 ProcList

 Timestamp is 5f5c3d93 (Sat Sep 12 04:16:35 2020)

 Preferred load address is 0000000180000000

 Start         Length     Name                   Class
 0001:00000000 00000008H .CRT$XCA                CODE
 0001:00000008 00000018H .CRT$XCC                CODE
 0001:00000020 00000010H .CRT$XCL                CODE
 0001:00000030 00000018H .CRT$XCU                CODE
 0001:00000048 00000008H .CRT$XCZ                CODE
 0001:00000050 00000008H .CRT$XIA                CODE
 0001:00000058 00000030H .CRT$XIC                CODE
 0001:00000088 00000008H .CRT$XIZ                CODE
 0001:00000090 00000008H .CRT$XPA                CODE
 0001:00000098 00000010H .CRT$XPX                CODE
 0001:000000a8 00000008H .CRT$XPXA               CODE
 0001:000000b0 00000008H .CRT$XPZ                CODE
 0001:000000b8 00000008H .CRT$XTA                CODE
 0001:000000c0 00000010H .CRT$XTZ                CODE
 0001:000000c8 00000000H .gfids$y                CODE
 0001:000000d0 000115c8H .rdata                  CODE
 0001:00011698 000007f4H .rdata$r                CODE
 0001:00011e8c 0000032cH .rdata$zzzdbg           CODE
 0001:000121b8 00000008H .rtc$IAA                CODE
 0001:000121c0 00000008H .rtc$IZZ                CODE
 0001:000121c8 00000008H .rtc$TAA                CODE
 0001:000121d0 00000010H .rtc$TZZ                CODE
 0001:000121e0 00000090H .text$di                CODE
 0001:00012270 00041900H .text$mn                CODE
 0001:00053b70 00000020H .text$mn$00             CODE
 0001:00053b90 00001530H .text$x                 CODE
 0001:000550c0 00000210H .text$yd                CODE
 0001:000552d0 00003bb8H .xdata                  CODE
 0001:00058e88 000003d8H .xdata$x                CODE
 0001:00059260 00000192H .edata                  CODE
 0002:00000000 00000bc0H .data                   DATA
 0002:00000bc0 000003d0H .data$r                 DATA
 0002:00000f90 00003124H .bss                    DATA
 0003:00000000 00002c58H .pdata                  DATA
 0004:00000000 000004a8H .idata$5                DATA
 0004:000004a8 00000010H .00cfg                  DATA
 0004:000004b8 000000a0H .idata$2                DATA
 0004:00000558 00000018H .idata$3                DATA
 0004:00000570 000004a8H .idata$4                DATA
 0004:00000a18 00000a7eH .idata$6                DATA
 0005:00000000 00000094H _RDATA                  DATA
 0006:00000000 00000060H .rsrc$01                DATA
 0006:00000060 00000378H .rsrc$02                DATA

  Address         Publics by Value              Rva+Base               Lib:Object

 0000:00000000       __hybrid_code_map          0000000000000000     <absolute>
 0000:00000000       __hybrid_code_map_count    0000000000000000     <absolute>
 0000:00000000       __guard_fids_count         0000000000000000     <absolute>
 0000:00000000       __volatile_metadata        0000000000000000     <absolute>
 0000:00000000       __guard_longjmp_count      0000000000000000     <absolute>
 0000:00000000       __guard_longjmp_table      0000000000000000     <absolute>
 0000:00000000       __guard_iat_count          0000000000000000     <absolute>
 0000:00000000       __guard_iat_table          0000000000000000     <absolute>
 0000:00000000       ___safe_se_handler_count   0000000000000000     <absolute>
 0000:00000000       __enclave_config           0000000000000000     <absolute>
 0000:00000000       __AbsoluteZero             0000000000000000     <absolute>
 0000:00000000       ___safe_se_handler_table   0000000000000000     <absolute>
 0000:00000000       __guard_fids_table         0000000000000000     <absolute>
 0000:00000000       __hybrid_auxiliary_iat     0000000000000000     <absolute>
 0000:00000000       __dynamic_value_reloc_table 0000000000000000     <absolute>
 0000:00000100       __guard_flags              0000000000000100     <absolute>
 0000:00000000       __ImageBase                0000000180000000     <linker-defined>
 0001:00000000       __xc_a                     0000000180001000     LIBCMT:initializers.obj
 0001:00000048       __xc_z                     0000000180001048     LIBCMT:initializers.obj
 0001:00000050       __xi_a                     0000000180001050     LIBCMT:initializers.obj
 0001:00000068       __acrt_stdio_initializer   0000000180001068     libucrt:stdio_initializer.obj
 0001:00000070       __acrt_tran_fma3_initializer 0000000180001070     libucrt:fma3_initializer.obj
 0001:00000078       __acrt_timeset_initializer 0000000180001078     libucrt:timeset_initializer.obj
 0001:00000080       __acrt_multibyte_initializer 0000000180001080     libucrt:multibyte_initializer.obj
 0001:00000088       __xi_z                     0000000180001088     LIBCMT:initializers.obj
 0001:00000090       __xp_a                     0000000180001090     LIBCMT:initializers.obj
 0001:00000098       __acrt_locale_terminator   0000000180001098     libucrt:locale_initializer.obj
 0001:000000a0       __dcrt_console_output_terminator 00000001800010a0     libucrt:console_output_initializer.obj
 0001:000000a8       __acrt_stdio_terminator    00000001800010a8     libucrt:stdio_initializer.obj
 0001:000000b0       __xp_z                     00000001800010b0     LIBCMT:initializers.obj
 0001:000000b8       __xt_a                     00000001800010b8     LIBCMT:initializers.obj
 0001:000000c0       __xt_z                     00000001800010c0     LIBCMT:initializers.obj
 0001:000000d0       ?powers_of_10_64@?$basic_data@X@detail@v6@fmt@@2QB_KB 00000001800010d0     format.obj
 0001:00000170       ?zero_or_powers_of_10_32@?$basic_data@X@detail@v6@fmt@@2QBIB 0000000180001170     format.obj
 0001:000001a0       ?zero_or_powers_of_10_64@?$basic_data@X@detail@v6@fmt@@2QB_KB 00000001800011a0     format.obj
 0001:00000240       ?pow10_significands@?$basic_data@X@detail@v6@fmt@@2QB_KB 0000000180001240     format.obj
 0001:00000500       ?pow10_exponents@?$basic_data@X@detail@v6@fmt@@2QBFB 0000000180001500     format.obj
 0001:000005b0       ?digits@?$basic_data@X@detail@v6@fmt@@2QAY01$$CBDA 00000001800015b0     format.obj
 0001:00000678       ?hex_digits@?$basic_data@X@detail@v6@fmt@@2QBDB 0000000180001678     format.obj
 0001:0000068c       ?signs@?$basic_data@X@detail@v6@fmt@@2QBDB 000000018000168c     format.obj
 0001:00000690       ?left_padding_shifts@?$basic_data@X@detail@v6@fmt@@2QBDB 0000000180001690     format.obj
 0001:00000698       ?right_padding_shifts@?$basic_data@X@detail@v6@fmt@@2QBDB 0000000180001698     format.obj
 0001:000006a0       ??_C@_0BC@EOODALEL@Unknown?5exception@ 00000001800016a0     format.obj
 0001:000006b8       ??_C@_0BF@KINCDENJ@bad?5array?5new?5length@ 00000001800016b8     format.obj
 0001:000006d0       ??_C@_08EPJLHIJG@bad?5cast@ 00000001800016d0     format.obj
 0001:000006d9       ??_C@_00CNPNBAHC@@         00000001800016d9     format.obj
 0001:000006e0       ??_C@_0BA@ELKIONDK@bad?5locale?5name@ 00000001800016e0     format.obj
 0001:000006f0       ??_C@_05LAPONLG@false@     00000001800016f0     format.obj
 0001:000006f8       ??_C@_04LOAJBDKD@true@     00000001800016f8     format.obj
 0001:00000700       ??_7format_error@v6@fmt@@6B@ 0000000180001700     format.obj
 0001:00000710       ??_7?$basic_memory_buffer@_W$0BPE@V?$allocator@_W@std@@@v6@fmt@@6B@ 0000000180001710     format.obj
 0001:00000720       ??_7?$basic_memory_buffer@D$0BPE@V?$allocator@D@std@@@v6@fmt@@6B@ 0000000180001720     format.obj
 0001:00000730       ??_7?$basic_memory_buffer@I$0CA@V?$allocator@I@std@@@v6@fmt@@6B@ 0000000180001730     format.obj
 0001:00000740       ??_C@_0BD@DBEDGLNA@argument?5not?5found@ 0000000180001740     format.obj
 0001:00000758       ??_C@_0BA@JFNIOLAK@string?5too?5long@ 0000000180001758     format.obj
 0001:00000768       ??_C@_0BP@NMGMJOEM@unmatched?5?8?$HN?8?5in?5format?5string@ 0000000180001768     format.obj
 0001:00000788       ??_C@_0BG@PEJKJNLA@invalid?5format?5string@ 0000000180001788     format.obj
 0001:000007a0       ??_C@_0BJ@JNDNOEDN@unknown?5format?5specifier@ 00000001800017a0     format.obj
 0001:000007c0       ??_C@_0BN@JNLAGDD@missing?5?8?$HN?8?5in?5format?5string@ 00000001800017c0     format.obj
 0001:000007e0       ??_C@_0DJ@LMIJFHJI@cannot?5switch?5from?5automatic?5to@ 00000001800017e0     format.obj
 0001:00000820       ??_C@_0BL@KNEDAEPA@invalid?5fill?5character?5?8?$HL?8@ 0000000180001820     format.obj
 0001:00000840       ??_C@_0CL@CFEEEDMP@format?5specifier?5requires?5numer@ 0000000180001840     format.obj
 0001:00000870       ??_C@_0BC@MDEIBHGE@number?5is?5too?5big@ 0000000180001870     format.obj
 0001:00000888       ??_C@_0BH@CIKPCHEG@invalid?5type?5specifier@ 0000000180001888     format.obj
 0001:000008a0       ??_C@_0CK@IBNNAPH@format?5specifier?5requires?5signe@ 00000001800018a0     format.obj
 0001:000008d0       ??_C@_0N@EFEDKJEI@invalid?5fill@ 00000001800018d0     format.obj
 0001:000008e0       ??_C@_0DJ@GHJONFIH@cannot?5switch?5from?5manual?5to?5au@ 00000001800018e0     format.obj
 0001:00000920       ??_C@_0CC@ELFJMMCC@invalid?5format?5specifier?5for?5ch@ 0000000180001920     format.obj
 0001:00000948       ??_C@_0BM@IEKLBNBK@missing?5precision?5specifier@ 0000000180001948     format.obj
 0001:00000968       ??_C@_0BH@IEEDMHI@string?5pointer?5is?5null@ 0000000180001968     format.obj
 0001:00000980       ??_C@_0CN@KMEDLGAJ@precision?5not?5allowed?5for?5this?5@ 0000000180001980     format.obj
 0001:000009b0       ??_C@_03OEIAHPBN@INF@      00000001800019b0     format.obj
 0001:000009b4       ??_C@_03OJHLLCGB@inf@      00000001800019b4     format.obj
 0001:000009b8       ??_C@_03LKNCIKJB@NAN@      00000001800019b8     format.obj
 0001:000009bc       ??_C@_03LHCJEHON@nan@      00000001800019bc     format.obj
 0001:000009c0       ??_C@_0BB@JGGOGLEG@0123456789ABCDEF@ 00000001800019c0     format.obj
 0001:000009d8       ??_C@_0BD@PKKFPMLC@negative?5precision@ 00000001800019d8     format.obj
 0001:000009f0       ??_C@_0P@DAPDPGEO@negative?5width@ 00000001800019f0     format.obj
 0001:00000a00       ??_C@_0BJ@KKLAKOOL@precision?5is?5not?5integer@ 0000000180001a00     format.obj
 0001:00000a20       ??_C@_0BF@KEAPHPPE@width?5is?5not?5integer@ 0000000180001a20     format.obj
 0001:00000a40       __xmm@80000000000000008000000000000000 0000000180001a40     format.obj
 0001:00000a50       __xmm@80000000800000008000000080000000 0000000180001a50     format.obj
 0001:00000a88       ??_C@_11LOCGONAA@@         0000000180001a88     handles.obj
 0001:00000a90       ??_C@_1BA@NMDNJJOO@?$AAP?$AAr?$AAo?$AAc?$AAe?$AAs?$AAs@ 0000000180001a90     handles.obj
 0001:00000aa0       ??_C@_1O@CDOGJPJJ@?$AAT?$AAh?$AAr?$AAe?$AAa?$AAd@ 0000000180001aa0     handles.obj
 0001:00000ab0       ??_C@_17KACEIPNC@?$AAK?$AAe?$AAy@ 0000000180001ab0     handles.obj
 0001:00000ab8       ??_C@_19DDLLJDOO@?$AAF?$AAi?$AAl?$AAe@ 0000000180001ab8     handles.obj
 0001:00000ac8       ??_C@_1O@ECECHNAE@?$AA?$DM?$AAp?$AAi?$AAp?$AAe?$AA?$DO@ 0000000180001ac8     handles.obj
 0001:00000ad8       ??_C@_1BE@FGECLHKD@?$AA?$HL?$AA0?$AA?$HN?$AA?5?$AA?$CI?$AA?$HL?$AA1?$AA?$HN?$AA?$CJ@ 0000000180001ad8     handles.obj
 0001:00000af0       ??_C@_1BC@HBCEGEJN@?$AAT?$AAI?$AAD?$AA?3?$AA?5?$AA?$HL?$AA0?$AA?$HN@ 0000000180001af0     handles.obj
 0001:00000b08       ??_C@_1BE@ELICABCK@?$AA?$DM?$AAu?$AAn?$AAk?$AAn?$AAo?$AAw?$AAn?$AA?$DO@ 0000000180001b08     handles.obj
 0001:00000b20       ??_C@_1DC@OIDKFHBF@?$AAM?$AAA?$AAC?$AAH?$AAI?$AAN?$AAE?$AA?2?$AAS?$AAO?$AAF?$AAT?$AAW?$AAA?$AAR@ 0000000180001b20     handles.obj
 0001:00000b58       ??_C@_19DIHHCHDI@?$AAH?$AAK?$AAU?$AA?2@ 0000000180001b58     handles.obj
 0001:00000b68       ??_C@_19JAPAIJDE@?$AAH?$AAK?$AAC?$AAU@ 0000000180001b68     handles.obj
 0001:00000b78       ??_C@_1BK@OEABCBLA@?$AAH?$AAK?$AAC?$AAU?$AA?2?$AAC?$AAl?$AAa?$AAs?$AAs?$AAe?$AAs@ 0000000180001b78     handles.obj
 0001:00000b98       ??_C@_17PJOJPMPB@?$AAH?$AAK?$AAU@ 0000000180001b98     handles.obj
 0001:00000ba0       ??_C@_19NCHLBIN@?$AAH?$AAK?$AAC?$AAR@ 0000000180001ba0     handles.obj
 0001:00000bb0       ??_C@_19PEALEEJB@?$AAH?$AAK?$AAL?$AAM@ 0000000180001bb0     handles.obj
 0001:00000bc0       ??_C@_1DK@KBLGALJE@?$AA?6?$AA?$HL?$AA0?$AA?$HN?$AA?6?$AA?$HL?$AA1?$AA?3?$AA6?$AA?$HN?$AA?5?$AA?$HL?$AA2?$AA?3?$AA8@ 0000000180001bc0     handles.obj
 0001:00000c00       ??_C@_1DG@HOLPNCNP@?$AA?$HL?$AA0?$AA?3?$AA6?$AAX?$AA?$HN?$AA?5?$AA?$HL?$AA1?$AA?3?$AA0?$AA8?$AAX?$AA?$HN?$AA?5@ 0000000180001c00     handles.obj
 0001:00000c38       ??_7PluginCheckBoxBinding@@6B@ 0000000180001c38     Pcfg.obj
 0001:00000c48       ??_C@_1O@BJPKKLLM@?$AAC?$AAo?$AAn?$AAf?$AAi?$AAg@ 0000000180001c48     Pcfg.obj
 0001:00000c58       ??_C@_1BO@NGDOFANC@?$AAA?$AAd?$AAd?$AAT?$AAo?$AAD?$AAi?$AAs?$AAk?$AAs?$AAM?$AAe?$AAn?$AAu@ 0000000180001c58     Pcfg.obj
 0001:00000c78       ??_C@_1CC@PNNAOHJC@?$AAA?$AAd?$AAd?$AAT?$AAo?$AAP?$AAl?$AAu?$AAg?$AAi?$AAn?$AAs?$AAM?$AAe?$AAn@ 0000000180001c78     Pcfg.obj
 0001:00000ca0       ??_C@_1CE@JIPJNDMD@?$AAE?$AAx?$AAp?$AAo?$AAr?$AAt?$AAE?$AAn?$AAv?$AAi?$AAr?$AAo?$AAn?$AAm?$AAe@ 0000000180001ca0     Pcfg.obj
 0001:00000cc8       ??_C@_1CC@OABICAMP@?$AAE?$AAx?$AAp?$AAo?$AAr?$AAt?$AAM?$AAo?$AAd?$AAu?$AAl?$AAe?$AAI?$AAn?$AAf@ 0000000180001cc8     Pcfg.obj
 0001:00000cf0       ??_C@_1CI@OFLGHPDG@?$AAE?$AAx?$AAp?$AAo?$AAr?$AAt?$AAM?$AAo?$AAd?$AAu?$AAl?$AAe?$AAV?$AAe?$AAr@ 0000000180001cf0     Pcfg.obj
 0001:00000d18       ??_C@_1CE@GNMOKOAL@?$AAE?$AAx?$AAp?$AAo?$AAr?$AAt?$AAP?$AAe?$AAr?$AAf?$AAo?$AAr?$AAm?$AAa?$AAn@ 0000000180001d18     Pcfg.obj
 0001:00000d40       ??_C@_1BM@KMCHODLM@?$AAE?$AAx?$AAp?$AAo?$AAr?$AAt?$AAH?$AAa?$AAn?$AAd?$AAl?$AAe?$AAs@ 0000000180001d40     Pcfg.obj
 0001:00000d60       ??_C@_1CK@CLFOOHFA@?$AAE?$AAx?$AAp?$AAo?$AAr?$AAt?$AAH?$AAa?$AAn?$AAd?$AAl?$AAe?$AAs?$AAU?$AAn@ 0000000180001d60     Pcfg.obj
 0001:00000d90       ??_C@_1BE@PKILIDFH@?$AAE?$AAn?$AAa?$AAb?$AAl?$AAe?$AAW?$AAM?$AAI@ 0000000180001d90     Pcfg.obj
 0001:00000db0       __xmm@00000000000000020000000000000000 0000000180001db0     Pcfg.obj
 0001:00000dc0       __xmm@ffffffffffffffffffffffffffffffff 0000000180001dc0     Pcfg.obj
 0001:00000dd0       ??_7PluginEditFieldBinding@@6B@ 0000000180001dd0     Pclass.obj
 0001:00000de0       ??_C@_1BK@GMMKGKID@?$AA?$HL?$AA0?$AA?$HN?$AA?4?$AA?$HL?$AA1?$AA?3?$AA0?$AA?$HL?$AA2?$AA?$HN?$AA?$HN@ 0000000180001de0     Pclass.obj
 0001:00000e00       ??_C@_1BA@BHJJFMCM@?$AAB?$AAK?$AAM?$AAG?$AAT?$AAP?$AAE@ 0000000180001e00     Pclass.obj
 0001:00000e10       ??_C@_1BC@HGOMHBK@?$AA?$HL?$AA0?$AA?3?$AA?$DM?$AA2?$AA1?$AA?$HN?$AA?5@ 0000000180001e10     Pclass.obj
 0001:00000e28       ??_C@_1BC@IALIJCAM@?$AAS?$AAo?$AAr?$AAt?$AAM?$AAo?$AAd?$AAe@ 0000000180001e28     Pclass.obj
 0001:00000e40       ??_C@_1BO@OMKAPLPJ@?$AAS?$AAt?$AAa?$AAr?$AAt?$AAP?$AAa?$AAn?$AAe?$AAl?$AAM?$AAo?$AAd?$AAe@ 0000000180001e40     Pclass.obj
 0001:00000e80       ??_C@_1BA@JOLGFBLP@?$AAM?$AAo?$AAd?$AAe?$AA?$HL?$AA0?$AA?$HN@ 0000000180001e80     Pclass.obj
 0001:00000e90       ??_C@_1CM@KGJLHHPG@?$AAN?$AA?0?$AAX?$AA1?$AA5?$AAF?$AA?0?$AAX?$AA1?$AA6?$AAF?$AA?0?$AAX?$AA1?$AA7@ 0000000180001e90     Pclass.obj
 0001:00000ec0       ??_C@_1BG@MNPGDOEP@?$AA1?$AA2?$AA?0?$AA0?$AA?0?$AA0?$AA?0?$AA0?$AA?0?$AA4@ 0000000180001ec0     Pclass.obj
 0001:00000ed8       ??_C@_1CG@OHFJBKLN@?$AAN?$AA?0?$AAX?$AAI?$AA?0?$AAX?$AAB?$AA?0?$AAX?$AAP?$AA?0?$AAX?$AA0?$AAS?$AA?0@ 0000000180001ed8     Pclass.obj
 0001:00000f00       ??_C@_1BI@EFANNANC@?$AA0?$AA?0?$AA6?$AA?0?$AA2?$AA?0?$AA2?$AA?0?$AA3?$AA?0?$AA9@ 0000000180001f00     Pclass.obj
 0001:00000f18       ??_C@_17KNGPBKAK@?$AAN?$AA?0?$AAN@ 0000000180001f18     Pclass.obj
 0001:00000f20       ??_C@_17JPFFEOAH@?$AA0?$AA?0?$AA0@ 0000000180001f20     Pclass.obj
 0001:00000f28       ??_C@_1BO@JAFIOFIL@?$AAN?$AA?0?$AAX?$AAI?$AA?0?$AAX?$AAB?$AA?0?$AAX?$AAC?$AA?0?$AAD?$AA?0?$AAT@ 0000000180001f28     Pclass.obj
 0001:00000f48       ??_C@_1BI@LFIMKDME@?$AA0?$AA?0?$AA6?$AA?0?$AA2?$AA?0?$AA6?$AA?0?$AA0?$AA?0?$AA0@ 0000000180001f48     Pclass.obj
 0001:00000f60       ??_C@_1BK@IEHCCPMO@?$AAN?$AA?0?$AAX?$AAI?$AA?0?$AAX?$AA4?$AAF?$AA?0?$AAX?$AA6?$AAF@ 0000000180001f60     Pclass.obj
 0001:00000f80       ??_C@_1BA@MMHHFCDG@?$AA0?$AA?0?$AA6?$AA?0?$AA9?$AA?0?$AA9@ 0000000180001f80     Pclass.obj
 0001:00000f90       ??_C@_1EA@CMHCGANC@?$AAN?$AA?0?$AAX?$AAI?$AA?0?$AAX?$AA4?$AAF?$AA?0?$AAX?$AA6?$AAF?$AA?0?$AAX?$AA1@ 0000000180001f90     Pclass.obj
 0001:00000fd0       ??_C@_1CE@LPFIEDMN@?$AA0?$AA?0?$AA6?$AA?0?$AA9?$AA?0?$AA9?$AA?0?$AA9?$AA?0?$AA9?$AA?0?$AA8?$AA?0?$AA8@ 0000000180001fd0     Pclass.obj
 0001:00000ff8       ??_C@_19ILLMDDHI@?$AAN?$AA?0?$AAZ?$AAD@ 0000000180001ff8     Pclass.obj
 0001:00001008       ??_C@_19NMOJBHGD@?$AA1?$AA2?$AA?0?$AA0@ 0000000180002008     Pclass.obj
 0001:00001020       ??_C@_1EC@OFLHMCFD@?$AAN?$AA?0?$AAX?$AAP?$AA?0?$AAX?$AA0?$AAS?$AA?0?$AAX?$AA1?$AAS?$AA?0?$AAX?$AA2@ 0000000180002020     Pclass.obj
 0001:00001068       ??_C@_1CA@MGMNHCLL@?$AA0?$AA?0?$AA2?$AA?0?$AA3?$AA?0?$AA2?$AA?0?$AA2?$AA?0?$AA3?$AA?0?$AA4?$AA?0?$AA3@ 0000000180002068     Pclass.obj
 0001:00001088       ??_C@_1O@JGFFCAGM@?$AAN?$AA?0?$AAX?$AAI?$AA?0?$AAO@ 0000000180002088     Pclass.obj
 0001:00001098       ??_C@_1O@FLEOANAI@?$AA0?$AA?0?$AA6?$AA?0?$AA1?$AA5@ 0000000180002098     Pclass.obj
 0001:000010a8       ??_C@_1CC@FANCGEGE@?$AAN?$AA?0?$AAX?$AAI?$AA?0?$AAX?$AAT?$AA?0?$AAX?$AA3?$AA?0?$AAX?$AAG?$AA?0?$AAX@ 00000001800020a8     Pclass.obj
 0001:000010d0       ??_C@_1BI@PMPHDFGH@?$AA0?$AA?0?$AA6?$AA?0?$AA3?$AA?0?$AA4?$AA?0?$AA4?$AA?0?$AA4@ 00000001800020d0     Pclass.obj
 0001:000010e8       ??_C@_1BG@COBJEPBB@?$AAN?$AA?0?$AAX?$AAI?$AA?0?$AAX?$AAT?$AA?0?$AAX?$AA3@ 00000001800020e8     Pclass.obj
 0001:00001100       ??_C@_1BA@KPNNJGCD@?$AA0?$AA?0?$AA6?$AA?0?$AA3?$AA?0?$AA4@ 0000000180002100     Pclass.obj
 0001:00001110       ??_C@_1CA@HLBJOHGN@?$AAF?$AAu?$AAl?$AAl?$AAS?$AAc?$AAr?$AAe?$AAe?$AAn?$AAL?$AAo?$AAc?$AAa?$AAl@ 0000000180002110     Pclass.obj
 0001:00001130       ??_C@_1CC@EBBNDNOD@?$AAF?$AAu?$AAl?$AAl?$AAS?$AAc?$AAr?$AAe?$AAe?$AAn?$AAR?$AAe?$AAm?$AAo?$AAt@ 0000000180002130     Pclass.obj
 0001:00001158       ??_C@_1BK@HMOODHKK@?$AAC?$AAo?$AAl?$AAu?$AAm?$AAn?$AAs?$AAL?$AAo?$AAc?$AAa?$AAl@ 0000000180002158     Pclass.obj
 0001:00001178       ??_C@_1BM@EDHFKJEJ@?$AAC?$AAo?$AAl?$AAu?$AAm?$AAn?$AAs?$AAR?$AAe?$AAm?$AAo?$AAt?$AAe@ 0000000180002178     Pclass.obj
 0001:00001198       ??_C@_1BI@FOOHDOCI@?$AAW?$AAi?$AAd?$AAt?$AAh?$AAs?$AAL?$AAo?$AAc?$AAa?$AAl@ 0000000180002198     Pclass.obj
 0001:000011b0       ??_C@_1BK@DDBMMJCN@?$AAW?$AAi?$AAd?$AAt?$AAh?$AAs?$AAR?$AAe?$AAm?$AAo?$AAt?$AAe@ 00000001800021b0     Pclass.obj
 0001:000011cc       ??_C@_13DEFPDAGF@?$AA?0@   00000001800021cc     Pclass.obj
 0001:000011d0       ??_C@_15LNKNCLHH@?$AAS?$AAs@ 00000001800021d0     Pclass.obj
 0001:000011d8       ??_C@_1M@PBHOFL@?$AA?5?$AA?$HL?$AA0?$AA?$HN?$AA?5@ 00000001800021d8     Pclass.obj
 0001:000011e8       ??_C@_1BE@JJMDGICA@?$AA?$HL?$AA0?$AA?$HN?$AA?3?$AA?5?$AA?$HL?$AA1?$AA?$HN?$AA?5@ 00000001800021e8     Pclass.obj
 0001:000011fc       ??_C@_15JOGBDECP@?$AA?0?$AA?5@ 00000001800021fc     Pclass.obj
 0001:00001204       ??_C@_15DNHPCDHG@?$AAT?$AAt@ 0000000180002204     Pclass.obj
 0001:0000120c       ??_C@_15IJHBBPPC@?$AAF?$AAf@ 000000018000220c     Pclass.obj
 0001:00001218       ??_C@_1BC@OMEIHGFC@?$AAW?$AAS?$AA_?$AAP?$AAO?$AAP?$AAU?$AAP@ 0000000180002218     Pclass.obj
 0001:00001230       ??_C@_1BC@ONEEOLLM@?$AAW?$AAS?$AA_?$AAC?$AAH?$AAI?$AAL?$AAD@ 0000000180002230     Pclass.obj
 0001:00001248       ??_C@_1BI@GHDIGAD@?$AAW?$AAS?$AA_?$AAM?$AAI?$AAN?$AAI?$AAM?$AAI?$AAZ?$AAE@ 0000000180002248     Pclass.obj
 0001:00001260       ??_C@_1BG@KLPFHNBP@?$AAW?$AAS?$AA_?$AAV?$AAI?$AAS?$AAI?$AAB?$AAL?$AAE@ 0000000180002260     Pclass.obj
 0001:00001278       ??_C@_1BI@NKODCGOF@?$AAW?$AAS?$AA_?$AAD?$AAI?$AAS?$AAA?$AAB?$AAL?$AAE?$AAD@ 0000000180002278     Pclass.obj
 0001:00001290       ??_C@_1CA@PCFJBBHH@?$AAW?$AAS?$AA_?$AAC?$AAL?$AAI?$AAP?$AAS?$AAI?$AAB?$AAL?$AAI?$AAN?$AAG?$AAS@ 0000000180002290     Pclass.obj
 0001:000012b0       ??_C@_1CA@MPLGGIO@?$AAW?$AAS?$AA_?$AAC?$AAL?$AAI?$AAP?$AAC?$AAH?$AAI?$AAL?$AAD?$AAR?$AAE?$AAN@ 00000001800022b0     Pclass.obj
 0001:000012d0       ??_C@_1BI@OLBAGOJG@?$AAW?$AAS?$AA_?$AAM?$AAA?$AAX?$AAI?$AAM?$AAI?$AAZ?$AAE@ 00000001800022d0     Pclass.obj
 0001:000012e8       ??_C@_1BE@DAMMEKNP@?$AAW?$AAS?$AA_?$AAB?$AAO?$AAR?$AAD?$AAE?$AAR@ 00000001800022e8     Pclass.obj
 0001:00001300       ??_C@_1BI@EDHINADK@?$AAW?$AAS?$AA_?$AAD?$AAL?$AAG?$AAF?$AAR?$AAA?$AAM?$AAE@ 0000000180002300     Pclass.obj
 0001:00001318       ??_C@_1BG@CKCLFGFA@?$AAW?$AAS?$AA_?$AAV?$AAS?$AAC?$AAR?$AAO?$AAL?$AAL@ 0000000180002318     Pclass.obj
 0001:00001330       ??_C@_1BG@OMIOJOGF@?$AAW?$AAS?$AA_?$AAH?$AAS?$AAC?$AAR?$AAO?$AAL?$AAL@ 0000000180002330     Pclass.obj
 0001:00001348       ??_C@_1BG@KJOBMDJC@?$AAW?$AAS?$AA_?$AAS?$AAY?$AAS?$AAM?$AAE?$AAN?$AAU@ 0000000180002348     Pclass.obj
 0001:00001360       ??_C@_1BM@GPNNOPCH@?$AAW?$AAS?$AA_?$AAT?$AAH?$AAI?$AAC?$AAK?$AAF?$AAR?$AAA?$AAM?$AAE@ 0000000180002360     Pclass.obj
 0001:00001380       ??_C@_1BO@FODKBODI@?$AAW?$AAS?$AA_?$AAM?$AAI?$AAN?$AAI?$AAM?$AAI?$AAZ?$AAE?$AAB?$AAO?$AAX@ 0000000180002380     Pclass.obj
 0001:000013a0       ??_C@_1BO@IDJMAOMI@?$AAW?$AAS?$AA_?$AAM?$AAA?$AAX?$AAI?$AAM?$AAI?$AAZ?$AAE?$AAB?$AAO?$AAX@ 00000001800023a0     Pclass.obj
 0001:000013c0       ??_C@_1CI@PKBCIOPN@?$AAW?$AAS?$AA_?$AAE?$AAX?$AA_?$AAD?$AAL?$AAG?$AAM?$AAO?$AAD?$AAA?$AAL?$AAF@ 00000001800023c0     Pclass.obj
 0001:000013e8       ??_C@_1CK@KJECLHMG@?$AAW?$AAS?$AA_?$AAE?$AAX?$AA_?$AAN?$AAO?$AAP?$AAA?$AAR?$AAE?$AAN?$AAT?$AAN@ 00000001800023e8     Pclass.obj
 0001:00001418       ??_C@_1BM@OCBKBALE@?$AAW?$AAS?$AA_?$AAE?$AAX?$AA_?$AAT?$AAO?$AAP?$AAM?$AAO?$AAS?$AAT@ 0000000180002418     Pclass.obj
 0001:00001438       ??_C@_1CE@JIDMMICL@?$AAW?$AAS?$AA_?$AAE?$AAX?$AA_?$AAA?$AAC?$AAC?$AAE?$AAP?$AAT?$AAF?$AAI?$AAL@ 0000000180002438     Pclass.obj
 0001:00001460       ??_C@_1CE@PFFPBMCF@?$AAW?$AAS?$AA_?$AAE?$AAX?$AA_?$AAT?$AAR?$AAA?$AAN?$AAS?$AAP?$AAA?$AAR?$AAE@ 0000000180002460     Pclass.obj
 0001:00001488       ??_C@_1BO@MEOEJPLO@?$AAW?$AAS?$AA_?$AAE?$AAX?$AA_?$AAM?$AAD?$AAI?$AAC?$AAH?$AAI?$AAL?$AAD@ 0000000180002488     Pclass.obj
 0001:000014a8       ??_C@_1CC@IEIGGJGG@?$AAW?$AAS?$AA_?$AAE?$AAX?$AA_?$AAT?$AAO?$AAO?$AAL?$AAW?$AAI?$AAN?$AAD?$AAO@ 00000001800024a8     Pclass.obj
 0001:000014d0       ??_C@_1CC@PLPNIKGL@?$AAW?$AAS?$AA_?$AAE?$AAX?$AA_?$AAW?$AAI?$AAN?$AAD?$AAO?$AAW?$AAE?$AAD?$AAG@ 00000001800024d0     Pclass.obj
 0001:000014f8       ??_C@_1CC@IAPGCLEG@?$AAW?$AAS?$AA_?$AAE?$AAX?$AA_?$AAC?$AAL?$AAI?$AAE?$AAN?$AAT?$AAE?$AAD?$AAG@ 00000001800024f8     Pclass.obj
 0001:00001520       ??_C@_1CE@EANKNCIF@?$AAW?$AAS?$AA_?$AAE?$AAX?$AA_?$AAC?$AAO?$AAN?$AAT?$AAE?$AAX?$AAT?$AAH?$AAE@ 0000000180002520     Pclass.obj
 0001:00001548       ??_C@_1BI@GFIADCMK@?$AAW?$AAS?$AA_?$AAE?$AAX?$AA_?$AAR?$AAI?$AAG?$AAH?$AAT@ 0000000180002548     Pclass.obj
 0001:00001560       ??_C@_1CC@JOFCJJPB@?$AAW?$AAS?$AA_?$AAE?$AAX?$AA_?$AAR?$AAT?$AAL?$AAR?$AAE?$AAA?$AAD?$AAI?$AAN@ 0000000180002560     Pclass.obj
 0001:00001588       ??_C@_1CI@EFLDECAB@?$AAW?$AAS?$AA_?$AAE?$AAX?$AA_?$AAL?$AAE?$AAF?$AAT?$AAS?$AAC?$AAR?$AAO?$AAL@ 0000000180002588     Pclass.obj
 0001:000015b0       ??_C@_1CI@CIFGFFJB@?$AAW?$AAS?$AA_?$AAE?$AAX?$AA_?$AAC?$AAO?$AAN?$AAT?$AAR?$AAO?$AAL?$AAP?$AAA@ 00000001800025b0     Pclass.obj
 0001:000015d8       ??_C@_1CC@BGEPLDCA@?$AAW?$AAS?$AA_?$AAE?$AAX?$AA_?$AAS?$AAT?$AAA?$AAT?$AAI?$AAC?$AAE?$AAD?$AAG@ 00000001800025d8     Pclass.obj
 0001:00001600       ??_C@_1CA@DOAIHHLO@?$AAW?$AAS?$AA_?$AAE?$AAX?$AA_?$AAA?$AAP?$AAP?$AAW?$AAI?$AAN?$AAD?$AAO?$AAW@ 0000000180002600     Pclass.obj
 0001:00001620       ??_C@_1BM@FAODAMGD@?$AAW?$AAS?$AA_?$AAE?$AAX?$AA_?$AAL?$AAA?$AAY?$AAE?$AAR?$AAE?$AAD@ 0000000180002620     Pclass.obj
 0001:00001640       ??_C@_1CM@DJKNBOGD@?$AAW?$AAS?$AA_?$AAE?$AAX?$AA_?$AAN?$AAO?$AAI?$AAN?$AAH?$AAE?$AAR?$AAI?$AAT@ 0000000180002640     Pclass.obj
 0001:00001670       ??_C@_1CA@KMHLBMFI@?$AAW?$AAS?$AA_?$AAE?$AAX?$AA_?$AAL?$AAA?$AAY?$AAO?$AAU?$AAT?$AAR?$AAT?$AAL@ 0000000180002670     Pclass.obj
 0001:00001690       ??_C@_1CC@LOFMDOPL@?$AAW?$AAS?$AA_?$AAE?$AAX?$AA_?$AAN?$AAO?$AAA?$AAC?$AAT?$AAI?$AAV?$AAA?$AAT@ 0000000180002690     Pclass.obj
 0001:000016b8       ??_C@_1BA@PCPLEJNM@?$AA?$HL?$AA0?$AA?3?$AA2?$AA0?$AA?$HN?$AA?6@ 00000001800026b8     Pclass.obj
 0001:000016c8       ??_C@_1CA@PGPHFLML@?$AA?$HL?$AA0?$AA?3?$AA?$DO?$AA2?$AA0?$AA?$HN?$AA?5?$AA?$HL?$AA1?$AA?3?$AA7?$AA?$HN?$AA?$CF?$AA?6@ 00000001800026c8     Pclass.obj
 0001:000016e8       ??_C@_1CE@BCAPNIMO@?$AA?$HL?$AA0?$AA?3?$AA2?$AA0?$AA?$HN?$AA?5?$AA?5?$AA?$HL?$AA1?$AA?3?$AA7?$AA?$HN?$AA?$HL?$AA2@ 00000001800026e8     Pclass.obj
 0001:00001728       ??_C@_1CA@CGMHBFCH@?$AA?$HL?$AA0?$AA?$HN?$AA?$HL?$AA1?$AA?$HN?$AA?0?$AA?5?$AA?$HL?$AA2?$AA?$HN?$AA?$HL?$AA3?$AA?$HN?$AA?6@ 0000000180002728     Pclass.obj
 0001:00001748       ??_C@_1BA@BIAFDLFH@?$AA?$HL?$AA0?$AA?$HN?$AA?$HL?$AA1?$AA?$HN?$AA?6@ 0000000180002748     Pclass.obj
 0001:00001758       ??_C@_1BI@DHFBAHCI@?$AA?$HL?$AA0?$AA?$HN?$AA?5?$AA?5?$AA?$CI?$AA?$HL?$AA1?$AA?$HN?$AA?$CJ?$AA?6@ 0000000180002758     Pclass.obj
 0001:00001770       ??_C@_19EPBAEEOA@?$AA?$HL?$AA0?$AA?$HN?$AA?6@ 0000000180002770     Pclass.obj
 0001:00001780       ??_C@_1BK@FKNCLDML@?$AA?6?$AA?$HL?$AA0?$AA?$HN?$AA?$HL?$AA1?$AA?$HN?$AA?5?$AA?$HL?$AA2?$AA?$HN?$AA?6@ 0000000180002780     Pclass.obj
 0001:000017a0       ??_C@_1BC@IBCAHKMA@?$AA?6?$AA?$HL?$AA0?$AA?$HN?$AA?$HL?$AA1?$AA?$HN?$AA?6@ 00000001800027a0     Pclass.obj
 0001:000017b8       ??_C@_1BE@EKPFJOAB@?$AA?6?$AA?$HL?$AA0?$AA?$HN?$AA?6?$AA?$HL?$AA1?$AA?$HN?$AA?6@ 00000001800027b8     Pclass.obj
 0001:000017d0       ??_C@_1CA@MEPGLLIO@?$AA?$HL?$AA0?$AA?$HN?$AA?$HL?$AA1?$AA?3?$AA0?$AA8?$AAX?$AA?$HN?$AA?5?$AA?$HL?$AA2?$AA?$HN?$AA?6@ 00000001800027d0     Pclass.obj
 0001:000017f0       ??_C@_1DE@IMIBLDFN@?$AA?6?$AA?$HL?$AA0?$AA?$HN?$AA?6?$AA?$HL?$AA1?$AA?3?$AA?$DM?$AA?$HL?$AA2?$AA?$HN?$AA?$HN?$AA?5?$AA?$HL@ 00000001800027f0     Pclass.obj
 0001:00001828       ??_C@_19GGNHIDOH@?$AA?4?$AAt?$AAx?$AAt@ 0000000180002828     Pclass.obj
 0001:00001838       ??_C@_19OPNPIOHE@?$AAH?$AAW?$AAN?$AAD@ 0000000180002838     Pclass.obj
 0001:00001844       ??_C@_15GKIJICBO@?$AAZ?$AAC@ 0000000180002844     Pclass.obj
 0001:00001850       ??_C@_17JJIMNMHK@?$AA?5?$AA?$CG?$AA?$FO@ 0000000180002850     Pclass.obj
 0001:00001858       ??_C@_13HOIJIPNN@?$AA?5@   0000000180002858     Pclass.obj
 0001:0000185c       ??_C@_15LEKKCGMK@?$AA?2?$AA?2@ 000000018000285c     Pclass.obj
 0001:00001880       ??_C@_1M@CHPAGEIC@?$AA?$CF?$AA?5?$AA?$HL?$AA0?$AA?$HN@ 0000000180002880     Pclass.obj
 0001:00001890       ??_C@_1O@DLMEBHDD@?$AA?$HL?$AA0?$AA?$HN?$AA?$HL?$AA1?$AA?$HN@ 0000000180002890     Pclass.obj
 0001:000018a0       ??_C@_15DDHGOCBH@?$AA?4?$AA?4@ 00000001800028a0     Pclass.obj
 0001:000018a8       ??_C@_17FJPEEFCB@?$AAp?$AAr?$AAc@ 00000001800028a8     Pclass.obj
 0001:000018b0       ??_C@_1BC@ENICKDH@?$AAC?$AAo?$AAn?$AAt?$AAe?$AAn?$AAt?$AAs@ 00000001800028b0     Pclass.obj
 0001:000018c8       ??_C@_1CK@DGKCELDD@?$AAP?$AAr?$AAo?$AAc?$AAe?$AAs?$AAs?$AAL?$AAi?$AAs?$AAt?$AA?4?$AAC?$AAo?$AAm@ 00000001800028c8     Pclass.obj
 0001:000018f8       ??_C@_1CK@ECJCGOEK@?$AAP?$AAr?$AAo?$AAc?$AAe?$AAs?$AAs?$AAL?$AAi?$AAs?$AAt?$AA?4?$AAU?$AAs?$AAe@ 00000001800028f8     Pclass.obj
 0001:00001930       ??_C@_1EA@IELLPLEF@?$AA?$HL?$AA0?$AA?$HN?$AA?5?$AA?$HL?$AA1?$AA?3?$AA0?$AA2?$AA?$HN?$AA?3?$AA?$HL?$AA2?$AA?3?$AA0@ 0000000180002930     Pclass.obj
 0001:00001970       ??_C@_1DI@BCOMPFMM@?$AA?$HL?$AA0?$AA?3?$AA0?$AA2?$AA?$HN?$AA?3?$AA?$HL?$AA1?$AA?3?$AA0?$AA2?$AA?$HN?$AA?3?$AA?$HL@ 0000000180002970     Pclass.obj
 0001:000019b0       ??_C@_1EA@HECKBAAG@?$AA?2?$AAS?$AAt?$AAr?$AAi?$AAn?$AAg?$AAF?$AAi?$AAl?$AAe?$AAI?$AAn?$AAf?$AAo@ 00000001800029b0     Pclass.obj
 0001:000019f0       ??_C@_19JHEHLFPM@?$AA?2?$AA?$DP?$AA?$DP?$AA?2@ 00000001800029f0     Pclass.obj
 0001:00001a00       ??_C@_1DC@HCLBMGIA@?$AA?2?$AAV?$AAa?$AAr?$AAF?$AAi?$AAl?$AAe?$AAI?$AAn?$AAf?$AAo?$AA?2?$AAT?$AAr@ 0000000180002a00     Pclass.obj
 0001:00001a38       ??_C@_1BI@HCCAONKE@?$AAF?$AAi?$AAl?$AAe?$AAV?$AAe?$AAr?$AAs?$AAi?$AAo?$AAn@ 0000000180002a38     Pclass.obj
 0001:00001a50       ??_C@_1CA@JGBAIPOO@?$AAF?$AAi?$AAl?$AAe?$AAD?$AAe?$AAs?$AAc?$AAr?$AAi?$AAp?$AAt?$AAi?$AAo?$AAn@ 0000000180002a50     Pclass.obj
 0001:00001a70       ??_C@_19KBHGBEJO@?$AA?$HL?$AA0?$AA?$HN?$AA?2@ 0000000180002a70     Pclass.obj
 0001:00001a80       ??_C@_1O@BMPPIAFP@?$AA?5?$AA?$CI?$AA?$HL?$AA0?$AA?$HN?$AA?$CJ@ 0000000180002a80     Pclass.obj
 0001:00001a90       ??_C@_1BC@OMEIBLAI@?$AAw?$AAb?$AAe?$AAm?$AAc?$AAo?$AAm?$AAn@ 0000000180002a90     Pclass.obj
 0001:00001aa8       ??_C@_0BI@CFPLBAOH@invalid?5string?5position@ 0000000180002aa8     Pclass.obj
 0001:00001ac0       ??_C@_15LGINNLBP@?$AA?$HL?$AA?$HN@ 0000000180002ac0     Pclass.obj
 0001:00001ac8       ??_C@_0BA@FOIKENOD@vector?5too?5long@ 0000000180002ac8     Pclass.obj
 0001:00001ad8       ??_C@_0BL@GOIGLPKN@unordered_map?1set?5too?5long@ 0000000180002ad8     Pclass.obj
 0001:00001af8       ??_C@_0BK@OGNNAFAB@invalid?5hash?5bucket?5count@ 0000000180002af8     Pclass.obj
 0001:00001b14       __real@3f800000            0000000180002b14     Pclass.obj
 0001:00001b18       __real@4024000000000000    0000000180002b18     Pclass.obj
 0001:00001b20       __real@43e0000000000000    0000000180002b20     Pclass.obj
 0001:00001b28       __real@5f000000            0000000180002b28     Pclass.obj
 0001:00001b30       ?Counters@@3QBUcounters@@B 0000000180002b30     perfthread.obj
 0001:00001c90       ??_C@_1CC@DNHMJIKH@?$AA?$CF?$AA?5?$AAP?$AAr?$AAo?$AAc?$AAe?$AAs?$AAs?$AAo?$AAr?$AA?5?$AAT?$AAi?$AAm@ 0000000180002c90     perfthread.obj
 0001:00001cb8       ??_C@_1CE@FNEMIHOD@?$AA?$CF?$AA?5?$AAP?$AAr?$AAi?$AAv?$AAi?$AAl?$AAe?$AAg?$AAe?$AAd?$AA?5?$AAT?$AAi@ 0000000180002cb8     perfthread.obj
 0001:00001ce0       ??_C@_1BI@IIOPEKIO@?$AA?$CF?$AA?5?$AAU?$AAs?$AAe?$AAr?$AA?5?$AAT?$AAi?$AAm?$AAe@ 0000000180002ce0     perfthread.obj
 0001:00001cf8       ??_C@_1BK@FAAJNJIB@?$AAH?$AAa?$AAn?$AAd?$AAl?$AAe?$AA?5?$AAC?$AAo?$AAu?$AAn?$AAt@ 0000000180002cf8     perfthread.obj
 0001:00001d18       ??_C@_1CA@KJMNGIDJ@?$AAP?$AAa?$AAg?$AAe?$AA?5?$AAF?$AAi?$AAl?$AAe?$AA?5?$AAB?$AAy?$AAt?$AAe?$AAs@ 0000000180002d18     perfthread.obj
 0001:00001d38       ??_C@_1CK@FGGMBBIH@?$AAP?$AAa?$AAg?$AAe?$AA?5?$AAF?$AAi?$AAl?$AAe?$AA?5?$AAB?$AAy?$AAt?$AAe?$AAs@ 0000000180002d38     perfthread.obj
 0001:00001d68       ??_C@_1BI@GCOMDKEO@?$AAW?$AAo?$AAr?$AAk?$AAi?$AAn?$AAg?$AA?5?$AAS?$AAe?$AAt@ 0000000180002d68     perfthread.obj
 0001:00001d80       ??_C@_1CC@OFJLEPCP@?$AAW?$AAo?$AAr?$AAk?$AAi?$AAn?$AAg?$AA?5?$AAS?$AAe?$AAt?$AA?5?$AAP?$AAe?$AAa@ 0000000180002d80     perfthread.obj
 0001:00001da8       ??_C@_1CI@LLKMGPEG@?$AAP?$AAo?$AAo?$AAl?$AA?5?$AAN?$AAo?$AAn?$AAp?$AAa?$AAg?$AAe?$AAd?$AA?5?$AAB@ 0000000180002da8     perfthread.obj
 0001:00001dd0       ??_C@_1CC@IMBAECJF@?$AAP?$AAo?$AAo?$AAl?$AA?5?$AAP?$AAa?$AAg?$AAe?$AAd?$AA?5?$AAB?$AAy?$AAt?$AAe@ 0000000180002dd0     perfthread.obj
 0001:00001df8       ??_C@_1BM@DGDPAMAA@?$AAP?$AAr?$AAi?$AAv?$AAa?$AAt?$AAe?$AA?5?$AAB?$AAy?$AAt?$AAe?$AAs@ 0000000180002df8     perfthread.obj
 0001:00001e18       ??_C@_1CA@GADAGCME@?$AAP?$AAa?$AAg?$AAe?$AA?5?$AAF?$AAa?$AAu?$AAl?$AAt?$AAs?$AA?1?$AAs?$AAe?$AAc@ 0000000180002e18     perfthread.obj
 0001:00001e38       ??_C@_1BM@FMIOMJAE@?$AAV?$AAi?$AAr?$AAt?$AAu?$AAa?$AAl?$AA?5?$AAB?$AAy?$AAt?$AAe?$AAs@ 0000000180002e38     perfthread.obj
 0001:00001e58       ??_C@_1CG@KJOKFONA@?$AAV?$AAi?$AAr?$AAt?$AAu?$AAa?$AAl?$AA?5?$AAB?$AAy?$AAt?$AAe?$AAs?$AA?5?$AAP@ 0000000180002e58     perfthread.obj
 0001:00001e80       ??_C@_1CE@DFDFLLAO@?$AAI?$AAO?$AA?5?$AAD?$AAa?$AAt?$AAa?$AA?5?$AAB?$AAy?$AAt?$AAe?$AAs?$AA?1?$AAs@ 0000000180002e80     perfthread.obj
 0001:00001ea8       ??_C@_1CE@EFLEKJAB@?$AAI?$AAO?$AA?5?$AAR?$AAe?$AAa?$AAd?$AA?5?$AAB?$AAy?$AAt?$AAe?$AAs?$AA?1?$AAs@ 0000000180002ea8     perfthread.obj
 0001:00001ed0       ??_C@_1CG@MEJHKKKF@?$AAI?$AAO?$AA?5?$AAW?$AAr?$AAi?$AAt?$AAe?$AA?5?$AAB?$AAy?$AAt?$AAe?$AAs?$AA?1@ 0000000180002ed0     perfthread.obj
 0001:00001ef8       ??_C@_1CG@LBBBPCJA@?$AAI?$AAO?$AA?5?$AAO?$AAt?$AAh?$AAe?$AAr?$AA?5?$AAB?$AAy?$AAt?$AAe?$AAs?$AA?1@ 0000000180002ef8     perfthread.obj
 0001:00001f20       ??_C@_1CO@LIEOHDCC@?$AAI?$AAO?$AA?5?$AAD?$AAa?$AAt?$AAa?$AA?5?$AAO?$AAp?$AAe?$AAr?$AAa?$AAt?$AAi@ 0000000180002f20     perfthread.obj
 0001:00001f50       ??_C@_1CO@LIIKBHDH@?$AAI?$AAO?$AA?5?$AAR?$AAe?$AAa?$AAd?$AA?5?$AAO?$AAp?$AAe?$AAr?$AAa?$AAt?$AAi@ 0000000180002f50     perfthread.obj
 0001:00001f80       ??_C@_1DA@HICMAFKK@?$AAI?$AAO?$AA?5?$AAW?$AAr?$AAi?$AAt?$AAe?$AA?5?$AAO?$AAp?$AAe?$AAr?$AAa?$AAt@ 0000000180002f80     perfthread.obj
 0001:00001fb0       ??_C@_1DA@BEHINMGJ@?$AAI?$AAO?$AA?5?$AAO?$AAt?$AAh?$AAe?$AAr?$AA?5?$AAO?$AAp?$AAe?$AAr?$AAa?$AAt@ 0000000180002fb0     perfthread.obj
 0001:00001fe0       ??_C@_1HK@MEBPBHGJ@?$AAS?$AAo?$AAf?$AAt?$AAw?$AAa?$AAr?$AAe?$AA?2?$AAM?$AAi?$AAc?$AAr?$AAo?$AAs@ 0000000180002fe0     perfthread.obj
 0001:00002060       ??_C@_1BC@IICCDNLG@?$AAC?$AAo?$AAu?$AAn?$AAt?$AAe?$AAr?$AAs@ 0000000180003060     perfthread.obj
 0001:00002078       ??_C@_1BG@NKNJPBCD@?$AAI?$AAD?$AA?5?$AAP?$AAr?$AAo?$AAc?$AAe?$AAs?$AAs@ 0000000180003078     perfthread.obj
 0001:00002090       ??_C@_1BM@KCAKLHJN@?$AAP?$AAr?$AAi?$AAo?$AAr?$AAi?$AAt?$AAy?$AA?5?$AAB?$AAa?$AAs?$AAe@ 0000000180003090     perfthread.obj
 0001:000020b0       ??_C@_1BK@KCHPPKHP@?$AAT?$AAh?$AAr?$AAe?$AAa?$AAd?$AA?5?$AAC?$AAo?$AAu?$AAn?$AAt@ 00000001800030b0     perfthread.obj
 0001:000020d0       ??_C@_1CI@FNIEMNAI@?$AAC?$AAr?$AAe?$AAa?$AAt?$AAi?$AAn?$AAg?$AA?5?$AAP?$AAr?$AAo?$AAc?$AAe?$AAs@ 00000001800030d0     perfthread.obj
 0001:000020f8       ??_C@_1BK@IKAFHKBD@?$AAE?$AAl?$AAa?$AAp?$AAs?$AAe?$AAd?$AA?5?$AAT?$AAi?$AAm?$AAe@ 00000001800030f8     perfthread.obj
 0001:00002118       ??_C@_19DLCFHDFF@?$AAP?$AAE?$AAR?$AAF@ 0000000180003118     perfthread.obj
 0001:00002128       ??_C@_19DOGDICKI@?$AA?4?$AAe?$AAx?$AAe@ 0000000180003128     perfthread.obj
 0001:00002138       ??_C@_1O@NKAIMMPD@?$AA_?$AAT?$AAo?$AAt?$AAa?$AAl@ 0000000180003138     Plist.obj
 0001:00002148       ??_C@_1CC@DMDJMJLM@?$AAS?$AAe?$AAD?$AAe?$AAb?$AAu?$AAg?$AAP?$AAr?$AAi?$AAv?$AAi?$AAl?$AAe?$AAg@ 0000000180003148     Plist.obj
 0001:00002170       ??_C@_1BC@HFCOGKPP@?$AA?$HL?$AA0?$AA?$HN?$AA?6?$AA?$HL?$AA1?$AA?$HN?$AA?6@ 0000000180003170     Plist.obj
 0001:00002188       ??_C@_1M@DNHIACJI@?$AA?6?$AA?$HL?$AA0?$AA?$HN?$AA?6@ 0000000180003188     Plist.obj
 0001:00002198       ??_C@_1BG@JBKHLPML@?$AA?$HL?$AA0?$AA?$HN?$AA?5?$AA?$HL?$AA1?$AA?3?$AA8?$AAX?$AA?$HN@ 0000000180003198     Plist.obj
 0001:000021b0       ??_C@_19DPDNGGHD@?$AA?5?$AA?$HL?$AA0?$AA?$HN@ 00000001800031b0     Plist.obj
 0001:000021c0       ??_C@_1BE@EMDGEBAH@?$AA?$HL?$AA0?$AA?3?$AA0?$AA?$HL?$AA1?$AA?$HN?$AAX?$AA?$HN@ 00000001800031c0     Plist.obj
 0001:00002208       ??_7?$_Func_impl_no_alloc@V<lambda_c6a5923e4ab0669d9f7c2a6c892502eb>@@_NPEA_W_K@std@@6B@ 0000000180003208     Plist.obj
 0001:00002238       ??_C@_1CA@CCAFOKCB@?$AAE?$AAr?$AAr?$AAo?$AAr?$AA?5?$AA0?$AAx?$AA?$HL?$AA0?$AA?3?$AA0?$AA8?$AAX?$AA?$HN@ 0000000180003238     Pmix.obj
 0001:00002258       ??_C@_15JNBOKNOG@?$AA?$AN?$AA?6@ 0000000180003258     Pmix.obj
 0001:00002260       IID_IWbemLocator           0000000180003260     WMI.obj
 0001:00002270       CLSID_WbemLocator          0000000180003270     WMI.obj
 0001:00002280       ??_C@_1DC@LAIEFOLO@?$AAW?$AAi?$AAn?$AA3?$AA2?$AA_?$AAP?$AAr?$AAo?$AAc?$AAe?$AAs?$AAs?$AA?4?$AAH@ 0000000180003280     WMI.obj
 0001:000022b8       ??_C@_1BO@CLCOBGDE@?$AAE?$AAx?$AAe?$AAc?$AAu?$AAt?$AAa?$AAb?$AAl?$AAe?$AAP?$AAa?$AAt?$AAh@ 00000001800032b8     WMI.obj
 0001:000022d8       ??_C@_1BI@LPJNJKGA@?$AAC?$AAo?$AAm?$AAm?$AAa?$AAn?$AAd?$AAL?$AAi?$AAn?$AAe@ 00000001800032d8     WMI.obj
 0001:000022f0       ??_C@_1BC@JHNNEHFE@?$AAP?$AAr?$AAi?$AAo?$AAr?$AAi?$AAt?$AAy@ 00000001800032f0     WMI.obj
 0001:00002308       ??_C@_1BC@HJJANEGO@?$AAG?$AAe?$AAt?$AAO?$AAw?$AAn?$AAe?$AAr@ 0000000180003308     WMI.obj
 0001:00002320       ??_C@_19PIJILKAI@?$AAU?$AAs?$AAe?$AAr@ 0000000180003320     WMI.obj
 0001:00002330       ??_C@_1O@OAMNPMOM@?$AAD?$AAo?$AAm?$AAa?$AAi?$AAn@ 0000000180003330     WMI.obj
 0001:00002340       ??_C@_1BI@OIPNMPCL@?$AAG?$AAe?$AAt?$AAO?$AAw?$AAn?$AAe?$AAr?$AAS?$AAi?$AAd@ 0000000180003340     WMI.obj
 0001:00002358       ??_C@_17NKMLOKHF@?$AAS?$AAi?$AAd@ 0000000180003358     WMI.obj
 0001:00002360       ??_C@_1BE@CFEJJKFE@?$AAS?$AAe?$AAs?$AAs?$AAi?$AAo?$AAn?$AAI?$AAd@ 0000000180003360     WMI.obj
 0001:00002378       ??_C@_1BM@MLGLIGHJ@?$AAW?$AAi?$AAn?$AA3?$AA2?$AA_?$AAP?$AAr?$AAo?$AAc?$AAe?$AAs?$AAs@ 0000000180003378     WMI.obj
 0001:00002398       ??_C@_1BI@FLOHINJE@?$AAR?$AAe?$AAt?$AAu?$AAr?$AAn?$AAV?$AAa?$AAl?$AAu?$AAe@ 0000000180003398     WMI.obj
 0001:000023b0       ??_C@_1BI@NKNJJIDM@?$AAS?$AAe?$AAt?$AAP?$AAr?$AAi?$AAo?$AAr?$AAi?$AAt?$AAy@ 00000001800033b0     WMI.obj
 0001:000023c8       ??_C@_1O@GGHBFGJC@?$AAR?$AAe?$AAa?$AAs?$AAo?$AAn@ 00000001800033c8     WMI.obj
 0001:000023d8       ??_C@_1BE@PBPGMODO@?$AAT?$AAe?$AAr?$AAm?$AAi?$AAn?$AAa?$AAt?$AAe@ 00000001800033d8     WMI.obj
 0001:000023f0       ??_C@_1CC@OGNCBAIB@?$AA?2?$AA?2?$AA?$HL?$AA0?$AA?$HN?$AA?2?$AAr?$AAo?$AAo?$AAt?$AA?2?$AAc?$AAi?$AAm?$AAv@ 00000001800033f0     WMI.obj
 0001:00002414       ??_C@_13JOFGPIOO@?$AA?4@   0000000180003414     WMI.obj
 0001:00002478       MainGuid                   0000000180003478     Proclist.obj
 0001:00002488       MenuGuid                   0000000180003488     Proclist.obj
 0001:00002498       ConfigDialogGuid           0000000180003498     Proclist.obj
 0001:000024a8       ??_C@_1M@OAIMIKLP@?$AAn?$AAt?$AAd?$AAl?$AAl@ 00000001800034a8     Proclist.obj
 0001:000024b8       ??_C@_0BK@EGDDIFMK@NtQueryInformationProcess@ 00000001800034b8     Proclist.obj
 0001:000024d8       ??_C@_0BJ@HKKELGGC@NtQueryInformationThread@ 00000001800034d8     Proclist.obj
 0001:000024f8       ??_C@_0O@IFMDHOMC@NtQueryObject@ 00000001800034f8     Proclist.obj
 0001:00002508       ??_C@_0BJ@NDLOPGCH@NtQuerySystemInformation@ 0000000180003508     Proclist.obj
 0001:00002528       ??_C@_0BH@DLPGICA@NtQueryInformationFile@ 0000000180003528     Proclist.obj
 0001:00002540       ??_C@_0CB@GDPHBMJN@NtWow64QueryInformationProcess6@ 0000000180003540     Proclist.obj
 0001:00002568       ??_C@_0BL@NJDHCDMK@NtWow64ReadVirtualMemory64@ 0000000180003568     Proclist.obj
 0001:00002588       ??_C@_1BC@GDMECMAK@?$AAk?$AAe?$AAr?$AAn?$AAe?$AAl?$AA3?$AA2@ 0000000180003588     Proclist.obj
 0001:000025a0       ??_C@_0P@LKABJJMO@IsWow64Process@ 00000001800035a0     Proclist.obj
 0001:000025b0       ??_C@_1BC@DNHGCMLG@?$AAa?$AAd?$AAv?$AAa?$AAp?$AAi?$AA3?$AA2@ 00000001800035b0     Proclist.obj
 0001:000025c8       ??_C@_0L@KJHKJIPF@IsValidSid@ 00000001800035c8     Proclist.obj
 0001:000025d8       ??_C@_0BK@FIHGNING@GetSidIdentifierAuthority@ 00000001800035d8     Proclist.obj
 0001:000025f8       ??_C@_0BI@LPFJALDI@GetSidSubAuthorityCount@ 00000001800035f8     Proclist.obj
 0001:00002610       ??_C@_0BD@LMGFHOAE@GetSidSubAuthority@ 0000000180003610     Proclist.obj
 0001:00002628       ??_C@_1O@BCCLBEOE@?$AAu?$AAs?$AAe?$AAr?$AA3?$AA2@ 0000000180003628     Proclist.obj
 0001:00002638       ??_C@_0BA@FKGDNIJG@GetGuiResources@ 0000000180003638     Proclist.obj
 0001:00002648       ??_C@_1M@FFPAMFOB@?$AAo?$AAl?$AAe?$AA3?$AA2@ 0000000180003648     Proclist.obj
 0001:00002658       ??_C@_0BC@IOEGILCE@CoSetProxyBlanket@ 0000000180003658     Proclist.obj
 0001:00002670       ??_C@_1M@OMFDJDJC@?$AAp?$AAs?$AAa?$AAp?$AAi@ 0000000180003670     Proclist.obj
 0001:00002680       ??_C@_0BF@LEEEDPDK@EnumProcessModulesEx@ 0000000180003680     Proclist.obj
 0001:00002698       ??_C@_1BC@PDEABLIN@?$AAP?$AAr?$AAo?$AAc?$AAL?$AAi?$AAs?$AAt@ 0000000180003698     Proclist.obj
 0001:000026b0       ??_C@_1DK@DCAMPEPJ@?$AAP?$AAr?$AAo?$AAc?$AAe?$AAs?$AAs?$AA?5?$AAL?$AAi?$AAs?$AAt?$AA?5?$AAf?$AAo@ 00000001800036b0     Proclist.obj
 0001:000026f0       ??_C@_1DE@BGKMIKPD@?$AAE?$AAu?$AAg?$AAe?$AAn?$AAe?$AA?5?$AAR?$AAo?$AAs?$AAh?$AAa?$AAl?$AA?5?$AA?$CG@ 00000001800036f0     Proclist.obj
 0001:00002728       ??_C@_1M@MNPEKPKO@?$AAp?$AAl?$AAi?$AAs?$AAt@ 0000000180003728     Proclist.obj
 0001:00002740       ??_7exception@std@@6B@     0000000180003740     libcpmt:xthrow.obj
 0001:00002758       ??_7bad_alloc@std@@6B@     0000000180003758     libcpmt:xthrow.obj
 0001:00002768       ??_C@_0P@GHFPNOJB@bad?5allocation@ 0000000180003768     libcpmt:xthrow.obj
 0001:00002780       ??_7logic_error@std@@6B@   0000000180003780     libcpmt:xthrow.obj
 0001:00002798       ??_7length_error@std@@6B@  0000000180003798     libcpmt:xthrow.obj
 0001:000027b0       ??_7out_of_range@std@@6B@  00000001800037b0     libcpmt:xthrow.obj
 0001:000027c8       ??_7runtime_error@std@@6B@ 00000001800037c8     libcpmt:xthrow.obj
 0001:000027e0       ??_7bad_function_call@std@@6B@ 00000001800037e0     libcpmt:xthrow.obj
 0001:000027f0       ??_C@_0BC@DPJNKNAF@bad?5function?5call@ 00000001800037f0     libcpmt:xthrow.obj
 0001:00002838       ??_7_Facet_base@std@@6B@   0000000180003838     libcpmt:locale0.obj
 0001:00002858       ??_7_Locimp@locale@std@@6B@ 0000000180003858     libcpmt:locale0.obj
 0001:00002870       ??_C@_01NBENCBCI@?$CK@     0000000180003870     libcpmt:locale0.obj
 0001:00002874       ??_C@_01GFHCPBMG@C@        0000000180003874     libcpmt:locale0.obj
 0001:00002880       ??_7bad_array_new_length@std@@6B@ 0000000180003880     libcpmt:locale.obj
 0001:00002898       ??_7bad_cast@std@@6B@      0000000180003898     libcpmt:locale.obj
 0001:000028d0       ??_C@_1BK@MGMFAEKH@?$AAk?$AAe?$AAr?$AAn?$AAe?$AAl?$AA3?$AA2?$AA?4?$AAd?$AAl?$AAl@ 00000001800038d0     libcpmt:winapisupp.obj
 0001:000028f0       ??_C@_08KNHFBNJ@FlsAlloc@  00000001800038f0     libcpmt:winapisupp.obj
 0001:00002900       ??_C@_07PEJMOBNF@FlsFree@  0000000180003900     libcpmt:winapisupp.obj
 0001:00002908       ??_C@_0M@GDNOONDI@FlsGetValue@ 0000000180003908     libcpmt:winapisupp.obj
 0001:00002918       ??_C@_0M@JCPCPOEF@FlsSetValue@ 0000000180003918     libcpmt:winapisupp.obj
 0001:00002928       ??_C@_0BM@HCFOFFN@InitializeCriticalSectionEx@ 0000000180003928     libcpmt:winapisupp.obj
 0001:00002948       ??_C@_0BE@GPLMMCMH@InitOnceExecuteOnce@ 0000000180003948     libcpmt:winapisupp.obj
 0001:00002960       ??_C@_0P@DLHPPCNH@CreateEventExW@ 0000000180003960     libcpmt:winapisupp.obj
 0001:00002970       ??_C@_0BB@MEFPJLHN@CreateSemaphoreW@ 0000000180003970     libcpmt:winapisupp.obj
 0001:00002988       ??_C@_0BD@KIEEOEEH@CreateSemaphoreExW@ 0000000180003988     libcpmt:winapisupp.obj
 0001:000029a0       ??_C@_0BG@OGFAJCKC@CreateThreadpoolTimer@ 00000001800039a0     libcpmt:winapisupp.obj
 0001:000029b8       ??_C@_0BD@LPLEMMDI@SetThreadpoolTimer@ 00000001800039b8     libcpmt:winapisupp.obj
 0001:000029d0       ??_C@_0CA@FMNJENH@WaitForThreadpoolTimerCallbacks@ 00000001800039d0     libcpmt:winapisupp.obj
 0001:000029f0       ??_C@_0BF@DCFCCNOC@CloseThreadpoolTimer@ 00000001800039f0     libcpmt:winapisupp.obj
 0001:00002a08       ??_C@_0BF@FLABGKKM@CreateThreadpoolWait@ 0000000180003a08     libcpmt:winapisupp.obj
 0001:00002a20       ??_C@_0BC@MGCOHNA@SetThreadpoolWait@ 0000000180003a20     libcpmt:winapisupp.obj
 0001:00002a38       ??_C@_0BE@OCIOMIMP@CloseThreadpoolWait@ 0000000180003a38     libcpmt:winapisupp.obj
 0001:00002a50       ??_C@_0BJ@LKGHFHBO@FlushProcessWriteBuffers@ 0000000180003a50     libcpmt:winapisupp.obj
 0001:00002a70       ??_C@_0BP@KALKKPMO@FreeLibraryWhenCallbackReturns@ 0000000180003a70     libcpmt:winapisupp.obj
 0001:00002a90       ??_C@_0BK@DFNBACLA@GetCurrentProcessorNumber@ 0000000180003a90     libcpmt:winapisupp.obj
 0001:00002ab0       ??_C@_0BE@FKKLLFLM@CreateSymbolicLinkW@ 0000000180003ab0     libcpmt:winapisupp.obj
 0001:00002ac8       ??_C@_0BE@JOGNEJCI@GetCurrentPackageId@ 0000000180003ac8     libcpmt:winapisupp.obj
 0001:00002ae0       ??_C@_0P@CDHHOHKP@GetTickCount64@ 0000000180003ae0     libcpmt:winapisupp.obj
 0001:00002af0       ??_C@_0BN@NEEHBBPO@GetFileInformationByHandleEx@ 0000000180003af0     libcpmt:winapisupp.obj
 0001:00002b10       ??_C@_0BL@KBBHGKCM@SetFileInformationByHandle@ 0000000180003b10     libcpmt:winapisupp.obj
 0001:00002b30       ??_C@_0BP@FPNJPEJC@GetSystemTimePreciseAsFileTime@ 0000000180003b30     libcpmt:winapisupp.obj
 0001:00002b50       ??_C@_0BM@HLJJNPAH@InitializeConditionVariable@ 0000000180003b50     libcpmt:winapisupp.obj
 0001:00002b70       ??_C@_0BG@BFNILBLN@WakeConditionVariable@ 0000000180003b70     libcpmt:winapisupp.obj
 0001:00002b88       ??_C@_0BJ@PGPPEPCC@WakeAllConditionVariable@ 0000000180003b88     libcpmt:winapisupp.obj
 0001:00002ba8       ??_C@_0BJ@JEBJOJFJ@SleepConditionVariableCS@ 0000000180003ba8     libcpmt:winapisupp.obj
 0001:00002bc8       ??_C@_0BC@MMLHEBPB@InitializeSRWLock@ 0000000180003bc8     libcpmt:winapisupp.obj
 0001:00002be0       ??_C@_0BI@OMNLIJDB@AcquireSRWLockExclusive@ 0000000180003be0     libcpmt:winapisupp.obj
 0001:00002bf8       ??_C@_0BL@OGHFEMNA@TryAcquireSRWLockExclusive@ 0000000180003bf8     libcpmt:winapisupp.obj
 0001:00002c18       ??_C@_0BI@HMIEPCNJ@ReleaseSRWLockExclusive@ 0000000180003c18     libcpmt:winapisupp.obj
 0001:00002c30       ??_C@_0BK@LGACAGIC@SleepConditionVariableSRW@ 0000000180003c30     libcpmt:winapisupp.obj
 0001:00002c50       ??_C@_0BF@GGPHFPJA@CreateThreadpoolWork@ 0000000180003c50     libcpmt:winapisupp.obj
 0001:00002c68       ??_C@_0BF@NHDAIMMO@SubmitThreadpoolWork@ 0000000180003c68     libcpmt:winapisupp.obj
 0001:00002c80       ??_C@_0BE@NPHIPNPD@CloseThreadpoolWork@ 0000000180003c80     libcpmt:winapisupp.obj
 0001:00002c98       ??_C@_0BA@IHGNDAEB@CompareStringEx@ 0000000180003c98     libcpmt:winapisupp.obj
 0001:00002ca8       ??_C@_0BA@ONOKGCMP@GetLocaleInfoEx@ 0000000180003ca8     libcpmt:winapisupp.obj
 0001:00002cb8       ??_C@_0O@KKBNKAPF@LCMapStringEx@ 0000000180003cb8     libcpmt:winapisupp.obj
 0001:00002cd0       ??_7?$numpunct@_W@std@@6B@ 0000000180003cd0     libcpmt:wlocale.obj
 0001:00002d10       ??_C@_13IMODFHAA@?$AA?9@   0000000180003d10     libcpmt:wlocale.obj
 0001:00002d14       ??_C@_01JOAMLHOP@?9@       0000000180003d14     libcpmt:wlocale.obj
 0001:00004a40       ??_C@_15EMKDOKLE@?$AAa?$AAr@ 0000000180005a40     libcpmt:winapinls.obj
 0001:00004a48       ??_C@_15KNPADPLH@?$AAb?$AAg@ 0000000180005a48     libcpmt:winapinls.obj
 0001:00004a50       ??_C@_15EDMHLDMO@?$AAc?$AAa@ 0000000180005a50     libcpmt:winapinls.obj
 0001:00004a58       ??_C@_1O@BPEAJADD@?$AAz?$AAh?$AA?9?$AAC?$AAH?$AAS@ 0000000180005a58     libcpmt:winapinls.obj
 0001:00004a68       ??_C@_15LJNHCMNK@?$AAc?$AAs@ 0000000180005a68     libcpmt:winapinls.obj
 0001:00004a70       ??_C@_15FOMCIDHG@?$AAd?$AAa@ 0000000180005a70     libcpmt:winapinls.obj
 0001:00004a78       ??_C@_15NBKABECB@?$AAd?$AAe@ 0000000180005a78     libcpmt:winapinls.obj
 0001:00004a80       ??_C@_15GHPEIIAO@?$AAe?$AAl@ 0000000180005a80     libcpmt:winapinls.obj
 0001:00004a88       ??_C@_15MNPNEAIF@?$AAe?$AAn@ 0000000180005a88     libcpmt:winapinls.obj
 0001:00004a90       ??_C@_15GPIOMPMH@?$AAe?$AAs@ 0000000180005a90     libcpmt:winapinls.obj
 0001:00004a98       ??_C@_15NGLOAKJC@?$AAf?$AAi@ 0000000180005a98     libcpmt:winapinls.obj
 0001:00004aa0       ??_C@_15FBKGNKAM@?$AAf?$AAr@ 0000000180005aa0     libcpmt:winapinls.obj
 0001:00004aa8       ??_C@_15KGGCNEFK@?$AAh?$AAe@ 0000000180005aa8     libcpmt:winapinls.obj
 0001:00004ab0       ??_C@_15PGHLIDMF@?$AAh?$AAu@ 0000000180005ab0     libcpmt:winapinls.obj
 0001:00004ab8       ??_C@_15BIEMAPLM@?$AAi?$AAs@ 0000000180005ab8     libcpmt:winapinls.obj
 0001:00004ac0       ??_C@_15IFJLDHAF@?$AAi?$AAt@ 0000000180005ac0     libcpmt:winapinls.obj
 0001:00004ac8       ??_C@_15GEMIOCAG@?$AAj?$AAa@ 0000000180005ac8     libcpmt:winapinls.obj
 0001:00004ad0       ??_C@_15EPELEGJA@?$AAk?$AAo@ 0000000180005ad0     libcpmt:winapinls.obj
 0001:00004ad8       ??_C@_15NDDHIMN@?$AAn?$AAl@ 0000000180005ad8     libcpmt:winapinls.obj
 0001:00004ae0       ??_C@_15BPIGNHCD@?$AAn?$AAo@ 0000000180005ae0     libcpmt:winapinls.obj
 0001:00004ae8       ??_C@_15DEOPBLCG@?$AAp?$AAl@ 0000000180005ae8     libcpmt:winapinls.obj
 0001:00004af0       ??_C@_15KBECGEFG@?$AAp?$AAt@ 0000000180005af0     libcpmt:winapinls.obj
 0001:00004af8       ??_C@_15GLJCBFMD@?$AAr?$AAo@ 0000000180005af8     libcpmt:winapinls.obj
 0001:00004b00       ??_C@_15FEDGKCDI@?$AAr?$AAu@ 0000000180005b00     libcpmt:winapinls.obj
 0001:00004b08       ??_C@_15GLKMLLHM@?$AAh?$AAr@ 0000000180005b08     libcpmt:winapinls.obj
 0001:00004b10       ??_C@_15CPKMFBDB@?$AAs?$AAk@ 0000000180005b10     libcpmt:winapinls.obj
 0001:00004b18       ??_C@_15BAAIOGMK@?$AAs?$AAq@ 0000000180005b18     libcpmt:winapinls.obj
 0001:00004b20       ??_C@_15INNPNOHD@?$AAs?$AAv@ 0000000180005b20     libcpmt:winapinls.obj
 0001:00004b28       ??_C@_15CABMMOGH@?$AAt?$AAh@ 0000000180005b28     libcpmt:winapinls.obj
 0001:00004b30       ??_C@_15BPLIHJJM@?$AAt?$AAr@ 0000000180005b30     libcpmt:winapinls.obj
 0001:00004b38       ??_C@_15NEOEKKDJ@?$AAu?$AAr@ 0000000180005b38     libcpmt:winapinls.obj
 0001:00004b40       ??_C@_15NFICGAJK@?$AAi?$AAd@ 0000000180005b40     libcpmt:winapinls.obj
 0001:00004b48       ??_C@_15PJPFLCCM@?$AAu?$AAk@ 0000000180005b48     libcpmt:winapinls.obj
 0001:00004b50       ??_C@_15HPJPHDM@?$AAb?$AAe@ 0000000180005b50     libcpmt:winapinls.obj
 0001:00004b58       ??_C@_15LCHLGJII@?$AAs?$AAl@ 0000000180005b58     libcpmt:winapinls.obj
 0001:00004b60       ??_C@_15PCFJPHHO@?$AAe?$AAt@ 0000000180005b60     libcpmt:winapinls.obj
 0001:00004b68       ??_C@_15HPFPGODN@?$AAl?$AAv@ 0000000180005b68     libcpmt:winapinls.obj
 0001:00004b70       ??_C@_15NFFGKGLG@?$AAl?$AAt@ 0000000180005b70     libcpmt:winapinls.obj
 0001:00004b78       ??_C@_15BDAKCCHN@?$AAf?$AAa@ 0000000180005b78     libcpmt:winapinls.obj
 0001:00004b80       ??_C@_15NFGIAIAJ@?$AAv?$AAi@ 0000000180005b80     libcpmt:winapinls.obj
 0001:00004b88       ??_C@_15LMKNDMHN@?$AAh?$AAy@ 0000000180005b88     libcpmt:winapinls.obj
 0001:00004b90       ??_C@_15IJBHMCFL@?$AAa?$AAz@ 0000000180005b90     libcpmt:winapinls.obj
 0001:00004b98       ??_C@_15EKOFJABL@?$AAe?$AAu@ 0000000180005b98     libcpmt:winapinls.obj
 0001:00004ba0       ??_C@_15BGHADCNK@?$AAm?$AAk@ 0000000180005ba0     libcpmt:winapinls.obj
 0001:00004ba8       ??_C@_15JDNICKHM@?$AAa?$AAf@ 0000000180005ba8     libcpmt:winapinls.obj
 0001:00004bb0       ??_C@_15KPJEDBKD@?$AAk?$AAa@ 0000000180005bb0     libcpmt:winapinls.obj
 0001:00004bb8       ??_C@_15PDNFFFEO@?$AAf?$AAo@ 0000000180005bb8     libcpmt:winapinls.obj
 0001:00004bc0       ??_C@_15OMLEGLOC@?$AAh?$AAi@ 0000000180005bc0     libcpmt:winapinls.obj
 0001:00004bc8       ??_C@_15IDNNENKK@?$AAm?$AAs@ 0000000180005bc8     libcpmt:winapinls.obj
 0001:00004bd0       ??_C@_15MACJNBMH@?$AAk?$AAk@ 0000000180005bd0     libcpmt:winapinls.obj
 0001:00004bd8       ??_C@_15DKDJEOND@?$AAk?$AAy@ 0000000180005bd8     libcpmt:winapinls.obj
 0001:00004be0       ??_C@_15DFGDLJBG@?$AAs?$AAw@ 0000000180005be0     libcpmt:winapinls.obj
 0001:00004be8       ??_C@_15BBFAICNG@?$AAu?$AAz@ 0000000180005be8     libcpmt:winapinls.obj
 0001:00004bf0       ??_C@_15DKNDCGEA@?$AAt?$AAt@ 0000000180005bf0     libcpmt:winapinls.obj
 0001:00004bf8       ??_C@_15MGIFMDPL@?$AAp?$AAa@ 0000000180005bf8     libcpmt:winapinls.obj
 0001:00004c00       ??_C@_15HCNDBBA@?$AAg?$AAu@ 0000000180005c00     libcpmt:winapinls.obj
 0001:00004c08       ??_C@_15FNBEIBON@?$AAt?$AAa@ 0000000180005c08     libcpmt:winapinls.obj
 0001:00004c10       ??_C@_15NCHGBGLK@?$AAt?$AAe@ 0000000180005c10     libcpmt:winapinls.obj
 0001:00004c18       ??_C@_15PHPHCBPF@?$AAk?$AAn@ 0000000180005c18     libcpmt:winapinls.obj
 0001:00004c20       ??_C@_15DLGBCKMP@?$AAm?$AAr@ 0000000180005c20     libcpmt:winapinls.obj
 0001:00004c28       ??_C@_15EABBLBFF@?$AAs?$AAa@ 0000000180005c28     libcpmt:winapinls.obj
 0001:00004c30       ??_C@_15CBKOMCOI@?$AAm?$AAn@ 0000000180005c30     libcpmt:winapinls.obj
 0001:00004c38       ??_C@_15CKDMCJAF@?$AAg?$AAl@ 0000000180005c38     libcpmt:winapinls.obj
 0001:00004c40       ??_C@_17CNJFBPG@?$AAk?$AAo?$AAk@ 0000000180005c40     libcpmt:winapinls.obj
 0001:00004c48       ??_C@_17FFBJICPL@?$AAs?$AAy?$AAr@ 0000000180005c48     libcpmt:winapinls.obj
 0001:00004c50       ??_C@_17KPNDCPAF@?$AAd?$AAi?$AAv@ 0000000180005c50     libcpmt:winapinls.obj
 0001:00004c58       ??_C@_1M@OKAHONE@?$AAa?$AAr?$AA?9?$AAS?$AAA@ 0000000180005c58     libcpmt:winapinls.obj
 0001:00004c68       ??_C@_1M@FFFIGIGK@?$AAb?$AAg?$AA?9?$AAB?$AAG@ 0000000180005c68     libcpmt:winapinls.obj
 0001:00004c78       ??_C@_1M@BJNKEDC@?$AAc?$AAa?$AA?9?$AAE?$AAS@ 0000000180005c78     libcpmt:winapinls.obj
 0001:00004c88       ??_C@_1M@CLNBBOPM@?$AAz?$AAh?$AA?9?$AAT?$AAW@ 0000000180005c88     libcpmt:winapinls.obj
 0001:00004c98       ??_C@_1M@IJJHFJHA@?$AAc?$AAs?$AA?9?$AAC?$AAZ@ 0000000180005c98     libcpmt:winapinls.obj
 0001:00004ca8       ??_C@_1M@CLPEOBGI@?$AAd?$AAa?$AA?9?$AAD?$AAK@ 0000000180005ca8     libcpmt:winapinls.obj
 0001:00004cb8       ??_C@_1M@MCMADGCB@?$AAd?$AAe?$AA?9?$AAD?$AAE@ 0000000180005cb8     libcpmt:winapinls.obj
 0001:00004cc8       ??_C@_1M@OOCKEMAM@?$AAe?$AAl?$AA?9?$AAG?$AAR@ 0000000180005cc8     libcpmt:winapinls.obj
 0001:00004cd8       ??_C@_1M@BMHNFIME@?$AAe?$AAn?$AA?9?$AAU?$AAS@ 0000000180005cd8     libcpmt:winapinls.obj
 0001:00004ce8       ??_C@_1M@DDNJFGID@?$AAf?$AAi?$AA?9?$AAF?$AAI@ 0000000180005ce8     libcpmt:winapinls.obj
 0001:00004cf8       ??_C@_1M@GLIPPMAC@?$AAf?$AAr?$AA?9?$AAF?$AAR@ 0000000180005cf8     libcpmt:winapinls.obj
 0001:00004d08       ??_C@_1M@GFMCHPE@?$AAh?$AAe?$AA?9?$AAI?$AAL@ 0000000180005d08     libcpmt:winapinls.obj
 0001:00004d18       ??_C@_1M@MHLPGNKM@?$AAh?$AAu?$AA?9?$AAH?$AAU@ 0000000180005d18     libcpmt:winapinls.obj
 0001:00004d28       ??_C@_1M@LPDDNNPN@?$AAi?$AAs?$AA?9?$AAI?$AAS@ 0000000180005d28     libcpmt:winapinls.obj
 0001:00004d38       ??_C@_1M@MADIPODN@?$AAi?$AAt?$AA?9?$AAI?$AAT@ 0000000180005d38     libcpmt:winapinls.obj
 0001:00004d48       ??_C@_1M@HPNHIDJI@?$AAj?$AAa?$AA?9?$AAJ?$AAP@ 0000000180005d48     libcpmt:winapinls.obj
 0001:00004d58       ??_C@_1M@JLOOOEGK@?$AAk?$AAo?$AA?9?$AAK?$AAR@ 0000000180005d58     libcpmt:winapinls.obj
 0001:00004d68       ??_C@_1M@IHBJJGG@?$AAn?$AAl?$AA?9?$AAN?$AAL@ 0000000180005d68     libcpmt:winapinls.obj
 0001:00004d78       ??_C@_1M@EANAGDL@?$AAn?$AAb?$AA?9?$AAN?$AAO@ 0000000180005d78     libcpmt:winapinls.obj
 0001:00004d88       ??_C@_1M@NEIEMEGP@?$AAp?$AAl?$AA?9?$AAP?$AAL@ 0000000180005d88     libcpmt:winapinls.obj
 0001:00004d98       ??_C@_1M@BOCFIGEP@?$AAp?$AAt?$AA?9?$AAB?$AAR@ 0000000180005d98     libcpmt:winapinls.obj
 0001:00004da8       ??_C@_1M@IMPFOPBG@?$AAr?$AAo?$AA?9?$AAR?$AAO@ 0000000180005da8     libcpmt:winapinls.obj
 0001:00004db8       ??_C@_1M@IDNNEJMM@?$AAr?$AAu?$AA?9?$AAR?$AAU@ 0000000180005db8     libcpmt:winapinls.obj
 0001:00004dc8       ??_C@_1M@LILEEOGM@?$AAh?$AAr?$AA?9?$AAH?$AAR@ 0000000180005dc8     libcpmt:winapinls.obj
 0001:00004dd8       ??_C@_1M@FKIFEHPB@?$AAs?$AAk?$AA?9?$AAS?$AAK@ 0000000180005dd8     libcpmt:winapinls.obj
 0001:00004de8       ??_C@_1M@LJMAMNPJ@?$AAs?$AAq?$AA?9?$AAA?$AAL@ 0000000180005de8     libcpmt:winapinls.obj
 0001:00004df8       ??_C@_1M@GIAKDKJK@?$AAs?$AAv?$AA?9?$AAS?$AAE@ 0000000180005df8     libcpmt:winapinls.obj
 0001:00004e08       ??_C@_1M@MKJKIKCL@?$AAt?$AAh?$AA?9?$AAT?$AAH@ 0000000180005e08     libcpmt:winapinls.obj
 0001:00004e18       ??_C@_1M@MFLCCMPB@?$AAt?$AAr?$AA?9?$AAT?$AAR@ 0000000180005e18     libcpmt:winapinls.obj
 0001:00004e28       ??_C@_1M@OIJHDKJN@?$AAu?$AAr?$AA?9?$AAP?$AAK@ 0000000180005e28     libcpmt:winapinls.obj
 0001:00004e38       ??_C@_1M@LHIPCIEK@?$AAi?$AAd?$AA?9?$AAI?$AAD@ 0000000180005e38     libcpmt:winapinls.obj
 0001:00004e48       ??_C@_1M@MFMOBGI@?$AAu?$AAk?$AA?9?$AAU?$AAA@ 0000000180005e48     libcpmt:winapinls.obj
 0001:00004e58       ??_C@_1M@OBGLJIPL@?$AAb?$AAe?$AA?9?$AAB?$AAY@ 0000000180005e58     libcpmt:winapinls.obj
 0001:00004e68       ??_C@_1M@BCFAJEAD@?$AAs?$AAl?$AA?9?$AAS?$AAI@ 0000000180005e68     libcpmt:winapinls.obj
 0001:00004e78       ??_C@_1M@FKFFEDDN@?$AAe?$AAt?$AA?9?$AAE?$AAE@ 0000000180005e78     libcpmt:winapinls.obj
 0001:00004e88       ??_C@_1M@KGKKAACI@?$AAl?$AAv?$AA?9?$AAL?$AAV@ 0000000180005e88     libcpmt:winapinls.obj
 0001:00004e98       ??_C@_1M@IFGBIJO@?$AAl?$AAt?$AA?9?$AAL?$AAT@ 0000000180005e98     libcpmt:winapinls.obj
 0001:00004ea8       ??_C@_1M@FGEAHEDM@?$AAf?$AAa?$AA?9?$AAI?$AAR@ 0000000180005ea8     libcpmt:winapinls.obj
 0001:00004eb8       ??_C@_1M@KBMAIBFN@?$AAv?$AAi?$AA?9?$AAV?$AAN@ 0000000180005eb8     libcpmt:winapinls.obj
 0001:00004ec8       ??_C@_1M@GPCBKDJK@?$AAh?$AAy?$AA?9?$AAA?$AAM@ 0000000180005ec8     libcpmt:winapinls.obj
 0001:00004ed8       ??_C@_1BG@BECMDDJB@?$AAa?$AAz?$AA?9?$AAA?$AAZ?$AA?9?$AAL?$AAa?$AAt?$AAn@ 0000000180005ed8     libcpmt:winapinls.obj
 0001:00004ef0       ??_C@_1M@MAOFCAEA@?$AAe?$AAu?$AA?9?$AAE?$AAS@ 0000000180005ef0     libcpmt:winapinls.obj
 0001:00004f00       ??_C@_1M@IGHABKPI@?$AAm?$AAk?$AA?9?$AAM?$AAK@ 0000000180005f00     libcpmt:winapinls.obj
 0001:00004f10       ??_C@_1M@IAIGNEJG@?$AAt?$AAn?$AA?9?$AAZ?$AAA@ 0000000180005f10     libcpmt:winapinls.obj
 0001:00004f20       ??_C@_1M@IIJCOJFA@?$AAx?$AAh?$AA?9?$AAZ?$AAA@ 0000000180005f20     libcpmt:winapinls.obj
 0001:00004f30       ??_C@_1M@LGPJHNJH@?$AAz?$AAu?$AA?9?$AAZ?$AAA@ 0000000180005f30     libcpmt:winapinls.obj
 0001:00004f40       ??_C@_1M@HOKAOIO@?$AAa?$AAf?$AA?9?$AAZ?$AAA@ 0000000180005f40     libcpmt:winapinls.obj
 0001:00004f50       ??_C@_1M@DPCLHLIE@?$AAk?$AAa?$AA?9?$AAG?$AAE@ 0000000180005f50     libcpmt:winapinls.obj
 0001:00004f60       ??_C@_1M@BLKMHJBI@?$AAf?$AAo?$AA?9?$AAF?$AAO@ 0000000180005f60     libcpmt:winapinls.obj
 0001:00004f70       ??_C@_1M@LGGJAPPB@?$AAh?$AAi?$AA?9?$AAI?$AAN@ 0000000180005f70     libcpmt:winapinls.obj
 0001:00004f80       ??_C@_1M@FIKPIHFE@?$AAm?$AAt?$AA?9?$AAM?$AAT@ 0000000180005f80     libcpmt:winapinls.obj
 0001:00004f90       ??_C@_1M@HEGGPBFA@?$AAs?$AAe?$AA?9?$AAN?$AAO@ 0000000180005f90     libcpmt:winapinls.obj
 0001:00004fa0       ??_C@_1M@EIBJEEPA@?$AAm?$AAs?$AA?9?$AAM?$AAY@ 0000000180005fa0     libcpmt:winapinls.obj
 0001:00004fb0       ??_C@_1M@FHLBGMPP@?$AAk?$AAk?$AA?9?$AAK?$AAZ@ 0000000180005fb0     libcpmt:winapinls.obj
 0001:00004fc0       ??_C@_1M@NGJJLCGI@?$AAk?$AAy?$AA?9?$AAK?$AAG@ 0000000180005fc0     libcpmt:winapinls.obj
 0001:00004fd0       ??_C@_1M@GIENNBFC@?$AAs?$AAw?$AA?9?$AAK?$AAE@ 0000000180005fd0     libcpmt:winapinls.obj
 0001:00004fe0       ??_C@_1BG@NDGMJIMJ@?$AAu?$AAz?$AA?9?$AAU?$AAZ?$AA?9?$AAL?$AAa?$AAt?$AAn@ 0000000180005fe0     libcpmt:winapinls.obj
 0001:00004ff8       ??_C@_1M@IDCCIHBC@?$AAt?$AAt?$AA?9?$AAR?$AAU@ 0000000180005ff8     libcpmt:winapinls.obj
 0001:00005008       ??_C@_1M@LOICPMOJ@?$AAb?$AAn?$AA?9?$AAI?$AAN@ 0000000180006008     libcpmt:winapinls.obj
 0001:00005018       ??_C@_1M@KPKKNEAH@?$AAp?$AAa?$AA?9?$AAI?$AAN@ 0000000180006018     libcpmt:winapinls.obj
 0001:00005028       ??_C@_1M@PJGPPBOG@?$AAg?$AAu?$AA?9?$AAI?$AAN@ 0000000180006028     libcpmt:winapinls.obj
 0001:00005038       ??_C@_1M@KMKMOPHI@?$AAt?$AAa?$AA?9?$AAI?$AAN@ 0000000180006038     libcpmt:winapinls.obj
 0001:00005048       ??_C@_1M@KFEHEPAC@?$AAt?$AAe?$AA?9?$AAI?$AAN@ 0000000180006048     libcpmt:winapinls.obj
 0001:00005058       ??_C@_1M@CDCLMGHI@?$AAk?$AAn?$AA?9?$AAI?$AAN@ 0000000180006058     libcpmt:winapinls.obj
 0001:00005068       ??_C@_1M@MIODLDKF@?$AAm?$AAl?$AA?9?$AAI?$AAN@ 0000000180006068     libcpmt:winapinls.obj
 0001:00005078       ??_C@_1M@PBIEACPO@?$AAm?$AAr?$AA?9?$AAI?$AAN@ 0000000180006078     libcpmt:winapinls.obj
 0001:00005088       ??_C@_1M@NIDEAGPH@?$AAs?$AAa?$AA?9?$AAI?$AAN@ 0000000180006088     libcpmt:winapinls.obj
 0001:00005098       ??_C@_1M@FHIHCBIO@?$AAm?$AAn?$AA?9?$AAM?$AAN@ 0000000180006098     libcpmt:winapinls.obj
 0001:000050a8       ??_C@_1M@JAIJPENP@?$AAc?$AAy?$AA?9?$AAG?$AAB@ 00000001800060a8     libcpmt:winapinls.obj
 0001:000050b8       ??_C@_1M@PHGFBEPN@?$AAg?$AAl?$AA?9?$AAE?$AAS@ 00000001800060b8     libcpmt:winapinls.obj
 0001:000050c8       ??_C@_1O@KPIPDNCP@?$AAk?$AAo?$AAk?$AA?9?$AAI?$AAN@ 00000001800060c8     libcpmt:winapinls.obj
 0001:000050d8       ??_C@_1O@KNHJLDJA@?$AAs?$AAy?$AAr?$AA?9?$AAS?$AAY@ 00000001800060d8     libcpmt:winapinls.obj
 0001:000050e8       ??_C@_1O@MKEKBLAH@?$AAd?$AAi?$AAv?$AA?9?$AAM?$AAV@ 00000001800060e8     libcpmt:winapinls.obj
 0001:000050f8       ??_C@_1O@OHDCKDDF@?$AAq?$AAu?$AAz?$AA?9?$AAB?$AAO@ 00000001800060f8     libcpmt:winapinls.obj
 0001:00005108       ??_C@_1M@LEPJNLFD@?$AAn?$AAs?$AA?9?$AAZ?$AAA@ 0000000180006108     libcpmt:winapinls.obj
 0001:00005118       ??_C@_1M@OMLEIIJB@?$AAm?$AAi?$AA?9?$AAN?$AAZ@ 0000000180006118     libcpmt:winapinls.obj
 0001:00005128       ??_C@_1M@PMPEAILG@?$AAa?$AAr?$AA?9?$AAI?$AAQ@ 0000000180006128     libcpmt:winapinls.obj
 0001:00005138       ??_C@_1M@BIBDDEMK@?$AAz?$AAh?$AA?9?$AAC?$AAN@ 0000000180006138     libcpmt:winapinls.obj
 0001:00005148       ??_C@_1M@CNKPNOEE@?$AAd?$AAe?$AA?9?$AAC?$AAH@ 0000000180006148     libcpmt:winapinls.obj
 0001:00005158       ??_C@_1M@LKMGMLKO@?$AAe?$AAn?$AA?9?$AAG?$AAB@ 0000000180006158     libcpmt:winapinls.obj
 0001:00005168       ??_C@_1M@PGKJFFGL@?$AAe?$AAs?$AA?9?$AAM?$AAX@ 0000000180006168     libcpmt:winapinls.obj
 0001:00005178       ??_C@_1M@DNNANBDC@?$AAf?$AAr?$AA?9?$AAB?$AAE@ 0000000180006178     libcpmt:winapinls.obj
 0001:00005188       ??_C@_1M@HLGMDFHM@?$AAi?$AAt?$AA?9?$AAC?$AAH@ 0000000180006188     libcpmt:winapinls.obj
 0001:00005198       ??_C@_1M@CLLBGJH@?$AAn?$AAl?$AA?9?$AAB?$AAE@ 0000000180006198     libcpmt:winapinls.obj
 0001:000051a8       ??_C@_1M@BODBOGLF@?$AAn?$AAn?$AA?9?$AAN?$AAO@ 00000001800061a8     libcpmt:winapinls.obj
 0001:000051b8       ??_C@_1M@HFFAHKAD@?$AAp?$AAt?$AA?9?$AAP?$AAT@ 00000001800061b8     libcpmt:winapinls.obj
 0001:000051c8       ??_C@_1BG@LNOAKHIE@?$AAs?$AAr?$AA?9?$AAS?$AAP?$AA?9?$AAL?$AAa?$AAt?$AAn@ 00000001800061c8     libcpmt:winapinls.obj
 0001:000051e0       ??_C@_1M@HBMHBGAK@?$AAs?$AAv?$AA?9?$AAF?$AAI@ 00000001800061e0     libcpmt:winapinls.obj
 0001:000051f0       ??_C@_1BG@DGCJGJBE@?$AAa?$AAz?$AA?9?$AAA?$AAZ?$AA?9?$AAC?$AAy?$AAr?$AAl@ 00000001800061f0     libcpmt:winapinls.obj
 0001:00005208       ??_C@_1M@KEJDAAHB@?$AAs?$AAe?$AA?9?$AAS?$AAE@ 0000000180006208     libcpmt:winapinls.obj
 0001:00005218       ??_C@_1M@HEIBJJAD@?$AAm?$AAs?$AA?9?$AAB?$AAN@ 0000000180006218     libcpmt:winapinls.obj
 0001:00005228       ??_C@_1BG@PBGJMCEM@?$AAu?$AAz?$AA?9?$AAU?$AAZ?$AA?9?$AAC?$AAy?$AAr?$AAl@ 0000000180006228     libcpmt:winapinls.obj
 0001:00005240       ??_C@_1O@LAOBCMDF@?$AAq?$AAu?$AAz?$AA?9?$AAE?$AAC@ 0000000180006240     libcpmt:winapinls.obj
 0001:00005250       ??_C@_1M@POEEMAIO@?$AAa?$AAr?$AA?9?$AAE?$AAG@ 0000000180006250     libcpmt:winapinls.obj
 0001:00005260       ??_C@_1M@EFAKDEDL@?$AAz?$AAh?$AA?9?$AAH?$AAK@ 0000000180006260     libcpmt:winapinls.obj
 0001:00005270       ??_C@_1M@HKKIJHGI@?$AAd?$AAe?$AA?9?$AAA?$AAT@ 0000000180006270     libcpmt:winapinls.obj
 0001:00005280       ??_C@_1M@KBFBEHJF@?$AAe?$AAn?$AA?9?$AAA?$AAU@ 0000000180006280     libcpmt:winapinls.obj
 0001:00005290       ??_C@_1M@MNPLFAAH@?$AAe?$AAs?$AA?9?$AAE?$AAS@ 0000000180006290     libcpmt:winapinls.obj
 0001:000052a0       ??_C@_1M@HJOOJFMA@?$AAf?$AAr?$AA?9?$AAC?$AAA@ 00000001800062a0     libcpmt:winapinls.obj
 0001:000052b0       ??_C@_1BG@JPOFPNAB@?$AAs?$AAr?$AA?9?$AAS?$AAP?$AA?9?$AAC?$AAy?$AAr?$AAl@ 00000001800062b0     libcpmt:winapinls.obj
 0001:000052c8       ??_C@_1M@LNFOCMOB@?$AAs?$AAe?$AA?9?$AAF?$AAI@ 00000001800062c8     libcpmt:winapinls.obj
 0001:000052d8       ??_C@_1O@MGJBOAMB@?$AAq?$AAu?$AAz?$AA?9?$AAP?$AAE@ 00000001800062d8     libcpmt:winapinls.obj
 0001:000052e8       ??_C@_1M@GJINLBOK@?$AAa?$AAr?$AA?9?$AAL?$AAY@ 00000001800062e8     libcpmt:winapinls.obj
 0001:000052f8       ??_C@_1M@GGMNHJNL@?$AAz?$AAh?$AA?9?$AAS?$AAG@ 00000001800062f8     libcpmt:winapinls.obj
 0001:00005308       ??_C@_1M@HOIKODND@?$AAd?$AAe?$AA?9?$AAL?$AAU@ 0000000180006308     libcpmt:winapinls.obj
 0001:00005318       ??_C@_1M@DDOCCGFG@?$AAe?$AAn?$AA?9?$AAC?$AAA@ 0000000180006318     libcpmt:winapinls.obj
 0001:00005328       ??_C@_1M@BNOEMJLF@?$AAe?$AAs?$AA?9?$AAG?$AAT@ 0000000180006328     libcpmt:winapinls.obj
 0001:00005338       ??_C@_1M@EOGNKEK@?$AAf?$AAr?$AA?9?$AAC?$AAH@ 0000000180006338     libcpmt:winapinls.obj
 0001:00005348       ??_C@_1M@FLIDJFHL@?$AAh?$AAr?$AA?9?$AAB?$AAA@ 0000000180006348     libcpmt:winapinls.obj
 0001:00005358       ??_C@_1O@FMCELNAJ@?$AAs?$AAm?$AAj?$AA?9?$AAN?$AAO@ 0000000180006358     libcpmt:winapinls.obj
 0001:00005368       ??_C@_1M@JHGLJMGJ@?$AAa?$AAr?$AA?9?$AAD?$AAZ@ 0000000180006368     libcpmt:winapinls.obj
 0001:00005378       ??_C@_1M@JKKFDCNP@?$AAz?$AAh?$AA?9?$AAM?$AAO@ 0000000180006378     libcpmt:winapinls.obj
 0001:00005388       ??_C@_1M@GEEFALPE@?$AAd?$AAe?$AA?9?$AAL?$AAI@ 0000000180006388     libcpmt:winapinls.obj
 0001:00005398       ??_C@_1M@IGEOFBG@?$AAe?$AAn?$AA?9?$AAN?$AAZ@ 0000000180006398     libcpmt:winapinls.obj
 0001:000053a8       ??_C@_1M@KDBONEHP@?$AAe?$AAs?$AA?9?$AAC?$AAR@ 00000001800063a8     libcpmt:winapinls.obj
 0001:000053b8       ??_C@_1M@FHMDOHNN@?$AAf?$AAr?$AA?9?$AAL?$AAU@ 00000001800063b8     libcpmt:winapinls.obj
 0001:000053c8       ??_C@_1BG@NFKKMAFG@?$AAb?$AAs?$AA?9?$AAB?$AAA?$AA?9?$AAL?$AAa?$AAt?$AAn@ 00000001800063c8     libcpmt:winapinls.obj
 0001:000053e0       ??_C@_1O@IMNBEMCI@?$AAs?$AAm?$AAj?$AA?9?$AAS?$AAE@ 00000001800063e0     libcpmt:winapinls.obj
 0001:000053f0       ??_C@_1M@DHHMBNDP@?$AAa?$AAr?$AA?9?$AAM?$AAA@ 00000001800063f0     libcpmt:winapinls.obj
 0001:00005400       ??_C@_1M@BNBLJCGH@?$AAe?$AAn?$AA?9?$AAI?$AAE@ 0000000180006400     libcpmt:winapinls.obj
 0001:00005410       ??_C@_1M@GEPAFMDL@?$AAe?$AAs?$AA?9?$AAP?$AAA@ 0000000180006410     libcpmt:winapinls.obj
 0001:00005420       ??_C@_1M@OJONDMDL@?$AAf?$AAr?$AA?9?$AAM?$AAC@ 0000000180006420     libcpmt:winapinls.obj
 0001:00005430       ??_C@_1BG@OBCNFJB@?$AAs?$AAr?$AA?9?$AAB?$AAA?$AA?9?$AAL?$AAa?$AAt?$AAn@ 0000000180006430     libcpmt:winapinls.obj
 0001:00005448       ??_C@_1O@KEMEEGPO@?$AAs?$AAm?$AAa?$AA?9?$AAN?$AAO@ 0000000180006448     libcpmt:winapinls.obj
 0001:00005458       ??_C@_1M@ELMGFODK@?$AAa?$AAr?$AA?9?$AAT?$AAN@ 0000000180006458     libcpmt:winapinls.obj
 0001:00005468       ??_C@_1M@BHDLHFAF@?$AAe?$AAn?$AA?9?$AAZ?$AAA@ 0000000180006468     libcpmt:winapinls.obj
 0001:00005478       ??_C@_1M@BMGIGLIF@?$AAe?$AAs?$AA?9?$AAD?$AAO@ 0000000180006478     libcpmt:winapinls.obj
 0001:00005488       ??_C@_1BG@CMBHIPBE@?$AAs?$AAr?$AA?9?$AAB?$AAA?$AA?9?$AAC?$AAy?$AAr?$AAl@ 0000000180006488     libcpmt:winapinls.obj
 0001:000054a0       ??_C@_1O@HEDBLHNP@?$AAs?$AAm?$AAa?$AA?9?$AAS?$AAE@ 00000001800064a0     libcpmt:winapinls.obj
 0001:000054b0       ??_C@_1M@DAGCADIM@?$AAa?$AAr?$AA?9?$AAO?$AAM@ 00000001800064b0     libcpmt:winapinls.obj
 0001:000054c0       ??_C@_1M@FODLMICG@?$AAe?$AAn?$AA?9?$AAJ?$AAM@ 00000001800064c0     libcpmt:winapinls.obj
 0001:000054d0       ??_C@_1M@DNMLCIHB@?$AAe?$AAs?$AA?9?$AAV?$AAE@ 00000001800064d0     libcpmt:winapinls.obj
 0001:000054e0       ??_C@_1O@EOKHMKJK@?$AAs?$AAm?$AAs?$AA?9?$AAF?$AAI@ 00000001800064e0     libcpmt:winapinls.obj
 0001:000054f0       ??_C@_1M@CAFJMKOF@?$AAa?$AAr?$AA?9?$AAY?$AAE@ 00000001800064f0     libcpmt:winapinls.obj
 0001:00005500       ??_C@_1M@CBFHIJLI@?$AAe?$AAn?$AA?9?$AAC?$AAB@ 0000000180006500     libcpmt:winapinls.obj
 0001:00005510       ??_C@_1M@BGNFLDN@?$AAe?$AAs?$AA?9?$AAC?$AAO@ 0000000180006510     libcpmt:winapinls.obj
 0001:00005520       ??_C@_1O@JMPHMAMC@?$AAs?$AAm?$AAn?$AA?9?$AAF?$AAI@ 0000000180006520     libcpmt:winapinls.obj
 0001:00005530       ??_C@_1M@JLANABKE@?$AAa?$AAr?$AA?9?$AAS?$AAY@ 0000000180006530     libcpmt:winapinls.obj
 0001:00005540       ??_C@_1M@HPKGCFGN@?$AAe?$AAn?$AA?9?$AAB?$AAZ@ 0000000180006540     libcpmt:winapinls.obj
 0001:00005550       ??_C@_1M@OLJCMLGM@?$AAe?$AAs?$AA?9?$AAP?$AAE@ 0000000180006550     libcpmt:winapinls.obj
 0001:00005560       ??_C@_1M@MKKGFKLE@?$AAa?$AAr?$AA?9?$AAJ?$AAO@ 0000000180006560     libcpmt:winapinls.obj
 0001:00005570       ??_C@_1M@EKPGLDNI@?$AAe?$AAn?$AA?9?$AAT?$AAT@ 0000000180006570     libcpmt:winapinls.obj
 0001:00005580       ??_C@_1M@OONGHFHE@?$AAe?$AAs?$AA?9?$AAA?$AAR@ 0000000180006580     libcpmt:winapinls.obj
 0001:00005590       ??_C@_1M@OOJFGBHE@?$AAa?$AAr?$AA?9?$AAL?$AAB@ 0000000180006590     libcpmt:winapinls.obj
 0001:000055a0       ??_C@_1M@GCEJHNEG@?$AAe?$AAn?$AA?9?$AAZ?$AAW@ 00000001800065a0     libcpmt:winapinls.obj
 0001:000055b0       ??_C@_1M@JNOCAHJI@?$AAe?$AAs?$AA?9?$AAE?$AAC@ 00000001800065b0     libcpmt:winapinls.obj
 0001:000055c0       ??_C@_1M@JEFHPGGB@?$AAa?$AAr?$AA?9?$AAK?$AAW@ 00000001800065c0     libcpmt:winapinls.obj
 0001:000055d0       ??_C@_1M@MLKIBJOJ@?$AAe?$AAn?$AA?9?$AAP?$AAH@ 00000001800065d0     libcpmt:winapinls.obj
 0001:000055e0       ??_C@_1M@BDNIPEND@?$AAe?$AAs?$AA?9?$AAC?$AAL@ 00000001800065e0     libcpmt:winapinls.obj
 0001:000055f0       ??_C@_1M@MPNMEKBD@?$AAa?$AAr?$AA?9?$AAA?$AAE@ 00000001800065f0     libcpmt:winapinls.obj
 0001:00005600       ??_C@_1M@KBJALCPI@?$AAe?$AAs?$AA?9?$AAU?$AAY@ 0000000180006600     libcpmt:winapinls.obj
 0001:00005610       ??_C@_1M@LLCCOAGA@?$AAa?$AAr?$AA?9?$AAB?$AAH@ 0000000180006610     libcpmt:winapinls.obj
 0001:00005620       ??_C@_1M@PBFNCDEL@?$AAe?$AAs?$AA?9?$AAP?$AAY@ 0000000180006620     libcpmt:winapinls.obj
 0001:00005630       ??_C@_1M@EDGINPNP@?$AAa?$AAr?$AA?9?$AAQ?$AAA@ 0000000180006630     libcpmt:winapinls.obj
 0001:00005640       ??_C@_1M@MKDBIIJI@?$AAe?$AAs?$AA?9?$AAB?$AAO@ 0000000180006640     libcpmt:winapinls.obj
 0001:00005650       ??_C@_1M@CPKKEBLD@?$AAe?$AAs?$AA?9?$AAS?$AAV@ 0000000180006650     libcpmt:winapinls.obj
 0001:00005660       ??_C@_1M@NDBGMMJL@?$AAe?$AAs?$AA?9?$AAH?$AAN@ 0000000180006660     libcpmt:winapinls.obj
 0001:00005670       ??_C@_1M@JIJIBHDP@?$AAe?$AAs?$AA?9?$AAN?$AAI@ 0000000180006670     libcpmt:winapinls.obj
 0001:00005680       ??_C@_1M@CGFMKEEK@?$AAe?$AAs?$AA?9?$AAP?$AAR@ 0000000180006680     libcpmt:winapinls.obj
 0001:00005690       ??_C@_1O@ICJHKIIK@?$AAz?$AAh?$AA?9?$AAC?$AAH?$AAT@ 0000000180006690     libcpmt:winapinls.obj
 0001:000056a0       ??_C@_15CLNEJCE@?$AAs?$AAr@ 00000001800066a0     libcpmt:winapinls.obj
 0001:000056a8       ??_C@_1M@KAHEKEIG@?$AAa?$AAf?$AA?9?$AAz?$AAa@ 00000001800066a8     libcpmt:winapinls.obj
 0001:000056b8       ??_C@_1M@GIECOABL@?$AAa?$AAr?$AA?9?$AAa?$AAe@ 00000001800066b8     libcpmt:winapinls.obj
 0001:000056c8       ??_C@_1M@BMLMEKGI@?$AAa?$AAr?$AA?9?$AAb?$AAh@ 00000001800066c8     libcpmt:winapinls.obj
 0001:000056d8       ??_C@_1M@DAPFDGGB@?$AAa?$AAr?$AA?9?$AAd?$AAz@ 00000001800066d8     libcpmt:winapinls.obj
 0001:000056e8       ??_C@_1M@FJNKGKIG@?$AAa?$AAr?$AA?9?$AAe?$AAg@ 00000001800066e8     libcpmt:winapinls.obj
 0001:000056f8       ??_C@_1M@FLGKKCLO@?$AAa?$AAr?$AA?9?$AAi?$AAq@ 00000001800066f8     libcpmt:winapinls.obj
 0001:00005708       ??_C@_1M@GNDIPALM@?$AAa?$AAr?$AA?9?$AAj?$AAo@ 0000000180006708     libcpmt:winapinls.obj
 0001:00005718       ??_C@_1M@DDMJFMGJ@?$AAa?$AAr?$AA?9?$AAk?$AAw@ 0000000180006718     libcpmt:winapinls.obj
 0001:00005728       ??_C@_1M@EJALMLHM@?$AAa?$AAr?$AA?9?$AAl?$AAb@ 0000000180006728     libcpmt:winapinls.obj
 0001:00005738       ??_C@_1M@MOBDBLOC@?$AAa?$AAr?$AA?9?$AAl?$AAy@ 0000000180006738     libcpmt:winapinls.obj
 0001:00005748       ??_C@_1M@JAOCLHDH@?$AAa?$AAr?$AA?9?$AAm?$AAa@ 0000000180006748     libcpmt:winapinls.obj
 0001:00005758       ??_C@_1M@JHPMKJIE@?$AAa?$AAr?$AA?9?$AAo?$AAm@ 0000000180006758     libcpmt:winapinls.obj
 0001:00005768       ??_C@_1M@OEPGHFNH@?$AAa?$AAr?$AA?9?$AAq?$AAa@ 0000000180006768     libcpmt:winapinls.obj
 0001:00005778       ??_C@_1M@KJDONENM@?$AAa?$AAr?$AA?9?$AAs?$AAa@ 0000000180006778     libcpmt:winapinls.obj
 0001:00005788       ??_C@_1M@DMJDKLKM@?$AAa?$AAr?$AA?9?$AAs?$AAy@ 0000000180006788     libcpmt:winapinls.obj
 0001:00005798       ??_C@_1M@OMFIPEDC@?$AAa?$AAr?$AA?9?$AAt?$AAn@ 0000000180006798     libcpmt:winapinls.obj
 0001:000057a8       ??_C@_1M@IHMHGAON@?$AAa?$AAr?$AA?9?$AAy?$AAe@ 00000001800067a8     libcpmt:winapinls.obj
 0001:000057b8       ??_C@_1BG@KDCPGJGB@?$AAa?$AAz?$AA?9?$AAa?$AAz?$AA?9?$AAc?$AAy?$AAr?$AAl@ 00000001800067b8     libcpmt:winapinls.obj
 0001:000057d0       ??_C@_1BG@IBCKDDOE@?$AAa?$AAz?$AA?9?$AAa?$AAz?$AA?9?$AAl?$AAa?$AAt?$AAn@ 00000001800067d0     libcpmt:winapinls.obj
 0001:000057e8       ??_C@_1M@EGPFDCPD@?$AAb?$AAe?$AA?9?$AAb?$AAy@ 00000001800067e8     libcpmt:winapinls.obj
 0001:000057f8       ??_C@_1M@PCMGMCGC@?$AAb?$AAg?$AA?9?$AAb?$AAg@ 00000001800067f8     libcpmt:winapinls.obj
 0001:00005808       ??_C@_1M@BJBMFGOB@?$AAb?$AAn?$AA?9?$AAi?$AAn@ 0000000180006808     libcpmt:winapinls.obj
 0001:00005818       ??_C@_1BG@EAKMMACD@?$AAb?$AAs?$AA?9?$AAb?$AAa?$AA?9?$AAl?$AAa?$AAt?$AAn@ 0000000180006818     libcpmt:winapinls.obj
 0001:00005830       ??_C@_1M@KGADAODK@?$AAc?$AAa?$AA?9?$AAe?$AAs@ 0000000180006830     libcpmt:winapinls.obj
 0001:00005840       ??_C@_1M@COAJPDHI@?$AAc?$AAs?$AA?9?$AAc?$AAz@ 0000000180006840     libcpmt:winapinls.obj
 0001:00005850       ??_C@_1M@DHBHFONH@?$AAc?$AAy?$AA?9?$AAg?$AAb@ 0000000180006850     libcpmt:winapinls.obj
 0001:00005860       ??_C@_1M@IMGKELGA@?$AAd?$AAa?$AA?9?$AAd?$AAk@ 0000000180006860     libcpmt:winapinls.obj
 0001:00005870       ??_C@_1M@NNDGDNGA@?$AAd?$AAe?$AA?9?$AAa?$AAt@ 0000000180006870     libcpmt:winapinls.obj
 0001:00005880       ??_C@_1M@IKDBHEEM@?$AAd?$AAe?$AA?9?$AAc?$AAh@ 0000000180006880     libcpmt:winapinls.obj
 0001:00005890       ??_C@_1M@GFFOJMCJ@?$AAd?$AAe?$AA?9?$AAd?$AAe@ 0000000180006890     libcpmt:winapinls.obj
 0001:000058a0       ??_C@_1M@MDNLKBPM@?$AAd?$AAe?$AA?9?$AAl?$AAi@ 00000001800068a0     libcpmt:winapinls.obj
 0001:000058b0       ??_C@_1M@NJBEEJNL@?$AAd?$AAe?$AA?9?$AAl?$AAu@ 00000001800068b0     libcpmt:winapinls.obj
 0001:000058c0       ??_C@_1O@GNNELBAP@?$AAd?$AAi?$AAv?$AA?9?$AAm?$AAv@ 00000001800068c0     libcpmt:winapinls.obj
 0001:000058d0       ??_C@_1M@EJLEOGAE@?$AAe?$AAl?$AA?9?$AAg?$AAr@ 00000001800068d0     libcpmt:winapinls.obj
 0001:000058e0       ??_C@_1M@GMPONJN@?$AAe?$AAn?$AA?9?$AAa?$AAu@ 00000001800068e0     libcpmt:winapinls.obj
 0001:000058f0       ??_C@_1M@NIDIIPGF@?$AAe?$AAn?$AA?9?$AAb?$AAz@ 00000001800068f0     libcpmt:winapinls.obj
 0001:00005900       ??_C@_1M@JEHMIMFO@?$AAe?$AAn?$AA?9?$AAc?$AAa@ 0000000180006900     libcpmt:winapinls.obj
 0001:00005910       ??_C@_1M@IGMJCDLA@?$AAe?$AAn?$AA?9?$AAc?$AAb@ 0000000180006910     libcpmt:winapinls.obj
 0001:00005920       ??_C@_1M@BNFIGBKG@?$AAe?$AAn?$AA?9?$AAg?$AAb@ 0000000180006920     libcpmt:winapinls.obj
 0001:00005930       ??_C@_1M@LKIFDIGP@?$AAe?$AAn?$AA?9?$AAi?$AAe@ 0000000180006930     libcpmt:winapinls.obj
 0001:00005940       ??_C@_1M@PJKFGCCO@?$AAe?$AAn?$AA?9?$AAj?$AAm@ 0000000180006940     libcpmt:winapinls.obj
 0001:00005950       ??_C@_1M@KPPKEPBO@?$AAe?$AAn?$AA?9?$AAn?$AAz@ 0000000180006950     libcpmt:winapinls.obj
 0001:00005960       ??_C@_1M@GMDGLDOB@?$AAe?$AAn?$AA?9?$AAp?$AAh@ 0000000180006960     libcpmt:winapinls.obj
 0001:00005970       ??_C@_1M@ONGIBJNA@?$AAe?$AAn?$AA?9?$AAt?$AAt@ 0000000180006970     libcpmt:winapinls.obj
 0001:00005980       ??_C@_1M@LLODPCMM@?$AAe?$AAn?$AA?9?$AAu?$AAs@ 0000000180006980     libcpmt:winapinls.obj
 0001:00005990       ??_C@_1M@LAKFNPAN@?$AAe?$AAn?$AA?9?$AAz?$AAa@ 0000000180006990     libcpmt:winapinls.obj
 0001:000059a0       ??_C@_1M@MFNHNHEO@?$AAe?$AAn?$AA?9?$AAz?$AAw@ 00000001800069a0     libcpmt:winapinls.obj
 0001:000059b0       ??_C@_1M@EJEINPHM@?$AAe?$AAs?$AA?9?$AAa?$AAr@ 00000001800069b0     libcpmt:winapinls.obj
 0001:000059c0       ??_C@_1M@GNKPCCJA@?$AAe?$AAs?$AA?9?$AAb?$AAo@ 00000001800069c0     libcpmt:winapinls.obj
 0001:000059d0       ??_C@_1M@LEEGFONL@?$AAe?$AAs?$AA?9?$AAc?$AAl@ 00000001800069d0     libcpmt:winapinls.obj
 0001:000059e0       ??_C@_1M@KGPDPBDF@?$AAe?$AAs?$AA?9?$AAc?$AAo@ 00000001800069e0     libcpmt:winapinls.obj
 0001:000059f0       ??_C@_1M@EIAHOHH@?$AAe?$AAs?$AA?9?$AAc?$AAr@ 00000001800069f0     libcpmt:winapinls.obj
 0001:00005a00       ??_C@_1M@LLPGMBIN@?$AAe?$AAs?$AA?9?$AAd?$AAo@ 0000000180006a00     libcpmt:winapinls.obj
 0001:00005a10       ??_C@_1M@DKHMKNJA@?$AAe?$AAs?$AA?9?$AAe?$AAc@ 0000000180006a10     libcpmt:winapinls.obj
 0001:00005a20       ??_C@_1M@GKGFPKAP@?$AAe?$AAs?$AA?9?$AAe?$AAs@ 0000000180006a20     libcpmt:winapinls.obj
 0001:00005a30       ??_C@_1M@LKHKGDLN@?$AAe?$AAs?$AA?9?$AAg?$AAt@ 0000000180006a30     libcpmt:winapinls.obj
 0001:00005a40       ??_C@_1M@HEIIGGJD@?$AAe?$AAs?$AA?9?$AAh?$AAn@ 0000000180006a40     libcpmt:winapinls.obj
 0001:00005a50       ??_C@_1M@FBDHPPGD@?$AAe?$AAs?$AA?9?$AAm?$AAx@ 0000000180006a50     libcpmt:winapinls.obj
 0001:00005a60       ??_C@_1M@DPAGLNDH@?$AAe?$AAs?$AA?9?$AAn?$AAi@ 0000000180006a60     libcpmt:winapinls.obj
 0001:00005a70       ??_C@_1M@MDGOPGDD@?$AAe?$AAs?$AA?9?$AAp?$AAa@ 0000000180006a70     libcpmt:winapinls.obj
 0001:00005a80       ??_C@_1M@EMAMGBGE@?$AAe?$AAs?$AA?9?$AAp?$AAe@ 0000000180006a80     libcpmt:winapinls.obj
 0001:00005a90       ??_C@_1M@IBMCAOEC@?$AAe?$AAs?$AA?9?$AAp?$AAr@ 0000000180006a90     libcpmt:winapinls.obj
 0001:00005aa0       ??_C@_1M@FGMDIJED@?$AAe?$AAs?$AA?9?$AAp?$AAy@ 0000000180006aa0     libcpmt:winapinls.obj
 0001:00005ab0       ??_C@_1M@IIDEOLLL@?$AAe?$AAs?$AA?9?$AAs?$AAv@ 0000000180006ab0     libcpmt:winapinls.obj
 0001:00005ac0       ??_C@_1M@GAOBIPA@?$AAe?$AAs?$AA?9?$AAu?$AAy@ 0000000180006ac0     libcpmt:winapinls.obj
 0001:00005ad0       ??_C@_1M@JKFFICHJ@?$AAe?$AAs?$AA?9?$AAv?$AAe@ 0000000180006ad0     libcpmt:winapinls.obj
 0001:00005ae0       ??_C@_1M@PNMLOJDF@?$AAe?$AAt?$AA?9?$AAe?$AAe@ 0000000180006ae0     libcpmt:winapinls.obj
 0001:00005af0       ??_C@_1M@GHHLIKEI@?$AAe?$AAu?$AA?9?$AAe?$AAs@ 0000000180006af0     libcpmt:winapinls.obj
 0001:00005b00       ??_C@_1M@PBNONODE@?$AAf?$AAa?$AA?9?$AAi?$AAr@ 0000000180006b00     libcpmt:winapinls.obj
 0001:00005b10       ??_C@_1M@JEEHPMIL@?$AAf?$AAi?$AA?9?$AAf?$AAi@ 0000000180006b10     libcpmt:winapinls.obj
 0001:00005b20       ??_C@_1M@LMDCNDBA@?$AAf?$AAo?$AA?9?$AAf?$AAo@ 0000000180006b20     libcpmt:winapinls.obj
 0001:00005b30       ??_C@_1M@JKEOHLDK@?$AAf?$AAr?$AA?9?$AAb?$AAe@ 0000000180006b30     libcpmt:winapinls.obj
 0001:00005b40       ??_C@_1M@NOHADPMI@?$AAf?$AAr?$AA?9?$AAc?$AAa@ 0000000180006b40     libcpmt:winapinls.obj
 0001:00005b50       ??_C@_1M@KDHIHAEC@?$AAf?$AAr?$AA?9?$AAc?$AAh@ 0000000180006b50     libcpmt:winapinls.obj
 0001:00005b60       ??_C@_1M@MMBBFGAK@?$AAf?$AAr?$AA?9?$AAf?$AAr@ 0000000180006b60     libcpmt:winapinls.obj
 0001:00005b70       ??_C@_1M@PAFNENNF@?$AAf?$AAr?$AA?9?$AAl?$AAu@ 0000000180006b70     libcpmt:winapinls.obj
 0001:00005b80       ??_C@_1M@EOHDJGDD@?$AAf?$AAr?$AA?9?$AAm?$AAc@ 0000000180006b80     libcpmt:winapinls.obj
 0001:00005b90       ??_C@_1M@FAPLLOPF@?$AAg?$AAl?$AA?9?$AAe?$AAs@ 0000000180006b90     libcpmt:winapinls.obj
 0001:00005ba0       ??_C@_1M@FOPBFLOO@?$AAg?$AAu?$AA?9?$AAi?$AAn@ 0000000180006ba0     libcpmt:winapinls.obj
 0001:00005bb0       ??_C@_1M@KBMCINPM@?$AAh?$AAe?$AA?9?$AAi?$AAl@ 0000000180006bb0     libcpmt:winapinls.obj
 0001:00005bc0       ??_C@_1M@BBPHKFPJ@?$AAh?$AAi?$AA?9?$AAi?$AAn@ 0000000180006bc0     libcpmt:winapinls.obj
 0001:00005bd0       ??_C@_1M@PMBNDPHD@?$AAh?$AAr?$AA?9?$AAb?$AAa@ 0000000180006bd0     libcpmt:winapinls.obj
 0001:00005be0       ??_C@_1M@BPCKOEGE@?$AAh?$AAr?$AA?9?$AAh?$AAr@ 0000000180006be0     libcpmt:winapinls.obj
 0001:00005bf0       ??_C@_1M@GACBMHKE@?$AAh?$AAu?$AA?9?$AAh?$AAu@ 0000000180006bf0     libcpmt:winapinls.obj
 0001:00005c00       ??_C@_1M@MILPAJJC@?$AAh?$AAy?$AA?9?$AAa?$AAm@ 0000000180006c00     libcpmt:winapinls.obj
 0001:00005c10       ??_C@_1M@BABBICEC@?$AAi?$AAd?$AA?9?$AAi?$AAd@ 0000000180006c10     libcpmt:winapinls.obj
 0001:00005c20       ??_C@_1M@BIKNHHPF@?$AAi?$AAs?$AA?9?$AAi?$AAs@ 0000000180006c20     libcpmt:winapinls.obj
 0001:00005c30       ??_C@_1M@NMPCJPHE@?$AAi?$AAt?$AA?9?$AAc?$AAh@ 0000000180006c30     libcpmt:winapinls.obj
 0001:00005c40       ??_C@_1M@GHKGFEDF@?$AAi?$AAt?$AA?9?$AAi?$AAt@ 0000000180006c40     libcpmt:winapinls.obj
 0001:00005c50       ??_C@_1M@NIEJCJJA@?$AAj?$AAa?$AA?9?$AAj?$AAp@ 0000000180006c50     libcpmt:winapinls.obj
 0001:00005c60       ??_C@_1M@JILFNBIM@?$AAk?$AAa?$AA?9?$AAg?$AAe@ 0000000180006c60     libcpmt:winapinls.obj
 0001:00005c70       ??_C@_1M@PACPMGPH@?$AAk?$AAk?$AA?9?$AAk?$AAz@ 0000000180006c70     libcpmt:winapinls.obj
 0001:00005c80       ??_C@_1M@IELFGMHA@?$AAk?$AAn?$AA?9?$AAi?$AAn@ 0000000180006c80     libcpmt:winapinls.obj
 0001:00005c90       ??_C@_1M@DMHAEOGC@?$AAk?$AAo?$AA?9?$AAk?$AAr@ 0000000180006c90     libcpmt:winapinls.obj
 0001:00005ca0       ??_C@_1O@IBBJHCH@?$AAk?$AAo?$AAk?$AA?9?$AAi?$AAn@ 0000000180006ca0     libcpmt:winapinls.obj
 0001:00005cb0       ??_C@_1M@HBAHBIGA@?$AAk?$AAy?$AA?9?$AAk?$AAg@ 0000000180006cb0     libcpmt:winapinls.obj
 0001:00005cc0       ??_C@_1M@KPMILCJG@?$AAl?$AAt?$AA?9?$AAl?$AAt@ 0000000180006cc0     libcpmt:winapinls.obj
 0001:00005cd0       ??_C@_1M@BDEKKCA@?$AAl?$AAv?$AA?9?$AAl?$AAv@ 0000000180006cd0     libcpmt:winapinls.obj
 0001:00005ce0       ??_C@_1M@ELCKCCJJ@?$AAm?$AAi?$AA?9?$AAn?$AAz@ 0000000180006ce0     libcpmt:winapinls.obj
 0001:00005cf0       ??_C@_1M@CBOOLAPA@?$AAm?$AAk?$AA?9?$AAm?$AAk@ 0000000180006cf0     libcpmt:winapinls.obj
 0001:00005d00       ??_C@_1M@GPHNBJKN@?$AAm?$AAl?$AA?9?$AAi?$AAn@ 0000000180006d00     libcpmt:winapinls.obj
 0001:00005d10       ??_C@_1M@PABJILIG@?$AAm?$AAn?$AA?9?$AAm?$AAn@ 0000000180006d10     libcpmt:winapinls.obj
 0001:00005d20       ??_C@_1M@FGBKKIPG@?$AAm?$AAr?$AA?9?$AAi?$AAn@ 0000000180006d20     libcpmt:winapinls.obj
 0001:00005d30       ??_C@_1M@NDBPDDAL@?$AAm?$AAs?$AA?9?$AAb?$AAn@ 0000000180006d30     libcpmt:winapinls.obj
 0001:00005d40       ??_C@_1M@OPIHOOPI@?$AAm?$AAs?$AA?9?$AAm?$AAy@ 0000000180006d40     libcpmt:winapinls.obj
 0001:00005d50       ??_C@_1M@PPDBCNFM@?$AAm?$AAt?$AA?9?$AAm?$AAt@ 0000000180006d50     libcpmt:winapinls.obj
 0001:00005d60       ??_C@_1M@KDJDKMDD@?$AAn?$AAb?$AA?9?$AAn?$AAo@ 0000000180006d60     libcpmt:winapinls.obj
 0001:00005d70       ??_C@_1M@KFCFLMJP@?$AAn?$AAl?$AA?9?$AAb?$AAe@ 0000000180006d70     libcpmt:winapinls.obj
 0001:00005d80       ??_C@_1M@KPOPDDGO@?$AAn?$AAl?$AA?9?$AAn?$AAl@ 0000000180006d80     libcpmt:winapinls.obj
 0001:00005d90       ??_C@_1M@LJKPEMLN@?$AAn?$AAn?$AA?9?$AAn?$AAo@ 0000000180006d90     libcpmt:winapinls.obj
 0001:00005da0       ??_C@_1M@BDGHHBFL@?$AAn?$AAs?$AA?9?$AAz?$AAa@ 0000000180006da0     libcpmt:winapinls.obj
 0001:00005db0       ??_C@_1M@IDEHOAP@?$AAp?$AAa?$AA?9?$AAi?$AAn@ 0000000180006db0     libcpmt:winapinls.obj
 0001:00005dc0       ??_C@_1M@HDBKGOGH@?$AAp?$AAl?$AA?9?$AAp?$AAl@ 0000000180006dc0     libcpmt:winapinls.obj
 0001:00005dd0       ??_C@_1M@LJLLCMEH@?$AAp?$AAt?$AA?9?$AAb?$AAr@ 0000000180006dd0     libcpmt:winapinls.obj
 0001:00005de0       ??_C@_1M@NCMONAAL@?$AAp?$AAt?$AA?9?$AAp?$AAt@ 0000000180006de0     libcpmt:winapinls.obj
 0001:00005df0       ??_C@_1O@EAKMAJDN@?$AAq?$AAu?$AAz?$AA?9?$AAb?$AAo@ 0000000180006df0     libcpmt:winapinls.obj
 0001:00005e00       ??_C@_1O@BHHPIGDN@?$AAq?$AAu?$AAz?$AA?9?$AAe?$AAc@ 0000000180006e00     libcpmt:winapinls.obj
 0001:00005e10       ??_C@_1O@GBAPEKMJ@?$AAq?$AAu?$AAz?$AA?9?$AAp?$AAe@ 0000000180006e10     libcpmt:winapinls.obj
 0001:00005e20       ??_C@_1M@CLGLEFBO@?$AAr?$AAo?$AA?9?$AAr?$AAo@ 0000000180006e20     libcpmt:winapinls.obj
 0001:00005e30       ??_C@_1M@CEEDODME@?$AAr?$AAu?$AA?9?$AAr?$AAu@ 0000000180006e30     libcpmt:winapinls.obj
 0001:00005e40       ??_C@_1M@HPKKKMPP@?$AAs?$AAa?$AA?9?$AAi?$AAn@ 0000000180006e40     libcpmt:winapinls.obj
 0001:00005e50       ??_C@_1M@BKMAIGOJ@?$AAs?$AAe?$AA?9?$AAf?$AAi@ 0000000180006e50     libcpmt:winapinls.obj
 0001:00005e60       ??_C@_1M@NDPIFLFI@?$AAs?$AAe?$AA?9?$AAn?$AAo@ 0000000180006e60     libcpmt:winapinls.obj
 0001:00005e70       ??_C@_1M@DANKKHJ@?$AAs?$AAe?$AA?9?$AAs?$AAe@ 0000000180006e70     libcpmt:winapinls.obj
 0001:00005e80       ??_C@_1M@PNBLONPJ@?$AAs?$AAk?$AA?9?$AAs?$AAk@ 0000000180006e80     libcpmt:winapinls.obj
 0001:00005e90       ??_C@_1M@LFMODOAL@?$AAs?$AAl?$AA?9?$AAs?$AAi@ 0000000180006e90     libcpmt:winapinls.obj
 0001:00005ea0       ??_C@_1O@DFKOMPG@?$AAs?$AAm?$AAa?$AA?9?$AAn?$AAo@ 0000000180006ea0     libcpmt:winapinls.obj
 0001:00005eb0       ??_C@_1O@NDKPBNNH@?$AAs?$AAm?$AAa?$AA?9?$AAs?$AAe@ 0000000180006eb0     libcpmt:winapinls.obj
 0001:00005ec0       ??_C@_1O@PLLKBHAB@?$AAs?$AAm?$AAj?$AA?9?$AAn?$AAo@ 0000000180006ec0     libcpmt:winapinls.obj
 0001:00005ed0       ??_C@_1O@CLEPOGCA@?$AAs?$AAm?$AAj?$AA?9?$AAs?$AAe@ 0000000180006ed0     libcpmt:winapinls.obj
 0001:00005ee0       ??_C@_1O@DLGJGKMK@?$AAs?$AAm?$AAn?$AA?9?$AAf?$AAi@ 0000000180006ee0     libcpmt:winapinls.obj
 0001:00005ef0       ??_C@_1O@OJDJGAJC@?$AAs?$AAm?$AAs?$AA?9?$AAf?$AAi@ 0000000180006ef0     libcpmt:winapinls.obj
 0001:00005f00       ??_C@_1M@BOFOGHPB@?$AAs?$AAq?$AA?9?$AAa?$AAl@ 0000000180006f00     libcpmt:winapinls.obj
 0001:00005f10       ??_C@_1BG@LJBBIPGB@?$AAs?$AAr?$AA?9?$AAb?$AAa?$AA?9?$AAc?$AAy?$AAr?$AAl@ 0000000180006f10     libcpmt:winapinls.obj
 0001:00005f28       ??_C@_1BG@JLBENFOE@?$AAs?$AAr?$AA?9?$AAb?$AAa?$AA?9?$AAl?$AAa?$AAt?$AAn@ 0000000180006f28     libcpmt:winapinls.obj
 0001:00005f40       ??_C@_1BG@KODPNHE@?$AAs?$AAr?$AA?9?$AAs?$AAp?$AA?9?$AAc?$AAy?$AAr?$AAl@ 0000000180006f40     libcpmt:winapinls.obj
 0001:00005f58       ??_C@_1BG@CIOGKHPB@?$AAs?$AAr?$AA?9?$AAs?$AAp?$AA?9?$AAl?$AAa?$AAt?$AAn@ 0000000180006f58     libcpmt:winapinls.obj
 0001:00005f70       ??_C@_1M@NGFJLMAC@?$AAs?$AAv?$AA?9?$AAf?$AAi@ 0000000180006f70     libcpmt:winapinls.obj
 0001:00005f80       ??_C@_1M@MPJEJAJC@?$AAs?$AAv?$AA?9?$AAs?$AAe@ 0000000180006f80     libcpmt:winapinls.obj
 0001:00005f90       ??_C@_1M@MPNDHLFK@?$AAs?$AAw?$AA?9?$AAk?$AAe@ 0000000180006f90     libcpmt:winapinls.obj
 0001:00005fa0       ??_C@_1O@KOHBJJI@?$AAs?$AAy?$AAr?$AA?9?$AAs?$AAy@ 0000000180006fa0     libcpmt:winapinls.obj
 0001:00005fb0       ??_C@_1M@LDCEFHA@?$AAt?$AAa?$AA?9?$AAi?$AAn@ 0000000180006fb0     libcpmt:winapinls.obj
 0001:00005fc0       ??_C@_1M@CNJOFAK@?$AAt?$AAe?$AA?9?$AAi?$AAn@ 0000000180006fc0     libcpmt:winapinls.obj
 0001:00005fd0       ??_C@_1M@GNAECACD@?$AAt?$AAh?$AA?9?$AAt?$AAh@ 0000000180006fd0     libcpmt:winapinls.obj
 0001:00005fe0       ??_C@_1M@CHBIHOJO@?$AAt?$AAn?$AA?9?$AAz?$AAa@ 0000000180006fe0     libcpmt:winapinls.obj
 0001:00005ff0       ??_C@_1M@GCCMIGPJ@?$AAt?$AAr?$AA?9?$AAt?$AAr@ 0000000180006ff0     libcpmt:winapinls.obj
 0001:00006000       ??_C@_1M@CELMCNBK@?$AAt?$AAt?$AA?9?$AAr?$AAu@ 0000000180007000     libcpmt:winapinls.obj
 0001:00006010       ??_C@_1M@KLMCELGA@?$AAu?$AAk?$AA?9?$AAu?$AAa@ 0000000180007010     libcpmt:winapinls.obj
 0001:00006020       ??_C@_1M@EPAJJAJF@?$AAu?$AAr?$AA?9?$AAp?$AAk@ 0000000180007020     libcpmt:winapinls.obj
 0001:00006030       ??_C@_1BG@GEGPMCDJ@?$AAu?$AAz?$AA?9?$AAu?$AAz?$AA?9?$AAc?$AAy?$AAr?$AAl@ 0000000180007030     libcpmt:winapinls.obj
 0001:00006048       ??_C@_1BG@EGGKJILM@?$AAu?$AAz?$AA?9?$AAu?$AAz?$AA?9?$AAl?$AAa?$AAt?$AAn@ 0000000180007048     libcpmt:winapinls.obj
 0001:00006060       ??_C@_1M@GFOCLFF@?$AAv?$AAi?$AA?9?$AAv?$AAn@ 0000000180007060     libcpmt:winapinls.obj
 0001:00006070       ??_C@_1M@CPAMEDFI@?$AAx?$AAh?$AA?9?$AAz?$AAa@ 0000000180007070     libcpmt:winapinls.obj
 0001:00006080       ??_C@_1O@EBKIFIGN@?$AAz?$AAh?$AA?9?$AAc?$AAh?$AAs@ 0000000180007080     libcpmt:winapinls.obj
 0001:00006090       ??_C@_1O@NMHPGANE@?$AAz?$AAh?$AA?9?$AAc?$AAh?$AAt@ 0000000180007090     libcpmt:winapinls.obj
 0001:000060a0       ??_C@_1M@LPINJOMC@?$AAz?$AAh?$AA?9?$AAc?$AAn@ 00000001800070a0     libcpmt:winapinls.obj
 0001:000060b0       ??_C@_1M@OCJEJODD@?$AAz?$AAh?$AA?9?$AAh?$AAk@ 00000001800070b0     libcpmt:winapinls.obj
 0001:000060c0       ??_C@_1M@DNDLJINH@?$AAz?$AAh?$AA?9?$AAm?$AAo@ 00000001800070c0     libcpmt:winapinls.obj
 0001:000060d0       ??_C@_1M@MBFDNDND@?$AAz?$AAh?$AA?9?$AAs?$AAg@ 00000001800070d0     libcpmt:winapinls.obj
 0001:000060e0       ??_C@_1M@IMEPLEPE@?$AAz?$AAh?$AA?9?$AAt?$AAw@ 00000001800070e0     libcpmt:winapinls.obj
 0001:000060f0       ??_C@_1M@BBGHNHJP@?$AAz?$AAu?$AA?9?$AAz?$AAa@ 00000001800070f0     libcpmt:winapinls.obj
 0001:00006108       ??_7type_info@@6B@         0000000180007108     LIBCMT:std_type_info_static.obj
 0001:00006110       _pRawDllMain               0000000180007110     LIBCMT:dll_dllmain.obj
 0001:00006110       _pDefaultRawDllMain        0000000180007110     LIBCMT:dll_dllmain.obj
 0001:00006128       _pDestructExceptionObject  0000000180007128     libvcruntime:ehhelpers.obj
 0001:00006130       ?s_negLengthTab@FH4@@3QBCB 0000000180007130     libvcruntime:risctrnsctrl.obj
 0001:00006140       ?s_shiftTab@FH4@@3QBEB     0000000180007140     libvcruntime:risctrnsctrl.obj
 0001:00006290       ??_7bad_exception@std@@6B@ 0000000180007290     libvcruntime:frame.obj
 0001:000062a0       ??_C@_0O@DPKOEFFH@bad?5exception@ 00000001800072a0     libvcruntime:frame.obj
 0001:000069b0       ??_C@_08EHJDFFNH@__based?$CI@ 00000001800079b0     libvcruntime:undname.obj
 0001:000069c0       ??_C@_07KOLFKCDI@__cdecl@  00000001800079c0     libvcruntime:undname.obj
 0001:000069c8       ??_C@_08GHMPAG@__pascal@   00000001800079c8     libvcruntime:undname.obj
 0001:000069d8       ??_C@_09IFJBGAPI@__stdcall@ 00000001800079d8     libvcruntime:undname.obj
 0001:000069e8       ??_C@_0L@NPHFGOKO@__thiscall@ 00000001800079e8     libvcruntime:undname.obj
 0001:000069f8       ??_C@_0L@JMKHOMEK@__fastcall@ 00000001800079f8     libvcruntime:undname.obj
 0001:00006a08       ??_C@_0N@BCKKPABJ@__vectorcall@ 0000000180007a08     libvcruntime:undname.obj
 0001:00006a18       ??_C@_09HIJEGCPM@__clrcall@ 0000000180007a18     libvcruntime:undname.obj
 0001:00006a24       ??_C@_06GHPCKEAG@__eabi@   0000000180007a24     libvcruntime:undname.obj
 0001:00006a30       ??_C@_09IOPIDJLG@__swift_1@ 0000000180007a30     libvcruntime:undname.obj
 0001:00006a40       ??_C@_09KFNFGKHF@__swift_2@ 0000000180007a40     libvcruntime:undname.obj
 0001:00006a50       ??_C@_07JOMMBBKO@__ptr64@  0000000180007a50     libvcruntime:undname.obj
 0001:00006a58       ??_C@_0L@PILCLIHE@__restrict@ 0000000180007a58     libvcruntime:undname.obj
 0001:00006a68       ??_C@_0M@GFIIJFMG@__unaligned@ 0000000180007a68     libvcruntime:undname.obj
 0001:00006a78       ??_C@_09DHDLOLLB@restrict?$CI@ 0000000180007a78     libvcruntime:undname.obj
 0001:00006a84       ??_C@_04NIHEBCM@?5new@     0000000180007a84     libvcruntime:undname.obj
 0001:00006a90       ??_C@_07FPCDHGMM@?5delete@ 0000000180007a90     libvcruntime:undname.obj
 0001:00006a98       ??_C@_01NEMOKFLO@?$DN@     0000000180007a98     libvcruntime:undname.obj
 0001:00006a9c       ??_C@_02GPIOPFAK@?$DO?$DO@ 0000000180007a9c     libvcruntime:undname.obj
 0001:00006aa0       ??_C@_02FODMEDOG@?$DM?$DM@ 0000000180007aa0     libvcruntime:undname.obj
 0001:00006aa4       ??_C@_01DCLJPIOD@?$CB@     0000000180007aa4     libvcruntime:undname.obj
 0001:00006aa8       ??_C@_02EGOFBIJA@?$DN?$DN@ 0000000180007aa8     libvcruntime:undname.obj
 0001:00006aac       ??_C@_02FDNJECIE@?$CB?$DN@ 0000000180007aac     libvcruntime:undname.obj
 0001:00006ab0       ??_C@_02GPECMEKF@?$FL?$FN@ 0000000180007ab0     libvcruntime:undname.obj
 0001:00006ab8       ??_C@_08LHJFAFGD@operator@ 0000000180007ab8     libvcruntime:undname.obj
 0001:00006ac4       ??_C@_02HBOOOICD@?9?$DO@   0000000180007ac4     libvcruntime:undname.obj
 0001:00006ac8       ??_C@_02ECNGHCIF@?$CL?$CL@ 0000000180007ac8     libvcruntime:undname.obj
 0001:00006acc       ??_C@_02BAABKJLB@?9?9@     0000000180007acc     libvcruntime:undname.obj
 0001:00006ad0       ??_C@_01MIFGBAGJ@?$CL@     0000000180007ad0     libvcruntime:undname.obj
 0001:00006ad4       ??_C@_01HNPIGOCE@?$CG@     0000000180007ad4     libvcruntime:undname.obj
 0001:00006ad8       ??_C@_03MNHNFDLC@?9?$DO?$CK@ 0000000180007ad8     libvcruntime:undname.obj
 0001:00006adc       ??_C@_01KMDKNFGN@?1@       0000000180007adc     libvcruntime:undname.obj
 0001:00006ae0       ??_C@_01FGNFDNOH@?$CF@     0000000180007ae0     libvcruntime:undname.obj
 0001:00006ae4       ??_C@_01MNNFJEPP@?$DM@     0000000180007ae4     libvcruntime:undname.obj
 0001:00006ae8       ??_C@_02EHCHHCKH@?$DM?$DN@ 0000000180007ae8     libvcruntime:undname.obj
 0001:00006aec       ??_C@_01PPODPGHN@?$DO@     0000000180007aec     libvcruntime:undname.obj
 0001:00006af0       ??_C@_02EEKDKGMJ@?$DO?$DN@ 0000000180007af0     libvcruntime:undname.obj
 0001:00006af4       ??_C@_01IHBHIGKO@?0@       0000000180007af4     libvcruntime:undname.obj
 0001:00006af8       ??_C@_02HCKGKOFO@?$CI?$CJ@ 0000000180007af8     libvcruntime:undname.obj
 0001:00006afc       ??_C@_01PJKLJHI@?$HO@      0000000180007afc     libvcruntime:undname.obj
 0001:00006b00       ??_C@_01JKBOJNNK@?$FO@     0000000180007b00     libvcruntime:undname.obj
 0001:00006b04       ??_C@_01DNKMNLPK@?$HM@     0000000180007b04     libvcruntime:undname.obj
 0001:00006b08       ??_C@_02PPKAJPJL@?$CG?$CG@ 0000000180007b08     libvcruntime:undname.obj
 0001:00006b0c       ??_C@_02NONPIBCD@?$HM?$HM@ 0000000180007b0c     libvcruntime:undname.obj
 0001:00006b10       ??_C@_02FPIMKNGF@?$CK?$DN@ 0000000180007b10     libvcruntime:undname.obj
 0001:00006b14       ??_C@_02FOEOMHFC@?$CL?$DN@ 0000000180007b14     libvcruntime:undname.obj
 0001:00006b18       ??_C@_02FKMDLLOA@?9?$DN@   0000000180007b18     libvcruntime:undname.obj
 0001:00006b1c       ??_C@_02FJEHGPIO@?1?$DN@   0000000180007b1c     libvcruntime:undname.obj
 0001:00006b20       ??_C@_02FENAOKFI@?$CF?$DN@ 0000000180007b20     libvcruntime:undname.obj
 0001:00006b24       ??_C@_03IKFCCPFF@?$DO?$DO?$DN@ 0000000180007b24     libvcruntime:undname.obj
 0001:00006b28       ??_C@_03CDNPDDLA@?$DM?$DM?$DN@ 0000000180007b28     libvcruntime:undname.obj
 0001:00006b2c       ??_C@_02FGJGFEAB@?$CG?$DN@ 0000000180007b2c     libvcruntime:undname.obj
 0001:00006b30       ??_C@_02DHLNPPGH@?$HM?$DN@ 0000000180007b30     libvcruntime:undname.obj
 0001:00006b34       ??_C@_02MHEGNOJ@?$FO?$DN@  0000000180007b34     libvcruntime:undname.obj
 0001:00006b38       ??_C@_09IFPLHPGF@?$GAvftable?8@ 0000000180007b38     libvcruntime:undname.obj
 0001:00006b48       ??_C@_09BLBHBJP@?$GAvbtable?8@ 0000000180007b48     libvcruntime:undname.obj
 0001:00006b58       ??_C@_07FEEIOKP@?$GAvcall?8@ 0000000180007b58     libvcruntime:undname.obj
 0001:00006b60       ??_C@_08LLFFHHDJ@?$GAtypeof?8@ 0000000180007b60     libvcruntime:undname.obj
 0001:00006b70       ??_C@_0BF@KDPPACIK@?$GAlocal?5static?5guard?8@ 0000000180007b70     libvcruntime:undname.obj
 0001:00006b88       ??_C@_08OBABFOLI@?$GAstring?8@ 0000000180007b88     libvcruntime:undname.obj
 0001:00006b98       ??_C@_0BD@JDLKDPAB@?$GAvbase?5destructor?8@ 0000000180007b98     libvcruntime:undname.obj
 0001:00006bb0       ??_C@_0BN@DEGPLNFK@?$GAvector?5deleting?5destructor?8@ 0000000180007bb0     libvcruntime:undname.obj
 0001:00006bd0       ??_C@_0BO@OBMKPJIG@?$GAdefault?5constructor?5closure?8@ 0000000180007bd0     libvcruntime:undname.obj
 0001:00006bf0       ??_C@_0BN@IMDCHIKM@?$GAscalar?5deleting?5destructor?8@ 0000000180007bf0     libvcruntime:undname.obj
 0001:00006c10       ??_C@_0BO@PFGOCPJJ@?$GAvector?5constructor?5iterator?8@ 0000000180007c10     libvcruntime:undname.obj
 0001:00006c30       ??_C@_0BN@LFPFMEDL@?$GAvector?5destructor?5iterator?8@ 0000000180007c30     libvcruntime:undname.obj
 0001:00006c50       ??_C@_0CE@IKBNEHA@?$GAvector?5vbase?5constructor?5itera@ 0000000180007c50     libvcruntime:undname.obj
 0001:00006c78       ??_C@_0BL@NILFHHPC@?$GAvirtual?5displacement?5map?8@ 0000000180007c78     libvcruntime:undname.obj
 0001:00006c98       ??_C@_0CB@JONCMFFK@?$GAeh?5vector?5constructor?5iterator@ 0000000180007c98     libvcruntime:undname.obj
 0001:00006cc0       ??_C@_0CA@GCEOPDGL@?$GAeh?5vector?5destructor?5iterator?8@ 0000000180007cc0     libvcruntime:undname.obj
 0001:00006ce0       ??_C@_0CH@OOJPLCPH@?$GAeh?5vector?5vbase?5constructor?5it@ 0000000180007ce0     libvcruntime:undname.obj
 0001:00006d08       ??_C@_0BL@LLKPOHJI@?$GAcopy?5constructor?5closure?8@ 0000000180007d08     libvcruntime:undname.obj
 0001:00006d28       ??_C@_0BA@KBCDOMBN@?$GAudt?5returning?8@ 0000000180007d28     libvcruntime:undname.obj
 0001:00006d38       ??_C@_03KLGMFNMG@?$GAEH@   0000000180007d38     libvcruntime:undname.obj
 0001:00006d3c       ??_C@_05KHLCHHI@?$GARTTI@  0000000180007d3c     libvcruntime:undname.obj
 0001:00006d48       ??_C@_0BA@KKLDJDLB@?$GAlocal?5vftable?8@ 0000000180007d48     libvcruntime:undname.obj
 0001:00006d58       ??_C@_0CE@IIHCMGGL@?$GAlocal?5vftable?5constructor?5clos@ 0000000180007d58     libvcruntime:undname.obj
 0001:00006d7c       ??_C@_06FHBGPFGH@?5new?$FL?$FN@ 0000000180007d7c     libvcruntime:undname.obj
 0001:00006d88       ??_C@_09LBNFPBCA@?5delete?$FL?$FN@ 0000000180007d88     libvcruntime:undname.obj
 0001:00006d98       ??_C@_0P@HJKNJFNN@?$GAomni?5callsig?8@ 0000000180007d98     libvcruntime:undname.obj
 0001:00006da8       ??_C@_0BL@CNOONJFP@?$GAplacement?5delete?5closure?8@ 0000000180007da8     libvcruntime:undname.obj
 0001:00006dc8       ??_C@_0BN@CKNJLHMB@?$GAplacement?5delete?$FL?$FN?5closure?8@ 0000000180007dc8     libvcruntime:undname.obj
 0001:00006de8       ??_C@_0CG@CFDHKGGD@?$GAmanaged?5vector?5constructor?5ite@ 0000000180007de8     libvcruntime:undname.obj
 0001:00006e10       ??_C@_0CF@IMGKMJNO@?$GAmanaged?5vector?5destructor?5iter@ 0000000180007e10     libvcruntime:undname.obj
 0001:00006e38       ??_C@_0CG@HLDDJMAG@?$GAeh?5vector?5copy?5constructor?5ite@ 0000000180007e38     libvcruntime:undname.obj
 0001:00006e60       ??_C@_0CM@FCBBDIGB@?$GAeh?5vector?5vbase?5copy?5construct@ 0000000180007e60     libvcruntime:undname.obj
 0001:00006e90       ??_C@_0BL@CLIPGLGB@?$GAdynamic?5initializer?5for?5?8@ 0000000180007e90     libvcruntime:undname.obj
 0001:00006eb0       ??_C@_0CB@PDBIFEP@?$GAdynamic?5atexit?5destructor?5for?5@ 0000000180007eb0     libvcruntime:undname.obj
 0001:00006ed8       ??_C@_0CD@CGAJBKEJ@?$GAvector?5copy?5constructor?5iterat@ 0000000180007ed8     libvcruntime:undname.obj
 0001:00006f00       ??_C@_0CJ@GJELGAMM@?$GAvector?5vbase?5copy?5constructor?5@ 0000000180007f00     libvcruntime:undname.obj
 0001:00006f30       ??_C@_0CL@FGIJHLCE@?$GAmanaged?5vector?5copy?5constructo@ 0000000180007f30     libvcruntime:undname.obj
 0001:00006f60       ??_C@_0BM@PMGGMLDN@?$GAlocal?5static?5thread?5guard?8@ 0000000180007f60     libvcruntime:undname.obj
 0001:00006f80       ??_C@_0N@BDNMDMOL@operator?5?$CC?$CC?5@ 0000000180007f80     libvcruntime:undname.obj
 0001:00006f90       ??_C@_0BC@GGEBGALA@operator?5co_await@ 0000000180007f90     libvcruntime:undname.obj
 0001:00006fa8       ??_C@_0M@GAAIMMOH@operator?$DM?$DN?$DO@ 0000000180007fa8     libvcruntime:undname.obj
 0001:00006fb8       ??_C@_0BC@DAFEJGAK@?5Type?5Descriptor?8@ 0000000180007fb8     libvcruntime:undname.obj
 0001:00006fd0       ??_C@_0BM@LDKODKLH@?5Base?5Class?5Descriptor?5at?5?$CI@ 0000000180007fd0     libvcruntime:undname.obj
 0001:00006ff0       ??_C@_0BD@LGICGFMM@?5Base?5Class?5Array?8@ 0000000180007ff0     libvcruntime:undname.obj
 0001:00007008       ??_C@_0BN@MECKDCOJ@?5Class?5Hierarchy?5Descriptor?8@ 0000000180008008     libvcruntime:undname.obj
 0001:00007028       ??_C@_0BK@CFCOFLF@?5Complete?5Object?5Locator?8@ 0000000180008028     libvcruntime:undname.obj
 0001:00007048       ??_C@_0BG@JNJLAMPM@?$GAanonymous?5namespace?8@ 0000000180008048     libvcruntime:undname.obj
 0001:00007078       ??_C@_1DM@KHCHBNEB@?$AAa?$AAp?$AAi?$AA?9?$AAm?$AAs?$AA?9?$AAw?$AAi?$AAn?$AA?9?$AAc?$AAo?$AAr?$AAe@ 0000000180008078     libvcruntime:winapi_downlevel.obj
 0001:000070b8       ??_C@_1DK@LPPGFMPP@?$AAa?$AAp?$AAi?$AA?9?$AAm?$AAs?$AA?9?$AAw?$AAi?$AAn?$AA?9?$AAc?$AAo?$AAr?$AAe@ 00000001800080b8     libvcruntime:winapi_downlevel.obj
 0001:000070f8       ??_C@_1BA@PFFKHIOG@?$AAa?$AAp?$AAi?$AA?9?$AAm?$AAs?$AA?9@ 00000001800080f8     libvcruntime:winapi_downlevel.obj
 0001:000072a0       format_validation_lookup_table 00000001800082a0     libucrt:output.obj
 0001:00007300       ??_C@_1O@CEDCILHN@?$AA?$CI?$AAn?$AAu?$AAl?$AAl?$AA?$CJ@ 0000000180008300     libucrt:output.obj
 0001:00007310       ??_C@_06OJHGLDPL@?$CInull?$CJ@ 0000000180008310     libucrt:output.obj
 0001:00007738       ??_C@_04KGLCPMCP@log2@     0000000180008738     libucrt:log2.obj
 0001:00007740       __real@03d0000000000000    0000000180008740     libucrt:log2.obj
 0001:00007748       __real@3ecb295c17f0bbbe    0000000180008748     libucrt:log2.obj
 0001:00007750       __real@3f3c8034c85dfff0    0000000180008750     libucrt:log2.obj
 0001:00007758       __real@3f62492307f1519f    0000000180008758     libucrt:log2.obj
 0001:00007760       __real@3f6249423bd94741    0000000180008760     libucrt:log2.obj
 0001:00007768       __real@3f80000000000000    0000000180008768     libucrt:log2.obj
 0001:00007770       __real@3f89999999865ede    0000000180008770     libucrt:log2.obj
 0001:00007778       __real@3f89999999bac6d4    0000000180008778     libucrt:log2.obj
 0001:00007780       __real@3fb55555555554e6    0000000180008780     libucrt:log2.obj
 0001:00007788       __real@3fb5555555555557    0000000180008788     libucrt:log2.obj
 0001:00007790       __real@3fe0000000000000    0000000180008790     libucrt:log2.obj
 0001:00007798       __real@3ff0000000000000    0000000180008798     libucrt:log2.obj
 0001:000077a0       __real@3ff7154400000000    00000001800087a0     libucrt:log2.obj
 0001:000077a8       __real@4000000000000000    00000001800087a8     libucrt:log2.obj
 0001:000077b0       __real@8000000000000000    00000001800087b0     libucrt:modf.obj
 0001:000077b8       __real@bff0000000000000    00000001800087b8     libucrt:round.obj
 0001:00008dc0       __newctype                 0000000180009dc0     libucrt:ctype.obj
 0001:000090c0       __newclmap                 000000018000a0c0     libucrt:ctype.obj
 0001:00009240       __newcumap                 000000018000a240     libucrt:ctype.obj
 0001:000093c0       _wctype                    000000018000a3c0     libucrt:ctype.obj
 0001:000095d0       ?large_power_data@?1??multiply_by_power_of_ten@__crt_strtox@@YA_NAEAUbig_integer@2@I@Z@4QBIB 000000018000a5d0     libucrt:strtod.obj
 0001:00009ed8       ?small_powers_of_ten@?1??multiply_by_power_of_ten@__crt_strtox@@YA_NAEAUbig_integer@2@I@Z@4QBIB 000000018000aed8     libucrt:strtod.obj
 0001:0000a800       __acrt_exception_action_table 000000018000b800     libucrt:exception_filter.obj
 0001:0000a8c0       __acrt_signal_action_table_count 000000018000b8c0     libucrt:exception_filter.obj
 0001:0000a8c8       __acrt_signal_action_first_fpe_index 000000018000b8c8     libucrt:exception_filter.obj
 0001:0000a8d0       __acrt_signal_action_fpe_count 000000018000b8d0     libucrt:exception_filter.obj
 0001:0000a8d8       ??_C@_1BI@BGOHAHKC@?$AAm?$AAs?$AAc?$AAo?$AAr?$AAe?$AAe?$AA?4?$AAd?$AAl?$AAl@ 000000018000b8d8     libucrt:exit.obj
 0001:0000a8f0       ??_C@_0P@MIGLKIOC@CorExitProcess@ 000000018000b8f0     libucrt:exit.obj
 0001:0000aae0       ??_C@_1EA@JGEFHKEI@?$AAa?$AAp?$AAi?$AA?9?$AAm?$AAs?$AA?9?$AAw?$AAi?$AAn?$AA?9?$AAc?$AAo?$AAr?$AAe@ 000000018000bae0     libucrt:winapi_thunks.obj
 0001:0000ab20       ??_C@_1DI@IJCEHOCB@?$AAa?$AAp?$AAi?$AA?9?$AAm?$AAs?$AA?9?$AAw?$AAi?$AAn?$AA?9?$AAc?$AAo?$AAr?$AAe@ 000000018000bb20     libucrt:winapi_thunks.obj
 0001:0000ab60       ??_C@_1EI@MPIAOHOC@?$AAa?$AAp?$AAi?$AA?9?$AAm?$AAs?$AA?9?$AAw?$AAi?$AAn?$AA?9?$AAc?$AAo?$AAr?$AAe@ 000000018000bb60     libucrt:winapi_thunks.obj
 0001:0000abb0       ??_C@_1FK@FPHCKFIE@?$AAa?$AAp?$AAi?$AA?9?$AAm?$AAs?$AA?9?$AAw?$AAi?$AAn?$AA?9?$AAc?$AAo?$AAr?$AAe@ 000000018000bbb0     libucrt:winapi_thunks.obj
 0001:0000ac10       ??_C@_1EM@DILCGIIO@?$AAa?$AAp?$AAi?$AA?9?$AAm?$AAs?$AA?9?$AAw?$AAi?$AAn?$AA?9?$AAc?$AAo?$AAr?$AAe@ 000000018000bc10     libucrt:winapi_thunks.obj
 0001:0000ac60       ??_C@_1DM@LNCGDDPN@?$AAa?$AAp?$AAi?$AA?9?$AAm?$AAs?$AA?9?$AAw?$AAi?$AAn?$AA?9?$AAc?$AAo?$AAr?$AAe@ 000000018000bc60     libucrt:winapi_thunks.obj
 0001:0000aca0       ??_C@_1DO@FPAPJEMD@?$AAa?$AAp?$AAi?$AA?9?$AAm?$AAs?$AA?9?$AAw?$AAi?$AAn?$AA?9?$AAc?$AAo?$AAr?$AAe@ 000000018000bca0     libucrt:winapi_thunks.obj
 0001:0000ace0       ??_C@_1DK@NDHNAHIO@?$AAa?$AAp?$AAi?$AA?9?$AAm?$AAs?$AA?9?$AAw?$AAi?$AAn?$AA?9?$AAc?$AAo?$AAr?$AAe@ 000000018000bce0     libucrt:winapi_thunks.obj
 0001:0000ad20       ??_C@_1DM@KGHDGBCM@?$AAa?$AAp?$AAi?$AA?9?$AAm?$AAs?$AA?9?$AAw?$AAi?$AAn?$AA?9?$AAc?$AAo?$AAr?$AAe@ 000000018000bd20     libucrt:winapi_thunks.obj
 0001:0000ad60       ??_C@_1EO@IJIOEFOH@?$AAa?$AAp?$AAi?$AA?9?$AAm?$AAs?$AA?9?$AAw?$AAi?$AAn?$AA?9?$AAr?$AAt?$AAc?$AAo@ 000000018000bd60     libucrt:winapi_thunks.obj
 0001:0000adb0       ??_C@_1FG@HHGEKANL@?$AAa?$AAp?$AAi?$AA?9?$AAm?$AAs?$AA?9?$AAw?$AAi?$AAn?$AA?9?$AAs?$AAe?$AAc?$AAu@ 000000018000bdb0     libucrt:winapi_thunks.obj
 0001:0000ae10       ??_C@_1EG@DBIOJECG@?$AAe?$AAx?$AAt?$AA?9?$AAm?$AAs?$AA?9?$AAw?$AAi?$AAn?$AA?9?$AAn?$AAt?$AAu?$AAs@ 000000018000be10     libucrt:winapi_thunks.obj
 0001:0000ae60       ??_C@_1EO@FIHMJCLF@?$AAe?$AAx?$AAt?$AA?9?$AAm?$AAs?$AA?9?$AAw?$AAi?$AAn?$AA?9?$AAn?$AAt?$AAu?$AAs@ 000000018000be60     libucrt:winapi_thunks.obj
 0001:0000aeb0       ??_C@_1EG@DPGNFKGC@?$AAa?$AAp?$AAi?$AA?9?$AAm?$AAs?$AA?9?$AAw?$AAi?$AAn?$AA?9?$AAa?$AAp?$AAp?$AAm@ 000000018000beb0     libucrt:winapi_thunks.obj
 0001:0000aef8       ??_C@_1BA@IAIFMGEF@?$AAe?$AAx?$AAt?$AA?9?$AAm?$AAs?$AA?9@ 000000018000bef8     libucrt:winapi_thunks.obj
 0001:0000af10       ??_C@_0BA@FHFNEAED@AreFileApisANSI@ 000000018000bf10     libucrt:winapi_thunks.obj
 0001:0000af30       ??_C@_0BE@LJANKFHF@EnumSystemLocalesEx@ 000000018000bf30     libucrt:winapi_thunks.obj
 0001:0000af70       ??_C@_0BA@EPCJIIPD@GetDateFormatEx@ 000000018000bf70     libucrt:winapi_thunks.obj
 0001:0000af90       ??_C@_0BA@CIJJKCJJ@GetTimeFormatEx@ 000000018000bf90     libucrt:winapi_thunks.obj
 0001:0000afa8       ??_C@_0BJ@PBCCBIPI@GetUserDefaultLocaleName@ 000000018000bfa8     libucrt:winapi_thunks.obj
 0001:0000afd8       ??_C@_0BC@CELBKLLA@IsValidLocaleName@ 000000018000bfd8     libucrt:winapi_thunks.obj
 0001:0000b000       ??_C@_0BB@CDHDDLLP@LCIDToLocaleName@ 000000018000c000     libucrt:winapi_thunks.obj
 0001:0000b020       ??_C@_0BB@HBDEELFH@LocaleNameToLCID@ 000000018000c020     libucrt:winapi_thunks.obj
 0001:0000b038       ??_C@_0CF@OJOFEIGO@AppPolicyGetProcessTerminationM@ 000000018000c038     libucrt:winapi_thunks.obj
 0001:0000b0e0       ??_C@_09OFJJIMPC@NAN?$CISNAN?$CJ@ 000000018000c0e0     libucrt:cvt.obj
 0001:0000b0f0       ??_C@_09IPFBKMDL@nan?$CIsnan?$CJ@ 000000018000c0f0     libucrt:cvt.obj
 0001:0000b100       ??_C@_08IKHNHAJ@NAN?$CIIND?$CJ@ 000000018000c100     libucrt:cvt.obj
 0001:0000b110       ??_C@_08OFCDMILK@nan?$CIind?$CJ@ 000000018000c110     libucrt:cvt.obj
 0001:0000b11c       ??_C@_05KLBDPFGC@e?$CL000@ 000000018000c11c     libucrt:cvt.obj
 0001:0000b1b0       __lc_category              000000018000c1b0     libucrt:wsetlocale.obj
 0001:0000b240       ??_C@_1O@GIFLHMA@?$AAL?$AAC?$AA_?$AAA?$AAL?$AAL@ 000000018000c240     libucrt:wsetlocale.obj
 0001:0000b250       ??_C@_1BG@PPOMIBNJ@?$AAL?$AAC?$AA_?$AAC?$AAO?$AAL?$AAL?$AAA?$AAT?$AAE@ 000000018000c250     libucrt:wsetlocale.obj
 0001:0000b268       ??_C@_1BC@FFJGAPJM@?$AAL?$AAC?$AA_?$AAC?$AAT?$AAY?$AAP?$AAE@ 000000018000c268     libucrt:wsetlocale.obj
 0001:0000b280       ??_C@_1BI@PCKFNJFB@?$AAL?$AAC?$AA_?$AAM?$AAO?$AAN?$AAE?$AAT?$AAA?$AAR?$AAY@ 000000018000c280     libucrt:wsetlocale.obj
 0001:0000b298       ??_C@_1BG@ENIEDKID@?$AAL?$AAC?$AA_?$AAN?$AAU?$AAM?$AAE?$AAR?$AAI?$AAC@ 000000018000c298     libucrt:wsetlocale.obj
 0001:0000b2b0       ??_C@_1BA@HAAOMIIG@?$AAL?$AAC?$AA_?$AAT?$AAI?$AAM?$AAE@ 000000018000c2b0     libucrt:wsetlocale.obj
 0001:0000b2c0       ??_C@_15NBPDDFIP@?$AA?$DN?$AA?$DL@ 000000018000c2c0     libucrt:wsetlocale.obj
 0001:0000b2c8       ??_C@_13PJJBFPED@?$AA?$DL@ 000000018000c2c8     libucrt:wsetlocale.obj
 0001:0000b2cc       ??_C@_13NMPKAAJP@?$AA?$DN@ 000000018000c2cc     libucrt:wsetlocale.obj
 0001:0000b2d0       ??_C@_17EFJLDFDO@?$AA?9?$AA_?$AA?4@ 000000018000c2d0     libucrt:wsetlocale.obj
 0001:0000b2d8       ??_C@_13FHBKNHDA@?$AAC@    000000018000c2d8     libucrt:wsetlocale.obj
 0001:0000b2e0       ??_C@_17MBJJLFDM@?$AA_?$AA?4?$AA?0@ 000000018000c2e0     libucrt:wsetlocale.obj
 0001:0000b2e8       ??_C@_13ENNFDPBH@?$AA_@    000000018000c2e8     libucrt:wsetlocale.obj
 0001:0000b2f0       __lc_time_c                000000018000c2f0     libucrt:nlsdata.obj
 0001:0000b5b0       ??_C@_03KOEHGMDN@Sun@      000000018000c5b0     libucrt:nlsdata.obj
 0001:0000b5b4       ??_C@_03PDAGKDH@Mon@       000000018000c5b4     libucrt:nlsdata.obj
 0001:0000b5b8       ??_C@_03NAGEINEP@Tue@      000000018000c5b8     libucrt:nlsdata.obj
 0001:0000b5bc       ??_C@_03MHOMLAJA@Wed@      000000018000c5bc     libucrt:nlsdata.obj
 0001:0000b5c0       ??_C@_03IOFIKPDN@Thu@      000000018000c5c0     libucrt:nlsdata.obj
 0001:0000b5c4       ??_C@_03IDIOELNC@Fri@      000000018000c5c4     libucrt:nlsdata.obj
 0001:0000b5c8       ??_C@_03FEFJNEK@Sat@       000000018000c5c8     libucrt:nlsdata.obj
 0001:0000b5cc       ??_C@_06OOPIFAJ@Sunday@    000000018000c5cc     libucrt:nlsdata.obj
 0001:0000b5d4       ??_C@_06JLEDEDGH@Monday@   000000018000c5d4     libucrt:nlsdata.obj
 0001:0000b5e0       ??_C@_07BAAGCFCM@Tuesday@  000000018000c5e0     libucrt:nlsdata.obj
 0001:0000b5e8       ??_C@_09DLIGFAKA@Wednesday@ 000000018000c5e8     libucrt:nlsdata.obj
 0001:0000b5f8       ??_C@_08HACCIKIA@Thursday@ 000000018000c5f8     libucrt:nlsdata.obj
 0001:0000b604       ??_C@_06JECMNKMI@Friday@   000000018000c604     libucrt:nlsdata.obj
 0001:0000b610       ??_C@_08INBOOONO@Saturday@ 000000018000c610     libucrt:nlsdata.obj
 0001:0000b61c       ??_C@_03JIHJHPIE@Jan@      000000018000c61c     libucrt:nlsdata.obj
 0001:0000b620       ??_C@_03HJBDCHOM@Feb@      000000018000c620     libucrt:nlsdata.obj
 0001:0000b624       ??_C@_03ODNJBKGA@Mar@      000000018000c624     libucrt:nlsdata.obj
 0001:0000b628       ??_C@_03LEOLGMJP@Apr@      000000018000c628     libucrt:nlsdata.obj
 0001:0000b62c       ??_C@_03CNMDKL@May@        000000018000c62c     libucrt:nlsdata.obj
 0001:0000b630       ??_C@_03IDFGHECI@Jun@      000000018000c630     libucrt:nlsdata.obj
 0001:0000b634       ??_C@_03LBGABGKK@Jul@      000000018000c634     libucrt:nlsdata.obj
 0001:0000b638       ??_C@_03IFJFEIGA@Aug@      000000018000c638     libucrt:nlsdata.obj
 0001:0000b63c       ??_C@_03GGCAPAJC@Sep@      000000018000c63c     libucrt:nlsdata.obj
 0001:0000b640       ??_C@_03BMAOKBAD@Oct@      000000018000c640     libucrt:nlsdata.obj
 0001:0000b644       ??_C@_03JPJOFNIA@Nov@      000000018000c644     libucrt:nlsdata.obj
 0001:0000b648       ??_C@_03MKABNOCG@Dec@      000000018000c648     libucrt:nlsdata.obj
 0001:0000b650       ??_C@_07CGJPFGJA@January@  000000018000c650     libucrt:nlsdata.obj
 0001:0000b658       ??_C@_08GNJGEPFN@February@ 000000018000c658     libucrt:nlsdata.obj
 0001:0000b664       ??_C@_05HPCKOFNC@March@    000000018000c664     libucrt:nlsdata.obj
 0001:0000b66c       ??_C@_05DMJDNLEJ@April@    000000018000c66c     libucrt:nlsdata.obj
 0001:0000b674       ??_C@_04CNLMGBGM@June@     000000018000c674     libucrt:nlsdata.obj
 0001:0000b67c       ??_C@_04MIEPOIFP@July@     000000018000c67c     libucrt:nlsdata.obj
 0001:0000b684       ??_C@_06LBBHFDDG@August@   000000018000c684     libucrt:nlsdata.obj
 0001:0000b690       ??_C@_09BHHEALKD@September@ 000000018000c690     libucrt:nlsdata.obj
 0001:0000b6a0       ??_C@_07JJNFCEND@October@  000000018000c6a0     libucrt:nlsdata.obj
 0001:0000b6a8       ??_C@_08HCHEGEOA@November@ 000000018000c6a8     libucrt:nlsdata.obj
 0001:0000b6b8       ??_C@_08EDHMEBNP@December@ 000000018000c6b8     libucrt:nlsdata.obj
 0001:0000b6c4       ??_C@_02DEDBPAFC@AM@       000000018000c6c4     libucrt:nlsdata.obj
 0001:0000b6c8       ??_C@_02CJNFDJBF@PM@       000000018000c6c8     libucrt:nlsdata.obj
 0001:0000b6d0       ??_C@_08BPBNCDIB@MM?1dd?1yy@ 000000018000c6d0     libucrt:nlsdata.obj
 0001:0000b6e0       ??_C@_0BE@CKGJFCPC@dddd?0?5MMMM?5dd?0?5yyyy@ 000000018000c6e0     libucrt:nlsdata.obj
 0001:0000b6f8       ??_C@_08JCCMCCIL@HH?3mm?3ss@ 000000018000c6f8     libucrt:nlsdata.obj
 0001:0000b708       ??_C@_17MBGCMIPB@?$AAS?$AAu?$AAn@ 000000018000c708     libucrt:nlsdata.obj
 0001:0000b710       ??_C@_17KBOMKBF@?$AAM?$AAo?$AAn@ 000000018000c710     libucrt:nlsdata.obj
 0001:0000b718       ??_C@_17BMKGEGOJ@?$AAT?$AAu?$AAe@ 000000018000c718     libucrt:nlsdata.obj
 0001:0000b720       ??_C@_17CJEDCEPE@?$AAW?$AAe?$AAd@ 000000018000c720     libucrt:nlsdata.obj
 0001:0000b728       ??_C@_17PDPHAADD@?$AAT?$AAh?$AAu@ 000000018000c728     libucrt:nlsdata.obj
 0001:0000b730       ??_C@_17HFOLPPLP@?$AAF?$AAr?$AAi@ 000000018000c730     libucrt:nlsdata.obj
 0001:0000b738       ??_C@_17GGIBDPIH@?$AAS?$AAa?$AAt@ 000000018000c738     libucrt:nlsdata.obj
 0001:0000b740       ??_C@_1O@IHNHDHPB@?$AAS?$AAu?$AAn?$AAd?$AAa?$AAy@ 000000018000c740     libucrt:nlsdata.obj
 0001:0000b750       ??_C@_1O@MMNBFLIA@?$AAM?$AAo?$AAn?$AAd?$AAa?$AAy@ 000000018000c750     libucrt:nlsdata.obj
 0001:0000b760       ??_C@_1BA@ENFBFFEK@?$AAT?$AAu?$AAe?$AAs?$AAd?$AAa?$AAy@ 000000018000c760     libucrt:nlsdata.obj
 0001:0000b770       ??_C@_1BE@EBOGMDOH@?$AAW?$AAe?$AAd?$AAn?$AAe?$AAs?$AAd?$AAa?$AAy@ 000000018000c770     libucrt:nlsdata.obj
 0001:0000b788       ??_C@_1BC@HHMNLIHE@?$AAT?$AAh?$AAu?$AAr?$AAs?$AAd?$AAa?$AAy@ 000000018000c788     libucrt:nlsdata.obj
 0001:0000b7a0       ??_C@_1O@PDICJHAG@?$AAF?$AAr?$AAi?$AAd?$AAa?$AAy@ 000000018000c7a0     libucrt:nlsdata.obj
 0001:0000b7b0       ??_C@_1BC@ENMNNPAJ@?$AAS?$AAa?$AAt?$AAu?$AAr?$AAd?$AAa?$AAy@ 000000018000c7b0     libucrt:nlsdata.obj
 0001:0000b7c8       ??_C@_17DKNBKCHM@?$AAJ?$AAa?$AAn@ 000000018000c7c8     libucrt:nlsdata.obj
 0001:0000b7d0       ??_C@_17LMDJEKJN@?$AAF?$AAe?$AAb@ 000000018000c7d0     libucrt:nlsdata.obj
 0001:0000b7d8       ??_C@_17CKNLEDEC@?$AAM?$AAa?$AAr@ 000000018000c7d8     libucrt:nlsdata.obj
 0001:0000b7e0       ??_C@_17LFPOIHDD@?$AAA?$AAp?$AAr@ 000000018000c7e0     libucrt:nlsdata.obj
 0001:0000b7e8       ??_C@_17PNNKMEED@?$AAM?$AAa?$AAy@ 000000018000c7e8     libucrt:nlsdata.obj
 0001:0000b7f0       ??_C@_17KCJGOCPB@?$AAJ?$AAu?$AAn@ 000000018000c7f0     libucrt:nlsdata.obj
 0001:0000b7f8       ??_C@_17IJPCKHK@?$AAJ?$AAu?$AAl@ 000000018000c7f8     libucrt:nlsdata.obj
 0001:0000b800       ??_C@_17ICPELBCN@?$AAA?$AAu?$AAg@ 000000018000c800     libucrt:nlsdata.obj
 0001:0000b808       ??_C@_17HCHCOKMG@?$AAS?$AAe?$AAp@ 000000018000c808     libucrt:nlsdata.obj
 0001:0000b810       ??_C@_17FNLKOI@?$AAO?$AAc?$AAt@ 000000018000c810     libucrt:nlsdata.obj
 0001:0000b818       ??_C@_17BBDMLCIG@?$AAN?$AAo?$AAv@ 000000018000c818     libucrt:nlsdata.obj
 0001:0000b820       ??_C@_17EGKACKIF@?$AAD?$AAe?$AAc@ 000000018000c820     libucrt:nlsdata.obj
 0001:0000b828       ??_C@_1BA@EFMEIEBA@?$AAJ?$AAa?$AAn?$AAu?$AAa?$AAr?$AAy@ 000000018000c828     libucrt:nlsdata.obj
 0001:0000b838       ??_C@_1BC@JGDDFFAM@?$AAF?$AAe?$AAb?$AAr?$AAu?$AAa?$AAr?$AAy@ 000000018000c838     libucrt:nlsdata.obj
 0001:0000b850       ??_C@_1M@IKEENEDF@?$AAM?$AAa?$AAr?$AAc?$AAh@ 000000018000c850     libucrt:nlsdata.obj
 0001:0000b860       ??_C@_1M@GJNLMHFD@?$AAA?$AAp?$AAr?$AAi?$AAl@ 000000018000c860     libucrt:nlsdata.obj
 0001:0000b870       ??_C@_19EPFLPGAP@?$AAJ?$AAu?$AAn?$AAe@ 000000018000c870     libucrt:nlsdata.obj
 0001:0000b880       ??_C@_19BIFMLPCD@?$AAJ?$AAu?$AAl?$AAy@ 000000018000c880     libucrt:nlsdata.obj
 0001:0000b890       ??_C@_1O@PAHLKOAC@?$AAA?$AAu?$AAg?$AAu?$AAs?$AAt@ 000000018000c890     libucrt:nlsdata.obj
 0001:0000b8a0       ??_C@_1BE@DKAAMBJL@?$AAS?$AAe?$AAp?$AAt?$AAe?$AAm?$AAb?$AAe?$AAr@ 000000018000c8a0     libucrt:nlsdata.obj
 0001:0000b8b8       ??_C@_1BA@EPANDLNG@?$AAO?$AAc?$AAt?$AAo?$AAb?$AAe?$AAr@ 000000018000c8b8     libucrt:nlsdata.obj
 0001:0000b8c8       ??_C@_1BC@BGLIFPF@?$AAN?$AAo?$AAv?$AAe?$AAm?$AAb?$AAe?$AAr@ 000000018000c8c8     libucrt:nlsdata.obj
 0001:0000b8e0       ??_C@_1BC@FEMKIFH@?$AAD?$AAe?$AAc?$AAe?$AAm?$AAb?$AAe?$AAr@ 000000018000c8e0     libucrt:nlsdata.obj
 0001:0000b8f4       ??_C@_15ODEHAHHF@?$AAA?$AAM@ 000000018000c8f4     libucrt:nlsdata.obj
 0001:0000b8fc       ??_C@_15CLMNNGEL@?$AAP?$AAM@ 000000018000c8fc     libucrt:nlsdata.obj
 0001:0000b908       ??_C@_1BC@IEBCMHCM@?$AAM?$AAM?$AA?1?$AAd?$AAd?$AA?1?$AAy?$AAy@ 000000018000c908     libucrt:nlsdata.obj
 0001:0000b920       ??_C@_1CI@KNAKOEBC@?$AAd?$AAd?$AAd?$AAd?$AA?0?$AA?5?$AAM?$AAM?$AAM?$AAM?$AA?5?$AAd?$AAd?$AA?0?$AA?5@ 000000018000c920     libucrt:nlsdata.obj
 0001:0000b948       ??_C@_1BC@GDGBMEMK@?$AAH?$AAH?$AA?3?$AAm?$AAm?$AA?3?$AAs?$AAs@ 000000018000c948     libucrt:nlsdata.obj
 0001:0000b960       __log10_256_lead           000000018000c960     libucrt:log10_256_lead_tail_table.obj
 0001:0000c170       __log10_256_tail           000000018000d170     libucrt:log10_256_lead_tail_table.obj
 0001:0000c980       __log_F_inv_qword          000000018000d980     libucrt:log_f_inv_qword_table.obj
 0001:0000d190       ??_C@_05HGHHAHAP@log10@    000000018000e190     libucrt:log_special.obj
 0001:0000d1a0       __log_256_lead             000000018000e1a0     libucrt:log_256_lead_tail_table.obj
 0001:0000d9b0       __log_256_tail             000000018000e9b0     libucrt:log_256_lead_tail_table.obj
 0001:0000e1c0       __two_to_jby64_head_table  000000018000f1c0     libucrt:two_to_jby64_head_tail_table.obj
 0001:0000e3c0       __two_to_jby64_tail_table  000000018000f3c0     libucrt:two_to_jby64_head_tail_table.obj
 0001:0000e5c0       ??_C@_04MBFDLNIM@powf@     000000018000f5c0     libucrt:pow_special.obj
 0001:0000e5c8       ??_C@_03JGHBODFD@pow@      000000018000f5c8     libucrt:pow_special.obj
 0001:0000e600       __two_to_jby64_table       000000018000f600     libucrt:two_to_jby64_table.obj
 0001:00010538       ??_C@_01GBGANLPD@0@        0000000180011538     libucrt:cfout.obj
 0001:0001053c       ??_C@_05DNEBIAHO@1?$CDINF@ 000000018001153c     libucrt:cfout.obj
 0001:00010544       ??_C@_06IMKFLFPG@1?$CDQNAN@ 0000000180011544     libucrt:cfout.obj
 0001:0001054c       ??_C@_06PGGFOGJG@1?$CDSNAN@ 000000018001154c     libucrt:cfout.obj
 0001:00010554       ??_C@_05PHHOCPM@1?$CDIND@  0000000180011554     libucrt:cfout.obj
 0001:00010560       __acrt_rg_language         0000000180011560     libucrt:get_qualified_locale.obj
 0001:00010970       __acrt_rg_language_count   0000000180011970     libucrt:get_qualified_locale.obj
 0001:00010980       __acrt_rg_country          0000000180011980     libucrt:get_qualified_locale.obj
 0001:00010af0       __acrt_rg_country_count    0000000180011af0     libucrt:get_qualified_locale.obj
 0001:00010af8       ??_C@_1BC@LLOKLNP@?$AAa?$AAm?$AAe?$AAr?$AAi?$AAc?$AAa?$AAn@ 0000000180011af8     libucrt:get_qualified_locale.obj
 0001:00010b10       ??_C@_1CC@HEIGCDGG@?$AAa?$AAm?$AAe?$AAr?$AAi?$AAc?$AAa?$AAn?$AA?5?$AAe?$AAn?$AAg?$AAl?$AAi?$AAs@ 0000000180011b10     libucrt:get_qualified_locale.obj
 0001:00010b38       ??_C@_1CC@IHCNOMIN@?$AAa?$AAm?$AAe?$AAr?$AAi?$AAc?$AAa?$AAn?$AA?9?$AAe?$AAn?$AAg?$AAl?$AAi?$AAs@ 0000000180011b38     libucrt:get_qualified_locale.obj
 0001:00010b60       ??_C@_1BG@GKAGPCGG@?$AAa?$AAu?$AAs?$AAt?$AAr?$AAa?$AAl?$AAi?$AAa?$AAn@ 0000000180011b60     libucrt:get_qualified_locale.obj
 0001:00010b78       ??_C@_1BA@GMENCENF@?$AAb?$AAe?$AAl?$AAg?$AAi?$AAa?$AAn@ 0000000180011b78     libucrt:get_qualified_locale.obj
 0001:00010b88       ??_C@_1BC@PJMIIAAN@?$AAc?$AAa?$AAn?$AAa?$AAd?$AAi?$AAa?$AAn@ 0000000180011b88     libucrt:get_qualified_locale.obj
 0001:00010ba0       ??_C@_17NOIMNFBF@?$AAc?$AAh?$AAh@ 0000000180011ba0     libucrt:get_qualified_locale.obj
 0001:00010ba8       ??_C@_17GGDALCHA@?$AAc?$AAh?$AAi@ 0000000180011ba8     libucrt:get_qualified_locale.obj
 0001:00010bb0       ??_C@_1BA@NPNJKIBL@?$AAc?$AAh?$AAi?$AAn?$AAe?$AAs?$AAe@ 0000000180011bb0     libucrt:get_qualified_locale.obj
 0001:00010bc0       ??_C@_1CC@DINBAMMJ@?$AAc?$AAh?$AAi?$AAn?$AAe?$AAs?$AAe?$AA?9?$AAh?$AAo?$AAn?$AAg?$AAk?$AAo?$AAn@ 0000000180011bc0     libucrt:get_qualified_locale.obj
 0001:00010be8       ??_C@_1CG@IOBJPACO@?$AAc?$AAh?$AAi?$AAn?$AAe?$AAs?$AAe?$AA?9?$AAs?$AAi?$AAm?$AAp?$AAl?$AAi?$AAf@ 0000000180011be8     libucrt:get_qualified_locale.obj
 0001:00010c10       ??_C@_1CE@GAJNDCKG@?$AAc?$AAh?$AAi?$AAn?$AAe?$AAs?$AAe?$AA?9?$AAs?$AAi?$AAn?$AAg?$AAa?$AAp?$AAo@ 0000000180011c10     libucrt:get_qualified_locale.obj
 0001:00010c38       ??_C@_1CI@PAJPIOOD@?$AAc?$AAh?$AAi?$AAn?$AAe?$AAs?$AAe?$AA?9?$AAt?$AAr?$AAa?$AAd?$AAi?$AAt?$AAi@ 0000000180011c38     libucrt:get_qualified_locale.obj
 0001:00010c60       ??_C@_1BM@NILJBMMD@?$AAd?$AAu?$AAt?$AAc?$AAh?$AA?9?$AAb?$AAe?$AAl?$AAg?$AAi?$AAa?$AAn@ 0000000180011c60     libucrt:get_qualified_locale.obj
 0001:00010c80       ??_C@_1CC@OOJPJNEJ@?$AAe?$AAn?$AAg?$AAl?$AAi?$AAs?$AAh?$AA?9?$AAa?$AAm?$AAe?$AAr?$AAi?$AAc?$AAa@ 0000000180011c80     libucrt:get_qualified_locale.obj
 0001:00010ca8       ??_C@_1BI@IOLFEEM@?$AAe?$AAn?$AAg?$AAl?$AAi?$AAs?$AAh?$AA?9?$AAa?$AAu?$AAs@ 0000000180011ca8     libucrt:get_qualified_locale.obj
 0001:00010cc0       ??_C@_1BO@HFFNLENJ@?$AAe?$AAn?$AAg?$AAl?$AAi?$AAs?$AAh?$AA?9?$AAb?$AAe?$AAl?$AAi?$AAz?$AAe@ 0000000180011cc0     libucrt:get_qualified_locale.obj
 0001:00010ce0       ??_C@_1BI@HAPKJMPO@?$AAe?$AAn?$AAg?$AAl?$AAi?$AAs?$AAh?$AA?9?$AAc?$AAa?$AAn@ 0000000180011ce0     libucrt:get_qualified_locale.obj
 0001:00010cf8       ??_C@_1CE@HLNDMIOJ@?$AAe?$AAn?$AAg?$AAl?$AAi?$AAs?$AAh?$AA?9?$AAc?$AAa?$AAr?$AAi?$AAb?$AAb?$AAe@ 0000000180011cf8     libucrt:get_qualified_locale.obj
 0001:00010d20       ??_C@_1BI@LDHJHHAC@?$AAe?$AAn?$AAg?$AAl?$AAi?$AAs?$AAh?$AA?9?$AAi?$AAr?$AAe@ 0000000180011d20     libucrt:get_qualified_locale.obj
 0001:00010d38       ??_C@_1CA@NJMMCFOC@?$AAe?$AAn?$AAg?$AAl?$AAi?$AAs?$AAh?$AA?9?$AAj?$AAa?$AAm?$AAa?$AAi?$AAc?$AAa@ 0000000180011d38     libucrt:get_qualified_locale.obj
 0001:00010d58       ??_C@_1BG@BHJEBBGG@?$AAe?$AAn?$AAg?$AAl?$AAi?$AAs?$AAh?$AA?9?$AAn?$AAz@ 0000000180011d58     libucrt:get_qualified_locale.obj
 0001:00010d70       ??_C@_1CK@FGOEJJCO@?$AAe?$AAn?$AAg?$AAl?$AAi?$AAs?$AAh?$AA?9?$AAs?$AAo?$AAu?$AAt?$AAh?$AA?5?$AAa@ 0000000180011d70     libucrt:get_qualified_locale.obj
 0001:00010da0       ??_C@_1DE@PDBJPCJ@?$AAe?$AAn?$AAg?$AAl?$AAi?$AAs?$AAh?$AA?9?$AAt?$AAr?$AAi?$AAn?$AAi?$AAd?$AAa@ 0000000180011da0     libucrt:get_qualified_locale.obj
 0001:00010dd8       ??_C@_1BG@JGCANDME@?$AAe?$AAn?$AAg?$AAl?$AAi?$AAs?$AAh?$AA?9?$AAu?$AAk@ 0000000180011dd8     libucrt:get_qualified_locale.obj
 0001:00010df0       ??_C@_1BG@DINKMLE@?$AAe?$AAn?$AAg?$AAl?$AAi?$AAs?$AAh?$AA?9?$AAu?$AAs@ 0000000180011df0     libucrt:get_qualified_locale.obj
 0001:00010e08       ??_C@_1BI@NMFDBHJE@?$AAe?$AAn?$AAg?$AAl?$AAi?$AAs?$AAh?$AA?9?$AAu?$AAs?$AAa@ 0000000180011e08     libucrt:get_qualified_locale.obj
 0001:00010e20       ??_C@_1BO@OIHKJKII@?$AAf?$AAr?$AAe?$AAn?$AAc?$AAh?$AA?9?$AAb?$AAe?$AAl?$AAg?$AAi?$AAa?$AAn@ 0000000180011e20     libucrt:get_qualified_locale.obj
 0001:00010e40       ??_C@_1CA@NKAELJKI@?$AAf?$AAr?$AAe?$AAn?$AAc?$AAh?$AA?9?$AAc?$AAa?$AAn?$AAa?$AAd?$AAi?$AAa?$AAn@ 0000000180011e40     libucrt:get_qualified_locale.obj
 0001:00010e60       ??_C@_1CE@MGKCNLGN@?$AAf?$AAr?$AAe?$AAn?$AAc?$AAh?$AA?9?$AAl?$AAu?$AAx?$AAe?$AAm?$AAb?$AAo?$AAu@ 0000000180011e60     libucrt:get_qualified_locale.obj
 0001:00010e88       ??_C@_1BK@CEGEAILM@?$AAf?$AAr?$AAe?$AAn?$AAc?$AAh?$AA?9?$AAs?$AAw?$AAi?$AAs?$AAs@ 0000000180011e88     libucrt:get_qualified_locale.obj
 0001:00010ea8       ??_C@_1CA@PAFKEOCC@?$AAg?$AAe?$AAr?$AAm?$AAa?$AAn?$AA?9?$AAa?$AAu?$AAs?$AAt?$AAr?$AAi?$AAa?$AAn@ 0000000180011ea8     libucrt:get_qualified_locale.obj
 0001:00010ec8       ??_C@_1CI@HCFHGOFD@?$AAg?$AAe?$AAr?$AAm?$AAa?$AAn?$AA?9?$AAl?$AAi?$AAc?$AAh?$AAt?$AAe?$AAn?$AAs@ 0000000180011ec8     libucrt:get_qualified_locale.obj
 0001:00010ef0       ??_C@_1CE@FEDDNPDG@?$AAg?$AAe?$AAr?$AAm?$AAa?$AAn?$AA?9?$AAl?$AAu?$AAx?$AAe?$AAm?$AAb?$AAo?$AAu@ 0000000180011ef0     libucrt:get_qualified_locale.obj
 0001:00010f18       ??_C@_1BK@LIMINNMN@?$AAg?$AAe?$AAr?$AAm?$AAa?$AAn?$AA?9?$AAs?$AAw?$AAi?$AAs?$AAs@ 0000000180011f18     libucrt:get_qualified_locale.obj
 0001:00010f38       ??_C@_1BM@LGMDBEPD@?$AAi?$AAr?$AAi?$AAs?$AAh?$AA?9?$AAe?$AAn?$AAg?$AAl?$AAi?$AAs?$AAh@ 0000000180011f38     libucrt:get_qualified_locale.obj
 0001:00010f58       ??_C@_1BM@NNCFBAEE@?$AAi?$AAt?$AAa?$AAl?$AAi?$AAa?$AAn?$AA?9?$AAs?$AAw?$AAi?$AAs?$AAs@ 0000000180011f58     libucrt:get_qualified_locale.obj
 0001:00010f78       ??_C@_1BE@FEDJNPIB@?$AAn?$AAo?$AAr?$AAw?$AAe?$AAg?$AAi?$AAa?$AAn@ 0000000180011f78     libucrt:get_qualified_locale.obj
 0001:00010f90       ??_C@_1CC@CILKDEIE@?$AAn?$AAo?$AAr?$AAw?$AAe?$AAg?$AAi?$AAa?$AAn?$AA?9?$AAb?$AAo?$AAk?$AAm?$AAa@ 0000000180011f90     libucrt:get_qualified_locale.obj
 0001:00010fb8       ??_C@_1CE@DHMMHEPL@?$AAn?$AAo?$AAr?$AAw?$AAe?$AAg?$AAi?$AAa?$AAn?$AA?9?$AAn?$AAy?$AAn?$AAo?$AAr@ 0000000180011fb8     libucrt:get_qualified_locale.obj
 0001:00010fe0       ??_C@_1CK@OPNMHECD@?$AAp?$AAo?$AAr?$AAt?$AAu?$AAg?$AAu?$AAe?$AAs?$AAe?$AA?9?$AAb?$AAr?$AAa?$AAz@ 0000000180011fe0     libucrt:get_qualified_locale.obj
 0001:00011010       ??_C@_1CE@KEEHCDB@?$AAs?$AAp?$AAa?$AAn?$AAi?$AAs?$AAh?$AA?9?$AAa?$AAr?$AAg?$AAe?$AAn?$AAt?$AAi@ 0000000180012010     libucrt:get_qualified_locale.obj
 0001:00011038       ??_C@_1CA@GIAOLHJD@?$AAs?$AAp?$AAa?$AAn?$AAi?$AAs?$AAh?$AA?9?$AAb?$AAo?$AAl?$AAi?$AAv?$AAi?$AAa@ 0000000180012038     libucrt:get_qualified_locale.obj
 0001:00011058       ??_C@_1BM@OJNDFNPD@?$AAs?$AAp?$AAa?$AAn?$AAi?$AAs?$AAh?$AA?9?$AAc?$AAh?$AAi?$AAl?$AAe@ 0000000180012058     libucrt:get_qualified_locale.obj
 0001:00011078       ??_C@_1CC@OCOLPALL@?$AAs?$AAp?$AAa?$AAn?$AAi?$AAs?$AAh?$AA?9?$AAc?$AAo?$AAl?$AAo?$AAm?$AAb?$AAi@ 0000000180012078     libucrt:get_qualified_locale.obj
 0001:000110a0       ??_C@_1CG@BPOFMKBB@?$AAs?$AAp?$AAa?$AAn?$AAi?$AAs?$AAh?$AA?9?$AAc?$AAo?$AAs?$AAt?$AAa?$AA?5?$AAr@ 00000001800120a0     libucrt:get_qualified_locale.obj
 0001:000110c8       ??_C@_1DG@IGOBAPBB@?$AAs?$AAp?$AAa?$AAn?$AAi?$AAs?$AAh?$AA?9?$AAd?$AAo?$AAm?$AAi?$AAn?$AAi?$AAc@ 00000001800120c8     libucrt:get_qualified_locale.obj
 0001:00011100       ??_C@_1CA@JHAPGEGI@?$AAs?$AAp?$AAa?$AAn?$AAi?$AAs?$AAh?$AA?9?$AAe?$AAc?$AAu?$AAa?$AAd?$AAo?$AAr@ 0000000180012100     libucrt:get_qualified_locale.obj
 0001:00011120       ??_C@_1CI@LAPALJPP@?$AAs?$AAp?$AAa?$AAn?$AAi?$AAs?$AAh?$AA?9?$AAe?$AAl?$AA?5?$AAs?$AAa?$AAl?$AAv@ 0000000180012120     libucrt:get_qualified_locale.obj
 0001:00011148       ??_C@_1CE@PDGBOFOM@?$AAs?$AAp?$AAa?$AAn?$AAi?$AAs?$AAh?$AA?9?$AAg?$AAu?$AAa?$AAt?$AAe?$AAm?$AAa@ 0000000180012148     libucrt:get_qualified_locale.obj
 0001:00011170       ??_C@_1CC@NBEBAODI@?$AAs?$AAp?$AAa?$AAn?$AAi?$AAs?$AAh?$AA?9?$AAh?$AAo?$AAn?$AAd?$AAu?$AAr?$AAa@ 0000000180012170     libucrt:get_qualified_locale.obj
 0001:00011198       ??_C@_1CA@LLKGHBMF@?$AAs?$AAp?$AAa?$AAn?$AAi?$AAs?$AAh?$AA?9?$AAm?$AAe?$AAx?$AAi?$AAc?$AAa?$AAn@ 0000000180012198     libucrt:get_qualified_locale.obj
 0001:000111b8       ??_C@_1BO@LKNDOIGD@?$AAs?$AAp?$AAa?$AAn?$AAi?$AAs?$AAh?$AA?9?$AAm?$AAo?$AAd?$AAe?$AAr?$AAn@ 00000001800121b8     libucrt:get_qualified_locale.obj
 0001:000111d8       ??_C@_1CE@NMDMOEEB@?$AAs?$AAp?$AAa?$AAn?$AAi?$AAs?$AAh?$AA?9?$AAn?$AAi?$AAc?$AAa?$AAr?$AAa?$AAg@ 00000001800121d8     libucrt:get_qualified_locale.obj
 0001:00011200       ??_C@_1BO@LLCBEJGB@?$AAs?$AAp?$AAa?$AAn?$AAi?$AAs?$AAh?$AA?9?$AAp?$AAa?$AAn?$AAa?$AAm?$AAa@ 0000000180012200     libucrt:get_qualified_locale.obj
 0001:00011220       ??_C@_1CC@FKPGGIHO@?$AAs?$AAp?$AAa?$AAn?$AAi?$AAs?$AAh?$AA?9?$AAp?$AAa?$AAr?$AAa?$AAg?$AAu?$AAa@ 0000000180012220     libucrt:get_qualified_locale.obj
 0001:00011248       ??_C@_1BK@CDEIHOOP@?$AAs?$AAp?$AAa?$AAn?$AAi?$AAs?$AAh?$AA?9?$AAp?$AAe?$AAr?$AAu@ 0000000180012248     libucrt:get_qualified_locale.obj
 0001:00011268       ??_C@_1CI@GAHAKKGP@?$AAs?$AAp?$AAa?$AAn?$AAi?$AAs?$AAh?$AA?9?$AAp?$AAu?$AAe?$AAr?$AAt?$AAo?$AA?5@ 0000000180012268     libucrt:get_qualified_locale.obj
 0001:00011290       ??_C@_1CA@NKJBCAGP@?$AAs?$AAp?$AAa?$AAn?$AAi?$AAs?$AAh?$AA?9?$AAu?$AAr?$AAu?$AAg?$AAu?$AAa?$AAy@ 0000000180012290     libucrt:get_qualified_locale.obj
 0001:000112b0       ??_C@_1CE@ODILCONM@?$AAs?$AAp?$AAa?$AAn?$AAi?$AAs?$AAh?$AA?9?$AAv?$AAe?$AAn?$AAe?$AAz?$AAu?$AAe@ 00000001800122b0     libucrt:get_qualified_locale.obj
 0001:000112d8       ??_C@_1CA@OBNMCGFO@?$AAs?$AAw?$AAe?$AAd?$AAi?$AAs?$AAh?$AA?9?$AAf?$AAi?$AAn?$AAl?$AAa?$AAn?$AAd@ 00000001800122d8     libucrt:get_qualified_locale.obj
 0001:000112f8       ??_C@_1M@PIPDDPPI@?$AAs?$AAw?$AAi?$AAs?$AAs@ 00000001800122f8     libucrt:get_qualified_locale.obj
 0001:00011304       ??_C@_15GMFIMNFM@?$AAu?$AAs@ 0000000180012304     libucrt:get_qualified_locale.obj
 0001:00011310       ??_C@_17HAEBFAGL@?$AAu?$AAs?$AAa@ 0000000180012310     libucrt:get_qualified_locale.obj
 0001:00011318       ??_C@_1BA@DPFJEPHB@?$AAa?$AAm?$AAe?$AAr?$AAi?$AAc?$AAa@ 0000000180012318     libucrt:get_qualified_locale.obj
 0001:00011328       ??_C@_1BA@ELOGGFK@?$AAb?$AAr?$AAi?$AAt?$AAa?$AAi?$AAn@ 0000000180012328     libucrt:get_qualified_locale.obj
 0001:00011338       ??_C@_1M@GHBGIGDA@?$AAc?$AAh?$AAi?$AAn?$AAa@ 0000000180012338     libucrt:get_qualified_locale.obj
 0001:00011348       ??_C@_1M@NCHEJOPO@?$AAc?$AAz?$AAe?$AAc?$AAh@ 0000000180012348     libucrt:get_qualified_locale.obj
 0001:00011358       ??_C@_1BA@BKPAPBLA@?$AAe?$AAn?$AAg?$AAl?$AAa?$AAn?$AAd@ 0000000180012358     libucrt:get_qualified_locale.obj
 0001:00011368       ??_C@_1BM@HKBCKIPC@?$AAg?$AAr?$AAe?$AAa?$AAt?$AA?5?$AAb?$AAr?$AAi?$AAt?$AAa?$AAi?$AAn@ 0000000180012368     libucrt:get_qualified_locale.obj
 0001:00011388       ??_C@_1BA@PPCHPGJB@?$AAh?$AAo?$AAl?$AAl?$AAa?$AAn?$AAd@ 0000000180012388     libucrt:get_qualified_locale.obj
 0001:00011398       ??_C@_1BE@JBMPEGDG@?$AAh?$AAo?$AAn?$AAg?$AA?9?$AAk?$AAo?$AAn?$AAg@ 0000000180012398     libucrt:get_qualified_locale.obj
 0001:000113b0       ??_C@_1BI@KOELBBPJ@?$AAn?$AAe?$AAw?$AA?9?$AAz?$AAe?$AAa?$AAl?$AAa?$AAn?$AAd@ 00000001800123b0     libucrt:get_qualified_locale.obj
 0001:000113c8       ??_C@_15HIEBHAIO@?$AAn?$AAz@ 00000001800123c8     libucrt:get_qualified_locale.obj
 0001:000113d0       ??_C@_1BC@CHBCPFPI@?$AAp?$AAr?$AA?5?$AAc?$AAh?$AAi?$AAn?$AAa@ 00000001800123d0     libucrt:get_qualified_locale.obj
 0001:000113e8       ??_C@_1BC@JAOIIFKD@?$AAp?$AAr?$AA?9?$AAc?$AAh?$AAi?$AAn?$AAa@ 00000001800123e8     libucrt:get_qualified_locale.obj
 0001:00011400       ??_C@_1BI@BEHPPHKC@?$AAp?$AAu?$AAe?$AAr?$AAt?$AAo?$AA?9?$AAr?$AAi?$AAc?$AAo@ 0000000180012400     libucrt:get_qualified_locale.obj
 0001:00011418       ??_C@_1O@PAEOFKDI@?$AAs?$AAl?$AAo?$AAv?$AAa?$AAk@ 0000000180012418     libucrt:get_qualified_locale.obj
 0001:00011428       ??_C@_1BK@FIHMCKAM@?$AAs?$AAo?$AAu?$AAt?$AAh?$AA?5?$AAa?$AAf?$AAr?$AAi?$AAc?$AAa@ 0000000180012428     libucrt:get_qualified_locale.obj
 0001:00011448       ??_C@_1BI@NAEOODKB@?$AAs?$AAo?$AAu?$AAt?$AAh?$AA?5?$AAk?$AAo?$AAr?$AAe?$AAa@ 0000000180012448     libucrt:get_qualified_locale.obj
 0001:00011460       ??_C@_1BK@FBDGGIFF@?$AAs?$AAo?$AAu?$AAt?$AAh?$AA?9?$AAa?$AAf?$AAr?$AAi?$AAc?$AAa@ 0000000180012460     libucrt:get_qualified_locale.obj
 0001:00011480       ??_C@_1BI@GHLEJDPK@?$AAs?$AAo?$AAu?$AAt?$AAh?$AA?9?$AAk?$AAo?$AAr?$AAe?$AAa@ 0000000180012480     libucrt:get_qualified_locale.obj
 0001:00011498       ??_C@_1CE@PLHLOMJF@?$AAt?$AAr?$AAi?$AAn?$AAi?$AAd?$AAa?$AAd?$AA?5?$AA?$CG?$AA?5?$AAt?$AAo?$AAb?$AAa@ 0000000180012498     libucrt:get_qualified_locale.obj
 0001:000114c0       ??_C@_1BO@MODIMHHI@?$AAu?$AAn?$AAi?$AAt?$AAe?$AAd?$AA?9?$AAk?$AAi?$AAn?$AAg?$AAd?$AAo?$AAm@ 00000001800124c0     libucrt:get_qualified_locale.obj
 0001:000114e0       ??_C@_1BM@FFHJONBJ@?$AAu?$AAn?$AAi?$AAt?$AAe?$AAd?$AA?9?$AAs?$AAt?$AAa?$AAt?$AAe?$AAs@ 00000001800124e0     libucrt:get_qualified_locale.obj
 0001:00011500       ??_C@_19MPDNHKDG@?$AAu?$AAt?$AAf?$AA8@ 0000000180012500     libucrt:get_qualified_locale.obj
 0001:00011510       ??_C@_17DNCLJFIF@?$AAA?$AAC?$AAP@ 0000000180012510     libucrt:get_qualified_locale.obj
 0001:00011518       ??_C@_1M@FPEIIFAM@?$AAu?$AAt?$AAf?$AA?9?$AA8@ 0000000180012518     libucrt:get_qualified_locale.obj
 0001:00011528       ??_C@_17CIKBIHLH@?$AAO?$AAC?$AAP@ 0000000180012528     libucrt:get_qualified_locale.obj
 0001:00011530       __rglangidNotDefault       0000000180012530     libucrt:getqloc_downlevel.obj
 0001:00011560       ??_C@_1BA@BALFACEM@?$AAC?$AAO?$AAN?$AAO?$AAU?$AAT?$AA$@ 0000000180012560     libucrt:initcon.obj
 0001:00011590       _load_config_used          0000000180012590     LIBCMT:loadcfg.obj
 0001:00011698       ??_R4exception@std@@6B@    0000000180012698     libcpmt:xthrow.obj
 0001:000116c0       ??_R3exception@std@@8      00000001800126c0     libcpmt:xthrow.obj
 0001:000116d8       ??_R2exception@std@@8      00000001800126d8     libcpmt:xthrow.obj
 0001:000116e8       ??_R1A@?0A@EA@exception@std@@8 00000001800126e8     libcpmt:xthrow.obj
 0001:00011710       ??_R4bad_alloc@std@@6B@    0000000180012710     libcpmt:xthrow.obj
 0001:00011738       ??_R3bad_alloc@std@@8      0000000180012738     libcpmt:xthrow.obj
 0001:00011750       ??_R2bad_alloc@std@@8      0000000180012750     libcpmt:xthrow.obj
 0001:00011768       ??_R1A@?0A@EA@bad_alloc@std@@8 0000000180012768     libcpmt:xthrow.obj
 0001:00011790       ??_R4logic_error@std@@6B@  0000000180012790     libcpmt:xthrow.obj
 0001:000117b8       ??_R3logic_error@std@@8    00000001800127b8     libcpmt:xthrow.obj
 0001:000117d0       ??_R2logic_error@std@@8    00000001800127d0     libcpmt:xthrow.obj
 0001:000117e8       ??_R1A@?0A@EA@logic_error@std@@8 00000001800127e8     libcpmt:xthrow.obj
 0001:00011810       ??_R4length_error@std@@6B@ 0000000180012810     libcpmt:xthrow.obj
 0001:00011838       ??_R3length_error@std@@8   0000000180012838     libcpmt:xthrow.obj
 0001:00011850       ??_R2length_error@std@@8   0000000180012850     libcpmt:xthrow.obj
 0001:00011870       ??_R1A@?0A@EA@length_error@std@@8 0000000180012870     libcpmt:xthrow.obj
 0001:00011898       ??_R4out_of_range@std@@6B@ 0000000180012898     libcpmt:xthrow.obj
 0001:000118c0       ??_R3out_of_range@std@@8   00000001800128c0     libcpmt:xthrow.obj
 0001:000118d8       ??_R2out_of_range@std@@8   00000001800128d8     libcpmt:xthrow.obj
 0001:000118f8       ??_R1A@?0A@EA@out_of_range@std@@8 00000001800128f8     libcpmt:xthrow.obj
 0001:00011920       ??_R4runtime_error@std@@6B@ 0000000180012920     libcpmt:xthrow.obj
 0001:00011948       ??_R3runtime_error@std@@8  0000000180012948     libcpmt:xthrow.obj
 0001:00011960       ??_R2runtime_error@std@@8  0000000180012960     libcpmt:xthrow.obj
 0001:00011978       ??_R1A@?0A@EA@runtime_error@std@@8 0000000180012978     libcpmt:xthrow.obj
 0001:000119a0       ??_R4bad_function_call@std@@6B@ 00000001800129a0     libcpmt:xthrow.obj
 0001:000119c8       ??_R3bad_function_call@std@@8 00000001800129c8     libcpmt:xthrow.obj
 0001:000119e0       ??_R2bad_function_call@std@@8 00000001800129e0     libcpmt:xthrow.obj
 0001:000119f8       ??_R1A@?0A@EA@bad_function_call@std@@8 00000001800129f8     libcpmt:xthrow.obj
 0001:00011a20       ??_R4_Facet_base@std@@6B@  0000000180012a20     libcpmt:locale0.obj
 0001:00011a48       ??_R3_Facet_base@std@@8    0000000180012a48     libcpmt:locale0.obj
 0001:00011a60       ??_R2_Facet_base@std@@8    0000000180012a60     libcpmt:locale0.obj
 0001:00011a70       ??_R1A@?0A@EA@_Facet_base@std@@8 0000000180012a70     libcpmt:locale0.obj
 0001:00011a98       ??_R4_Locimp@locale@std@@6B@ 0000000180012a98     libcpmt:locale0.obj
 0001:00011ac0       ??_R3_Locimp@locale@std@@8 0000000180012ac0     libcpmt:locale0.obj
 0001:00011ad8       ??_R2_Locimp@locale@std@@8 0000000180012ad8     libcpmt:locale0.obj
 0001:00011b00       ??_R1A@?0A@EA@_Locimp@locale@std@@8 0000000180012b00     libcpmt:locale0.obj
 0001:00011b28       ??_R1A@?0A@EA@facet@locale@std@@8 0000000180012b28     libcpmt:locale0.obj
 0001:00011b50       ??_R3facet@locale@std@@8   0000000180012b50     libcpmt:locale0.obj
 0001:00011b68       ??_R2facet@locale@std@@8   0000000180012b68     libcpmt:locale0.obj
 0001:00011b88       ??_R17?0A@EA@_Crt_new_delete@std@@8 0000000180012b88     libcpmt:locale0.obj
 0001:00011bb0       ??_R3_Crt_new_delete@std@@8 0000000180012bb0     libcpmt:locale0.obj
 0001:00011bc8       ??_R2_Crt_new_delete@std@@8 0000000180012bc8     libcpmt:locale0.obj
 0001:00011bd8       ??_R1A@?0A@EA@_Crt_new_delete@std@@8 0000000180012bd8     libcpmt:locale0.obj
 0001:00011c00       ??_R4bad_array_new_length@std@@6B@ 0000000180012c00     libcpmt:locale.obj
 0001:00011c28       ??_R3bad_array_new_length@std@@8 0000000180012c28     libcpmt:locale.obj
 0001:00011c40       ??_R2bad_array_new_length@std@@8 0000000180012c40     libcpmt:locale.obj
 0001:00011c60       ??_R1A@?0A@EA@bad_array_new_length@std@@8 0000000180012c60     libcpmt:locale.obj
 0001:00011c88       ??_R4bad_cast@std@@6B@     0000000180012c88     libcpmt:locale.obj
 0001:00011cb0       ??_R3bad_cast@std@@8       0000000180012cb0     libcpmt:locale.obj
 0001:00011cc8       ??_R2bad_cast@std@@8       0000000180012cc8     libcpmt:locale.obj
 0001:00011ce0       ??_R1A@?0A@EA@bad_cast@std@@8 0000000180012ce0     libcpmt:locale.obj
 0001:00011d08       ??_R4?$numpunct@_W@std@@6B@ 0000000180012d08     libcpmt:wlocale.obj
 0001:00011d30       ??_R3?$numpunct@_W@std@@8  0000000180012d30     libcpmt:wlocale.obj
 0001:00011d48       ??_R2?$numpunct@_W@std@@8  0000000180012d48     libcpmt:wlocale.obj
 0001:00011d70       ??_R1A@?0A@EA@?$numpunct@_W@std@@8 0000000180012d70     libcpmt:wlocale.obj
 0001:00011d98       ??_R4type_info@@6B@        0000000180012d98     LIBCMT:std_type_info_static.obj
 0001:00011dc0       ??_R3type_info@@8          0000000180012dc0     LIBCMT:std_type_info_static.obj
 0001:00011dd8       ??_R2type_info@@8          0000000180012dd8     LIBCMT:std_type_info_static.obj
 0001:00011de8       ??_R1A@?0A@EA@type_info@@8 0000000180012de8     LIBCMT:std_type_info_static.obj
 0001:00011e10       ??_R4bad_exception@std@@6B@ 0000000180012e10     libvcruntime:frame.obj
 0001:00011e38       ??_R3bad_exception@std@@8  0000000180012e38     libvcruntime:frame.obj
 0001:00011e50       ??_R2bad_exception@std@@8  0000000180012e50     libvcruntime:frame.obj
 0001:00011e68       ??_R1A@?0A@EA@bad_exception@std@@8 0000000180012e68     libvcruntime:frame.obj
 0001:000121b8       __rtc_iaa                  00000001800131b8     LIBCMT:initsect.obj
 0001:000121c0       __rtc_izz                  00000001800131c0     LIBCMT:initsect.obj
 0001:000121c8       __rtc_taa                  00000001800131c8     LIBCMT:initsect.obj
 0001:000121d0       __rtc_tzz                  00000001800131d0     LIBCMT:initsect.obj
 0001:00012280       _alloca_probe              0000000180013280 f   chkstk.obj
 0001:00012280       __chkstk                   0000000180013280 f   chkstk.obj
 0001:000122e0       ??$_Destroy_range@V?$allocator@Umode@@@std@@@std@@YAXPEAUmode@@QEAU1@AEAV?$allocator@Umode@@@0@@Z 00000001800132e0 f i fileio.obj
 0001:00012350       ??1?$basic_string@_WU?$char_traits@_W@std@@V?$allocator@_W@2@@std@@QEAA@XZ 0000000180013350 f i fileio.obj
 0001:00012350       ?_Tidy_deallocate@?$basic_string@_WU?$char_traits@_W@std@@V?$allocator@_W@2@@std@@AEAAXXZ 0000000180013350 f i fileio.obj
 0001:000123c0       ??1?$vector@Umode@@V?$allocator@Umode@@@std@@@std@@QEAA@XZ 00000001800133c0 f i fileio.obj
 0001:000124c0       ??1columns@@QEAA@XZ        00000001800134c0 f i fileio.obj
 0001:000124f0       ??1mode@@QEAA@XZ           00000001800134f0 f i fileio.obj
 0001:00012550       ?WriteToFile@@YA_KPEAXAEBV?$basic_string_view@_WU?$char_traits@_W@std@@@std@@@Z 0000000180013550 f   fileio.obj
 0001:00012590       ?WriteToFile@@YA_KPEAX_W@Z 0000000180013590 f   fileio.obj
 0001:000125d0       ?deallocate@?$allocator@_W@std@@QEAAXQEA_W_K@Z 00000001800135d0 f i fileio.obj
 0001:00012610       ??$format_float@N@detail@v6@fmt@@YAHNHUfloat_specs@012@AEAV?$buffer@D@012@@Z 0000000180013610 f i format.obj
 0001:00012ce0       ??$_Allocate@$0BA@U_Default_allocate_traits@std@@$0A@@std@@YAPEAX_K@Z 0000000180013ce0 f i format.obj
 0001:00012d40       ??$_Maklocstr@D@std@@YAPEADPEBDPEADAEBU_Cvtvec@@@Z 0000000180013d40 f i format.obj
 0001:00012db0       ??$decimal_point_impl@_W@detail@v6@fmt@@YA_WVlocale_ref@012@@Z 0000000180013db0 f i format.obj
 0001:00012e10       ??$do_throw@Vformat_error@v6@fmt@@@detail@v6@fmt@@YAXAEBVformat_error@12@@Z 0000000180013e10 f i format.obj
 0001:00012e40       ??$fallback_format@O@detail@v6@fmt@@YAXOAEAV?$buffer@D@012@AEAH@Z 0000000180013e40 f i format.obj
 0001:00012e40       ??$fallback_format@N@detail@v6@fmt@@YAXNAEAV?$buffer@D@012@AEAH@Z 0000000180013e40 f i format.obj
 0001:00013f40       ??$format_float@O@detail@v6@fmt@@YAHOHUfloat_specs@012@AEAV?$buffer@D@012@@Z 0000000180014f40 f i format.obj
 0001:00014610       ??$get@Vlocale@std@@@locale_ref@detail@v6@fmt@@QEBA?AVlocale@std@@XZ 0000000180015610 f i format.obj
 0001:000146f0       ??$grisu_gen_digits@Ufixed_handler@detail@v6@fmt@@@detail@v6@fmt@@YA?AW4result@digits@012@Vfp@012@_KAEAHAEAUfixed_handler@012@@Z 00000001800156f0 f i format.obj
 0001:00014b30       ??$grisu_gen_digits@Ugrisu_shortest_handler@detail@v6@fmt@@@detail@v6@fmt@@YA?AW4result@digits@012@Vfp@012@_KAEAHAEAUgrisu_shortest_handler@012@@Z 0000000180015b30 f i format.obj
 0001:00014ed0       ??$grouping_impl@_W@detail@v6@fmt@@YA?AV?$basic_string@DU?$char_traits@D@std@@V?$allocator@D@2@@std@@Vlocale_ref@012@@Z 0000000180015ed0 f i format.obj
 0001:00014f40       ??$snprintf_float@N@detail@v6@fmt@@YAHNHUfloat_specs@012@AEAV?$buffer@D@012@@Z 0000000180015f40 f i format.obj
 0001:000151c0       ??$snprintf_float@O@detail@v6@fmt@@YAHOHUfloat_specs@012@AEAV?$buffer@D@012@@Z 00000001800161c0 f i format.obj
 0001:00015440       ??$thousands_sep_impl@_W@detail@v6@fmt@@YA_WVlocale_ref@012@@Z 0000000180016440 f i format.obj
 0001:000154a0       ??$use_facet@V?$numpunct@_W@std@@@std@@YAAEBV?$numpunct@_W@0@AEBVlocale@0@@Z 00000001800164a0 f i format.obj
 0001:000155b0       ??0bad_alloc@std@@QEAA@AEBV01@@Z 00000001800165b0 f i format.obj
 0001:000155f0       ??0bad_array_new_length@std@@QEAA@AEBV01@@Z 00000001800165f0 f i format.obj
 0001:00015630       ??0bad_array_new_length@std@@QEAA@XZ 0000000180016630 f i format.obj
 0001:00015660       ??0bad_cast@std@@QEAA@AEBV01@@Z 0000000180016660 f i format.obj
 0001:000156a0       ??0bad_cast@std@@QEAA@XZ   00000001800166a0 f i format.obj
 0001:000156d0       ??0exception@std@@QEAA@AEBV01@@Z 00000001800166d0 f i format.obj
 0001:00015710       ??0format_error@v6@fmt@@QEAA@AEBV012@@Z 0000000180016710 f i format.obj
 0001:00015750       ??0runtime_error@std@@QEAA@AEBV01@@Z 0000000180016750 f i format.obj
 0001:00015790       ??0runtime_error@std@@QEAA@PEBD@Z 0000000180016790 f i format.obj
 0001:000157e0       ??1?$_Tidy_guard@V?$numpunct@_W@std@@@std@@QEAA@XZ 00000001800167e0 f i format.obj
 0001:00015820       ??1?$_Yarn@D@std@@QEAA@XZ  0000000180016820 f i format.obj
 0001:00015820       ??1?$_Yarn@_W@std@@QEAA@XZ 0000000180016820 f i format.obj
 0001:00015850       ??1?$basic_memory_buffer@D$0BPE@V?$allocator@D@std@@@v6@fmt@@UEAA@XZ 0000000180016850 f i format.obj
 0001:000158b0       ??1?$basic_memory_buffer@I$0CA@V?$allocator@I@std@@@v6@fmt@@UEAA@XZ 00000001800168b0 f i format.obj
 0001:000158b0       ??1bigint@detail@v6@fmt@@QEAA@XZ 00000001800168b0 f i format.obj
 0001:00015910       ??1?$basic_memory_buffer@_W$0BPE@V?$allocator@_W@std@@@v6@fmt@@UEAA@XZ 0000000180016910 f i format.obj
 0001:00015970       ??1?$basic_string@DU?$char_traits@D@std@@V?$allocator@D@2@@std@@QEAA@XZ 0000000180016970 f i format.obj
 0001:000159d0       ??1?$unique_ptr@V_Facet_base@std@@U?$default_delete@V_Facet_base@std@@@2@@std@@QEAA@XZ 00000001800169d0 f i format.obj
 0001:000159f0       ??1_Locinfo@std@@QEAA@XZ   00000001800169f0 f i format.obj
 0001:00015a90       ??1bad_function_call@std@@UEAA@XZ 0000000180016a90 f i libcpmt:xthrow.obj
 0001:00015a90       ??1bad_cast@std@@UEAA@XZ   0000000180016a90 f i format.obj
 0001:00015a90       ??1format_error@v6@fmt@@UEAA@XZ 0000000180016a90 f i format.obj
 0001:00015a90       ??1bad_exception@std@@UEAA@XZ 0000000180016a90 f i libvcruntime:frame.obj
 0001:00015a90       ??1out_of_range@std@@UEAA@XZ 0000000180016a90 f i libcpmt:xthrow.obj
 0001:00015a90       ??1bad_alloc@std@@UEAA@XZ  0000000180016a90 f i format.obj
 0001:00015a90       ??1runtime_error@std@@UEAA@XZ 0000000180016a90 f i format.obj
 0001:00015a90       ??1length_error@std@@UEAA@XZ 0000000180016a90 f i libcpmt:xthrow.obj
 0001:00015a90       ??1bad_array_new_length@std@@UEAA@XZ 0000000180016a90 f i format.obj
 0001:00015ab0       ??1facet@locale@std@@MEAA@XZ 0000000180016ab0 f i format.obj
 0001:00015ac0       ??1locale@std@@QEAA@XZ     0000000180016ac0 f i format.obj
 0001:00015af0       ??_3bigint@detail@v6@fmt@@QEAAAEAV0123@H@Z 0000000180016af0 f i format.obj
 0001:00015bb0       ??_E?$basic_memory_buffer@D$0BPE@V?$allocator@D@std@@@v6@fmt@@UEAAPEAXI@Z 0000000180016bb0 f i format.obj
 0001:00015bb0       ??_G?$basic_memory_buffer@D$0BPE@V?$allocator@D@std@@@v6@fmt@@UEAAPEAXI@Z 0000000180016bb0 f i format.obj
 0001:00015c30       ??_E?$basic_memory_buffer@I$0CA@V?$allocator@I@std@@@v6@fmt@@UEAAPEAXI@Z 0000000180016c30 f i format.obj
 0001:00015c30       ??_G?$basic_memory_buffer@I$0CA@V?$allocator@I@std@@@v6@fmt@@UEAAPEAXI@Z 0000000180016c30 f i format.obj
 0001:00015cb0       ??_G?$basic_memory_buffer@_W$0BPE@V?$allocator@_W@std@@@v6@fmt@@UEAAPEAXI@Z 0000000180016cb0 f i format.obj
 0001:00015cb0       ??_E?$basic_memory_buffer@_W$0BPE@V?$allocator@_W@std@@@v6@fmt@@UEAAPEAXI@Z 0000000180016cb0 f i format.obj
 0001:00015d30       ??_G?$numpunct@_W@std@@MEAAPEAXI@Z 0000000180016d30 f i format.obj
 0001:00015d30       ??_E?$numpunct@_W@std@@MEAAPEAXI@Z 0000000180016d30 f i format.obj
 0001:00015d90       ??_E_Facet_base@std@@UEAAPEAXI@Z 0000000180016d90 f i format.obj
 0001:00015d90       ??_G_Facet_base@std@@UEAAPEAXI@Z 0000000180016d90 f i format.obj
 0001:00015dc0       ??_Gout_of_range@std@@UEAAPEAXI@Z 0000000180016dc0 f i libcpmt:xthrow.obj
 0001:00015dc0       ??_Elength_error@std@@UEAAPEAXI@Z 0000000180016dc0 f i libcpmt:xthrow.obj
 0001:00015dc0       ??_Ebad_function_call@std@@UEAAPEAXI@Z 0000000180016dc0 f i libcpmt:xthrow.obj
 0001:00015dc0       ??_Eformat_error@v6@fmt@@UEAAPEAXI@Z 0000000180016dc0 f i format.obj
 0001:00015dc0       ??_Gruntime_error@std@@UEAAPEAXI@Z 0000000180016dc0 f i format.obj
 0001:00015dc0       ??_Gexception@std@@UEAAPEAXI@Z 0000000180016dc0 f i format.obj
 0001:00015dc0       ??_Ebad_cast@std@@UEAAPEAXI@Z 0000000180016dc0 f i format.obj
 0001:00015dc0       ??_Gbad_array_new_length@std@@UEAAPEAXI@Z 0000000180016dc0 f i format.obj
 0001:00015dc0       ??_Glength_error@std@@UEAAPEAXI@Z 0000000180016dc0 f i libcpmt:xthrow.obj
 0001:00015dc0       ??_Gbad_function_call@std@@UEAAPEAXI@Z 0000000180016dc0 f i libcpmt:xthrow.obj
 0001:00015dc0       ??_Elogic_error@std@@UEAAPEAXI@Z 0000000180016dc0 f i libcpmt:xthrow.obj
 0001:00015dc0       ??_Ebad_exception@std@@UEAAPEAXI@Z 0000000180016dc0 f i libvcruntime:frame.obj
 0001:00015dc0       ??_Ebad_array_new_length@std@@UEAAPEAXI@Z 0000000180016dc0 f i format.obj
 0001:00015dc0       ??_Eexception@std@@UEAAPEAXI@Z 0000000180016dc0 f i format.obj
 0001:00015dc0       ??_Ebad_alloc@std@@UEAAPEAXI@Z 0000000180016dc0 f i format.obj
 0001:00015dc0       ??_Glogic_error@std@@UEAAPEAXI@Z 0000000180016dc0 f i libcpmt:xthrow.obj
 0001:00015dc0       ??_Gbad_exception@std@@UEAAPEAXI@Z 0000000180016dc0 f i libvcruntime:frame.obj
 0001:00015dc0       ??_Gformat_error@v6@fmt@@UEAAPEAXI@Z 0000000180016dc0 f i format.obj
 0001:00015dc0       ??_Eout_of_range@std@@UEAAPEAXI@Z 0000000180016dc0 f i libcpmt:xthrow.obj
 0001:00015dc0       ??_Eruntime_error@std@@UEAAPEAXI@Z 0000000180016dc0 f i format.obj
 0001:00015dc0       ??_Gbad_cast@std@@UEAAPEAXI@Z 0000000180016dc0 f i format.obj
 0001:00015dc0       ??_Gbad_alloc@std@@UEAAPEAXI@Z 0000000180016dc0 f i format.obj
 0001:00015e10       ?_Decref@facet@locale@std@@UEAAPEAV_Facet_base@3@XZ 0000000180016e10 f i format.obj
 0001:00015e20       ?_Getcat@?$numpunct@_W@std@@SA_KPEAPEBVfacet@locale@2@PEBV42@@Z 0000000180016e20 f i format.obj
 0001:00015fd0       ?_Incref@facet@locale@std@@UEAAXXZ 0000000180016fd0 f i format.obj
 0001:00015fe0       ?_Init@?$numpunct@_W@std@@IEAAXAEBV_Locinfo@2@_N@Z 0000000180016fe0 f i format.obj
 0001:00016280       ?_Throw_bad_array_new_length@std@@YAXXZ 0000000180017280 f i format.obj
 0001:00016280       ?__scrt_throw_std_bad_array_new_length@@YAXXZ 0000000180017280 f i LIBCMT:throw_bad_alloc.obj
 0001:000162a0       ?_Throw_bad_cast@std@@YAXXZ 00000001800172a0 f i format.obj
 0001:000162c0       ?_Xlen@?$basic_string@DU?$char_traits@D@std@@V?$allocator@D@2@@std@@CAXXZ 00000001800172c0 f i format.obj
 0001:000162c0       ?_Xlen@?$basic_string@_WU?$char_traits@_W@std@@V?$allocator@_W@2@@std@@CAXXZ 00000001800172c0 f i format.obj
 0001:000162e0       ?allocate@?$allocator@_W@std@@QEAAPEA_W_K@Z 00000001800172e0 f i format.obj
 0001:00016350       ?assign@?$basic_string@DU?$char_traits@D@std@@V?$allocator@D@2@@std@@QEAAAEAV12@QEBD_K@Z 0000000180017350 f i format.obj
 0001:000164b0       ?assign@?$basic_string@_WU?$char_traits@_W@std@@V?$allocator@_W@2@@std@@QEAAAEAV12@QEB_W_K@Z 00000001800174b0 f i format.obj
 0001:000165e0       ?assign_pow10@bigint@detail@v6@fmt@@QEAAXH@Z 00000001800175e0 f i format.obj
 0001:00016700       ?do_decimal_point@?$numpunct@_W@std@@MEBA_WXZ 0000000180017700 f i format.obj
 0001:00016710       ?do_falsename@?$numpunct@_W@std@@MEBA?AV?$basic_string@_WU?$char_traits@_W@std@@V?$allocator@_W@2@@2@XZ 0000000180017710 f i format.obj
 0001:00016750       ?do_grouping@?$numpunct@_W@std@@MEBA?AV?$basic_string@DU?$char_traits@D@std@@V?$allocator@D@2@@2@XZ 0000000180017750 f i format.obj
 0001:000167a0       ?do_thousands_sep@?$numpunct@_W@std@@MEBA_WXZ 00000001800177a0 f i format.obj
 0001:000167b0       ?do_truename@?$numpunct@_W@std@@MEBA?AV?$basic_string@_WU?$char_traits@_W@std@@V?$allocator@_W@2@@2@XZ 00000001800177b0 f i format.obj
 0001:000167f0       ?fmt_snprintf@detail@v6@fmt@@YAHPEAD_KPEBDZZ 00000001800177f0 f i format.obj
 0001:00016860       ?grisu_count_digits@detail@v6@fmt@@YAHI@Z 0000000180017860 f i format.obj
 0001:000168e0       ?grow@?$basic_memory_buffer@D$0BPE@V?$allocator@D@std@@@v6@fmt@@MEAAX_K@Z 00000001800178e0 f i format.obj
 0001:000169d0       ?grow@?$basic_memory_buffer@I$0CA@V?$allocator@I@std@@@v6@fmt@@MEAAX_K@Z 00000001800179d0 f i format.obj
 0001:00016af0       ?grow@?$basic_memory_buffer@_W$0BPE@V?$allocator@_W@std@@@v6@fmt@@MEAAX_K@Z 0000000180017af0 f i format.obj
 0001:00016c00       ?on_error@error_handler@detail@v6@fmt@@QEAAXPEBD@Z 0000000180017c00 f   format.obj
 0001:00016c70       ?resize@?$buffer@D@detail@v6@fmt@@QEAAX_K@Z 0000000180017c70 f i format.obj
 0001:00016cb0       ?square@bigint@detail@v6@fmt@@QEAAXXZ 0000000180017cb0 f i format.obj
 0001:00016f30       ?what@exception@std@@UEBAPEBDXZ 0000000180017f30 f i format.obj
 0001:00016f50       __local_stdio_printf_options 0000000180017f50 f i format.obj
 0001:00016f60       ??$?RH$0A@@?$arg_formatter_base@V?$back_insert_iterator@V?$buffer@_W@detail@v6@fmt@@@std@@_WUerror_handler@detail@v6@fmt@@@detail@v6@fmt@@QEAA?AV?$back_insert_iterator@V?$buffer@_W@detail@v6@fmt@@@std@@H@Z 0000000180017f60 f i handles.obj
 0001:00016fc0       ??$copy_str@_WPEBDPEA_W$0A@@detail@v6@fmt@@YAPEA_WPEBD0PEA_W@Z 0000000180017fc0 f i handles.obj
 0001:00017080       ??$fill@PEA_W_W@detail@v6@fmt@@YAPEA_WPEA_W_KAEBU?$fill_t@_W@012@@Z 0000000180018080 f i handles.obj
 0001:00017110       ??$format_decimal@_W_K@detail@v6@fmt@@YA?AU?$format_decimal_result@PEA_W@012@PEA_W_KH@Z 0000000180018110 f i handles.obj
 0001:000171d0       ??$get_dynamic_spec@Vprecision_checker@detail@v6@fmt@@V?$basic_format_arg@V?$basic_format_context@V?$back_insert_iterator@V?$buffer@_W@detail@v6@fmt@@@std@@_W@v6@fmt@@@34@Uerror_handler@234@@detail@v6@fmt@@YAHV?$basic_format_arg@V?$basic_format_context@V?$back_insert_iterator@V?$buffer@_W@detail@v6@fmt@@@std@@_W@v6@fmt@@@12@Uerror_handler@012@@Z 00000001800181d0 f i handles.obj
 0001:000172a0       ??$get_dynamic_spec@Vwidth_checker@detail@v6@fmt@@V?$basic_format_arg@V?$basic_format_context@V?$back_insert_iterator@V?$buffer@_W@detail@v6@fmt@@@std@@_W@v6@fmt@@@34@Uerror_handler@234@@detail@v6@fmt@@YAHV?$basic_format_arg@V?$basic_format_context@V?$back_insert_iterator@V?$buffer@_W@detail@v6@fmt@@@std@@_W@v6@fmt@@@12@Uerror_handler@012@@Z 00000001800182a0 f i handles.obj
 0001:00017370       ??$get_id@_W@?$basic_format_args@V?$basic_format_context@V?$back_insert_iterator@V?$buffer@_W@detail@v6@fmt@@@std@@_W@v6@fmt@@@v6@fmt@@QEBAHV?$basic_string_view@_W@12@@Z 0000000180018370 f i handles.obj
 0001:000174a0       ??$handle_int_type_spec@AEAU?$int_writer@V?$back_insert_iterator@V?$buffer@_W@detail@v6@fmt@@@std@@_WI@detail@v6@fmt@@@detail@v6@fmt@@YAXDAEAU?$int_writer@V?$back_insert_iterator@V?$buffer@_W@detail@v6@fmt@@@std@@_WI@012@@Z 00000001800184a0 f i handles.obj
 0001:000177c0       ??$handle_int_type_spec@AEAU?$int_writer@V?$back_insert_iterator@V?$buffer@_W@detail@v6@fmt@@@std@@_W_K@detail@v6@fmt@@@detail@v6@fmt@@YAXDAEAU?$int_writer@V?$back_insert_iterator@V?$buffer@_W@detail@v6@fmt@@@std@@_W_K@012@@Z 00000001800187c0 f i handles.obj
 0001:00017af0       ??$make_unique@$$BY0A@_W$0A@@std@@YA?AV?$unique_ptr@$$BY0A@_WU?$default_delete@$$BY0A@_W@std@@@0@_K@Z 0000000180018af0 f i handles.obj
 0001:00017b70       ??$parse_arg_id@_WAEAU?$id_adapter@AEAU?$format_handler@V?$arg_formatter@V?$back_insert_iterator@V?$buffer@_W@detail@v6@fmt@@@std@@_W@detail@v6@fmt@@_WV?$basic_format_context@V?$back_insert_iterator@V?$buffer@_W@detail@v6@fmt@@@std@@_W@34@@detail@v6@fmt@@_W@detail@v6@fmt@@@detail@v6@fmt@@YAPEB_WPEB_W0AEAU?$id_adapter@AEAU?$format_handler@V?$arg_formatter@V?$back_insert_iterator@V?$buffer@_W@detail@v6@fmt@@@std@@_W@detail@v6@fmt@@_WV?$basic_format_context@V?$back_insert_iterator@V?$buffer@_W@detail@v6@fmt@@@std@@_W@34@@detail@v6@fmt@@_W@012@@Z 0000000180018b70 f i handles.obj
 0001:00017d70       ??$parse_arg_id@_WU?$precision_adapter@AEAV?$specs_checker@V?$specs_handler@V?$basic_format_parse_context@_WUerror_handler@detail@v6@fmt@@@v6@fmt@@V?$basic_format_context@V?$back_insert_iterator@V?$buffer@_W@detail@v6@fmt@@@std@@_W@23@@detail@v6@fmt@@@detail@v6@fmt@@_W@detail@v6@fmt@@@detail@v6@fmt@@YAPEB_WPEB_W0$$QEAU?$precision_adapter@AEAV?$specs_checker@V?$specs_handler@V?$basic_format_parse_context@_WUerror_handler@detail@v6@fmt@@@v6@fmt@@V?$basic_format_context@V?$back_insert_iterator@V?$buffer@_W@detail@v6@fmt@@@std@@_W@23@@detail@v6@fmt@@@detail@v6@fmt@@_W@012@@Z 0000000180018d70 f i handles.obj
 0001:00018170       ??$parse_arg_id@_WU?$width_adapter@AEAV?$specs_checker@V?$specs_handler@V?$basic_format_parse_context@_WUerror_handler@detail@v6@fmt@@@v6@fmt@@V?$basic_format_context@V?$back_insert_iterator@V?$buffer@_W@detail@v6@fmt@@@std@@_W@23@@detail@v6@fmt@@@detail@v6@fmt@@_W@detail@v6@fmt@@@detail@v6@fmt@@YAPEB_WPEB_W0$$QEAU?$width_adapter@AEAV?$specs_checker@V?$specs_handler@V?$basic_format_parse_context@_WUerror_handler@detail@v6@fmt@@@v6@fmt@@V?$basic_format_context@V?$back_insert_iterator@V?$buffer@_W@detail@v6@fmt@@@std@@_W@23@@detail@v6@fmt@@@detail@v6@fmt@@_W@012@@Z 0000000180019170 f i handles.obj
 0001:00018570       ??$parse_float_type_spec@Uerror_handler@detail@v6@fmt@@_W@detail@v6@fmt@@YA?AUfloat_specs@012@AEBU?$basic_format_specs@_W@12@$$QEAUerror_handler@012@@Z 0000000180019570 f i handles.obj
 0001:00018700       ??$parse_format_specs@_WAEAV?$specs_checker@V?$specs_handler@V?$basic_format_parse_context@_WUerror_handler@detail@v6@fmt@@@v6@fmt@@V?$basic_format_context@V?$back_insert_iterator@V?$buffer@_W@detail@v6@fmt@@@std@@_W@23@@detail@v6@fmt@@@detail@v6@fmt@@@detail@v6@fmt@@YAPEB_WPEB_W0AEAV?$specs_checker@V?$specs_handler@V?$basic_format_parse_context@_WUerror_handler@detail@v6@fmt@@@v6@fmt@@V?$basic_format_context@V?$back_insert_iterator@V?$buffer@_W@detail@v6@fmt@@@std@@_W@23@@detail@v6@fmt@@@012@@Z 0000000180019700 f i handles.obj
 0001:00018ac0       ??$parse_format_string@$0A@_WAEAU?$format_handler@V?$arg_formatter@V?$back_insert_iterator@V?$buffer@_W@detail@v6@fmt@@@std@@_W@detail@v6@fmt@@_WV?$basic_format_context@V?$back_insert_iterator@V?$buffer@_W@detail@v6@fmt@@@std@@_W@34@@detail@v6@fmt@@@detail@v6@fmt@@YAXV?$basic_string_view@_W@12@AEAU?$format_handler@V?$arg_formatter@V?$back_insert_iterator@V?$buffer@_W@detail@v6@fmt@@@std@@_W@detail@v6@fmt@@_WV?$basic_format_context@V?$back_insert_iterator@V?$buffer@_W@detail@v6@fmt@@@std@@_W@34@@012@@Z 0000000180019ac0 f i handles.obj
 0001:00018eb0       ??$prettify@PEA_W@?$float_writer@_W@detail@v6@fmt@@AEBAPEA_WPEA_W@Z 0000000180019eb0 f i handles.obj
 0001:000191e0       ??$reserve@V?$buffer@_W@detail@v6@fmt@@$0A@@detail@v6@fmt@@YAPEA_WV?$back_insert_iterator@V?$buffer@_W@detail@v6@fmt@@@std@@_K@Z 000000018001a1e0 f i handles.obj
 0001:00019230       ??$vformat@_W$0A@@detail@v6@fmt@@YA?AV?$basic_string@_WU?$char_traits@_W@std@@V?$allocator@_W@2@@std@@V?$basic_string_view@_W@12@V?$basic_format_args@V?$basic_format_context@V?$back_insert_iterator@V?$buffer@_W@detail@v6@fmt@@@std@@_W@v6@fmt@@@12@@Z 000000018001a230 f i handles.obj
 0001:00019410       ??$visit_format_arg@U?$default_arg_formatter@V?$back_insert_iterator@V?$buffer@_W@detail@v6@fmt@@@std@@_W@detail@v6@fmt@@V?$basic_format_context@V?$back_insert_iterator@V?$buffer@_W@detail@v6@fmt@@@std@@_W@34@@v6@fmt@@YA?AV?$back_insert_iterator@V?$buffer@_W@detail@v6@fmt@@@std@@$$QEAU?$default_arg_formatter@V?$back_insert_iterator@V?$buffer@_W@detail@v6@fmt@@@std@@_W@detail@01@AEBV?$basic_format_arg@V?$basic_format_context@V?$back_insert_iterator@V?$buffer@_W@detail@v6@fmt@@@std@@_W@v6@fmt@@@01@@Z 000000018001a410 f i handles.obj
 0001:000196e0       ??$visit_format_arg@V?$arg_formatter@V?$back_insert_iterator@V?$buffer@_W@detail@v6@fmt@@@std@@_W@detail@v6@fmt@@V?$basic_format_context@V?$back_insert_iterator@V?$buffer@_W@detail@v6@fmt@@@std@@_W@34@@v6@fmt@@YA?AV?$back_insert_iterator@V?$buffer@_W@detail@v6@fmt@@@std@@$$QEAV?$arg_formatter@V?$back_insert_iterator@V?$buffer@_W@detail@v6@fmt@@@std@@_W@detail@01@AEBV?$basic_format_arg@V?$basic_format_context@V?$back_insert_iterator@V?$buffer@_W@detail@v6@fmt@@@std@@_W@v6@fmt@@@01@@Z 000000018001a6e0 f i handles.obj
 0001:00019e60       ??$write@_WV?$back_insert_iterator@V?$buffer@_W@detail@v6@fmt@@@std@@@detail@v6@fmt@@YA?AV?$back_insert_iterator@V?$buffer@_W@detail@v6@fmt@@@std@@V34@_N@Z 000000018001ae60 f i handles.obj
 0001:00019f00       ??$write@_WV?$back_insert_iterator@V?$buffer@_W@detail@v6@fmt@@@std@@@detail@v6@fmt@@YA?AV?$back_insert_iterator@V?$buffer@_W@detail@v6@fmt@@@std@@V34@_W@Z 000000018001af00 f i handles.obj
 0001:00019f70       ??$write@_WV?$back_insert_iterator@V?$buffer@_W@detail@v6@fmt@@@std@@H$0A@@detail@v6@fmt@@YA?AV?$back_insert_iterator@V?$buffer@_W@detail@v6@fmt@@@std@@V34@H@Z 000000018001af70 f i handles.obj
 0001:0001a0b0       ??$write@_WV?$back_insert_iterator@V?$buffer@_W@detail@v6@fmt@@@std@@I$0A@@detail@v6@fmt@@YA?AV?$back_insert_iterator@V?$buffer@_W@detail@v6@fmt@@@std@@V34@I@Z 000000018001b0b0 f i handles.obj
 0001:0001a1c0       ??$write@_WV?$back_insert_iterator@V?$buffer@_W@detail@v6@fmt@@@std@@M$0A@@detail@v6@fmt@@YA?AV?$back_insert_iterator@V?$buffer@_W@detail@v6@fmt@@@std@@V34@M@Z 000000018001b1c0 f i handles.obj
 0001:0001a3c0       ??$write@_WV?$back_insert_iterator@V?$buffer@_W@detail@v6@fmt@@@std@@M$0A@@detail@v6@fmt@@YA?AV?$back_insert_iterator@V?$buffer@_W@detail@v6@fmt@@@std@@V34@MU?$basic_format_specs@_W@12@Vlocale_ref@012@@Z 000000018001b3c0 f i handles.obj
 0001:0001a750       ??$write@_WV?$back_insert_iterator@V?$buffer@_W@detail@v6@fmt@@@std@@N$0A@@detail@v6@fmt@@YA?AV?$back_insert_iterator@V?$buffer@_W@detail@v6@fmt@@@std@@V34@N@Z 000000018001b750 f i handles.obj
 0001:0001a950       ??$write@_WV?$back_insert_iterator@V?$buffer@_W@detail@v6@fmt@@@std@@N$0A@@detail@v6@fmt@@YA?AV?$back_insert_iterator@V?$buffer@_W@detail@v6@fmt@@@std@@V34@NU?$basic_format_specs@_W@12@Vlocale_ref@012@@Z 000000018001b950 f i handles.obj
 0001:0001acd0       ??$write@_WV?$back_insert_iterator@V?$buffer@_W@detail@v6@fmt@@@std@@O$0A@@detail@v6@fmt@@YA?AV?$back_insert_iterator@V?$buffer@_W@detail@v6@fmt@@@std@@V34@O@Z 000000018001bcd0 f i handles.obj
 0001:0001aed0       ??$write@_WV?$back_insert_iterator@V?$buffer@_W@detail@v6@fmt@@@std@@O$0A@@detail@v6@fmt@@YA?AV?$back_insert_iterator@V?$buffer@_W@detail@v6@fmt@@@std@@V34@OU?$basic_format_specs@_W@12@Vlocale_ref@012@@Z 000000018001bed0 f i handles.obj
 0001:0001b250       ??$write@_WV?$back_insert_iterator@V?$buffer@_W@detail@v6@fmt@@@std@@_J$0A@@detail@v6@fmt@@YA?AV?$back_insert_iterator@V?$buffer@_W@detail@v6@fmt@@@std@@V34@_J@Z 000000018001c250 f i handles.obj
 0001:0001b320       ??$write@_WV?$back_insert_iterator@V?$buffer@_W@detail@v6@fmt@@@std@@_K$0A@@detail@v6@fmt@@YA?AV?$back_insert_iterator@V?$buffer@_W@detail@v6@fmt@@@std@@V34@_K@Z 000000018001c320 f i handles.obj
 0001:0001b3d0       ??$write@_W_WV?$back_insert_iterator@V?$buffer@_W@detail@v6@fmt@@@std@@@detail@v6@fmt@@YA?AV?$back_insert_iterator@V?$buffer@_W@detail@v6@fmt@@@std@@V34@V?$basic_string_view@_W@12@AEBU?$basic_format_specs@_W@12@@Z 000000018001c3d0 f i handles.obj
 0001:0001b4f0       ??$write_bytes@_WV?$back_insert_iterator@V?$buffer@_W@detail@v6@fmt@@@std@@@detail@v6@fmt@@YA?AV?$back_insert_iterator@V?$buffer@_W@detail@v6@fmt@@@std@@V34@V?$basic_string_view@D@12@AEBU?$basic_format_specs@_W@12@@Z 000000018001c4f0 f i handles.obj
 0001:0001b5e0       ??$write_int@H@?$arg_formatter_base@V?$back_insert_iterator@V?$buffer@_W@detail@v6@fmt@@@std@@_WUerror_handler@detail@v6@fmt@@@detail@v6@fmt@@AEAAXHAEBU?$basic_format_specs@_W@23@@Z 000000018001c5e0 f i handles.obj
 0001:0001b670       ??$write_int@V?$back_insert_iterator@V?$buffer@_W@detail@v6@fmt@@@std@@_WV<lambda_0273f2d8c97c19346923ccbca9d35cd0>@@@detail@v6@fmt@@YA?AV?$back_insert_iterator@V?$buffer@_W@detail@v6@fmt@@@std@@V34@HV?$basic_string_view@D@12@AEBU?$basic_format_specs@_W@12@V<lambda_0273f2d8c97c19346923ccbca9d35cd0>@@@Z 000000018001c670 f i handles.obj
 0001:0001b820       ??$write_int@V?$back_insert_iterator@V?$buffer@_W@detail@v6@fmt@@@std@@_WV<lambda_1584a04d9a5f951756080462468a1c79>@@@detail@v6@fmt@@YA?AV?$back_insert_iterator@V?$buffer@_W@detail@v6@fmt@@@std@@V34@HV?$basic_string_view@D@12@AEBU?$basic_format_specs@_W@12@V<lambda_1584a04d9a5f951756080462468a1c79>@@@Z 000000018001c820 f i handles.obj
 0001:0001b9f0       ??$write_int@V?$back_insert_iterator@V?$buffer@_W@detail@v6@fmt@@@std@@_WV<lambda_46028ac11bf91aacf0795357afd8c72d>@@@detail@v6@fmt@@YA?AV?$back_insert_iterator@V?$buffer@_W@detail@v6@fmt@@@std@@V34@HV?$basic_string_view@D@12@AEBU?$basic_format_specs@_W@12@V<lambda_46028ac11bf91aacf0795357afd8c72d>@@@Z 000000018001c9f0 f i handles.obj
 0001:0001bbb0       ??$write_int@V?$back_insert_iterator@V?$buffer@_W@detail@v6@fmt@@@std@@_WV<lambda_766228445ed89183d7065b0051936627>@@@detail@v6@fmt@@YA?AV?$back_insert_iterator@V?$buffer@_W@detail@v6@fmt@@@std@@V34@HV?$basic_string_view@D@12@AEBU?$basic_format_specs@_W@12@V<lambda_766228445ed89183d7065b0051936627>@@@Z 000000018001cbb0 f i handles.obj
 0001:0001bd50       ??$write_int@V?$back_insert_iterator@V?$buffer@_W@detail@v6@fmt@@@std@@_WV<lambda_c4159916ea5054600e9c49615e89ce82>@@@detail@v6@fmt@@YA?AV?$back_insert_iterator@V?$buffer@_W@detail@v6@fmt@@@std@@V34@HV?$basic_string_view@D@12@AEBU?$basic_format_specs@_W@12@V<lambda_c4159916ea5054600e9c49615e89ce82>@@@Z 000000018001cd50 f i handles.obj
 0001:0001bf00       ??$write_int@V?$back_insert_iterator@V?$buffer@_W@detail@v6@fmt@@@std@@_WV<lambda_dbc99c5d30ad811266da5b27d7d4d7eb>@@@detail@v6@fmt@@YA?AV?$back_insert_iterator@V?$buffer@_W@detail@v6@fmt@@@std@@V34@HV?$basic_string_view@D@12@AEBU?$basic_format_specs@_W@12@V<lambda_dbc99c5d30ad811266da5b27d7d4d7eb>@@@Z 000000018001cf00 f i handles.obj
 0001:0001c0b0       ??$write_int@V?$back_insert_iterator@V?$buffer@_W@detail@v6@fmt@@@std@@_WV<lambda_ee8e8661040b0e68e19c307d8706693d>@@@detail@v6@fmt@@YA?AV?$back_insert_iterator@V?$buffer@_W@detail@v6@fmt@@@std@@V34@HV?$basic_string_view@D@12@AEBU?$basic_format_specs@_W@12@V<lambda_ee8e8661040b0e68e19c307d8706693d>@@@Z 000000018001d0b0 f i handles.obj
 0001:0001c250       ??$write_nonfinite@_WV?$back_insert_iterator@V?$buffer@_W@detail@v6@fmt@@@std@@@detail@v6@fmt@@YA?AV?$back_insert_iterator@V?$buffer@_W@detail@v6@fmt@@@std@@V34@_NAEBU?$basic_format_specs@_W@12@AEBUfloat_specs@012@@Z 000000018001d250 f i handles.obj
 0001:0001c530       ??$write_padded@$01V?$back_insert_iterator@V?$buffer@_W@detail@v6@fmt@@@std@@_WV?$float_writer@_W@detail@v6@fmt@@@detail@v6@fmt@@YA?AV?$back_insert_iterator@V?$buffer@_W@detail@v6@fmt@@@std@@V34@AEBU?$basic_format_specs@_W@12@_KAEBV?$float_writer@_W@012@@Z 000000018001d530 f i handles.obj
 0001:0001c630       ??$write_ptr@_WV?$back_insert_iterator@V?$buffer@_W@detail@v6@fmt@@@std@@_K@detail@v6@fmt@@YA?AV?$back_insert_iterator@V?$buffer@_W@detail@v6@fmt@@@std@@V34@_KPEBU?$basic_format_specs@_W@12@@Z 000000018001d630 f i handles.obj
 0001:0001c7e0       ??0?$basic_string@_WU?$char_traits@_W@std@@V?$allocator@_W@2@@std@@QEAA@AEBV01@@Z 000000018001d7e0 f i handles.obj
 0001:0001c880       ??0?$float_writer@_W@detail@v6@fmt@@QEAA@PEBDHHUfloat_specs@123@_W@Z 000000018001d880 f i handles.obj
 0001:0001cad0       ??1?$scoped_lock@VPerfThread@@@std@@QEAA@XZ 000000018001dad0 f i handles.obj
 0001:0001caf0       ??1?$unique_ptr@$$BY0A@_WU?$default_delete@$$BY0A@_W@std@@@std@@QEAA@XZ 000000018001daf0 f i handles.obj
 0001:0001caf0       ??1?$unique_ptr@$$BY0A@DU?$default_delete@$$BY0A@D@std@@@std@@QEAA@XZ 000000018001daf0 f i handles.obj
 0001:0001cb00       ??1?$unique_ptr@USYSTEM_HANDLE_INFORMATION@@Uvirtual_deleter@@@std@@QEAA@XZ 000000018001db00 f i handles.obj
 0001:0001cb20       ??1?$unique_ptr@XUfree_deleter@@@std@@QEAA@XZ 000000018001db20 f i handles.obj
 0001:0001cb20       ??1?$unique_ptr@UPluginPanelItem@@Ufree_deleter@@@std@@QEAA@XZ 000000018001db20 f i Pclass.obj
 0001:0001cb30       ??1?$unique_ptr@XUhandle_closer@@@std@@QEAA@XZ 000000018001db30 f i handles.obj
 0001:0001cb40       ??1?$unique_ptr@_WUlocal_deleter@@@std@@QEAA@XZ 000000018001db40 f i handles.obj
 0001:0001cb50       ??1DebugToken@@QEAA@XZ     000000018001db50 f i handles.obj
 0001:0001cd90       ??Rwriter@?1???$parse_format_string@$0A@_WAEAU?$format_handler@V?$arg_formatter@V?$back_insert_iterator@V?$buffer@_W@detail@v6@fmt@@@std@@_W@detail@v6@fmt@@_WV?$basic_format_context@V?$back_insert_iterator@V?$buffer@_W@detail@v6@fmt@@@std@@_W@34@@detail@v6@fmt@@@detail@v6@fmt@@YAXV?$basic_string_view@_W@23@AEAU?$format_handler@V?$arg_formatter@V?$back_insert_iterator@V?$buffer@_W@detail@v6@fmt@@@std@@_W@detail@v6@fmt@@_WV?$basic_format_context@V?$back_insert_iterator@V?$buffer@_W@detail@v6@fmt@@@std@@_W@34@@123@@Z@QEAAXPEB_W2@Z 000000018001dd90 f i handles.obj
 0001:0001d560       ?PrintHandleInfo@@YA_NKPEAX_NPEAVPerfThread@@@Z 000000018001e560 f   handles.obj
 0001:0001dbb0       ?append@?$basic_string@_WU?$char_traits@_W@std@@V?$allocator@_W@2@@std@@QEAAAEAV12@QEB_W_K@Z 000000018001ebb0 f i handles.obj
 0001:0001dd30       ?check_sign@?$numeric_specs_checker@V?$specs_handler@V?$basic_format_parse_context@_WUerror_handler@detail@v6@fmt@@@v6@fmt@@V?$basic_format_context@V?$back_insert_iterator@V?$buffer@_W@detail@v6@fmt@@@std@@_W@23@@detail@v6@fmt@@@detail@v6@fmt@@QEAAXXZ 000000018001ed30 f i handles.obj
 0001:0001ded0       ?on_char@char_spec_handler@?$arg_formatter_base@V?$back_insert_iterator@V?$buffer@_W@detail@v6@fmt@@@std@@_WUerror_handler@detail@v6@fmt@@@detail@v6@fmt@@QEAAXXZ 000000018001eed0 f i handles.obj
 0001:0001dfe0       ?on_dec@?$int_writer@V?$back_insert_iterator@V?$buffer@_W@detail@v6@fmt@@@std@@_WI@detail@v6@fmt@@QEAAXXZ 000000018001efe0 f i handles.obj
 0001:0001e0e0       ?on_dec@?$int_writer@V?$back_insert_iterator@V?$buffer@_W@detail@v6@fmt@@@std@@_W_K@detail@v6@fmt@@QEAAXXZ 000000018001f0e0 f i handles.obj
 0001:0001e180       ?on_fill@?$specs_setter@_W@detail@v6@fmt@@QEAAXV?$basic_string_view@_W@34@@Z 000000018001f180 f i handles.obj
 0001:0001e250       ?on_format_specs@?$format_handler@V?$arg_formatter@V?$back_insert_iterator@V?$buffer@_W@detail@v6@fmt@@@std@@_W@detail@v6@fmt@@_WV?$basic_format_context@V?$back_insert_iterator@V?$buffer@_W@detail@v6@fmt@@@std@@_W@34@@detail@v6@fmt@@QEAAPEB_WHPEB_W0@Z 000000018001f250 f i handles.obj
 0001:0001e470       ?on_num@?$int_writer@V?$back_insert_iterator@V?$buffer@_W@detail@v6@fmt@@@std@@_WI@detail@v6@fmt@@QEAAXXZ 000000018001f470 f i handles.obj
 0001:0001e810       ?on_num@?$int_writer@V?$back_insert_iterator@V?$buffer@_W@detail@v6@fmt@@@std@@_W_K@detail@v6@fmt@@QEAAXXZ 000000018001f810 f i handles.obj
 0001:0001ebb0       ?on_replacement_field@?$format_handler@V?$arg_formatter@V?$back_insert_iterator@V?$buffer@_W@detail@v6@fmt@@@std@@_W@detail@v6@fmt@@_WV?$basic_format_context@V?$back_insert_iterator@V?$buffer@_W@detail@v6@fmt@@@std@@_W@34@@detail@v6@fmt@@QEAAXHPEB_W@Z 000000018001fbb0 f i handles.obj
 0001:0001ec80       ?on_text@?$format_handler@V?$arg_formatter@V?$back_insert_iterator@V?$buffer@_W@detail@v6@fmt@@@std@@_W@detail@v6@fmt@@_WV?$basic_format_context@V?$back_insert_iterator@V?$buffer@_W@detail@v6@fmt@@@std@@_W@34@@detail@v6@fmt@@QEAAXPEB_W0@Z 000000018001fc80 f i handles.obj
 0001:0001edc0       ?write@?$arg_formatter_base@V?$back_insert_iterator@V?$buffer@_W@detail@v6@fmt@@@std@@_WUerror_handler@detail@v6@fmt@@@detail@v6@fmt@@IEAAXPEB_W@Z 000000018001fdc0 f i handles.obj
 0001:0001eef0       ?write@?$arg_formatter_base@V?$back_insert_iterator@V?$buffer@_W@detail@v6@fmt@@@std@@_WUerror_handler@detail@v6@fmt@@@detail@v6@fmt@@IEAAX_N@Z 000000018001fef0 f i handles.obj
 0001:0001f0b0       ??1PluginDialogBuilder@@QEAA@XZ 00000001800200b0 f i Pcfg.obj
 0001:0001f130       ??1PluginSettings@@QEAA@XZ 0000000180020130 f i Pcfg.obj
 0001:0001f150       ??_GPluginEditFieldBinding@@UEAAPEAXI@Z 0000000180020150 f i Pclass.obj
 0001:0001f150       ??_EPluginCheckBoxBinding@@UEAAPEAXI@Z 0000000180020150 f i Pcfg.obj
 0001:0001f150       ??_GPluginCheckBoxBinding@@UEAAPEAXI@Z 0000000180020150 f i Pcfg.obj
 0001:0001f150       ??_EPluginEditFieldBinding@@UEAAPEAXI@Z 0000000180020150 f i Pclass.obj
 0001:0001f180       ?AddButtons@PluginDialogBuilder@@QEAAXHPEBHHH@Z 0000000180020180 f i Pcfg.obj
 0001:0001f4b0       ?AddDialogItem@PluginDialogBuilder@@AEAAPEAUFarDialogItem@@W4FARDIALOGITEMTYPES@@PEB_W@Z 00000001800204b0 f i Pcfg.obj
 0001:0001f660       ?Config@@YAHXZ             0000000180020660 f   Pcfg.obj
 0001:00020cc0       ?ItemWidth@PluginDialogBuilder@@CA_JAEBUFarDialogItem@@@Z 0000000180021cc0 f i Pcfg.obj
 0001:00020d50       ?Read@options@@QEAAXXZ     0000000180021d50 f   Pcfg.obj
 0001:00021050       ?SaveValue@PluginCheckBoxBinding@@UEAAXPEBUFarDialogItem@@H@Z 0000000180022050 f i Pcfg.obj
 0001:000210b0       ?ShowDialogEx@PluginDialogBuilder@@QEAA_JXZ 00000001800220b0 f i Pcfg.obj
 0001:00021400       ?Write@options@@QEBAXXZ    0000000180022400 f   Pcfg.obj
 0001:00021680       ??$_Assign_range@PEBUmode@@@?$vector@Umode@@V?$allocator@Umode@@@std@@@std@@AEAAXPEBUmode@@0Uforward_iterator_tag@1@@Z 0000000180022680 f i Pclass.obj
 0001:00021840       ??$_Copy_unchecked@PEBUmode@@PEAU1@@std@@YAPEAUmode@@PEBU1@0PEAU1@@Z 0000000180022840 f i Pclass.obj
 0001:000218b0       ??$_Emplace_reallocate@V?$basic_string@_WU?$char_traits@_W@std@@V?$allocator@_W@2@@std@@@?$vector@V?$basic_string@_WU?$char_traits@_W@std@@V?$allocator@_W@2@@std@@V?$allocator@V?$basic_string@_WU?$char_traits@_W@std@@V?$allocator@_W@2@@std@@@2@@std@@QEAAPEAV?$basic_string@_WU?$char_traits@_W@std@@V?$allocator@_W@2@@1@QEAV21@$$QEAV21@@Z 00000001800228b0 f i Pclass.obj
 0001:00021b60       ??$_Reallocate_grow_by@V<lambda_51c4cb9729979bd953fe6d1bff5c73b0>@@_K_K_W@?$basic_string@_WU?$char_traits@_W@std@@V?$allocator@_W@2@@std@@AEAAAEAV01@_KV<lambda_51c4cb9729979bd953fe6d1bff5c73b0>@@_K2_W@Z 0000000180022b60 f i Pclass.obj
 0001:00021ce0       ??$_Reallocate_grow_by@V<lambda_967c2ed818824c5314a20ec3af46b793>@@_KPEB_W_K@?$basic_string@_WU?$char_traits@_W@std@@V?$allocator@_W@2@@std@@AEAAAEAV01@_KV<lambda_967c2ed818824c5314a20ec3af46b793>@@_KPEB_W2@Z 0000000180022ce0 f i Pclass.obj
 0001:00021e60       ??$_Resize_reallocate@U_Value_init_tag@std@@@?$vector@PEB_WV?$allocator@PEB_W@std@@@std@@AEAAX_KAEBU_Value_init_tag@1@@Z 0000000180022e60 f i Pclass.obj
 0001:00021fc0       ??$_Try_emplace@AEBK$$V@?$_Hash@V?$_Umap_traits@KPEAUHWND__@@V?$_Uhash_compare@KU?$hash@K@std@@U?$equal_to@K@2@@std@@V?$allocator@U?$pair@$$CBKPEAUHWND__@@@std@@@3@$0A@@std@@@std@@IEAA?AU?$pair@PEAU?$_List_node@U?$pair@$$CBKPEAUHWND__@@@std@@PEAX@std@@_N@1@AEBK@Z 0000000180022fc0 f i Pclass.obj
 0001:00022280       ??$fill@PEAV?$_List_unchecked_iterator@V?$_List_val@U?$_List_simple_types@U?$pair@$$CBKPEAUHWND__@@@std@@@std@@@std@@@std@@V12@@std@@YAXQEAV?$_List_unchecked_iterator@V?$_List_val@U?$_List_simple_types@U?$pair@$$CBKPEAUHWND__@@@std@@@std@@@std@@@0@0AEBV10@@Z 0000000180023280 f i Pclass.obj
 0001:00022310       ??0Plist@@QEAA@XZ          0000000180023310 f   Pclass.obj
 0001:000224d0       ??1?$_List_node_emplace_op2@V?$allocator@U?$_List_node@U?$pair@$$CBKPEAUHWND__@@@std@@PEAX@std@@@std@@@std@@QEAA@XZ 00000001800234d0 f i Pclass.obj
 0001:000224d0       ??1?$_Alloc_construct_ptr@V?$allocator@U?$_List_node@U?$pair@$$CBKPEAUHWND__@@@std@@PEAX@std@@@std@@@std@@QEAA@XZ 00000001800234d0 f i Pclass.obj
 0001:000224f0       ??1?$_Hash@V?$_Umap_traits@KPEAUHWND__@@V?$_Uhash_compare@KU?$hash@K@std@@U?$equal_to@K@2@@std@@V?$allocator@U?$pair@$$CBKPEAUHWND__@@@std@@@3@$0A@@std@@@std@@QEAA@XZ 00000001800234f0 f i Pclass.obj
 0001:000225a0       ??1?$_Hash_vec@V?$allocator@V?$_List_unchecked_iterator@V?$_List_val@U?$_List_simple_types@U?$pair@$$CBKPEAUHWND__@@@std@@@std@@@std@@@std@@@std@@@std@@QEAA@XZ 00000001800235a0 f i Pclass.obj
 0001:00022600       ??1?$_Uninitialized_backout_al@V?$allocator@Umode@@@std@@@std@@QEAA@XZ 0000000180023600 f i Pclass.obj
 0001:00022610       ??1?$list@U?$pair@$$CBKPEAUHWND__@@@std@@V?$allocator@U?$pair@$$CBKPEAUHWND__@@@std@@@2@@std@@QEAA@XZ 0000000180023610 f i Pclass.obj
 0001:00022670       ??1?$pair@KV?$basic_string@_WU?$char_traits@_W@std@@V?$allocator@_W@2@@std@@@std@@QEAA@XZ 0000000180023670 f i Pclass.obj
 0001:00022670       ??1?$pair@_JV?$basic_string@_WU?$char_traits@_W@std@@V?$allocator@_W@2@@std@@@std@@QEAA@XZ 0000000180023670 f i Pclass.obj
 0001:00022680       ??1?$unique_ptr@VPerfThread@@U?$default_delete@VPerfThread@@@std@@@std@@QEAA@XZ 0000000180023680 f i Pclass.obj
 0001:000226b0       ??1?$unique_ptr@VWMIConnection@@U?$default_delete@VWMIConnection@@@std@@@std@@QEAA@XZ 00000001800236b0 f i Pclass.obj
 0001:000226e0       ??1?$unordered_map@KPEAUHWND__@@U?$hash@K@std@@U?$equal_to@K@3@V?$allocator@U?$pair@$$CBKPEAUHWND__@@@std@@@3@@std@@QEAA@XZ 00000001800236e0 f i Pclass.obj
 0001:000226f0       ??1?$vector@UFarMenuItem@@V?$allocator@UFarMenuItem@@@std@@@std@@QEAA@XZ 00000001800236f0 f i Pclass.obj
 0001:00022700       ??1?$vector@V?$basic_string@_WU?$char_traits@_W@std@@V?$allocator@_W@2@@std@@V?$allocator@V?$basic_string@_WU?$char_traits@_W@std@@V?$allocator@_W@2@@std@@@2@@std@@QEAA@XZ 0000000180023700 f i Pclass.obj
 0001:00022710       ??1Plist@@QEAA@XZ          0000000180023710 f   Pclass.obj
 0001:000227c0       ??1ProcessData@@QEAA@XZ    00000001800237c0 f i Pclass.obj
 0001:000227e0       ??1StrTok@@QEAA@XZ         00000001800237e0 f i Pclass.obj
 0001:000227f0       ??4?$unique_ptr@VPerfThread@@U?$default_delete@VPerfThread@@@std@@@std@@QEAAAEAV01@$$QEAV01@@Z 00000001800237f0 f i Pclass.obj
 0001:00022850       ??4columns@@QEAAAEAU0@AEBU0@@Z 0000000180023850 f i Pclass.obj
 0001:000228d0       ?AddEditField@PluginDialogBuilder@@QEAAPEAUFarDialogItem@@PEA_WHHPEB_W_N@Z 00000001800238d0 f i Pclass.obj
 0001:000229e0       ?Compare@Plist@@QEBAHPEBUPluginPanelItem@@0I@Z 00000001800239e0 f   Pclass.obj
 0001:00022b50       ?Connect@Plist@@QEAA_NPEB_W00@Z 0000000180023b50 f   Pclass.obj
 0001:00022e20       ?ConnectWMI@Plist@@AEAA_NXZ 0000000180023e20 f   Pclass.obj
 0001:00022f20       ?DeleteFiles@Plist@@QEAAHPEAUPluginPanelItem@@_K1@Z 0000000180023f20 f   Pclass.obj
 0001:00023470       ?DumpNTCounters@@YAXPEAXAEAVPerfThread@@KK@Z 0000000180024470 f   Pclass.obj
 0001:00023ac0       ?DurationToText@@YA?AV?$basic_string@_WU?$char_traits@_W@std@@V?$allocator@_W@2@@std@@_K@Z 0000000180024ac0 f   Pclass.obj
 0001:00023c40       ?EnumWndProc@@YAHPEAUHWND__@@_J@Z 0000000180024c40 f   Pclass.obj
 0001:00023d60       ?FreeFindData@Plist@@SAXPEAUPluginPanelItem@@_K@Z 0000000180024d60 f   Pclass.obj
 0001:00023e60       ?GetFiles@Plist@@QEAAHPEAUPluginPanelItem@@_KHPEAPEB_W1AEAUoptions@@@Z 0000000180024e60 f   Pclass.obj
 0001:00025e50       ?GetFindData@Plist@@QEAAHAEAPEAUPluginPanelItem@@AEA_K_K@Z 0000000180026e50 f   Pclass.obj
 0001:00026c20       ?GetOpenPanelInfo@Plist@@QEAAXPEAUOpenPanelInfo@@@Z 0000000180027c20 f   Pclass.obj
 0001:00026f00       ?GetVersionInfo@Plist@@SA_NPEB_WAEAV?$unique_ptr@$$BY0A@DU?$default_delete@$$BY0A@D@std@@@std@@AEAPEB_W2@Z 0000000180027f00 f   Pclass.obj
 0001:000273c0       ?InitializePanelModes@Plist@@SAXXZ 00000001800283c0 f   Pclass.obj
 0001:00028920       ?PanelModes@Plist@@QEAAPEAUPanelMode@@AEA_K@Z 0000000180029920 f   Pclass.obj
 0001:00028b60       ?PrintOwnerInfo@Plist@@AEAAXPEAXK@Z 0000000180029b60 f   Pclass.obj
 0001:000291b0       ?PrintVersionInfo@Plist@@CAXPEAXPEB_W@Z 000000018002a1b0 f   Pclass.obj
 0001:00029560       ?ProcessEvent@Plist@@QEAAH_JPEAX@Z 000000018002a560 f   Pclass.obj
 0001:00029700       ?ProcessKey@Plist@@QEAAHPEBU_INPUT_RECORD@@@Z 000000018002a700 f   Pclass.obj
 0001:0002c6e0       ?Reread@Plist@@AEAAXXZ     000000018002d6e0 f   Pclass.obj
 0001:0002c790       ?SavePanelModes@Plist@@SAXXZ 000000018002d790 f   Pclass.obj
 0001:0002caf0       ?SaveValue@PluginEditFieldBinding@@UEAAXPEBUFarDialogItem@@H@Z 000000018002daf0 f i Pclass.obj
 0001:0002d330       ?WmiError@Plist@@AEBAXXZ   000000018002e330 f   Pclass.obj
 0001:0002d380       ?_Assign_grow@?$_Hash_vec@V?$allocator@V?$_List_unchecked_iterator@V?$_List_val@U?$_List_simple_types@U?$pair@$$CBKPEAUHWND__@@@std@@@std@@@std@@@std@@@std@@@std@@QEAAX_KV?$_List_unchecked_iterator@V?$_List_val@U?$_List_simple_types@U?$pair@$$CBKPEAUHWND__@@@std@@@std@@@std@@@2@@Z 000000018002e380 f i Pclass.obj
 0001:0002d4b0       ?_Clear_and_reserve_geometric@?$vector@Umode@@V?$allocator@Umode@@@std@@@std@@AEAAX_K@Z 000000018002e4b0 f i Pclass.obj
 0001:0002d630       ?_Destroy@?$vector@V?$basic_string@_WU?$char_traits@_W@std@@V?$allocator@_W@2@@std@@V?$allocator@V?$basic_string@_WU?$char_traits@_W@std@@V?$allocator@_W@2@@std@@@2@@std@@AEAAXPEAV?$basic_string@_WU?$char_traits@_W@std@@V?$allocator@_W@2@@2@0@Z 000000018002e630 f i Pclass.obj
 0001:0002d670       ?_Forced_rehash@?$_Hash@V?$_Umap_traits@KPEAUHWND__@@V?$_Uhash_compare@KU?$hash@K@std@@U?$equal_to@K@2@@std@@V?$allocator@U?$pair@$$CBKPEAUHWND__@@@std@@@3@$0A@@std@@@std@@IEAAX_K@Z 000000018002e670 f i Pclass.obj
 0001:0002d830       ?_Getal@?$vector@PEB_WV?$allocator@PEB_W@std@@@std@@AEAAAEAV?$allocator@PEB_W@2@XZ 000000018002e830 f i Pclass.obj
 0001:0002d830       ?_Getal@?$vector@PEAUHINSTANCE__@@V?$allocator@PEAUHINSTANCE__@@@std@@@std@@AEAAAEAV?$allocator@PEAUHINSTANCE__@@@2@XZ 000000018002e830 f i Plist.obj
 0001:0002d830       ?_Getal@?$vector@EV?$allocator@E@std@@@std@@AEAAAEAV?$allocator@E@2@XZ 000000018002e830 f i perfthread.obj
 0001:0002d840       ?_Tidy@?$vector@UFarMenuItem@@V?$allocator@UFarMenuItem@@@std@@@std@@AEAAXXZ 000000018002e840 f i Pclass.obj
 0001:0002d8c0       ?_Tidy@?$vector@V?$basic_string@_WU?$char_traits@_W@std@@V?$allocator@_W@2@@std@@V?$allocator@V?$basic_string@_WU?$char_traits@_W@std@@V?$allocator@_W@2@@std@@@2@@std@@AEAAXXZ 000000018002e8c0 f i Pclass.obj
 0001:0002d950       ?_Xlength@?$vector@Umode@@V?$allocator@Umode@@@std@@@std@@CAXXZ 000000018002e950 f i Pclass.obj
 0001:0002d950       ?_Xlength@?$vector@V?$basic_string@_WU?$char_traits@_W@std@@V?$allocator@_W@2@@std@@V?$allocator@V?$basic_string@_WU?$char_traits@_W@std@@V?$allocator@_W@2@@std@@@2@@std@@CAXXZ 000000018002e950 f i Pclass.obj
 0001:0002d950       ?_Xlength@?$vector@UProcessPerfData@@V?$allocator@UProcessPerfData@@@std@@@std@@CAXXZ 000000018002e950 f i perfthread.obj
 0001:0002d950       ?_Xlength@?$vector@PEAUHINSTANCE__@@V?$allocator@PEAUHINSTANCE__@@@std@@@std@@CAXXZ 000000018002e950 f i Plist.obj
 0001:0002d950       ?_Xlength@?$vector@PEB_WV?$allocator@PEB_W@std@@@std@@CAXXZ 000000018002e950 f i Pclass.obj
 0001:0002d950       ?_Xlength@?$vector@EV?$allocator@E@std@@@std@@CAXXZ 000000018002e950 f i perfthread.obj
 0001:0002d970       ?_Xran@?$_String_val@U?$_Simple_types@_W@std@@@std@@SAXXZ 000000018002e970 f i Pclass.obj
 0001:0002d990       ?append@?$basic_string@_WU?$char_traits@_W@std@@V?$allocator@_W@2@@std@@QEAAAEAV12@_K_W@Z 000000018002e990 f i Pclass.obj
 0001:0002db10       ?deallocate@?$allocator@PEB_W@std@@QEAAXQEAPEB_W_K@Z 000000018002eb10 f i Pclass.obj
 0001:0002db10       ?deallocate@?$allocator@PEAUHINSTANCE__@@@std@@QEAAXQEAPEAUHINSTANCE__@@_K@Z 000000018002eb10 f i Plist.obj
 0001:0002db60       ?deallocate@?$allocator@V?$basic_string@_WU?$char_traits@_W@std@@V?$allocator@_W@2@@std@@@std@@QEAAXQEAV?$basic_string@_WU?$char_traits@_W@std@@V?$allocator@_W@2@@2@_K@Z 000000018002eb60 f i Pclass.obj
 0001:0002de30       ?insert@?$basic_string@_WU?$char_traits@_W@std@@V?$allocator@_W@2@@std@@QEAAAEAV12@_KQEB_W0@Z 000000018002ee30 f i Pclass.obj
 0001:0002ecb0       ??$_Construct_n_copies_of_ty@U_Value_init_tag@std@@@?$vector@UProcessPerfData@@V?$allocator@UProcessPerfData@@@std@@@std@@AEAAX_KAEBU_Value_init_tag@1@@Z 000000018002fcb0 f i perfthread.obj
 0001:0002ee40       ??$_Resize_reallocate@U_Value_init_tag@std@@@?$vector@EV?$allocator@E@std@@@std@@AEAAX_KAEBU_Value_init_tag@1@@Z 000000018002fe40 f i perfthread.obj
 0001:0002ef70       ??0PerfThread@@QEAA@PEB_W00@Z 000000018002ff70 f   perfthread.obj
 0001:0002f900       ??1?$_Tidy_guard@V?$vector@UProcessPerfData@@V?$allocator@UProcessPerfData@@@std@@@std@@@std@@QEAA@XZ 0000000180030900 f i perfthread.obj
 0001:0002f910       ??1?$_Uninitialized_backout_al@V?$allocator@UProcessPerfData@@@std@@@std@@QEAA@XZ 0000000180030910 f i perfthread.obj
 0001:0002f980       ??1?$vector@EV?$allocator@E@std@@@std@@QEAA@XZ 0000000180030980 f i perfthread.obj
 0001:0002f9e0       ??1?$vector@UProcessPerfData@@V?$allocator@UProcessPerfData@@@std@@@std@@QEAA@XZ 00000001800309e0 f i perfthread.obj
 0001:0002f9f0       ??1?$vector@_WV?$allocator@_W@std@@@std@@QEAA@XZ 00000001800309f0 f i perfthread.obj
 0001:0002fa50       ??1PerfLib@@QEAA@XZ        0000000180030a50 f i perfthread.obj
 0001:0002fa60       ??1PerfThread@@QEAA@XZ     0000000180030a60 f   perfthread.obj
 0001:0002fb40       ??1RegKey@@QEAA@XZ         0000000180030b40 f i perfthread.obj
 0001:0002fb50       ??4ProcessPerfData@@QEAAAEAU0@AEBU0@@Z 0000000180030b50 f i perfthread.obj
 0001:0002fea0       ?GetProcessData@PerfThread@@QEAAPEAUProcessPerfData@@KK@Z 0000000180030ea0 f   perfthread.obj
 0001:0002ffc0       ?Refresh@PerfThread@@AEAAXXZ 0000000180030fc0 f   perfthread.obj
 0001:00031320       ?RefreshWMIData@PerfThread@@AEAAXXZ 0000000180032320 f   perfthread.obj
 0001:00031760       ?SyncReread@PerfThread@@QEAAXXZ 0000000180032760 f   perfthread.obj
 0001:000317a0       ?ThreadProc@PerfThread@@CAKPEAX@Z 00000001800327a0 f   perfthread.obj
 0001:000318a0       ?_Tidy@?$vector@UProcessPerfData@@V?$allocator@UProcessPerfData@@@std@@@std@@AEAAXXZ 00000001800328a0 f i perfthread.obj
 0001:00031990       ?deallocate@?$allocator@E@std@@QEAAXQEAE_K@Z 0000000180032990 f i perfthread.obj
 0001:000319d0       ?lock@PerfThread@@QEAAXXZ  00000001800329d0 f   perfthread.obj
 0001:000319f0       ?unlock@PerfThread@@QEAAXXZ 00000001800329f0 f   perfthread.obj
 0001:00031a00       ??$_Resize_reallocate@U_Value_init_tag@std@@@?$vector@PEAUHINSTANCE__@@V?$allocator@PEAUHINSTANCE__@@@std@@@std@@AEAAX_KAEBU_Value_init_tag@1@@Z 0000000180032a00 f i Plist.obj
 0001:00031c70       ??0?$basic_string@_WU?$char_traits@_W@std@@V?$allocator@_W@2@@std@@QEAA@_K_W@Z 0000000180032c70 f i Plist.obj
 0001:00031d50       ??0?$vector@UProcessPerfData@@V?$allocator@UProcessPerfData@@@std@@@std@@QEAA@AEBV01@@Z 0000000180032d50 f i Plist.obj
 0001:00032030       ??1?$function@$$A6AXAEBUtagVARIANT@@@Z@std@@QEAA@XZ 0000000180033030 f i WMI.obj
 0001:00032030       ??1?$function@$$A6A_NPEA_W_K@Z@std@@QEAA@XZ 0000000180033030 f i Plist.obj
 0001:00032060       ??1?$vector@PEAUHINSTANCE__@@V?$allocator@PEAUHINSTANCE__@@@std@@@std@@QEAA@XZ 0000000180033060 f i Plist.obj
 0001:00032160       ?CreateToken@DebugToken@@SA_NXZ 0000000180033160 f   Plist.obj
 0001:00032260       ?Enable@DebugToken@@QEAA_NXZ 0000000180033260 f   Plist.obj
 0001:00032340       ?GetList@@YA_NAEAPEAUPluginPanelItem@@AEA_KAEAVPerfThread@@@Z 0000000180033340 f   Plist.obj
 0001:00032700       ?GetOpenProcessData@?$ipc_functions@$0A@@@SAXPEAXPEAV?$basic_string@_WU?$char_traits@_W@std@@V?$allocator@_W@2@@std@@1111@Z 0000000180033700 f i Plist.obj
 0001:00032bd0       ?GetOpenProcessData@@YAXPEAXPEAV?$basic_string@_WU?$char_traits@_W@std@@V?$allocator@_W@2@@std@@1111@Z 0000000180033bd0 f   Plist.obj
 0001:00032be0       ?GetPData@@YA_NAEAUProcessData@@AEBUProcessPerfData@@@Z 0000000180033be0 f   Plist.obj
 0001:00032de0       ?KillProcess@@YA_NKPEAUHWND__@@@Z 0000000180033de0 f   Plist.obj
 0001:00032f90       ?OpenProcessForced@@YAPEAXPEAVDebugToken@@KKH@Z 0000000180033f90 f   Plist.obj
 0001:00033000       ?PrintModules@@YAXPEAXKAEAUoptions@@@Z 0000000180034000 f   Plist.obj
 0001:000335e0       ?PrintNTCurDirAndEnv@@YAXPEAX0H@Z 00000001800345e0 f   Plist.obj
 0001:000339e0       ?Revert@DebugToken@@QEAA_NXZ 00000001800349e0 f   Plist.obj
 0001:00033a50       ?_Move@?$_Func_impl_no_alloc@V<lambda_c6a5923e4ab0669d9f7c2a6c892502eb>@@_NPEA_W_K@std@@EEAAPEAV?$_Func_base@_NPEA_W_K@2@PEAX@Z 0000000180034a50 f i Plist.obj
 0001:00033a50       ?_Copy@?$_Func_impl_no_alloc@V<lambda_c6a5923e4ab0669d9f7c2a6c892502eb>@@_NPEA_W_K@std@@EEBAPEAV?$_Func_base@_NPEA_W_K@2@PEAX@Z 0000000180034a50 f i Plist.obj
 0001:00033a70       ?_Delete_this@?$_Func_impl_no_alloc@V<lambda_c6a5923e4ab0669d9f7c2a6c892502eb>@@_NPEA_W_K@std@@EEAAX_N@Z 0000000180034a70 f   Plist.obj
 0001:00033ab0       ?_Do_call@?$_Func_impl_no_alloc@V<lambda_c6a5923e4ab0669d9f7c2a6c892502eb>@@_NPEA_W_K@std@@EEAA_N$$QEAPEA_W$$QEA_K@Z 0000000180034ab0 f i Plist.obj
 0001:00033af0       ?_Get@?$_Func_impl_no_alloc@V<lambda_c6a5923e4ab0669d9f7c2a6c892502eb>@@_NPEA_W_K@std@@EEBAPEBXXZ 0000000180034af0 f   Plist.obj
 0001:00033b10       ?_Target_type@?$_Func_impl_no_alloc@V<lambda_c6a5923e4ab0669d9f7c2a6c892502eb>@@_NPEA_W_K@std@@EEBAAEBVtype_info@@XZ 0000000180034b10 f i Plist.obj
 0001:00033b20       ?allocate@?$allocator@PEAUHINSTANCE__@@@std@@QEAAPEAPEAUHINSTANCE__@@_K@Z 0000000180034b20 f i Plist.obj
 0001:00033ef0       ?read_string@?$ipc_functions@$0A@@@SA?AV?$basic_string@_WU?$char_traits@_W@std@@V?$allocator@_W@2@@std@@PEAXAEBUUNICODE_STRING_SAME@detail@@@Z 0000000180034ef0 f i Plist.obj
 0001:00033fe0       ?ConvertDate@@YAXAEBU_FILETIME@@PEA_W1@Z 0000000180034fe0 f   Pmix.obj
 0001:00034090       ?GetMsg@@YAPEB_WH@Z        0000000180035090 f   Pmix.obj
 0001:000340b0       ?WinError@@YAHPEB_W@Z      00000001800350b0 f   Pmix.obj
 0001:000344b0       ??0WMIConnection@@QEAA@XZ  00000001800354b0 f   WMI.obj
 0001:000344e0       ??1?$ptr_setter@V?$unique_ptr@UIWbemClassObject@@Ucom_closer@@@std@@@@QEAA@XZ 00000001800354e0 f i WMI.obj
 0001:00034510       ??1?$unique_ptr@UIWbemLocator@@Ucom_closer@@@std@@QEAA@XZ 0000000180035510 f i WMI.obj
 0001:00034510       ??1?$unique_ptr@UIWbemClassObject@@Ucom_closer@@@std@@QEAA@XZ 0000000180035510 f i WMI.obj
 0001:00034530       ??1WMIConnection@@QEAA@XZ  0000000180035530 f   WMI.obj
 0001:00034570       ??1bstr@@QEAA@XZ           0000000180035570 f i WMI.obj
 0001:00034580       ?Connect@WMIConnection@@QEAA_NPEB_W00@Z 0000000180035580 f   WMI.obj
 0001:00034800       ?Disconnect@WMIConnection@@QEAAXXZ 0000000180035800 f   WMI.obj
 0001:00034830       ?ExecMethod@WMIConnection@@AEAAHKPEB_W0K@Z 0000000180035830 f   WMI.obj
 0001:00034b50       ?GetProcessCommandLine@WMIConnection@@QEAA?AV?$basic_string@_WU?$char_traits@_W@std@@V?$allocator@_W@2@@std@@K@Z 0000000180035b50 f   WMI.obj
 0001:00034be0       ?GetProcessExecutablePath@WMIConnection@@QEAA?AV?$basic_string@_WU?$char_traits@_W@std@@V?$allocator@_W@2@@std@@K@Z 0000000180035be0 f   WMI.obj
 0001:00034c70       ?GetProcessOwner@WMIConnection@@QEAA?AV?$basic_string@_WU?$char_traits@_W@std@@V?$allocator@_W@2@@std@@KPEAV23@@Z 0000000180035c70 f   WMI.obj
 0001:00034e80       ?GetProcessPriority@WMIConnection@@QEAAKK@Z 0000000180035e80 f   WMI.obj
 0001:00034ef0       ?GetProcessProperty@WMIConnection@@AEAA_NKPEB_WAEBV?$function@$$A6AXAEBUtagVARIANT@@@Z@std@@@Z 0000000180035ef0 f   WMI.obj
 0001:00035020       ?GetProcessSessionId@WMIConnection@@QEAAKK@Z 0000000180036020 f   WMI.obj
 0001:00035090       ?GetProcessUserSid@WMIConnection@@QEAA?AV?$basic_string@_WU?$char_traits@_W@std@@V?$allocator@_W@2@@std@@K@Z 0000000180036090 f   WMI.obj
 0001:00035300       ?SetProcessPriority@WMIConnection@@QEAAHKK@Z 0000000180036300 f   WMI.obj
 0001:00035330       ?TerminateProcess@WMIConnection@@QEAAHK@Z 0000000180036330 f   WMI.obj
 0001:00035440       ?Message@@YAHIPEB_WPEAPEB_W_K2@Z 0000000180036440 f   Proclist.obj
 0001:00035750       ?is_wow64_process@@YA_NPEAX@Z 0000000180036750 f   Proclist.obj
 0001:00035780       ClosePanelW                0000000180036780 f   Proclist.obj
 0001:000357b0       CompareW                   00000001800367b0 f   Proclist.obj
 0001:000357d0       ConfigureW                 00000001800367d0 f   Proclist.obj
 0001:000357e0       DeleteFilesW               00000001800367e0 f   Proclist.obj
 0001:00035800       _guard_check_icall_nop     0000000180036800 f   LIBCMT:guard_support.obj
 0001:00035800       ExitFARW                   0000000180036800 f   Proclist.obj
 0001:00035810       FreeFindDataW              0000000180036810 f   Proclist.obj
 0001:00035820       GetFilesW                  0000000180036820 f   Proclist.obj
 0001:00035860       GetFindDataW               0000000180036860 f   Proclist.obj
 0001:00035880       GetGlobalInfoW             0000000180036880 f   Proclist.obj
 0001:00035900       GetOpenPanelInfoW          0000000180036900 f   Proclist.obj
 0001:00035910       GetPluginInfoW             0000000180036910 f   Proclist.obj
 0001:000359e0       OpenW                      00000001800369e0 f   Proclist.obj
 0001:00035a80       ProcessPanelEventW         0000000180036a80 f   Proclist.obj
 0001:00035aa0       ProcessPanelInputW         0000000180036aa0 f   Proclist.obj
 0001:00035ac0       SetStartupInfoW            0000000180036ac0 f   Proclist.obj
 0001:00035bd6       ConvertSidToStringSidW     0000000180036bd6 f   advapi32:ADVAPI32.dll
 0001:00035bdc       WNetAddConnection2W        0000000180036bdc f   mpr:MPR.dll
 0001:00035be2       WNetCancelConnection2W     0000000180036be2 f   mpr:MPR.dll
 0001:00035be8       GetFileVersionInfoSizeW    0000000180036be8 f   version:VERSION.dll
 0001:00035bee       GetFileVersionInfoW        0000000180036bee f   version:VERSION.dll
 0001:00035bf4       VerQueryValueW             0000000180036bf4 f   version:VERSION.dll
 0001:00035bfa       GetModuleFileNameExW       0000000180036bfa f   psapi:PSAPI.DLL
 0001:00035c00       GetModuleInformation       0000000180036c00 f   psapi:PSAPI.DLL
 0001:00035c08       ??0_Init_locks@std@@QEAA@XZ 0000000180036c08 f   libcpmt:xlock.obj
 0001:00035c4c       ??0_Lockit@std@@QEAA@H@Z   0000000180036c4c f   libcpmt:xlock.obj
 0001:00035c88       ??1_Init_locks@std@@QEAA@XZ 0000000180036c88 f   libcpmt:xlock.obj
 0001:00035cc4       ??1_Lockit@std@@QEAA@XZ    0000000180036cc4 f   libcpmt:xlock.obj
 0001:00035cf8       ??0bad_alloc@std@@QEAA@XZ  0000000180036cf8 f i libcpmt:xthrow.obj
 0001:00035d18       ??0bad_function_call@std@@QEAA@AEBV01@@Z 0000000180036d18 f i libcpmt:xthrow.obj
 0001:00035d54       ??0bad_function_call@std@@QEAA@XZ 0000000180036d54 f i libcpmt:xthrow.obj
 0001:00035d6c       ??0length_error@std@@QEAA@AEBV01@@Z 0000000180036d6c f i libcpmt:xthrow.obj
 0001:00035da8       ??0length_error@std@@QEAA@PEBD@Z 0000000180036da8 f i libcpmt:xthrow.obj
 0001:00035df0       ??0logic_error@std@@QEAA@AEBV01@@Z 0000000180036df0 f i libcpmt:xthrow.obj
 0001:00035e2c       ??0out_of_range@std@@QEAA@AEBV01@@Z 0000000180036e2c f i libcpmt:xthrow.obj
 0001:00035e68       ??0out_of_range@std@@QEAA@PEBD@Z 0000000180036e68 f i libcpmt:xthrow.obj
 0001:00035eb0       ?__scrt_throw_std_bad_alloc@@YAXXZ 0000000180036eb0 f   LIBCMT:throw_bad_alloc.obj
 0001:00035eb0       ?_Xbad_alloc@std@@YAXXZ    0000000180036eb0 f   libcpmt:xthrow.obj
 0001:00035ed0       ?_Xbad_function_call@std@@YAXXZ 0000000180036ed0 f   libcpmt:xthrow.obj
 0001:00035ef0       ?_Xlength_error@std@@YAXPEBD@Z 0000000180036ef0 f   libcpmt:xthrow.obj
 0001:00035f14       ?_Xout_of_range@std@@YAXPEBD@Z 0000000180036f14 f   libcpmt:xthrow.obj
 0001:00035f38       ?_Xruntime_error@std@@YAXPEBD@Z 0000000180036f38 f   libcpmt:xthrow.obj
 0001:00035f5c       ?what@bad_function_call@std@@UEBAPEBDXZ 0000000180036f5c f i libcpmt:xthrow.obj
 0001:00035f64       ??4?$_Yarn@D@std@@QEAAAEAV01@PEBD@Z 0000000180036f64 f i libcpmt:locale0.obj
 0001:00035fdc       ??_E_Locimp@locale@std@@MEAAPEAXI@Z 0000000180036fdc f i libcpmt:locale0.obj
 0001:00035fdc       ??_G_Locimp@locale@std@@MEAAPEAXI@Z 0000000180036fdc f i libcpmt:locale0.obj
 0001:00036038       ?_Facet_Register@std@@YAXPEAV_Facet_base@1@@Z 0000000180037038 f   libcpmt:locale0.obj
 0001:00036070       ?_Getgloballocale@locale@std@@CAPEAV_Locimp@12@XZ 0000000180037070 f   libcpmt:locale0.obj
 0001:00036078       ?_Init@locale@std@@CAPEAV_Locimp@12@_N@Z 0000000180037078 f   libcpmt:locale0.obj
 0001:00036124       ?_Locimp_dtor@_Locimp@locale@std@@CAXPEAV123@@Z 0000000180037124 f   libcpmt:locale0.obj
 0001:000361a0       ?_Locinfo_ctor@_Locinfo@std@@SAXPEAV12@PEBD@Z 00000001800371a0 f   libcpmt:locale0.obj
 0001:0003620c       ?_Locinfo_dtor@_Locinfo@std@@SAXPEAV12@@Z 000000018003720c f   libcpmt:locale0.obj
 0001:00036228       ?_New_Locimp@_Locimp@locale@std@@CAPEAV123@_N@Z 0000000180037228 f   libcpmt:locale0.obj
 0001:00036298       ?_Setgloballocale@locale@std@@CAXPEAX@Z 0000000180037298 f   libcpmt:locale0.obj
 0001:000362cc       _Deletegloballocale        00000001800372cc f   libcpmt:locale0.obj
 0001:0003633c       _Getcvt                    000000018003733c f   libcpmt:xwctomb.obj
 0001:000363d4       _Mbrtowc                   00000001800373d4 f   libcpmt:xmbtowc.obj
 0001:00036570       _Mtxdst                    0000000180037570 f   libcpmt:xmtx.obj
 0001:00036578       _Mtxinit                   0000000180037578 f   libcpmt:xmtx.obj
 0001:00036588       _Mtxlock                   0000000180037588 f   libcpmt:xmtx.obj
 0001:00036590       _Mtxunlock                 0000000180037590 f   libcpmt:xmtx.obj
 0001:00036598       ?_Atexit@@YAXP6AXXZ@Z      0000000180037598 f   libcpmt:iosptrs.obj
 0001:0003698c       __crtInitializeCriticalSectionEx 000000018003798c f   libcpmt:winapisupp.obj
 0001:000369b8       ??3@YAXPEAX_K@Z            00000001800379b8 f   LIBCMT:delete_scalar_size.obj
 0001:000369b8       ??_V@YAXPEAX@Z             00000001800379b8 f   LIBCMT:delete_array.obj
 0001:000369c0       __scrt_acquire_startup_lock 00000001800379c0 f   LIBCMT:utility.obj
 0001:000369fc       __scrt_dllmain_after_initialize_c 00000001800379fc f   LIBCMT:utility.obj
 0001:00036a30       __scrt_dllmain_before_initialize_c 0000000180037a30 f   LIBCMT:utility.obj
 0001:00036a48       __scrt_dllmain_crt_thread_attach 0000000180037a48 f   LIBCMT:utility.obj
 0001:00036a70       __scrt_dllmain_crt_thread_detach 0000000180037a70 f   LIBCMT:utility.obj
 0001:00036a88       __scrt_dllmain_exception_filter 0000000180037a88 f   LIBCMT:utility.obj
 0001:00036ae8       __scrt_dllmain_uninitialize_c 0000000180037ae8 f   LIBCMT:utility.obj
 0001:00036b18       __scrt_dllmain_uninitialize_critical 0000000180037b18 f   LIBCMT:utility.obj
 0001:00036b2c       __scrt_initialize_crt      0000000180037b2c f   LIBCMT:utility.obj
 0001:00036b78       __scrt_initialize_onexit_tables 0000000180037b78 f   LIBCMT:utility.obj
 0001:00036c04       __scrt_is_nonwritable_in_current_image 0000000180037c04 f   LIBCMT:utility.obj
 0001:00036c9c       __scrt_release_startup_lock 0000000180037c9c f   LIBCMT:utility.obj
 0001:00036cc0       __scrt_uninitialize_crt    0000000180037cc0 f   LIBCMT:utility.obj
 0001:00036cec       _onexit                    0000000180037cec f   LIBCMT:utility.obj
 0001:00036d28       atexit                     0000000180037d28 f   LIBCMT:utility.obj
 0001:00036d40       ??2@YAPEAX_K@Z             0000000180037d40 f   LIBCMT:new_scalar.obj
 0001:00036d7c       ??_Gtype_info@@UEAAPEAXI@Z 0000000180037d7c f i LIBCMT:std_type_info_static.obj
 0001:00036d7c       ??_Etype_info@@UEAAPEAXI@Z 0000000180037d7c f i LIBCMT:std_type_info_static.obj
 0001:00036da8       ??_U@YAPEAX_K@Z            0000000180037da8 f   LIBCMT:new_array.obj
 0001:00036db0       ??_M@YAXPEAX_K1P6AX0@Z@Z   0000000180037db0 f   LIBCMT:ehvecdtr.obj
 0001:00036e1c       ?__ArrayUnwind@@YAXPEAX_K1P6AX0@Z@Z 0000000180037e1c f   LIBCMT:ehvecdtr.obj
 0001:000371a0       _DllMainCRTStartup         00000001800381a0 f   LIBCMT:dll_dllmain.obj
 0001:000371e0       __GSHandlerCheck           00000001800381e0 f   LIBCMT:gshandler.obj
 0001:00037200       __GSHandlerCheckCommon     0000000180038200 f   LIBCMT:gshandler.obj
 0001:0003725c       __GSHandlerCheck_EH        000000018003825c f   LIBCMT:gshandlereh.obj
 0001:000372f0       __security_check_cookie    00000001800382f0 f   LIBCMT:amdsecgs.obj
 0001:00037314       ??3@YAXPEAX@Z              0000000180038314 f   LIBCMT:delete_scalar.obj
 0001:0003731c       __isa_available_init       000000018003831c f   LIBCMT:cpu_disp.obj
 0001:000374c0       _get_startup_argv_mode     00000001800384c0 f   LIBCMT:argv_mode.obj
 0001:000374c0       DllMain                    00000001800384c0 f   LIBCMT:dll_dllmain_stub.obj
 0001:000374c8       __scrt_is_ucrt_dll_in_use  00000001800384c8 f   LIBCMT:ucrt_detection.obj
 0001:000374d4       __crt_debugger_hook        00000001800384d4 f   LIBCMT:utility_desktop.obj
 0001:000374dc       __scrt_fastfail            00000001800384dc f   LIBCMT:utility_desktop.obj
 0001:00037628       __security_init_cookie     0000000180038628 f   LIBCMT:gs_support.obj
 0001:000376d4       ?__scrt_initialize_type_info@@YAXXZ 00000001800386d4 f   LIBCMT:tncleanup.obj
 0001:000376e4       ?__scrt_uninitialize_type_info@@YAXXZ 00000001800386e4 f   LIBCMT:tncleanup.obj
 0001:000376f0       __local_stdio_scanf_options 00000001800386f0 f i LIBCMT:default_local_stdio_options.obj
 0001:000376f8       __scrt_initialize_default_local_stdio_options 00000001800386f8 f   LIBCMT:default_local_stdio_options.obj
 0001:00037714       __scrt_get_dyn_tls_init_callback 0000000180038714 f   LIBCMT:dyn_tls_init.obj
 0001:0003771c       _RTC_Initialize            000000018003871c f   LIBCMT:initsect.obj
 0001:00037758       _RTC_Terminate             0000000180038758 f   LIBCMT:initsect.obj
 0001:000377a0       __raise_securityfailure    00000001800387a0 f   LIBCMT:gs_report.obj
 0001:000377d4       __report_gsfailure         00000001800387d4 f   LIBCMT:gs_report.obj
 0001:000378a8       __report_rangecheckfailure 00000001800388a8 f   LIBCMT:gs_report.obj
 0001:000378bc       __report_securityfailure   00000001800388bc f   LIBCMT:gs_report.obj
 0001:00037a3c       _get_purecall_handler      0000000180038a3c f   libvcruntime:purevirt.obj
 0001:00037a44       _purecall                  0000000180038a44 f   libvcruntime:purevirt.obj
 0001:00037a60       __DestructExceptionObject  0000000180038a60 f   libvcruntime:ehhelpers.obj
 0001:00037ad0       ?_CallMemberFunction0@@YAXQEAX0@Z 0000000180038ad0 f i libvcruntime:ehhelpers.obj
 0001:00037ad4       _IsExceptionObjectToBeDestroyed 0000000180038ad4 f   libvcruntime:ehhelpers.obj
 0001:00037b04       __AdjustPointer            0000000180038b04 f   libvcruntime:ehhelpers.obj
 0001:00037b28       __FrameUnwindFilter        0000000180038b28 f   libvcruntime:ehhelpers.obj
 0001:00037b90       __current_exception        0000000180038b90 f   libvcruntime:ehhelpers.obj
 0001:00037ba4       __current_exception_context 0000000180038ba4 f   libvcruntime:ehhelpers.obj
 0001:00037bb8       __std_terminate            0000000180038bb8 f   libvcruntime:ehhelpers.obj
 0001:00037bc4       __std_exception_copy       0000000180038bc4 f   libvcruntime:std_exception.obj
 0001:00037c54       __std_exception_destroy    0000000180038c54 f   libvcruntime:std_exception.obj
 0001:00037c7c       _CxxThrowException         0000000180038c7c f   libvcruntime:throw.obj
 0001:00037d1c       ??$_CallSETranslator@V__FrameHandler3@@@@YAHPEAUEHExceptionRecord@@PEA_KPEAU_CONTEXT@@PEAU_xDISPATCHER_CONTEXT@@PEBU_s_FuncInfo@@K1@Z 0000000180038d1c f i libvcruntime:risctrnsctrl.obj
 0001:00037d70       ??$_CallSETranslator@V__FrameHandler4@@@@YAHPEAUEHExceptionRecord@@PEA_KPEAU_CONTEXT@@PEAU_xDISPATCHER_CONTEXT@@PEAUFuncInfo4@FH4@@K1@Z 0000000180038d70 f i libvcruntime:risctrnsctrl.obj
 0001:00037dc4       ?CatchTryBlock@__FrameHandler3@@SAPEBU_s_TryBlockMapEntry@@PEBU_s_FuncInfo@@H@Z 0000000180038dc4 f   libvcruntime:risctrnsctrl.obj
 0001:00037e18       ?DecompFuncInfo@FH4@@YA_JPEAEAEAUFuncInfo4@1@_KH_N@Z 0000000180038e18 f i libvcruntime:risctrnsctrl.obj
 0001:00037f3c       ?ExecutionInCatch@__FrameHandler3@@SA_NPEAU_xDISPATCHER_CONTEXT@@PEBU_s_FuncInfo@@@Z 0000000180038f3c f   libvcruntime:risctrnsctrl.obj
 0001:00037f68       ?ExecutionInCatch@__FrameHandler4@@SA_NPEAU_xDISPATCHER_CONTEXT@@PEAUFuncInfo4@FH4@@@Z 0000000180038f68 f   libvcruntime:risctrnsctrl.obj
 0001:00037f70       ?FrameUnwindToEmptyState@__FrameHandler3@@SAXPEA_KPEAU_xDISPATCHER_CONTEXT@@PEBU_s_FuncInfo@@@Z 0000000180038f70 f   libvcruntime:risctrnsctrl.obj
 0001:00037fd4       ?FrameUnwindToEmptyState@__FrameHandler4@@SAXPEA_KPEAU_xDISPATCHER_CONTEXT@@PEAUFuncInfo4@FH4@@@Z 0000000180038fd4 f   libvcruntime:risctrnsctrl.obj
 0001:00038008       ?GetEstablisherFrame@__FrameHandler3@@SAPEA_KPEA_KPEAU_xDISPATCHER_CONTEXT@@PEBU_s_FuncInfo@@0@Z 0000000180039008 f   libvcruntime:risctrnsctrl.obj
 0001:000380d4       ?GetEstablisherFrame@__FrameHandler4@@SAPEA_KPEA_KPEAU_xDISPATCHER_CONTEXT@@PEAUFuncInfo4@FH4@@0@Z 00000001800390d4 f   libvcruntime:risctrnsctrl.obj
 0001:000380f8       ?GetRangeOfTrysToCheck@__FrameHandler3@@SA?AU?$pair@Viterator@TryBlockMap@__FrameHandler3@@V123@@std@@AEAVTryBlockMap@1@HPEAU_xDISPATCHER_CONTEXT@@PEBU_s_FuncInfo@@H@Z 00000001800390f8 f   libvcruntime:risctrnsctrl.obj
 0001:00038238       ?GetRangeOfTrysToCheck@__FrameHandler4@@SA?AU?$pair@Viterator@TryBlockMap4@FH4@@V123@@std@@AEAVTryBlockMap4@FH4@@HPEAU_xDISPATCHER_CONTEXT@@PEAUFuncInfo4@5@H@Z 0000000180039238 f   libvcruntime:risctrnsctrl.obj
 0001:00038390       ?UnwindNestedFrames@__FrameHandler3@@SAXPEA_KPEAUEHExceptionRecord@@PEAU_CONTEXT@@0PEAXPEBU_s_FuncInfo@@HHPEBU_s_HandlerType@@PEAU_xDISPATCHER_CONTEXT@@E@Z 0000000180039390 f   libvcruntime:risctrnsctrl.obj
 0001:00038494       ?UnwindNestedFrames@__FrameHandler4@@SAXPEA_KPEAUEHExceptionRecord@@PEAU_CONTEXT@@0PEAXPEAUFuncInfo4@FH4@@HHPEAUHandlerType4@5@PEAU_xDISPATCHER_CONTEXT@@E@Z 0000000180039494 f   libvcruntime:risctrnsctrl.obj
 0001:000385d4       ?setBuffer@TryBlockMap4@FH4@@QEAAXViterator@12@@Z 00000001800395d4 f i libvcruntime:risctrnsctrl.obj
 0001:00038798       _CreateFrameInfo           0000000180039798 f   libvcruntime:risctrnsctrl.obj
 0001:000387d4       _FindAndUnlinkFrame        00000001800397d4 f   libvcruntime:risctrnsctrl.obj
 0001:00038828       _GetImageBase              0000000180039828 f   libvcruntime:risctrnsctrl.obj
 0001:0003883c       _GetThrowImageBase         000000018003983c f   libvcruntime:risctrnsctrl.obj
 0001:00038850       _SetImageBase              0000000180039850 f   libvcruntime:risctrnsctrl.obj
 0001:00038868       _SetThrowImageBase         0000000180039868 f   libvcruntime:risctrnsctrl.obj
 0001:00038880       __CxxFrameHandler3         0000000180039880 f   libvcruntime:risctrnsctrl.obj
 0001:00038908       __CxxFrameHandler4         0000000180039908 f   libvcruntime:risctrnsctrl.obj
 0001:000389e0       memchr                     00000001800399e0 f   libvcruntime:memchr.obj
 0001:00038a60       memcmp                     0000000180039a60 f   libvcruntime:memcmp.obj
 0001:00038b40       memcpy_repmovs             0000000180039b40 f   libvcruntime:memcpy.obj
 0001:00038b60       memmove                    0000000180039b60 f   libvcruntime:memcpy.obj
 0001:00038b60       memcpy                     0000000180039b60 f   libvcruntime:memcpy.obj
 0001:00038f50       memset_repmovs             0000000180039f50 f   libvcruntime:memset.obj
 0001:00038f70       memset                     0000000180039f70 f   libvcruntime:memset.obj
 0001:00039100       wcschr                     000000018003a100 f   libvcruntime:wcschr.obj
 0001:0003917c       __vcrt_initialize          000000018003a17c f   libvcruntime:initialization.obj
 0001:000391a4       __vcrt_thread_attach       000000018003a1a4 f   libvcruntime:initialization.obj
 0001:000391b8       __vcrt_thread_detach       000000018003a1b8 f   libvcruntime:initialization.obj
 0001:000391cc       __vcrt_uninitialize        000000018003a1cc f   libvcruntime:initialization.obj
 0001:000391e8       __vcrt_uninitialize_critical 000000018003a1e8 f   libvcruntime:initialization.obj
 0001:000391f8       __C_specific_handler       000000018003a1f8 f   libvcruntime:riscchandler.obj
 0001:00039404       __std_type_info_compare    000000018003a404 f   libvcruntime:std_type_info.obj
 0001:0003942c       __std_type_info_destroy_list 000000018003a42c f   libvcruntime:std_type_info.obj
 0001:00039458       __vcrt_freefls             000000018003a458 f   libvcruntime:per_thread_data.obj
 0001:00039478       __vcrt_freeptd             000000018003a478 f   libvcruntime:per_thread_data.obj
 0001:000394c8       __vcrt_getptd              000000018003a4c8 f   libvcruntime:per_thread_data.obj
 0001:000394e4       __vcrt_getptd_noexit       000000018003a4e4 f   libvcruntime:per_thread_data.obj
 0001:000395a4       __vcrt_initialize_ptd      000000018003a5a4 f   libvcruntime:per_thread_data.obj
 0001:000395ec       __vcrt_uninitialize_ptd    000000018003a5ec f   libvcruntime:per_thread_data.obj
 0001:00039610       ?GetCurrentState@__FrameHandler3@@SAHPEA_KPEAU_xDISPATCHER_CONTEXT@@PEBU_s_FuncInfo@@@Z 000000018003a610 f   libvcruntime:ehstate.obj
 0001:00039638       ?GetUnwindTryBlock@__FrameHandler3@@SAHPEA_KPEAU_xDISPATCHER_CONTEXT@@PEBU_s_FuncInfo@@@Z 000000018003a638 f   libvcruntime:ehstate.obj
 0001:00039664       ?SetState@__FrameHandler3@@SAXPEA_KPEBU_s_FuncInfo@@H@Z 000000018003a664 f   libvcruntime:ehstate.obj
 0001:00039670       ?SetUnwindTryBlock@__FrameHandler3@@SAXPEA_KPEAU_xDISPATCHER_CONTEXT@@PEBU_s_FuncInfo@@H@Z 000000018003a670 f   libvcruntime:ehstate.obj
 0001:000396ac       ?StateFromControlPc@__FrameHandler3@@SAHPEBU_s_FuncInfo@@PEAU_xDISPATCHER_CONTEXT@@@Z 000000018003a6ac f   libvcruntime:ehstate.obj
 0001:000396b4       ?StateFromControlPc@__FrameHandler4@@SAHPEAUFuncInfo4@FH4@@PEAU_xDISPATCHER_CONTEXT@@@Z 000000018003a6b4 f   libvcruntime:ehstate.obj
 0001:000396bc       ?StateFromIp@__FrameHandler3@@SAHPEBU_s_FuncInfo@@PEAU_xDISPATCHER_CONTEXT@@_K@Z 000000018003a6bc f   libvcruntime:ehstate.obj
 0001:00039724       ?StateFromIp@__FrameHandler4@@SAHPEAUFuncInfo4@FH4@@PEAU_xDISPATCHER_CONTEXT@@_K@Z 000000018003a724 f   libvcruntime:ehstate.obj
 0001:0003ae50       ??$TypeMatchHelper@V__FrameHandler3@@@@YAHPEBU_s_HandlerType@@PEBU_s_CatchableType@@PEBU_s_ThrowInfo@@@Z 000000018003be50 f i libvcruntime:frame.obj
 0001:0003af94       ??$TypeMatchHelper@V__FrameHandler4@@@@YAHPEAUHandlerType4@FH4@@PEBU_s_CatchableType@@PEBU_s_ThrowInfo@@@Z 000000018003bf94 f i libvcruntime:frame.obj
 0001:0003b0dc       ??$__InternalCxxFrameHandler@V__FrameHandler3@@@@YA?AW4_EXCEPTION_DISPOSITION@@PEAUEHExceptionRecord@@PEA_KPEAU_CONTEXT@@PEAU_xDISPATCHER_CONTEXT@@PEBU_s_FuncInfo@@H1E@Z 000000018003c0dc f i libvcruntime:frame.obj
 0001:0003b324       ??$__InternalCxxFrameHandler@V__FrameHandler4@@@@YA?AW4_EXCEPTION_DISPOSITION@@PEAUEHExceptionRecord@@PEA_KPEAU_CONTEXT@@PEAU_xDISPATCHER_CONTEXT@@PEAUFuncInfo4@FH4@@H1E@Z 000000018003c324 f i libvcruntime:frame.obj
 0001:0003b5c4       ??0HandlerMap4@FH4@@QEAA@PEBUTryBlockMapEntry4@1@_KH@Z 000000018003c5c4 f i libvcruntime:frame.obj
 0001:0003b640       ??0TryBlockMap4@FH4@@QEAA@PEBUFuncInfo4@1@_K@Z 000000018003c640 f i libvcruntime:frame.obj
 0001:0003b718       ??0bad_exception@std@@QEAA@AEBV01@@Z 000000018003c718 f i libvcruntime:frame.obj
 0001:0003b754       ??0bad_exception@std@@QEAA@XZ 000000018003c754 f i libvcruntime:frame.obj
 0001:0003b774       ?CxxCallCatchBlock@__FrameHandler3@@SAPEAXPEAU_EXCEPTION_RECORD@@@Z 000000018003c774 f   libvcruntime:frame.obj
 0001:0003b960       ?CxxCallCatchBlock@__FrameHandler4@@SAPEAXPEAU_EXCEPTION_RECORD@@@Z 000000018003c960 f   libvcruntime:frame.obj
 0001:0003bbb0       ?DecompHandler@HandlerMap4@FH4@@AEAAXXZ 000000018003cbb0 f i libvcruntime:frame.obj
 0001:0003bdf0       ?FrameUnwindToState@__FrameHandler3@@SAXPEA_KPEAU_xDISPATCHER_CONTEXT@@PEBU_s_FuncInfo@@H@Z 000000018003cdf0 f   libvcruntime:frame.obj
 0001:0003bf7c       ?FrameUnwindToState@__FrameHandler4@@SAXPEA_KPEAU_xDISPATCHER_CONTEXT@@PEAUFuncInfo4@FH4@@H@Z 000000018003cf7c f   libvcruntime:frame.obj
 0001:0003c250       ?GetHandlerSearchState@__FrameHandler3@@SAHPEA_KPEAU_xDISPATCHER_CONTEXT@@PEBU_s_FuncInfo@@@Z 000000018003d250 f i libvcruntime:frame.obj
 0001:0003c460       ?ReadEntry@UWMap4@FH4@@AEAAXPEAPEAE@Z 000000018003d460 f i libvcruntime:frame.obj
 0001:0003c500       ?_CallMemberFunction1@@YAXQEAX00@Z 000000018003d500 f i libvcruntime:frame.obj
 0001:0003c50c       ?_CallMemberFunction2@@YAXQEAX00H@Z 000000018003d50c f i libvcruntime:frame.obj
 0001:0003c51c       ?getStartStop@UWMap4@FH4@@QEAAXHHAEAViterator@12@0@Z 000000018003d51c f i libvcruntime:frame.obj
 0001:0003c5ec       ?getStateFromIterators@UWMap4@FH4@@SAHAEBViterator@12@H0H0@Z 000000018003d5ec f i libvcruntime:frame.obj
 0001:0003c6b4       __vcrt_initialize_locks    000000018003d6b4 f   libvcruntime:locks.obj
 0001:0003c6e8       __vcrt_uninitialize_locks  000000018003d6e8 f   libvcruntime:locks.obj
 0001:0003c730       _NLG_Notify                000000018003d730 f   libvcruntime:notify.obj
 0001:0003c750       __NLG_Dispatch2            000000018003d750 f   libvcruntime:notify.obj
 0001:0003c760       __NLG_Return2              000000018003d760 f   libvcruntime:notify.obj
 0001:0003c764       __except_validate_context_record 000000018003d764 f   libvcruntime:jbcxrval.obj
 0001:0003c8f8       __vcrt_FlsAlloc            000000018003d8f8 f   libvcruntime:winapi_downlevel.obj
 0001:0003c940       __vcrt_FlsFree             000000018003d940 f   libvcruntime:winapi_downlevel.obj
 0001:0003c988       __vcrt_FlsGetValue         000000018003d988 f   libvcruntime:winapi_downlevel.obj
 0001:0003c9d0       __vcrt_FlsSetValue         000000018003d9d0 f   libvcruntime:winapi_downlevel.obj
 0001:0003ca24       __vcrt_InitializeCriticalSectionEx 000000018003da24 f   libvcruntime:winapi_downlevel.obj
 0001:0003caa0       _CallSettingFrame          000000018003daa0 f   libvcruntime:handlers.obj
 0001:0003caf0       _CallSettingFrame_LookupContinuationIndex 000000018003daf0 f   libvcruntime:handlers.obj
 0001:0003cb20       _CallSettingFrame_NotifyContinuationAddr 000000018003db20 f   libvcruntime:handlers.obj
 0001:0003cb50       _CallSettingFrameEncoded   000000018003db50 f   libvcruntime:handlers.obj
 0001:0003cb98       __acrt_call_reportfault    000000018003db98 f   libucrt:invalid_parameter.obj
 0001:0003ccf4       __acrt_initialize_invalid_parameter_handler 000000018003dcf4 f   libucrt:invalid_parameter.obj
 0001:0003ccfc       _invalid_parameter         000000018003dcfc f   libucrt:invalid_parameter.obj
 0001:0003cdac       _invalid_parameter_noinfo  000000018003ddac f   libucrt:invalid_parameter.obj
 0001:0003cdcc       _invalid_parameter_noinfo_noreturn 000000018003ddcc f   libucrt:invalid_parameter.obj
 0001:0003cdfc       _invoke_watson             000000018003ddfc f   libucrt:invalid_parameter.obj
 0001:0003ce44       _dclass                    000000018003de44 f   libucrt:nan.obj
 0001:0003ce60       _dsign                     000000018003de60 f   libucrt:nan.obj
 0001:0003ce60       _ldsign                    000000018003de60 f   libucrt:nanl.obj
 0001:0003ce78       _ldclass                   000000018003de78 f   libucrt:nanl.obj
 0001:0003ce94       _fdclass                   000000018003de94 f   libucrt:nanf.obj
 0001:0003ceb0       _fdsign                    000000018003deb0 f   libucrt:nanf.obj
 0001:0003cec4       calloc                     000000018003dec4 f   libucrt:calloc.obj
 0001:0003cecc       free                       000000018003decc f   libucrt:free.obj
 0001:0003cee0       __acrt_errno_from_os_error 000000018003dee0 f   libucrt:errno.obj
 0001:0003cf28       __acrt_errno_map_os_error  000000018003df28 f   libucrt:errno.obj
 0001:0003cf78       __doserrno                 000000018003df78 f   libucrt:errno.obj
 0001:0003cf98       _errno                     000000018003df98 f   libucrt:errno.obj
 0001:0003cfb8       __acrt_initialize_stdio    000000018003dfb8 f   libucrt:_file.obj
 0001:0003d0d8       __acrt_uninitialize_stdio  000000018003e0d8 f   libucrt:_file.obj
 0001:0003d134       _lock_file                 000000018003e134 f   libucrt:_file.obj
 0001:0003d140       _unlock_file               000000018003e140 f   libucrt:_file.obj
 0001:0003d14c       _fileno                    000000018003e14c f   libucrt:fileno.obj
 0001:0003d340       ??$ensure_buffer_is_big_enough@D@formatting_buffer@__crt_stdio_output@@QEAA_N_K@Z 000000018003e340 f i libucrt:output.obj
 0001:0003d3e8       ??$type_case_integer_parse_into_buffer@I@?$output_processor@DV?$string_output_adapter@D@__crt_stdio_output@@V?$format_validation_base@DV?$string_output_adapter@D@__crt_stdio_output@@@2@@__crt_stdio_output@@AEAAXII_N@Z 000000018003e3e8 f i libucrt:output.obj
 0001:0003d470       ??$type_case_integer_parse_into_buffer@_K@?$output_processor@DV?$string_output_adapter@D@__crt_stdio_output@@V?$format_validation_base@DV?$string_output_adapter@D@__crt_stdio_output@@@2@@__crt_stdio_output@@AEAAX_KI_N@Z 000000018003e470 f i libucrt:output.obj
 0001:0003d500       ??$write_multiple_characters@V?$string_output_adapter@D@__crt_stdio_output@@D@__crt_stdio_output@@YAXAEBV?$string_output_adapter@D@0@DHQEAH@Z 000000018003e500 f i libucrt:output.obj
 0001:0003d578       ??0_LocaleUpdate@@QEAA@QEAU__crt_locale_pointers@@@Z 000000018003e578 f i libucrt:output.obj
 0001:0003d614       ??1_LocaleUpdate@@QEAA@XZ  000000018003e614 f i libucrt:output.obj
 0001:0003d628       ?crop_zeroes@__crt_stdio_output@@YAXPEADQEAU__crt_locale_pointers@@@Z 000000018003e628 f i libucrt:output.obj
 0001:0003d694       ?parse_int_from_format_string@?$output_processor@DV?$string_output_adapter@D@__crt_stdio_output@@V?$format_validation_base@DV?$string_output_adapter@D@__crt_stdio_output@@@2@@__crt_stdio_output@@AEAA_NQEAH@Z 000000018003e694 f i libucrt:output.obj
 0001:0003d738       ?process@?$output_processor@DV?$string_output_adapter@D@__crt_stdio_output@@V?$format_validation_base@DV?$string_output_adapter@D@__crt_stdio_output@@@2@@__crt_stdio_output@@QEAAHXZ 000000018003e738 f i libucrt:output.obj
 0001:0003d950       ?state_case_normal@?$output_processor@DV?$string_output_adapter@D@__crt_stdio_output@@V?$format_validation_base@DV?$string_output_adapter@D@__crt_stdio_output@@@2@@__crt_stdio_output@@AEAA_NXZ 000000018003e950 f i libucrt:output.obj
 0001:0003d9c4       ?state_case_normal_tchar@?$output_processor@DV?$string_output_adapter@D@__crt_stdio_output@@V?$format_validation_base@DV?$string_output_adapter@D@__crt_stdio_output@@@2@@__crt_stdio_output@@AEAA_ND@Z 000000018003e9c4 f i libucrt:output.obj
 0001:0003da6c       ?state_case_size@?$output_processor@DV?$string_output_adapter@D@__crt_stdio_output@@V?$format_validation_base@DV?$string_output_adapter@D@__crt_stdio_output@@@2@@__crt_stdio_output@@AEAA_NXZ 000000018003ea6c f i libucrt:output.obj
 0001:0003dbe0       ?state_case_type@?$output_processor@DV?$string_output_adapter@D@__crt_stdio_output@@V?$format_validation_base@DV?$string_output_adapter@D@__crt_stdio_output@@@2@@__crt_stdio_output@@AEAA_NXZ 000000018003ebe0 f i libucrt:output.obj
 0001:0003de48       ?type_case_Z@?$output_processor@DV?$string_output_adapter@D@__crt_stdio_output@@V?$format_validation_base@DV?$string_output_adapter@D@__crt_stdio_output@@@2@@__crt_stdio_output@@AEAA_NXZ 000000018003ee48 f i libucrt:output.obj
 0001:0003debc       ?type_case_a@?$output_processor@DV?$string_output_adapter@D@__crt_stdio_output@@V?$format_validation_base@DV?$string_output_adapter@D@__crt_stdio_output@@@2@@__crt_stdio_output@@AEAA_NXZ 000000018003eebc f i libucrt:output.obj
 0001:0003e0d4       ?type_case_c_tchar@?$output_processor@DV?$string_output_adapter@D@__crt_stdio_output@@V?$format_validation_base@DV?$string_output_adapter@D@__crt_stdio_output@@@2@@__crt_stdio_output@@AEAA_ND@Z 000000018003f0d4 f i libucrt:output.obj
 0001:0003e190       ?type_case_integer@?$output_processor@DV?$string_output_adapter@D@__crt_stdio_output@@V?$format_validation_base@DV?$string_output_adapter@D@__crt_stdio_output@@@2@@__crt_stdio_output@@AEAA_NI_N@Z 000000018003f190 f i libucrt:output.obj
 0001:0003e358       ?type_case_n@?$output_processor@DV?$string_output_adapter@D@__crt_stdio_output@@V?$format_validation_base@DV?$string_output_adapter@D@__crt_stdio_output@@@2@@__crt_stdio_output@@AEAA_NXZ 000000018003f358 f i libucrt:output.obj
 0001:0003e434       ?type_case_s@?$output_processor@DV?$string_output_adapter@D@__crt_stdio_output@@V?$format_validation_base@DV?$string_output_adapter@D@__crt_stdio_output@@@2@@__crt_stdio_output@@AEAA_NXZ 000000018003f434 f i libucrt:output.obj
 0001:0003e4cc       ?write_stored_string_tchar@?$output_processor@DV?$string_output_adapter@D@__crt_stdio_output@@V?$format_validation_base@DV?$string_output_adapter@D@__crt_stdio_output@@@2@@__crt_stdio_output@@AEAA_ND@Z 000000018003f4cc f i libucrt:output.obj
 0001:0003e5a4       ?write_string@?$string_output_adapter@D@__crt_stdio_output@@QEBAXQEBDHQEAHAEAV__crt_deferred_errno_cache@@@Z 000000018003f5a4 f i libucrt:output.obj
 0001:0003e648       __stdio_common_vsnprintf_s 000000018003f648 f   libucrt:output.obj
 0001:0003e77c       terminate                  000000018003f77c f   libucrt:terminate.obj
 0001:0003e79c       localeconv                 000000018003f79c f   libucrt:localeconv.obj
 0001:0003e7d0       __acrt_lowio_create_handle_array 000000018003f7d0 f   libucrt:osfinfo.obj
 0001:0003e878       __acrt_lowio_destroy_handle_array 000000018003f878 f   libucrt:osfinfo.obj
 0001:0003e8c8       __acrt_lowio_ensure_fh_exists 000000018003f8c8 f   libucrt:osfinfo.obj
 0001:0003e970       __acrt_lowio_lock_fh       000000018003f970 f   libucrt:osfinfo.obj
 0001:0003e998       __acrt_lowio_unlock_fh     000000018003f998 f   libucrt:osfinfo.obj
 0001:0003e9c0       _free_osfhnd               000000018003f9c0 f   libucrt:osfinfo.obj
 0001:0003ea7c       _get_osfhandle             000000018003fa7c f   libucrt:osfinfo.obj
 0001:0003eaf4       _isatty                    000000018003faf4 f   libucrt:isatty.obj
 0001:0003eb54       malloc                     000000018003fb54 f   libucrt:malloc.obj
 0001:0003eb5c       log2                       000000018003fb5c f   libucrt:log2.obj
 0001:0003ee84       modf                       000000018003fe84 f   libucrt:modf.obj
 0001:0003ef64       round                      000000018003ff64 f   libucrt:round.obj
 0001:0003efcc       _isleadbyte_l              000000018003ffcc f i libucrt:_wctype.obj
 0001:0003f018       iswdigit                   0000000180040018 f i libucrt:_wctype.obj
 0001:0003f024       wcscspn                    0000000180040024 f   libucrt:wcscspn.obj
 0001:0003f064       wcsncpy                    0000000180040064 f   libucrt:wcsncpy.obj
 0001:0003f0ac       wcspbrk                    00000001800400ac f   libucrt:wcspbrk.obj
 0001:0003f0e0       wcstok                     00000001800400e0 f   libucrt:wcstok.obj
 0001:0003f11c       ceilf                      000000018004011c f   libucrt:ceilf.obj
 0001:0003f1b0       log10                      00000001800401b0 f   libucrt:log10.obj
 0001:0003f760       pow                        0000000180040760 f   libucrt:pow.obj
 0001:00040df4       __acrt_initialize_locks    0000000180041df4 f   libucrt:locks.obj
 0001:00040e3c       __acrt_lock                0000000180041e3c f   libucrt:locks.obj
 0001:00040e58       __acrt_uninitialize_locks  0000000180041e58 f   libucrt:locks.obj
 0001:00040e90       __acrt_unlock              0000000180041e90 f   libucrt:locks.obj
 0001:00040eac       _lock_locales              0000000180041eac f   libucrt:locks.obj
 0001:00040ec8       _unlock_locales            0000000180041ec8 f   libucrt:locks.obj
 0001:000411b8       setlocale                  00000001800421b8 f   libucrt:setlocale.obj
 0001:00041204       ___lc_codepage_func        0000000180042204 f   libucrt:initctype.obj
 0001:00041234       ___lc_locale_name_func     0000000180042234 f   libucrt:initctype.obj
 0001:00041268       ___mb_cur_max_func         0000000180042268 f   libucrt:initctype.obj
 0001:00041298       __acrt_locale_initialize_ctype 0000000180042298 f   libucrt:initctype.obj
 0001:000418fc       __pctype_func              00000001800428fc f   libucrt:ctype.obj
 0001:00041930       ?divide@__crt_strtox@@YA_KAEAUbig_integer@1@AEBU21@@Z 0000000180042930 f i libucrt:strtod.obj
 0001:00041d5c       _ischartype_l              0000000180042d5c f i libucrt:strtod.obj
 0001:00041e60       powf                       0000000180042e60 f   libucrt:powf.obj
 0001:00042d28       abort                      0000000180043d28 f   libucrt:abort.obj
 0001:00042d80       wcsdup                     0000000180043d80 f   libucrt:wcsdup.obj
 0001:00042d80       _wcsdup                    0000000180043d80 f   libucrt:wcsdup.obj
 0001:00042e04       ??$__acrt_mbs_to_wcs_cp@U__crt_win32_buffer_internal_dynamic_resizing@@@@YAHQEBDAEAV?$__crt_win32_buffer@_WU__crt_win32_buffer_internal_dynamic_resizing@@@@I@Z 0000000180043e04 f i libucrt:strftime.obj
 0001:00042f7c       ??$__acrt_wcs_to_mbs_cp@U__crt_win32_buffer_no_resizing@@@@YAHQEB_WAEAV?$__crt_win32_buffer@DU__crt_win32_buffer_no_resizing@@@@I@Z 0000000180043f7c f i libucrt:strftime.obj
 0001:00043090       __strncnt                  0000000180044090 f   libucrt:strncnt.obj
 0001:000430a8       wcscpy_s                   00000001800440a8 f   libucrt:wcscpy_s.obj
 0001:00043110       strnlen                    0000000180044110 f   libucrt:strnlen.obj
 0001:00043260       wcsnlen                    0000000180044260 f   libucrt:strnlen.obj
 0001:00043438       _seh_filter_dll            0000000180044438 f   libucrt:exception_filter.obj
 0001:0004344c       _seh_filter_exe            000000018004444c f   libucrt:exception_filter.obj
 0001:0004383c       __acrt_initialize_thread_local_exit_callback 000000018004483c f   libucrt:exit.obj
 0001:00043844       _cexit                     0000000180044844 f   libucrt:exit.obj
 0001:00043854       _exit                      0000000180044854 f   libucrt:exit.obj
 0001:00043860       _is_c_termination_complete 0000000180044860 f   libucrt:exit.obj
 0001:00043a2c       __acrt_allocate_buffer_for_argv 0000000180044a2c f   libucrt:argv_parsing.obj
 0001:00043a8c       _configure_narrow_argv     0000000180044a8c f   libucrt:argv_parsing.obj
 0001:00043e04       __dcrt_uninitialize_environments_nolock 0000000180044e04 f   libucrt:environment_initialization.obj
 0001:00043e3c       _initialize_narrow_environment 0000000180044e3c f   libucrt:environment_initialization.obj
 0001:00044184       _crt_atexit                0000000180045184 f   libucrt:onexit.obj
 0001:00044194       _execute_onexit_table      0000000180045194 f   libucrt:onexit.obj
 0001:000441d0       _initialize_onexit_table   00000001800451d0 f   libucrt:onexit.obj
 0001:000441f8       _register_onexit_function  00000001800451f8 f   libucrt:onexit.obj
 0001:00044278       __acrt_uninitialize_command_line 0000000180045278 f   libucrt:argv_data.obj
 0001:00044370       __acrt_initialize          0000000180045370 f   libucrt:initialization.obj
 0001:00044384       __acrt_thread_attach       0000000180045384 f   libucrt:initialization.obj
 0001:00044398       __acrt_thread_detach       0000000180045398 f   libucrt:initialization.obj
 0001:000443a8       __acrt_uninitialize        00000001800453a8 f   libucrt:initialization.obj
 0001:000443e0       __acrt_uninitialize_critical 00000001800453e0 f   libucrt:initialization.obj
 0001:000443f0       __initialize_lconv_for_unsigned_char 00000001800453f0 f   libucrt:lconv_unsigned_char_initialization.obj
 0001:000443fc       __acrt_initialize_new_handler 00000001800453fc f   libucrt:new_handler.obj
 0001:00044404       _callnewh                  0000000180045404 f   libucrt:new_handler.obj
 0001:00044434       _query_new_handler         0000000180045434 f   libucrt:new_handler.obj
 0001:00044468       _initterm                  0000000180045468 f   libucrt:initterm.obj
 0001:000444cc       _initterm_e                00000001800454cc f   libucrt:initterm.obj
 0001:0004450c       strcpy_s                   000000018004550c f   libucrt:strcpy_s.obj
 0001:0004456c       ??$parse_integer@KV?$c_string_character_source@D@__crt_strtox@@@__crt_strtox@@YAKQEAU__crt_locale_pointers@@V?$c_string_character_source@D@0@H_N@Z 000000018004556c f i libucrt:atox.obj
 0001:00044874       ??$parse_integer@KV?$c_string_character_source@_W@__crt_strtox@@@__crt_strtox@@YAKQEAU__crt_locale_pointers@@V?$c_string_character_source@_W@0@H_N@Z 0000000180045874 f i libucrt:atox.obj
 0001:00044f1c       _wtol                      0000000180045f1c f   libucrt:atox.obj
 0001:00044f60       strncmp                    0000000180045f60 f   libucrt:strncmp.obj
 0001:00044fe0       wcsncmp                    0000000180045fe0 f   libucrt:wcsncmp.obj
 0001:00045384       __acrt_freeptd             0000000180046384 f   libucrt:per_thread_data.obj
 0001:000453c8       __acrt_getptd              00000001800463c8 f   libucrt:per_thread_data.obj
 0001:0004549c       __acrt_getptd_head         000000018004649c f   libucrt:per_thread_data.obj
 0001:00045544       __acrt_getptd_noexit       0000000180046544 f   libucrt:per_thread_data.obj
 0001:00045610       __acrt_initialize_ptd      0000000180046610 f   libucrt:per_thread_data.obj
 0001:0004564c       __acrt_uninitialize_ptd    000000018004664c f   libucrt:per_thread_data.obj
 0001:00045670       _d_int                     0000000180046670 f   libucrt:_test.obj
 0001:00045788       _dtest                     0000000180046788 f   libucrt:_test.obj
 0001:000457ec       _fdtest                    00000001800467ec f   libucrt:_test.obj
 0001:00045838       _ldtest                    0000000180046838 f   libucrt:_test.obj
 0001:00045840       _calloc_base               0000000180046840 f   libucrt:calloc_base.obj
 0001:000458b8       _free_base                 00000001800468b8 f   libucrt:free_base.obj
 0001:00045b74       __acrt_AppPolicyGetProcessTerminationMethodInternal 0000000180046b74 f   libucrt:winapi_thunks.obj
 0001:00045bc4       __acrt_AreFileApisANSI     0000000180046bc4 f   libucrt:winapi_thunks.obj
 0001:00045c00       __acrt_EnumSystemLocalesEx 0000000180046c00 f   libucrt:winapi_thunks.obj
 0001:00045c98       __acrt_FlsAlloc            0000000180046c98 f   libucrt:winapi_thunks.obj
 0001:00045ce0       __acrt_FlsFree             0000000180046ce0 f   libucrt:winapi_thunks.obj
 0001:00045d28       __acrt_FlsGetValue         0000000180046d28 f   libucrt:winapi_thunks.obj
 0001:00045d70       __acrt_FlsSetValue         0000000180046d70 f   libucrt:winapi_thunks.obj
 0001:00045dc4       __acrt_GetLocaleInfoEx     0000000180046dc4 f   libucrt:winapi_thunks.obj
 0001:00045e48       __acrt_GetUserDefaultLocaleName 0000000180046e48 f   libucrt:winapi_thunks.obj
 0001:00045eac       __acrt_InitializeCriticalSectionEx 0000000180046eac f   libucrt:winapi_thunks.obj
 0001:00045f10       __acrt_IsValidLocaleName   0000000180046f10 f   libucrt:winapi_thunks.obj
 0001:00045f68       __acrt_LCIDToLocaleName    0000000180046f68 f   libucrt:winapi_thunks.obj
 0001:00045fd8       __acrt_LCMapStringEx       0000000180046fd8 f   libucrt:winapi_thunks.obj
 0001:000460b4       __acrt_LocaleNameToLCID    00000001800470b4 f   libucrt:winapi_thunks.obj
 0001:00046104       __acrt_can_use_vista_locale_apis 0000000180047104 f   libucrt:winapi_thunks.obj
 0001:00046134       __acrt_eagerly_load_locale_apis 0000000180047134 f   libucrt:winapi_thunks.obj
 0001:00046290       __acrt_initialize_winapi_thunks 0000000180047290 f   libucrt:winapi_thunks.obj
 0001:000462c4       __acrt_uninitialize_winapi_thunks 00000001800472c4 f   libucrt:winapi_thunks.obj
 0001:00046308       _fcloseall                 0000000180047308 f   libucrt:closeall.obj
 0001:00046598       __acrt_stdio_flush_nolock  0000000180047598 f   libucrt:fflush.obj
 0001:00046614       _fflush_nolock             0000000180047614 f   libucrt:fflush.obj
 0001:00046660       _flushall                  0000000180047660 f   libucrt:fflush.obj
 0001:00046668       __acrt_stdio_free_buffer_nolock 0000000180047668 f   libucrt:_freebuf.obj
 0001:000468a4       __acrt_initialize_lowio    00000001800478a4 f   libucrt:ioinit.obj
 0001:000468e0       __acrt_uninitialize_lowio  00000001800478e0 f   libucrt:ioinit.obj
 0001:00047180       _write                     0000000180048180 f   libucrt:write.obj
 0001:0004726c       _write_nolock              000000018004826c f   libucrt:write.obj
 0001:00047548       _malloc_base               0000000180048548 f   libucrt:malloc_base.obj
 0001:000475a8       strtol                     00000001800485a8 f   libucrt:strtox.obj
 0001:000475d4       _mbtowc_l                  00000001800485d4 f   libucrt:mbtowc.obj
 0001:00047754       mbtowc                     0000000180048754 f   libucrt:mbtowc.obj
 0001:0004775c       _wctomb_s_l                000000018004875c f   libucrt:wctomb.obj
 0001:000478f8       wctomb_s                   00000001800488f8 f   libucrt:wctomb.obj
 0001:0004790c       __acrt_update_locale_info  000000018004890c f   libucrt:locale_update.obj
 0001:00047940       __acrt_update_multibyte_info 0000000180048940 f   libucrt:locale_update.obj
 0001:0004820c       __acrt_fp_format           000000018004920c f   libucrt:cvt.obj
 0001:00048510       _get_printf_count_output   0000000180049510 f   libucrt:printf_count_output.obj
 0001:00048790       ?commit_locale_name@_expandlocale_locale_name_cache@@QEAAXQEB_W_K@Z 0000000180049790 f i libucrt:wsetlocale.obj
 0001:00048808       __acrt_copy_locale_name    0000000180049808 f   libucrt:wsetlocale.obj
 0001:0004888c       __acrt_set_locale_changed  000000018004988c f   libucrt:wsetlocale.obj
 0001:00048898       __acrt_uninitialize_locale 0000000180049898 f   libucrt:wsetlocale.obj
 0001:000488c8       __lc_lctowcs               00000001800498c8 f   libucrt:wsetlocale.obj
 0001:0004896c       __lc_wcstolc               000000018004996c f   libucrt:wsetlocale.obj
 0001:00049014       _wcscats                   000000018004a014 f   libucrt:wsetlocale.obj
 0001:0004907c       _wsetlocale                000000018004a07c f   libucrt:wsetlocale.obj
 0001:00049fdc       _mbstowcs_s_l              000000018004afdc f   libucrt:mbstowcs.obj
 0001:0004a110       mbstowcs_s                 000000018004b110 f   libucrt:mbstowcs.obj
 0001:0004a130       strncpy_s                  000000018004b130 f   libucrt:strncpy_s.obj
 0001:0004a204       _query_app_type            000000018004b204 f   libucrt:report_runtime_error.obj
 0001:0004a330       _handle_error              000000018004b330 f   libucrt:libm_error.obj
 0001:0004a458       _handle_errorf             000000018004b458 f   libucrt:libm_error.obj
 0001:0004a58c       _handle_nan                000000018004b58c f   libucrt:libm_error.obj
 0001:0004a5a8       _handle_nanf               000000018004b5a8 f   libucrt:libm_error.obj
 0001:0004a5b8       iswctype                   000000018004b5b8 f   libucrt:iswctype.obj
 0001:0004a628       __acrt_wcstok_s_novalidation 000000018004b628 f   libucrt:wcstok_s.obj
 0001:0004a6e0       __acrt_initialize_fma3     000000018004b6e0 f   libucrt:fma3_available.obj
 0001:0004a750       _log10_special             000000018004b750 f   libucrt:log_special.obj
 0001:0004a810       _pow_special               000000018004b810 f   libucrt:pow_special.obj
 0001:0004a934       _powf_special              000000018004b934 f   libucrt:pow_special.obj
 0001:0004ae28       _wcstombs_s_l              000000018004be28 f   libucrt:wcstombs.obj
 0001:0004b090       __acrt_GetLocaleInfoA      000000018004c090 f   libucrt:getlocaleinfoa.obj
 0001:0004b258       __acrt_GetStringTypeA      000000018004c258 f   libucrt:getstringtypea.obj
 0001:0004b700       __acrt_LCMapStringA        000000018004c700 f   libucrt:lcmapstringa.obj
 0001:0004b798       _raise_exc                 000000018004c798 f   libucrt:fpexcept.obj
 0001:0004b7c0       _raise_exc_ex              000000018004c7c0 f   libucrt:fpexcept.obj
 0001:0004bad0       _raise_excf                000000018004cad0 f   libucrt:fpexcept.obj
 0001:0004bafc       _set_errno_from_matherr    000000018004cafc f   libucrt:fpexcept.obj
 0001:0004bb2c       _clrfp                     000000018004cb2c f   libucrt:fpctrl.obj
 0001:0004bb4c       _ctrlfp                    000000018004cb4c f   libucrt:fpctrl.obj
 0001:0004bbc8       _set_statfp                000000018004cbc8 f   libucrt:fpctrl.obj
 0001:0004bbe8       _statfp                    000000018004cbe8 f   libucrt:fpctrl.obj
 0001:0004bbfc       _realloc_base              000000018004cbfc f   libucrt:realloc_base.obj
 0001:0004bc78       _isctype_l                 000000018004cc78 f   libucrt:isctype.obj
 0001:0004bdc8       __acrt_get_sigabrt_handler 000000018004cdc8 f   libucrt:signal.obj
 0001:0004bdf8       __acrt_initialize_signal_handlers 000000018004cdf8 f   libucrt:signal.obj
 0001:0004be18       raise                      000000018004ce18 f   libucrt:signal.obj
 0001:0004c084       __acrt_MultiByteToWideChar 000000018004d084 f   libucrt:multibytetowidechar.obj
 0001:0004c0e0       __acrt_WideCharToMultiByte 000000018004d0e0 f   libucrt:widechartomultibyte.obj
 0001:0004c178       __ascii_wcsicmp            000000018004d178 f   libucrt:wcsicmp.obj
 0001:0004c1b8       _wcsicmp                   000000018004d1b8 f   libucrt:wcsicmp.obj
 0001:0004c200       _wcsicmp_l                 000000018004d200 f   libucrt:wcsicmp.obj
 0001:0004c328       __acrt_initialize_timeset  000000018004d328 f   libucrt:timeset.obj
 0001:0004c36c       __acrt_get_process_end_policy 000000018004d36c f   libucrt:win_policies.obj
 0001:0004c3bc       ??$__acrt_wcs_to_mbs_cp@U__crt_win32_buffer_internal_dynamic_resizing@@@@YAHQEB_WAEAV?$__crt_win32_buffer@DU__crt_win32_buffer_internal_dynamic_resizing@@@@I@Z 000000018004d3bc f i libucrt:argv_wildcards.obj
 0001:0004cbec       __acrt_expand_narrow_argv_wildcards 000000018004dbec f   libucrt:argv_wildcards.obj
 0001:0004cbf4       __acrt_GetModuleFileNameA  000000018004dbf4 f   libucrt:getmodulefilenamea.obj
 0001:0004d440       __acrt_initialize_multibyte 000000018004e440 f   libucrt:mbctype.obj
 0001:0004d4a0       __acrt_update_thread_multibyte_data 000000018004e4a0 f   libucrt:mbctype.obj
 0001:0004d4bc       _setmbcp_nolock            000000018004e4bc f   libucrt:mbctype.obj
 0001:0004d7f0       _ismbblead                 000000018004e7f0 f   libucrt:ismbbyte.obj
 0001:0004d804       __acrt_initialize_command_line 000000018004e804 f   libucrt:argv_data.obj
 0001:0004d82c       __dcrt_get_narrow_environment_from_os 000000018004e82c f   libucrt:get_environment_from_os.obj
 0001:0004d930       _recalloc_base             000000018004e930 f   libucrt:recalloc.obj
 0001:0004d9c8       __acrt_initialize_heap     000000018004e9c8 f   libucrt:heap_handle.obj
 0001:0004d9e4       __acrt_uninitialize_heap   000000018004e9e4 f   libucrt:heap_handle.obj
 0001:0004d9f0       __acrt_execute_initializers 000000018004e9f0 f   libucrt:shared_initialization.obj
 0001:0004da70       __acrt_execute_uninitializers 000000018004ea70 f   libucrt:shared_initialization.obj
 0001:0004daac       __acrt_has_user_matherr    000000018004eaac f   libucrt:matherr.obj
 0001:0004dacc       __acrt_initialize_user_matherr 000000018004eacc f   libucrt:matherr.obj
 0001:0004dad4       __acrt_invoke_user_matherr 000000018004ead4 f   libucrt:matherr.obj
 0001:0004db04       __acrt_add_locale_ref      000000018004eb04 f   libucrt:locale_refcounting.obj
 0001:0004db90       __acrt_free_locale         000000018004eb90 f   libucrt:locale_refcounting.obj
 0001:0004dd08       __acrt_locale_add_lc_time_reference 000000018004ed08 f   libucrt:locale_refcounting.obj
 0001:0004dd30       __acrt_locale_free_lc_time_if_unreferenced 000000018004ed30 f   libucrt:locale_refcounting.obj
 0001:0004dd68       __acrt_locale_release_lc_time_reference 000000018004ed68 f   libucrt:locale_refcounting.obj
 0001:0004dd90       __acrt_release_locale_ref  000000018004ed90 f   libucrt:locale_refcounting.obj
 0001:0004de38       __acrt_update_thread_locale_data 000000018004ee38 f   libucrt:locale_refcounting.obj
 0001:0004dea4       _updatetlocinfoEx_nolock   000000018004eea4 f   libucrt:locale_refcounting.obj
 0001:0004df0c       __acrt_fenv_get_control    000000018004ef0c f   libucrt:_fenvutils.obj
 0001:0004e000       __acrt_fenv_get_status     000000018004f000 f   libucrt:_fenvutils.obj
 0001:0004e054       __acrt_fenv_set_control    000000018004f054 f   libucrt:_fenvutils.obj
 0001:0004e19c       __acrt_fenv_set_status     000000018004f19c f   libucrt:_fenvutils.obj
 0001:0004e220       _query_new_mode            000000018004f220 f   libucrt:new_mode.obj
 0001:0004e228       __acrt_DownlevelLCIDToLocaleName 000000018004f228 f   libucrt:lcidtoname_downlevel.obj
 0001:0004e31c       __acrt_DownlevelLocaleNameToLCID 000000018004f31c f   libucrt:lcidtoname_downlevel.obj
 0001:0004e3cc       _fclose_nolock             000000018004f3cc f   libucrt:fclose.obj
 0001:0004e450       fclose                     000000018004f450 f   libucrt:fclose.obj
 0001:0004e540       _commit                    000000018004f540 f   libucrt:commit.obj
 0001:0004e670       _lseeki64_nolock           000000018004f670 f   libucrt:lseek.obj
 0001:0004e678       ?__mbrtowc_utf8@__crt_mbstring@@YA_KPEA_WPEBD_KPEAU_Mbstatet@@@Z 000000018004f678 f   libucrt:mbrtowc.obj
 0001:0004e6b4       ?__mbsrtowcs_utf8@__crt_mbstring@@YA_KPEA_WPEAPEBD_KPEAU_Mbstatet@@@Z 000000018004f6b4 f   libucrt:mbrtowc.obj
 0001:0004e82c       _putwch_nolock             000000018004f82c f   libucrt:putwch.obj
 0001:0004e868       ?__c32rtomb_utf8@__crt_mbstring@@YA_KPEAD_UPEAU_Mbstatet@@@Z 000000018004f868 f   libucrt:c32rtomb.obj
 0001:0004e91c       c32rtomb                   000000018004f91c f   libucrt:c32rtomb.obj
 0001:0004e924       __acrt_fp_strflt_to_string 000000018004f924 f   libucrt:_fptostr.obj
 0001:0004ea08       __acrt_fltout              000000018004fa08 f   libucrt:cfout.obj
 0001:0004fc3c       __acrt_locale_free_monetary 0000000180050c3c f   libucrt:initmon.obj
 0001:0004fd48       __acrt_locale_initialize_monetary 0000000180050d48 f   libucrt:initmon.obj
 0001:0005027c       __acrt_locale_free_numeric 000000018005127c f   libucrt:initnum.obj
 0001:000502e8       __acrt_locale_initialize_numeric 00000001800512e8 f   libucrt:initnum.obj
 0001:00050968       __acrt_locale_free_time    0000000180051968 f   libucrt:inittime.obj
 0001:00050a70       __acrt_locale_initialize_time 0000000180051a70 f   libucrt:inittime.obj
 0001:00050b0c       wcscat_s                   0000000180051b0c f   libucrt:wcscat_s.obj
 0001:00050b8c       wcsncat_s                  0000000180051b8c f   libucrt:wcsncat_s.obj
 0001:00050c8c       wcsncpy_s                  0000000180051c8c f   libucrt:wcsncpy_s.obj
 0001:00051524       __acrt_get_qualified_locale 0000000180052524 f   libucrt:get_qualified_locale.obj
 0001:00051f58       __acrt_get_qualified_locale_downlevel 0000000180052f58 f   libucrt:getqloc_downlevel.obj
 0001:000521d8       __acrt_GetStringTypeW      00000001800531d8 f   libucrt:getstringtypew.obj
 0001:000521e0       ?__wcsrtombs_utf8@__crt_mbstring@@YA_KPEADPEAPEB_W_KPEAU_Mbstatet@@@Z 00000001800531e0 f   libucrt:wcrtomb.obj
 0001:00052310       _get_fpsr                  0000000180053310 f   libucrt:fpsr.obj
 0001:00052320       _set_fpsr                  0000000180053320 f   libucrt:fpsr.obj
 0001:0005232a       _fclrf                     000000018005332a f   libucrt:fpsr.obj
 0001:0005233e       _frnd                      000000018005333e f   libucrt:fpsr.obj
 0001:00052360       _towlower_l                0000000180053360 f   libucrt:towlower.obj
 0001:00052420       qsort                      0000000180053420 f   libucrt:qsort.obj
 0001:00052870       strpbrk                    0000000180053870 f   libucrt:strpbrk.obj
 0001:00052c50       _mbsdec                    0000000180053c50 f   libucrt:mbsdec.obj
 0001:00052c58       _mbsdec_l                  0000000180053c58 f   libucrt:mbsdec.obj
 0001:00052d04       _msize_base                0000000180053d04 f   libucrt:msize.obj
 0001:00052d40       __ascii_wcsnicmp           0000000180053d40 f   libucrt:wcsnicmp.obj
 0001:00052d8c       _wcsnicmp                  0000000180053d8c f   libucrt:wcsnicmp.obj
 0001:00052dd4       _wcsnicmp_l                0000000180053dd4 f   libucrt:wcsnicmp.obj
 0001:00052f98       _close                     0000000180053f98 f   libucrt:close.obj
 0001:0005303c       _close_nolock              000000018005403c f   libucrt:close.obj
 0001:000530fc       ?__acrt_stdio_free_stream@@YAXV__crt_stdio_stream@@@Z 00000001800540fc f   libucrt:stream.obj
 0001:00053118       ?__mbrtoc32_utf8@__crt_mbstring@@YA_KPEA_UPEBD_KPEAU_Mbstatet@@@Z 0000000180054118 f   libucrt:mbrtoc32.obj
 0001:000532f4       __dcrt_lowio_ensure_console_output_initialized 00000001800542f4 f   libucrt:initcon.obj
 0001:00053348       __dcrt_terminate_console_output 0000000180054348 f   libucrt:initcon.obj
 0001:00053364       __dcrt_write_console       0000000180054364 f   libucrt:initcon.obj
 0001:00053424       fegetenv                   0000000180054424 f   libucrt:fegetenv.obj
 0001:00053444       fesetenv                   0000000180054444 f   libucrt:fesetenv.obj
 0001:00053490       feholdexcept               0000000180054490 f   libucrt:feholdexcept.obj
 0001:000534e0       ceil                       00000001800544e0 f   libucrt:ceil.obj
 0001:000536e4       _itow_s                    00000001800546e4 f   libucrt:xtoa.obj
 0001:00053704       wcscmp                     0000000180054704 f   libucrt:wcscmp.obj
 0001:0005373c       ?__c16rtomb_utf8@__crt_mbstring@@YA_KPEAD_SPEAU_Mbstatet@@@Z 000000018005473c f   libucrt:c16rtomb.obj
 0001:000537e4       __acrt_LCMapStringW        00000001800547e4 f   libucrt:lcmapstringw.obj
 0001:0005386c       _clearfp                   000000018005486c f   libucrt:ieee.obj
 0001:000538da       IsProcessorFeaturePresent  00000001800548da f   kernel32:KERNEL32.dll
 0001:000538e0       _FindPESection             00000001800548e0 f   LIBCMT:pesect.obj
 0001:00053930       _IsNonwritableInCurrentImage 0000000180054930 f   LIBCMT:pesect.obj
 0001:00053980       _ValidateImageBase         0000000180054980 f   LIBCMT:pesect.obj
 0001:000539b0       __GSHandlerCheck_SEH       00000001800549b0 f   LIBCMT:gshandlerseh.obj
 0001:00053a38       strrchr                    0000000180054a38 f   libvcruntime:strrchr.obj
 0001:00053b80       _guard_dispatch_icall_nop  0000000180054b80 f   LIBCMT:guard_dispatch.obj
 0001:00058e88       _TI3?AVbad_array_new_length@std@@ 0000000180059e88     format.obj
 0001:00058ea8       _CTA3?AVbad_array_new_length@std@@ 0000000180059ea8     format.obj
 0001:00058ec8       _CT??_R0?AVbad_array_new_length@std@@@8??0bad_array_new_length@std@@QEAA@AEBV01@@Z24 0000000180059ec8     format.obj
 0001:00058ef0       _CT??_R0?AVbad_alloc@std@@@8??0bad_alloc@std@@QEAA@AEBV01@@Z24 0000000180059ef0     format.obj
 0001:00058f18       _CT??_R0?AVexception@std@@@8??0exception@std@@QEAA@AEBV01@@Z24 0000000180059f18     format.obj
 0001:00058f40       _TI2?AVbad_cast@std@@      0000000180059f40     format.obj
 0001:00058f60       _CTA2?AVbad_cast@std@@     0000000180059f60     format.obj
 0001:00058f78       _CT??_R0?AVbad_cast@std@@@8??0bad_cast@std@@QEAA@AEBV01@@Z24 0000000180059f78     format.obj
 0001:00058fa0       _CT??_R0?AVruntime_error@std@@@8??0runtime_error@std@@QEAA@AEBV01@@Z24 0000000180059fa0     format.obj
 0001:00058fc8       _TI2?AVruntime_error@std@@ 0000000180059fc8     format.obj
 0001:00058fe8       _CTA2?AVruntime_error@std@@ 0000000180059fe8     format.obj
 0001:00059000       _TI3?AVformat_error@v6@fmt@@ 000000018005a000     format.obj
 0001:00059020       _CTA3?AVformat_error@v6@fmt@@ 000000018005a020     format.obj
 0001:00059040       _CT??_R0?AVformat_error@v6@fmt@@@8??0format_error@v6@fmt@@QEAA@AEBV012@@Z24 000000018005a040     format.obj
 0001:00059068       _TI2?AVbad_alloc@std@@     000000018005a068     libcpmt:xthrow.obj
 0001:00059088       _CTA2?AVbad_alloc@std@@    000000018005a088     libcpmt:xthrow.obj
 0001:000590a0       _CT??_R0?AVlogic_error@std@@@8??0logic_error@std@@QEAA@AEBV01@@Z24 000000018005a0a0     libcpmt:xthrow.obj
 0001:000590c8       _TI3?AVlength_error@std@@  000000018005a0c8     libcpmt:xthrow.obj
 0001:000590e8       _CTA3?AVlength_error@std@@ 000000018005a0e8     libcpmt:xthrow.obj
 0001:00059108       _CT??_R0?AVlength_error@std@@@8??0length_error@std@@QEAA@AEBV01@@Z24 000000018005a108     libcpmt:xthrow.obj
 0001:00059130       _TI3?AVout_of_range@std@@  000000018005a130     libcpmt:xthrow.obj
 0001:00059150       _CTA3?AVout_of_range@std@@ 000000018005a150     libcpmt:xthrow.obj
 0001:00059170       _CT??_R0?AVout_of_range@std@@@8??0out_of_range@std@@QEAA@AEBV01@@Z24 000000018005a170     libcpmt:xthrow.obj
 0001:00059198       _TI2?AVbad_function_call@std@@ 000000018005a198     libcpmt:xthrow.obj
 0001:000591b8       _CTA2?AVbad_function_call@std@@ 000000018005a1b8     libcpmt:xthrow.obj
 0001:000591d0       _CT??_R0?AVbad_function_call@std@@@8??0bad_function_call@std@@QEAA@AEBV01@@Z24 000000018005a1d0     libcpmt:xthrow.obj
 0001:000591f8       _TI2?AVbad_exception@std@@ 000000018005a1f8     libvcruntime:frame.obj
 0001:00059218       _CTA2?AVbad_exception@std@@ 000000018005a218     libvcruntime:frame.obj
 0001:00059230       _CT??_R0?AVbad_exception@std@@@8??0bad_exception@std@@QEAA@AEBV01@@Z24 000000018005a230     libvcruntime:frame.obj
 0002:00000000       ?instantiate_format_float@v6@fmt@@3P6AHNHUfloat_specs@detail@12@AEAV?$buffer@D@412@@ZEA 000000018005b000     format.obj
 0002:00000088       ?pNtQueryInformationProcess@@3P6AJPEAXW4_PROCESSINFOCLASS@@0KPEAK@ZEA 000000018005b088     Proclist.obj
 0002:00000090       ?pNtQueryInformationThread@@3P6AJPEAXK0KPEAK@ZEA 000000018005b090     Proclist.obj
 0002:00000098       ?pNtQueryObject@@3P6AJPEAXK0K0@ZEA 000000018005b098     Proclist.obj
 0002:000000a0       ?pNtQuerySystemInformation@@3P6AJKPEAXKPEAK@ZEA 000000018005b0a0     Proclist.obj
 0002:000000a8       ?pNtQueryInformationFile@@3P6AJPEAX00KK@ZEA 000000018005b0a8     Proclist.obj
 0002:000000b0       ?pNtWow64QueryInformationProcess64@@3P6AJPEAXW4_PROCESSINFOCLASS@@0KPEAK@ZEA 000000018005b0b0     Proclist.obj
 0002:000000b8       ?pNtWow64ReadVirtualMemory64@@3P6AJPEAX_K01PEA_K@ZEA 000000018005b0b8     Proclist.obj
 0002:000000c0       ?pIsValidSid@@3P6AHPEAX@ZEA 000000018005b0c0     Proclist.obj
 0002:000000c8       ?pGetSidIdentifierAuthority@@3P6APEAU_SID_IDENTIFIER_AUTHORITY@@PEAX@ZEA 000000018005b0c8     Proclist.obj
 0002:000000d0       ?pGetSidSubAuthorityCount@@3P6APEAEPEAX@ZEA 000000018005b0d0     Proclist.obj
 0002:000000d8       ?pGetSidSubAuthority@@3P6APEAKPEAXK@ZEA 000000018005b0d8     Proclist.obj
 0002:000000e0       ?pIsWow64Process@@3P6AHPEAXPEAH@ZEA 000000018005b0e0     Proclist.obj
 0002:000000e8       ?pGetGuiResources@@3P6AKPEAXK@ZEA 000000018005b0e8     Proclist.obj
 0002:000000f0       ?pCoSetProxyBlanket@@3P6AJPEAUIUnknown@@KKPEA_WKKPEAXK@ZEA 000000018005b0f0     Proclist.obj
 0002:000000f8       ?pEnumProcessModulesEx@@3P6AHPEAXPEAPEAUHINSTANCE__@@KPEAKK@ZEA 000000018005b0f8     Proclist.obj
 0002:00000110       __scrt_native_dllmain_reason 000000018005b110     LIBCMT:utility.obj
 0002:00000114       __do_unsigned_char_lconv_initialization 000000018005b114     LIBCMT:lconv_unsigned_char.obj
 0002:00000118       _fltused                   000000018005b118     LIBCMT:fltused.obj
 0002:00000120       __security_cookie_complement 000000018005b120     LIBCMT:gs_cookie.obj
 0002:00000128       __security_cookie          000000018005b128     LIBCMT:gs_cookie.obj
 0002:00000130       __isa_available            000000018005b130     LIBCMT:cpu_disp.obj
 0002:00000134       __isa_enabled              000000018005b134     LIBCMT:cpu_disp.obj
 0002:00000138       __memcpy_nt_iters          000000018005b138     LIBCMT:cpu_disp.obj
 0002:00000140       __memset_nt_iters          000000018005b140     LIBCMT:cpu_disp.obj
 0002:00000170       _iob                       000000018005b170     libucrt:_file.obj
 0002:00000280       __acrt_lconv_c             000000018005b280     libucrt:localeconv.obj
 0002:00000318       __acrt_lconv               000000018005b318     libucrt:localeconv.obj
 0002:00000320       __acrt_lconv_static_decimal 000000018005b320     libucrt:localeconv.obj
 0002:00000324       __acrt_lconv_static_W_decimal 000000018005b324     libucrt:localeconv.obj
 0002:00000330       _pctype                    000000018005b330     libucrt:ctype.obj
 0002:00000338       _pwctype                   000000018005b338     libucrt:ctype.obj
 0002:00000340       __abort_behavior           000000018005b340     libucrt:abort.obj
 0002:00000360       __acrt_initial_locale_data 000000018005b360     libucrt:nlsdata.obj
 0002:000004b8       __acrt_initial_locale_pointers 000000018005b4b8     libucrt:nlsdata.obj
 0002:000004c8       __acrt_wide_c_locale_string 000000018005b4c8     libucrt:nlsdata.obj
 0002:000004cc       __mb_cur_max               000000018005b4cc     libucrt:nlsdata.obj
 0002:000004d0       __globallocalestatus       000000018005b4d0     libucrt:glstatus.obj
 0002:00000570       __acrt_initial_multibyte_data 000000018005b570     libucrt:mbctype.obj
 0002:00000ab0       _lookuptrailbytes          000000018005bab0     libucrt:read.obj
 0002:00000bc0       ??_R0?AVbad_array_new_length@std@@@8 000000018005bbc0     format.obj
 0002:00000bf0       ??_R0?AVbad_alloc@std@@@8  000000018005bbf0     format.obj
 0002:00000c18       ??_R0?AVexception@std@@@8  000000018005bc18     format.obj
 0002:00000c40       ??_R0?AVbad_cast@std@@@8   000000018005bc40     format.obj
 0002:00000c68       ??_R0?AVruntime_error@std@@@8 000000018005bc68     format.obj
 0002:00000c90       ??_R0?AVformat_error@v6@fmt@@@8 000000018005bc90     format.obj
 0002:00000cc0       ??_R0?AV<lambda_c6a5923e4ab0669d9f7c2a6c892502eb>@@@8 000000018005bcc0     Plist.obj
 0002:00000dc0       ??_R0?AVlogic_error@std@@@8 000000018005bdc0     libcpmt:xthrow.obj
 0002:00000de8       ??_R0?AVlength_error@std@@@8 000000018005bde8     libcpmt:xthrow.obj
 0002:00000e10       ??_R0?AVout_of_range@std@@@8 000000018005be10     libcpmt:xthrow.obj
 0002:00000e38       ??_R0?AVbad_function_call@std@@@8 000000018005be38     libcpmt:xthrow.obj
 0002:00000e68       ??_R0?AV_Facet_base@std@@@8 000000018005be68     libcpmt:locale0.obj
 0002:00000e90       ??_R0?AV_Locimp@locale@std@@@8 000000018005be90     libcpmt:locale0.obj
 0002:00000ec0       ??_R0?AVfacet@locale@std@@@8 000000018005bec0     libcpmt:locale0.obj
 0002:00000ee8       ??_R0?AU_Crt_new_delete@std@@@8 000000018005bee8     libcpmt:locale0.obj
 0002:00000f18       ??_R0?AV?$numpunct@_W@std@@@8 000000018005bf18     libcpmt:wlocale.obj
 0002:00000f40       ??_R0?AVtype_info@@@8      000000018005bf40     LIBCMT:std_type_info_static.obj
 0002:00000f60       ??_R0?AVbad_exception@std@@@8 000000018005bf60     libvcruntime:frame.obj
 0002:00000f90       ?m_PanelModesDataLocal@Plist@@0V?$vector@Umode@@V?$allocator@Umode@@@std@@@std@@A 000000018005bf90     fileio.obj
 0002:00000fa8       ?m_PanelModesDataRemote@Plist@@0V?$vector@Umode@@V?$allocator@Umode@@@std@@@std@@A 000000018005bfa8     fileio.obj
 0002:00000fc0       ?_OptionsStorage@?1??__local_stdio_printf_options@@9@4_KA 000000018005bfc0     format.obj
 0002:00000fc8       ?id@?$numpunct@_W@std@@2V0locale@2@A 000000018005bfc8     format.obj
 0002:00000fd0       ?id@?$numpunct@D@std@@2V0locale@2@A 000000018005bfd0     format.obj
 0002:00000fd8       ?_Psave@?$_Facetptr@V?$numpunct@_W@std@@@std@@2PEBVfacet@locale@2@EB 000000018005bfd8     format.obj
 0002:00002680       ?Info@@3UPluginStartupInfo@@A 000000018005d680     Proclist.obj
 0002:00002798       ?Opt@@3Uoptions@@A         000000018005d798     Proclist.obj
 0002:000027c0       ?FSF@@3UFarStandardFunctions@@A 000000018005d7c0     Proclist.obj
 0002:00002ac0       ?_Id_cnt@id@locale@std@@0HA 000000018005dac0     libcpmt:locale0.obj
 0002:00002ac8       ?_Clocptr@_Locimp@locale@std@@0PEAV123@EA 000000018005dac8     libcpmt:locale0.obj
 0002:00002ad0       ?id@?$ctype@_W@std@@2V0locale@2@A 000000018005dad0     libcpmt:locale0.obj
 0002:00002ad8       ?id@?$ctype@D@std@@2V0locale@2@A 000000018005dad8     libcpmt:locale0.obj
 0002:00002ae0       ?id@?$codecvt@GDU_Mbstatet@@@std@@2V0locale@2@A 000000018005dae0     libcpmt:locale0.obj
 0002:00002ae8       ?id@?$ctype@G@std@@2V0locale@2@A 000000018005dae8     libcpmt:locale0.obj
 0002:00002b00       ?id@?$codecvt@_WDU_Mbstatet@@@std@@2V0locale@2@A 000000018005db00     libcpmt:locale0.obj
 0002:00002b28       ?id@?$num_get@DV?$istreambuf_iterator@DU?$char_traits@D@std@@@std@@@std@@2V0locale@2@A 000000018005db28     libcpmt:locale.obj
 0002:00002b30       ?id@?$num_put@DV?$ostreambuf_iterator@DU?$char_traits@D@std@@@std@@@std@@2V0locale@2@A 000000018005db30     libcpmt:locale.obj
 0002:00002b38       ?id@?$codecvt@DDU_Mbstatet@@@std@@2V0locale@2@A 000000018005db38     libcpmt:locale.obj
 0002:00002b40       ?_Ptr_cin@std@@3PEAV?$basic_istream@DU?$char_traits@D@std@@@1@EA 000000018005db40     libcpmt:iosptrs.obj
 0002:00002b48       ?_Ptr_cout@std@@3PEAV?$basic_ostream@DU?$char_traits@D@std@@@1@EA 000000018005db48     libcpmt:iosptrs.obj
 0002:00002b50       ?_Ptr_cerr@std@@3PEAV?$basic_ostream@DU?$char_traits@D@std@@@1@EA 000000018005db50     libcpmt:iosptrs.obj
 0002:00002b58       ?_Ptr_clog@std@@3PEAV?$basic_ostream@DU?$char_traits@D@std@@@1@EA 000000018005db58     libcpmt:iosptrs.obj
 0002:00002b60       ?_Ptr_wcin@std@@3PEAV?$basic_istream@_WU?$char_traits@_W@std@@@1@EA 000000018005db60     libcpmt:iosptrs.obj
 0002:00002b68       ?_Ptr_wcout@std@@3PEAV?$basic_ostream@_WU?$char_traits@_W@std@@@1@EA 000000018005db68     libcpmt:iosptrs.obj
 0002:00002b70       ?_Ptr_wcerr@std@@3PEAV?$basic_ostream@_WU?$char_traits@_W@std@@@1@EA 000000018005db70     libcpmt:iosptrs.obj
 0002:00002b78       ?_Ptr_wclog@std@@3PEAV?$basic_ostream@_WU?$char_traits@_W@std@@@1@EA 000000018005db78     libcpmt:iosptrs.obj
 0002:00002be0       __KERNEL32Functions        000000018005dbe0     libcpmt:winapisupp.obj
 0002:00002d20       ?id@?$time_put@_WV?$ostreambuf_iterator@_WU?$char_traits@_W@std@@@std@@@std@@2V0locale@2@A 000000018005dd20     libcpmt:wlocale.obj
 0002:00002d28       ?id@?$num_get@_WV?$istreambuf_iterator@_WU?$char_traits@_W@std@@@std@@@std@@2V0locale@2@A 000000018005dd28     libcpmt:wlocale.obj
 0002:00002d30       ?id@?$num_put@_WV?$ostreambuf_iterator@_WU?$char_traits@_W@std@@@std@@@std@@2V0locale@2@A 000000018005dd30     libcpmt:wlocale.obj
 0002:00002d38       ?id@?$collate@_W@std@@2V0locale@2@A 000000018005dd38     libcpmt:wlocale.obj
 0002:00002d40       ?id@?$messages@_W@std@@2V0locale@2@A 000000018005dd40     libcpmt:wlocale.obj
 0002:00002d48       ?id@?$money_get@_WV?$istreambuf_iterator@_WU?$char_traits@_W@std@@@std@@@std@@2V0locale@2@A 000000018005dd48     libcpmt:wlocale.obj
 0002:00002d50       ?id@?$money_put@_WV?$ostreambuf_iterator@_WU?$char_traits@_W@std@@@std@@@std@@2V0locale@2@A 000000018005dd50     libcpmt:wlocale.obj
 0002:00002d58       ?id@?$moneypunct@_W$0A@@std@@2V0locale@2@A 000000018005dd58     libcpmt:wlocale.obj
 0002:00002d60       ?id@?$moneypunct@_W$00@std@@2V0locale@2@A 000000018005dd60     libcpmt:wlocale.obj
 0002:00002d68       ?id@?$time_get@_WV?$istreambuf_iterator@_WU?$char_traits@_W@std@@@std@@@std@@2V0locale@2@A 000000018005dd68     libcpmt:wlocale.obj
 0002:00002d70       ?id@?$num_get@GV?$istreambuf_iterator@GU?$char_traits@G@std@@@std@@@std@@2V0locale@2@A 000000018005dd70     libcpmt:wlocale.obj
 0002:00002d78       ?id@?$num_put@GV?$ostreambuf_iterator@GU?$char_traits@G@std@@@std@@@std@@2V0locale@2@A 000000018005dd78     libcpmt:wlocale.obj
 0002:00002d80       ?id@?$numpunct@G@std@@2V0locale@2@A 000000018005dd80     libcpmt:wlocale.obj
 0002:00002d88       ?id@?$collate@G@std@@2V0locale@2@A 000000018005dd88     libcpmt:wlocale.obj
 0002:00002d90       ?id@?$messages@G@std@@2V0locale@2@A 000000018005dd90     libcpmt:wlocale.obj
 0002:00002d98       ?id@?$money_get@GV?$istreambuf_iterator@GU?$char_traits@G@std@@@std@@@std@@2V0locale@2@A 000000018005dd98     libcpmt:wlocale.obj
 0002:00002da0       ?id@?$money_put@GV?$ostreambuf_iterator@GU?$char_traits@G@std@@@std@@@std@@2V0locale@2@A 000000018005dda0     libcpmt:wlocale.obj
 0002:00002da8       ?id@?$moneypunct@G$0A@@std@@2V0locale@2@A 000000018005dda8     libcpmt:wlocale.obj
 0002:00002db0       ?id@?$moneypunct@G$00@std@@2V0locale@2@A 000000018005ddb0     libcpmt:wlocale.obj
 0002:00002db8       ?id@?$time_get@GV?$istreambuf_iterator@GU?$char_traits@G@std@@@std@@@std@@2V0locale@2@A 000000018005ddb8     libcpmt:wlocale.obj
 0002:00002dc0       ?id@?$time_put@GV?$ostreambuf_iterator@GU?$char_traits@G@std@@@std@@@std@@2V0locale@2@A 000000018005ddc0     libcpmt:wlocale.obj
 0002:00002dc8       ?id@?$collate@D@std@@2V0locale@2@A 000000018005ddc8     libcpmt:xlocale.obj
 0002:00002dd0       ?id@?$messages@D@std@@2V0locale@2@A 000000018005ddd0     libcpmt:xlocale.obj
 0002:00002dd8       ?id@?$money_get@DV?$istreambuf_iterator@DU?$char_traits@D@std@@@std@@@std@@2V0locale@2@A 000000018005ddd8     libcpmt:xlocale.obj
 0002:00002de0       ?id@?$money_put@DV?$ostreambuf_iterator@DU?$char_traits@D@std@@@std@@@std@@2V0locale@2@A 000000018005dde0     libcpmt:xlocale.obj
 0002:00002de8       ?id@?$moneypunct@D$0A@@std@@2V0locale@2@A 000000018005dde8     libcpmt:xlocale.obj
 0002:00002df0       ?id@?$moneypunct@D$00@std@@2V0locale@2@A 000000018005ddf0     libcpmt:xlocale.obj
 0002:00002df8       ?id@?$time_get@DV?$istreambuf_iterator@DU?$char_traits@D@std@@@std@@@std@@2V0locale@2@A 000000018005ddf8     libcpmt:xlocale.obj
 0002:00002e00       ?id@?$time_put@DV?$ostreambuf_iterator@DU?$char_traits@D@std@@@std@@@std@@2V0locale@2@A 000000018005de00     libcpmt:xlocale.obj
 0002:00002e08       __scrt_current_native_startup_state 000000018005de08     LIBCMT:utility.obj
 0002:00002e10       __scrt_native_startup_lock 000000018005de10     LIBCMT:utility.obj
 0002:00002e54       __favor                    000000018005de54     LIBCMT:cpu_disp.obj
 0002:00002e58       __scrt_debugger_hook_flag  000000018005de58     LIBCMT:utility_desktop.obj
 0002:00002e60       ?__type_info_root_node@@3U__type_info_node@@A 000000018005de60     LIBCMT:tncleanup.obj
 0002:00002e70       ?_OptionsStorage@?1??__local_stdio_scanf_options@@9@4_KA 000000018005de70     LIBCMT:default_local_stdio_options.obj
 0002:000033f0       ?__WinRTOutOfMemoryExceptionCallback@@3P6APEAXXZEA 000000018005e3f0     libvcruntime:ehhelpers.obj
 0002:000033f8       __pPurecall                000000018005e3f8     libvcruntime:purevirt_data.obj
 0002:000034b0       ?pArgList@UnDecorator@@0PEAVReplicator@@EA 000000018005e4b0     libvcruntime:undname.obj
 0002:000034b8       ?pZNameList@UnDecorator@@0PEAVReplicator@@EA 000000018005e4b8     libvcruntime:undname.obj
 0002:000034c0       ?pTemplateArgList@UnDecorator@@0PEAVReplicator@@EA 000000018005e4c0     libvcruntime:undname.obj
 0002:000034c8       ?gName@UnDecorator@@0PEBDEB 000000018005e4c8     libvcruntime:undname.obj
 0002:000034d0       ?name@UnDecorator@@0PEBDEB 000000018005e4d0     libvcruntime:undname.obj
 0002:000034d8       ?disableFlags@UnDecorator@@0KA 000000018005e4d8     libvcruntime:undname.obj
 0002:000034dc       ?fExplicitTemplateParams@UnDecorator@@0_NA 000000018005e4dc     libvcruntime:undname.obj
 0002:000034dd       ?fGetTemplateArgumentList@UnDecorator@@0_NA 000000018005e4dd     libvcruntime:undname.obj
 0002:000034e0       ?m_pGetParameter@UnDecorator@@0P6APEADJ@ZEA 000000018005e4e0     libvcruntime:undname.obj
 0002:000034e8       ?m_CHPENameOffset@UnDecorator@@0KA 000000018005e4e8     libvcruntime:undname.obj
 0002:000034ec       ?m_recursionLevel@UnDecorator@@0KA 000000018005e4ec     libvcruntime:undname.obj
 0002:00003560       _nstream                   000000018005e560     libucrt:_file.obj
 0002:00003568       __piob                     000000018005e568     libucrt:_file.obj
 0002:00003570       __acrt_lconv_static_null   000000018005e570     libucrt:localeconv.obj
 0002:00003574       __acrt_lconv_static_W_null 000000018005e574     libucrt:localeconv.obj
 0002:000037c0       ?c_exit_complete@?1???R<lambda_6e4b09c48022b2350581041d5f6b0c4c>@@QEBA@XZ@4_NA 000000018005e7c0     libucrt:exit.obj
 0002:000038d8       _environ_table             000000018005e8d8     libucrt:environment_initialization.obj
 0002:000038e0       _wenviron_table            000000018005e8e0     libucrt:environment_initialization.obj
 0002:000038e8       __dcrt_initial_wide_environment 000000018005e8e8     libucrt:environment_initialization.obj
 0002:000038f0       __dcrt_initial_narrow_environment 000000018005e8f0     libucrt:environment_initialization.obj
 0002:000038f8       __acrt_atexit_table        000000018005e8f8     libucrt:onexit.obj
 0002:00003910       __acrt_at_quick_exit_table 000000018005e910     libucrt:onexit.obj
 0002:00003af0       __pioinfo                  000000018005eaf0     libucrt:ioinit.obj
 0002:00003ef0       _nhandle                   000000018005eef0     libucrt:ioinit.obj
 0002:00003ef8       __acrt_stdout_buffer       000000018005eef8     libucrt:_sftbuf.obj
 0002:00003f00       __acrt_stderr_buffer       000000018005ef00     libucrt:_sftbuf.obj
 0002:00003f18       __acrt_locale_changed_data 000000018005ef18     libucrt:wsetlocale.obj
 0002:00003f20       __acrt_current_locale_data 000000018005ef20     libucrt:nlsdata.obj
 0002:00003f2c       __fma3_is_available        000000018005ef2c     libucrt:fma3_available.obj
 0002:00003f30       __use_fma3_lib             000000018005ef30     libucrt:fma3_available.obj
 0002:00003f58       ?_timezone@@3V?$dual_state_global@J@__crt_state_management@@A 000000018005ef58     libucrt:timeset.obj
 0002:00003f5c       ?_daylight@@3V?$dual_state_global@H@__crt_state_management@@A 000000018005ef5c     libucrt:timeset.obj
 0002:00003f60       ?_dstbias@@3V?$dual_state_global@J@__crt_state_management@@A 000000018005ef60     libucrt:timeset.obj
 0002:00004030       _mbctype                   000000018005f030     libucrt:mbctype.obj
 0002:00004038       _mbcasemap                 000000018005f038     libucrt:mbctype.obj
 0002:00004040       __acrt_current_multibyte_data 000000018005f040     libucrt:mbctype.obj
 0002:00004050       _pgmptr                    000000018005f050     libucrt:argv_data.obj
 0002:00004058       __argc                     000000018005f058     libucrt:argv_data.obj
 0002:00004060       __argv                     000000018005f060     libucrt:argv_data.obj
 0002:00004068       __wargv                    000000018005f068     libucrt:argv_data.obj
 0002:00004070       _acmdln                    000000018005f070     libucrt:argv_data.obj
 0002:00004078       _wcmdln                    000000018005f078     libucrt:argv_data.obj
 0002:00004080       __acrt_heap                000000018005f080     libucrt:heap_handle.obj
 0002:000040a8       __dyn_tls_init_callback    000000018005f0a8     <common>
 0002:000040b0       __scrt_ucrt_dll_is_in_use  000000018005f0b0     <common>
 0004:00000000       __imp_LookupPrivilegeValueW 0000000180063000     advapi32:ADVAPI32.dll
 0004:00000008       __imp_DuplicateTokenEx     0000000180063008     advapi32:ADVAPI32.dll
 0004:00000010       __imp_AdjustTokenPrivileges 0000000180063010     advapi32:ADVAPI32.dll
 0004:00000018       __imp_OpenThreadToken      0000000180063018     advapi32:ADVAPI32.dll
 0004:00000020       __imp_OpenProcessToken     0000000180063020     advapi32:ADVAPI32.dll
 0004:00000028       __imp_SetThreadToken       0000000180063028     advapi32:ADVAPI32.dll
 0004:00000030       __imp_RegQueryValueExW     0000000180063030     advapi32:ADVAPI32.dll
 0004:00000038       __imp_RegOpenKeyExW        0000000180063038     advapi32:ADVAPI32.dll
 0004:00000040       __imp_RegConnectRegistryW  0000000180063040     advapi32:ADVAPI32.dll
 0004:00000048       __imp_RegCloseKey          0000000180063048     advapi32:ADVAPI32.dll
 0004:00000050       __imp_ConvertSidToStringSidW 0000000180063050     advapi32:ADVAPI32.dll
 0004:00000058       __imp_GetUserNameW         0000000180063058     advapi32:ADVAPI32.dll
 0004:00000060       __imp_LookupAccountNameW   0000000180063060     advapi32:ADVAPI32.dll
 0004:00000068       \177ADVAPI32_NULL_THUNK_DATA 0000000180063068     advapi32:ADVAPI32.dll
 0004:00000070       __imp_CreateFileW          0000000180063070     kernel32:KERNEL32.dll
 0004:00000078       __imp_SetLastError         0000000180063078     kernel32:KERNEL32.dll
 0004:00000080       __imp_SetEvent             0000000180063080     kernel32:KERNEL32.dll
 0004:00000088       __imp_GetCurrentThreadId   0000000180063088     kernel32:KERNEL32.dll
 0004:00000090       __imp_SetPriorityClass     0000000180063090     kernel32:KERNEL32.dll
 0004:00000098       __imp_GetPriorityClass     0000000180063098     kernel32:KERNEL32.dll
 0004:000000a0       __imp_GetSystemTimeAsFileTime 00000001800630a0     kernel32:KERNEL32.dll
 0004:000000a8       __imp_GetLocalTime         00000001800630a8     kernel32:KERNEL32.dll
 0004:000000b0       __imp_GetTickCount         00000001800630b0     kernel32:KERNEL32.dll
 0004:000000b8       __imp_lstrcmpW             00000001800630b8     kernel32:KERNEL32.dll
 0004:000000c0       __imp_lstrcpynW            00000001800630c0     kernel32:KERNEL32.dll
 0004:000000c8       __imp_SystemTimeToTzSpecificLocalTime 00000001800630c8     kernel32:KERNEL32.dll
 0004:000000d0       __imp_FileTimeToSystemTime 00000001800630d0     kernel32:KERNEL32.dll
 0004:000000d8       __imp_ResetEvent           00000001800630d8     kernel32:KERNEL32.dll
 0004:000000e0       __imp_ReleaseMutex         00000001800630e0     kernel32:KERNEL32.dll
 0004:000000e8       __imp_CreateMutexW         00000001800630e8     kernel32:KERNEL32.dll
 0004:000000f0       __imp_CreateEventW         00000001800630f0     kernel32:KERNEL32.dll
 0004:000000f8       __imp_WaitForMultipleObjects 00000001800630f8     kernel32:KERNEL32.dll
 0004:00000100       __imp_GetProcessTimes      0000000180063100     kernel32:KERNEL32.dll
 0004:00000108       __imp_GetLastError         0000000180063108     kernel32:KERNEL32.dll
 0004:00000110       __imp_TerminateProcess     0000000180063110     kernel32:KERNEL32.dll
 0004:00000118       __imp_lstrlenW             0000000180063118     kernel32:KERNEL32.dll
 0004:00000120       __imp_OpenProcess          0000000180063120     kernel32:KERNEL32.dll
 0004:00000128       __imp_ReadProcessMemory    0000000180063128     kernel32:KERNEL32.dll
 0004:00000130       __imp_FileTimeToLocalFileTime 0000000180063130     kernel32:KERNEL32.dll
 0004:00000138       __imp_GetModuleHandleW     0000000180063138     kernel32:KERNEL32.dll
 0004:00000140       __imp_FormatMessageW       0000000180063140     kernel32:KERNEL32.dll
 0004:00000148       __imp_GetDateFormatW       0000000180063148     kernel32:KERNEL32.dll
 0004:00000150       __imp_GetTimeFormatW       0000000180063150     kernel32:KERNEL32.dll
 0004:00000158       __imp_GetProcAddress       0000000180063158     kernel32:KERNEL32.dll
 0004:00000160       __imp_HeapSize             0000000180063160     kernel32:KERNEL32.dll
 0004:00000168       __imp_FlushFileBuffers     0000000180063168     kernel32:KERNEL32.dll
 0004:00000170       __imp_GetProcessHeap       0000000180063170     kernel32:KERNEL32.dll
 0004:00000178       __imp_FreeEnvironmentStringsW 0000000180063178     kernel32:KERNEL32.dll
 0004:00000180       __imp_GetEnvironmentStringsW 0000000180063180     kernel32:KERNEL32.dll
 0004:00000188       __imp_GetCommandLineW      0000000180063188     kernel32:KERNEL32.dll
 0004:00000190       __imp_GetCommandLineA      0000000180063190     kernel32:KERNEL32.dll
 0004:00000198       __imp_GetOEMCP             0000000180063198     kernel32:KERNEL32.dll
 0004:000001a0       __imp_GetACP               00000001800631a0     kernel32:KERNEL32.dll
 0004:000001a8       __imp_IsValidCodePage      00000001800631a8     kernel32:KERNEL32.dll
 0004:000001b0       __imp_LocalFree            00000001800631b0     kernel32:KERNEL32.dll
 0004:000001b8       __imp_VirtualFree          00000001800631b8     kernel32:KERNEL32.dll
 0004:000001c0       __imp_VirtualAlloc         00000001800631c0     kernel32:KERNEL32.dll
 0004:000001c8       __imp_TerminateThread      00000001800631c8     kernel32:KERNEL32.dll
 0004:000001d0       __imp_CreateThread         00000001800631d0     kernel32:KERNEL32.dll
 0004:000001d8       __imp_GetCurrentProcessId  00000001800631d8     kernel32:KERNEL32.dll
 0004:000001e0       __imp_GetCurrentProcess    00000001800631e0     kernel32:KERNEL32.dll
 0004:000001e8       __imp_WaitForSingleObject  00000001800631e8     kernel32:KERNEL32.dll
 0004:000001f0       __imp_DuplicateHandle      00000001800631f0     kernel32:KERNEL32.dll
 0004:000001f8       __imp_CloseHandle          00000001800631f8     kernel32:KERNEL32.dll
 0004:00000200       __imp_GetFileType          0000000180063200     kernel32:KERNEL32.dll
 0004:00000208       __imp_WriteConsoleW        0000000180063208     kernel32:KERNEL32.dll
 0004:00000210       __imp_GetCurrentThread     0000000180063210     kernel32:KERNEL32.dll
 0004:00000218       __imp_WriteFile            0000000180063218     kernel32:KERNEL32.dll
 0004:00000220       __imp_FindNextFileW        0000000180063220     kernel32:KERNEL32.dll
 0004:00000228       __imp_FindFirstFileExW     0000000180063228     kernel32:KERNEL32.dll
 0004:00000230       __imp_FindClose            0000000180063230     kernel32:KERNEL32.dll
 0004:00000238       __imp_HeapReAlloc          0000000180063238     kernel32:KERNEL32.dll
 0004:00000240       __imp_GetConsoleMode       0000000180063240     kernel32:KERNEL32.dll
 0004:00000248       __imp_GetConsoleCP         0000000180063248     kernel32:KERNEL32.dll
 0004:00000250       __imp_SetFilePointerEx     0000000180063250     kernel32:KERNEL32.dll
 0004:00000258       __imp_GetStdHandle         0000000180063258     kernel32:KERNEL32.dll
 0004:00000260       __imp_EnumSystemLocalesW   0000000180063260     kernel32:KERNEL32.dll
 0004:00000268       __imp_GetUserDefaultLCID   0000000180063268     kernel32:KERNEL32.dll
 0004:00000270       __imp_IsValidLocale        0000000180063270     kernel32:KERNEL32.dll
 0004:00000278       __imp_HeapFree             0000000180063278     kernel32:KERNEL32.dll
 0004:00000280       __imp_HeapAlloc            0000000180063280     kernel32:KERNEL32.dll
 0004:00000288       __imp_GetModuleFileNameW   0000000180063288     kernel32:KERNEL32.dll
 0004:00000290       __imp_WideCharToMultiByte  0000000180063290     kernel32:KERNEL32.dll
 0004:00000298       __imp_MultiByteToWideChar  0000000180063298     kernel32:KERNEL32.dll
 0004:000002a0       __imp_EnterCriticalSection 00000001800632a0     kernel32:KERNEL32.dll
 0004:000002a8       __imp_LeaveCriticalSection 00000001800632a8     kernel32:KERNEL32.dll
 0004:000002b0       __imp_DeleteCriticalSection 00000001800632b0     kernel32:KERNEL32.dll
 0004:000002b8       __imp_EncodePointer        00000001800632b8     kernel32:KERNEL32.dll
 0004:000002c0       __imp_DecodePointer        00000001800632c0     kernel32:KERNEL32.dll
 0004:000002c8       __imp_InitializeCriticalSectionAndSpinCount 00000001800632c8     kernel32:KERNEL32.dll
 0004:000002d0       __imp_TlsAlloc             00000001800632d0     kernel32:KERNEL32.dll
 0004:000002d8       __imp_TlsGetValue          00000001800632d8     kernel32:KERNEL32.dll
 0004:000002e0       __imp_TlsSetValue          00000001800632e0     kernel32:KERNEL32.dll
 0004:000002e8       __imp_TlsFree              00000001800632e8     kernel32:KERNEL32.dll
 0004:000002f0       __imp_GetStringTypeW       00000001800632f0     kernel32:KERNEL32.dll
 0004:000002f8       __imp_LCMapStringW         00000001800632f8     kernel32:KERNEL32.dll
 0004:00000300       __imp_GetLocaleInfoW       0000000180063300     kernel32:KERNEL32.dll
 0004:00000308       __imp_GetCPInfo            0000000180063308     kernel32:KERNEL32.dll
 0004:00000310       __imp_RtlCaptureContext    0000000180063310     kernel32:KERNEL32.dll
 0004:00000318       __imp_RtlLookupFunctionEntry 0000000180063318     kernel32:KERNEL32.dll
 0004:00000320       __imp_RtlVirtualUnwind     0000000180063320     kernel32:KERNEL32.dll
 0004:00000328       __imp_IsDebuggerPresent    0000000180063328     kernel32:KERNEL32.dll
 0004:00000330       __imp_UnhandledExceptionFilter 0000000180063330     kernel32:KERNEL32.dll
 0004:00000338       __imp_SetUnhandledExceptionFilter 0000000180063338     kernel32:KERNEL32.dll
 0004:00000340       __imp_GetStartupInfoW      0000000180063340     kernel32:KERNEL32.dll
 0004:00000348       __imp_IsProcessorFeaturePresent 0000000180063348     kernel32:KERNEL32.dll
 0004:00000350       __imp_QueryPerformanceCounter 0000000180063350     kernel32:KERNEL32.dll
 0004:00000358       __imp_InitializeSListHead  0000000180063358     kernel32:KERNEL32.dll
 0004:00000360       __imp_RtlPcToFileHeader    0000000180063360     kernel32:KERNEL32.dll
 0004:00000368       __imp_RaiseException       0000000180063368     kernel32:KERNEL32.dll
 0004:00000370       __imp_RtlUnwindEx          0000000180063370     kernel32:KERNEL32.dll
 0004:00000378       __imp_InterlockedFlushSList 0000000180063378     kernel32:KERNEL32.dll
 0004:00000380       __imp_FreeLibrary          0000000180063380     kernel32:KERNEL32.dll
 0004:00000388       __imp_LoadLibraryExW       0000000180063388     kernel32:KERNEL32.dll
 0004:00000390       __imp_SetStdHandle         0000000180063390     kernel32:KERNEL32.dll
 0004:00000398       __imp_ExitProcess          0000000180063398     kernel32:KERNEL32.dll
 0004:000003a0       __imp_GetModuleHandleExW   00000001800633a0     kernel32:KERNEL32.dll
 0004:000003a8       \177KERNEL32_NULL_THUNK_DATA 00000001800633a8     kernel32:KERNEL32.dll
 0004:000003b0       __imp_WNetCancelConnection2W 00000001800633b0     mpr:MPR.dll
 0004:000003b8       __imp_WNetAddConnection2W  00000001800633b8     mpr:MPR.dll
 0004:000003c0       \177MPR_NULL_THUNK_DATA    00000001800633c0     mpr:MPR.dll
 0004:000003c8       __imp_VariantClear         00000001800633c8     oleaut32:OLEAUT32.dll
 0004:000003d0       __imp_SysFreeString        00000001800633d0     oleaut32:OLEAUT32.dll
 0004:000003d8       __imp_SysAllocString       00000001800633d8     oleaut32:OLEAUT32.dll
 0004:000003e0       \177OLEAUT32_NULL_THUNK_DATA 00000001800633e0     oleaut32:OLEAUT32.dll
 0004:000003e8       __imp_GetModuleInformation 00000001800633e8     psapi:PSAPI.DLL
 0004:000003f0       __imp_GetModuleFileNameExW 00000001800633f0     psapi:PSAPI.DLL
 0004:000003f8       \177PSAPI_NULL_THUNK_DATA  00000001800633f8     psapi:PSAPI.DLL
 0004:00000400       __imp_GetWindowTextW       0000000180063400     user32:USER32.dll
 0004:00000408       __imp_SetForegroundWindow  0000000180063408     user32:USER32.dll
 0004:00000410       __imp_ShowWindowAsync      0000000180063410     user32:USER32.dll
 0004:00000418       __imp_IsWindowVisible      0000000180063418     user32:USER32.dll
 0004:00000420       __imp_IsIconic             0000000180063420     user32:USER32.dll
 0004:00000428       __imp_GetWindowLongPtrW    0000000180063428     user32:USER32.dll
 0004:00000430       __imp_GetParent            0000000180063430     user32:USER32.dll
 0004:00000438       __imp_GetAncestor          0000000180063438     user32:USER32.dll
 0004:00000440       __imp_GetLastActivePopup   0000000180063440     user32:USER32.dll
 0004:00000448       __imp_GetWindowThreadProcessId 0000000180063448     user32:USER32.dll
 0004:00000450       __imp_EnumWindows          0000000180063450     user32:USER32.dll
 0004:00000458       __imp_CharUpperBuffW       0000000180063458     user32:USER32.dll
 0004:00000460       \177USER32_NULL_THUNK_DATA 0000000180063460     user32:USER32.dll
 0004:00000468       __imp_VerQueryValueW       0000000180063468     version:VERSION.dll
 0004:00000470       __imp_GetFileVersionInfoSizeW 0000000180063470     version:VERSION.dll
 0004:00000478       __imp_GetFileVersionInfoW  0000000180063478     version:VERSION.dll
 0004:00000480       \177VERSION_NULL_THUNK_DATA 0000000180063480     version:VERSION.dll
 0004:00000488       __imp_CoUninitialize       0000000180063488     ole32:ole32.dll
 0004:00000490       __imp_CoCreateInstance     0000000180063490     ole32:ole32.dll
 0004:00000498       __imp_CoInitialize         0000000180063498     ole32:ole32.dll
 0004:000004a0       \177ole32_NULL_THUNK_DATA  00000001800634a0     ole32:ole32.dll
 0004:000004a8       __guard_check_icall_fptr   00000001800634a8     LIBCMT:guard_support.obj
 0004:000004b0       __guard_dispatch_icall_fptr 00000001800634b0     LIBCMT:guard_support.obj
 0004:000004b8       __IMPORT_DESCRIPTOR_KERNEL32 00000001800634b8     kernel32:KERNEL32.dll
 0004:000004cc       __IMPORT_DESCRIPTOR_USER32 00000001800634cc     user32:USER32.dll
 0004:000004e0       __IMPORT_DESCRIPTOR_ADVAPI32 00000001800634e0     advapi32:ADVAPI32.dll
 0004:000004f4       __IMPORT_DESCRIPTOR_ole32  00000001800634f4     ole32:ole32.dll
 0004:00000508       __IMPORT_DESCRIPTOR_MPR    0000000180063508     mpr:MPR.dll
 0004:0000051c       __IMPORT_DESCRIPTOR_VERSION 000000018006351c     version:VERSION.dll
 0004:00000530       __IMPORT_DESCRIPTOR_OLEAUT32 0000000180063530     oleaut32:OLEAUT32.dll
 0004:00000544       __IMPORT_DESCRIPTOR_PSAPI  0000000180063544     psapi:PSAPI.DLL
 0004:00000558       __NULL_IMPORT_DESCRIPTOR   0000000180063558     kernel32:KERNEL32.dll

 entry point at        0001:000371a0

 Static symbols

 0001:00000008       ?initlocks$initializer$@std@@3P6AXXZEA 0000000180001008     libcpmt:xlock.obj
 0001:00000010       ?initlocks$initializer$@std@@3P6AXXZEA 0000000180001010     libcpmt:iosptrs.obj
 0001:00000018       ?init_atexit$initializer$@@3P6AXXZEA 0000000180001018     libcpmt:iosptrs.obj
 0001:00000020       ?_Fac_tidy_reg$initializer$@std@@3P6AXXZEA 0000000180001020     libcpmt:locale0.obj
 0001:00000028       ?classic_locale$initializer$@std@@3P6AXXZEA 0000000180001028     libcpmt:locale0.obj
 0001:00000030       ??m_PanelModesDataLocal$initializer$@Plist@@0P6AXXZEA@@3P6AXXZEA 0000000180001030     fileio.obj
 0001:00000038       ??m_PanelModesDataRemote$initializer$@Plist@@0P6AXXZEA@@3P6AXXZEA 0000000180001038     fileio.obj
 0001:00000040       ?hDebugToken$initializer$@@3P6AXXZEA 0000000180001040     Plist.obj
 0001:00000058       ?pinit@@3P6AHXZEA          0000000180001058     libcpmt:winapisupp.obj
 0001:00000060       pinit                      0000000180001060     LIBCMT:lconv_unsigned_char.obj
 0001:00000a60       ?constStrTypes@@3QBQEB_WB  0000000180001a60     handles.obj
 0001:00000e60       ?StatusCols@?1??InitializePanelModes@Plist@@SAXXZ@4QB_WB 0000000180001e60     Pclass.obj
 0001:00000e70       ?StatusWidths@?1??InitializePanelModes@Plist@@SAXXZ@4QB_WB 0000000180001e70     Pclass.obj
 0001:00001710       ?invalid_chars@?1??GetFiles@Plist@@QEAAHPEAUPluginPanelItem@@_KHPEAPEB_W1AEAUoptions@@@Z@4QB_WB 0000000180002710     Pclass.obj
 0001:00001868       ?PrClasses@?EH@??ProcessKey@Plist@@QEAAHPEBU_INPUT_RECORD@@@Z@4QBGB 0000000180002868     Pclass.obj
 0001:00001874       ?Pr@?HF@??ProcessKey@Plist@@QEAAHPEBU_INPUT_RECORD@@@Z@4QBEB 0000000180002874     Pclass.obj
 0001:000021d8       ??_7?$_Func_impl_no_alloc@V<lambda_87e110110aa5c29eaf754372c3484d5b>@@_NPEA_W_K@std@@6B@ 00000001800031d8     Plist.obj
 0001:00002418       ??_7?$_Func_impl_no_alloc@V<lambda_aac7a801b46524f039ecb4f6852a8dbe>@@XAEBUtagVARIANT@@@std@@6B@ 0000000180003418     WMI.obj
 0001:00002448       ??_7?$_Func_impl_no_alloc@V<lambda_6ecd11d6a952986d4bf89c34edf08f5f>@@XAEBUtagVARIANT@@@std@@6B@ 0000000180003448     WMI.obj
 0001:00002808       $cppxdata$?_Init@locale@std@@CAPEAV_Locimp@12@_N@Z 0000000180003808     libcpmt:locale0.obj
 0001:000028a8       $cppxdata$??__Finit_atexit@@YAXXZ 00000001800038a8     libcpmt:iosptrs.obj
 0001:00002d18       digits                     0000000180003d18     libcpmt:xstoul.obj
 0001:00002d40       ndigs                      0000000180003d40     libcpmt:xstoul.obj
 0001:00002d68       digits                     0000000180003d68     libcpmt:xstoull.obj
 0001:00002d90       ndigs                      0000000180003d90     libcpmt:xstoull.obj
 0001:00002dc0       ?LcidToLocaleNameTable@@3QBULcidToLocaleName@@B 0000000180003dc0     libcpmt:winapinls.obj
 0001:00003c00       ?LocaleNameToIndexTable@@3QBULocaleNameIndex@@B 0000000180004c00     libcpmt:winapinls.obj
 0001:00006118       GS_ExceptionPointers       0000000180007118     LIBCMT:gs_report.obj
 0001:00006150       ?ExceptionTemplate@?1??UnwindNestedFrames@__FrameHandler4@@SAXPEA_KPEAUEHExceptionRecord@@PEAU_CONTEXT@@0PEAXPEAUFuncInfo4@FH4@@HHPEAUHandlerType4@6@PEAU_xDISPATCHER_CONTEXT@@E@Z@4U_EXCEPTION_RECORD@@B 0000000180007150     libvcruntime:risctrnsctrl.obj
 0001:000061f0       ?ExceptionTemplate@?1??UnwindNestedFrames@__FrameHandler3@@SAXPEA_KPEAUEHExceptionRecord@@PEAU_CONTEXT@@0PEAXPEBU_s_FuncInfo@@HHPEBU_s_HandlerType@@PEAU_xDISPATCHER_CONTEXT@@E@Z@4U_EXCEPTION_RECORD@@B 00000001800071f0     libvcruntime:risctrnsctrl.obj
 0001:000062b0       ?tokenTable@@3QBUStringLiteral@@B 00000001800072b0     libvcruntime:undname.obj
 0001:000063b0       ?nameTable@@3QBUStringLiteral@@B 00000001800073b0     libvcruntime:undname.obj
 0001:000068e0       ?rttiTable@@3QBUStringLiteral@@B 00000001800078e0     libvcruntime:undname.obj
 0001:00006930       ?IndirectionName@@3QBUStringLiteral@@B 0000000180007930     libvcruntime:undname.obj
 0001:00006990       ?PrefixName@@3QBUStringLiteral@@B 0000000180007990     libvcruntime:undname.obj
 0001:00007060       ?module_names@?A0x81a78551@@3QBQEB_WB 0000000180008060     libvcruntime:winapi_downlevel.obj
 0001:00007108       ?candidate_modules@?1??try_get_FlsAlloc@@YAP6AKP6AXPEAX@Z@ZXZ@4QBW4module_id@?A0x81a78551@@B 0000000180008108     libvcruntime:winapi_downlevel.obj
 0001:00007110       ?candidate_modules@?1??try_get_FlsFree@@YAP6AHK@ZXZ@4QBW4module_id@?A0x81a78551@@B 0000000180008110     libvcruntime:winapi_downlevel.obj
 0001:00007118       ?candidate_modules@?1??try_get_FlsGetValue@@YAP6APEAXK@ZXZ@4QBW4module_id@?A0x81a78551@@B 0000000180008118     libvcruntime:winapi_downlevel.obj
 0001:00007120       ?candidate_modules@?1??try_get_FlsSetValue@@YAP6AHKPEAX@ZXZ@4QBW4module_id@?A0x81a78551@@B 0000000180008120     libvcruntime:winapi_downlevel.obj
 0001:00007128       ?candidate_modules@?1??try_get_InitializeCriticalSectionEx@@YAP6AHPEAU_RTL_CRITICAL_SECTION@@KK@ZXZ@4QBW4module_id@?A0x81a78551@@B 0000000180008128     libvcruntime:winapi_downlevel.obj
 0001:00007130       ?errtable@@3QBUerrentry@?A0x31fdb9ec@@B 0000000180008130     libucrt:errno.obj
 0001:00007320       ?ln_lead_table@?1??log2@@9@9 0000000180008320     libucrt:log2.obj
 0001:00007530       ?ln_tail_table@?1??log2@@9@9 0000000180008530     libucrt:log2.obj
 0001:000077c0       __real_ninf                00000001800087c0     libucrt:log10.obj
 0001:000077d0       __real_inf                 00000001800087d0     libucrt:log10.obj
 0001:000077e0       __real_neg_qnan            00000001800087e0     libucrt:log10.obj
 0001:000077f0       __real_qnanbit             00000001800087f0     libucrt:log10.obj
 0001:00007800       __int_1023                 0000000180008800     libucrt:log10.obj
 0001:00007810       __mask_001                 0000000180008810     libucrt:log10.obj
 0001:00007820       __mask_mant                0000000180008820     libucrt:log10.obj
 0001:00007830       __mask_mant_top8           0000000180008830     libucrt:log10.obj
 0001:00007840       __mask_mant9               0000000180008840     libucrt:log10.obj
 0001:00007850       __real_log10_e             0000000180008850     libucrt:log10.obj
 0001:00007860       __real_log10_e_lead        0000000180008860     libucrt:log10.obj
 0001:00007870       __real_log10_e_tail        0000000180008870     libucrt:log10.obj
 0001:00007880       __real_log10_2_lead        0000000180008880     libucrt:log10.obj
 0001:00007890       __real_log10_2_tail        0000000180008890     libucrt:log10.obj
 0001:000078a0       __real_two                 00000001800088a0     libucrt:log10.obj
 0001:000078b0       __real_one                 00000001800088b0     libucrt:log10.obj
 0001:000078c0       __real_half                00000001800088c0     libucrt:log10.obj
 0001:000078d0       __mask_100                 00000001800088d0     libucrt:log10.obj
 0001:000078e0       __real_1_over_512          00000001800088e0     libucrt:log10.obj
 0001:000078f0       __real_1_over_2            00000001800088f0     libucrt:log10.obj
 0001:00007900       __real_1_over_3            0000000180008900     libucrt:log10.obj
 0001:00007910       __real_1_over_4            0000000180008910     libucrt:log10.obj
 0001:00007920       __real_1_over_5            0000000180008920     libucrt:log10.obj
 0001:00007930       __real_1_over_6            0000000180008930     libucrt:log10.obj
 0001:00007940       __real_neg_1023            0000000180008940     libucrt:log10.obj
 0001:00007950       __mask_2045                0000000180008950     libucrt:log10.obj
 0001:00007960       __real_threshold           0000000180008960     libucrt:log10.obj
 0001:00007970       __real_near_one_lt         0000000180008970     libucrt:log10.obj
 0001:00007980       __real_near_one_gt         0000000180008980     libucrt:log10.obj
 0001:00007990       __real_min_norm            0000000180008990     libucrt:log10.obj
 0001:000079a0       __real_notsign             00000001800089a0     libucrt:log10.obj
 0001:000079b0       __real_ca1                 00000001800089b0     libucrt:log10.obj
 0001:000079c0       __real_ca2                 00000001800089c0     libucrt:log10.obj
 0001:000079d0       __real_ca3                 00000001800089d0     libucrt:log10.obj
 0001:000079e0       __real_ca4                 00000001800089e0     libucrt:log10.obj
 0001:000079f0       __mask_lower               00000001800089f0     libucrt:log10.obj
 0001:00007a00       __flag_x_zero              0000000180008a00     libucrt:log10.obj
 0001:00007a04       __flag_x_neg               0000000180008a04     libucrt:log10.obj
 0001:00007a08       __flag_x_nan               0000000180008a08     libucrt:log10.obj
 0001:00007a10       __flag_x_one_y_snan        0000000180008a10     libucrt:pow.obj
 0001:00007a14       __flag_x_zero_z_inf        0000000180008a14     libucrt:pow.obj
 0001:00007a18       __flag_x_nan               0000000180008a18     libucrt:pow.obj
 0001:00007a1c       __flag_y_nan               0000000180008a1c     libucrt:pow.obj
 0001:00007a20       __flag_x_nan_y_nan         0000000180008a20     libucrt:pow.obj
 0001:00007a24       __flag_x_neg_y_notint      0000000180008a24     libucrt:pow.obj
 0001:00007a28       __flag_z_zero              0000000180008a28     libucrt:pow.obj
 0001:00007a2c       __flag_z_denormal          0000000180008a2c     libucrt:pow.obj
 0001:00007a30       __flag_z_inf               0000000180008a30     libucrt:pow.obj
 0001:00007a40       __ay_max_bound             0000000180008a40     libucrt:pow.obj
 0001:00007a48       __ay_min_bound             0000000180008a48     libucrt:pow.obj
 0001:00007a50       __sign_mask                0000000180008a50     libucrt:pow.obj
 0001:00007a58       __sign_and_exp_mask        0000000180008a58     libucrt:pow.obj
 0001:00007a60       __exp_mask                 0000000180008a60     libucrt:pow.obj
 0001:00007a68       __neg_inf                  0000000180008a68     libucrt:pow.obj
 0001:00007a70       __pos_inf                  0000000180008a70     libucrt:pow.obj
 0001:00007a78       __pos_one                  0000000180008a78     libucrt:pow.obj
 0001:00007a80       __pos_zero                 0000000180008a80     libucrt:pow.obj
 0001:00007a88       __exp_mant_mask            0000000180008a88     libucrt:pow.obj
 0001:00007a90       __mant_mask                0000000180008a90     libucrt:pow.obj
 0001:00007a98       __ind_pattern              0000000180008a98     libucrt:pow.obj
 0001:00007aa0       __neg_qnan                 0000000180008aa0     libucrt:pow.obj
 0001:00007aa8       __qnan                     0000000180008aa8     libucrt:pow.obj
 0001:00007ab0       __qnan_set                 0000000180008ab0     libucrt:pow.obj
 0001:00007ab8       __neg_one                  0000000180008ab8     libucrt:pow.obj
 0001:00007ac0       __neg_zero                 0000000180008ac0     libucrt:pow.obj
 0001:00007ac8       __exp_shift                0000000180008ac8     libucrt:pow.obj
 0001:00007ad0       __exp_bias                 0000000180008ad0     libucrt:pow.obj
 0001:00007ad8       __exp_bias_m1              0000000180008ad8     libucrt:pow.obj
 0001:00007ae0       __yexp_53                  0000000180008ae0     libucrt:pow.obj
 0001:00007ae8       __mant_full                0000000180008ae8     libucrt:pow.obj
 0001:00007af0       __1_before_mant            0000000180008af0     libucrt:pow.obj
 0001:00007af8       __mask_mant_all8           0000000180008af8     libucrt:pow.obj
 0001:00007b00       __mask_mant9               0000000180008b00     libucrt:pow.obj
 0001:00007b10       __real_fffffffff8000000    0000000180008b10     libucrt:pow.obj
 0001:00007b20       __mask_8000000000000000    0000000180008b20     libucrt:pow.obj
 0001:00007b30       __real_4090040000000000    0000000180008b30     libucrt:pow.obj
 0001:00007b40       __real_C090C80000000000    0000000180008b40     libucrt:pow.obj
 0001:00007b50       __real_ninf                0000000180008b50     libucrt:pow.obj
 0001:00007b60       __real_inf                 0000000180008b60     libucrt:pow.obj
 0001:00007b70       __real_nan                 0000000180008b70     libucrt:pow.obj
 0001:00007b80       __real_mant                0000000180008b80     libucrt:pow.obj
 0001:00007b90       __mask_1023                0000000180008b90     libucrt:pow.obj
 0001:00007ba0       __mask_001                 0000000180008ba0     libucrt:pow.obj
 0001:00007bb0       __real_log2_lead           0000000180008bb0     libucrt:pow.obj
 0001:00007bc0       __real_log2_tail           0000000180008bc0     libucrt:pow.obj
 0001:00007bd0       __real_two                 0000000180008bd0     libucrt:pow.obj
 0001:00007be0       __real_one                 0000000180008be0     libucrt:pow.obj
 0001:00007bf0       __real_half                0000000180008bf0     libucrt:pow.obj
 0001:00007c00       __mask_100                 0000000180008c00     libucrt:pow.obj
 0001:00007c10       __real_1_over_2            0000000180008c10     libucrt:pow.obj
 0001:00007c20       __real_1_over_3            0000000180008c20     libucrt:pow.obj
 0001:00007c30       __real_1_over_4            0000000180008c30     libucrt:pow.obj
 0001:00007c40       __real_1_over_5            0000000180008c40     libucrt:pow.obj
 0001:00007c50       __real_1_over_6            0000000180008c50     libucrt:pow.obj
 0001:00007c60       __real_1_over_7            0000000180008c60     libucrt:pow.obj
 0001:00007c70       __mask_1023_f              0000000180008c70     libucrt:pow.obj
 0001:00007c80       __mask_2045                0000000180008c80     libucrt:pow.obj
 0001:00007c90       __real_threshold           0000000180008c90     libucrt:pow.obj
 0001:00007ca0       __real_notsign             0000000180008ca0     libucrt:pow.obj
 0001:00007cb0       __log_F_inv_head           0000000180008cb0     libucrt:pow.obj
 0001:000084c0       __log_F_inv_tail           00000001800094c0     libucrt:pow.obj
 0001:00008cd0       __denormal_threshold       0000000180009cd0     libucrt:pow.obj
 0001:00008ce0       __enable_almost_inf        0000000180009ce0     libucrt:pow.obj
 0001:00008cf0       __real_zero                0000000180009cf0     libucrt:pow.obj
 0001:00008d00       __real_smallest_denormal   0000000180009d00     libucrt:pow.obj
 0001:00008d10       __denormal_tiny_threshold  0000000180009d10     libucrt:pow.obj
 0001:00008d20       __real_p65536              0000000180009d20     libucrt:pow.obj
 0001:00008d30       __real_m68800              0000000180009d30     libucrt:pow.obj
 0001:00008d40       __real_64_by_log2          0000000180009d40     libucrt:pow.obj
 0001:00008d50       __real_log2_by_64_head     0000000180009d50     libucrt:pow.obj
 0001:00008d60       __real_log2_by_64_tail     0000000180009d60     libucrt:pow.obj
 0001:00008d70       __real_1_by_720            0000000180009d70     libucrt:pow.obj
 0001:00008d80       __real_1_by_120            0000000180009d80     libucrt:pow.obj
 0001:00008d90       __real_1_by_24             0000000180009d90     libucrt:pow.obj
 0001:00008da0       __real_1_by_6              0000000180009da0     libucrt:pow.obj
 0001:00008db0       __real_1_by_2              0000000180009db0     libucrt:pow.obj
 0001:00009f00       __flag_x_one_y_snan        000000018000af00     libucrt:powf.obj
 0001:00009f04       __flag_x_zero_z_inf        000000018000af04     libucrt:powf.obj
 0001:00009f08       __flag_x_nan               000000018000af08     libucrt:powf.obj
 0001:00009f0c       __flag_y_nan               000000018000af0c     libucrt:powf.obj
 0001:00009f10       __flag_x_nan_y_nan         000000018000af10     libucrt:powf.obj
 0001:00009f14       __flag_x_neg_y_notint      000000018000af14     libucrt:powf.obj
 0001:00009f18       __flag_z_zero              000000018000af18     libucrt:powf.obj
 0001:00009f1c       __flag_z_denormal          000000018000af1c     libucrt:powf.obj
 0001:00009f20       __flag_z_inf               000000018000af20     libucrt:powf.obj
 0001:00009f24       L__1_by_3                  000000018000af24     libucrt:powf.obj
 0001:00009f2c       L__log2                    000000018000af2c     libucrt:powf.obj
 0001:00009f34       L__max_exp_arg             000000018000af34     libucrt:powf.obj
 0001:00009f3c       L__min_exp_arg             000000018000af3c     libucrt:powf.obj
 0001:00009f44       L__real_log2_by_64         000000018000af44     libucrt:powf.obj
 0001:00009f4c       L__1_by_6                  000000018000af4c     libucrt:powf.obj
 0001:00009f54       L__real_threshold          000000018000af54     libucrt:powf.obj
 0001:00009f5c       L__real_one                000000018000af5c     libucrt:powf.obj
 0001:00009f64       L__real_two                000000018000af64     libucrt:powf.obj
 0001:00009f6c       L__neg_zero                000000018000af6c     libucrt:powf.obj
 0001:00009f80       L__real_ca42               000000018000af80     libucrt:powf.obj
 0001:00009f88       L__real_ca4                000000018000af88     libucrt:powf.obj
 0001:00009f90       L__real_ca31               000000018000af90     libucrt:powf.obj
 0001:00009f98       L__real_ca3                000000018000af98     libucrt:powf.obj
 0001:00009fa0       L__clear_sign              000000018000afa0     libucrt:powf.obj
 0001:00009fb0       L__real_64_by_log2         000000018000afb0     libucrt:powf.obj
 0001:00009fc0       L__1_by_2                  000000018000afc0     libucrt:powf.obj
 0001:00009fd0       L__1023                    000000018000afd0     libucrt:powf.obj
 0001:00009fe0       L__xexp_bits_xmantissa_bits 000000018000afe0     libucrt:powf.obj
 0001:0000a900       __acrt_initializers        000000018000b900     libucrt:initialization.obj
 0001:0000aa00       ?mask@?P@??_d_int@@9@4QBGB 000000018000ba00     libucrt:_test.obj
 0001:0000aa20       ?sub@?P@??_d_int@@9@4QB_KB 000000018000ba20     libucrt:_test.obj
 0001:0000aa40       ?module_names@?A0x391cf84c@@3QBQEB_WB 000000018000ba40     libucrt:winapi_thunks.obj
 0001:0000af08       ?candidate_modules@?1??try_get_AreFileApisANSI@@YAP6AHXZXZ@4QBW4module_id@?A0x391cf84c@@B 000000018000bf08     libucrt:winapi_thunks.obj
 0001:0000af20       ?candidate_modules@?1??try_get_CompareStringEx@@YAP6AHPEB_WK0H0HPEAU_nlsversioninfo@@PEAX_J@ZXZ@4QBW4module_id@?A0x391cf84c@@B 000000018000bf20     libucrt:winapi_thunks.obj
 0001:0000af28       ?candidate_modules@?1??try_get_EnumSystemLocalesEx@@YAP6AHP6AHPEA_WK_J@ZK1PEAX@ZXZ@4QBW4module_id@?A0x391cf84c@@B 000000018000bf28     libucrt:winapi_thunks.obj
 0001:0000af48       ?candidate_modules@?1??try_get_FlsAlloc@@YAP6AKP6AXPEAX@Z@ZXZ@4QBW4module_id@?A0x391cf84c@@B 000000018000bf48     libucrt:winapi_thunks.obj
 0001:0000af50       ?candidate_modules@?1??try_get_FlsFree@@YAP6AHK@ZXZ@4QBW4module_id@?A0x391cf84c@@B 000000018000bf50     libucrt:winapi_thunks.obj
 0001:0000af58       ?candidate_modules@?1??try_get_FlsGetValue@@YAP6APEAXK@ZXZ@4QBW4module_id@?A0x391cf84c@@B 000000018000bf58     libucrt:winapi_thunks.obj
 0001:0000af60       ?candidate_modules@?1??try_get_FlsSetValue@@YAP6AHKPEAX@ZXZ@4QBW4module_id@?A0x391cf84c@@B 000000018000bf60     libucrt:winapi_thunks.obj
 0001:0000af68       ?candidate_modules@?1??try_get_GetDateFormatEx@@YAP6AHPEB_WKPEBU_SYSTEMTIME@@0PEA_WH0@ZXZ@4QBW4module_id@?A0x391cf84c@@B 000000018000bf68     libucrt:winapi_thunks.obj
 0001:0000af80       ?candidate_modules@?1??try_get_GetLocaleInfoEx@@YAP6AHPEB_WKPEA_WH@ZXZ@4QBW4module_id@?A0x391cf84c@@B 000000018000bf80     libucrt:winapi_thunks.obj
 0001:0000af88       ?candidate_modules@?1??try_get_GetTimeFormatEx@@YAP6AHPEB_WKPEBU_SYSTEMTIME@@0PEA_WH@ZXZ@4QBW4module_id@?A0x391cf84c@@B 000000018000bf88     libucrt:winapi_thunks.obj
 0001:0000afa0       ?candidate_modules@?1??try_get_GetUserDefaultLocaleName@@YAP6AHPEA_WH@ZXZ@4QBW4module_id@?A0x391cf84c@@B 000000018000bfa0     libucrt:winapi_thunks.obj
 0001:0000afc8       ?candidate_modules@?1??try_get_InitializeCriticalSectionEx@@YAP6AHPEAU_RTL_CRITICAL_SECTION@@KK@ZXZ@4QBW4module_id@?A0x391cf84c@@B 000000018000bfc8     libucrt:winapi_thunks.obj
 0001:0000afd0       ?candidate_modules@?1??try_get_IsValidLocaleName@@YAP6AHPEB_W@ZXZ@4QBW4module_id@?A0x391cf84c@@B 000000018000bfd0     libucrt:winapi_thunks.obj
 0001:0000aff0       ?candidate_modules@?1??try_get_LCMapStringEx@@YAP6AHPEB_WK0HPEA_WHPEAU_nlsversioninfo@@PEAX_J@ZXZ@4QBW4module_id@?A0x391cf84c@@B 000000018000bff0     libucrt:winapi_thunks.obj
 0001:0000aff8       ?candidate_modules@?1??try_get_LCIDToLocaleName@@YAP6AHKPEA_WHK@ZXZ@4QBW4module_id@?A0x391cf84c@@B 000000018000bff8     libucrt:winapi_thunks.obj
 0001:0000b018       ?candidate_modules@?1??try_get_LocaleNameToLCID@@YAP6AKPEB_WK@ZXZ@4QBW4module_id@?A0x391cf84c@@B 000000018000c018     libucrt:winapi_thunks.obj
 0001:0000b034       ?candidate_modules@?1??try_get_AppPolicyGetProcessTerminationMethod@@YAP6AJPEAXPEAW4AppPolicyProcessTerminationMethod@@@ZXZ@4QBW4module_id@?A0x391cf84c@@B 000000018000c034     libucrt:winapi_thunks.obj
 0001:0000b060       ?strings@?1??fp_format_nan_or_infinity@@YAHW4__acrt_fp_class@@_NPEAD_K1@Z@4QAY03QEBDA 000000018000c060     libucrt:cvt.obj
 0001:0000b130       _first_127char             000000018000c130     libucrt:wsetlocale.obj
 0001:0000e5d0       $cppxdata$?_wcstombs_l_helper@@YA_KPEADPEB_W_KPEAU__crt_locale_pointers@@@Z 000000018000f5d0     libucrt:wcstombs.obj
 0001:0000e800       ?_mb_locale_names@@3QBQEB_WB 000000018000f800     libucrt:mbctype.obj
 0001:0000e820       ?LcidToLocaleNameTable@?A0x881e4c05@@3QBULcidToLocaleName@1@B 000000018000f820     libucrt:lcidtoname_downlevel.obj
 0001:0000f660       ?LocaleNameToIndexTable@?A0x881e4c05@@3QBULocaleNameIndex@1@B 0000000180010660     libucrt:lcidtoname_downlevel.obj
 0001:000104a0       ?large_power_indices@?1??multiply_by_power_of_ten@__crt_strtox@@YA_NAEAUbig_integer@2@I@Z@4QBUunpack_index@?1??12@YA_N0I@Z@B 00000001800114a0     libucrt:cfout.obj
 0001:00011550       __real@433fffffffffffff    0000000180012550     libucrt:fpsr.obj
 0001:00011558       __real@c33fffffffffffff    0000000180012558     libucrt:fpsr.obj
 0001:000121e0       ??__E?m_PanelModesDataLocal@Plist@@0V?$vector@Umode@@V?$allocator@Umode@@@std@@@std@@A@@YAXXZ 00000001800131e0 f   fileio.obj
 0001:000121f0       ??__E?m_PanelModesDataRemote@Plist@@0V?$vector@Umode@@V?$allocator@Umode@@@std@@@std@@A@@YAXXZ 00000001800131f0 f   fileio.obj
 0001:00012200       ??__EhDebugToken@@YAXXZ    0000000180013200 f   Plist.obj
 0001:0001220c       ??__Einitlocks@std@@YAXXZ  000000018001320c f   libcpmt:xlock.obj
 0001:0001222c       ??__E_Fac_tidy_reg@std@@YAXXZ 000000018001322c f   libcpmt:locale0.obj
 0001:00012238       ??__Eclassic_locale@std@@YAXXZ 0000000180013238 f   libcpmt:locale0.obj
 0001:00012244       ??__Einit_atexit@@YAXXZ    0000000180013244 f   libcpmt:iosptrs.obj
 0001:00012250       ??__Einitlocks@std@@YAXXZ  0000000180013250 f   libcpmt:iosptrs.obj
 0001:00012270       $$000000                   0000000180013270     chkstk.obj
 0001:00014afc       $LN130                     0000000180015afc     format.obj
 0001:00014ea0       $LN110                     0000000180015ea0     format.obj
 0001:00017260       $LN62                      0000000180018260     handles.obj
 0001:00017330       $LN62                      0000000180018330     handles.obj
 0001:00017724       $LN93                      0000000180018724     handles.obj
 0001:00017740       $LN92                      0000000180018740     handles.obj
 0001:00017a54       $LN93                      0000000180018a54     handles.obj
 0001:00017a70       $LN92                      0000000180018a70     handles.obj
 0001:00018660       $LN17                      0000000180019660     handles.obj
 0001:0001868c       $LN16                      000000018001968c     handles.obj
 0001:0001969c       $LN130                     000000018001a69c     handles.obj
 0001:00019e18       $LN223                     000000018001ae18     handles.obj
 0001:0001c3a0       ??$write_padded@$01V?$back_insert_iterator@V?$buffer@_W@detail@v6@fmt@@@std@@_WV<lambda_2c6139bafe179ad98da6b2e77db1d169>@@@detail@v6@fmt@@YA?AV?$back_insert_iterator@V?$buffer@_W@detail@v6@fmt@@@std@@V34@AEBU?$basic_format_specs@_W@12@_K2AEBV<lambda_2c6139bafe179ad98da6b2e77db1d169>@@@Z 000000018001d3a0 f   handles.obj
 0001:0001cb80       ??R<lambda_c3630acb37279cf92411e07a2b271fdf>@@QEBA?AV?$basic_string@_WU?$char_traits@_W@std@@V?$allocator@_W@2@@std@@XZ 000000018001db80 f   handles.obj
 0001:0001ce30       ?GetFileNameThread@test@?4??GetFileName@@YA?AV?$basic_string@_WU?$char_traits@_W@std@@V?$allocator@_W@2@@std@@PEAX@Z@SAK0@Z 000000018001de30 f   handles.obj
 0001:0001ce70       ?GetNameByType@@YA?AV?$basic_string@_WU?$char_traits@_W@std@@V?$allocator@_W@2@@std@@PEAXGPEAVPerfThread@@@Z 000000018001de70 f   handles.obj
 0001:0001dda0       ?duplicate_handle@@YA?AV?$unique_ptr@XUhandle_closer@@@std@@PEAXK@Z 000000018001eda0 f   handles.obj
 0001:0001e42c       $LN106                     000000018001f42c     handles.obj
 0001:0001ed00       ?query_object@@YA?AV?$unique_ptr@$$BY0A@DU?$default_delete@$$BY0A@D@std@@@std@@PEAXW4OBJECT_INFORMATION_CLASS@@@Z 000000018001fd00 f   handles.obj
 0001:0001f478       $LN46                      0000000180020478     Pcfg.obj
 0001:00020d1c       $LN13                      0000000180021d1c     Pcfg.obj
 0001:000213d0       $LN69                      00000001800223d0     Pcfg.obj
 0001:00026bcc       $LN884                     0000000180027bcc     Pclass.obj
 0001:00029120       ?PrintTitle@@YA?AV?$basic_string@_WU?$char_traits@_W@std@@V?$allocator@_W@2@@std@@H@Z 000000018002a120 f   Pclass.obj
 0001:0002c6ac       $LN1371                    000000018002d6ac     Pclass.obj
 0001:0002cb30       ?TranslateMode@@YA_NAEBV?$basic_string@_WU?$char_traits@_W@std@@V?$allocator@_W@2@@std@@AEAV12@@Z 000000018002db30 f   Pclass.obj
 0001:0002d314       $LN483                     000000018002e314     Pclass.obj
 0001:0002d31c       $LN482                     000000018002e31c     Pclass.obj
 0001:0002dbb0       ?generate_titles@@YAXAEBV?$basic_string@_WU?$char_traits@_W@std@@V?$allocator@_W@2@@std@@AEAUPanelMode@@@Z 000000018002ebb0 f   Pclass.obj
 0001:0002dde0       $LN85                      000000018002ede0     Pclass.obj
 0001:0002df40       ?ui64toa_width@@YA?AV?$basic_string@_WU?$char_traits@_W@std@@V?$allocator@_W@2@@std@@_KI_N@Z 000000018002ef40 f   Pclass.obj
 0001:0002e3d0       ?window_ex_style@@YA@PEAUHWND__@@@Z 000000018002f3d0 f   Pclass.obj
 0001:0002e870       ?window_style@@YA@PEAUHWND__@@@Z 000000018002f870 f   Pclass.obj
 0001:00031b10       ??$print_module@PEAX@@YAXQEAXPEAXKAEAUoptions@@AEBV?$function@$$A6A_NPEA_W_K@Z@std@@@Z 0000000180032b10 f   Plist.obj
 0001:000320c0       ??R<lambda_fbad59960194a21b5f35257a64aadaa4>@@QEBAXXZ 00000001800330c0 f   Plist.obj
 0001:00032300       ?FreeUserData@@YAXQEAXQEBUFarPanelItemFreeInfo@@@Z 0000000180033300 f   Plist.obj
 0001:00033a30       ?_Copy@?$_Func_impl_no_alloc@V<lambda_87e110110aa5c29eaf754372c3484d5b>@@_NPEA_W_K@std@@EEBAPEAV?$_Func_base@_NPEA_W_K@2@PEAX@Z 0000000180034a30 f   Plist.obj
 0001:00033a30       ?_Move@?$_Func_impl_no_alloc@V<lambda_87e110110aa5c29eaf754372c3484d5b>@@_NPEA_W_K@std@@EEAAPEAV?$_Func_base@_NPEA_W_K@2@PEAX@Z 0000000180034a30 f   Plist.obj
 0001:00033a70       ?_Delete_this@?$_Func_impl_no_alloc@V<lambda_87e110110aa5c29eaf754372c3484d5b>@@_NPEA_W_K@std@@EEAAX_N@Z 0000000180034a70 f   Plist.obj
 0001:00033a80       ?_Do_call@?$_Func_impl_no_alloc@V<lambda_87e110110aa5c29eaf754372c3484d5b>@@_NPEA_W_K@std@@EEAA_N$$QEAPEA_W$$QEA_K@Z 0000000180034a80 f   Plist.obj
 0001:00033af0       ?_Get@?$_Func_impl_no_alloc@V<lambda_87e110110aa5c29eaf754372c3484d5b>@@_NPEA_W_K@std@@EEBAPEBXXZ 0000000180034af0 f   Plist.obj
 0001:00033af0       ?_Get@?$_Func_impl_no_alloc@V<lambda_6ecd11d6a952986d4bf89c34edf08f5f>@@XAEBUtagVARIANT@@@std@@EEBAPEBXXZ 0000000180034af0 f   WMI.obj
 0001:00033af0       ?_Get@?$_Func_impl_no_alloc@V<lambda_aac7a801b46524f039ecb4f6852a8dbe>@@XAEBUtagVARIANT@@@std@@EEBAPEBXXZ 0000000180034af0 f   WMI.obj
 0001:00033b00       ?_Target_type@?$_Func_impl_no_alloc@V<lambda_87e110110aa5c29eaf754372c3484d5b>@@_NPEA_W_K@std@@EEBAAEBVtype_info@@XZ 0000000180034b00 f   Plist.obj
 0001:00033b90       ?print_module_impl@@YAXQEAXAEBV?$basic_string@_WU?$char_traits@_W@std@@V?$allocator@_W@2@@std@@KAEBUoptions@@AEBV?$function@$$A6A_NPEA_W_K@Z@2@@Z 0000000180034b90 f   Plist.obj
 0001:00035240       ?ProcessPath@@YA@K@Z       0000000180036240 f   WMI.obj
 0001:00035360       ?_Copy@?$_Func_impl_no_alloc@V<lambda_6ecd11d6a952986d4bf89c34edf08f5f>@@XAEBUtagVARIANT@@@std@@EEBAPEAV?$_Func_base@XAEBUtagVARIANT@@@2@PEAX@Z 0000000180036360 f   WMI.obj
 0001:00035360       ?_Move@?$_Func_impl_no_alloc@V<lambda_6ecd11d6a952986d4bf89c34edf08f5f>@@XAEBUtagVARIANT@@@std@@EEAAPEAV?$_Func_base@XAEBUtagVARIANT@@@2@PEAX@Z 0000000180036360 f   WMI.obj
 0001:00035380       ?_Copy@?$_Func_impl_no_alloc@V<lambda_aac7a801b46524f039ecb4f6852a8dbe>@@XAEBUtagVARIANT@@@std@@EEBAPEAV?$_Func_base@XAEBUtagVARIANT@@@2@PEAX@Z 0000000180036380 f   WMI.obj
 0001:00035380       ?_Move@?$_Func_impl_no_alloc@V<lambda_aac7a801b46524f039ecb4f6852a8dbe>@@XAEBUtagVARIANT@@@std@@EEAAPEAV?$_Func_base@XAEBUtagVARIANT@@@2@PEAX@Z 0000000180036380 f   WMI.obj
 0001:000353a0       ?_Delete_this@?$_Func_impl_no_alloc@V<lambda_6ecd11d6a952986d4bf89c34edf08f5f>@@XAEBUtagVARIANT@@@std@@EEAAX_N@Z 00000001800363a0 f   WMI.obj
 0001:000353a0       ?_Delete_this@?$_Func_impl_no_alloc@V<lambda_aac7a801b46524f039ecb4f6852a8dbe>@@XAEBUtagVARIANT@@@std@@EEAAX_N@Z 00000001800363a0 f   WMI.obj
 0001:000353b0       ?_Do_call@?$_Func_impl_no_alloc@V<lambda_6ecd11d6a952986d4bf89c34edf08f5f>@@XAEBUtagVARIANT@@@std@@EEAAXAEBUtagVARIANT@@@Z 00000001800363b0 f   WMI.obj
 0001:000353e0       ?_Do_call@?$_Func_impl_no_alloc@V<lambda_aac7a801b46524f039ecb4f6852a8dbe>@@XAEBUtagVARIANT@@@std@@EEAAXAEBUtagVARIANT@@@Z 00000001800363e0 f   WMI.obj
 0001:000353f0       ?_Target_type@?$_Func_impl_no_alloc@V<lambda_6ecd11d6a952986d4bf89c34edf08f5f>@@XAEBUtagVARIANT@@@std@@EEBAAEBVtype_info@@XZ 00000001800363f0 f   WMI.obj
 0001:00035400       ?_Target_type@?$_Func_impl_no_alloc@V<lambda_aac7a801b46524f039ecb4f6852a8dbe>@@XAEBUtagVARIANT@@@std@@EEBAAEBVtype_info@@XZ 0000000180036400 f   WMI.obj
 0001:00035410       ?fNtQueryInformationFile@@YAJPEAX00KK@Z 0000000180036410 f   Proclist.obj
 0001:00035410       ?fNtQueryInformationProcess@@YAJPEAXW4_PROCESSINFOCLASS@@0KPEAK@Z 0000000180036410 f   Proclist.obj
 0001:00035410       ?fNtQueryInformationThread@@YAJPEAXK0KPEAK@Z 0000000180036410 f   Proclist.obj
 0001:00035410       ?fNtQueryObject@@YAJPEAXK0K0@Z 0000000180036410 f   Proclist.obj
 0001:00035410       ?fNtQuerySystemInformation@@YAJKPEAXKPEAK@Z 0000000180036410 f   Proclist.obj
 0001:00035410       ?fNtWow64QueryInformationProcess64@@YAJPEAXW4_PROCESSINFOCLASS@@0KPEAK@Z 0000000180036410 f   Proclist.obj
 0001:00035410       ?fNtWow64ReadVirtualMemory64@@YAJPEAX_K01PEA_K@Z 0000000180036410 f   Proclist.obj
 0001:00035420       ?fEnumProcessModulesEx@@YAHPEAXPEAPEAUHINSTANCE__@@KPEAKK@Z 0000000180036420 f   Proclist.obj
 0001:00035420       ?fGetGuiResources@@YAKPEAXK@Z 0000000180036420 f   Proclist.obj
 0001:00035420       ?fGetSidIdentifierAuthority@@YAPEAU_SID_IDENTIFIER_AUTHORITY@@PEAX@Z 0000000180036420 f   Proclist.obj
 0001:00035420       ?fGetSidSubAuthority@@YAPEAKPEAXK@Z 0000000180036420 f   Proclist.obj
 0001:00035420       ?fGetSidSubAuthorityCount@@YAPEAEPEAX@Z 0000000180036420 f   Proclist.obj
 0001:00035420       ?fIsValidSid@@YAHPEAX@Z    0000000180036420 f   Proclist.obj
 0001:00035420       ?fIsWow64Process@@YAHPEAXPEAH@Z 0000000180036420 f   Proclist.obj
 0001:00035420       no_op_initialize           0000000180036420 f   libucrt:wsetlocale.obj
 0001:00035430       ?fCoSetProxyBlanket@@YAJPEAUIUnknown@@KKPEA_WKKPEAXK@Z 0000000180036430 f   Proclist.obj
 0001:00035480       ?dynamic_bind@@YAXXZ       0000000180036480 f   Proclist.obj
 0001:00036308       tidy_global                0000000180037308 f   libcpmt:locale0.obj
 0001:000365d4       ?initialize_pointers@@YAHXZ 00000001800375d4 f   libcpmt:winapisupp.obj
 0001:00036e80       ?dllmain_crt_dispatch@@YAHQEAUHINSTANCE__@@KQEAX@Z 0000000180037e80 f   LIBCMT:dll_dllmain.obj
 0001:00036ed0       ?dllmain_crt_process_attach@@YAHQEAUHINSTANCE__@@QEAX@Z 0000000180037ed0 f   LIBCMT:dll_dllmain.obj
 0001:00036fe8       ?dllmain_crt_process_detach@@YAH_N@Z 0000000180037fe8 f   LIBCMT:dll_dllmain.obj
 0001:0003706c       ?dllmain_dispatch@@YAHQEAUHINSTANCE__@@KQEAX@Z 000000018003806c f   LIBCMT:dll_dllmain.obj
 0001:000372e0       $$000000                   00000001800382e0     LIBCMT:amdsecgs.obj
 0001:00037958       capture_current_context    0000000180038958 f   LIBCMT:gs_report.obj
 0001:000379c8       capture_previous_context   00000001800389c8 f   LIBCMT:gs_report.obj
 0001:000389d0       $$000000                   00000001800399d0     libvcruntime:memchr.obj
 0001:00038a50       $$000000                   0000000180039a50     libvcruntime:memcmp.obj
 0001:00038b30       $$000000                   0000000180039b30     libvcruntime:memcpy.obj
 0001:00038f40       $$000000                   0000000180039f40     libvcruntime:memset.obj
 0001:0003980c       ??$BuildCatchObjectHelperInternal@V__FrameHandler3@@@@YAHPEAUEHExceptionRecord@@PEAXPEBU_s_HandlerType@@PEBU_s_CatchableType@@@Z 000000018003a80c f   libvcruntime:frame.obj
 0001:00039a0c       ??$BuildCatchObjectHelperInternal@V__FrameHandler4@@@@YAHPEAUEHExceptionRecord@@PEAXPEAUHandlerType4@FH4@@PEBU_s_CatchableType@@@Z 000000018003aa0c f   libvcruntime:frame.obj
 0001:00039c10       ??$BuildCatchObjectInternal@V__FrameHandler3@@@@YAXPEAUEHExceptionRecord@@PEAXPEBU_s_HandlerType@@PEBU_s_CatchableType@@@Z 000000018003ac10 f   libvcruntime:frame.obj
 0001:00039cd0       ??$BuildCatchObjectInternal@V__FrameHandler4@@@@YAXPEAUEHExceptionRecord@@PEAXPEAUHandlerType4@FH4@@PEBU_s_CatchableType@@@Z 000000018003acd0 f   libvcruntime:frame.obj
 0001:00039d94       ??$CatchIt@V__FrameHandler3@@@@YAXPEAUEHExceptionRecord@@PEA_KPEAU_CONTEXT@@PEAU_xDISPATCHER_CONTEXT@@PEBU_s_FuncInfo@@PEBU_s_HandlerType@@PEBU_s_CatchableType@@PEBU_s_TryBlockMapEntry@@H1EE@Z 000000018003ad94 f   libvcruntime:frame.obj
 0001:00039e68       ??$CatchIt@V__FrameHandler4@@@@YAXPEAUEHExceptionRecord@@PEA_KPEAU_CONTEXT@@PEAU_xDISPATCHER_CONTEXT@@PEAUFuncInfo4@FH4@@PEAUHandlerType4@4@PEBU_s_CatchableType@@PEAUTryBlockMapEntry4@4@H1EE@Z 000000018003ae68 f   libvcruntime:frame.obj
 0001:00039f3c       ??$FindHandler@V__FrameHandler3@@@@YAXPEAUEHExceptionRecord@@PEA_KPEAU_CONTEXT@@PEAU_xDISPATCHER_CONTEXT@@PEBU_s_FuncInfo@@EH1@Z 000000018003af3c f   libvcruntime:frame.obj
 0001:0003a434       ??$FindHandler@V__FrameHandler4@@@@YAXPEAUEHExceptionRecord@@PEA_KPEAU_CONTEXT@@PEAU_xDISPATCHER_CONTEXT@@PEAUFuncInfo4@FH4@@EH1@Z 000000018003b434 f   libvcruntime:frame.obj
 0001:0003a944       ??$FindHandlerForForeignException@V__FrameHandler3@@@@YAXPEAUEHExceptionRecord@@PEA_KPEAU_CONTEXT@@PEAU_xDISPATCHER_CONTEXT@@PEBU_s_FuncInfo@@HH1@Z 000000018003b944 f   libvcruntime:frame.obj
 0001:0003ab58       ??$FindHandlerForForeignException@V__FrameHandler4@@@@YAXPEAUEHExceptionRecord@@PEA_KPEAU_CONTEXT@@PEAU_xDISPATCHER_CONTEXT@@PEAUFuncInfo4@FH4@@HH1@Z 000000018003bb58 f   libvcruntime:frame.obj
 0001:0003bd38       ?ExFilterRethrow@@YAHPEAU_EXCEPTION_POINTERS@@PEAUEHExceptionRecord@@PEAH@Z 000000018003cd38 f   libvcruntime:frame.obj
 0001:0003bdc0       ?ExFilterRethrowFH4@@YAHPEAU_EXCEPTION_POINTERS@@PEAUEHExceptionRecord@@HPEAH@Z 000000018003cdc0 f   libvcruntime:frame.obj
 0001:0003c2e8       ?IsInExceptionSpec@@YAEPEAUEHExceptionRecord@@PEBU_s_ESTypeList@@@Z 000000018003d2e8 f   libvcruntime:frame.obj
 0001:0003c3d8       ?Is_bad_exception_allowed@@YAEPEBU_s_ESTypeList@@@Z 000000018003d3d8 f   libvcruntime:frame.obj
 0001:0003c720       $$000000                   000000018003d720     libvcruntime:notify.obj
 0001:0003c79c       ?try_get_function@@YAPEAXW4function_id@?A0x81a78551@@QEBDQEBW4module_id@2@2@Z 000000018003d79c f   libvcruntime:winapi_downlevel.obj
 0001:0003ca90       $$000000                   000000018003da90     libvcruntime:handlers.obj
 0001:0003d174       ??$common_vsprintf@Vformat_validation_base@__crt_stdio_output@@D@@YAH_KQEAD0QEBDQEAU__crt_locale_pointers@@1@Z 000000018003e174 f   libucrt:output.obj
 0001:0003f1b0       $$000000                   00000001800401b0     libucrt:log10.obj
 0001:0003f760       $$000000                   0000000180040760     libucrt:pow.obj
 0001:00040ed8       ??$?RV<lambda_41e84717acc955b55e9d0d529e507b68>@@AEAV<lambda_b37934c380d97b75fd242ea49540127a>@@V<lambda_bb6db9f9ac473960206e0d4b942b5506>@@@?$__crt_seh_guarded_call@PEAD@@QEAAPEAD$$QEAV<lambda_41e84717acc955b55e9d0d529e507b68>@@AEAV<lambda_b37934c380d97b75fd242ea49540127a>@@$$QEAV<lambda_bb6db9f9ac473960206e0d4b942b5506>@@@Z 0000000180041ed8 f   libucrt:setlocale.obj
 0001:00040f18       ??R<lambda_b37934c380d97b75fd242ea49540127a>@@QEBAPEADXZ 0000000180041f18 f   libucrt:setlocale.obj
 0001:00041dd4       memcpy_s                   0000000180042dd4 f   libucrt:cfout.obj
 0001:00041dd4       memcpy_s                   0000000180042dd4 f   libucrt:strtod.obj
 0001:00041e60       $$000000                   0000000180042e60     libucrt:powf.obj
 0001:000435d0       ??$?RV<lambda_d80eeec6fff315bfe5c115232f3240e3>@@AEAV<lambda_6e4b09c48022b2350581041d5f6b0c4c>@@V<lambda_2358e3775559c9db80273638284d5e45>@@@?$__crt_seh_guarded_call@X@@QEAAX$$QEAV<lambda_d80eeec6fff315bfe5c115232f3240e3>@@AEAV<lambda_6e4b09c48022b2350581041d5f6b0c4c>@@$$QEAV<lambda_2358e3775559c9db80273638284d5e45>@@@Z 00000001800445d0 f   libucrt:exit.obj
 0001:00043608       ??R<lambda_6e4b09c48022b2350581041d5f6b0c4c>@@QEBA@XZ 0000000180044608 f   libucrt:exit.obj
 0001:000436cc       ?atexit_exception_filter@@YAHK@Z 00000001800446cc f   libucrt:exit.obj
 0001:000436d8       ?common_exit@@YAXHW4_crt_exit_cleanup_mode@@W4_crt_exit_return_mode@@@Z 00000001800446d8 f   libucrt:exit.obj
 0001:00043794       ?exit_or_terminate_process@@YAXI@Z 0000000180044794 f   libucrt:exit.obj
 0001:000437e0       ?try_cor_exit_process@@YAXI@Z 00000001800447e0 f   libucrt:exit.obj
 0001:00043868       ??$parse_command_line@D@@YAXPEADPEAPEAD0PEA_K2@Z 0000000180044868 f   libucrt:argv_parsing.obj
 0001:00043c14       ??$common_initialize_environment_nolock@D@@YAHXZ 0000000180044c14 f   libucrt:environment_initialization.obj
 0001:00043c80       ??$create_environment@D@@YAQEAPEADQEAD@Z 0000000180044c80 f   libucrt:environment_initialization.obj
 0001:00043d88       ??$free_environment@D@@YAXQEAPEAD@Z 0000000180044d88 f   libucrt:environment_initialization.obj
 0001:00043d88       ??$free_environment@_W@@YAXQEAPEA_W@Z 0000000180044d88 f   libucrt:environment_initialization.obj
 0001:00043dcc       ??$uninitialize_environment_internal@D@@YAXAEAPEAPEAD@Z 0000000180044dcc f   libucrt:environment_initialization.obj
 0001:00043de8       ??$uninitialize_environment_internal@_W@@YAXAEAPEAPEA_W@Z 0000000180044de8 f   libucrt:environment_initialization.obj
 0001:00043e44       ??$?RV<lambda_638799b9deba96c50f710eeac98168cd>@@AEAV<lambda_22ebabd17bc4fa466a2aca6d8deb888d>@@V<lambda_a6f7d7db0129f75315ebf26d50c089f1>@@@?$__crt_seh_guarded_call@H@@QEAAH$$QEAV<lambda_638799b9deba96c50f710eeac98168cd>@@AEAV<lambda_22ebabd17bc4fa466a2aca6d8deb888d>@@$$QEAV<lambda_a6f7d7db0129f75315ebf26d50c089f1>@@@Z 0000000180044e44 f   libucrt:onexit.obj
 0001:00043e80       ??$?RV<lambda_7777bce6b2f8c936911f934f8298dc43>@@AEAV<lambda_f03950bc5685219e0bcd2087efbe011e>@@V<lambda_3883c3dff614d5e0c5f61bb1ac94921c>@@@?$__crt_seh_guarded_call@H@@QEAAH$$QEAV<lambda_7777bce6b2f8c936911f934f8298dc43>@@AEAV<lambda_f03950bc5685219e0bcd2087efbe011e>@@$$QEAV<lambda_3883c3dff614d5e0c5f61bb1ac94921c>@@@Z 0000000180044e80 f   libucrt:onexit.obj
 0001:00043ebc       ??R<lambda_22ebabd17bc4fa466a2aca6d8deb888d>@@QEBAHXZ 0000000180044ebc f   libucrt:onexit.obj
 0001:0004406c       ??R<lambda_f03950bc5685219e0bcd2087efbe011e>@@QEBAHXZ 000000018004506c f   libucrt:onexit.obj
 0001:00044240       initialize_global_variables 0000000180045240 f   libucrt:initialization.obj
 0001:00044254       initialize_c               0000000180045254 f   libucrt:initialization.obj
 0001:00044278       initialize_environment     0000000180045278 f   libucrt:initialization.obj
 0001:00044278       initialize_global_state_isolation 0000000180045278 f   libucrt:initialization.obj
 0001:00044278       report_memory_leaks        0000000180045278 f   libucrt:initialization.obj
 0001:00044278       uninitialize_c             0000000180045278 f   libucrt:initialization.obj
 0001:00044278       uninitialize_global_state_isolation 0000000180045278 f   libucrt:initialization.obj
 0001:0004427c       uninitialize_environment   000000018004527c f   libucrt:initialization.obj
 0001:0004428c       initialize_pointers        000000018004528c f   libucrt:initialization.obj
 0001:000442cc       uninitialize_vcruntime     00000001800452cc f   libucrt:initialization.obj
 0001:000442d4       uninitialize_allocated_memory 00000001800452d4 f   libucrt:initialization.obj
 0001:00044314       uninitialize_allocated_io_buffers 0000000180045314 f   libucrt:initialization.obj
 0001:00044f50       $$000000                   0000000180045f50     libucrt:strncmp.obj
 0001:0004500c       ??$?RV<lambda_0ae27a3a962d80f24befdcbee591983d>@@AEAV<lambda_8d0ee55de4b1038c4002e0adecdf1839>@@V<lambda_dc504788e8f1664fe9b84e20bfb512f2>@@@?$__crt_seh_guarded_call@X@@QEAAX$$QEAV<lambda_0ae27a3a962d80f24befdcbee591983d>@@AEAV<lambda_8d0ee55de4b1038c4002e0adecdf1839>@@$$QEAV<lambda_dc504788e8f1664fe9b84e20bfb512f2>@@@Z 000000018004600c f   libucrt:per_thread_data.obj
 0001:0004504c       ??$?RV<lambda_2d41944a1d46af3157314b8a01080d33>@@AEAV<lambda_8f455de75cd7d7f24b4096f044d8b9e6>@@V<lambda_aa500f224e6afead328df44964fe2772>@@@?$__crt_seh_guarded_call@X@@QEAAX$$QEAV<lambda_2d41944a1d46af3157314b8a01080d33>@@AEAV<lambda_8f455de75cd7d7f24b4096f044d8b9e6>@@$$QEAV<lambda_aa500f224e6afead328df44964fe2772>@@@Z 000000018004604c f   libucrt:per_thread_data.obj
 0001:0004508c       ??$?RV<lambda_aa87e3671a710a21b5dc78c0bdf72e11>@@AEAV<lambda_92619d2358a28f41a33ba319515a20b9>@@V<lambda_6992ecaafeb10aed2b74cb1fae11a551>@@@?$__crt_seh_guarded_call@X@@QEAAX$$QEAV<lambda_aa87e3671a710a21b5dc78c0bdf72e11>@@AEAV<lambda_92619d2358a28f41a33ba319515a20b9>@@$$QEAV<lambda_6992ecaafeb10aed2b74cb1fae11a551>@@@Z 000000018004608c f   libucrt:per_thread_data.obj
 0001:000450d4       ??$?RV<lambda_f2e299630e499de9f9a165e60fcd3db5>@@AEAV<lambda_2ae9d31cdba2644fcbeaf08da7c24588>@@V<lambda_40d01ff24d0e7b3814fdbdcee8eab3c7>@@@?$__crt_seh_guarded_call@X@@QEAAX$$QEAV<lambda_f2e299630e499de9f9a165e60fcd3db5>@@AEAV<lambda_2ae9d31cdba2644fcbeaf08da7c24588>@@$$QEAV<lambda_40d01ff24d0e7b3814fdbdcee8eab3c7>@@@Z 00000001800460d4 f   libucrt:per_thread_data.obj
 0001:00045134       ?construct_ptd_array@@YAXQEAU__acrt_ptd@@@Z 0000000180046134 f   libucrt:per_thread_data.obj
 0001:00045204       ?destroy_fls@@YAXPEAX@Z    0000000180046204 f   libucrt:per_thread_data.obj
 0001:00045224       ?destroy_ptd_array@@YAXQEAU__acrt_ptd@@@Z 0000000180046224 f   libucrt:per_thread_data.obj
 0001:0004531c       ?replace_current_thread_locale_nolock@@YAXQEAU__acrt_ptd@@QEAU__crt_locale_data@@@Z 000000018004631c f   libucrt:per_thread_data.obj
 0001:000458f8       ?<lambda_invoker_cdecl>@<lambda_795c6bd18aed400428efeb9a5f0e1479>@@CAHPEA_W@Z 00000001800468f8 f   libucrt:winapi_thunks.obj
 0001:00045920       ??$?RV<lambda_48fc4a32460bb0512d3b13f8499328be>@@AEAV<lambda_6c3dac0a4f3f9cefca9bb494422f9b77>@@V<lambda_0a2f2c9f9a56eb2b08bfa6ff61d331c5>@@@?$__crt_seh_guarded_call@H@@QEAAH$$QEAV<lambda_48fc4a32460bb0512d3b13f8499328be>@@AEAV<lambda_6c3dac0a4f3f9cefca9bb494422f9b77>@@$$QEAV<lambda_0a2f2c9f9a56eb2b08bfa6ff61d331c5>@@@Z 0000000180046920 f   libucrt:winapi_thunks.obj
 0001:0004599c       ?try_get_function@@YAPEAXW4function_id@?A0x391cf84c@@QEBDQEBW4module_id@2@2@Z 000000018004699c f   libucrt:winapi_thunks.obj
 0001:000463bc       ??$?RV<lambda_842d9ff0dc9ef11c61343bbaebe7f885>@@AEAV<lambda_c5860995281e5c4ce005b3de8f5874ee>@@V<lambda_d90129c13df834fdcbf8d2b88dafcf2d>@@@?$__crt_seh_guarded_call@X@@QEAAX$$QEAV<lambda_842d9ff0dc9ef11c61343bbaebe7f885>@@AEAV<lambda_c5860995281e5c4ce005b3de8f5874ee>@@$$QEAV<lambda_d90129c13df834fdcbf8d2b88dafcf2d>@@@Z 00000001800473bc f   libucrt:fflush.obj
 0001:00046458       ??$?RV<lambda_886d6c58226a84441f68b9f2b8217b83>@@AEAV<lambda_ab61a845afdef5b7c387490eaf3616ee>@@V<lambda_f7f22ab5edc0698d5f6905b0d3f44752>@@@?$__crt_seh_guarded_call@X@@QEAAX$$QEAV<lambda_886d6c58226a84441f68b9f2b8217b83>@@AEAV<lambda_ab61a845afdef5b7c387490eaf3616ee>@@$$QEAV<lambda_f7f22ab5edc0698d5f6905b0d3f44752>@@@Z 0000000180047458 f   libucrt:fflush.obj
 0001:00046538       ?common_flush_all@@YAH_N@Z 0000000180047538 f   libucrt:fflush.obj
 0001:000466a8       ?initialize_inherited_file_handles_nolock@@YAXXZ 00000001800476a8 f   libucrt:ioinit.obj
 0001:00046798       ?initialize_stdio_handles_nolock@@YAXXZ 0000000180047798 f   libucrt:ioinit.obj
 0001:00046920       ?write_double_translated_ansi_nolock@@YA?AUwrite_result@?A0x17268360@@HQEBDI@Z 0000000180047920 f   libucrt:write.obj
 0001:00046df0       ?write_text_ansi_nolock@@YA?AUwrite_result@?A0x17268360@@HQEBDI@Z 0000000180047df0 f   libucrt:write.obj
 0001:00046ef4       ?write_text_utf16le_nolock@@YA?AUwrite_result@?A0x17268360@@HQEBDI@Z 0000000180047ef4 f   libucrt:write.obj
 0001:00047010       ?write_text_utf8_nolock@@YA?AUwrite_result@?A0x17268360@@HQEBDI@Z 0000000180048010 f   libucrt:write.obj
 0001:00047974       ?fp_format_a@@YAHQEBNPEAD_KQEAD2H_NIQEAU__crt_locale_pointers@@@Z 0000000180048974 f   libucrt:cvt.obj
 0001:00047ce4       ?fp_format_e@@YAHQEBNQEAD_K12H_NIQEAU__crt_locale_pointers@@@Z 0000000180048ce4 f   libucrt:cvt.obj
 0001:00047dc0       ?fp_format_e_internal@@YAHQEAD_KH_NIQEAU_strflt@@2QEAU__crt_locale_pointers@@@Z 0000000180048dc0 f   libucrt:cvt.obj
 0001:00047f94       ?fp_format_f_internal@@YAHQEAD_KHQEAU_strflt@@_NQEAU__crt_locale_pointers@@@Z 0000000180048f94 f   libucrt:cvt.obj
 0001:000480d8       ?fp_format_g@@YAHQEBNQEAD_K12H_NIQEAU__crt_locale_pointers@@@Z 00000001800490d8 f   libucrt:cvt.obj
 0001:00048528       ??$?RV<lambda_1d892b297fdedeee07ed8124eeb2f2fa>@@AEAV<lambda_ffc046909424fd52df0ac47e64813305>@@V<lambda_01a7098693036236037e7cdb9bca3d73>@@@?$__crt_seh_guarded_call@X@@QEAAX$$QEAV<lambda_1d892b297fdedeee07ed8124eeb2f2fa>@@AEAV<lambda_ffc046909424fd52df0ac47e64813305>@@$$QEAV<lambda_01a7098693036236037e7cdb9bca3d73>@@@Z 0000000180049528 f   libucrt:wsetlocale.obj
 0001:00048664       ??$?RV<lambda_410d79af7f07d98d83a3f525b3859a53>@@AEAV<lambda_3e16ef9562a7dcce91392c22ab16ea36>@@V<lambda_38119f0e861e05405d8a144b9b982f0a>@@@?$__crt_seh_guarded_call@X@@QEAAX$$QEAV<lambda_410d79af7f07d98d83a3f525b3859a53>@@AEAV<lambda_3e16ef9562a7dcce91392c22ab16ea36>@@$$QEAV<lambda_38119f0e861e05405d8a144b9b982f0a>@@@Z 0000000180049664 f   libucrt:wsetlocale.obj
 0001:000486d4       ??$?RV<lambda_7f2adfce497ff2baa965cd4f576ecfd1>@@AEAV<lambda_2a444430fde8c29194d880d93eed5e8f>@@AEAV<lambda_8dff2cf36a5417162780cd64fa2883ef>@@@?$__crt_seh_guarded_call@X@@QEAAX$$QEAV<lambda_7f2adfce497ff2baa965cd4f576ecfd1>@@AEAV<lambda_2a444430fde8c29194d880d93eed5e8f>@@AEAV<lambda_8dff2cf36a5417162780cd64fa2883ef>@@@Z 00000001800496d4 f   libucrt:wsetlocale.obj
 0001:00048700       ??R<lambda_2a444430fde8c29194d880d93eed5e8f>@@QEBA@XZ 0000000180049700 f   libucrt:wsetlocale.obj
 0001:00048ad4       _copytlocinfo_nolock       0000000180049ad4 f   libucrt:wsetlocale.obj
 0001:00048b94       _expandlocale              0000000180049b94 f   libucrt:wsetlocale.obj
 0001:00049120       _wsetlocale_get_all        000000018004a120 f   libucrt:wsetlocale.obj
 0001:0004930c       _wsetlocale_nolock         000000018004a30c f   libucrt:wsetlocale.obj
 0001:000495a4       _wsetlocale_set_cat        000000018004a5a4 f   libucrt:wsetlocale.obj
 0001:000498f8       parse_bcp47                000000018004a8f8 f   libucrt:wsetlocale.obj
 0001:00049af8       parse_bcp47_code_page      000000018004aaf8 f   libucrt:wsetlocale.obj
 0001:00049b40       parse_bcp47_language       000000018004ab40 f   libucrt:wsetlocale.obj
 0001:00049bcc       parse_bcp47_region         000000018004abcc f   libucrt:wsetlocale.obj
 0001:00049cd8       parse_bcp47_script         000000018004acd8 f   libucrt:wsetlocale.obj
 0001:00049d68       string_is_alpha            000000018004ad68 f   libucrt:wsetlocale.obj
 0001:00049ddc       ?_mbstowcs_l_helper@@YA_KPEA_WPEBD_KPEAU__crt_locale_pointers@@@Z 000000018004addc f   libucrt:mbstowcs.obj
 0001:0004a20c       _call_matherr              000000018004b20c f   libucrt:libm_error.obj
 0001:0004a274       _exception_enabled         000000018004b274 f   libucrt:libm_error.obj
 0001:0004a770       _log_special_common        000000018004b770 f   libucrt:log_special.obj
 0001:0004aac0       ?_wcstombs_l_helper@@YA_KPEADPEB_W_KPEAU__crt_locale_pointers@@@Z 000000018004bac0 f   libucrt:wcstombs.obj
 0001:0004af14       ?InternalGetLocaleInfoA@@YAHQEAU__crt_locale_pointers@@QEB_WKQEADH@Z 000000018004bf14 f   libucrt:getlocaleinfoa.obj
 0001:0004b3e8       ?__acrt_LCMapStringA_stat@@YAHPEAU__crt_locale_pointers@@PEB_WKPEBDHPEADHHH@Z 000000018004c3e8 f   libucrt:lcmapstringa.obj
 0001:0004bd80       ??$?RV<lambda_450d765d439847d4c735a33c368b5fc0>@@AEAV<lambda_44731a7d0e6d81c3e6aa82d741081786>@@V<lambda_601a2a7da3b7a96e9554ac7215c4b07c>@@@?$__crt_seh_guarded_call@P6AXH@Z@@QEAAP6AXH@Z$$QEAV<lambda_450d765d439847d4c735a33c368b5fc0>@@AEAV<lambda_44731a7d0e6d81c3e6aa82d741081786>@@$$QEAV<lambda_601a2a7da3b7a96e9554ac7215c4b07c>@@@Z 000000018004cd80 f   libucrt:signal.obj
 0001:0004c3a8       ?<lambda_invoker_cdecl>@<lambda_a1ce4c8ae42411fd470c77163914f50e>@@CAHPEBX0@Z 000000018004d3a8 f   libucrt:argv_wildcards.obj
 0001:0004c548       ??$common_expand_argv_wildcards@D@@YAHQEAPEADQEAPEAPEAD@Z 000000018004d548 f   libucrt:argv_wildcards.obj
 0001:0004c754       ??$copy_and_add_argument_to_buffer@D@@YAHQEBD0_KAEAV?$argument_list@D@?A0x5f5c8891@@@Z 000000018004d754 f   libucrt:argv_wildcards.obj
 0001:0004c8dc       ??$expand_argument_wildcards@D@@YAHQEAD0AEAV?$argument_list@D@?A0x5f5c8891@@@Z 000000018004d8dc f   libucrt:argv_wildcards.obj
 0001:0004cd14       ??$?RV<lambda_efdfa57d1f175319df784efa44bb7b81>@@AEAV<lambda_5f0a4c1567f8adc6734073e5d1e1b35c>@@V<lambda_2e8a7d3640ea6ccb4c2413664c2db6fd>@@@?$__crt_seh_guarded_call@X@@QEAAX$$QEAV<lambda_efdfa57d1f175319df784efa44bb7b81>@@AEAV<lambda_5f0a4c1567f8adc6734073e5d1e1b35c>@@$$QEAV<lambda_2e8a7d3640ea6ccb4c2413664c2db6fd>@@@Z 000000018004dd14 f   libucrt:mbctype.obj
 0001:0004ced0       ?getSystemCP@@YAHH@Z       000000018004ded0 f   libucrt:mbctype.obj
 0001:0004cf50       ?setSBCS@@YAXPEAU__crt_multibyte_data@@@Z 000000018004df50 f   libucrt:mbctype.obj
 0001:0004cfe0       ?setSBUpLow@@YAXPEAU__crt_multibyte_data@@@Z 000000018004dfe0 f   libucrt:mbctype.obj
 0001:0004d1c4       ?setmbcp_internal@@YAHH_NQEAU__acrt_ptd@@QEAPEAU__crt_multibyte_data@@@Z 000000018004e1c4 f   libucrt:mbctype.obj
 0001:0004d388       ?update_thread_multibyte_data_internal@@YAPEAU__crt_multibyte_data@@QEAU__acrt_ptd@@QEAPEAU1@@Z 000000018004e388 f   libucrt:mbctype.obj
 0001:0004d778       ?x_ismbbtype_l@@YAHPEAU__crt_locale_pointers@@IHH@Z 000000018004e778 f   libucrt:ismbbyte.obj
 0001:0004e4b4       ??$?RV<lambda_a37b2b86f63e897a80ea819b0eb08c01>@@AEAV<lambda_38ce7e780aa69e748d6df282ebc68efe>@@V<lambda_99fb1378e971ab6e7edea83e3a7a83a2>@@@?$__crt_seh_guarded_call@H@@QEAAH$$QEAV<lambda_a37b2b86f63e897a80ea819b0eb08c01>@@AEAV<lambda_38ce7e780aa69e748d6df282ebc68efe>@@$$QEAV<lambda_99fb1378e971ab6e7edea83e3a7a83a2>@@@Z 000000018004f4b4 f   libucrt:commit.obj
 0001:0004e5d4       ??$common_lseek_nolock@_J@@YA_JH_JH@Z 000000018004f5d4 f   libucrt:lseek.obj
 0001:000505d0       ?free_crt_array_internal@@YAXQEAPEBX_K@Z 00000001800515d0 f   libucrt:inittime.obj
 0001:00050628       ?initialize_lc_time@@YA_NQEAU__crt_lc_time_data@@QEAU__crt_locale_data@@@Z 0000000180051628 f   libucrt:inittime.obj
 0001:00050d70       GetLocaleNameFromDefault   0000000180051d70 f   libucrt:get_qualified_locale.obj
 0001:00050e18       GetLocaleNameFromLangCountry 0000000180051e18 f   libucrt:get_qualified_locale.obj
 0001:00050ee8       GetLocaleNameFromLanguage  0000000180051ee8 f   libucrt:get_qualified_locale.obj
 0001:00050f80       LangCountryEnumProcEx      0000000180051f80 f   libucrt:get_qualified_locale.obj
 0001:0005126c       LanguageEnumProcEx         000000018005226c f   libucrt:get_qualified_locale.obj
 0001:00051358       ProcessCodePage            0000000180052358 f   libucrt:get_qualified_locale.obj
 0001:00051424       TestDefaultCountry         0000000180052424 f   libucrt:get_qualified_locale.obj
 0001:00051488       TranslateName              0000000180052488 f   libucrt:get_qualified_locale.obj
 0001:00051788       CountryEnumProc            0000000180052788 f   libucrt:getqloc_downlevel.obj
 0001:00051870       GetLcidFromLangCountry     0000000180052870 f   libucrt:getqloc_downlevel.obj
 0001:00051940       GetLcidFromLanguage        0000000180052940 f   libucrt:getqloc_downlevel.obj
 0001:000519d8       LangCountryEnumProc        00000001800529d8 f   libucrt:getqloc_downlevel.obj
 0001:00051c24       LanguageEnumProc           0000000180052c24 f   libucrt:getqloc_downlevel.obj
 0001:00051d2c       LcidFromHexString          0000000180052d2c f   libucrt:getqloc_downlevel.obj
 0001:00051d7c       ProcessCodePage            0000000180052d7c f   libucrt:getqloc_downlevel.obj
 0001:00051e2c       TestDefaultLanguage        0000000180052e2c f   libucrt:getqloc_downlevel.obj
 0001:00051ed8       TranslateName              0000000180052ed8 f   libucrt:getqloc_downlevel.obj
 0001:00052300       $$000000                   0000000180053300     libucrt:fpsr.obj
 0001:000527d0       fallbackMethod             00000001800537d0 f   libucrt:strpbrk.obj
 0001:00052b94       $LN78                      0000000180053b94     libucrt:strpbrk.obj
 0001:00052bd0       $LN77                      0000000180053bd0     libucrt:strpbrk.obj
 0001:00052c10       $LN76                      0000000180053c10     libucrt:strpbrk.obj
 0001:00052cec       ?initialize_multibyte@@YAHXZ 0000000180053cec f   libucrt:multibyte_initializer.obj
 0001:00052f24       ??$?RV<lambda_751a882b2c74d4b022dec766aa51a29a>@@AEAV<lambda_628dfdc04ba53c8bfc02c9951375f3f5>@@V<lambda_f6c7be5f7998530c34de24c7437d6b54>@@@?$__crt_seh_guarded_call@H@@QEAAH$$QEAV<lambda_751a882b2c74d4b022dec766aa51a29a>@@AEAV<lambda_628dfdc04ba53c8bfc02c9951375f3f5>@@$$QEAV<lambda_f6c7be5f7998530c34de24c7437d6b54>@@@Z 0000000180053f24 f   libucrt:close.obj
 0001:000535a4       ??$common_xtox@K_W@@YAHKQEA_W_KI_N@Z 00000001800545a4 f   libucrt:xtoa.obj
 0001:00053678       ??$common_xtox_s@K_W@@YAHKQEA_W_KI_N@Z 0000000180054678 f   libucrt:xtoa.obj
 0001:00053b70       $$000000                   0000000180054b70     LIBCMT:guard_dispatch.obj
 0001:00053b90       ?dtor$0@?0???$decimal_point_impl@_W@detail@v6@fmt@@YA_WVlocale_ref@012@@Z@4HA 0000000180054b90 f   format.obj
 0001:00053b90       ?dtor$0@?0???$grouping_impl@_W@detail@v6@fmt@@YA?AV?$basic_string@DU?$char_traits@D@std@@V?$allocator@D@2@@std@@Vlocale_ref@012@@Z@4HA 0000000180054b90 f   format.obj
 0001:00053b90       ?dtor$0@?0???$thousands_sep_impl@_W@detail@v6@fmt@@YA_WVlocale_ref@012@@Z@4HA 0000000180054b90 f   format.obj
 0001:00053ba0       ?dtor$0@?0???$fallback_format@N@detail@v6@fmt@@YAXNAEAV?$buffer@D@012@AEAH@Z@4HA 0000000180054ba0 f   format.obj
 0001:00053ba0       ?dtor$0@?0???$fallback_format@O@detail@v6@fmt@@YAXOAEAV?$buffer@D@012@AEAH@Z@4HA 0000000180054ba0 f   format.obj
 0001:00053bb0       ?dtor$1@?0???$fallback_format@N@detail@v6@fmt@@YAXNAEAV?$buffer@D@012@AEAH@Z@4HA 0000000180054bb0 f   format.obj
 0001:00053bb0       ?dtor$1@?0???$fallback_format@O@detail@v6@fmt@@YAXOAEAV?$buffer@D@012@AEAH@Z@4HA 0000000180054bb0 f   format.obj
 0001:00053bc0       ?dtor$2@?0???$fallback_format@N@detail@v6@fmt@@YAXNAEAV?$buffer@D@012@AEAH@Z@4HA 0000000180054bc0 f   format.obj
 0001:00053bc0       ?dtor$2@?0???$fallback_format@O@detail@v6@fmt@@YAXOAEAV?$buffer@D@012@AEAH@Z@4HA 0000000180054bc0 f   format.obj
 0001:00053bd0       ?dtor$3@?0???$fallback_format@N@detail@v6@fmt@@YAXNAEAV?$buffer@D@012@AEAH@Z@4HA 0000000180054bd0 f   format.obj
 0001:00053bd0       ?dtor$3@?0???$fallback_format@O@detail@v6@fmt@@YAXOAEAV?$buffer@D@012@AEAH@Z@4HA 0000000180054bd0 f   format.obj
 0001:00053be0       ?dtor$0@?0???$use_facet@V?$numpunct@_W@std@@@std@@YAAEBV?$numpunct@_W@0@AEBVlocale@0@@Z@4HA 0000000180054be0 f   format.obj
 0001:00053bf0       ?dtor$1@?0???$use_facet@V?$numpunct@_W@std@@@std@@YAAEBV?$numpunct@_W@0@AEBVlocale@0@@Z@4HA 0000000180054bf0 f   format.obj
 0001:00053c00       ?dtor$0@?0??_Getcat@?$numpunct@_W@std@@SA_KPEAPEBVfacet@locale@2@PEBV42@@Z@4HA 0000000180054c00 f   format.obj
 0001:00053c20       ?dtor$1@?0??_Getcat@?$numpunct@_W@std@@SA_KPEAPEBVfacet@locale@2@PEBV42@@Z@4HA 0000000180054c20 f   format.obj
 0001:00053c50       ?dtor$2@?0??_Getcat@?$numpunct@_W@std@@SA_KPEAPEBVfacet@locale@2@PEBV42@@Z@4HA 0000000180054c50 f   format.obj
 0001:00053c60       ?dtor$3@?0??_Getcat@?$numpunct@_W@std@@SA_KPEAPEBVfacet@locale@2@PEBV42@@Z@4HA 0000000180054c60 f   format.obj
 0001:00053c70       ?dtor$4@?0??_Getcat@?$numpunct@_W@std@@SA_KPEAPEBVfacet@locale@2@PEBV42@@Z@4HA 0000000180054c70 f   format.obj
 0001:00053c80       ?dtor$5@?0??_Getcat@?$numpunct@_W@std@@SA_KPEAPEBVfacet@locale@2@PEBV42@@Z@4HA 0000000180054c80 f   format.obj
 0001:00053c90       ?dtor$6@?0??_Getcat@?$numpunct@_W@std@@SA_KPEAPEBVfacet@locale@2@PEBV42@@Z@4HA 0000000180054c90 f   format.obj
 0001:00053ca0       ?dtor$7@?0??_Getcat@?$numpunct@_W@std@@SA_KPEAPEBVfacet@locale@2@PEBV42@@Z@4HA 0000000180054ca0 f   format.obj
 0001:00053cb0       ?dtor$8@?0??_Getcat@?$numpunct@_W@std@@SA_KPEAPEBVfacet@locale@2@PEBV42@@Z@4HA 0000000180054cb0 f   format.obj
 0001:00053cc0       ?dtor$9@?0??_Getcat@?$numpunct@_W@std@@SA_KPEAPEBVfacet@locale@2@PEBV42@@Z@4HA 0000000180054cc0 f   format.obj
 0001:00053cd0       ?dtor$0@?0??_Init@?$numpunct@_W@std@@IEAAXAEBV_Locinfo@2@_N@Z@4HA 0000000180054cd0 f   format.obj
 0001:00053ce0       ?dtor$0@?0??on_error@error_handler@detail@v6@fmt@@QEAAXPEBD@Z@4HA 0000000180054ce0 f   format.obj
 0001:00053ce0       ?dtor$0@?0???$visit_format_arg@U?$default_arg_formatter@V?$back_insert_iterator@V?$buffer@_W@detail@v6@fmt@@@std@@_W@detail@v6@fmt@@V?$basic_format_context@V?$back_insert_iterator@V?$buffer@_W@detail@v6@fmt@@@std@@_W@34@@v6@fmt@@YA?AV?$back_insert_iterator@V?$buffer@_W@detail@v6@fmt@@@std@@$$QEAU?$default_arg_formatter@V?$back_insert_iterator@V?$buffer@_W@detail@v6@fmt@@@std@@_W@detail@01@AEBV?$basic_format_arg@V?$basic_format_context@V?$back_insert_iterator@V?$buffer@_W@detail@v6@fmt@@@std@@_W@v6@fmt@@@01@@Z@4HA 0000000180054ce0 f   handles.obj
 0001:00053ce0       ?dtor$0@?0??on_fill@?$specs_setter@_W@detail@v6@fmt@@QEAAXV?$basic_string_view@_W@34@@Z@4HA 0000000180054ce0 f   handles.obj
 0001:00053ce0       ?dtor$0@?0??write@?$arg_formatter_base@V?$back_insert_iterator@V?$buffer@_W@detail@v6@fmt@@@std@@_WUerror_handler@detail@v6@fmt@@@detail@v6@fmt@@IEAAXPEB_W@Z@4HA 0000000180054ce0 f   handles.obj
 0001:00053cf0       ?dtor$0@?0??square@bigint@detail@v6@fmt@@QEAAXXZ@4HA 0000000180054cf0 f   format.obj
 0001:00053d00       ?dtor$0@?0???$handle_int_type_spec@AEAU?$int_writer@V?$back_insert_iterator@V?$buffer@_W@detail@v6@fmt@@@std@@_WI@detail@v6@fmt@@@detail@v6@fmt@@YAXDAEAU?$int_writer@V?$back_insert_iterator@V?$buffer@_W@detail@v6@fmt@@@std@@_WI@012@@Z@4HA 0000000180054d00 f   handles.obj
 0001:00053d00       ?dtor$0@?0???$handle_int_type_spec@AEAU?$int_writer@V?$back_insert_iterator@V?$buffer@_W@detail@v6@fmt@@@std@@_W_K@detail@v6@fmt@@@detail@v6@fmt@@YAXDAEAU?$int_writer@V?$back_insert_iterator@V?$buffer@_W@detail@v6@fmt@@@std@@_W_K@012@@Z@4HA 0000000180054d00 f   handles.obj
 0001:00053d10       ?dtor$0@?0???$vformat@_W$0A@@detail@v6@fmt@@YA?AV?$basic_string@_WU?$char_traits@_W@std@@V?$allocator@_W@2@@std@@V?$basic_string_view@_W@12@V?$basic_format_args@V?$basic_format_context@V?$back_insert_iterator@V?$buffer@_W@detail@v6@fmt@@@std@@_W@v6@fmt@@@12@@Z@4HA 0000000180054d10 f   handles.obj
 0001:00053d20       ?dtor$0@?0???$write@_WV?$back_insert_iterator@V?$buffer@_W@detail@v6@fmt@@@std@@M$0A@@detail@v6@fmt@@YA?AV?$back_insert_iterator@V?$buffer@_W@detail@v6@fmt@@@std@@V34@M@Z@4HA 0000000180054d20 f   handles.obj
 0001:00053d20       ?dtor$0@?0???$write@_WV?$back_insert_iterator@V?$buffer@_W@detail@v6@fmt@@@std@@N$0A@@detail@v6@fmt@@YA?AV?$back_insert_iterator@V?$buffer@_W@detail@v6@fmt@@@std@@V34@N@Z@4HA 0000000180054d20 f   handles.obj
 0001:00053d20       ?dtor$0@?0???$write@_WV?$back_insert_iterator@V?$buffer@_W@detail@v6@fmt@@@std@@O$0A@@detail@v6@fmt@@YA?AV?$back_insert_iterator@V?$buffer@_W@detail@v6@fmt@@@std@@V34@O@Z@4HA 0000000180054d20 f   handles.obj
 0001:00053d30       ?dtor$0@?0???$write@_WV?$back_insert_iterator@V?$buffer@_W@detail@v6@fmt@@@std@@M$0A@@detail@v6@fmt@@YA?AV?$back_insert_iterator@V?$buffer@_W@detail@v6@fmt@@@std@@V34@MU?$basic_format_specs@_W@12@Vlocale_ref@012@@Z@4HA 0000000180054d30 f   handles.obj
 0001:00053d30       ?dtor$0@?0???$write@_WV?$back_insert_iterator@V?$buffer@_W@detail@v6@fmt@@@std@@N$0A@@detail@v6@fmt@@YA?AV?$back_insert_iterator@V?$buffer@_W@detail@v6@fmt@@@std@@V34@NU?$basic_format_specs@_W@12@Vlocale_ref@012@@Z@4HA 0000000180054d30 f   handles.obj
 0001:00053d30       ?dtor$0@?0???$write@_WV?$back_insert_iterator@V?$buffer@_W@detail@v6@fmt@@@std@@O$0A@@detail@v6@fmt@@YA?AV?$back_insert_iterator@V?$buffer@_W@detail@v6@fmt@@@std@@V34@OU?$basic_format_specs@_W@12@Vlocale_ref@012@@Z@4HA 0000000180054d30 f   handles.obj
 0001:00053d40       ?dtor$1@?0???$write@_WV?$back_insert_iterator@V?$buffer@_W@detail@v6@fmt@@@std@@M$0A@@detail@v6@fmt@@YA?AV?$back_insert_iterator@V?$buffer@_W@detail@v6@fmt@@@std@@V34@MU?$basic_format_specs@_W@12@Vlocale_ref@012@@Z@4HA 0000000180054d40 f   handles.obj
 0001:00053d40       ?dtor$1@?0???$write@_WV?$back_insert_iterator@V?$buffer@_W@detail@v6@fmt@@@std@@N$0A@@detail@v6@fmt@@YA?AV?$back_insert_iterator@V?$buffer@_W@detail@v6@fmt@@@std@@V34@NU?$basic_format_specs@_W@12@Vlocale_ref@012@@Z@4HA 0000000180054d40 f   handles.obj
 0001:00053d40       ?dtor$1@?0???$write@_WV?$back_insert_iterator@V?$buffer@_W@detail@v6@fmt@@@std@@O$0A@@detail@v6@fmt@@YA?AV?$back_insert_iterator@V?$buffer@_W@detail@v6@fmt@@@std@@V34@OU?$basic_format_specs@_W@12@Vlocale_ref@012@@Z@4HA 0000000180054d40 f   handles.obj
 0001:00053d50       ?dtor$1@?0???R<lambda_c3630acb37279cf92411e07a2b271fdf>@@QEBA?AV?$basic_string@_WU?$char_traits@_W@std@@V?$allocator@_W@2@@std@@XZ@4HA 0000000180054d50 f   handles.obj
 0001:00053d60       ?dtor$2@?0???R<lambda_c3630acb37279cf92411e07a2b271fdf>@@QEBA?AV?$basic_string@_WU?$char_traits@_W@std@@V?$allocator@_W@2@@std@@XZ@4HA 0000000180054d60 f   handles.obj
 0001:00053d70       ?dtor$3@?0???R<lambda_c3630acb37279cf92411e07a2b271fdf>@@QEBA?AV?$basic_string@_WU?$char_traits@_W@std@@V?$allocator@_W@2@@std@@XZ@4HA 0000000180054d70 f   handles.obj
 0001:00053d80       ?dtor$1@?0??GetNameByType@@YA?AV?$basic_string@_WU?$char_traits@_W@std@@V?$allocator@_W@2@@std@@PEAXGPEAVPerfThread@@@Z@4HA 0000000180054d80 f   handles.obj
 0001:00053d90       ?dtor$0@?0??query_object@@YA?AV?$unique_ptr@$$BY0A@DU?$default_delete@$$BY0A@D@std@@@std@@PEAXW4OBJECT_INFORMATION_CLASS@@@Z@4HA 0000000180054d90 f   handles.obj
 0001:00053d90       ?dtor$2@?0??GetNameByType@@YA?AV?$basic_string@_WU?$char_traits@_W@std@@V?$allocator@_W@2@@std@@PEAXGPEAVPerfThread@@@Z@4HA 0000000180054d90 f   handles.obj
 0001:00053da0       ?dtor$0@?0??Connect@Plist@@QEAA_NPEB_W00@Z@4HA 0000000180054da0 f   Pclass.obj
 0001:00053da0       ?dtor$0@?0??DeleteFiles@Plist@@QEAAHPEAUPluginPanelItem@@_K1@Z@4HA 0000000180054da0 f   Pclass.obj
 0001:00053da0       ?dtor$11@?0??GetFiles@Plist@@QEAAHPEAUPluginPanelItem@@_KHPEAPEB_W1AEAUoptions@@@Z@4HA 0000000180054da0 f   Pclass.obj
 0001:00053da0       ?dtor$12@?0??GetFiles@Plist@@QEAAHPEAUPluginPanelItem@@_KHPEAPEB_W1AEAUoptions@@@Z@4HA 0000000180054da0 f   Pclass.obj
 0001:00053da0       ?dtor$13@?0??GetFiles@Plist@@QEAAHPEAUPluginPanelItem@@_KHPEAPEB_W1AEAUoptions@@@Z@4HA 0000000180054da0 f   Pclass.obj
 0001:00053da0       ?dtor$15@?0??GetFiles@Plist@@QEAAHPEAUPluginPanelItem@@_KHPEAPEB_W1AEAUoptions@@@Z@4HA 0000000180054da0 f   Pclass.obj
 0001:00053da0       ?dtor$18@?0??GetFiles@Plist@@QEAAHPEAUPluginPanelItem@@_KHPEAPEB_W1AEAUoptions@@@Z@4HA 0000000180054da0 f   Pclass.obj
 0001:00053da0       ?dtor$20@?0??GetFiles@Plist@@QEAAHPEAUPluginPanelItem@@_KHPEAPEB_W1AEAUoptions@@@Z@4HA 0000000180054da0 f   Pclass.obj
 0001:00053da0       ?dtor$23@?0??GetFiles@Plist@@QEAAHPEAUPluginPanelItem@@_KHPEAPEB_W1AEAUoptions@@@Z@4HA 0000000180054da0 f   Pclass.obj
 0001:00053da0       ?dtor$24@?0??GetFiles@Plist@@QEAAHPEAUPluginPanelItem@@_KHPEAPEB_W1AEAUoptions@@@Z@4HA 0000000180054da0 f   Pclass.obj
 0001:00053da0       ?dtor$29@?0??GetFiles@Plist@@QEAAHPEAUPluginPanelItem@@_KHPEAPEB_W1AEAUoptions@@@Z@4HA 0000000180054da0 f   Pclass.obj
 0001:00053da0       ?dtor$2@?0??PrintVersionInfo@Plist@@CAXPEAXPEB_W@Z@4HA 0000000180054da0 f   Pclass.obj
 0001:00053da0       ?dtor$31@?0??GetFiles@Plist@@QEAAHPEAUPluginPanelItem@@_KHPEAPEB_W1AEAUoptions@@@Z@4HA 0000000180054da0 f   Pclass.obj
 0001:00053da0       ?dtor$33@?0??GetFiles@Plist@@QEAAHPEAUPluginPanelItem@@_KHPEAPEB_W1AEAUoptions@@@Z@4HA 0000000180054da0 f   Pclass.obj
 0001:00053da0       ?dtor$35@?0??GetFiles@Plist@@QEAAHPEAUPluginPanelItem@@_KHPEAPEB_W1AEAUoptions@@@Z@4HA 0000000180054da0 f   Pclass.obj
 0001:00053da0       ?dtor$38@?0??GetFiles@Plist@@QEAAHPEAUPluginPanelItem@@_KHPEAPEB_W1AEAUoptions@@@Z@4HA 0000000180054da0 f   Pclass.obj
 0001:00053da0       ?dtor$3@?0??DeleteFiles@Plist@@QEAAHPEAUPluginPanelItem@@_K1@Z@4HA 0000000180054da0 f   Pclass.obj
 0001:00053da0       ?dtor$3@?0??GetFiles@Plist@@QEAAHPEAUPluginPanelItem@@_KHPEAPEB_W1AEAUoptions@@@Z@4HA 0000000180054da0 f   Pclass.obj
 0001:00053da0       ?dtor$3@?0??PrintOwnerInfo@Plist@@AEAAXPEAXK@Z@4HA 0000000180054da0 f   Pclass.obj
 0001:00053da0       ?dtor$41@?0??GetFiles@Plist@@QEAAHPEAUPluginPanelItem@@_KHPEAPEB_W1AEAUoptions@@@Z@4HA 0000000180054da0 f   Pclass.obj
 0001:00053da0       ?dtor$42@?0??GetFiles@Plist@@QEAAHPEAUPluginPanelItem@@_KHPEAPEB_W1AEAUoptions@@@Z@4HA 0000000180054da0 f   Pclass.obj
 0001:00053da0       ?dtor$4@?0??PrintOwnerInfo@Plist@@AEAAXPEAXK@Z@4HA 0000000180054da0 f   Pclass.obj
 0001:00053da0       ?dtor$4@?0??PrintVersionInfo@Plist@@CAXPEAXPEB_W@Z@4HA 0000000180054da0 f   Pclass.obj
 0001:00053da0       ?dtor$5@?0??GetFiles@Plist@@QEAAHPEAUPluginPanelItem@@_KHPEAPEB_W1AEAUoptions@@@Z@4HA 0000000180054da0 f   Pclass.obj
 0001:00053da0       ?dtor$5@?0??PrintOwnerInfo@Plist@@AEAAXPEAXK@Z@4HA 0000000180054da0 f   Pclass.obj
 0001:00053da0       ?dtor$7@?0??GetFiles@Plist@@QEAAHPEAUPluginPanelItem@@_KHPEAPEB_W1AEAUoptions@@@Z@4HA 0000000180054da0 f   Pclass.obj
 0001:00053da0       ?dtor$9@?0??GetFiles@Plist@@QEAAHPEAUPluginPanelItem@@_KHPEAPEB_W1AEAUoptions@@@Z@4HA 0000000180054da0 f   Pclass.obj
 0001:00053da0       ?dtor$1@?0??WinError@@YAHPEB_W@Z@4HA 0000000180054da0 f   Pmix.obj
 0001:00053da0       ?dtor$3@?0??GetNameByType@@YA?AV?$basic_string@_WU?$char_traits@_W@std@@V?$allocator@_W@2@@std@@PEAXGPEAVPerfThread@@@Z@4HA 0000000180054da0 f   handles.obj
 0001:00053db0       ?dtor$12@?0??GetNameByType@@YA?AV?$basic_string@_WU?$char_traits@_W@std@@V?$allocator@_W@2@@std@@PEAXGPEAVPerfThread@@@Z@4HA 0000000180054db0 f   handles.obj
 0001:00053db0       ?dtor$3@?0??PrintHandleInfo@@YA_NKPEAX_NPEAVPerfThread@@@Z@4HA 0000000180054db0 f   handles.obj
 0001:00053dc0       ?dtor$14@?0??GetNameByType@@YA?AV?$basic_string@_WU?$char_traits@_W@std@@V?$allocator@_W@2@@std@@PEAXGPEAVPerfThread@@@Z@4HA 0000000180054dc0 f   handles.obj
 0001:00053dd0       ?dtor$20@?0??GetNameByType@@YA?AV?$basic_string@_WU?$char_traits@_W@std@@V?$allocator@_W@2@@std@@PEAXGPEAVPerfThread@@@Z@4HA 0000000180054dd0 f   handles.obj
 0001:00053df0       ?dtor$0@?0??PrintHandleInfo@@YA_NKPEAX_NPEAVPerfThread@@@Z@4HA 0000000180054df0 f   handles.obj
 0001:00053e00       ?dtor$1@?0??GetVersionInfo@Plist@@SA_NPEB_WAEAV?$unique_ptr@$$BY0A@DU?$default_delete@$$BY0A@D@std@@@std@@AEAPEB_W2@Z@4HA 0000000180054e00 f   Pclass.obj
 0001:00053e00       ?dtor$3@?0??DumpNTCounters@@YAXPEAXAEAVPerfThread@@KK@Z@4HA 0000000180054e00 f   Pclass.obj
 0001:00053e00       ?dtor$6@?0??DumpNTCounters@@YAXPEAXAEAVPerfThread@@KK@Z@4HA 0000000180054e00 f   Pclass.obj
 0001:00053e00       ?dtor$7@?0??PrintOwnerInfo@Plist@@AEAAXPEAXK@Z@4HA 0000000180054e00 f   Pclass.obj
 0001:00053e00       ?dtor$0@?0??print_module_impl@@YAXQEAXAEBV?$basic_string@_WU?$char_traits@_W@std@@V?$allocator@_W@2@@std@@KAEBUoptions@@AEBV?$function@$$A6A_NPEA_W_K@Z@2@@Z@4HA 0000000180054e00 f   Plist.obj
 0001:00053e00       ?dtor$2@?0??PrintHandleInfo@@YA_NKPEAX_NPEAVPerfThread@@@Z@4HA 0000000180054e00 f   handles.obj
 0001:00053e00       ?dtor$6@?0??PrintHandleInfo@@YA_NKPEAX_NPEAVPerfThread@@@Z@4HA 0000000180054e00 f   handles.obj
 0001:00053e00       ?dtor$2@?0??RefreshWMIData@PerfThread@@AEAAXXZ@4HA 0000000180054e00 f   perfthread.obj
 0001:00053e10       ?dtor$5@?0??PrintHandleInfo@@YA_NKPEAX_NPEAVPerfThread@@@Z@4HA 0000000180054e10 f   handles.obj
 0001:00053e20       ?dtor$7@?0??PrintHandleInfo@@YA_NKPEAX_NPEAVPerfThread@@@Z@4HA 0000000180054e20 f   handles.obj
 0001:00053e30       ?dtor$20@?0??PrintHandleInfo@@YA_NKPEAX_NPEAVPerfThread@@@Z@4HA 0000000180054e30 f   handles.obj
 0001:00053e30       ?dtor$22@?0??PrintHandleInfo@@YA_NKPEAX_NPEAVPerfThread@@@Z@4HA 0000000180054e30 f   handles.obj
 0001:00053e40       ?dtor$0@?0??duplicate_handle@@YA?AV?$unique_ptr@XUhandle_closer@@@std@@PEAXK@Z@4HA 0000000180054e40 f   handles.obj
 0001:00053e50       ?dtor$0@?0??on_num@?$int_writer@V?$back_insert_iterator@V?$buffer@_W@detail@v6@fmt@@@std@@_WI@detail@v6@fmt@@QEAAXXZ@4HA 0000000180054e50 f   handles.obj
 0001:00053e50       ?dtor$0@?0??on_num@?$int_writer@V?$back_insert_iterator@V?$buffer@_W@detail@v6@fmt@@@std@@_W_K@detail@v6@fmt@@QEAAXXZ@4HA 0000000180054e50 f   handles.obj
 0001:00053e60       ?dtor$1@?0??on_num@?$int_writer@V?$back_insert_iterator@V?$buffer@_W@detail@v6@fmt@@@std@@_WI@detail@v6@fmt@@QEAAXXZ@4HA 0000000180054e60 f   handles.obj
 0001:00053e60       ?dtor$1@?0??on_num@?$int_writer@V?$back_insert_iterator@V?$buffer@_W@detail@v6@fmt@@@std@@_W_K@detail@v6@fmt@@QEAAXXZ@4HA 0000000180054e60 f   handles.obj
 0001:00053e70       ?dtor$0@?0??Config@@YAHXZ@4HA 0000000180054e70 f   Pcfg.obj
 0001:00053e80       ?dtor$0@?0??Read@options@@QEAAXXZ@4HA 0000000180054e80 f   Pcfg.obj
 0001:00053e80       ?dtor$0@?0??Write@options@@QEBAXXZ@4HA 0000000180054e80 f   Pcfg.obj
 0001:00053e80       ?dtor$3@?0???0Plist@@QEAA@XZ@4HA 0000000180054e80 f   Pclass.obj
 0001:00053e90       ?dtor$0@?0???$_Assign_range@PEBUmode@@@?$vector@Umode@@V?$allocator@Umode@@@std@@@std@@AEAAXPEBUmode@@0Uforward_iterator_tag@1@@Z@4HA 0000000180054e90 f   Pclass.obj
 0001:00053ea0       ?dtor$1@?0???$_Assign_range@PEBUmode@@@?$vector@Umode@@V?$allocator@Umode@@@std@@@std@@AEAAXPEBUmode@@0Uforward_iterator_tag@1@@Z@4HA 0000000180054ea0 f   Pclass.obj
 0001:00053eb0       ?dtor$3@?0???$_Assign_range@PEBUmode@@@?$vector@Umode@@V?$allocator@Umode@@@std@@@std@@AEAAXPEBUmode@@0Uforward_iterator_tag@1@@Z@4HA 0000000180054eb0 f   Pclass.obj
 0001:00053eb0       ?dtor$6@?0???$_Assign_range@PEBUmode@@@?$vector@Umode@@V?$allocator@Umode@@@std@@@std@@AEAAXPEBUmode@@0Uforward_iterator_tag@1@@Z@4HA 0000000180054eb0 f   Pclass.obj
 0001:00053ec0       ?dtor$4@?0???$_Assign_range@PEBUmode@@@?$vector@Umode@@V?$allocator@Umode@@@std@@@std@@AEAAXPEBUmode@@0Uforward_iterator_tag@1@@Z@4HA 0000000180054ec0 f   Pclass.obj
 0001:00053ec0       ?dtor$7@?0???$_Assign_range@PEBUmode@@@?$vector@Umode@@V?$allocator@Umode@@@std@@@std@@AEAAXPEBUmode@@0Uforward_iterator_tag@1@@Z@4HA 0000000180054ec0 f   Pclass.obj
 0001:00053ed0       ?catch$8@?0???$_Emplace_reallocate@V?$basic_string@_WU?$char_traits@_W@std@@V?$allocator@_W@2@@std@@@?$vector@V?$basic_string@_WU?$char_traits@_W@std@@V?$allocator@_W@2@@std@@V?$allocator@V?$basic_string@_WU?$char_traits@_W@std@@V?$allocator@_W@2@@std@@@2@@std@@QEAAPEAV?$basic_string@_WU?$char_traits@_W@std@@V?$allocator@_W@2@@1@QEAV21@$$QEAV21@@Z@4HA 0000000180054ed0 f   Pclass.obj
 0001:00053ede       __catch$??$_Emplace_reallocate@V?$basic_string@_WU?$char_traits@_W@std@@V?$allocator@_W@2@@std@@@?$vector@V?$basic_string@_WU?$char_traits@_W@std@@V?$allocator@_W@2@@std@@V?$allocator@V?$basic_string@_WU?$char_traits@_W@std@@V?$allocator@_W@2@@std@@@2@@std@@QEAAPEAV?$basic_string@_WU?$char_traits@_W@std@@V?$allocator@_W@2@@1@QEAV21@$$QEAV21@@Z$0 0000000180054ede f   Pclass.obj
 0001:00053f20       ?catch$0@?0???$_Resize_reallocate@U_Value_init_tag@std@@@?$vector@PEB_WV?$allocator@PEB_W@std@@@std@@AEAAX_KAEBU_Value_init_tag@1@@Z@4HA 0000000180054f20 f   Pclass.obj
 0001:00053f2d       __catch$??$_Resize_reallocate@U_Value_init_tag@std@@@?$vector@PEB_WV?$allocator@PEB_W@std@@@std@@AEAAX_KAEBU_Value_init_tag@1@@Z$0 0000000180054f2d f   Pclass.obj
 0001:00053f50       ?dtor$0@?0???$_Try_emplace@AEBK$$V@?$_Hash@V?$_Umap_traits@KPEAUHWND__@@V?$_Uhash_compare@KU?$hash@K@std@@U?$equal_to@K@2@@std@@V?$allocator@U?$pair@$$CBKPEAUHWND__@@@std@@@3@$0A@@std@@@std@@IEAA?AU?$pair@PEAU?$_List_node@U?$pair@$$CBKPEAUHWND__@@@std@@PEAX@std@@_N@1@AEBK@Z@4HA 0000000180054f50 f   Pclass.obj
 0001:00053f50       ?dtor$1@?0???$_Try_emplace@AEBK$$V@?$_Hash@V?$_Umap_traits@KPEAUHWND__@@V?$_Uhash_compare@KU?$hash@K@std@@U?$equal_to@K@2@@std@@V?$allocator@U?$pair@$$CBKPEAUHWND__@@@std@@@3@$0A@@std@@@std@@IEAA?AU?$pair@PEAU?$_List_node@U?$pair@$$CBKPEAUHWND__@@@std@@PEAX@std@@_N@1@AEBK@Z@4HA 0000000180054f50 f   Pclass.obj
 0001:00053f60       ?dtor$0@?0???0Plist@@QEAA@XZ@4HA 0000000180054f60 f   Pclass.obj
 0001:00053f70       ?dtor$1@?0???0Plist@@QEAA@XZ@4HA 0000000180054f70 f   Pclass.obj
 0001:00053f80       ?dtor$2@?0???0Plist@@QEAA@XZ@4HA 0000000180054f80 f   Pclass.obj
 0001:00053f90       ?dtor$7@?0???0Plist@@QEAA@XZ@4HA 0000000180054f90 f   Pclass.obj
 0001:00053fb0       ?dtor$0@?0??Compare@Plist@@QEBAHPEBUPluginPanelItem@@0I@Z@4HA 0000000180054fb0 f   Pclass.obj
 0001:00053fc0       ?dtor$1@?0??Connect@Plist@@QEAA_NPEB_W00@Z@4HA 0000000180054fc0 f   Pclass.obj
 0001:00053fd0       ?dtor$3@?0??Connect@Plist@@QEAA_NPEB_W00@Z@4HA 0000000180054fd0 f   Pclass.obj
 0001:00053ff0       ?dtor$1@?0??ConnectWMI@Plist@@AEAA_NXZ@4HA 0000000180054ff0 f   Pclass.obj
 0001:00054010       ?dtor$0@?0??DumpNTCounters@@YAXPEAXAEAVPerfThread@@KK@Z@4HA 0000000180055010 f   Pclass.obj
 0001:00054020       ?dtor$0@?0??TranslateMode@@YA_NAEBV?$basic_string@_WU?$char_traits@_W@std@@V?$allocator@_W@2@@std@@AEAV12@@Z@4HA 0000000180055020 f   Pclass.obj
 0001:00054020       ?dtor$0@?0??window_ex_style@@YA@PEAUHWND__@@@Z@4HA 0000000180055020 f   Pclass.obj
 0001:00054020       ?dtor$0@?0??window_style@@YA@PEAUHWND__@@@Z@4HA 0000000180055020 f   Pclass.obj
 0001:00054020       ?dtor$183@?0??InitializePanelModes@Plist@@SAXXZ@4HA 0000000180055020 f   Pclass.obj
 0001:00054020       ?dtor$1@?0??DumpNTCounters@@YAXPEAXAEAVPerfThread@@KK@Z@4HA 0000000180055020 f   Pclass.obj
 0001:00054020       ?dtor$1@?0??SavePanelModes@Plist@@SAXXZ@4HA 0000000180055020 f   Pclass.obj
 0001:00054020       ?dtor$4@?0??DumpNTCounters@@YAXPEAXAEAVPerfThread@@KK@Z@4HA 0000000180055020 f   Pclass.obj
 0001:00054020       ?dtor$7@?0??DumpNTCounters@@YAXPEAXAEAVPerfThread@@KK@Z@4HA 0000000180055020 f   Pclass.obj
 0001:00054030       ?dtor$2@?0??DumpNTCounters@@YAXPEAXAEAVPerfThread@@KK@Z@4HA 0000000180055030 f   Pclass.obj
 0001:00054030       ?dtor$2@?0??GetVersionInfo@Plist@@SA_NPEB_WAEAV?$unique_ptr@$$BY0A@DU?$default_delete@$$BY0A@D@std@@@std@@AEAPEB_W2@Z@4HA 0000000180055030 f   Pclass.obj
 0001:00054030       ?dtor$5@?0??DumpNTCounters@@YAXPEAXAEAVPerfThread@@KK@Z@4HA 0000000180055030 f   Pclass.obj
 0001:00054030       ?dtor$0@?0???$print_module@PEAX@@YAXQEAXPEAXKAEAUoptions@@AEBV?$function@$$A6A_NPEA_W_K@Z@std@@@Z@4HA 0000000180055030 f   Plist.obj
 0001:00054030       ?dtor$1@?0??print_module_impl@@YAXQEAXAEBV?$basic_string@_WU?$char_traits@_W@std@@V?$allocator@_W@2@@std@@KAEBUoptions@@AEBV?$function@$$A6A_NPEA_W_K@Z@2@@Z@4HA 0000000180055030 f   Plist.obj
 0001:00054040       ?dtor$0@?0??GetFiles@Plist@@QEAAHPEAUPluginPanelItem@@_KHPEAPEB_W1AEAUoptions@@@Z@4HA 0000000180055040 f   Pclass.obj
 0001:00054050       ?dtor$1@?0??GetFiles@Plist@@QEAAHPEAUPluginPanelItem@@_KHPEAPEB_W1AEAUoptions@@@Z@4HA 0000000180055050 f   Pclass.obj
 0001:00054050       ?dtor$0@?0??PrintNTCurDirAndEnv@@YAXPEAX0H@Z@4HA 0000000180055050 f   Plist.obj
 0001:00054060       ?dtor$2@?0??GetFiles@Plist@@QEAAHPEAUPluginPanelItem@@_KHPEAPEB_W1AEAUoptions@@@Z@4HA 0000000180055060 f   Pclass.obj
 0001:00054070       ?dtor$4@?0??GetFiles@Plist@@QEAAHPEAUPluginPanelItem@@_KHPEAPEB_W1AEAUoptions@@@Z@4HA 0000000180055070 f   Pclass.obj
 0001:00054070       ?dtor$6@?0??GetFiles@Plist@@QEAAHPEAUPluginPanelItem@@_KHPEAPEB_W1AEAUoptions@@@Z@4HA 0000000180055070 f   Pclass.obj
 0001:00054070       ?dtor$8@?0??GetFiles@Plist@@QEAAHPEAUPluginPanelItem@@_KHPEAPEB_W1AEAUoptions@@@Z@4HA 0000000180055070 f   Pclass.obj
 0001:00054070       ?dtor$2@?0??PrintNTCurDirAndEnv@@YAXPEAX0H@Z@4HA 0000000180055070 f   Plist.obj
 0001:00054070       ?dtor$3@?0??PrintNTCurDirAndEnv@@YAXPEAX0H@Z@4HA 0000000180055070 f   Plist.obj
 0001:00054080       ?dtor$10@?0??GetFiles@Plist@@QEAAHPEAUPluginPanelItem@@_KHPEAPEB_W1AEAUoptions@@@Z@4HA 0000000180055080 f   Pclass.obj
 0001:00054090       ?dtor$14@?0??GetFiles@Plist@@QEAAHPEAUPluginPanelItem@@_KHPEAPEB_W1AEAUoptions@@@Z@4HA 0000000180055090 f   Pclass.obj
 0001:00054090       ?dtor$16@?0??GetFiles@Plist@@QEAAHPEAUPluginPanelItem@@_KHPEAPEB_W1AEAUoptions@@@Z@4HA 0000000180055090 f   Pclass.obj
 0001:00054090       ?dtor$19@?0??GetFiles@Plist@@QEAAHPEAUPluginPanelItem@@_KHPEAPEB_W1AEAUoptions@@@Z@4HA 0000000180055090 f   Pclass.obj
 0001:00054090       ?dtor$1@?0??PrintVersionInfo@Plist@@CAXPEAXPEB_W@Z@4HA 0000000180055090 f   Pclass.obj
 0001:00054090       ?dtor$21@?0??GetFiles@Plist@@QEAAHPEAUPluginPanelItem@@_KHPEAPEB_W1AEAUoptions@@@Z@4HA 0000000180055090 f   Pclass.obj
 0001:00054090       ?dtor$3@?0??PrintVersionInfo@Plist@@CAXPEAXPEB_W@Z@4HA 0000000180055090 f   Pclass.obj
 0001:00054090       ?dtor$7@?0??GetFindData@Plist@@QEAAHAEAPEAUPluginPanelItem@@AEA_K_K@Z@4HA 0000000180055090 f   Pclass.obj
 0001:00054090       ?dtor$1@?0??PrintNTCurDirAndEnv@@YAXPEAX0H@Z@4HA 0000000180055090 f   Plist.obj
 0001:000540a0       ?dtor$17@?0??GetFiles@Plist@@QEAAHPEAUPluginPanelItem@@_KHPEAPEB_W1AEAUoptions@@@Z@4HA 00000001800550a0 f   Pclass.obj
 0001:000540a0       ?dtor$4@?0??PrintNTCurDirAndEnv@@YAXPEAX0H@Z@4HA 00000001800550a0 f   Plist.obj
 0001:000540b0       ?dtor$22@?0??GetFiles@Plist@@QEAAHPEAUPluginPanelItem@@_KHPEAPEB_W1AEAUoptions@@@Z@4HA 00000001800550b0 f   Pclass.obj
 0001:000540b0       ?dtor$34@?0??GetFiles@Plist@@QEAAHPEAUPluginPanelItem@@_KHPEAPEB_W1AEAUoptions@@@Z@4HA 00000001800550b0 f   Pclass.obj
 0001:000540b0       ?dtor$6@?0??PrintOwnerInfo@Plist@@AEAAXPEAXK@Z@4HA 00000001800550b0 f   Pclass.obj
 0001:000540c0       ?dtor$25@?0??GetFiles@Plist@@QEAAHPEAUPluginPanelItem@@_KHPEAPEB_W1AEAUoptions@@@Z@4HA 00000001800550c0 f   Pclass.obj
 0001:000540d0       ?dtor$26@?0??GetFiles@Plist@@QEAAHPEAUPluginPanelItem@@_KHPEAPEB_W1AEAUoptions@@@Z@4HA 00000001800550d0 f   Pclass.obj
 0001:000540e0       ?dtor$27@?0??GetFiles@Plist@@QEAAHPEAUPluginPanelItem@@_KHPEAPEB_W1AEAUoptions@@@Z@4HA 00000001800550e0 f   Pclass.obj
 0001:000540f0       ?dtor$28@?0??GetFiles@Plist@@QEAAHPEAUPluginPanelItem@@_KHPEAPEB_W1AEAUoptions@@@Z@4HA 00000001800550f0 f   Pclass.obj
 0001:000540f0       ?dtor$30@?0??GetFiles@Plist@@QEAAHPEAUPluginPanelItem@@_KHPEAPEB_W1AEAUoptions@@@Z@4HA 00000001800550f0 f   Pclass.obj
 0001:000540f0       ?dtor$32@?0??GetFiles@Plist@@QEAAHPEAUPluginPanelItem@@_KHPEAPEB_W1AEAUoptions@@@Z@4HA 00000001800550f0 f   Pclass.obj
 0001:000540f0       ?dtor$37@?0??GetFiles@Plist@@QEAAHPEAUPluginPanelItem@@_KHPEAPEB_W1AEAUoptions@@@Z@4HA 00000001800550f0 f   Pclass.obj
 0001:000540f0       ?dtor$40@?0??GetFiles@Plist@@QEAAHPEAUPluginPanelItem@@_KHPEAPEB_W1AEAUoptions@@@Z@4HA 00000001800550f0 f   Pclass.obj
 0001:00054100       ?dtor$36@?0??GetFiles@Plist@@QEAAHPEAUPluginPanelItem@@_KHPEAPEB_W1AEAUoptions@@@Z@4HA 0000000180055100 f   Pclass.obj
 0001:00054110       ?dtor$39@?0??GetFiles@Plist@@QEAAHPEAUPluginPanelItem@@_KHPEAPEB_W1AEAUoptions@@@Z@4HA 0000000180055110 f   Pclass.obj
 0001:00054120       ?dtor$0@?0??GetFindData@Plist@@QEAAHAEAPEAUPluginPanelItem@@AEA_K_K@Z@4HA 0000000180055120 f   Pclass.obj
 0001:00054130       ?dtor$1@?0??GetFindData@Plist@@QEAAHAEAPEAUPluginPanelItem@@AEA_K_K@Z@4HA 0000000180055130 f   Pclass.obj
 0001:00054140       ?dtor$2@?0??GetFindData@Plist@@QEAAHAEAPEAUPluginPanelItem@@AEA_K_K@Z@4HA 0000000180055140 f   Pclass.obj
 0001:00054150       ?dtor$3@?0??GetFindData@Plist@@QEAAHAEAPEAUPluginPanelItem@@AEA_K_K@Z@4HA 0000000180055150 f   Pclass.obj
 0001:00054160       ?dtor$4@?0??GetFindData@Plist@@QEAAHAEAPEAUPluginPanelItem@@AEA_K_K@Z@4HA 0000000180055160 f   Pclass.obj
 0001:00054160       ?dtor$6@?0??GetFindData@Plist@@QEAAHAEAPEAUPluginPanelItem@@AEA_K_K@Z@4HA 0000000180055160 f   Pclass.obj
 0001:00054170       ?dtor$5@?0??GetFindData@Plist@@QEAAHAEAPEAUPluginPanelItem@@AEA_K_K@Z@4HA 0000000180055170 f   Pclass.obj
 0001:00054180       ?dtor$13@?0??GetFindData@Plist@@QEAAHAEAPEAUPluginPanelItem@@AEA_K_K@Z@4HA 0000000180055180 f   Pclass.obj
 0001:00054190       ?dtor$14@?0??GetFindData@Plist@@QEAAHAEAPEAUPluginPanelItem@@AEA_K_K@Z@4HA 0000000180055190 f   Pclass.obj
 0001:000541a0       ?dtor$0@?0??ui64toa_width@@YA?AV?$basic_string@_WU?$char_traits@_W@std@@V?$allocator@_W@2@@std@@_KI_N@Z@4HA 00000001800551a0 f   Pclass.obj
 0001:000541a0       ?dtor$4@?0??GetVersionInfo@Plist@@SA_NPEB_WAEAV?$unique_ptr@$$BY0A@DU?$default_delete@$$BY0A@D@std@@@std@@AEAPEB_W2@Z@4HA 00000001800551a0 f   Pclass.obj
 0001:000541b0       ?dtor$0@?0??InitializePanelModes@Plist@@SAXXZ@4HA 00000001800551b0 f   Pclass.obj
 0001:000541c0       ?dtor$8@?0??InitializePanelModes@Plist@@SAXXZ@4HA 00000001800551c0 f   Pclass.obj
 0001:000541d0       ?dtor$9@?0??InitializePanelModes@Plist@@SAXXZ@4HA 00000001800551d0 f   Pclass.obj
 0001:000541e0       ?dtor$17@?0??InitializePanelModes@Plist@@SAXXZ@4HA 00000001800551e0 f   Pclass.obj
 0001:000541f0       ?dtor$18@?0??InitializePanelModes@Plist@@SAXXZ@4HA 00000001800551f0 f   Pclass.obj
 0001:00054200       ?dtor$26@?0??InitializePanelModes@Plist@@SAXXZ@4HA 0000000180055200 f   Pclass.obj
 0001:00054210       ?dtor$27@?0??InitializePanelModes@Plist@@SAXXZ@4HA 0000000180055210 f   Pclass.obj
 0001:00054220       ?dtor$35@?0??InitializePanelModes@Plist@@SAXXZ@4HA 0000000180055220 f   Pclass.obj
 0001:00054230       ?dtor$36@?0??InitializePanelModes@Plist@@SAXXZ@4HA 0000000180055230 f   Pclass.obj
 0001:00054240       ?dtor$44@?0??InitializePanelModes@Plist@@SAXXZ@4HA 0000000180055240 f   Pclass.obj
 0001:00054250       ?dtor$45@?0??InitializePanelModes@Plist@@SAXXZ@4HA 0000000180055250 f   Pclass.obj
 0001:00054260       ?dtor$53@?0??InitializePanelModes@Plist@@SAXXZ@4HA 0000000180055260 f   Pclass.obj
 0001:00054270       ?dtor$54@?0??InitializePanelModes@Plist@@SAXXZ@4HA 0000000180055270 f   Pclass.obj
 0001:00054280       ?dtor$62@?0??InitializePanelModes@Plist@@SAXXZ@4HA 0000000180055280 f   Pclass.obj
 0001:00054290       ?dtor$63@?0??InitializePanelModes@Plist@@SAXXZ@4HA 0000000180055290 f   Pclass.obj
 0001:000542a0       ?dtor$71@?0??InitializePanelModes@Plist@@SAXXZ@4HA 00000001800552a0 f   Pclass.obj
 0001:000542b0       ?dtor$72@?0??InitializePanelModes@Plist@@SAXXZ@4HA 00000001800552b0 f   Pclass.obj
 0001:000542c0       ?dtor$80@?0??InitializePanelModes@Plist@@SAXXZ@4HA 00000001800552c0 f   Pclass.obj
 0001:000542d0       ?dtor$81@?0??InitializePanelModes@Plist@@SAXXZ@4HA 00000001800552d0 f   Pclass.obj
 0001:000542e0       ?dtor$90@?0??InitializePanelModes@Plist@@SAXXZ@4HA 00000001800552e0 f   Pclass.obj
 0001:00054310       ?dtor$91@?0??InitializePanelModes@Plist@@SAXXZ@4HA 0000000180055310 f   Pclass.obj
 0001:00054320       ?dtor$99@?0??InitializePanelModes@Plist@@SAXXZ@4HA 0000000180055320 f   Pclass.obj
 0001:00054330       ?dtor$100@?0??InitializePanelModes@Plist@@SAXXZ@4HA 0000000180055330 f   Pclass.obj
 0001:00054340       ?dtor$108@?0??InitializePanelModes@Plist@@SAXXZ@4HA 0000000180055340 f   Pclass.obj
 0001:00054350       ?dtor$109@?0??InitializePanelModes@Plist@@SAXXZ@4HA 0000000180055350 f   Pclass.obj
 0001:00054360       ?dtor$117@?0??InitializePanelModes@Plist@@SAXXZ@4HA 0000000180055360 f   Pclass.obj
 0001:00054370       ?dtor$118@?0??InitializePanelModes@Plist@@SAXXZ@4HA 0000000180055370 f   Pclass.obj
 0001:00054380       ?dtor$126@?0??InitializePanelModes@Plist@@SAXXZ@4HA 0000000180055380 f   Pclass.obj
 0001:00054390       ?dtor$127@?0??InitializePanelModes@Plist@@SAXXZ@4HA 0000000180055390 f   Pclass.obj
 0001:000543a0       ?dtor$135@?0??InitializePanelModes@Plist@@SAXXZ@4HA 00000001800553a0 f   Pclass.obj
 0001:000543b0       ?dtor$136@?0??InitializePanelModes@Plist@@SAXXZ@4HA 00000001800553b0 f   Pclass.obj
 0001:000543c0       ?dtor$144@?0??InitializePanelModes@Plist@@SAXXZ@4HA 00000001800553c0 f   Pclass.obj
 0001:000543d0       ?dtor$145@?0??InitializePanelModes@Plist@@SAXXZ@4HA 00000001800553d0 f   Pclass.obj
 0001:000543e0       ?dtor$153@?0??InitializePanelModes@Plist@@SAXXZ@4HA 00000001800553e0 f   Pclass.obj
 0001:000543f0       ?dtor$154@?0??InitializePanelModes@Plist@@SAXXZ@4HA 00000001800553f0 f   Pclass.obj
 0001:00054400       ?dtor$162@?0??InitializePanelModes@Plist@@SAXXZ@4HA 0000000180055400 f   Pclass.obj
 0001:00054410       ?dtor$163@?0??InitializePanelModes@Plist@@SAXXZ@4HA 0000000180055410 f   Pclass.obj
 0001:00054420       ?dtor$171@?0??InitializePanelModes@Plist@@SAXXZ@4HA 0000000180055420 f   Pclass.obj
 0001:00054430       ?dtor$172@?0??InitializePanelModes@Plist@@SAXXZ@4HA 0000000180055430 f   Pclass.obj
 0001:00054440       ?dtor$181@?0??InitializePanelModes@Plist@@SAXXZ@4HA 0000000180055440 f   Pclass.obj
 0001:00054470       ?dtor$182@?0??InitializePanelModes@Plist@@SAXXZ@4HA 0000000180055470 f   Pclass.obj
 0001:00054480       ?dtor$0@?0??PrintOwnerInfo@Plist@@AEAAXPEAXK@Z@4HA 0000000180055480 f   Pclass.obj
 0001:00054490       ?dtor$1@?0??PrintOwnerInfo@Plist@@AEAAXPEAXK@Z@4HA 0000000180055490 f   Pclass.obj
 0001:000544a0       ?dtor$2@?0??PrintOwnerInfo@Plist@@AEAAXPEAXK@Z@4HA 00000001800554a0 f   Pclass.obj
 0001:000544a0       ?dtor$2@?0??Connect@WMIConnection@@QEAA_NPEB_W00@Z@4HA 00000001800554a0 f   WMI.obj
 0001:000544b0       ?dtor$0@?0??PrintVersionInfo@Plist@@CAXPEAXPEB_W@Z@4HA 00000001800554b0 f   Pclass.obj
 0001:000544c0       ?dtor$0@?0??ProcessEvent@Plist@@QEAAH_JPEAX@Z@4HA 00000001800554c0 f   Pclass.obj
 0001:000544d0       ?dtor$0@?0??ProcessKey@Plist@@QEAAHPEBU_INPUT_RECORD@@@Z@4HA 00000001800554d0 f   Pclass.obj
 0001:000544d0       ?dtor$1@?0??ProcessKey@Plist@@QEAAHPEBU_INPUT_RECORD@@@Z@4HA 00000001800554d0 f   Pclass.obj
 0001:000544e0       ?dtor$2@?0??ProcessKey@Plist@@QEAAHPEBU_INPUT_RECORD@@@Z@4HA 00000001800554e0 f   Pclass.obj
 0001:000544e0       ?dtor$4@?0??ProcessKey@Plist@@QEAAHPEBU_INPUT_RECORD@@@Z@4HA 00000001800554e0 f   Pclass.obj
 0001:000544f0       ?dtor$3@?0??ProcessKey@Plist@@QEAAHPEBU_INPUT_RECORD@@@Z@4HA 00000001800554f0 f   Pclass.obj
 0001:00054500       ?dtor$7@?0??ProcessKey@Plist@@QEAAHPEBU_INPUT_RECORD@@@Z@4HA 0000000180055500 f   Pclass.obj
 0001:00054510       ?dtor$10@?0??ProcessKey@Plist@@QEAAHPEBU_INPUT_RECORD@@@Z@4HA 0000000180055510 f   Pclass.obj
 0001:00054510       ?dtor$8@?0??ProcessKey@Plist@@QEAAHPEBU_INPUT_RECORD@@@Z@4HA 0000000180055510 f   Pclass.obj
 0001:00054520       ?dtor$9@?0??ProcessKey@Plist@@QEAAHPEBU_INPUT_RECORD@@@Z@4HA 0000000180055520 f   Pclass.obj
 0001:00054530       ?dtor$11@?0??ProcessKey@Plist@@QEAAHPEBU_INPUT_RECORD@@@Z@4HA 0000000180055530 f   Pclass.obj
 0001:00054540       ?dtor$12@?0??ProcessKey@Plist@@QEAAHPEBU_INPUT_RECORD@@@Z@4HA 0000000180055540 f   Pclass.obj
 0001:00054550       ?dtor$25@?0??ProcessKey@Plist@@QEAAHPEBU_INPUT_RECORD@@@Z@4HA 0000000180055550 f   Pclass.obj
 0001:00054550       ?dtor$28@?0??ProcessKey@Plist@@QEAAHPEBU_INPUT_RECORD@@@Z@4HA 0000000180055550 f   Pclass.obj
 0001:00054570       ?dtor$32@?0??ProcessKey@Plist@@QEAAHPEBU_INPUT_RECORD@@@Z@4HA 0000000180055570 f   Pclass.obj
 0001:00054580       ?dtor$0@?0??SavePanelModes@Plist@@SAXXZ@4HA 0000000180055580 f   Pclass.obj
 0001:00054590       ?dtor$0@?0??generate_titles@@YAXAEBV?$basic_string@_WU?$char_traits@_W@std@@V?$allocator@_W@2@@std@@AEAUPanelMode@@@Z@4HA 0000000180055590 f   Pclass.obj
 0001:000545a0       ?catch$0@?0???$_Resize_reallocate@U_Value_init_tag@std@@@?$vector@EV?$allocator@E@std@@@std@@AEAAX_KAEBU_Value_init_tag@1@@Z@4HA 00000001800555a0 f   perfthread.obj
 0001:000545ad       __catch$??$_Resize_reallocate@U_Value_init_tag@std@@@?$vector@EV?$allocator@E@std@@@std@@AEAAX_KAEBU_Value_init_tag@1@@Z$0 00000001800555ad f   perfthread.obj
 0001:000545d0       ?dtor$0@?0???0PerfThread@@QEAA@PEB_W00@Z@4HA 00000001800555d0 f   perfthread.obj
 0001:000545e0       ?dtor$1@?0???0PerfThread@@QEAA@PEB_W00@Z@4HA 00000001800555e0 f   perfthread.obj
 0001:000545f0       ?dtor$2@?0???0PerfThread@@QEAA@PEB_W00@Z@4HA 00000001800555f0 f   perfthread.obj
 0001:00054600       ?dtor$3@?0???0PerfThread@@QEAA@PEB_W00@Z@4HA 0000000180055600 f   perfthread.obj
 0001:00054610       ?dtor$4@?0???0PerfThread@@QEAA@PEB_W00@Z@4HA 0000000180055610 f   perfthread.obj
 0001:00054620       ?dtor$5@?0???0PerfThread@@QEAA@PEB_W00@Z@4HA 0000000180055620 f   perfthread.obj
 0001:00054630       ?dtor$6@?0???0PerfThread@@QEAA@PEB_W00@Z@4HA 0000000180055630 f   perfthread.obj
 0001:00054650       ?dtor$7@?0???0PerfThread@@QEAA@PEB_W00@Z@4HA 0000000180055650 f   perfthread.obj
 0001:00054670       ?dtor$8@?0???0PerfThread@@QEAA@PEB_W00@Z@4HA 0000000180055670 f   perfthread.obj
 0001:00054690       ?dtor$9@?0???0PerfThread@@QEAA@PEB_W00@Z@4HA 0000000180055690 f   perfthread.obj
 0001:000546b0       ?dtor$10@?0???0PerfThread@@QEAA@PEB_W00@Z@4HA 00000001800556b0 f   perfthread.obj
 0001:000546d0       ?dtor$11@?0???0PerfThread@@QEAA@PEB_W00@Z@4HA 00000001800556d0 f   perfthread.obj
 0001:000546e0       ?dtor$13@?0???0PerfThread@@QEAA@PEB_W00@Z@4HA 00000001800556e0 f   perfthread.obj
 0001:000546f0       ?dtor$14@?0???0PerfThread@@QEAA@PEB_W00@Z@4HA 00000001800556f0 f   perfthread.obj
 0001:00054700       ?dtor$0@?0??Refresh@PerfThread@@AEAAXXZ@4HA 0000000180055700 f   perfthread.obj
 0001:00054710       ?dtor$1@?0??Refresh@PerfThread@@AEAAXXZ@4HA 0000000180055710 f   perfthread.obj
 0001:00054720       ?dtor$2@?0??Refresh@PerfThread@@AEAAXXZ@4HA 0000000180055720 f   perfthread.obj
 0001:00054730       ?dtor$5@?0??Refresh@PerfThread@@AEAAXXZ@4HA 0000000180055730 f   perfthread.obj
 0001:00054740       ?catch$0@?0???$_Resize_reallocate@U_Value_init_tag@std@@@?$vector@PEAUHINSTANCE__@@V?$allocator@PEAUHINSTANCE__@@@std@@@std@@AEAAX_KAEBU_Value_init_tag@1@@Z@4HA 0000000180055740 f   Plist.obj
 0001:0005474d       __catch$??$_Resize_reallocate@U_Value_init_tag@std@@@?$vector@PEAUHINSTANCE__@@V?$allocator@PEAUHINSTANCE__@@@std@@@std@@AEAAX_KAEBU_Value_init_tag@1@@Z$0 000000018005574d f   Plist.obj
 0001:00054770       ?dtor$0@?0???0?$vector@UProcessPerfData@@V?$allocator@UProcessPerfData@@@std@@@std@@QEAA@AEBV01@@Z@4HA 0000000180055770 f   Plist.obj
 0001:00054780       ?dtor$1@?0???0?$vector@UProcessPerfData@@V?$allocator@UProcessPerfData@@@std@@@std@@QEAA@AEBV01@@Z@4HA 0000000180055780 f   Plist.obj
 0001:00054790       ?dtor$2@?0???0?$vector@UProcessPerfData@@V?$allocator@UProcessPerfData@@@std@@@std@@QEAA@AEBV01@@Z@4HA 0000000180055790 f   Plist.obj
 0001:000547b0       ?dtor$3@?0???0?$vector@UProcessPerfData@@V?$allocator@UProcessPerfData@@@std@@@std@@QEAA@AEBV01@@Z@4HA 00000001800557b0 f   Plist.obj
 0001:000547d0       ?dtor$4@?0???0?$vector@UProcessPerfData@@V?$allocator@UProcessPerfData@@@std@@@std@@QEAA@AEBV01@@Z@4HA 00000001800557d0 f   Plist.obj
 0001:000547f0       ?dtor$0@?0??GetList@@YA_NAEAPEAUPluginPanelItem@@AEA_KAEAVPerfThread@@@Z@4HA 00000001800557f0 f   Plist.obj
 0001:00054800       ?dtor$0@?0??KillProcess@@YA_NKPEAUHWND__@@@Z@4HA 0000000180055800 f   Plist.obj
 0001:00054810       ?dtor$1@?0??KillProcess@@YA_NKPEAUHWND__@@@Z@4HA 0000000180055810 f   Plist.obj
 0001:00054820       ?dtor$0@?0??PrintModules@@YAXPEAXKAEAUoptions@@@Z@4HA 0000000180055820 f   Plist.obj
 0001:00054830       ?dtor$1@?0??PrintModules@@YAXPEAXKAEAUoptions@@@Z@4HA 0000000180055830 f   Plist.obj
 0001:00054840       ?dtor$2@?0??PrintModules@@YAXPEAXKAEAUoptions@@@Z@4HA 0000000180055840 f   Plist.obj
 0001:00054850       ?dtor$3@?0??PrintModules@@YAXPEAXKAEAUoptions@@@Z@4HA 0000000180055850 f   Plist.obj
 0001:00054850       ?dtor$8@?0??PrintModules@@YAXPEAXKAEAUoptions@@@Z@4HA 0000000180055850 f   Plist.obj
 0001:00054860       ?dtor$2@?0??print_module_impl@@YAXQEAXAEBV?$basic_string@_WU?$char_traits@_W@std@@V?$allocator@_W@2@@std@@KAEBUoptions@@AEBV?$function@$$A6A_NPEA_W_K@Z@2@@Z@4HA 0000000180055860 f   Plist.obj
 0001:00054870       ?dtor$0@?0??WinError@@YAHPEB_W@Z@4HA 0000000180055870 f   Pmix.obj
 0001:00054880       ?dtor$0@?0???0WMIConnection@@QEAA@XZ@4HA 0000000180055880 f   WMI.obj
 0001:00054890       ?dtor$0@?0??Connect@WMIConnection@@QEAA_NPEB_W00@Z@4HA 0000000180055890 f   WMI.obj
 0001:000548a0       ?dtor$3@?0??Connect@WMIConnection@@QEAA_NPEB_W00@Z@4HA 00000001800558a0 f   WMI.obj
 0001:000548b0       ?dtor$4@?0??Connect@WMIConnection@@QEAA_NPEB_W00@Z@4HA 00000001800558b0 f   WMI.obj
 0001:000548b0       ?dtor$9@?0??ExecMethod@WMIConnection@@AEAAHKPEB_W0K@Z@4HA 00000001800558b0 f   WMI.obj
 0001:000548c0       ?dtor$5@?0??Connect@WMIConnection@@QEAA_NPEB_W00@Z@4HA 00000001800558c0 f   WMI.obj
 0001:000548d0       ?dtor$0@?0??ExecMethod@WMIConnection@@AEAAHKPEB_W0K@Z@4HA 00000001800558d0 f   WMI.obj
 0001:000548e0       ?dtor$1@?0??ExecMethod@WMIConnection@@AEAAHKPEB_W0K@Z@4HA 00000001800558e0 f   WMI.obj
 0001:000548e0       ?dtor$4@?0??ExecMethod@WMIConnection@@AEAAHKPEB_W0K@Z@4HA 00000001800558e0 f   WMI.obj
 0001:000548e0       ?dtor$6@?0??ExecMethod@WMIConnection@@AEAAHKPEB_W0K@Z@4HA 00000001800558e0 f   WMI.obj
 0001:000548f0       ?dtor$10@?0??ExecMethod@WMIConnection@@AEAAHKPEB_W0K@Z@4HA 00000001800558f0 f   WMI.obj
 0001:000548f0       ?dtor$2@?0??ExecMethod@WMIConnection@@AEAAHKPEB_W0K@Z@4HA 00000001800558f0 f   WMI.obj
 0001:00054900       ?dtor$3@?0??ExecMethod@WMIConnection@@AEAAHKPEB_W0K@Z@4HA 0000000180055900 f   WMI.obj
 0001:00054910       ?dtor$5@?0??ExecMethod@WMIConnection@@AEAAHKPEB_W0K@Z@4HA 0000000180055910 f   WMI.obj
 0001:00054920       ?dtor$7@?0??ExecMethod@WMIConnection@@AEAAHKPEB_W0K@Z@4HA 0000000180055920 f   WMI.obj
 0001:00054930       ?dtor$8@?0??ExecMethod@WMIConnection@@AEAAHKPEB_W0K@Z@4HA 0000000180055930 f   WMI.obj
 0001:00054940       ?dtor$1@?0??GetProcessCommandLine@WMIConnection@@QEAA?AV?$basic_string@_WU?$char_traits@_W@std@@V?$allocator@_W@2@@std@@K@Z@4HA 0000000180055940 f   WMI.obj
 0001:00054940       ?dtor$1@?0??GetProcessExecutablePath@WMIConnection@@QEAA?AV?$basic_string@_WU?$char_traits@_W@std@@V?$allocator@_W@2@@std@@K@Z@4HA 0000000180055940 f   WMI.obj
 0001:00054970       ?dtor$2@?0??GetProcessCommandLine@WMIConnection@@QEAA?AV?$basic_string@_WU?$char_traits@_W@std@@V?$allocator@_W@2@@std@@K@Z@4HA 0000000180055970 f   WMI.obj
 0001:00054970       ?dtor$2@?0??GetProcessExecutablePath@WMIConnection@@QEAA?AV?$basic_string@_WU?$char_traits@_W@std@@V?$allocator@_W@2@@std@@K@Z@4HA 0000000180055970 f   WMI.obj
 0001:00054980       ?dtor$0@?0??GetProcessOwner@WMIConnection@@QEAA?AV?$basic_string@_WU?$char_traits@_W@std@@V?$allocator@_W@2@@std@@KPEAV23@@Z@4HA 0000000180055980 f   WMI.obj
 0001:00054990       ?dtor$1@?0??GetProcessOwner@WMIConnection@@QEAA?AV?$basic_string@_WU?$char_traits@_W@std@@V?$allocator@_W@2@@std@@KPEAV23@@Z@4HA 0000000180055990 f   WMI.obj
 0001:00054990       ?dtor$1@?0??GetProcessUserSid@WMIConnection@@QEAA?AV?$basic_string@_WU?$char_traits@_W@std@@V?$allocator@_W@2@@std@@K@Z@4HA 0000000180055990 f   WMI.obj
 0001:000549a0       ?dtor$2@?0??GetProcessOwner@WMIConnection@@QEAA?AV?$basic_string@_WU?$char_traits@_W@std@@V?$allocator@_W@2@@std@@KPEAV23@@Z@4HA 00000001800559a0 f   WMI.obj
 0001:000549a0       ?dtor$2@?0??GetProcessUserSid@WMIConnection@@QEAA?AV?$basic_string@_WU?$char_traits@_W@std@@V?$allocator@_W@2@@std@@K@Z@4HA 00000001800559a0 f   WMI.obj
 0001:000549b0       ?dtor$3@?0??GetProcessOwner@WMIConnection@@QEAA?AV?$basic_string@_WU?$char_traits@_W@std@@V?$allocator@_W@2@@std@@KPEAV23@@Z@4HA 00000001800559b0 f   WMI.obj
 0001:000549c0       ?dtor$5@?0??GetProcessOwner@WMIConnection@@QEAA?AV?$basic_string@_WU?$char_traits@_W@std@@V?$allocator@_W@2@@std@@KPEAV23@@Z@4HA 00000001800559c0 f   WMI.obj
 0001:000549c0       ?dtor$5@?0??GetProcessUserSid@WMIConnection@@QEAA?AV?$basic_string@_WU?$char_traits@_W@std@@V?$allocator@_W@2@@std@@K@Z@4HA 00000001800559c0 f   WMI.obj
 0001:000549d0       ?dtor$0@?0??GetProcessPriority@WMIConnection@@QEAAKK@Z@4HA 00000001800559d0 f   WMI.obj
 0001:000549d0       ?dtor$0@?0??GetProcessSessionId@WMIConnection@@QEAAKK@Z@4HA 00000001800559d0 f   WMI.obj
 0001:000549e0       ?dtor$0@?0??GetProcessProperty@WMIConnection@@AEAA_NKPEB_WAEBV?$function@$$A6AXAEBUtagVARIANT@@@Z@std@@@Z@4HA 00000001800559e0 f   WMI.obj
 0001:000549f0       ?dtor$1@?0??GetProcessProperty@WMIConnection@@AEAA_NKPEB_WAEBV?$function@$$A6AXAEBUtagVARIANT@@@Z@std@@@Z@4HA 00000001800559f0 f   WMI.obj
 0001:00054a00       ?dtor$2@?0??GetProcessProperty@WMIConnection@@AEAA_NKPEB_WAEBV?$function@$$A6AXAEBUtagVARIANT@@@Z@std@@@Z@4HA 0000000180055a00 f   WMI.obj
 0001:00054a10       ?dtor$0@?0??GetProcessUserSid@WMIConnection@@QEAA?AV?$basic_string@_WU?$char_traits@_W@std@@V?$allocator@_W@2@@std@@K@Z@4HA 0000000180055a10 f   WMI.obj
 0001:00054a20       ?dtor$3@?0??GetProcessUserSid@WMIConnection@@QEAA?AV?$basic_string@_WU?$char_traits@_W@std@@V?$allocator@_W@2@@std@@K@Z@4HA 0000000180055a20 f   WMI.obj
 0001:00054a2c       ?dtor$0@?0??_Init@locale@std@@CAPEAV_Locimp@12@_N@Z@4HA 0000000180055a2c f   libcpmt:locale0.obj
 0001:00054a38       __scrt_is_nonwritable_in_current_image$filt$0 0000000180055a38 f   LIBCMT:utility.obj
 0001:00054a50       ?fin$0@?0???_M@YAXPEAX_K1P6AX0@Z@Z@4HA 0000000180055a50 f   LIBCMT:ehvecdtr.obj
 0001:00054a7c       ?filt$0@?0??__ArrayUnwind@@YAXPEAX_K1P6AX0@Z@Z@4HA 0000000180055a7c f   LIBCMT:ehvecdtr.obj
 0001:00054adb       ?fin$0@?0??dllmain_crt_process_attach@@YAHQEAUHINSTANCE__@@QEAX@Z@4HA 0000000180055adb f   LIBCMT:dll_dllmain.obj
 0001:00054af2       ?fin$0@?0??dllmain_crt_process_detach@@YAH_N@Z@4HA 0000000180055af2 f   LIBCMT:dll_dllmain.obj
 0001:00054b0b       ?fin$1@?0??dllmain_crt_process_detach@@YAH_N@Z@4HA 0000000180055b0b f   LIBCMT:dll_dllmain.obj
 0001:00054b1f       ?filt$0@?0??dllmain_dispatch@@YAHQEAUHINSTANCE__@@KQEAX@Z@4HA 0000000180055b1f f   LIBCMT:dll_dllmain.obj
 0001:00054b55       __DestructExceptionObject$filt$0 0000000180055b55 f   libvcruntime:ehhelpers.obj
 0001:00054beb       ?filt$0@?0???$_CallSETranslator@V__FrameHandler3@@@@YAHPEAUEHExceptionRecord@@PEA_KPEAU_CONTEXT@@PEAU_xDISPATCHER_CONTEXT@@PEBU_s_FuncInfo@@K1@Z@4HA 0000000180055beb f   libvcruntime:risctrnsctrl.obj
 0001:00054c7c       ?filt$0@?0???$_CallSETranslator@V__FrameHandler4@@@@YAHPEAUEHExceptionRecord@@PEA_KPEAU_CONTEXT@@PEAU_xDISPATCHER_CONTEXT@@PEAUFuncInfo4@FH4@@K1@Z@4HA 0000000180055c7c f   libvcruntime:risctrnsctrl.obj
 0001:00054d0d       ?filt$0@?0??CxxCallCatchBlock@__FrameHandler3@@SAPEAXPEAU_EXCEPTION_RECORD@@@Z@4HA 0000000180055d0d f   libvcruntime:frame.obj
 0001:00054d32       ?fin$1@?0??CxxCallCatchBlock@__FrameHandler3@@SAPEAXPEAU_EXCEPTION_RECORD@@@Z@4HA 0000000180055d32 f   libvcruntime:frame.obj
 0001:00054daa       ?filt$0@?0??CxxCallCatchBlock@__FrameHandler4@@SAPEAXPEAU_EXCEPTION_RECORD@@@Z@4HA 0000000180055daa f   libvcruntime:frame.obj
 0001:00054dd9       ?fin$1@?0??CxxCallCatchBlock@__FrameHandler4@@SAPEAXPEAU_EXCEPTION_RECORD@@@Z@4HA 0000000180055dd9 f   libvcruntime:frame.obj
 0001:00054e5c       ?filt$0@?0??FrameUnwindToState@__FrameHandler3@@SAXPEA_KPEAU_xDISPATCHER_CONTEXT@@PEBU_s_FuncInfo@@H@Z@4HA 0000000180055e5c f   libvcruntime:frame.obj
 0001:00054e72       ?fin$1@?0??FrameUnwindToState@__FrameHandler3@@SAXPEA_KPEAU_xDISPATCHER_CONTEXT@@PEBU_s_FuncInfo@@H@Z@4HA 0000000180055e72 f   libvcruntime:frame.obj
 0001:00054e95       ?filt$0@?0??FrameUnwindToState@__FrameHandler4@@SAXPEA_KPEAU_xDISPATCHER_CONTEXT@@PEAUFuncInfo4@FH4@@H@Z@4HA 0000000180055e95 f   libvcruntime:frame.obj
 0001:00054eab       ?fin$1@?0??FrameUnwindToState@__FrameHandler4@@SAXPEA_KPEAU_xDISPATCHER_CONTEXT@@PEAUFuncInfo4@FH4@@H@Z@4HA 0000000180055eab f   libvcruntime:frame.obj
 0001:00054ece       __acrt_initialize_lowio$fin$0 0000000180055ece f   libucrt:ioinit.obj
 0001:00054ece       __acrt_lowio_ensure_fh_exists$fin$0 0000000180055ece f   libucrt:osfinfo.obj
 0001:00054ee7       ?fin$0@?0???$?RV<lambda_0ae27a3a962d80f24befdcbee591983d>@@AEAV<lambda_8d0ee55de4b1038c4002e0adecdf1839>@@V<lambda_dc504788e8f1664fe9b84e20bfb512f2>@@@?$__crt_seh_guarded_call@X@@QEAAX$$QEAV<lambda_0ae27a3a962d80f24befdcbee591983d>@@AEAV<lambda_8d0ee55de4b1038c4002e0adecdf1839>@@$$QEAV<lambda_dc504788e8f1664fe9b84e20bfb512f2>@@@Z@4HA 0000000180055ee7 f   libucrt:per_thread_data.obj
 0001:00054ee7       ?fin$0@?0???$?RV<lambda_2d41944a1d46af3157314b8a01080d33>@@AEAV<lambda_8f455de75cd7d7f24b4096f044d8b9e6>@@V<lambda_aa500f224e6afead328df44964fe2772>@@@?$__crt_seh_guarded_call@X@@QEAAX$$QEAV<lambda_2d41944a1d46af3157314b8a01080d33>@@AEAV<lambda_8f455de75cd7d7f24b4096f044d8b9e6>@@$$QEAV<lambda_aa500f224e6afead328df44964fe2772>@@@Z@4HA 0000000180055ee7 f   libucrt:per_thread_data.obj
 0001:00054ee7       ?fin$0@?0???$?RV<lambda_aa87e3671a710a21b5dc78c0bdf72e11>@@AEAV<lambda_92619d2358a28f41a33ba319515a20b9>@@V<lambda_6992ecaafeb10aed2b74cb1fae11a551>@@@?$__crt_seh_guarded_call@X@@QEAAX$$QEAV<lambda_aa87e3671a710a21b5dc78c0bdf72e11>@@AEAV<lambda_92619d2358a28f41a33ba319515a20b9>@@$$QEAV<lambda_6992ecaafeb10aed2b74cb1fae11a551>@@@Z@4HA 0000000180055ee7 f   libucrt:per_thread_data.obj
 0001:00054ee7       ?fin$0@?0???$?RV<lambda_f2e299630e499de9f9a165e60fcd3db5>@@AEAV<lambda_2ae9d31cdba2644fcbeaf08da7c24588>@@V<lambda_40d01ff24d0e7b3814fdbdcee8eab3c7>@@@?$__crt_seh_guarded_call@X@@QEAAX$$QEAV<lambda_f2e299630e499de9f9a165e60fcd3db5>@@AEAV<lambda_2ae9d31cdba2644fcbeaf08da7c24588>@@$$QEAV<lambda_40d01ff24d0e7b3814fdbdcee8eab3c7>@@@Z@4HA 0000000180055ee7 f   libucrt:per_thread_data.obj
 0001:00054ee7       ?fin$0@?0???$?RV<lambda_48fc4a32460bb0512d3b13f8499328be>@@AEAV<lambda_6c3dac0a4f3f9cefca9bb494422f9b77>@@V<lambda_0a2f2c9f9a56eb2b08bfa6ff61d331c5>@@@?$__crt_seh_guarded_call@H@@QEAAH$$QEAV<lambda_48fc4a32460bb0512d3b13f8499328be>@@AEAV<lambda_6c3dac0a4f3f9cefca9bb494422f9b77>@@$$QEAV<lambda_0a2f2c9f9a56eb2b08bfa6ff61d331c5>@@@Z@4HA 0000000180055ee7 f   libucrt:winapi_thunks.obj
 0001:00054ee7       ?fin$0@?0???$?RV<lambda_41e84717acc955b55e9d0d529e507b68>@@AEAV<lambda_b37934c380d97b75fd242ea49540127a>@@V<lambda_bb6db9f9ac473960206e0d4b942b5506>@@@?$__crt_seh_guarded_call@PEAD@@QEAAPEAD$$QEAV<lambda_41e84717acc955b55e9d0d529e507b68>@@AEAV<lambda_b37934c380d97b75fd242ea49540127a>@@$$QEAV<lambda_bb6db9f9ac473960206e0d4b942b5506>@@@Z@4HA 0000000180055ee7 f   libucrt:setlocale.obj
 0001:00054ee7       ?fin$0@?0???$?RV<lambda_1d892b297fdedeee07ed8124eeb2f2fa>@@AEAV<lambda_ffc046909424fd52df0ac47e64813305>@@V<lambda_01a7098693036236037e7cdb9bca3d73>@@@?$__crt_seh_guarded_call@X@@QEAAX$$QEAV<lambda_1d892b297fdedeee07ed8124eeb2f2fa>@@AEAV<lambda_ffc046909424fd52df0ac47e64813305>@@$$QEAV<lambda_01a7098693036236037e7cdb9bca3d73>@@@Z@4HA 0000000180055ee7 f   libucrt:wsetlocale.obj
 0001:00054ee7       ?fin$0@?0???$?RV<lambda_efdfa57d1f175319df784efa44bb7b81>@@AEAV<lambda_5f0a4c1567f8adc6734073e5d1e1b35c>@@V<lambda_2e8a7d3640ea6ccb4c2413664c2db6fd>@@@?$__crt_seh_guarded_call@X@@QEAAX$$QEAV<lambda_efdfa57d1f175319df784efa44bb7b81>@@AEAV<lambda_5f0a4c1567f8adc6734073e5d1e1b35c>@@$$QEAV<lambda_2e8a7d3640ea6ccb4c2413664c2db6fd>@@@Z@4HA 0000000180055ee7 f   libucrt:mbctype.obj
 0001:00054ee7       ?fin$0@?0???$?RV<lambda_450d765d439847d4c735a33c368b5fc0>@@AEAV<lambda_44731a7d0e6d81c3e6aa82d741081786>@@V<lambda_601a2a7da3b7a96e9554ac7215c4b07c>@@@?$__crt_seh_guarded_call@P6AXH@Z@@QEAAP6AXH@Z$$QEAV<lambda_450d765d439847d4c735a33c368b5fc0>@@AEAV<lambda_44731a7d0e6d81c3e6aa82d741081786>@@$$QEAV<lambda_601a2a7da3b7a96e9554ac7215c4b07c>@@@Z@4HA 0000000180055ee7 f   libucrt:signal.obj
 0001:00054ee7       ?fin$0@?0???$?RV<lambda_d80eeec6fff315bfe5c115232f3240e3>@@AEAV<lambda_6e4b09c48022b2350581041d5f6b0c4c>@@V<lambda_2358e3775559c9db80273638284d5e45>@@@?$__crt_seh_guarded_call@X@@QEAAX$$QEAV<lambda_d80eeec6fff315bfe5c115232f3240e3>@@AEAV<lambda_6e4b09c48022b2350581041d5f6b0c4c>@@$$QEAV<lambda_2358e3775559c9db80273638284d5e45>@@@Z@4HA 0000000180055ee7 f   libucrt:exit.obj
 0001:00054ee7       ?fin$0@?0???$?RV<lambda_638799b9deba96c50f710eeac98168cd>@@AEAV<lambda_22ebabd17bc4fa466a2aca6d8deb888d>@@V<lambda_a6f7d7db0129f75315ebf26d50c089f1>@@@?$__crt_seh_guarded_call@H@@QEAAH$$QEAV<lambda_638799b9deba96c50f710eeac98168cd>@@AEAV<lambda_22ebabd17bc4fa466a2aca6d8deb888d>@@$$QEAV<lambda_a6f7d7db0129f75315ebf26d50c089f1>@@@Z@4HA 0000000180055ee7 f   libucrt:onexit.obj
 0001:00054ee7       ?fin$0@?0???$?RV<lambda_7777bce6b2f8c936911f934f8298dc43>@@AEAV<lambda_f03950bc5685219e0bcd2087efbe011e>@@V<lambda_3883c3dff614d5e0c5f61bb1ac94921c>@@@?$__crt_seh_guarded_call@H@@QEAAH$$QEAV<lambda_7777bce6b2f8c936911f934f8298dc43>@@AEAV<lambda_f03950bc5685219e0bcd2087efbe011e>@@$$QEAV<lambda_3883c3dff614d5e0c5f61bb1ac94921c>@@@Z@4HA 0000000180055ee7 f   libucrt:onexit.obj
 0001:00054f01       ?filt$0@?0???R<lambda_6e4b09c48022b2350581041d5f6b0c4c>@@QEBA@XZ@4HA 0000000180055f01 f   libucrt:exit.obj
 0001:00054f1c       _query_new_handler$fin$0   0000000180055f1c f   libucrt:new_handler.obj
 0001:00054f32       _fcloseall$fin$0           0000000180055f32 f   libucrt:closeall.obj
 0001:00054f4b       ?fin$0@?0???$?RV<lambda_842d9ff0dc9ef11c61343bbaebe7f885>@@AEAV<lambda_c5860995281e5c4ce005b3de8f5874ee>@@V<lambda_d90129c13df834fdcbf8d2b88dafcf2d>@@@?$__crt_seh_guarded_call@X@@QEAAX$$QEAV<lambda_842d9ff0dc9ef11c61343bbaebe7f885>@@AEAV<lambda_c5860995281e5c4ce005b3de8f5874ee>@@$$QEAV<lambda_d90129c13df834fdcbf8d2b88dafcf2d>@@@Z@4HA 0000000180055f4b f   libucrt:fflush.obj
 0001:00054f66       ?fin$0@?0???$?RV<lambda_886d6c58226a84441f68b9f2b8217b83>@@AEAV<lambda_ab61a845afdef5b7c387490eaf3616ee>@@V<lambda_f7f22ab5edc0698d5f6905b0d3f44752>@@@?$__crt_seh_guarded_call@X@@QEAAX$$QEAV<lambda_886d6c58226a84441f68b9f2b8217b83>@@AEAV<lambda_ab61a845afdef5b7c387490eaf3616ee>@@$$QEAV<lambda_f7f22ab5edc0698d5f6905b0d3f44752>@@@Z@4HA 0000000180055f66 f   libucrt:fflush.obj
 0001:00054f83       _write$fin$0               0000000180055f83 f   libucrt:write.obj
 0001:00054f9a       ?fin$0@?0???$?RV<lambda_410d79af7f07d98d83a3f525b3859a53>@@AEAV<lambda_3e16ef9562a7dcce91392c22ab16ea36>@@V<lambda_38119f0e861e05405d8a144b9b982f0a>@@@?$__crt_seh_guarded_call@X@@QEAAX$$QEAV<lambda_410d79af7f07d98d83a3f525b3859a53>@@AEAV<lambda_3e16ef9562a7dcce91392c22ab16ea36>@@$$QEAV<lambda_38119f0e861e05405d8a144b9b982f0a>@@@Z@4HA 0000000180055f9a f   libucrt:wsetlocale.obj
 0001:00054fb4       ?fin$0@?0???$?RV<lambda_7f2adfce497ff2baa965cd4f576ecfd1>@@AEAV<lambda_2a444430fde8c29194d880d93eed5e8f>@@AEAV<lambda_8dff2cf36a5417162780cd64fa2883ef>@@@?$__crt_seh_guarded_call@X@@QEAAX$$QEAV<lambda_7f2adfce497ff2baa965cd4f576ecfd1>@@AEAV<lambda_2a444430fde8c29194d880d93eed5e8f>@@AEAV<lambda_8dff2cf36a5417162780cd64fa2883ef>@@@Z@4HA 0000000180055fb4 f   libucrt:wsetlocale.obj
 0001:00054fd5       ?dtor$0@?0??_wcstombs_l_helper@@YA_KPEADPEB_W_KPEAU__crt_locale_pointers@@@Z@4HA 0000000180055fd5 f   libucrt:wcstombs.obj
 0001:00054fe1       _ctrlfp$filt$0             0000000180055fe1 f   libucrt:fpctrl.obj
 0001:0005500d       raise$fin$0                000000018005600d f   libucrt:signal.obj
 0001:0005502e       ?fin$0@?0??update_thread_multibyte_data_internal@@YAPEAU__crt_multibyte_data@@QEAU__acrt_ptd@@QEAPEAU1@@Z@4HA 000000018005602e f   libucrt:mbctype.obj
 0001:00055047       __acrt_update_thread_locale_data$fin$0 0000000180056047 f   libucrt:locale_refcounting.obj
 0001:00055060       fclose$fin$0               0000000180056060 f   libucrt:fclose.obj
 0001:00055078       ?fin$0@?0???$?RV<lambda_751a882b2c74d4b022dec766aa51a29a>@@AEAV<lambda_628dfdc04ba53c8bfc02c9951375f3f5>@@V<lambda_f6c7be5f7998530c34de24c7437d6b54>@@@?$__crt_seh_guarded_call@H@@QEAAH$$QEAV<lambda_751a882b2c74d4b022dec766aa51a29a>@@AEAV<lambda_628dfdc04ba53c8bfc02c9951375f3f5>@@$$QEAV<lambda_f6c7be5f7998530c34de24c7437d6b54>@@@Z@4HA 0000000180056078 f   libucrt:close.obj
 0001:00055078       ?fin$0@?0???$?RV<lambda_a37b2b86f63e897a80ea819b0eb08c01>@@AEAV<lambda_38ce7e780aa69e748d6df282ebc68efe>@@V<lambda_99fb1378e971ab6e7edea83e3a7a83a2>@@@?$__crt_seh_guarded_call@H@@QEAAH$$QEAV<lambda_a37b2b86f63e897a80ea819b0eb08c01>@@AEAV<lambda_38ce7e780aa69e748d6df282ebc68efe>@@$$QEAV<lambda_99fb1378e971ab6e7edea83e3a7a83a2>@@@Z@4HA 0000000180056078 f   libucrt:commit.obj
 0001:000550a0       _IsNonwritableInCurrentImage$filt$0 00000001800560a0 f   LIBCMT:pesect.obj
 0001:000550c0       ??__F?m_PanelModesDataLocal@Plist@@0V?$vector@Umode@@V?$allocator@Umode@@@std@@@std@@A@@YAXXZ 00000001800560c0 f   fileio.obj
 0001:000550d0       ??__F?m_PanelModesDataRemote@Plist@@0V?$vector@Umode@@V?$allocator@Umode@@@std@@@std@@A@@YAXXZ 00000001800560d0 f   fileio.obj
 0001:000550e0       ??__FUserAccountID@?1??GetUserAccountID@@YA@XZ@YAXXZ 00000001800560e0 f   handles.obj
 0001:00055150       ??__FTitle@?1??GetOpenPanelInfo@Plist@@QEAAXPEAUOpenPanelInfo@@@Z@YAXXZ 0000000180056150 f   Pclass.obj
 0001:000551c0       ??__FhDebugToken@@YAXXZ    00000001800561c0 f   Plist.obj
 0001:000551d4       ??__Finitlocks@std@@YAXXZ  00000001800561d4 f   libcpmt:xlock.obj
 0001:000551e0       ??__F_Fac_tidy_reg@std@@YAXXZ 00000001800561e0 f   libcpmt:locale0.obj
 0001:0005523c       ??__Fclassic_locale@std@@YAXXZ 000000018005623c f   libcpmt:locale0.obj
 0001:0005527c       ??__Finit_atexit@@YAXXZ    000000018005627c f   libcpmt:iosptrs.obj
 0001:000552c4       ??__Finitlocks@std@@YAXXZ  00000001800562c4 f   libcpmt:iosptrs.obj
 0001:000552d0       $xdatasym                  00000001800562d0     chkstk.obj
 0001:000552d8       $unwind$?ItemWidth@PluginDialogBuilder@@CA_JAEBUFarDialogItem@@@Z 00000001800562d8     Pcfg.obj
 0001:000552d8       $unwind$??__FTitle@?1??GetOpenPanelInfo@Plist@@QEAAXPEAUOpenPanelInfo@@@Z@YAXXZ 00000001800562d8     Pclass.obj
 0001:000552d8       $unwind$?WmiError@Plist@@AEBAXXZ 00000001800562d8     Pclass.obj
 0001:000552d8       $unwind$?_Xlength@?$vector@PEB_WV?$allocator@PEB_W@std@@@std@@CAXXZ 00000001800562d8     Pclass.obj
 0001:000552d8       $unwind$?_Xlength@?$vector@Umode@@V?$allocator@Umode@@@std@@@std@@CAXXZ 00000001800562d8     Pclass.obj
 0001:000552d8       $unwind$?_Xlength@?$vector@V?$basic_string@_WU?$char_traits@_W@std@@V?$allocator@_W@2@@std@@V?$allocator@V?$basic_string@_WU?$char_traits@_W@std@@V?$allocator@_W@2@@std@@@2@@std@@CAXXZ 00000001800562d8     Pclass.obj
 0001:000552d8       $unwind$?_Xran@?$_String_val@U?$_Simple_types@_W@std@@@std@@SAXXZ 00000001800562d8     Pclass.obj
 0001:000552d8       $unwind$?deallocate@?$allocator@PEB_W@std@@QEAAXQEAPEB_W_K@Z 00000001800562d8     Pclass.obj
 0001:000552d8       $unwind$?deallocate@?$allocator@V?$basic_string@_WU?$char_traits@_W@std@@V?$allocator@_W@2@@std@@@std@@QEAAXQEAV?$basic_string@_WU?$char_traits@_W@std@@V?$allocator@_W@2@@2@_K@Z 00000001800562d8     Pclass.obj
 0001:000552d8       $unwind$?_Do_call@?$_Func_impl_no_alloc@V<lambda_87e110110aa5c29eaf754372c3484d5b>@@_NPEA_W_K@std@@EEAA_N$$QEAPEA_W$$QEA_K@Z 00000001800562d8     Plist.obj
 0001:000552d8       $unwind$?_Xlength@?$vector@PEAUHINSTANCE__@@V?$allocator@PEAUHINSTANCE__@@@std@@@std@@CAXXZ 00000001800562d8     Plist.obj
 0001:000552d8       $unwind$?allocate@?$allocator@PEAUHINSTANCE__@@@std@@QEAAPEAPEAUHINSTANCE__@@_K@Z 00000001800562d8     Plist.obj
 0001:000552d8       $unwind$?deallocate@?$allocator@PEAUHINSTANCE__@@@std@@QEAAXQEAPEAUHINSTANCE__@@_K@Z 00000001800562d8     Plist.obj
 0001:000552d8       $unwind$?dynamic_bind@@YAXXZ 00000001800562d8     Proclist.obj
 0001:000552d8       $unwind$?is_wow64_process@@YA_NPEAX@Z 00000001800562d8     Proclist.obj
 0001:000552d8       $unwind$CompareW           00000001800562d8     Proclist.obj
 0001:000552d8       $unwind$ConfigureW         00000001800562d8     Proclist.obj
 0001:000552d8       $unwind$DeleteFilesW       00000001800562d8     Proclist.obj
 0001:000552d8       $unwind$GetFindDataW       00000001800562d8     Proclist.obj
 0001:000552d8       $unwind$GetGlobalInfoW     00000001800562d8     Proclist.obj
 0001:000552d8       $unwind$ProcessPanelEventW 00000001800562d8     Proclist.obj
 0001:000552d8       $unwind$ProcessPanelInputW 00000001800562d8     Proclist.obj
 0001:000552d8       $unwind$?deallocate@?$allocator@_W@std@@QEAAXQEA_W_K@Z 00000001800562d8     fileio.obj
 0001:000552d8       $unwind$??$_Allocate@$0BA@U_Default_allocate_traits@std@@$0A@@std@@YAPEAX_K@Z 00000001800562d8     format.obj
 0001:000552d8       $unwind$??1?$basic_memory_buffer@D$0BPE@V?$allocator@D@std@@@v6@fmt@@UEAA@XZ 00000001800562d8     format.obj
 0001:000552d8       $unwind$??1?$basic_memory_buffer@I$0CA@V?$allocator@I@std@@@v6@fmt@@UEAA@XZ 00000001800562d8     format.obj
 0001:000552d8       $unwind$??1?$basic_memory_buffer@_W$0BPE@V?$allocator@_W@std@@@v6@fmt@@UEAA@XZ 00000001800562d8     format.obj
 0001:000552d8       $unwind$??1bigint@detail@v6@fmt@@QEAA@XZ 00000001800562d8     format.obj
 0001:000552d8       $unwind$??1locale@std@@QEAA@XZ 00000001800562d8     format.obj
 0001:000552d8       $unwind$?_Xlen@?$basic_string@DU?$char_traits@D@std@@V?$allocator@D@2@@std@@CAXXZ 00000001800562d8     format.obj
 0001:000552d8       $unwind$?_Xlen@?$basic_string@_WU?$char_traits@_W@std@@V?$allocator@_W@2@@std@@CAXXZ 00000001800562d8     format.obj
 0001:000552d8       $unwind$?allocate@?$allocator@_W@std@@QEAAPEA_W_K@Z 00000001800562d8     format.obj
 0001:000552d8       $unwind$??$get_id@_W@?$basic_format_args@V?$basic_format_context@V?$back_insert_iterator@V?$buffer@_W@detail@v6@fmt@@@std@@_W@v6@fmt@@@v6@fmt@@QEBAHV?$basic_string_view@_W@12@@Z 00000001800562d8     handles.obj
 0001:000552d8       $unwind$??__FUserAccountID@?1??GetUserAccountID@@YA@XZ@YAXXZ 00000001800562d8     handles.obj
 0001:000552d8       $unwind$?_Xlength@?$vector@EV?$allocator@E@std@@@std@@CAXXZ 00000001800562d8     perfthread.obj
 0001:000552d8       $unwind$?_Xlength@?$vector@UProcessPerfData@@V?$allocator@UProcessPerfData@@@std@@@std@@CAXXZ 00000001800562d8     perfthread.obj
 0001:000552d8       $unwind$?deallocate@?$allocator@E@std@@QEAAXQEAE_K@Z 00000001800562d8     perfthread.obj
 0001:000552d8       $unwind$__scrt_initialize_default_local_stdio_options 00000001800562d8     LIBCMT:default_local_stdio_options.obj
 0001:000552d8       $unwind$?dllmain_crt_dispatch@@YAHQEAUHINSTANCE__@@KQEAX@Z 00000001800562d8     LIBCMT:dll_dllmain.obj
 0001:000552d8       $unwind$__report_rangecheckfailure 00000001800562d8     LIBCMT:gs_report.obj
 0001:000552d8       $unwind$__GSHandlerCheck   00000001800562d8     LIBCMT:gshandler.obj
 0001:000552d8       $unwind$__scrt_acquire_startup_lock 00000001800562d8     LIBCMT:utility.obj
 0001:000552d8       $unwind$__scrt_dllmain_after_initialize_c 00000001800562d8     LIBCMT:utility.obj
 0001:000552d8       $unwind$__scrt_dllmain_before_initialize_c 00000001800562d8     LIBCMT:utility.obj
 0001:000552d8       $unwind$__scrt_dllmain_crt_thread_attach 00000001800562d8     LIBCMT:utility.obj
 0001:000552d8       $unwind$__scrt_dllmain_crt_thread_detach 00000001800562d8     LIBCMT:utility.obj
 0001:000552d8       $unwind$__scrt_dllmain_uninitialize_c 00000001800562d8     LIBCMT:utility.obj
 0001:000552d8       $unwind$__scrt_dllmain_uninitialize_critical 00000001800562d8     LIBCMT:utility.obj
 0001:000552d8       $unwind$atexit             00000001800562d8     LIBCMT:utility.obj
 0001:000552d8       $unwind$??__Einitlocks@std@@YAXXZ 00000001800562d8     libcpmt:iosptrs.obj
 0001:000552d8       $unwind$?_Atexit@@YAXP6AXXZ@Z 00000001800562d8     libcpmt:iosptrs.obj
 0001:000552d8       $unwind$??__Fclassic_locale@std@@YAXXZ 00000001800562d8     libcpmt:locale0.obj
 0001:000552d8       $unwind$?_Locinfo_dtor@_Locinfo@std@@SAXPEAV12@@Z 00000001800562d8     libcpmt:locale0.obj
 0001:000552d8       $unwind$_Deletegloballocale 00000001800562d8     libcpmt:locale0.obj
 0001:000552d8       $unwind$tidy_global        00000001800562d8     libcpmt:locale0.obj
 0001:000552d8       $unwind$__crtInitializeCriticalSectionEx 00000001800562d8     libcpmt:winapisupp.obj
 0001:000552d8       $unwind$??1_Lockit@std@@QEAA@XZ 00000001800562d8     libcpmt:xlock.obj
 0001:000552d8       $unwind$??__Einitlocks@std@@YAXXZ 00000001800562d8     libcpmt:xlock.obj
 0001:000552d8       $unwind$__current_exception 00000001800562d8     libvcruntime:ehhelpers.obj
 0001:000552d8       $unwind$__current_exception_context 00000001800562d8     libvcruntime:ehhelpers.obj
 0001:000552d8       $unwind$__std_terminate    00000001800562d8     libvcruntime:ehhelpers.obj
 0001:000552d8       $unwind$?GetCurrentState@__FrameHandler3@@SAHPEA_KPEAU_xDISPATCHER_CONTEXT@@PEBU_s_FuncInfo@@@Z 00000001800562d8     libvcruntime:ehstate.obj
 0001:000552d8       $unwind$__vcrt_initialize  00000001800562d8     libvcruntime:initialization.obj
 0001:000552d8       $unwind$__vcrt_thread_attach 00000001800562d8     libvcruntime:initialization.obj
 0001:000552d8       $unwind$__vcrt_thread_detach 00000001800562d8     libvcruntime:initialization.obj
 0001:000552d8       $unwind$__vcrt_uninitialize 00000001800562d8     libvcruntime:initialization.obj
 0001:000552d8       $unwind$__vcrt_uninitialize_critical 00000001800562d8     libvcruntime:initialization.obj
 0001:000552d8       $unwind$__vcrt_initialize_locks 00000001800562d8     libvcruntime:locks.obj
 0001:000552d8       $unwind$__vcrt_freefls     00000001800562d8     libvcruntime:per_thread_data.obj
 0001:000552d8       $unwind$__vcrt_getptd      00000001800562d8     libvcruntime:per_thread_data.obj
 0001:000552d8       $unwind$__vcrt_initialize_ptd 00000001800562d8     libvcruntime:per_thread_data.obj
 0001:000552d8       $unwind$__vcrt_uninitialize_ptd 00000001800562d8     libvcruntime:per_thread_data.obj
 0001:000552d8       $unwind$_purecall          00000001800562d8     libvcruntime:purevirt.obj
 0001:000552d8       $unwind$?FrameUnwindToEmptyState@__FrameHandler4@@SAXPEA_KPEAU_xDISPATCHER_CONTEXT@@PEAUFuncInfo4@FH4@@@Z 00000001800562d8     libvcruntime:risctrnsctrl.obj
 0001:000552d8       $unwind$_GetImageBase      00000001800562d8     libvcruntime:risctrnsctrl.obj
 0001:000552d8       $unwind$_GetThrowImageBase 00000001800562d8     libvcruntime:risctrnsctrl.obj
 0001:000552d8       $unwind$__dcrt_terminate_console_output 00000001800562d8     libucrt:initcon.obj
 0001:000552d8       $unwind$??$uninitialize_environment_internal@D@@YAXAEAPEAPEAD@Z 00000001800562d8     libucrt:environment_initialization.obj
 0001:000552d8       $unwind$??$uninitialize_environment_internal@_W@@YAXAEAPEAPEA_W@Z 00000001800562d8     libucrt:environment_initialization.obj
 0001:000552d8       $unwind$__dcrt_uninitialize_environments_nolock 00000001800562d8     libucrt:environment_initialization.obj
 0001:000552d8       $unwind$?__c32rtomb_utf8@__crt_mbstring@@YA_KPEAD_UPEAU_Mbstatet@@@Z 00000001800562d8     libucrt:c32rtomb.obj
 0001:000552d8       $unwind$__acrt_initialize_heap 00000001800562d8     libucrt:heap_handle.obj
 0001:000552d8       $unwind$_msize_base        00000001800562d8     libucrt:msize.obj
 0001:000552d8       $unwind$?initialize_multibyte@@YAHXZ 00000001800562d8     libucrt:multibyte_initializer.obj
 0001:000552d8       $unwind$__acrt_thread_attach 00000001800562d8     libucrt:initialization.obj
 0001:000552d8       $unwind$__acrt_thread_detach 00000001800562d8     libucrt:initialization.obj
 0001:000552d8       $unwind$__acrt_uninitialize 00000001800562d8     libucrt:initialization.obj
 0001:000552d8       $unwind$__acrt_uninitialize_critical 00000001800562d8     libucrt:initialization.obj
 0001:000552d8       $unwind$initialize_c       00000001800562d8     libucrt:initialization.obj
 0001:000552d8       $unwind$uninitialize_allocated_io_buffers 00000001800562d8     libucrt:initialization.obj
 0001:000552d8       $unwind$uninitialize_environment 00000001800562d8     libucrt:initialization.obj
 0001:000552d8       $unwind$_lock_locales      00000001800562d8     libucrt:locks.obj
 0001:000552d8       $unwind$__acrt_initialize_ptd 00000001800562d8     libucrt:per_thread_data.obj
 0001:000552d8       $unwind$__acrt_uninitialize_ptd 00000001800562d8     libucrt:per_thread_data.obj
 0001:000552d8       $unwind$__acrt_AreFileApisANSI 00000001800562d8     libucrt:winapi_thunks.obj
 0001:000552d8       $unwind$__acrt_can_use_vista_locale_apis 00000001800562d8     libucrt:winapi_thunks.obj
 0001:000552d8       $unwind$__acrt_eagerly_load_locale_apis 00000001800562d8     libucrt:winapi_thunks.obj
 0001:000552d8       $unwind$__pctype_func      00000001800562d8     libucrt:ctype.obj
 0001:000552d8       $unwind$___lc_codepage_func 00000001800562d8     libucrt:initctype.obj
 0001:000552d8       $unwind$___lc_locale_name_func 00000001800562d8     libucrt:initctype.obj
 0001:000552d8       $unwind$___mb_cur_max_func 00000001800562d8     libucrt:initctype.obj
 0001:000552d8       $unwind$__acrt_release_locale_ref 00000001800562d8     libucrt:locale_refcounting.obj
 0001:000552d8       $unwind$localeconv         00000001800562d8     libucrt:localeconv.obj
 0001:000552d8       $unwind$_copytlocinfo_nolock 00000001800562d8     libucrt:wsetlocale.obj
 0001:000552d8       $unwind$_isatty            00000001800562d8     libucrt:isatty.obj
 0001:000552d8       $unwind$_get_osfhandle     00000001800562d8     libucrt:osfinfo.obj
 0001:000552d8       $unwind$__acrt_initialize_multibyte 00000001800562d8     libucrt:mbctype.obj
 0001:000552d8       $unwind$__acrt_update_thread_multibyte_data 00000001800562d8     libucrt:mbctype.obj
 0001:000552d8       $unwind$__doserrno         00000001800562d8     libucrt:errno.obj
 0001:000552d8       $unwind$_errno             00000001800562d8     libucrt:errno.obj
 0001:000552d8       $unwind$_invoke_watson     00000001800562d8     libucrt:invalid_parameter.obj
 0001:000552d8       $unwind$abort              00000001800562d8     libucrt:abort.obj
 0001:000552d8       $unwind$__acrt_initialize_command_line 00000001800562d8     libucrt:argv_data.obj
 0001:000552d8       $unwind$_fileno            00000001800562d8     libucrt:fileno.obj
 0001:000552d8       $unwind$?state_case_normal_tchar@?$output_processor@DV?$string_output_adapter@D@__crt_stdio_output@@V?$format_validation_base@DV?$string_output_adapter@D@__crt_stdio_output@@@2@@__crt_stdio_output@@AEAA_ND@Z 00000001800562d8     libucrt:output.obj
 0001:000552d8       $unwind$?state_case_size@?$output_processor@DV?$string_output_adapter@D@__crt_stdio_output@@V?$format_validation_base@DV?$string_output_adapter@D@__crt_stdio_output@@@2@@__crt_stdio_output@@AEAA_NXZ 00000001800562d8     libucrt:output.obj
 0001:000552d8       $unwind$_wcsicmp           00000001800562d8     libucrt:wcsicmp.obj
 0001:000552d8       $unwind$_wcsnicmp          00000001800562d8     libucrt:wcsnicmp.obj
 0001:000552d8       $unwind$_statfp            00000001800562d8     libucrt:fpctrl.obj
 0001:000552d8       $unwind$_set_errno_from_matherr 00000001800562d8     libucrt:fpexcept.obj
 0001:000552e0       $unwind$??_GPluginCheckBoxBinding@@UEAAPEAXI@Z 00000001800562e0     Pcfg.obj
 0001:000552e0       $unwind$?SaveValue@PluginCheckBoxBinding@@UEAAXPEBUFarDialogItem@@H@Z 00000001800562e0     Pcfg.obj
 0001:000552e0       $unwind$??1?$_Hash_vec@V?$allocator@V?$_List_unchecked_iterator@V?$_List_val@U?$_List_simple_types@U?$pair@$$CBKPEAUHWND__@@@std@@@std@@@std@@@std@@@std@@@std@@QEAA@XZ 00000001800562e0     Pclass.obj
 0001:000552e0       $unwind$??1?$unique_ptr@VPerfThread@@U?$default_delete@VPerfThread@@@std@@@std@@QEAA@XZ 00000001800562e0     Pclass.obj
 0001:000552e0       $unwind$??1?$unique_ptr@VWMIConnection@@U?$default_delete@VWMIConnection@@@std@@@std@@QEAA@XZ 00000001800562e0     Pclass.obj
 0001:000552e0       $unwind$??1ProcessData@@QEAA@XZ 00000001800562e0     Pclass.obj
 0001:000552e0       $unwind$??4?$unique_ptr@VPerfThread@@U?$default_delete@VPerfThread@@@std@@@std@@QEAAAEAV01@$$QEAV01@@Z 00000001800562e0     Pclass.obj
 0001:000552e0       $unwind$??_GPluginEditFieldBinding@@UEAAPEAXI@Z 00000001800562e0     Pclass.obj
 0001:000552e0       $unwind$?SaveValue@PluginEditFieldBinding@@UEAAXPEBUFarDialogItem@@H@Z 00000001800562e0     Pclass.obj
 0001:000552e0       $unwind$?_Tidy@?$vector@UFarMenuItem@@V?$allocator@UFarMenuItem@@@std@@@std@@AEAAXXZ 00000001800562e0     Pclass.obj
 0001:000552e0       $unwind$??1?$function@$$A6A_NPEA_W_K@Z@std@@QEAA@XZ 00000001800562e0     Plist.obj
 0001:000552e0       $unwind$??1?$vector@PEAUHINSTANCE__@@V?$allocator@PEAUHINSTANCE__@@@std@@@std@@QEAA@XZ 00000001800562e0     Plist.obj
 0001:000552e0       $unwind$?Enable@DebugToken@@QEAA_NXZ 00000001800562e0     Plist.obj
 0001:000552e0       $unwind$?Revert@DebugToken@@QEAA_NXZ 00000001800562e0     Plist.obj
 0001:000552e0       $unwind$ClosePanelW        00000001800562e0     Proclist.obj
 0001:000552e0       $unwind$SetStartupInfoW    00000001800562e0     Proclist.obj
 0001:000552e0       $unwind$??1?$function@$$A6AXAEBUtagVARIANT@@@Z@std@@QEAA@XZ 00000001800562e0     WMI.obj
 0001:000552e0       $unwind$?Disconnect@WMIConnection@@QEAAXXZ 00000001800562e0     WMI.obj
 0001:000552e0       $unwind$??1?$basic_string@_WU?$char_traits@_W@std@@V?$allocator@_W@2@@std@@QEAA@XZ 00000001800562e0     fileio.obj
 0001:000552e0       $unwind$??1columns@@QEAA@XZ 00000001800562e0     fileio.obj
 0001:000552e0       $unwind$?_Tidy_deallocate@?$basic_string@_WU?$char_traits@_W@std@@V?$allocator@_W@2@@std@@AEAAXXZ 00000001800562e0     fileio.obj
 0001:000552e0       $unwind$??0bad_alloc@std@@QEAA@AEBV01@@Z 00000001800562e0     format.obj
 0001:000552e0       $unwind$??0bad_array_new_length@std@@QEAA@AEBV01@@Z 00000001800562e0     format.obj
 0001:000552e0       $unwind$??0bad_cast@std@@QEAA@AEBV01@@Z 00000001800562e0     format.obj
 0001:000552e0       $unwind$??0exception@std@@QEAA@AEBV01@@Z 00000001800562e0     format.obj
 0001:000552e0       $unwind$??0format_error@v6@fmt@@QEAA@AEBV012@@Z 00000001800562e0     format.obj
 0001:000552e0       $unwind$??0runtime_error@std@@QEAA@AEBV01@@Z 00000001800562e0     format.obj
 0001:000552e0       $unwind$??1?$_Tidy_guard@V?$numpunct@_W@std@@@std@@QEAA@XZ 00000001800562e0     format.obj
 0001:000552e0       $unwind$??1?$_Yarn@D@std@@QEAA@XZ 00000001800562e0     format.obj
 0001:000552e0       $unwind$??1?$_Yarn@_W@std@@QEAA@XZ 00000001800562e0     format.obj
 0001:000552e0       $unwind$??1?$basic_string@DU?$char_traits@D@std@@V?$allocator@D@2@@std@@QEAA@XZ 00000001800562e0     format.obj
 0001:000552e0       $unwind$??_3bigint@detail@v6@fmt@@QEAAAEAV0123@H@Z 00000001800562e0     format.obj
 0001:000552e0       $unwind$??_G_Facet_base@std@@UEAAPEAXI@Z 00000001800562e0     format.obj
 0001:000552e0       $unwind$?do_falsename@?$numpunct@_W@std@@MEBA?AV?$basic_string@_WU?$char_traits@_W@std@@V?$allocator@_W@2@@2@XZ 00000001800562e0     format.obj
 0001:000552e0       $unwind$?do_grouping@?$numpunct@_W@std@@MEBA?AV?$basic_string@DU?$char_traits@D@std@@V?$allocator@D@2@@2@XZ 00000001800562e0     format.obj
 0001:000552e0       $unwind$?do_truename@?$numpunct@_W@std@@MEBA?AV?$basic_string@_WU?$char_traits@_W@std@@V?$allocator@_W@2@@2@XZ 00000001800562e0     format.obj
 0001:000552e0       $unwind$??$parse_float_type_spec@Uerror_handler@detail@v6@fmt@@_W@detail@v6@fmt@@YA?AUfloat_specs@012@AEBU?$basic_format_specs@_W@12@$$QEAUerror_handler@012@@Z 00000001800562e0     handles.obj
 0001:000552e0       $unwind$?check_sign@?$numeric_specs_checker@V?$specs_handler@V?$basic_format_parse_context@_WUerror_handler@detail@v6@fmt@@@v6@fmt@@V?$basic_format_context@V?$back_insert_iterator@V?$buffer@_W@detail@v6@fmt@@@std@@_W@23@@detail@v6@fmt@@@detail@v6@fmt@@QEAAXXZ 00000001800562e0     handles.obj
 0001:000552e0       $unwind$??1?$vector@EV?$allocator@E@std@@@std@@QEAA@XZ 00000001800562e0     perfthread.obj
 0001:000552e0       $unwind$??1?$vector@_WV?$allocator@_W@std@@@std@@QEAA@XZ 00000001800562e0     perfthread.obj
 0001:000552e0       $unwind$??1PerfThread@@QEAA@XZ 00000001800562e0     perfthread.obj
 0001:000552e0       $unwind$?SyncReread@PerfThread@@QEAAXXZ 00000001800562e0     perfthread.obj
 0001:000552e0       $unwind$__raise_securityfailure 00000001800562e0     LIBCMT:gs_report.obj
 0001:000552e0       $unwind$??2@YAPEAX_K@Z     00000001800562e0     LIBCMT:new_scalar.obj
 0001:000552e0       $unwind$??_Gtype_info@@UEAAPEAXI@Z 00000001800562e0     LIBCMT:std_type_info_static.obj
 0001:000552e0       $unwind$__scrt_initialize_crt 00000001800562e0     LIBCMT:utility.obj
 0001:000552e0       $unwind$__scrt_initialize_onexit_tables 00000001800562e0     LIBCMT:utility.obj
 0001:000552e0       $unwind$__scrt_release_startup_lock 00000001800562e0     LIBCMT:utility.obj
 0001:000552e0       $unwind$__scrt_uninitialize_crt 00000001800562e0     LIBCMT:utility.obj
 0001:000552e0       $unwind$_onexit            00000001800562e0     LIBCMT:utility.obj
 0001:000552e0       $unwind$??__F_Fac_tidy_reg@std@@YAXXZ 00000001800562e0     libcpmt:locale0.obj
 0001:000552e0       $unwind$?_Facet_Register@std@@YAXPEAV_Facet_base@1@@Z 00000001800562e0     libcpmt:locale0.obj
 0001:000552e0       $unwind$?_Setgloballocale@locale@std@@CAXPEAX@Z 00000001800562e0     libcpmt:locale0.obj
 0001:000552e0       $unwind$?initialize_pointers@@YAHXZ 00000001800562e0     libcpmt:winapisupp.obj
 0001:000552e0       $unwind$??0_Lockit@std@@QEAA@H@Z 00000001800562e0     libcpmt:xlock.obj
 0001:000552e0       $unwind$??1_Init_locks@std@@QEAA@XZ 00000001800562e0     libcpmt:xlock.obj
 0001:000552e0       $unwind$??0bad_function_call@std@@QEAA@AEBV01@@Z 00000001800562e0     libcpmt:xthrow.obj
 0001:000552e0       $unwind$??0length_error@std@@QEAA@AEBV01@@Z 00000001800562e0     libcpmt:xthrow.obj
 0001:000552e0       $unwind$??0logic_error@std@@QEAA@AEBV01@@Z 00000001800562e0     libcpmt:xthrow.obj
 0001:000552e0       $unwind$??0out_of_range@std@@QEAA@AEBV01@@Z 00000001800562e0     libcpmt:xthrow.obj
 0001:000552e0       $unwind$_IsExceptionObjectToBeDestroyed 00000001800562e0     libvcruntime:ehhelpers.obj
 0001:000552e0       $unwind$?GetUnwindTryBlock@__FrameHandler3@@SAHPEA_KPEAU_xDISPATCHER_CONTEXT@@PEBU_s_FuncInfo@@@Z 00000001800562e0     libvcruntime:ehstate.obj
 0001:000552e0       $unwind$?StateFromIp@__FrameHandler3@@SAHPEBU_s_FuncInfo@@PEAU_xDISPATCHER_CONTEXT@@_K@Z 00000001800562e0     libvcruntime:ehstate.obj
 0001:000552e0       $unwind$??0HandlerMap4@FH4@@QEAA@PEBUTryBlockMapEntry4@1@_KH@Z 00000001800562e0     libvcruntime:frame.obj
 0001:000552e0       $unwind$??0bad_exception@std@@QEAA@AEBV01@@Z 00000001800562e0     libvcruntime:frame.obj
 0001:000552e0       $unwind$?ExFilterRethrow@@YAHPEAU_EXCEPTION_POINTERS@@PEAUEHExceptionRecord@@PEAH@Z 00000001800562e0     libvcruntime:frame.obj
 0001:000552e0       $unwind$__vcrt_uninitialize_locks 00000001800562e0     libvcruntime:locks.obj
 0001:000552e0       $unwind$__vcrt_freeptd     00000001800562e0     libvcruntime:per_thread_data.obj
 0001:000552e0       $unwind$?ExecutionInCatch@__FrameHandler3@@SA_NPEAU_xDISPATCHER_CONTEXT@@PEBU_s_FuncInfo@@@Z 00000001800562e0     libvcruntime:risctrnsctrl.obj
 0001:000552e0       $unwind$_CreateFrameInfo   00000001800562e0     libvcruntime:risctrnsctrl.obj
 0001:000552e0       $unwind$_SetImageBase      00000001800562e0     libvcruntime:risctrnsctrl.obj
 0001:000552e0       $unwind$_SetThrowImageBase 00000001800562e0     libvcruntime:risctrnsctrl.obj
 0001:000552e0       $unwind$__std_exception_destroy 00000001800562e0     libvcruntime:std_exception.obj
 0001:000552e0       $unwind$__std_type_info_destroy_list 00000001800562e0     libvcruntime:std_type_info.obj
 0001:000552e0       $unwind$__vcrt_FlsAlloc    00000001800562e0     libvcruntime:winapi_downlevel.obj
 0001:000552e0       $unwind$__vcrt_FlsFree     00000001800562e0     libvcruntime:winapi_downlevel.obj
 0001:000552e0       $unwind$__vcrt_FlsGetValue 00000001800562e0     libvcruntime:winapi_downlevel.obj
 0001:000552e0       $unwind$?__c16rtomb_utf8@__crt_mbstring@@YA_KPEAD_SPEAU_Mbstatet@@@Z 00000001800562e0     libucrt:c16rtomb.obj
 0001:000552e0       $unwind$_calloc_base       00000001800562e0     libucrt:calloc_base.obj
 0001:000552e0       $unwind$_malloc_base       00000001800562e0     libucrt:malloc_base.obj
 0001:000552e0       $unwind$_callnewh          00000001800562e0     libucrt:new_handler.obj
 0001:000552e0       $unwind$initialize_pointers 00000001800562e0     libucrt:initialization.obj
 0001:000552e0       $unwind$uninitialize_allocated_memory 00000001800562e0     libucrt:initialization.obj
 0001:000552e0       $unwind$__acrt_initialize_locks 00000001800562e0     libucrt:locks.obj
 0001:000552e0       $unwind$__acrt_uninitialize_locks 00000001800562e0     libucrt:locks.obj
 0001:000552e0       $unwind$__acrt_freeptd     00000001800562e0     libucrt:per_thread_data.obj
 0001:000552e0       $unwind$__acrt_getptd_head 00000001800562e0     libucrt:per_thread_data.obj
 0001:000552e0       $unwind$__acrt_get_process_end_policy 00000001800562e0     libucrt:win_policies.obj
 0001:000552e0       $unwind$__acrt_AppPolicyGetProcessTerminationMethodInternal 00000001800562e0     libucrt:winapi_thunks.obj
 0001:000552e0       $unwind$__acrt_FlsAlloc    00000001800562e0     libucrt:winapi_thunks.obj
 0001:000552e0       $unwind$__acrt_FlsFree     00000001800562e0     libucrt:winapi_thunks.obj
 0001:000552e0       $unwind$__acrt_FlsGetValue 00000001800562e0     libucrt:winapi_thunks.obj
 0001:000552e0       $unwind$__acrt_IsValidLocaleName 00000001800562e0     libucrt:winapi_thunks.obj
 0001:000552e0       $unwind$__acrt_uninitialize_winapi_thunks 00000001800562e0     libucrt:winapi_thunks.obj
 0001:000552e0       $unwind$__acrt_update_locale_info 00000001800562e0     libucrt:locale_update.obj
 0001:000552e0       $unwind$__acrt_update_multibyte_info 00000001800562e0     libucrt:locale_update.obj
 0001:000552e0       $unwind$__acrt_allocate_buffer_for_argv 00000001800562e0     libucrt:argv_parsing.obj
 0001:000552e0       $unwind$?exit_or_terminate_process@@YAXI@Z 00000001800562e0     libucrt:exit.obj
 0001:000552e0       $unwind$?try_cor_exit_process@@YAXI@Z 00000001800562e0     libucrt:exit.obj
 0001:000552e0       $unwind$__acrt_uninitialize_stdio 00000001800562e0     libucrt:_file.obj
 0001:000552e0       $unwind$__acrt_stdio_free_buffer_nolock 00000001800562e0     libucrt:_freebuf.obj
 0001:000552e0       $unwind$_fflush_nolock     00000001800562e0     libucrt:fflush.obj
 0001:000552e0       $unwind$?state_case_normal@?$output_processor@DV?$string_output_adapter@D@__crt_stdio_output@@V?$format_validation_base@DV?$string_output_adapter@D@__crt_stdio_output@@@2@@__crt_stdio_output@@AEAA_NXZ 00000001800562e0     libucrt:output.obj
 0001:000552e0       $unwind$?type_case_c_tchar@?$output_processor@DV?$string_output_adapter@D@__crt_stdio_output@@V?$format_validation_base@DV?$string_output_adapter@D@__crt_stdio_output@@@2@@__crt_stdio_output@@AEAA_ND@Z 00000001800562e0     libucrt:output.obj
 0001:000552e0       $unwind$?type_case_s@?$output_processor@DV?$string_output_adapter@D@__crt_stdio_output@@V?$format_validation_base@DV?$string_output_adapter@D@__crt_stdio_output@@@2@@__crt_stdio_output@@AEAA_NXZ 00000001800562e0     libucrt:output.obj
 0001:000552e0       $unwind$strcpy_s           00000001800562e0     libucrt:strcpy_s.obj
 0001:000552e0       $unwind$wcscat_s           00000001800562e0     libucrt:wcscat_s.obj
 0001:000552e0       $unwind$wcscpy_s           00000001800562e0     libucrt:wcscpy_s.obj
 0001:000552e0       $unwind$_clrfp             00000001800562e0     libucrt:fpctrl.obj
 0001:000552e0       $unwind$_set_statfp        00000001800562e0     libucrt:fpctrl.obj
 0001:000552e0       $unwind$_clearfp           00000001800562e0     libucrt:ieee.obj
 0001:000552e0       $unwind$fegetenv           00000001800562e0     libucrt:fegetenv.obj
 0001:000552e0       $unwind$feholdexcept       00000001800562e0     libucrt:feholdexcept.obj
 0001:000552e0       $unwind$fesetenv           00000001800562e0     libucrt:fesetenv.obj
 0001:000552e8       $unwind$??4columns@@QEAAAEAU0@AEBU0@@Z 00000001800562e8     Pclass.obj
 0001:000552e8       $unwind$GetPluginInfoW     00000001800562e8     Proclist.obj
 0001:000552e8       $unwind$OpenW              00000001800562e8     Proclist.obj
 0001:000552e8       $unwind$??1mode@@QEAA@XZ   00000001800562e8     fileio.obj
 0001:000552e8       $unwind$??_G?$basic_memory_buffer@D$0BPE@V?$allocator@D@std@@@v6@fmt@@UEAAPEAXI@Z 00000001800562e8     format.obj
 0001:000552e8       $unwind$??_G?$basic_memory_buffer@I$0CA@V?$allocator@I@std@@@v6@fmt@@UEAAPEAXI@Z 00000001800562e8     format.obj
 0001:000552e8       $unwind$??_G?$basic_memory_buffer@_W$0BPE@V?$allocator@_W@std@@@v6@fmt@@UEAAPEAXI@Z 00000001800562e8     format.obj
 0001:000552e8       $unwind$??_G?$numpunct@_W@std@@MEAAPEAXI@Z 00000001800562e8     format.obj
 0001:000552e8       $unwind$??_Gbad_alloc@std@@UEAAPEAXI@Z 00000001800562e8     format.obj
 0001:000552e8       $unwind$??_Gbad_array_new_length@std@@UEAAPEAXI@Z 00000001800562e8     format.obj
 0001:000552e8       $unwind$??_Gbad_cast@std@@UEAAPEAXI@Z 00000001800562e8     format.obj
 0001:000552e8       $unwind$??_Gexception@std@@UEAAPEAXI@Z 00000001800562e8     format.obj
 0001:000552e8       $unwind$??_Gformat_error@v6@fmt@@UEAAPEAXI@Z 00000001800562e8     format.obj
 0001:000552e8       $unwind$??_Gruntime_error@std@@UEAAPEAXI@Z 00000001800562e8     format.obj
 0001:000552e8       $unwind$?resize@?$buffer@D@detail@v6@fmt@@QEAAX_K@Z 00000001800562e8     format.obj
 0001:000552e8       $unwind$??1?$_Uninitialized_backout_al@V?$allocator@UProcessPerfData@@@std@@@std@@QEAA@XZ 00000001800562e8     perfthread.obj
 0001:000552e8       $unwind$??4ProcessPerfData@@QEAAAEAU0@AEBU0@@Z 00000001800562e8     perfthread.obj
 0001:000552e8       $unwind$_RTC_Initialize    00000001800562e8     LIBCMT:initsect.obj
 0001:000552e8       $unwind$_RTC_Terminate     00000001800562e8     LIBCMT:initsect.obj
 0001:000552e8       $unwind$??_G_Locimp@locale@std@@MEAAPEAXI@Z 00000001800562e8     libcpmt:locale0.obj
 0001:000552e8       $unwind$?_Locinfo_ctor@_Locinfo@std@@SAXPEAV12@PEBD@Z 00000001800562e8     libcpmt:locale0.obj
 0001:000552e8       $unwind$?_New_Locimp@_Locimp@locale@std@@CAPEAV123@_N@Z 00000001800562e8     libcpmt:locale0.obj
 0001:000552e8       $unwind$??0_Init_locks@std@@QEAA@XZ 00000001800562e8     libcpmt:xlock.obj
 0001:000552e8       $unwind$??_Gbad_function_call@std@@UEAAPEAXI@Z 00000001800562e8     libcpmt:xthrow.obj
 0001:000552e8       $unwind$??_Glength_error@std@@UEAAPEAXI@Z 00000001800562e8     libcpmt:xthrow.obj
 0001:000552e8       $unwind$??_Glogic_error@std@@UEAAPEAXI@Z 00000001800562e8     libcpmt:xthrow.obj
 0001:000552e8       $unwind$??_Gout_of_range@std@@UEAAPEAXI@Z 00000001800562e8     libcpmt:xthrow.obj
 0001:000552e8       $unwind$_Getcvt            00000001800562e8     libcpmt:xwctomb.obj
 0001:000552e8       $unwind$__FrameUnwindFilter 00000001800562e8     libvcruntime:ehhelpers.obj
 0001:000552e8       $unwind$?SetUnwindTryBlock@__FrameHandler3@@SAXPEA_KPEAU_xDISPATCHER_CONTEXT@@PEBU_s_FuncInfo@@H@Z 00000001800562e8     libvcruntime:ehstate.obj
 0001:000552e8       $unwind$??_Gbad_exception@std@@UEAAPEAXI@Z 00000001800562e8     libvcruntime:frame.obj
 0001:000552e8       $unwind$?ExFilterRethrowFH4@@YAHPEAU_EXCEPTION_POINTERS@@PEAUEHExceptionRecord@@HPEAH@Z 00000001800562e8     libvcruntime:frame.obj
 0001:000552e8       $unwind$_FindAndUnlinkFrame 00000001800562e8     libvcruntime:risctrnsctrl.obj
 0001:000552e8       $unwind$__vcrt_FlsSetValue 00000001800562e8     libvcruntime:winapi_downlevel.obj
 0001:000552e8       $unwind$??$common_initialize_environment_nolock@D@@YAHXZ 00000001800562e8     libucrt:environment_initialization.obj
 0001:000552e8       $unwind$__acrt_fp_strflt_to_string 00000001800562e8     libucrt:_fptostr.obj
 0001:000552e8       $unwind$_realloc_base      00000001800562e8     libucrt:realloc_base.obj
 0001:000552e8       $unwind$?replace_current_thread_locale_nolock@@YAXQEAU__acrt_ptd@@QEAU__crt_locale_data@@@Z 00000001800562e8     libucrt:per_thread_data.obj
 0001:000552e8       $unwind$__acrt_execute_uninitializers 00000001800562e8     libucrt:shared_initialization.obj
 0001:000552e8       $unwind$__acrt_FlsSetValue 00000001800562e8     libucrt:winapi_thunks.obj
 0001:000552e8       $unwind$__acrt_GetUserDefaultLocaleName 00000001800562e8     libucrt:winapi_thunks.obj
 0001:000552e8       $unwind$__acrt_LocaleNameToLCID 00000001800562e8     libucrt:winapi_thunks.obj
 0001:000552e8       $unwind$GetLocaleNameFromLangCountry 00000001800562e8     libucrt:get_qualified_locale.obj
 0001:000552e8       $unwind$GetLocaleNameFromLanguage 00000001800562e8     libucrt:get_qualified_locale.obj
 0001:000552e8       $unwind$GetLcidFromLangCountry 00000001800562e8     libucrt:getqloc_downlevel.obj
 0001:000552e8       $unwind$GetLcidFromLanguage 00000001800562e8     libucrt:getqloc_downlevel.obj
 0001:000552e8       $unwind$_updatetlocinfoEx_nolock 00000001800562e8     libucrt:locale_refcounting.obj
 0001:000552e8       $unwind$_close_nolock      00000001800562e8     libucrt:close.obj
 0001:000552e8       $unwind$__acrt_uninitialize_lowio 00000001800562e8     libucrt:ioinit.obj
 0001:000552e8       $unwind$__acrt_errno_map_os_error 00000001800562e8     libucrt:errno.obj
 0001:000552e8       $unwind$_initterm_e        00000001800562e8     libucrt:initterm.obj
 0001:000552e8       $unwind$_fclose_nolock     00000001800562e8     libucrt:fclose.obj
 0001:000552e8       $unwind$strncpy_s          00000001800562e8     libucrt:strncpy_s.obj
 0001:000552e8       $unwind$wcsncat_s          00000001800562e8     libucrt:wcsncat_s.obj
 0001:000552e8       $unwind$wcsncpy_s          00000001800562e8     libucrt:wcsncpy_s.obj
 0001:000552e8       $unwind$wcstok             00000001800562e8     libucrt:wcstok.obj
 0001:000552f4       $unwind$??1?$vector@Umode@@V?$allocator@Umode@@@std@@@std@@QEAA@XZ 00000001800562f4     fileio.obj
 0001:00055300       $chain$0$??1?$vector@Umode@@V?$allocator@Umode@@@std@@@std@@QEAA@XZ 0000000180056300     fileio.obj
 0001:00055314       $chain$1$??1?$vector@Umode@@V?$allocator@Umode@@@std@@@std@@QEAA@XZ 0000000180056314     fileio.obj
 0001:00055328       $chain$2$??1?$vector@Umode@@V?$allocator@Umode@@@std@@@std@@QEAA@XZ 0000000180056328     fileio.obj
 0001:00055338       $chain$3$??1?$vector@Umode@@V?$allocator@Umode@@@std@@@std@@QEAA@XZ 0000000180056338     fileio.obj
 0001:00055348       $unwind$?_Do_call@?$_Func_impl_no_alloc@V<lambda_c6a5923e4ab0669d9f7c2a6c892502eb>@@_NPEA_W_K@std@@EEAA_N$$QEAPEA_W$$QEA_K@Z 0000000180056348     Plist.obj
 0001:00055348       $unwind$?SetProcessPriority@WMIConnection@@QEAAHKK@Z 0000000180056348     WMI.obj
 0001:00055348       $unwind$?TerminateProcess@WMIConnection@@QEAAHK@Z 0000000180056348     WMI.obj
 0001:00055348       $unwind$?WriteToFile@@YA_KPEAXAEBV?$basic_string_view@_WU?$char_traits@_W@std@@@std@@@Z 0000000180056348     fileio.obj
 0001:00055348       $unwind$_wtol              0000000180056348     libucrt:atox.obj
 0001:00055348       $unwind$mbstowcs_s         0000000180056348     libucrt:mbstowcs.obj
 0001:00055348       $unwind$strtol             0000000180056348     libucrt:strtox.obj
 0001:00055348       $unwind$wctomb_s           0000000180056348     libucrt:wctomb.obj
 0001:00055348       $unwind$_itow_s            0000000180056348     libucrt:xtoa.obj
 0001:00055348       $unwind$parse_bcp47_code_page 0000000180056348     libucrt:wsetlocale.obj
 0001:00055348       $unwind$_invalid_parameter_noinfo 0000000180056348     libucrt:invalid_parameter.obj
 0001:00055348       $unwind$_invalid_parameter_noinfo_noreturn 0000000180056348     libucrt:invalid_parameter.obj
 0001:00055348       $unwind$_log10_special     0000000180056348     libucrt:log_special.obj
 0001:00055350       $unwind$?WriteToFile@@YA_KPEAX_W@Z 0000000180056350     fileio.obj
 0001:00055350       $unwind$__report_gsfailure 0000000180056350     LIBCMT:gs_report.obj
 0001:00055358       $unwind$??$_Destroy_range@V?$allocator@Umode@@@std@@@std@@YAXPEAUmode@@QEAU1@AEAV?$allocator@Umode@@@0@@Z 0000000180056358     fileio.obj
 0001:00055360       $chain$0$??$_Destroy_range@V?$allocator@Umode@@@std@@@std@@YAXPEAUmode@@QEAU1@AEAV?$allocator@Umode@@@0@@Z 0000000180056360     fileio.obj
 0001:00055374       $chain$1$??$_Destroy_range@V?$allocator@Umode@@@std@@@std@@YAXPEAUmode@@QEAU1@AEAV?$allocator@Umode@@@0@@Z 0000000180056374     fileio.obj
 0001:00055384       $unwind$?CreateToken@DebugToken@@SA_NXZ 0000000180056384     Plist.obj
 0001:00055384       $unwind$?Message@@YAHIPEB_WPEAPEB_W_K2@Z 0000000180056384     Proclist.obj
 0001:00055384       $unwind$GetFilesW          0000000180056384     Proclist.obj
 0001:00055384       $unwind$??$do_throw@Vformat_error@v6@fmt@@@detail@v6@fmt@@YAXAEBVformat_error@12@@Z 0000000180056384     format.obj
 0001:00055384       $unwind$?_Throw_bad_array_new_length@std@@YAXXZ 0000000180056384     format.obj
 0001:00055384       $unwind$?_Throw_bad_cast@std@@YAXXZ 0000000180056384     format.obj
 0001:00055384       $unwind$?__scrt_throw_std_bad_alloc@@YAXXZ 0000000180056384     LIBCMT:throw_bad_alloc.obj
 0001:00055384       $unwind$?__scrt_throw_std_bad_array_new_length@@YAXXZ 0000000180056384     LIBCMT:throw_bad_alloc.obj
 0001:00055384       $unwind$?_Xbad_alloc@std@@YAXXZ 0000000180056384     libcpmt:xthrow.obj
 0001:00055384       $unwind$?_Xbad_function_call@std@@YAXXZ 0000000180056384     libcpmt:xthrow.obj
 0001:00055384       $unwind$?_Xlength_error@std@@YAXPEBD@Z 0000000180056384     libcpmt:xthrow.obj
 0001:00055384       $unwind$?_Xout_of_range@std@@YAXPEBD@Z 0000000180056384     libcpmt:xthrow.obj
 0001:00055384       $unwind$?_Xruntime_error@std@@YAXPEBD@Z 0000000180056384     libcpmt:xthrow.obj
 0001:00055384       $unwind$_raise_exc         0000000180056384     libucrt:fpexcept.obj
 0001:00055384       $unwind$_raise_excf        0000000180056384     libucrt:fpexcept.obj
 0001:0005538c       $unwind$?assign@?$basic_string@DU?$char_traits@D@std@@V?$allocator@D@2@@std@@QEAAAEAV12@QEBD_K@Z 000000018005638c     format.obj
 0001:000553a0       $chain$0$?assign@?$basic_string@DU?$char_traits@D@std@@V?$allocator@D@2@@std@@QEAAAEAV12@QEBD_K@Z 00000001800563a0     format.obj
 0001:000553b4       $chain$1$?assign@?$basic_string@DU?$char_traits@D@std@@V?$allocator@D@2@@std@@QEAAAEAV12@QEBD_K@Z 00000001800563b4     format.obj
 0001:000553b4       $chain$3$?assign@?$basic_string@DU?$char_traits@D@std@@V?$allocator@D@2@@std@@QEAAAEAV12@QEBD_K@Z 00000001800563b4     format.obj
 0001:000553c4       $chain$2$?assign@?$basic_string@DU?$char_traits@D@std@@V?$allocator@D@2@@std@@QEAAAEAV12@QEBD_K@Z 00000001800563c4     format.obj
 0001:000553d8       $unwind$?FreeFindData@Plist@@SAXPEAUPluginPanelItem@@_K@Z 00000001800563d8     Pclass.obj
 0001:000553d8       $unwind$?assign@?$basic_string@_WU?$char_traits@_W@std@@V?$allocator@_W@2@@std@@QEAAAEAV12@QEB_W_K@Z 00000001800563d8     format.obj
 0001:000553d8       $unwind$??$write@_WV?$back_insert_iterator@V?$buffer@_W@detail@v6@fmt@@@std@@@detail@v6@fmt@@YA?AV?$back_insert_iterator@V?$buffer@_W@detail@v6@fmt@@@std@@V34@_N@Z 00000001800563d8     handles.obj
 0001:000553d8       $unwind$??$common_xtox@K_W@@YAHKQEA_W_KI_N@Z 00000001800563d8     libucrt:xtoa.obj
 0001:000553d8       $unwind$TranslateName      00000001800563d8     libucrt:getqloc_downlevel.obj
 0001:000553d8       $unwind$__acrt_DownlevelLocaleNameToLCID 00000001800563d8     libucrt:lcidtoname_downlevel.obj
 0001:000553d8       $unwind$??R<lambda_f03950bc5685219e0bcd2087efbe011e>@@QEBAHXZ 00000001800563d8     libucrt:onexit.obj
 0001:000553d8       $unwind$?type_case_integer@?$output_processor@DV?$string_output_adapter@D@__crt_stdio_output@@V?$format_validation_base@DV?$string_output_adapter@D@__crt_stdio_output@@@2@@__crt_stdio_output@@AEAA_NI_N@Z 00000001800563d8     libucrt:output.obj
 0001:000553f0       $unwind$??0runtime_error@std@@QEAA@PEBD@Z 00000001800563f0     format.obj
 0001:000553f0       $unwind$??0length_error@std@@QEAA@PEBD@Z 00000001800563f0     libcpmt:xthrow.obj
 0001:000553f0       $unwind$??0out_of_range@std@@QEAA@PEBD@Z 00000001800563f0     libcpmt:xthrow.obj
 0001:000553f0       $unwind$?__mbrtowc_utf8@__crt_mbstring@@YA_KPEA_WPEBD_KPEAU_Mbstatet@@@Z 00000001800563f0     libucrt:mbrtowc.obj
 0001:000553f0       $unwind$??$common_xtox_s@K_W@@YAHKQEA_W_KI_N@Z 00000001800563f0     libucrt:xtoa.obj
 0001:000553f8       $unwind$??1_Locinfo@std@@QEAA@XZ 00000001800563f8     format.obj
 0001:0005540c       $cppxdata$??1_Locinfo@std@@QEAA@XZ 000000018005640c     format.obj
 0001:00055411       $ip2state$??1_Locinfo@std@@QEAA@XZ 0000000180056411     format.obj
 0001:00055414       $unwind$??$_Copy_unchecked@PEBUmode@@PEAU1@@std@@YAPEAUmode@@PEBU1@0PEAU1@@Z 0000000180056414     Pclass.obj
 0001:00055414       $unwind$??1Plist@@QEAA@XZ  0000000180056414     Pclass.obj
 0001:00055414       $unwind$??$_Maklocstr@D@std@@YAPEADPEBDPEADAEBU_Cvtvec@@@Z 0000000180056414     format.obj
 0001:00055414       $unwind$??$make_unique@$$BY0A@_W$0A@@std@@YA?AV?$unique_ptr@$$BY0A@_WU?$default_delete@$$BY0A@_W@std@@@0@_K@Z 0000000180056414     handles.obj
 0001:00055414       $unwind$??$reserve@V?$buffer@_W@detail@v6@fmt@@$0A@@detail@v6@fmt@@YAPEA_WV?$back_insert_iterator@V?$buffer@_W@detail@v6@fmt@@@std@@_K@Z 0000000180056414     handles.obj
 0001:00055414       $unwind$_DllMainCRTStartup 0000000180056414     LIBCMT:dll_dllmain.obj
 0001:00055414       $unwind$??4?$_Yarn@D@std@@QEAAAEAV01@PEBD@Z 0000000180056414     libcpmt:locale0.obj
 0001:00055414       $unwind$__vcrt_getptd_noexit 0000000180056414     libvcruntime:per_thread_data.obj
 0001:00055414       $unwind$?CatchTryBlock@__FrameHandler3@@SAPEBU_s_TryBlockMapEntry@@PEBU_s_FuncInfo@@H@Z 0000000180056414     libvcruntime:risctrnsctrl.obj
 0001:00055414       $unwind$?FrameUnwindToEmptyState@__FrameHandler3@@SAXPEA_KPEAU_xDISPATCHER_CONTEXT@@PEBU_s_FuncInfo@@@Z 0000000180056414     libvcruntime:risctrnsctrl.obj
 0001:00055414       $unwind$__vcrt_InitializeCriticalSectionEx 0000000180056414     libvcruntime:winapi_downlevel.obj
 0001:00055414       $unwind$memcpy_s           0000000180056414     libucrt:cfout.obj
 0001:00055414       $unwind$memcpy_s           0000000180056414     libucrt:strtod.obj
 0001:00055414       $unwind$__acrt_getptd      0000000180056414     libucrt:per_thread_data.obj
 0001:00055414       $unwind$__acrt_getptd_noexit 0000000180056414     libucrt:per_thread_data.obj
 0001:00055414       $unwind$__acrt_execute_initializers 0000000180056414     libucrt:shared_initialization.obj
 0001:00055414       $unwind$__acrt_InitializeCriticalSectionEx 0000000180056414     libucrt:winapi_thunks.obj
 0001:00055414       $unwind$?free_crt_array_internal@@YAXQEAPEBX_K@Z 0000000180056414     libucrt:inittime.obj
 0001:00055414       $unwind$__acrt_locale_initialize_time 0000000180056414     libucrt:inittime.obj
 0001:00055414       $unwind$??$common_lseek_nolock@_J@@YA_JH_JH@Z 0000000180056414     libucrt:lseek.obj
 0001:00055414       $unwind$__acrt_stdio_flush_nolock 0000000180056414     libucrt:fflush.obj
 0001:00055414       $unwind$??0_LocaleUpdate@@QEAA@QEAU__crt_locale_pointers@@@Z 0000000180056414     libucrt:output.obj
 0001:00055414       $unwind$?type_case_n@?$output_processor@DV?$string_output_adapter@D@__crt_stdio_output@@V?$format_validation_base@DV?$string_output_adapter@D@__crt_stdio_output@@@2@@__crt_stdio_output@@AEAA_NXZ 0000000180056414     libucrt:output.obj
 0001:00055414       $unwind$_exception_enabled 0000000180056414     libucrt:libm_error.obj
 0001:00055424       $unwind$?on_error@error_handler@detail@v6@fmt@@QEAAXPEBD@Z 0000000180056424     format.obj
 0001:00055434       $cppxdata$?on_error@error_handler@detail@v6@fmt@@QEAAXPEBD@Z 0000000180056434     format.obj
 0001:0005543d       $stateUnwindMap$?on_error@error_handler@detail@v6@fmt@@QEAAXPEBD@Z 000000018005643d     format.obj
 0001:0005543d       $stateUnwindMap$??$visit_format_arg@U?$default_arg_formatter@V?$back_insert_iterator@V?$buffer@_W@detail@v6@fmt@@@std@@_W@detail@v6@fmt@@V?$basic_format_context@V?$back_insert_iterator@V?$buffer@_W@detail@v6@fmt@@@std@@_W@34@@v6@fmt@@YA?AV?$back_insert_iterator@V?$buffer@_W@detail@v6@fmt@@@std@@$$QEAU?$default_arg_formatter@V?$back_insert_iterator@V?$buffer@_W@detail@v6@fmt@@@std@@_W@detail@01@AEBV?$basic_format_arg@V?$basic_format_context@V?$back_insert_iterator@V?$buffer@_W@detail@v6@fmt@@@std@@_W@v6@fmt@@@01@@Z 000000018005643d     handles.obj
 0001:0005543d       $stateUnwindMap$?on_fill@?$specs_setter@_W@detail@v6@fmt@@QEAAXV?$basic_string_view@_W@34@@Z 000000018005643d     handles.obj
 0001:0005543d       $stateUnwindMap$?write@?$arg_formatter_base@V?$back_insert_iterator@V?$buffer@_W@detail@v6@fmt@@@std@@_WUerror_handler@detail@v6@fmt@@@detail@v6@fmt@@IEAAXPEB_W@Z 000000018005643d     handles.obj
 0001:00055444       $ip2state$?on_error@error_handler@detail@v6@fmt@@QEAAXPEBD@Z 0000000180056444     format.obj
 0001:00055448       $unwind$??$grouping_impl@_W@detail@v6@fmt@@YA?AV?$basic_string@DU?$char_traits@D@std@@V?$allocator@D@2@@std@@Vlocale_ref@012@@Z 0000000180056448     format.obj
 0001:00055458       $cppxdata$??$grouping_impl@_W@detail@v6@fmt@@YA?AV?$basic_string@DU?$char_traits@D@std@@V?$allocator@D@2@@std@@Vlocale_ref@012@@Z 0000000180056458     format.obj
 0001:00055461       $stateUnwindMap$??$decimal_point_impl@_W@detail@v6@fmt@@YA_WVlocale_ref@012@@Z 0000000180056461     format.obj
 0001:00055461       $stateUnwindMap$??$grouping_impl@_W@detail@v6@fmt@@YA?AV?$basic_string@DU?$char_traits@D@std@@V?$allocator@D@2@@std@@Vlocale_ref@012@@Z 0000000180056461     format.obj
 0001:00055461       $stateUnwindMap$??$thousands_sep_impl@_W@detail@v6@fmt@@YA_WVlocale_ref@012@@Z 0000000180056461     format.obj
 0001:00055468       $ip2state$??$grouping_impl@_W@detail@v6@fmt@@YA?AV?$basic_string@DU?$char_traits@D@std@@V?$allocator@D@2@@std@@Vlocale_ref@012@@Z 0000000180056468     format.obj
 0001:00055470       $unwind$??$decimal_point_impl@_W@detail@v6@fmt@@YA_WVlocale_ref@012@@Z 0000000180056470     format.obj
 0001:00055470       $unwind$??$thousands_sep_impl@_W@detail@v6@fmt@@YA_WVlocale_ref@012@@Z 0000000180056470     format.obj
 0001:00055480       $cppxdata$??$decimal_point_impl@_W@detail@v6@fmt@@YA_WVlocale_ref@012@@Z 0000000180056480     format.obj
 0001:00055480       $cppxdata$??$thousands_sep_impl@_W@detail@v6@fmt@@YA_WVlocale_ref@012@@Z 0000000180056480     format.obj
 0001:00055489       $ip2state$??$decimal_point_impl@_W@detail@v6@fmt@@YA_WVlocale_ref@012@@Z 0000000180056489     format.obj
 0001:00055489       $ip2state$??$thousands_sep_impl@_W@detail@v6@fmt@@YA_WVlocale_ref@012@@Z 0000000180056489     format.obj
 0001:00055490       $unwind$?AddEditField@PluginDialogBuilder@@QEAAPEAUFarDialogItem@@PEA_WHHPEB_W_N@Z 0000000180056490     Pclass.obj
 0001:00055490       $unwind$??0?$basic_string@_WU?$char_traits@_W@std@@V?$allocator@_W@2@@std@@QEAA@_K_W@Z 0000000180056490     Plist.obj
 0001:00055490       $unwind$?grow@?$basic_memory_buffer@D$0BPE@V?$allocator@D@std@@@v6@fmt@@MEAAX_K@Z 0000000180056490     format.obj
 0001:00055490       $unwind$?grow@?$basic_memory_buffer@I$0CA@V?$allocator@I@std@@@v6@fmt@@MEAAX_K@Z 0000000180056490     format.obj
 0001:00055490       $unwind$?grow@?$basic_memory_buffer@_W$0BPE@V?$allocator@_W@std@@@v6@fmt@@MEAAX_K@Z 0000000180056490     format.obj
 0001:00055490       $unwind$??$write@_WV?$back_insert_iterator@V?$buffer@_W@detail@v6@fmt@@@std@@@detail@v6@fmt@@YA?AV?$back_insert_iterator@V?$buffer@_W@detail@v6@fmt@@@std@@V34@_W@Z 0000000180056490     handles.obj
 0001:00055490       $unwind$?on_text@?$format_handler@V?$arg_formatter@V?$back_insert_iterator@V?$buffer@_W@detail@v6@fmt@@@std@@_W@detail@v6@fmt@@_WV?$basic_format_context@V?$back_insert_iterator@V?$buffer@_W@detail@v6@fmt@@@std@@_W@34@@detail@v6@fmt@@QEAAXPEB_W0@Z 0000000180056490     handles.obj
 0001:000554a8       $unwind$??$format_float@N@detail@v6@fmt@@YAHNHUfloat_specs@012@AEAV?$buffer@D@012@@Z 00000001800564a8     format.obj
 0001:000554a8       $unwind$??$format_float@O@detail@v6@fmt@@YAHOHUfloat_specs@012@AEAV?$buffer@D@012@@Z 00000001800564a8     format.obj
 0001:000554c0       $chain$1$??$format_float@N@detail@v6@fmt@@YAHNHUfloat_specs@012@AEAV?$buffer@D@012@@Z 00000001800564c0     format.obj
 0001:000554d8       $chain$2$??$format_float@N@detail@v6@fmt@@YAHNHUfloat_specs@012@AEAV?$buffer@D@012@@Z 00000001800564d8     format.obj
 0001:000554e8       $chain$1$??$format_float@O@detail@v6@fmt@@YAHOHUfloat_specs@012@AEAV?$buffer@D@012@@Z 00000001800564e8     format.obj
 0001:00055500       $chain$2$??$format_float@O@detail@v6@fmt@@YAHOHUfloat_specs@012@AEAV?$buffer@D@012@@Z 0000000180056500     format.obj
 0001:00055510       $unwind$??$snprintf_float@N@detail@v6@fmt@@YAHNHUfloat_specs@012@AEAV?$buffer@D@012@@Z 0000000180056510     format.obj
 0001:00055510       $unwind$??$snprintf_float@O@detail@v6@fmt@@YAHOHUfloat_specs@012@AEAV?$buffer@D@012@@Z 0000000180056510     format.obj
 0001:00055530       $unwind$?fmt_snprintf@detail@v6@fmt@@YAHPEAD_KPEBDZZ 0000000180056530     format.obj
 0001:00055540       $chain$1$??_3bigint@detail@v6@fmt@@QEAAAEAV0123@H@Z 0000000180056540     format.obj
 0001:00055558       $chain$2$??_3bigint@detail@v6@fmt@@QEAAAEAV0123@H@Z 0000000180056558     format.obj
 0001:00055568       $unwind$?assign_pow10@bigint@detail@v6@fmt@@QEAAXH@Z 0000000180056568     format.obj
 0001:00055578       $chain$1$?assign_pow10@bigint@detail@v6@fmt@@QEAAXH@Z 0000000180056578     format.obj
 0001:0005558c       $chain$2$?assign_pow10@bigint@detail@v6@fmt@@QEAAXH@Z 000000018005658c     format.obj
 0001:0005559c       $unwind$?square@bigint@detail@v6@fmt@@QEAAXXZ 000000018005659c     format.obj
 0001:000555c4       $cppxdata$?square@bigint@detail@v6@fmt@@QEAAXXZ 00000001800565c4     format.obj
 0001:000555cd       $stateUnwindMap$?square@bigint@detail@v6@fmt@@QEAAXXZ 00000001800565cd     format.obj
 0001:000555d9       $ip2state$?square@bigint@detail@v6@fmt@@QEAAXXZ 00000001800565d9     format.obj
 0001:000555e4       $unwind$??$get@Vlocale@std@@@locale_ref@detail@v6@fmt@@QEBA?AVlocale@std@@XZ 00000001800565e4     format.obj
 0001:00055600       $cppxdata$??$get@Vlocale@std@@@locale_ref@detail@v6@fmt@@QEBA?AVlocale@std@@XZ 0000000180056600     format.obj
 0001:00055609       $stateUnwindMap$??1?$ptr_setter@V?$unique_ptr@UIWbemClassObject@@Ucom_closer@@@std@@@@QEAA@XZ 0000000180056609     WMI.obj
 0001:00055609       $stateUnwindMap$??1WMIConnection@@QEAA@XZ 0000000180056609     WMI.obj
 0001:00055609       $stateUnwindMap$??$get@Vlocale@std@@@locale_ref@detail@v6@fmt@@QEBA?AVlocale@std@@XZ 0000000180056609     format.obj
 0001:0005560f       $ip2state$??$get@Vlocale@std@@@locale_ref@detail@v6@fmt@@QEBA?AVlocale@std@@XZ 000000018005660f     format.obj
 0001:00055614       $unwind$??$use_facet@V?$numpunct@_W@std@@@std@@YAAEBV?$numpunct@_W@0@AEBVlocale@0@@Z 0000000180056614     format.obj
 0001:0005562c       $cppxdata$??$use_facet@V?$numpunct@_W@std@@@std@@YAAEBV?$numpunct@_W@0@AEBVlocale@0@@Z 000000018005662c     format.obj
 0001:00055635       $stateUnwindMap$??$use_facet@V?$numpunct@_W@std@@@std@@YAAEBV?$numpunct@_W@0@AEBVlocale@0@@Z 0000000180056635     format.obj
 0001:00055642       $ip2state$??$use_facet@V?$numpunct@_W@std@@@std@@YAAEBV?$numpunct@_W@0@AEBVlocale@0@@Z 0000000180056642     format.obj
 0001:0005564c       $unwind$?_Getcat@?$numpunct@_W@std@@SA_KPEAPEBVfacet@locale@2@PEBV42@@Z 000000018005664c     format.obj
 0001:0005566c       $cppxdata$?_Getcat@?$numpunct@_W@std@@SA_KPEAPEBVfacet@locale@2@PEBV42@@Z 000000018005666c     format.obj
 0001:00055675       $stateUnwindMap$?_Getcat@?$numpunct@_W@std@@SA_KPEAPEBVfacet@locale@2@PEBV42@@Z 0000000180056675     format.obj
 0001:000556b8       $ip2state$?_Getcat@?$numpunct@_W@std@@SA_KPEAPEBVfacet@locale@2@PEBV42@@Z 00000001800566b8     format.obj
 0001:000556c8       $unwind$?dtor$181@?0??InitializePanelModes@Plist@@SAXXZ@4HA 00000001800566c8     Pclass.obj
 0001:000556c8       $unwind$?dtor$1@?0??ConnectWMI@Plist@@AEAA_NXZ@4HA 00000001800566c8     Pclass.obj
 0001:000556c8       $unwind$?dtor$25@?0??ProcessKey@Plist@@QEAAHPEBU_INPUT_RECORD@@@Z@4HA 00000001800566c8     Pclass.obj
 0001:000556c8       $unwind$?dtor$28@?0??ProcessKey@Plist@@QEAAHPEBU_INPUT_RECORD@@@Z@4HA 00000001800566c8     Pclass.obj
 0001:000556c8       $unwind$?dtor$3@?0??Connect@Plist@@QEAA_NPEB_W00@Z@4HA 00000001800566c8     Pclass.obj
 0001:000556c8       $unwind$?dtor$7@?0???0Plist@@QEAA@XZ@4HA 00000001800566c8     Pclass.obj
 0001:000556c8       $unwind$?dtor$90@?0??InitializePanelModes@Plist@@SAXXZ@4HA 00000001800566c8     Pclass.obj
 0001:000556c8       $unwind$?dtor$1@?0??GetProcessCommandLine@WMIConnection@@QEAA?AV?$basic_string@_WU?$char_traits@_W@std@@V?$allocator@_W@2@@std@@K@Z@4HA 00000001800566c8     WMI.obj
 0001:000556c8       $unwind$?dtor$1@?0??GetProcessExecutablePath@WMIConnection@@QEAA?AV?$basic_string@_WU?$char_traits@_W@std@@V?$allocator@_W@2@@std@@K@Z@4HA 00000001800566c8     WMI.obj
 0001:000556c8       $unwind$?dtor$0@?0??_Getcat@?$numpunct@_W@std@@SA_KPEAPEBVfacet@locale@2@PEBV42@@Z@4HA 00000001800566c8     format.obj
 0001:000556c8       $unwind$?dtor$1@?0??_Getcat@?$numpunct@_W@std@@SA_KPEAPEBVfacet@locale@2@PEBV42@@Z@4HA 00000001800566c8     format.obj
 0001:000556c8       $unwind$?fin$0@?0??dllmain_crt_process_attach@@YAHQEAUHINSTANCE__@@QEAX@Z@4HA 00000001800566c8     LIBCMT:dll_dllmain.obj
 0001:000556c8       $unwind$?fin$0@?0??dllmain_crt_process_detach@@YAH_N@Z@4HA 00000001800566c8     LIBCMT:dll_dllmain.obj
 0001:000556c8       $unwind$?fin$1@?0??dllmain_crt_process_detach@@YAH_N@Z@4HA 00000001800566c8     LIBCMT:dll_dllmain.obj
 0001:000556c8       $unwind$?fin$0@?0???_M@YAXPEAX_K1P6AX0@Z@Z@4HA 00000001800566c8     LIBCMT:ehvecdtr.obj
 0001:000556c8       $unwind$_IsNonwritableInCurrentImage$filt$0 00000001800566c8     LIBCMT:pesect.obj
 0001:000556c8       $unwind$?filt$0@?0??CxxCallCatchBlock@__FrameHandler3@@SAPEAXPEAU_EXCEPTION_RECORD@@@Z@4HA 00000001800566c8     libvcruntime:frame.obj
 0001:000556c8       $unwind$?filt$0@?0??CxxCallCatchBlock@__FrameHandler4@@SAPEAXPEAU_EXCEPTION_RECORD@@@Z@4HA 00000001800566c8     libvcruntime:frame.obj
 0001:000556c8       $unwind$?filt$0@?0??FrameUnwindToState@__FrameHandler3@@SAXPEA_KPEAU_xDISPATCHER_CONTEXT@@PEBU_s_FuncInfo@@H@Z@4HA 00000001800566c8     libvcruntime:frame.obj
 0001:000556c8       $unwind$?fin$1@?0??FrameUnwindToState@__FrameHandler3@@SAXPEA_KPEAU_xDISPATCHER_CONTEXT@@PEBU_s_FuncInfo@@H@Z@4HA 00000001800566c8     libvcruntime:frame.obj
 0001:000556c8       $unwind$_query_new_handler$fin$0 00000001800566c8     libucrt:new_handler.obj
 0001:000556c8       $unwind$?fin$0@?0???$?RV<lambda_0ae27a3a962d80f24befdcbee591983d>@@AEAV<lambda_8d0ee55de4b1038c4002e0adecdf1839>@@V<lambda_dc504788e8f1664fe9b84e20bfb512f2>@@@?$__crt_seh_guarded_call@X@@QEAAX$$QEAV<lambda_0ae27a3a962d80f24befdcbee591983d>@@AEAV<lambda_8d0ee55de4b1038c4002e0adecdf1839>@@$$QEAV<lambda_dc504788e8f1664fe9b84e20bfb512f2>@@@Z@4HA 00000001800566c8     libucrt:per_thread_data.obj
 0001:000556c8       $unwind$?fin$0@?0???$?RV<lambda_2d41944a1d46af3157314b8a01080d33>@@AEAV<lambda_8f455de75cd7d7f24b4096f044d8b9e6>@@V<lambda_aa500f224e6afead328df44964fe2772>@@@?$__crt_seh_guarded_call@X@@QEAAX$$QEAV<lambda_2d41944a1d46af3157314b8a01080d33>@@AEAV<lambda_8f455de75cd7d7f24b4096f044d8b9e6>@@$$QEAV<lambda_aa500f224e6afead328df44964fe2772>@@@Z@4HA 00000001800566c8     libucrt:per_thread_data.obj
 0001:000556c8       $unwind$?fin$0@?0???$?RV<lambda_aa87e3671a710a21b5dc78c0bdf72e11>@@AEAV<lambda_92619d2358a28f41a33ba319515a20b9>@@V<lambda_6992ecaafeb10aed2b74cb1fae11a551>@@@?$__crt_seh_guarded_call@X@@QEAAX$$QEAV<lambda_aa87e3671a710a21b5dc78c0bdf72e11>@@AEAV<lambda_92619d2358a28f41a33ba319515a20b9>@@$$QEAV<lambda_6992ecaafeb10aed2b74cb1fae11a551>@@@Z@4HA 00000001800566c8     libucrt:per_thread_data.obj
 0001:000556c8       $unwind$?fin$0@?0???$?RV<lambda_f2e299630e499de9f9a165e60fcd3db5>@@AEAV<lambda_2ae9d31cdba2644fcbeaf08da7c24588>@@V<lambda_40d01ff24d0e7b3814fdbdcee8eab3c7>@@@?$__crt_seh_guarded_call@X@@QEAAX$$QEAV<lambda_f2e299630e499de9f9a165e60fcd3db5>@@AEAV<lambda_2ae9d31cdba2644fcbeaf08da7c24588>@@$$QEAV<lambda_40d01ff24d0e7b3814fdbdcee8eab3c7>@@@Z@4HA 00000001800566c8     libucrt:per_thread_data.obj
 0001:000556c8       $unwind$?fin$0@?0???$?RV<lambda_48fc4a32460bb0512d3b13f8499328be>@@AEAV<lambda_6c3dac0a4f3f9cefca9bb494422f9b77>@@V<lambda_0a2f2c9f9a56eb2b08bfa6ff61d331c5>@@@?$__crt_seh_guarded_call@H@@QEAAH$$QEAV<lambda_48fc4a32460bb0512d3b13f8499328be>@@AEAV<lambda_6c3dac0a4f3f9cefca9bb494422f9b77>@@$$QEAV<lambda_0a2f2c9f9a56eb2b08bfa6ff61d331c5>@@@Z@4HA 00000001800566c8     libucrt:winapi_thunks.obj
 0001:000556c8       $unwind$__acrt_update_thread_locale_data$fin$0 00000001800566c8     libucrt:locale_refcounting.obj
 0001:000556c8       $unwind$?fin$0@?0???$?RV<lambda_41e84717acc955b55e9d0d529e507b68>@@AEAV<lambda_b37934c380d97b75fd242ea49540127a>@@V<lambda_bb6db9f9ac473960206e0d4b942b5506>@@@?$__crt_seh_guarded_call@PEAD@@QEAAPEAD$$QEAV<lambda_41e84717acc955b55e9d0d529e507b68>@@AEAV<lambda_b37934c380d97b75fd242ea49540127a>@@$$QEAV<lambda_bb6db9f9ac473960206e0d4b942b5506>@@@Z@4HA 00000001800566c8     libucrt:setlocale.obj
 0001:000556c8       $unwind$?fin$0@?0???$?RV<lambda_1d892b297fdedeee07ed8124eeb2f2fa>@@AEAV<lambda_ffc046909424fd52df0ac47e64813305>@@V<lambda_01a7098693036236037e7cdb9bca3d73>@@@?$__crt_seh_guarded_call@X@@QEAAX$$QEAV<lambda_1d892b297fdedeee07ed8124eeb2f2fa>@@AEAV<lambda_ffc046909424fd52df0ac47e64813305>@@$$QEAV<lambda_01a7098693036236037e7cdb9bca3d73>@@@Z@4HA 00000001800566c8     libucrt:wsetlocale.obj
 0001:000556c8       $unwind$?fin$0@?0???$?RV<lambda_410d79af7f07d98d83a3f525b3859a53>@@AEAV<lambda_3e16ef9562a7dcce91392c22ab16ea36>@@V<lambda_38119f0e861e05405d8a144b9b982f0a>@@@?$__crt_seh_guarded_call@X@@QEAAX$$QEAV<lambda_410d79af7f07d98d83a3f525b3859a53>@@AEAV<lambda_3e16ef9562a7dcce91392c22ab16ea36>@@$$QEAV<lambda_38119f0e861e05405d8a144b9b982f0a>@@@Z@4HA 00000001800566c8     libucrt:wsetlocale.obj
 0001:000556c8       $unwind$?fin$0@?0???$?RV<lambda_7f2adfce497ff2baa965cd4f576ecfd1>@@AEAV<lambda_2a444430fde8c29194d880d93eed5e8f>@@AEAV<lambda_8dff2cf36a5417162780cd64fa2883ef>@@@?$__crt_seh_guarded_call@X@@QEAAX$$QEAV<lambda_7f2adfce497ff2baa965cd4f576ecfd1>@@AEAV<lambda_2a444430fde8c29194d880d93eed5e8f>@@AEAV<lambda_8dff2cf36a5417162780cd64fa2883ef>@@@Z@4HA 00000001800566c8     libucrt:wsetlocale.obj
 0001:000556c8       $unwind$?fin$0@?0???$?RV<lambda_751a882b2c74d4b022dec766aa51a29a>@@AEAV<lambda_628dfdc04ba53c8bfc02c9951375f3f5>@@V<lambda_f6c7be5f7998530c34de24c7437d6b54>@@@?$__crt_seh_guarded_call@H@@QEAAH$$QEAV<lambda_751a882b2c74d4b022dec766aa51a29a>@@AEAV<lambda_628dfdc04ba53c8bfc02c9951375f3f5>@@$$QEAV<lambda_f6c7be5f7998530c34de24c7437d6b54>@@@Z@4HA 00000001800566c8     libucrt:close.obj
 0001:000556c8       $unwind$?fin$0@?0???$?RV<lambda_a37b2b86f63e897a80ea819b0eb08c01>@@AEAV<lambda_38ce7e780aa69e748d6df282ebc68efe>@@V<lambda_99fb1378e971ab6e7edea83e3a7a83a2>@@@?$__crt_seh_guarded_call@H@@QEAAH$$QEAV<lambda_a37b2b86f63e897a80ea819b0eb08c01>@@AEAV<lambda_38ce7e780aa69e748d6df282ebc68efe>@@$$QEAV<lambda_99fb1378e971ab6e7edea83e3a7a83a2>@@@Z@4HA 00000001800566c8     libucrt:commit.obj
 0001:000556c8       $unwind$__acrt_initialize_lowio$fin$0 00000001800566c8     libucrt:ioinit.obj
 0001:000556c8       $unwind$__acrt_lowio_ensure_fh_exists$fin$0 00000001800566c8     libucrt:osfinfo.obj
 0001:000556c8       $unwind$_write$fin$0       00000001800566c8     libucrt:write.obj
 0001:000556c8       $unwind$?fin$0@?0???$?RV<lambda_efdfa57d1f175319df784efa44bb7b81>@@AEAV<lambda_5f0a4c1567f8adc6734073e5d1e1b35c>@@V<lambda_2e8a7d3640ea6ccb4c2413664c2db6fd>@@@?$__crt_seh_guarded_call@X@@QEAAX$$QEAV<lambda_efdfa57d1f175319df784efa44bb7b81>@@AEAV<lambda_5f0a4c1567f8adc6734073e5d1e1b35c>@@$$QEAV<lambda_2e8a7d3640ea6ccb4c2413664c2db6fd>@@@Z@4HA 00000001800566c8     libucrt:mbctype.obj
 0001:000556c8       $unwind$?fin$0@?0??update_thread_multibyte_data_internal@@YAPEAU__crt_multibyte_data@@QEAU__acrt_ptd@@QEAPEAU1@@Z@4HA 00000001800566c8     libucrt:mbctype.obj
 0001:000556c8       $unwind$?fin$0@?0???$?RV<lambda_450d765d439847d4c735a33c368b5fc0>@@AEAV<lambda_44731a7d0e6d81c3e6aa82d741081786>@@V<lambda_601a2a7da3b7a96e9554ac7215c4b07c>@@@?$__crt_seh_guarded_call@P6AXH@Z@@QEAAP6AXH@Z$$QEAV<lambda_450d765d439847d4c735a33c368b5fc0>@@AEAV<lambda_44731a7d0e6d81c3e6aa82d741081786>@@$$QEAV<lambda_601a2a7da3b7a96e9554ac7215c4b07c>@@@Z@4HA 00000001800566c8     libucrt:signal.obj
 0001:000556c8       $unwind$raise$fin$0        00000001800566c8     libucrt:signal.obj
 0001:000556c8       $unwind$?filt$0@?0???R<lambda_6e4b09c48022b2350581041d5f6b0c4c>@@QEBA@XZ@4HA 00000001800566c8     libucrt:exit.obj
 0001:000556c8       $unwind$?fin$0@?0???$?RV<lambda_d80eeec6fff315bfe5c115232f3240e3>@@AEAV<lambda_6e4b09c48022b2350581041d5f6b0c4c>@@V<lambda_2358e3775559c9db80273638284d5e45>@@@?$__crt_seh_guarded_call@X@@QEAAX$$QEAV<lambda_d80eeec6fff315bfe5c115232f3240e3>@@AEAV<lambda_6e4b09c48022b2350581041d5f6b0c4c>@@$$QEAV<lambda_2358e3775559c9db80273638284d5e45>@@@Z@4HA 00000001800566c8     libucrt:exit.obj
 0001:000556c8       $unwind$?fin$0@?0???$?RV<lambda_638799b9deba96c50f710eeac98168cd>@@AEAV<lambda_22ebabd17bc4fa466a2aca6d8deb888d>@@V<lambda_a6f7d7db0129f75315ebf26d50c089f1>@@@?$__crt_seh_guarded_call@H@@QEAAH$$QEAV<lambda_638799b9deba96c50f710eeac98168cd>@@AEAV<lambda_22ebabd17bc4fa466a2aca6d8deb888d>@@$$QEAV<lambda_a6f7d7db0129f75315ebf26d50c089f1>@@@Z@4HA 00000001800566c8     libucrt:onexit.obj
 0001:000556c8       $unwind$?fin$0@?0???$?RV<lambda_7777bce6b2f8c936911f934f8298dc43>@@AEAV<lambda_f03950bc5685219e0bcd2087efbe011e>@@V<lambda_3883c3dff614d5e0c5f61bb1ac94921c>@@@?$__crt_seh_guarded_call@H@@QEAAH$$QEAV<lambda_7777bce6b2f8c936911f934f8298dc43>@@AEAV<lambda_f03950bc5685219e0bcd2087efbe011e>@@$$QEAV<lambda_3883c3dff614d5e0c5f61bb1ac94921c>@@@Z@4HA 00000001800566c8     libucrt:onexit.obj
 0001:000556c8       $unwind$_fcloseall$fin$0   00000001800566c8     libucrt:closeall.obj
 0001:000556c8       $unwind$fclose$fin$0       00000001800566c8     libucrt:fclose.obj
 0001:000556c8       $unwind$?fin$0@?0???$?RV<lambda_842d9ff0dc9ef11c61343bbaebe7f885>@@AEAV<lambda_c5860995281e5c4ce005b3de8f5874ee>@@V<lambda_d90129c13df834fdcbf8d2b88dafcf2d>@@@?$__crt_seh_guarded_call@X@@QEAAX$$QEAV<lambda_842d9ff0dc9ef11c61343bbaebe7f885>@@AEAV<lambda_c5860995281e5c4ce005b3de8f5874ee>@@$$QEAV<lambda_d90129c13df834fdcbf8d2b88dafcf2d>@@@Z@4HA 00000001800566c8     libucrt:fflush.obj
 0001:000556c8       $unwind$?fin$0@?0???$?RV<lambda_886d6c58226a84441f68b9f2b8217b83>@@AEAV<lambda_ab61a845afdef5b7c387490eaf3616ee>@@V<lambda_f7f22ab5edc0698d5f6905b0d3f44752>@@@?$__crt_seh_guarded_call@X@@QEAAX$$QEAV<lambda_886d6c58226a84441f68b9f2b8217b83>@@AEAV<lambda_ab61a845afdef5b7c387490eaf3616ee>@@$$QEAV<lambda_f7f22ab5edc0698d5f6905b0d3f44752>@@@Z@4HA 00000001800566c8     libucrt:fflush.obj
 0001:000556c8       $unwind$_ctrlfp$filt$0     00000001800566c8     libucrt:fpctrl.obj
 0001:000556d0       $unwind$?_Init@?$numpunct@_W@std@@IEAAXAEBV_Locinfo@2@_N@Z 00000001800566d0     format.obj
 0001:000556f4       $cppxdata$?_Init@?$numpunct@_W@std@@IEAAXAEBV_Locinfo@2@_N@Z 00000001800566f4     format.obj
 0001:000556fd       $stateUnwindMap$?_Init@?$numpunct@_W@std@@IEAAXAEBV_Locinfo@2@_N@Z 00000001800566fd     format.obj
 0001:00055704       $ip2state$?_Init@?$numpunct@_W@std@@IEAAXAEBV_Locinfo@2@_N@Z 0000000180056704     format.obj
 0001:00055708       $unwind$??$grisu_gen_digits@Ugrisu_shortest_handler@detail@v6@fmt@@@detail@v6@fmt@@YA?AW4result@digits@012@Vfp@012@_KAEAHAEAUgrisu_shortest_handler@012@@Z 0000000180056708     format.obj
 0001:00055708       $unwind$??$write_nonfinite@_WV?$back_insert_iterator@V?$buffer@_W@detail@v6@fmt@@@std@@@detail@v6@fmt@@YA?AV?$back_insert_iterator@V?$buffer@_W@detail@v6@fmt@@@std@@V34@_NAEBU?$basic_format_specs@_W@12@AEBUfloat_specs@012@@Z 0000000180056708     handles.obj
 0001:00055708       $unwind$??$write_padded@$01V?$back_insert_iterator@V?$buffer@_W@detail@v6@fmt@@@std@@_WV<lambda_2c6139bafe179ad98da6b2e77db1d169>@@@detail@v6@fmt@@YA?AV?$back_insert_iterator@V?$buffer@_W@detail@v6@fmt@@@std@@V34@AEBU?$basic_format_specs@_W@12@_K2AEBV<lambda_2c6139bafe179ad98da6b2e77db1d169>@@@Z 0000000180056708     handles.obj
 0001:00055708       $unwind$??$write_padded@$01V?$back_insert_iterator@V?$buffer@_W@detail@v6@fmt@@@std@@_WV?$float_writer@_W@detail@v6@fmt@@@detail@v6@fmt@@YA?AV?$back_insert_iterator@V?$buffer@_W@detail@v6@fmt@@@std@@V34@AEBU?$basic_format_specs@_W@12@_KAEBV?$float_writer@_W@012@@Z 0000000180056708     handles.obj
 0001:00055708       $unwind$?try_get_function@@YAPEAXW4function_id@?A0x81a78551@@QEBDQEBW4module_id@2@2@Z 0000000180056708     libvcruntime:winapi_downlevel.obj
 0001:00055708       $unwind$?try_get_function@@YAPEAXW4function_id@?A0x391cf84c@@QEBDQEBW4module_id@2@2@Z 0000000180056708     libucrt:winapi_thunks.obj
 0001:00055724       $unwind$??$fallback_format@N@detail@v6@fmt@@YAXNAEAV?$buffer@D@012@AEAH@Z 0000000180056724     format.obj
 0001:00055724       $unwind$??$fallback_format@O@detail@v6@fmt@@YAXOAEAV?$buffer@D@012@AEAH@Z 0000000180056724     format.obj
 0001:00055744       $cppxdata$??$fallback_format@N@detail@v6@fmt@@YAXNAEAV?$buffer@D@012@AEAH@Z 0000000180056744     format.obj
 0001:00055744       $cppxdata$??$fallback_format@O@detail@v6@fmt@@YAXOAEAV?$buffer@D@012@AEAH@Z 0000000180056744     format.obj
 0001:0005574d       $stateUnwindMap$??$fallback_format@N@detail@v6@fmt@@YAXNAEAV?$buffer@D@012@AEAH@Z 000000018005674d     format.obj
 0001:0005574d       $stateUnwindMap$??$fallback_format@O@detail@v6@fmt@@YAXOAEAV?$buffer@D@012@AEAH@Z 000000018005674d     format.obj
 0001:00055769       $ip2state$??$fallback_format@N@detail@v6@fmt@@YAXNAEAV?$buffer@D@012@AEAH@Z 0000000180056769     format.obj
 0001:00055769       $ip2state$??$fallback_format@O@detail@v6@fmt@@YAXOAEAV?$buffer@D@012@AEAH@Z 0000000180056769     format.obj
 0001:00055770       $unwind$??$grisu_gen_digits@Ufixed_handler@detail@v6@fmt@@@detail@v6@fmt@@YA?AW4result@digits@012@Vfp@012@_KAEAHAEAUfixed_handler@012@@Z 0000000180056770     format.obj
 0001:00055770       $unwind$??$write@_W_WV?$back_insert_iterator@V?$buffer@_W@detail@v6@fmt@@@std@@@detail@v6@fmt@@YA?AV?$back_insert_iterator@V?$buffer@_W@detail@v6@fmt@@@std@@V34@V?$basic_string_view@_W@12@AEBU?$basic_format_specs@_W@12@@Z 0000000180056770     handles.obj
 0001:0005578c       $unwind$?OpenProcessForced@@YAPEAXPEAVDebugToken@@KKH@Z 000000018005678c     Plist.obj
 0001:0005578c       $unwind$??0?$basic_string@_WU?$char_traits@_W@std@@V?$allocator@_W@2@@std@@QEAA@AEBV01@@Z 000000018005678c     handles.obj
 0001:0005578c       $unwind$__scrt_dllmain_exception_filter 000000018005678c     LIBCMT:utility.obj
 0001:0005578c       $unwind$?GetHandlerSearchState@__FrameHandler3@@SAHPEA_KPEAU_xDISPATCHER_CONTEXT@@PEBU_s_FuncInfo@@@Z 000000018005678c     libvcruntime:frame.obj
 0001:0005578c       $unwind$?Is_bad_exception_allowed@@YAEPEBU_s_ESTypeList@@@Z 000000018005678c     libvcruntime:frame.obj
 0001:0005578c       $unwind$_ischartype_l      000000018005678c     libucrt:strtod.obj
 0001:0005578c       $unwind$_recalloc_base     000000018005678c     libucrt:recalloc.obj
 0001:0005578c       $unwind$__acrt_free_locale 000000018005678c     libucrt:locale_refcounting.obj
 0001:0005578c       $unwind$__acrt_lowio_create_handle_array 000000018005678c     libucrt:osfinfo.obj
 0001:0005578c       $unwind$?setSBCS@@YAXPEAU__crt_multibyte_data@@@Z 000000018005678c     libucrt:mbctype.obj
 0001:0005578c       $unwind$_seh_filter_exe    000000018005678c     libucrt:exception_filter.obj
 0001:0005578c       $unwind$_initterm          000000018005678c     libucrt:initterm.obj
 0001:0005578c       $unwind$??$ensure_buffer_is_big_enough@D@formatting_buffer@__crt_stdio_output@@QEAA_N_K@Z 000000018005678c     libucrt:output.obj
 0001:000557a0       $unwind$?append@?$basic_string@_WU?$char_traits@_W@std@@V?$allocator@_W@2@@std@@QEAAAEAV12@QEB_W_K@Z 00000001800567a0     handles.obj
 0001:000557a0       $unwind$?on_char@char_spec_handler@?$arg_formatter_base@V?$back_insert_iterator@V?$buffer@_W@detail@v6@fmt@@@std@@_WUerror_handler@detail@v6@fmt@@@detail@v6@fmt@@QEAAXXZ 00000001800567a0     handles.obj
 0001:000557a0       $unwind$?GetEstablisherFrame@__FrameHandler3@@SAPEA_KPEA_KPEAU_xDISPATCHER_CONTEXT@@PEBU_s_FuncInfo@@0@Z 00000001800567a0     libvcruntime:risctrnsctrl.obj
 0001:000557b8       $chain$0$?append@?$basic_string@_WU?$char_traits@_W@std@@V?$allocator@_W@2@@std@@QEAAAEAV12@QEB_W_K@Z 00000001800567b8     handles.obj
 0001:000557cc       $chain$1$?append@?$basic_string@_WU?$char_traits@_W@std@@V?$allocator@_W@2@@std@@QEAAAEAV12@QEB_W_K@Z 00000001800567cc     handles.obj
 0001:000557cc       $chain$3$?append@?$basic_string@_WU?$char_traits@_W@std@@V?$allocator@_W@2@@std@@QEAAAEAV12@QEB_W_K@Z 00000001800567cc     handles.obj
 0001:000557dc       $chain$2$?append@?$basic_string@_WU?$char_traits@_W@std@@V?$allocator@_W@2@@std@@QEAAAEAV12@QEB_W_K@Z 00000001800567dc     handles.obj
 0001:000557f0       $unwind$??1DebugToken@@QEAA@XZ 00000001800567f0     handles.obj
 0001:00055800       $cppxdata$??1DebugToken@@QEAA@XZ 0000000180056800     handles.obj
 0001:00055805       $ip2state$??1DebugToken@@QEAA@XZ 0000000180056805     handles.obj
 0001:00055808       $unwind$?PrintHandleInfo@@YA_NKPEAX_NPEAVPerfThread@@@Z 0000000180056808     handles.obj
 0001:00055828       $cppxdata$?PrintHandleInfo@@YA_NKPEAX_NPEAVPerfThread@@@Z 0000000180056828     handles.obj
 0001:00055831       $stateUnwindMap$?PrintHandleInfo@@YA_NKPEAX_NPEAVPerfThread@@@Z 0000000180056831     handles.obj
 0001:0005585f       $ip2state$?PrintHandleInfo@@YA_NKPEAX_NPEAVPerfThread@@@Z 000000018005685f     handles.obj
 0001:0005587c       $unwind$?query_object@@YA?AV?$unique_ptr@$$BY0A@DU?$default_delete@$$BY0A@D@std@@@std@@PEAXW4OBJECT_INFORMATION_CLASS@@@Z 000000018005687c     handles.obj
 0001:00055898       $cppxdata$?query_object@@YA?AV?$unique_ptr@$$BY0A@DU?$default_delete@$$BY0A@D@std@@@std@@PEAXW4OBJECT_INFORMATION_CLASS@@@Z 0000000180056898     handles.obj
 0001:000558a1       $stateUnwindMap$?query_object@@YA?AV?$unique_ptr@$$BY0A@DU?$default_delete@$$BY0A@D@std@@@std@@PEAXW4OBJECT_INFORMATION_CLASS@@@Z 00000001800568a1     handles.obj
 0001:000558a8       $ip2state$?query_object@@YA?AV?$unique_ptr@$$BY0A@DU?$default_delete@$$BY0A@D@std@@@std@@PEAXW4OBJECT_INFORMATION_CLASS@@@Z 00000001800568a8     handles.obj
 0001:000558b0       $unwind$?GetFileNameThread@test@?4??GetFileName@@YA?AV?$basic_string@_WU?$char_traits@_W@std@@V?$allocator@_W@2@@std@@PEAX@Z@SAK0@Z 00000001800568b0     handles.obj
 0001:000558b8       $unwind$??R<lambda_c3630acb37279cf92411e07a2b271fdf>@@QEBA?AV?$basic_string@_WU?$char_traits@_W@std@@V?$allocator@_W@2@@std@@XZ 00000001800568b8     handles.obj
 0001:000558dc       $cppxdata$??R<lambda_c3630acb37279cf92411e07a2b271fdf>@@QEBA?AV?$basic_string@_WU?$char_traits@_W@std@@V?$allocator@_W@2@@std@@XZ 00000001800568dc     handles.obj
 0001:000558e5       $stateUnwindMap$??R<lambda_c3630acb37279cf92411e07a2b271fdf>@@QEBA?AV?$basic_string@_WU?$char_traits@_W@std@@V?$allocator@_W@2@@std@@XZ 00000001800568e5     handles.obj
 0001:000558f8       $ip2state$??R<lambda_c3630acb37279cf92411e07a2b271fdf>@@QEBA?AV?$basic_string@_WU?$char_traits@_W@std@@V?$allocator@_W@2@@std@@XZ 00000001800568f8     handles.obj
 0001:00055900       $unwind$?GetNameByType@@YA?AV?$basic_string@_WU?$char_traits@_W@std@@V?$allocator@_W@2@@std@@PEAXGPEAVPerfThread@@@Z 0000000180056900     handles.obj
 0001:00055928       $cppxdata$?GetNameByType@@YA?AV?$basic_string@_WU?$char_traits@_W@std@@V?$allocator@_W@2@@std@@PEAXGPEAVPerfThread@@@Z 0000000180056928     handles.obj
 0001:00055931       $stateUnwindMap$?GetNameByType@@YA?AV?$basic_string@_WU?$char_traits@_W@std@@V?$allocator@_W@2@@std@@PEAXGPEAVPerfThread@@@Z 0000000180056931     handles.obj
 0001:0005595b       $ip2state$?GetNameByType@@YA?AV?$basic_string@_WU?$char_traits@_W@std@@V?$allocator@_W@2@@std@@PEAXGPEAVPerfThread@@@Z 000000018005695b     handles.obj
 0001:00055978       $unwind$?dtor$20@?0??GetNameByType@@YA?AV?$basic_string@_WU?$char_traits@_W@std@@V?$allocator@_W@2@@std@@PEAXGPEAVPerfThread@@@Z@4HA 0000000180056978     handles.obj
 0001:00055978       $unwind$__scrt_is_nonwritable_in_current_image$filt$0 0000000180056978     LIBCMT:utility.obj
 0001:00055980       $unwind$??1?$scoped_lock@VPerfThread@@@std@@QEAA@XZ 0000000180056980     handles.obj
 0001:00055990       $cppxdata$??1?$scoped_lock@VPerfThread@@@std@@QEAA@XZ 0000000180056990     handles.obj
 0001:00055995       $ip2state$??1?$scoped_lock@VPerfThread@@@std@@QEAA@XZ 0000000180056995     handles.obj
 0001:00055998       $unwind$?duplicate_handle@@YA?AV?$unique_ptr@XUhandle_closer@@@std@@PEAXK@Z 0000000180056998     handles.obj
 0001:000559b4       $cppxdata$?duplicate_handle@@YA?AV?$unique_ptr@XUhandle_closer@@@std@@PEAXK@Z 00000001800569b4     handles.obj
 0001:000559bd       $stateUnwindMap$?duplicate_handle@@YA?AV?$unique_ptr@XUhandle_closer@@@std@@PEAXK@Z 00000001800569bd     handles.obj
 0001:000559c9       $ip2state$?duplicate_handle@@YA?AV?$unique_ptr@XUhandle_closer@@@std@@PEAXK@Z 00000001800569c9     handles.obj
 0001:000559d0       $unwind$??$vformat@_W$0A@@detail@v6@fmt@@YA?AV?$basic_string@_WU?$char_traits@_W@std@@V?$allocator@_W@2@@std@@V?$basic_string_view@_W@12@V?$basic_format_args@V?$basic_format_context@V?$back_insert_iterator@V?$buffer@_W@detail@v6@fmt@@@std@@_W@v6@fmt@@@12@@Z 00000001800569d0     handles.obj
 0001:000559f0       $cppxdata$??$vformat@_W$0A@@detail@v6@fmt@@YA?AV?$basic_string@_WU?$char_traits@_W@std@@V?$allocator@_W@2@@std@@V?$basic_string_view@_W@12@V?$basic_format_args@V?$basic_format_context@V?$back_insert_iterator@V?$buffer@_W@detail@v6@fmt@@@std@@_W@v6@fmt@@@12@@Z 00000001800569f0     handles.obj
 0001:000559f9       $stateUnwindMap$??$vformat@_W$0A@@detail@v6@fmt@@YA?AV?$basic_string@_WU?$char_traits@_W@std@@V?$allocator@_W@2@@std@@V?$basic_string_view@_W@12@V?$basic_format_args@V?$basic_format_context@V?$back_insert_iterator@V?$buffer@_W@detail@v6@fmt@@@std@@_W@v6@fmt@@@12@@Z 00000001800569f9     handles.obj
 0001:00055a01       $ip2state$??$vformat@_W$0A@@detail@v6@fmt@@YA?AV?$basic_string@_WU?$char_traits@_W@std@@V?$allocator@_W@2@@std@@V?$basic_string_view@_W@12@V?$basic_format_args@V?$basic_format_context@V?$back_insert_iterator@V?$buffer@_W@detail@v6@fmt@@@std@@_W@v6@fmt@@@12@@Z 0000000180056a01     handles.obj
 0001:00055a08       $unwind$?on_fill@?$specs_setter@_W@detail@v6@fmt@@QEAAXV?$basic_string_view@_W@34@@Z 0000000180056a08     handles.obj
 0001:00055a18       $cppxdata$?on_fill@?$specs_setter@_W@detail@v6@fmt@@QEAAXV?$basic_string_view@_W@34@@Z 0000000180056a18     handles.obj
 0001:00055a21       $ip2state$?on_fill@?$specs_setter@_W@detail@v6@fmt@@QEAAXV?$basic_string_view@_W@34@@Z 0000000180056a21     handles.obj
 0001:00055a28       $unwind$?write@?$arg_formatter_base@V?$back_insert_iterator@V?$buffer@_W@detail@v6@fmt@@@std@@_WUerror_handler@detail@v6@fmt@@@detail@v6@fmt@@IEAAX_N@Z 0000000180056a28     handles.obj
 0001:00055a3c       $chain$1$?write@?$arg_formatter_base@V?$back_insert_iterator@V?$buffer@_W@detail@v6@fmt@@@std@@_WUerror_handler@detail@v6@fmt@@@detail@v6@fmt@@IEAAX_N@Z 0000000180056a3c     handles.obj
 0001:00055a54       $chain$2$?write@?$arg_formatter_base@V?$back_insert_iterator@V?$buffer@_W@detail@v6@fmt@@@std@@_WUerror_handler@detail@v6@fmt@@@detail@v6@fmt@@IEAAX_N@Z 0000000180056a54     handles.obj
 0001:00055a64       $unwind$?write@?$arg_formatter_base@V?$back_insert_iterator@V?$buffer@_W@detail@v6@fmt@@@std@@_WUerror_handler@detail@v6@fmt@@@detail@v6@fmt@@IEAAXPEB_W@Z 0000000180056a64     handles.obj
 0001:00055a80       $cppxdata$?write@?$arg_formatter_base@V?$back_insert_iterator@V?$buffer@_W@detail@v6@fmt@@@std@@_WUerror_handler@detail@v6@fmt@@@detail@v6@fmt@@IEAAXPEB_W@Z 0000000180056a80     handles.obj
 0001:00055a89       $ip2state$?write@?$arg_formatter_base@V?$back_insert_iterator@V?$buffer@_W@detail@v6@fmt@@@std@@_WUerror_handler@detail@v6@fmt@@@detail@v6@fmt@@IEAAXPEB_W@Z 0000000180056a89     handles.obj
 0001:00055a90       $unwind$??$visit_format_arg@U?$default_arg_formatter@V?$back_insert_iterator@V?$buffer@_W@detail@v6@fmt@@@std@@_W@detail@v6@fmt@@V?$basic_format_context@V?$back_insert_iterator@V?$buffer@_W@detail@v6@fmt@@@std@@_W@34@@v6@fmt@@YA?AV?$back_insert_iterator@V?$buffer@_W@detail@v6@fmt@@@std@@$$QEAU?$default_arg_formatter@V?$back_insert_iterator@V?$buffer@_W@detail@v6@fmt@@@std@@_W@detail@01@AEBV?$basic_format_arg@V?$basic_format_context@V?$back_insert_iterator@V?$buffer@_W@detail@v6@fmt@@@std@@_W@v6@fmt@@@01@@Z 0000000180056a90     handles.obj
 0001:00055ab0       $cppxdata$??$visit_format_arg@U?$default_arg_formatter@V?$back_insert_iterator@V?$buffer@_W@detail@v6@fmt@@@std@@_W@detail@v6@fmt@@V?$basic_format_context@V?$back_insert_iterator@V?$buffer@_W@detail@v6@fmt@@@std@@_W@34@@v6@fmt@@YA?AV?$back_insert_iterator@V?$buffer@_W@detail@v6@fmt@@@std@@$$QEAU?$default_arg_formatter@V?$back_insert_iterator@V?$buffer@_W@detail@v6@fmt@@@std@@_W@detail@01@AEBV?$basic_format_arg@V?$basic_format_context@V?$back_insert_iterator@V?$buffer@_W@detail@v6@fmt@@@std@@_W@v6@fmt@@@01@@Z 0000000180056ab0     handles.obj
 0001:00055ab9       $ip2state$??$visit_format_arg@U?$default_arg_formatter@V?$back_insert_iterator@V?$buffer@_W@detail@v6@fmt@@@std@@_W@detail@v6@fmt@@V?$basic_format_context@V?$back_insert_iterator@V?$buffer@_W@detail@v6@fmt@@@std@@_W@34@@v6@fmt@@YA?AV?$back_insert_iterator@V?$buffer@_W@detail@v6@fmt@@@std@@$$QEAU?$default_arg_formatter@V?$back_insert_iterator@V?$buffer@_W@detail@v6@fmt@@@std@@_W@detail@01@AEBV?$basic_format_arg@V?$basic_format_context@V?$back_insert_iterator@V?$buffer@_W@detail@v6@fmt@@@std@@_W@v6@fmt@@@01@@Z 0000000180056ab9     handles.obj
 0001:00055ac0       $unwind$?on_replacement_field@?$format_handler@V?$arg_formatter@V?$back_insert_iterator@V?$buffer@_W@detail@v6@fmt@@@std@@_W@detail@v6@fmt@@_WV?$basic_format_context@V?$back_insert_iterator@V?$buffer@_W@detail@v6@fmt@@@std@@_W@34@@detail@v6@fmt@@QEAAXHPEB_W@Z 0000000180056ac0     handles.obj
 0001:00055ac8       $unwind$?on_format_specs@?$format_handler@V?$arg_formatter@V?$back_insert_iterator@V?$buffer@_W@detail@v6@fmt@@@std@@_W@detail@v6@fmt@@_WV?$basic_format_context@V?$back_insert_iterator@V?$buffer@_W@detail@v6@fmt@@@std@@_W@34@@detail@v6@fmt@@QEAAPEB_WHPEB_W0@Z 0000000180056ac8     handles.obj
 0001:00055ae4       $unwind$??$parse_format_string@$0A@_WAEAU?$format_handler@V?$arg_formatter@V?$back_insert_iterator@V?$buffer@_W@detail@v6@fmt@@@std@@_W@detail@v6@fmt@@_WV?$basic_format_context@V?$back_insert_iterator@V?$buffer@_W@detail@v6@fmt@@@std@@_W@34@@detail@v6@fmt@@@detail@v6@fmt@@YAXV?$basic_string_view@_W@12@AEAU?$format_handler@V?$arg_formatter@V?$back_insert_iterator@V?$buffer@_W@detail@v6@fmt@@@std@@_W@detail@v6@fmt@@_WV?$basic_format_context@V?$back_insert_iterator@V?$buffer@_W@detail@v6@fmt@@@std@@_W@34@@012@@Z 0000000180056ae4     handles.obj
 0001:00055afc       $unwind$??Rwriter@?1???$parse_format_string@$0A@_WAEAU?$format_handler@V?$arg_formatter@V?$back_insert_iterator@V?$buffer@_W@detail@v6@fmt@@@std@@_W@detail@v6@fmt@@_WV?$basic_format_context@V?$back_insert_iterator@V?$buffer@_W@detail@v6@fmt@@@std@@_W@34@@detail@v6@fmt@@@detail@v6@fmt@@YAXV?$basic_string_view@_W@23@AEAU?$format_handler@V?$arg_formatter@V?$back_insert_iterator@V?$buffer@_W@detail@v6@fmt@@@std@@_W@detail@v6@fmt@@_WV?$basic_format_context@V?$back_insert_iterator@V?$buffer@_W@detail@v6@fmt@@@std@@_W@34@@123@@Z@QEAAXPEB_W2@Z 0000000180056afc     handles.obj
 0001:00055b08       $chain$0$??Rwriter@?1???$parse_format_string@$0A@_WAEAU?$format_handler@V?$arg_formatter@V?$back_insert_iterator@V?$buffer@_W@detail@v6@fmt@@@std@@_W@detail@v6@fmt@@_WV?$basic_format_context@V?$back_insert_iterator@V?$buffer@_W@detail@v6@fmt@@@std@@_W@34@@detail@v6@fmt@@@detail@v6@fmt@@YAXV?$basic_string_view@_W@23@AEAU?$format_handler@V?$arg_formatter@V?$back_insert_iterator@V?$buffer@_W@detail@v6@fmt@@@std@@_W@detail@v6@fmt@@_WV?$basic_format_context@V?$back_insert_iterator@V?$buffer@_W@detail@v6@fmt@@@std@@_W@34@@123@@Z@QEAAXPEB_W2@Z 0000000180056b08     handles.obj
 0001:00055b1c       $chain$1$??Rwriter@?1???$parse_format_string@$0A@_WAEAU?$format_handler@V?$arg_formatter@V?$back_insert_iterator@V?$buffer@_W@detail@v6@fmt@@@std@@_W@detail@v6@fmt@@_WV?$basic_format_context@V?$back_insert_iterator@V?$buffer@_W@detail@v6@fmt@@@std@@_W@34@@detail@v6@fmt@@@detail@v6@fmt@@YAXV?$basic_string_view@_W@23@AEAU?$format_handler@V?$arg_formatter@V?$back_insert_iterator@V?$buffer@_W@detail@v6@fmt@@@std@@_W@detail@v6@fmt@@_WV?$basic_format_context@V?$back_insert_iterator@V?$buffer@_W@detail@v6@fmt@@@std@@_W@34@@123@@Z@QEAAXPEB_W2@Z 0000000180056b1c     handles.obj
 0001:00055b2c       $chain$2$??Rwriter@?1???$parse_format_string@$0A@_WAEAU?$format_handler@V?$arg_formatter@V?$back_insert_iterator@V?$buffer@_W@detail@v6@fmt@@@std@@_W@detail@v6@fmt@@_WV?$basic_format_context@V?$back_insert_iterator@V?$buffer@_W@detail@v6@fmt@@@std@@_W@34@@detail@v6@fmt@@@detail@v6@fmt@@YAXV?$basic_string_view@_W@23@AEAU?$format_handler@V?$arg_formatter@V?$back_insert_iterator@V?$buffer@_W@detail@v6@fmt@@@std@@_W@detail@v6@fmt@@_WV?$basic_format_context@V?$back_insert_iterator@V?$buffer@_W@detail@v6@fmt@@@std@@_W@34@@123@@Z@QEAAXPEB_W2@Z 0000000180056b2c     handles.obj
 0001:00055b40       $unwind$??$write@_WV?$back_insert_iterator@V?$buffer@_W@detail@v6@fmt@@@std@@H$0A@@detail@v6@fmt@@YA?AV?$back_insert_iterator@V?$buffer@_W@detail@v6@fmt@@@std@@V34@H@Z 0000000180056b40     handles.obj
 0001:00055b5c       $unwind$??$write@_WV?$back_insert_iterator@V?$buffer@_W@detail@v6@fmt@@@std@@I$0A@@detail@v6@fmt@@YA?AV?$back_insert_iterator@V?$buffer@_W@detail@v6@fmt@@@std@@V34@I@Z 0000000180056b5c     handles.obj
 0001:00055b74       $unwind$??$write@_WV?$back_insert_iterator@V?$buffer@_W@detail@v6@fmt@@@std@@_J$0A@@detail@v6@fmt@@YA?AV?$back_insert_iterator@V?$buffer@_W@detail@v6@fmt@@@std@@V34@_J@Z 0000000180056b74     handles.obj
 0001:00055b8c       $unwind$??$write@_WV?$back_insert_iterator@V?$buffer@_W@detail@v6@fmt@@@std@@_K$0A@@detail@v6@fmt@@YA?AV?$back_insert_iterator@V?$buffer@_W@detail@v6@fmt@@@std@@V34@_K@Z 0000000180056b8c     handles.obj
 0001:00055b8c       $unwind$?state_case_type@?$output_processor@DV?$string_output_adapter@D@__crt_stdio_output@@V?$format_validation_base@DV?$string_output_adapter@D@__crt_stdio_output@@@2@@__crt_stdio_output@@AEAA_NXZ 0000000180056b8c     libucrt:output.obj
 0001:00055ba4       $unwind$??$write@_WV?$back_insert_iterator@V?$buffer@_W@detail@v6@fmt@@@std@@M$0A@@detail@v6@fmt@@YA?AV?$back_insert_iterator@V?$buffer@_W@detail@v6@fmt@@@std@@V34@M@Z 0000000180056ba4     handles.obj
 0001:00055bcc       $cppxdata$??$write@_WV?$back_insert_iterator@V?$buffer@_W@detail@v6@fmt@@@std@@M$0A@@detail@v6@fmt@@YA?AV?$back_insert_iterator@V?$buffer@_W@detail@v6@fmt@@@std@@V34@M@Z 0000000180056bcc     handles.obj
 0001:00055bd5       $stateUnwindMap$??$write@_WV?$back_insert_iterator@V?$buffer@_W@detail@v6@fmt@@@std@@M$0A@@detail@v6@fmt@@YA?AV?$back_insert_iterator@V?$buffer@_W@detail@v6@fmt@@@std@@V34@M@Z 0000000180056bd5     handles.obj
 0001:00055bd5       $stateUnwindMap$??$write@_WV?$back_insert_iterator@V?$buffer@_W@detail@v6@fmt@@@std@@N$0A@@detail@v6@fmt@@YA?AV?$back_insert_iterator@V?$buffer@_W@detail@v6@fmt@@@std@@V34@N@Z 0000000180056bd5     handles.obj
 0001:00055bd5       $stateUnwindMap$??$write@_WV?$back_insert_iterator@V?$buffer@_W@detail@v6@fmt@@@std@@O$0A@@detail@v6@fmt@@YA?AV?$back_insert_iterator@V?$buffer@_W@detail@v6@fmt@@@std@@V34@O@Z 0000000180056bd5     handles.obj
 0001:00055bdd       $ip2state$??$write@_WV?$back_insert_iterator@V?$buffer@_W@detail@v6@fmt@@@std@@M$0A@@detail@v6@fmt@@YA?AV?$back_insert_iterator@V?$buffer@_W@detail@v6@fmt@@@std@@V34@M@Z 0000000180056bdd     handles.obj
 0001:00055be8       $unwind$??$write@_WV?$back_insert_iterator@V?$buffer@_W@detail@v6@fmt@@@std@@N$0A@@detail@v6@fmt@@YA?AV?$back_insert_iterator@V?$buffer@_W@detail@v6@fmt@@@std@@V34@N@Z 0000000180056be8     handles.obj
 0001:00055be8       $unwind$??$write@_WV?$back_insert_iterator@V?$buffer@_W@detail@v6@fmt@@@std@@O$0A@@detail@v6@fmt@@YA?AV?$back_insert_iterator@V?$buffer@_W@detail@v6@fmt@@@std@@V34@O@Z 0000000180056be8     handles.obj
 0001:00055c10       $cppxdata$??$write@_WV?$back_insert_iterator@V?$buffer@_W@detail@v6@fmt@@@std@@N$0A@@detail@v6@fmt@@YA?AV?$back_insert_iterator@V?$buffer@_W@detail@v6@fmt@@@std@@V34@N@Z 0000000180056c10     handles.obj
 0001:00055c10       $cppxdata$??$write@_WV?$back_insert_iterator@V?$buffer@_W@detail@v6@fmt@@@std@@O$0A@@detail@v6@fmt@@YA?AV?$back_insert_iterator@V?$buffer@_W@detail@v6@fmt@@@std@@V34@O@Z 0000000180056c10     handles.obj
 0001:00055c19       $ip2state$??$write@_WV?$back_insert_iterator@V?$buffer@_W@detail@v6@fmt@@@std@@N$0A@@detail@v6@fmt@@YA?AV?$back_insert_iterator@V?$buffer@_W@detail@v6@fmt@@@std@@V34@N@Z 0000000180056c19     handles.obj
 0001:00055c19       $ip2state$??$write@_WV?$back_insert_iterator@V?$buffer@_W@detail@v6@fmt@@@std@@O$0A@@detail@v6@fmt@@YA?AV?$back_insert_iterator@V?$buffer@_W@detail@v6@fmt@@@std@@V34@O@Z 0000000180056c19     handles.obj
 0001:00055c24       $unwind$??$parse_arg_id@_WAEAU?$id_adapter@AEAU?$format_handler@V?$arg_formatter@V?$back_insert_iterator@V?$buffer@_W@detail@v6@fmt@@@std@@_W@detail@v6@fmt@@_WV?$basic_format_context@V?$back_insert_iterator@V?$buffer@_W@detail@v6@fmt@@@std@@_W@34@@detail@v6@fmt@@_W@detail@v6@fmt@@@detail@v6@fmt@@YAPEB_WPEB_W0AEAU?$id_adapter@AEAU?$format_handler@V?$arg_formatter@V?$back_insert_iterator@V?$buffer@_W@detail@v6@fmt@@@std@@_W@detail@v6@fmt@@_WV?$basic_format_context@V?$back_insert_iterator@V?$buffer@_W@detail@v6@fmt@@@std@@_W@34@@detail@v6@fmt@@_W@012@@Z 0000000180056c24     handles.obj
 0001:00055c24       $unwind$__acrt_GetLocaleInfoEx 0000000180056c24     libucrt:winapi_thunks.obj
 0001:00055c24       $unwind$__acrt_LCIDToLocaleName 0000000180056c24     libucrt:winapi_thunks.obj
 0001:00055c24       $unwind$__acrt_DownlevelLCIDToLocaleName 0000000180056c24     libucrt:lcidtoname_downlevel.obj
 0001:00055c24       $unwind$__lc_lctowcs       0000000180056c24     libucrt:wsetlocale.obj
 0001:00055c24       $unwind$_invalid_parameter 0000000180056c24     libucrt:invalid_parameter.obj
 0001:00055c24       $unwind$_wcsdup            0000000180056c24     libucrt:wcsdup.obj
 0001:00055c38       $unwind$??$parse_format_specs@_WAEAV?$specs_checker@V?$specs_handler@V?$basic_format_parse_context@_WUerror_handler@detail@v6@fmt@@@v6@fmt@@V?$basic_format_context@V?$back_insert_iterator@V?$buffer@_W@detail@v6@fmt@@@std@@_W@23@@detail@v6@fmt@@@detail@v6@fmt@@@detail@v6@fmt@@YAPEB_WPEB_W0AEAV?$specs_checker@V?$specs_handler@V?$basic_format_parse_context@_WUerror_handler@detail@v6@fmt@@@v6@fmt@@V?$basic_format_context@V?$back_insert_iterator@V?$buffer@_W@detail@v6@fmt@@@std@@_W@23@@detail@v6@fmt@@@012@@Z 0000000180056c38     handles.obj
 0001:00055c48       $chain$1$??$parse_format_specs@_WAEAV?$specs_checker@V?$specs_handler@V?$basic_format_parse_context@_WUerror_handler@detail@v6@fmt@@@v6@fmt@@V?$basic_format_context@V?$back_insert_iterator@V?$buffer@_W@detail@v6@fmt@@@std@@_W@23@@detail@v6@fmt@@@detail@v6@fmt@@@detail@v6@fmt@@YAPEB_WPEB_W0AEAV?$specs_checker@V?$specs_handler@V?$basic_format_parse_context@_WUerror_handler@detail@v6@fmt@@@v6@fmt@@V?$basic_format_context@V?$back_insert_iterator@V?$buffer@_W@detail@v6@fmt@@@std@@_W@23@@detail@v6@fmt@@@012@@Z 0000000180056c48     handles.obj
 0001:00055c60       $chain$3$??$parse_format_specs@_WAEAV?$specs_checker@V?$specs_handler@V?$basic_format_parse_context@_WUerror_handler@detail@v6@fmt@@@v6@fmt@@V?$basic_format_context@V?$back_insert_iterator@V?$buffer@_W@detail@v6@fmt@@@std@@_W@23@@detail@v6@fmt@@@detail@v6@fmt@@@detail@v6@fmt@@YAPEB_WPEB_W0AEAV?$specs_checker@V?$specs_handler@V?$basic_format_parse_context@_WUerror_handler@detail@v6@fmt@@@v6@fmt@@V?$basic_format_context@V?$back_insert_iterator@V?$buffer@_W@detail@v6@fmt@@@std@@_W@23@@detail@v6@fmt@@@012@@Z 0000000180056c60     handles.obj
 0001:00055c78       $chain$4$??$parse_format_specs@_WAEAV?$specs_checker@V?$specs_handler@V?$basic_format_parse_context@_WUerror_handler@detail@v6@fmt@@@v6@fmt@@V?$basic_format_context@V?$back_insert_iterator@V?$buffer@_W@detail@v6@fmt@@@std@@_W@23@@detail@v6@fmt@@@detail@v6@fmt@@@detail@v6@fmt@@YAPEB_WPEB_W0AEAV?$specs_checker@V?$specs_handler@V?$basic_format_parse_context@_WUerror_handler@detail@v6@fmt@@@v6@fmt@@V?$basic_format_context@V?$back_insert_iterator@V?$buffer@_W@detail@v6@fmt@@@std@@_W@23@@detail@v6@fmt@@@012@@Z 0000000180056c78     handles.obj
 0001:00055c88       $unwind$?_Tidy@?$vector@V?$basic_string@_WU?$char_traits@_W@std@@V?$allocator@_W@2@@std@@V?$allocator@V?$basic_string@_WU?$char_traits@_W@std@@V?$allocator@_W@2@@std@@@2@@std@@AEAAXXZ 0000000180056c88     Pclass.obj
 0001:00055c88       $unwind$??$?RH$0A@@?$arg_formatter_base@V?$back_insert_iterator@V?$buffer@_W@detail@v6@fmt@@@std@@_WUerror_handler@detail@v6@fmt@@@detail@v6@fmt@@QEAA?AV?$back_insert_iterator@V?$buffer@_W@detail@v6@fmt@@@std@@H@Z 0000000180056c88     handles.obj
 0001:00055c88       $unwind$?_Tidy@?$vector@UProcessPerfData@@V?$allocator@UProcessPerfData@@@std@@@std@@AEAAXXZ 0000000180056c88     perfthread.obj
 0001:00055c88       $unwind$?_Locimp_dtor@_Locimp@locale@std@@CAXPEAV123@@Z 0000000180056c88     libcpmt:locale0.obj
 0001:00055c88       $unwind$iswctype           0000000180056c88     libucrt:iswctype.obj
 0001:00055c94       $unwind$??$visit_format_arg@V?$arg_formatter@V?$back_insert_iterator@V?$buffer@_W@detail@v6@fmt@@@std@@_W@detail@v6@fmt@@V?$basic_format_context@V?$back_insert_iterator@V?$buffer@_W@detail@v6@fmt@@@std@@_W@34@@v6@fmt@@YA?AV?$back_insert_iterator@V?$buffer@_W@detail@v6@fmt@@@std@@$$QEAV?$arg_formatter@V?$back_insert_iterator@V?$buffer@_W@detail@v6@fmt@@@std@@_W@detail@01@AEBV?$basic_format_arg@V?$basic_format_context@V?$back_insert_iterator@V?$buffer@_W@detail@v6@fmt@@@std@@_W@v6@fmt@@@01@@Z 0000000180056c94     handles.obj
 0001:00055cb4       $unwind$??$write_ptr@_WV?$back_insert_iterator@V?$buffer@_W@detail@v6@fmt@@@std@@_K@detail@v6@fmt@@YA?AV?$back_insert_iterator@V?$buffer@_W@detail@v6@fmt@@@std@@V34@_KPEBU?$basic_format_specs@_W@12@@Z 0000000180056cb4     handles.obj
 0001:00055ccc       $chain$2$??$write_ptr@_WV?$back_insert_iterator@V?$buffer@_W@detail@v6@fmt@@@std@@_K@detail@v6@fmt@@YA?AV?$back_insert_iterator@V?$buffer@_W@detail@v6@fmt@@@std@@V34@_KPEBU?$basic_format_specs@_W@12@@Z 0000000180056ccc     handles.obj
 0001:00055ce0       $chain$3$??$write_ptr@_WV?$back_insert_iterator@V?$buffer@_W@detail@v6@fmt@@@std@@_K@detail@v6@fmt@@YA?AV?$back_insert_iterator@V?$buffer@_W@detail@v6@fmt@@@std@@V34@_KPEBU?$basic_format_specs@_W@12@@Z 0000000180056ce0     handles.obj
 0001:00055cf0       $unwind$??$format_decimal@_W_K@detail@v6@fmt@@YA?AU?$format_decimal_result@PEA_W@012@PEA_W_KH@Z 0000000180056cf0     handles.obj
 0001:00055cf0       $unwind$__GSHandlerCheckCommon 0000000180056cf0     LIBCMT:gshandler.obj
 0001:00055cf0       $unwind$__acrt_WideCharToMultiByte 0000000180056cf0     libucrt:widechartomultibyte.obj
 0001:00055cf8       $chain$0$??$format_decimal@_W_K@detail@v6@fmt@@YA?AU?$format_decimal_result@PEA_W@012@PEA_W_KH@Z 0000000180056cf8     handles.obj
 0001:00055d0c       $chain$1$??$format_decimal@_W_K@detail@v6@fmt@@YA?AU?$format_decimal_result@PEA_W@012@PEA_W_KH@Z 0000000180056d0c     handles.obj
 0001:00055d1c       $unwind$??0?$float_writer@_W@detail@v6@fmt@@QEAA@PEBDHHUfloat_specs@123@_W@Z 0000000180056d1c     handles.obj
 0001:00055d2c       $chain$0$?on_char@char_spec_handler@?$arg_formatter_base@V?$back_insert_iterator@V?$buffer@_W@detail@v6@fmt@@@std@@_WUerror_handler@detail@v6@fmt@@@detail@v6@fmt@@QEAAXXZ 0000000180056d2c     handles.obj
 0001:00055d40       $chain$1$?on_char@char_spec_handler@?$arg_formatter_base@V?$back_insert_iterator@V?$buffer@_W@detail@v6@fmt@@@std@@_WUerror_handler@detail@v6@fmt@@@detail@v6@fmt@@QEAAXXZ 0000000180056d40     handles.obj
 0001:00055d50       $chain$5$??$get_id@_W@?$basic_format_args@V?$basic_format_context@V?$back_insert_iterator@V?$buffer@_W@detail@v6@fmt@@@std@@_W@v6@fmt@@@v6@fmt@@QEBAHV?$basic_string_view@_W@12@@Z 0000000180056d50     handles.obj
 0001:00055d78       $chain$7$??$get_id@_W@?$basic_format_args@V?$basic_format_context@V?$back_insert_iterator@V?$buffer@_W@detail@v6@fmt@@@std@@_W@v6@fmt@@@v6@fmt@@QEBAHV?$basic_string_view@_W@12@@Z 0000000180056d78     handles.obj
 0001:00055da0       $unwind$?PrintTitle@@YA?AV?$basic_string@_WU?$char_traits@_W@std@@V?$allocator@_W@2@@std@@H@Z 0000000180056da0     Pclass.obj
 0001:00055da0       $unwind$??$write_int@H@?$arg_formatter_base@V?$back_insert_iterator@V?$buffer@_W@detail@v6@fmt@@@std@@_WUerror_handler@detail@v6@fmt@@@detail@v6@fmt@@AEAAXHAEBU?$basic_format_specs@_W@23@@Z 0000000180056da0     handles.obj
 0001:00055da8       $unwind$??R<lambda_fbad59960194a21b5f35257a64aadaa4>@@QEBAXXZ 0000000180056da8     Plist.obj
 0001:00055da8       $unwind$??$prettify@PEA_W@?$float_writer@_W@detail@v6@fmt@@AEBAPEA_WPEA_W@Z 0000000180056da8     handles.obj
 0001:00055da8       $unwind$ProcessCodePage    0000000180056da8     libucrt:get_qualified_locale.obj
 0001:00055da8       $unwind$ProcessCodePage    0000000180056da8     libucrt:getqloc_downlevel.obj
 0001:00055da8       $unwind$TestDefaultLanguage 0000000180056da8     libucrt:getqloc_downlevel.obj
 0001:00055db8       $chain$0$??$prettify@PEA_W@?$float_writer@_W@detail@v6@fmt@@AEBAPEA_WPEA_W@Z 0000000180056db8     handles.obj
 0001:00055dcc       $unwind$??$parse_arg_id@_WU?$precision_adapter@AEAV?$specs_checker@V?$specs_handler@V?$basic_format_parse_context@_WUerror_handler@detail@v6@fmt@@@v6@fmt@@V?$basic_format_context@V?$back_insert_iterator@V?$buffer@_W@detail@v6@fmt@@@std@@_W@23@@detail@v6@fmt@@@detail@v6@fmt@@_W@detail@v6@fmt@@@detail@v6@fmt@@YAPEB_WPEB_W0$$QEAU?$precision_adapter@AEAV?$specs_checker@V?$specs_handler@V?$basic_format_parse_context@_WUerror_handler@detail@v6@fmt@@@v6@fmt@@V?$basic_format_context@V?$back_insert_iterator@V?$buffer@_W@detail@v6@fmt@@@std@@_W@23@@detail@v6@fmt@@@detail@v6@fmt@@_W@012@@Z 0000000180056dcc     handles.obj
 0001:00055dcc       $unwind$??$parse_arg_id@_WU?$width_adapter@AEAV?$specs_checker@V?$specs_handler@V?$basic_format_parse_context@_WUerror_handler@detail@v6@fmt@@@v6@fmt@@V?$basic_format_context@V?$back_insert_iterator@V?$buffer@_W@detail@v6@fmt@@@std@@_W@23@@detail@v6@fmt@@@detail@v6@fmt@@_W@detail@v6@fmt@@@detail@v6@fmt@@YAPEB_WPEB_W0$$QEAU?$width_adapter@AEAV?$specs_checker@V?$specs_handler@V?$basic_format_parse_context@_WUerror_handler@detail@v6@fmt@@@v6@fmt@@V?$basic_format_context@V?$back_insert_iterator@V?$buffer@_W@detail@v6@fmt@@@std@@_W@23@@detail@v6@fmt@@@detail@v6@fmt@@_W@012@@Z 0000000180056dcc     handles.obj
 0001:00055dec       $unwind$??$write@_WV?$back_insert_iterator@V?$buffer@_W@detail@v6@fmt@@@std@@M$0A@@detail@v6@fmt@@YA?AV?$back_insert_iterator@V?$buffer@_W@detail@v6@fmt@@@std@@V34@MU?$basic_format_specs@_W@12@Vlocale_ref@012@@Z 0000000180056dec     handles.obj
 0001:00055e18       $cppxdata$??$write@_WV?$back_insert_iterator@V?$buffer@_W@detail@v6@fmt@@@std@@M$0A@@detail@v6@fmt@@YA?AV?$back_insert_iterator@V?$buffer@_W@detail@v6@fmt@@@std@@V34@MU?$basic_format_specs@_W@12@Vlocale_ref@012@@Z 0000000180056e18     handles.obj
 0001:00055e21       $stateUnwindMap$??$write@_WV?$back_insert_iterator@V?$buffer@_W@detail@v6@fmt@@@std@@M$0A@@detail@v6@fmt@@YA?AV?$back_insert_iterator@V?$buffer@_W@detail@v6@fmt@@@std@@V34@MU?$basic_format_specs@_W@12@Vlocale_ref@012@@Z 0000000180056e21     handles.obj
 0001:00055e21       $stateUnwindMap$??$write@_WV?$back_insert_iterator@V?$buffer@_W@detail@v6@fmt@@@std@@N$0A@@detail@v6@fmt@@YA?AV?$back_insert_iterator@V?$buffer@_W@detail@v6@fmt@@@std@@V34@NU?$basic_format_specs@_W@12@Vlocale_ref@012@@Z 0000000180056e21     handles.obj
 0001:00055e21       $stateUnwindMap$??$write@_WV?$back_insert_iterator@V?$buffer@_W@detail@v6@fmt@@@std@@O$0A@@detail@v6@fmt@@YA?AV?$back_insert_iterator@V?$buffer@_W@detail@v6@fmt@@@std@@V34@OU?$basic_format_specs@_W@12@Vlocale_ref@012@@Z 0000000180056e21     handles.obj
 0001:00055e2f       $ip2state$??$write@_WV?$back_insert_iterator@V?$buffer@_W@detail@v6@fmt@@@std@@M$0A@@detail@v6@fmt@@YA?AV?$back_insert_iterator@V?$buffer@_W@detail@v6@fmt@@@std@@V34@MU?$basic_format_specs@_W@12@Vlocale_ref@012@@Z 0000000180056e2f     handles.obj
 0001:00055e40       $unwind$??$write@_WV?$back_insert_iterator@V?$buffer@_W@detail@v6@fmt@@@std@@N$0A@@detail@v6@fmt@@YA?AV?$back_insert_iterator@V?$buffer@_W@detail@v6@fmt@@@std@@V34@NU?$basic_format_specs@_W@12@Vlocale_ref@012@@Z 0000000180056e40     handles.obj
 0001:00055e40       $unwind$??$write@_WV?$back_insert_iterator@V?$buffer@_W@detail@v6@fmt@@@std@@O$0A@@detail@v6@fmt@@YA?AV?$back_insert_iterator@V?$buffer@_W@detail@v6@fmt@@@std@@V34@OU?$basic_format_specs@_W@12@Vlocale_ref@012@@Z 0000000180056e40     handles.obj
 0001:00055e6c       $cppxdata$??$write@_WV?$back_insert_iterator@V?$buffer@_W@detail@v6@fmt@@@std@@N$0A@@detail@v6@fmt@@YA?AV?$back_insert_iterator@V?$buffer@_W@detail@v6@fmt@@@std@@V34@NU?$basic_format_specs@_W@12@Vlocale_ref@012@@Z 0000000180056e6c     handles.obj
 0001:00055e6c       $cppxdata$??$write@_WV?$back_insert_iterator@V?$buffer@_W@detail@v6@fmt@@@std@@O$0A@@detail@v6@fmt@@YA?AV?$back_insert_iterator@V?$buffer@_W@detail@v6@fmt@@@std@@V34@OU?$basic_format_specs@_W@12@Vlocale_ref@012@@Z 0000000180056e6c     handles.obj
 0001:00055e75       $ip2state$??$write@_WV?$back_insert_iterator@V?$buffer@_W@detail@v6@fmt@@@std@@N$0A@@detail@v6@fmt@@YA?AV?$back_insert_iterator@V?$buffer@_W@detail@v6@fmt@@@std@@V34@NU?$basic_format_specs@_W@12@Vlocale_ref@012@@Z 0000000180056e75     handles.obj
 0001:00055e75       $ip2state$??$write@_WV?$back_insert_iterator@V?$buffer@_W@detail@v6@fmt@@@std@@O$0A@@detail@v6@fmt@@YA?AV?$back_insert_iterator@V?$buffer@_W@detail@v6@fmt@@@std@@V34@OU?$basic_format_specs@_W@12@Vlocale_ref@012@@Z 0000000180056e75     handles.obj
 0001:00055e84       $unwind$?on_dec@?$int_writer@V?$back_insert_iterator@V?$buffer@_W@detail@v6@fmt@@@std@@_WI@detail@v6@fmt@@QEAAXXZ 0000000180056e84     handles.obj
 0001:00055e90       $unwind$?on_num@?$int_writer@V?$back_insert_iterator@V?$buffer@_W@detail@v6@fmt@@@std@@_WI@detail@v6@fmt@@QEAAXXZ 0000000180056e90     handles.obj
 0001:00055eb4       $cppxdata$?on_num@?$int_writer@V?$back_insert_iterator@V?$buffer@_W@detail@v6@fmt@@@std@@_WI@detail@v6@fmt@@QEAAXXZ 0000000180056eb4     handles.obj
 0001:00055ebd       $stateUnwindMap$?on_num@?$int_writer@V?$back_insert_iterator@V?$buffer@_W@detail@v6@fmt@@@std@@_WI@detail@v6@fmt@@QEAAXXZ 0000000180056ebd     handles.obj
 0001:00055ebd       $stateUnwindMap$?on_num@?$int_writer@V?$back_insert_iterator@V?$buffer@_W@detail@v6@fmt@@@std@@_W_K@detail@v6@fmt@@QEAAXXZ 0000000180056ebd     handles.obj
 0001:00055ecb       $ip2state$?on_num@?$int_writer@V?$back_insert_iterator@V?$buffer@_W@detail@v6@fmt@@@std@@_WI@detail@v6@fmt@@QEAAXXZ 0000000180056ecb     handles.obj
 0001:00055edc       $unwind$??$handle_int_type_spec@AEAU?$int_writer@V?$back_insert_iterator@V?$buffer@_W@detail@v6@fmt@@@std@@_WI@detail@v6@fmt@@@detail@v6@fmt@@YAXDAEAU?$int_writer@V?$back_insert_iterator@V?$buffer@_W@detail@v6@fmt@@@std@@_WI@012@@Z 0000000180056edc     handles.obj
 0001:00055ef4       $cppxdata$??$handle_int_type_spec@AEAU?$int_writer@V?$back_insert_iterator@V?$buffer@_W@detail@v6@fmt@@@std@@_WI@detail@v6@fmt@@@detail@v6@fmt@@YAXDAEAU?$int_writer@V?$back_insert_iterator@V?$buffer@_W@detail@v6@fmt@@@std@@_WI@012@@Z 0000000180056ef4     handles.obj
 0001:00055efd       $stateUnwindMap$??$handle_int_type_spec@AEAU?$int_writer@V?$back_insert_iterator@V?$buffer@_W@detail@v6@fmt@@@std@@_WI@detail@v6@fmt@@@detail@v6@fmt@@YAXDAEAU?$int_writer@V?$back_insert_iterator@V?$buffer@_W@detail@v6@fmt@@@std@@_WI@012@@Z 0000000180056efd     handles.obj
 0001:00055efd       $stateUnwindMap$??$handle_int_type_spec@AEAU?$int_writer@V?$back_insert_iterator@V?$buffer@_W@detail@v6@fmt@@@std@@_W_K@detail@v6@fmt@@@detail@v6@fmt@@YAXDAEAU?$int_writer@V?$back_insert_iterator@V?$buffer@_W@detail@v6@fmt@@@std@@_W_K@012@@Z 0000000180056efd     handles.obj
 0001:00055f04       $ip2state$??$handle_int_type_spec@AEAU?$int_writer@V?$back_insert_iterator@V?$buffer@_W@detail@v6@fmt@@@std@@_WI@detail@v6@fmt@@@detail@v6@fmt@@YAXDAEAU?$int_writer@V?$back_insert_iterator@V?$buffer@_W@detail@v6@fmt@@@std@@_WI@012@@Z 0000000180056f04     handles.obj
 0001:00055f0c       $unwind$?on_dec@?$int_writer@V?$back_insert_iterator@V?$buffer@_W@detail@v6@fmt@@@std@@_W_K@detail@v6@fmt@@QEAAXXZ 0000000180056f0c     handles.obj
 0001:00055f0c       $unwind$_call_matherr      0000000180056f0c     libucrt:libm_error.obj
 0001:00055f14       $unwind$?on_num@?$int_writer@V?$back_insert_iterator@V?$buffer@_W@detail@v6@fmt@@@std@@_W_K@detail@v6@fmt@@QEAAXXZ 0000000180056f14     handles.obj
 0001:00055f38       $cppxdata$?on_num@?$int_writer@V?$back_insert_iterator@V?$buffer@_W@detail@v6@fmt@@@std@@_W_K@detail@v6@fmt@@QEAAXXZ 0000000180056f38     handles.obj
 0001:00055f41       $ip2state$?on_num@?$int_writer@V?$back_insert_iterator@V?$buffer@_W@detail@v6@fmt@@@std@@_W_K@detail@v6@fmt@@QEAAXXZ 0000000180056f41     handles.obj
 0001:00055f50       $unwind$??$handle_int_type_spec@AEAU?$int_writer@V?$back_insert_iterator@V?$buffer@_W@detail@v6@fmt@@@std@@_W_K@detail@v6@fmt@@@detail@v6@fmt@@YAXDAEAU?$int_writer@V?$back_insert_iterator@V?$buffer@_W@detail@v6@fmt@@@std@@_W_K@012@@Z 0000000180056f50     handles.obj
 0001:00055f68       $cppxdata$??$handle_int_type_spec@AEAU?$int_writer@V?$back_insert_iterator@V?$buffer@_W@detail@v6@fmt@@@std@@_W_K@detail@v6@fmt@@@detail@v6@fmt@@YAXDAEAU?$int_writer@V?$back_insert_iterator@V?$buffer@_W@detail@v6@fmt@@@std@@_W_K@012@@Z 0000000180056f68     handles.obj
 0001:00055f71       $ip2state$??$handle_int_type_spec@AEAU?$int_writer@V?$back_insert_iterator@V?$buffer@_W@detail@v6@fmt@@@std@@_W_K@detail@v6@fmt@@@detail@v6@fmt@@YAXDAEAU?$int_writer@V?$back_insert_iterator@V?$buffer@_W@detail@v6@fmt@@@std@@_W_K@012@@Z 0000000180056f71     handles.obj
 0001:00055f78       $unwind$??$write_bytes@_WV?$back_insert_iterator@V?$buffer@_W@detail@v6@fmt@@@std@@@detail@v6@fmt@@YA?AV?$back_insert_iterator@V?$buffer@_W@detail@v6@fmt@@@std@@V34@V?$basic_string_view@D@12@AEBU?$basic_format_specs@_W@12@@Z 0000000180056f78     handles.obj
 0001:00055f94       $unwind$??$fill@PEA_W_W@detail@v6@fmt@@YAPEA_WPEA_W_KAEBU?$fill_t@_W@012@@Z 0000000180056f94     handles.obj
 0001:00055fa8       $chain$0$??$fill@PEA_W_W@detail@v6@fmt@@YAPEA_WPEA_W_KAEBU?$fill_t@_W@012@@Z 0000000180056fa8     handles.obj
 0001:00055fbc       $chain$1$??$fill@PEA_W_W@detail@v6@fmt@@YAPEA_WPEA_W_KAEBU?$fill_t@_W@012@@Z 0000000180056fbc     handles.obj
 0001:00055fcc       $unwind$??$get_dynamic_spec@Vprecision_checker@detail@v6@fmt@@V?$basic_format_arg@V?$basic_format_context@V?$back_insert_iterator@V?$buffer@_W@detail@v6@fmt@@@std@@_W@v6@fmt@@@34@Uerror_handler@234@@detail@v6@fmt@@YAHV?$basic_format_arg@V?$basic_format_context@V?$back_insert_iterator@V?$buffer@_W@detail@v6@fmt@@@std@@_W@v6@fmt@@@12@Uerror_handler@012@@Z 0000000180056fcc     handles.obj
 0001:00055fcc       $unwind$??$get_dynamic_spec@Vwidth_checker@detail@v6@fmt@@V?$basic_format_arg@V?$basic_format_context@V?$back_insert_iterator@V?$buffer@_W@detail@v6@fmt@@@std@@_W@v6@fmt@@@34@Uerror_handler@234@@detail@v6@fmt@@YAHV?$basic_format_arg@V?$basic_format_context@V?$back_insert_iterator@V?$buffer@_W@detail@v6@fmt@@@std@@_W@v6@fmt@@@12@Uerror_handler@012@@Z 0000000180056fcc     handles.obj
 0001:00055fd4       $unwind$??$write_int@V?$back_insert_iterator@V?$buffer@_W@detail@v6@fmt@@@std@@_WV<lambda_0273f2d8c97c19346923ccbca9d35cd0>@@@detail@v6@fmt@@YA?AV?$back_insert_iterator@V?$buffer@_W@detail@v6@fmt@@@std@@V34@HV?$basic_string_view@D@12@AEBU?$basic_format_specs@_W@12@V<lambda_0273f2d8c97c19346923ccbca9d35cd0>@@@Z 0000000180056fd4     handles.obj
 0001:00055fd4       $unwind$??$write_int@V?$back_insert_iterator@V?$buffer@_W@detail@v6@fmt@@@std@@_WV<lambda_1584a04d9a5f951756080462468a1c79>@@@detail@v6@fmt@@YA?AV?$back_insert_iterator@V?$buffer@_W@detail@v6@fmt@@@std@@V34@HV?$basic_string_view@D@12@AEBU?$basic_format_specs@_W@12@V<lambda_1584a04d9a5f951756080462468a1c79>@@@Z 0000000180056fd4     handles.obj
 0001:00055fd4       $unwind$??$write_int@V?$back_insert_iterator@V?$buffer@_W@detail@v6@fmt@@@std@@_WV<lambda_46028ac11bf91aacf0795357afd8c72d>@@@detail@v6@fmt@@YA?AV?$back_insert_iterator@V?$buffer@_W@detail@v6@fmt@@@std@@V34@HV?$basic_string_view@D@12@AEBU?$basic_format_specs@_W@12@V<lambda_46028ac11bf91aacf0795357afd8c72d>@@@Z 0000000180056fd4     handles.obj
 0001:00055fd4       $unwind$??$write_int@V?$back_insert_iterator@V?$buffer@_W@detail@v6@fmt@@@std@@_WV<lambda_c4159916ea5054600e9c49615e89ce82>@@@detail@v6@fmt@@YA?AV?$back_insert_iterator@V?$buffer@_W@detail@v6@fmt@@@std@@V34@HV?$basic_string_view@D@12@AEBU?$basic_format_specs@_W@12@V<lambda_c4159916ea5054600e9c49615e89ce82>@@@Z 0000000180056fd4     handles.obj
 0001:00055fd4       $unwind$??$write_int@V?$back_insert_iterator@V?$buffer@_W@detail@v6@fmt@@@std@@_WV<lambda_dbc99c5d30ad811266da5b27d7d4d7eb>@@@detail@v6@fmt@@YA?AV?$back_insert_iterator@V?$buffer@_W@detail@v6@fmt@@@std@@V34@HV?$basic_string_view@D@12@AEBU?$basic_format_specs@_W@12@V<lambda_dbc99c5d30ad811266da5b27d7d4d7eb>@@@Z 0000000180056fd4     handles.obj
 0001:00055fd4       $unwind$??$write_int@V?$back_insert_iterator@V?$buffer@_W@detail@v6@fmt@@@std@@_WV<lambda_ee8e8661040b0e68e19c307d8706693d>@@@detail@v6@fmt@@YA?AV?$back_insert_iterator@V?$buffer@_W@detail@v6@fmt@@@std@@V34@HV?$basic_string_view@D@12@AEBU?$basic_format_specs@_W@12@V<lambda_ee8e8661040b0e68e19c307d8706693d>@@@Z 0000000180056fd4     handles.obj
 0001:00055ff0       $unwind$??$write_int@V?$back_insert_iterator@V?$buffer@_W@detail@v6@fmt@@@std@@_WV<lambda_766228445ed89183d7065b0051936627>@@@detail@v6@fmt@@YA?AV?$back_insert_iterator@V?$buffer@_W@detail@v6@fmt@@@std@@V34@HV?$basic_string_view@D@12@AEBU?$basic_format_specs@_W@12@V<lambda_766228445ed89183d7065b0051936627>@@@Z 0000000180056ff0     handles.obj
 0001:0005600c       $unwind$??1PluginSettings@@QEAA@XZ 000000018005700c     Pcfg.obj
 0001:0005601c       $cppxdata$??1PluginSettings@@QEAA@XZ 000000018005701c     Pcfg.obj
 0001:00056021       $ip2state$??1PluginSettings@@QEAA@XZ 0000000180057021     Pcfg.obj
 0001:00056024       $unwind$??1PluginDialogBuilder@@QEAA@XZ 0000000180057024     Pcfg.obj
 0001:0005603c       $cppxdata$??1PluginDialogBuilder@@QEAA@XZ 000000018005703c     Pcfg.obj
 0001:00056041       $ip2state$??1PluginDialogBuilder@@QEAA@XZ 0000000180057041     Pcfg.obj
 0001:00056044       $unwind$?AddButtons@PluginDialogBuilder@@QEAAXHPEBHHH@Z 0000000180057044     Pcfg.obj
 0001:00056050       $chain$4$?AddButtons@PluginDialogBuilder@@QEAAXHPEBHHH@Z 0000000180057050     Pcfg.obj
 0001:00056074       $chain$5$?AddButtons@PluginDialogBuilder@@QEAAXHPEBHHH@Z 0000000180057074     Pcfg.obj
 0001:00056084       $unwind$?ShowDialogEx@PluginDialogBuilder@@QEAA_JXZ 0000000180057084     Pcfg.obj
 0001:00056090       $chain$4$?ShowDialogEx@PluginDialogBuilder@@QEAA_JXZ 0000000180057090     Pcfg.obj
 0001:000560b4       $chain$6$?ShowDialogEx@PluginDialogBuilder@@QEAA_JXZ 00000001800570b4     Pcfg.obj
 0001:000560cc       $chain$7$?ShowDialogEx@PluginDialogBuilder@@QEAA_JXZ 00000001800570cc     Pcfg.obj
 0001:000560e0       $chain$8$?ShowDialogEx@PluginDialogBuilder@@QEAA_JXZ 00000001800570e0     Pcfg.obj
 0001:000560f0       $unwind$?AddDialogItem@PluginDialogBuilder@@AEAAPEAUFarDialogItem@@W4FARDIALOGITEMTYPES@@PEB_W@Z 00000001800570f0     Pcfg.obj
 0001:00056100       $chain$0$?AddDialogItem@PluginDialogBuilder@@AEAAPEAUFarDialogItem@@W4FARDIALOGITEMTYPES@@PEB_W@Z 0000000180057100     Pcfg.obj
 0001:00056114       $chain$1$?AddDialogItem@PluginDialogBuilder@@AEAAPEAUFarDialogItem@@W4FARDIALOGITEMTYPES@@PEB_W@Z 0000000180057114     Pcfg.obj
 0001:00056128       $chain$2$?AddDialogItem@PluginDialogBuilder@@AEAAPEAUFarDialogItem@@W4FARDIALOGITEMTYPES@@PEB_W@Z 0000000180057128     Pcfg.obj
 0001:00056138       $chain$3$?AddDialogItem@PluginDialogBuilder@@AEAAPEAUFarDialogItem@@W4FARDIALOGITEMTYPES@@PEB_W@Z 0000000180057138     Pcfg.obj
 0001:00056148       $unwind$?Read@options@@QEAAXXZ 0000000180057148     Pcfg.obj
 0001:00056168       $cppxdata$?Read@options@@QEAAXXZ 0000000180057168     Pcfg.obj
 0001:00056171       $stateUnwindMap$?Read@options@@QEAAXXZ 0000000180057171     Pcfg.obj
 0001:00056171       $stateUnwindMap$?Write@options@@QEBAXXZ 0000000180057171     Pcfg.obj
 0001:0005617d       $ip2state$?Read@options@@QEAAXXZ 000000018005717d     Pcfg.obj
 0001:00056188       $unwind$?Write@options@@QEBAXXZ 0000000180057188     Pcfg.obj
 0001:000561a8       $cppxdata$?Write@options@@QEBAXXZ 00000001800571a8     Pcfg.obj
 0001:000561b1       $ip2state$?Write@options@@QEBAXXZ 00000001800571b1     Pcfg.obj
 0001:000561bc       $unwind$?Config@@YAHXZ     00000001800571bc     Pcfg.obj
 0001:000561e4       $cppxdata$?Config@@YAHXZ   00000001800571e4     Pcfg.obj
 0001:000561ed       $stateUnwindMap$?Config@@YAHXZ 00000001800571ed     Pcfg.obj
 0001:000561fa       $ip2state$?Config@@YAHXZ   00000001800571fa     Pcfg.obj
 0001:00056208       $unwind$?append@?$basic_string@_WU?$char_traits@_W@std@@V?$allocator@_W@2@@std@@QEAAAEAV12@_K_W@Z 0000000180057208     Pclass.obj
 0001:0005621c       $chain$1$?append@?$basic_string@_WU?$char_traits@_W@std@@V?$allocator@_W@2@@std@@QEAAAEAV12@_K_W@Z 000000018005721c     Pclass.obj
 0001:00056234       $chain$2$?append@?$basic_string@_WU?$char_traits@_W@std@@V?$allocator@_W@2@@std@@QEAAAEAV12@_K_W@Z 0000000180057234     Pclass.obj
 0001:00056234       $chain$4$?append@?$basic_string@_WU?$char_traits@_W@std@@V?$allocator@_W@2@@std@@QEAAAEAV12@_K_W@Z 0000000180057234     Pclass.obj
 0001:00056244       $chain$3$?append@?$basic_string@_WU?$char_traits@_W@std@@V?$allocator@_W@2@@std@@QEAAAEAV12@_K_W@Z 0000000180057244     Pclass.obj
 0001:0005625c       $unwind$?insert@?$basic_string@_WU?$char_traits@_W@std@@V?$allocator@_W@2@@std@@QEAAAEAV12@_KQEB_W0@Z 000000018005725c     Pclass.obj
 0001:00056268       $chain$2$?insert@?$basic_string@_WU?$char_traits@_W@std@@V?$allocator@_W@2@@std@@QEAAAEAV12@_KQEB_W0@Z 0000000180057268     Pclass.obj
 0001:00056284       $chain$3$?insert@?$basic_string@_WU?$char_traits@_W@std@@V?$allocator@_W@2@@std@@QEAAAEAV12@_KQEB_W0@Z 0000000180057284     Pclass.obj
 0001:00056294       $unwind$??0Plist@@QEAA@XZ  0000000180057294     Pclass.obj
 0001:000562b0       $cppxdata$??0Plist@@QEAA@XZ 00000001800572b0     Pclass.obj
 0001:000562b9       $stateUnwindMap$??0Plist@@QEAA@XZ 00000001800572b9     Pclass.obj
 0001:000562d9       $ip2state$??0Plist@@QEAA@XZ 00000001800572d9     Pclass.obj
 0001:000562e8       $unwind$?Connect@Plist@@QEAA_NPEB_W00@Z 00000001800572e8     Pclass.obj
 0001:00056308       $cppxdata$?Connect@Plist@@QEAA_NPEB_W00@Z 0000000180057308     Pclass.obj
 0001:00056311       $stateUnwindMap$?Connect@Plist@@QEAA_NPEB_W00@Z 0000000180057311     Pclass.obj
 0001:00056324       $ip2state$?Connect@Plist@@QEAA_NPEB_W00@Z 0000000180057324     Pclass.obj
 0001:00056334       $unwind$?GetFindData@Plist@@QEAAHAEAPEAUPluginPanelItem@@AEA_K_K@Z 0000000180057334     Pclass.obj
 0001:00056358       $cppxdata$?GetFindData@Plist@@QEAAHAEAPEAUPluginPanelItem@@AEA_K_K@Z 0000000180057358     Pclass.obj
 0001:00056361       $stateUnwindMap$?GetFindData@Plist@@QEAAHAEAPEAUPluginPanelItem@@AEA_K_K@Z 0000000180057361     Pclass.obj
 0001:000563aa       $ip2state$?GetFindData@Plist@@QEAAHAEAPEAUPluginPanelItem@@AEA_K_K@Z 00000001800573aa     Pclass.obj
 0001:000563d8       $unwind$?GetOpenPanelInfo@Plist@@QEAAXPEAUOpenPanelInfo@@@Z 00000001800573d8     Pclass.obj
 0001:000563f0       $unwind$?GetFiles@Plist@@QEAAHPEAUPluginPanelItem@@_KHPEAPEB_W1AEAUoptions@@@Z 00000001800573f0     Pclass.obj
 0001:00056414       $cppxdata$?GetFiles@Plist@@QEAAHPEAUPluginPanelItem@@_KHPEAPEB_W1AEAUoptions@@@Z 0000000180057414     Pclass.obj
 0001:0005641d       $stateUnwindMap$?GetFiles@Plist@@QEAAHPEAUPluginPanelItem@@_KHPEAPEB_W1AEAUoptions@@@Z 000000018005741d     Pclass.obj
 0001:000564ef       $ip2state$?GetFiles@Plist@@QEAAHPEAUPluginPanelItem@@_KHPEAPEB_W1AEAUoptions@@@Z 00000001800574ef     Pclass.obj
 0001:000565a4       $unwind$?DeleteFiles@Plist@@QEAAHPEAUPluginPanelItem@@_K1@Z 00000001800575a4     Pclass.obj
 0001:000565cc       $cppxdata$?DeleteFiles@Plist@@QEAAHPEAUPluginPanelItem@@_K1@Z 00000001800575cc     Pclass.obj
 0001:000565d5       $stateUnwindMap$?DeleteFiles@Plist@@QEAAHPEAUPluginPanelItem@@_K1@Z 00000001800575d5     Pclass.obj
 0001:000565dc       $ip2state$?DeleteFiles@Plist@@QEAAHPEAUPluginPanelItem@@_K1@Z 00000001800575dc     Pclass.obj
 0001:000565ec       $unwind$?ProcessEvent@Plist@@QEAAH_JPEAX@Z 00000001800575ec     Pclass.obj
 0001:0005660c       $cppxdata$?ProcessEvent@Plist@@QEAAH_JPEAX@Z 000000018005760c     Pclass.obj
 0001:00056615       $stateUnwindMap$?ProcessEvent@Plist@@QEAAH_JPEAX@Z 0000000180057615     Pclass.obj
 0001:00056621       $ip2state$?ProcessEvent@Plist@@QEAAH_JPEAX@Z 0000000180057621     Pclass.obj
 0001:0005662c       $unwind$?Compare@Plist@@QEBAHPEBUPluginPanelItem@@0I@Z 000000018005762c     Pclass.obj
 0001:00056650       $cppxdata$?Compare@Plist@@QEBAHPEBUPluginPanelItem@@0I@Z 0000000180057650     Pclass.obj
 0001:00056659       $stateUnwindMap$?Compare@Plist@@QEBAHPEBUPluginPanelItem@@0I@Z 0000000180057659     Pclass.obj
 0001:00056666       $ip2state$?Compare@Plist@@QEBAHPEBUPluginPanelItem@@0I@Z 0000000180057666     Pclass.obj
 0001:00056674       $unwind$?ProcessKey@Plist@@QEAAHPEBU_INPUT_RECORD@@@Z 0000000180057674     Pclass.obj
 0001:00056698       $cppxdata$?ProcessKey@Plist@@QEAAHPEBU_INPUT_RECORD@@@Z 0000000180057698     Pclass.obj
 0001:000566a1       $stateUnwindMap$?ProcessKey@Plist@@QEAAHPEBU_INPUT_RECORD@@@Z 00000001800576a1     Pclass.obj
 0001:000566fc       $ip2state$?ProcessKey@Plist@@QEAAHPEBU_INPUT_RECORD@@@Z 00000001800576fc     Pclass.obj
 0001:00056754       $unwind$?PanelModes@Plist@@QEAAPEAUPanelMode@@AEA_K@Z 0000000180057754     Pclass.obj
 0001:00056764       $chain$2$?PanelModes@Plist@@QEAAPEAUPanelMode@@AEA_K@Z 0000000180057764     Pclass.obj
 0001:00056780       $chain$3$?PanelModes@Plist@@QEAAPEAUPanelMode@@AEA_K@Z 0000000180057780     Pclass.obj
 0001:00056794       $unwind$?GetVersionInfo@Plist@@SA_NPEB_WAEAV?$unique_ptr@$$BY0A@DU?$default_delete@$$BY0A@D@std@@@std@@AEAPEB_W2@Z 0000000180057794     Pclass.obj
 0001:000567bc       $cppxdata$?GetVersionInfo@Plist@@SA_NPEB_WAEAV?$unique_ptr@$$BY0A@DU?$default_delete@$$BY0A@D@std@@@std@@AEAPEB_W2@Z 00000001800577bc     Pclass.obj
 0001:000567c5       $stateUnwindMap$?GetVersionInfo@Plist@@SA_NPEB_WAEAV?$unique_ptr@$$BY0A@DU?$default_delete@$$BY0A@D@std@@@std@@AEAPEB_W2@Z 00000001800577c5     Pclass.obj
 0001:000567d8       $ip2state$?GetVersionInfo@Plist@@SA_NPEB_WAEAV?$unique_ptr@$$BY0A@DU?$default_delete@$$BY0A@D@std@@@std@@AEAPEB_W2@Z 00000001800577d8     Pclass.obj
 0001:000567ec       $unwind$?SavePanelModes@Plist@@SAXXZ 00000001800577ec     Pclass.obj
 0001:00056818       $cppxdata$?SavePanelModes@Plist@@SAXXZ 0000000180057818     Pclass.obj
 0001:00056821       $stateUnwindMap$?SavePanelModes@Plist@@SAXXZ 0000000180057821     Pclass.obj
 0001:00056834       $ip2state$?SavePanelModes@Plist@@SAXXZ 0000000180057834     Pclass.obj
 0001:00056844       $unwind$?InitializePanelModes@Plist@@SAXXZ 0000000180057844     Pclass.obj
 0001:00056868       $cppxdata$?InitializePanelModes@Plist@@SAXXZ 0000000180057868     Pclass.obj
 0001:00056871       $stateUnwindMap$?InitializePanelModes@Plist@@SAXXZ 0000000180057871     Pclass.obj
 0001:0005699c       $ip2state$?InitializePanelModes@Plist@@SAXXZ 000000018005799c     Pclass.obj
 0001:00056a14       $unwind$?PrintVersionInfo@Plist@@CAXPEAXPEB_W@Z 0000000180057a14     Pclass.obj
 0001:00056a38       $cppxdata$?PrintVersionInfo@Plist@@CAXPEAXPEB_W@Z 0000000180057a38     Pclass.obj
 0001:00056a41       $stateUnwindMap$?PrintVersionInfo@Plist@@CAXPEAXPEB_W@Z 0000000180057a41     Pclass.obj
 0001:00056a56       $ip2state$?PrintVersionInfo@Plist@@CAXPEAXPEB_W@Z 0000000180057a56     Pclass.obj
 0001:00056a6c       $unwind$?Reread@Plist@@AEAAXXZ 0000000180057a6c     Pclass.obj
 0001:00056a78       $unwind$?PrintOwnerInfo@Plist@@AEAAXPEAXK@Z 0000000180057a78     Pclass.obj
 0001:00056a9c       $cppxdata$?PrintOwnerInfo@Plist@@AEAAXPEAXK@Z 0000000180057a9c     Pclass.obj
 0001:00056aa5       $stateUnwindMap$?PrintOwnerInfo@Plist@@AEAAXPEAXK@Z 0000000180057aa5     Pclass.obj
 0001:00056ace       $ip2state$?PrintOwnerInfo@Plist@@AEAAXPEAXK@Z 0000000180057ace     Pclass.obj
 0001:00056aec       $unwind$?ConnectWMI@Plist@@AEAA_NXZ 0000000180057aec     Pclass.obj
 0001:00056b08       $cppxdata$?ConnectWMI@Plist@@AEAA_NXZ 0000000180057b08     Pclass.obj
 0001:00056b11       $stateUnwindMap$?ConnectWMI@Plist@@AEAA_NXZ 0000000180057b11     Pclass.obj
 0001:00056b17       $ip2state$?ConnectWMI@Plist@@AEAA_NXZ 0000000180057b17     Pclass.obj
 0001:00056b20       $chain$0$?WmiError@Plist@@AEBAXXZ 0000000180057b20     Pclass.obj
 0001:00056b34       $chain$1$?WmiError@Plist@@AEBAXXZ 0000000180057b34     Pclass.obj
 0001:00056b44       $chain$0$??4?$unique_ptr@VPerfThread@@U?$default_delete@VPerfThread@@@std@@@std@@QEAAAEAV01@$$QEAV01@@Z 0000000180057b44     Pclass.obj
 0001:00056b58       $chain$1$??4?$unique_ptr@VPerfThread@@U?$default_delete@VPerfThread@@@std@@@std@@QEAAAEAV01@$$QEAV01@@Z 0000000180057b58     Pclass.obj
 0001:00056b68       $unwind$?_Clear_and_reserve_geometric@?$vector@Umode@@V?$allocator@Umode@@@std@@@std@@AEAAX_K@Z 0000000180057b68     Pclass.obj
 0001:00056b78       $chain$0$?_Clear_and_reserve_geometric@?$vector@Umode@@V?$allocator@Umode@@@std@@@std@@AEAAX_K@Z 0000000180057b78     Pclass.obj
 0001:00056b8c       $chain$1$?_Clear_and_reserve_geometric@?$vector@Umode@@V?$allocator@Umode@@@std@@@std@@AEAAX_K@Z 0000000180057b8c     Pclass.obj
 0001:00056ba0       $chain$3$?_Clear_and_reserve_geometric@?$vector@Umode@@V?$allocator@Umode@@@std@@@std@@AEAAX_K@Z 0000000180057ba0     Pclass.obj
 0001:00056bb4       $chain$4$?_Clear_and_reserve_geometric@?$vector@Umode@@V?$allocator@Umode@@@std@@@std@@AEAAX_K@Z 0000000180057bb4     Pclass.obj
 0001:00056bc4       $unwind$?DurationToText@@YA?AV?$basic_string@_WU?$char_traits@_W@std@@V?$allocator@_W@2@@std@@_K@Z 0000000180057bc4     Pclass.obj
 0001:00056bdc       $unwind$?ui64toa_width@@YA?AV?$basic_string@_WU?$char_traits@_W@std@@V?$allocator@_W@2@@std@@_KI_N@Z 0000000180057bdc     Pclass.obj
 0001:00056c0c       $cppxdata$?ui64toa_width@@YA?AV?$basic_string@_WU?$char_traits@_W@std@@V?$allocator@_W@2@@std@@_KI_N@Z 0000000180057c0c     Pclass.obj
 0001:00056c15       $stateUnwindMap$?ui64toa_width@@YA?AV?$basic_string@_WU?$char_traits@_W@std@@V?$allocator@_W@2@@std@@_KI_N@Z 0000000180057c15     Pclass.obj
 0001:00056c1c       $ip2state$?ui64toa_width@@YA?AV?$basic_string@_WU?$char_traits@_W@std@@V?$allocator@_W@2@@std@@_KI_N@Z 0000000180057c1c     Pclass.obj
 0001:00056c28       $unwind$?TranslateMode@@YA_NAEBV?$basic_string@_WU?$char_traits@_W@std@@V?$allocator@_W@2@@std@@AEAV12@@Z 0000000180057c28     Pclass.obj
 0001:00056c48       $cppxdata$?TranslateMode@@YA_NAEBV?$basic_string@_WU?$char_traits@_W@std@@V?$allocator@_W@2@@std@@AEAV12@@Z 0000000180057c48     Pclass.obj
 0001:00056c51       $stateUnwindMap$?TranslateMode@@YA_NAEBV?$basic_string@_WU?$char_traits@_W@std@@V?$allocator@_W@2@@std@@AEAV12@@Z 0000000180057c51     Pclass.obj
 0001:00056c51       $stateUnwindMap$?window_ex_style@@YA@PEAUHWND__@@@Z 0000000180057c51     Pclass.obj
 0001:00056c51       $stateUnwindMap$?window_style@@YA@PEAUHWND__@@@Z 0000000180057c51     Pclass.obj
 0001:00056c58       $ip2state$?TranslateMode@@YA_NAEBV?$basic_string@_WU?$char_traits@_W@std@@V?$allocator@_W@2@@std@@AEAV12@@Z 0000000180057c58     Pclass.obj
 0001:00056c64       $unwind$?generate_titles@@YAXAEBV?$basic_string@_WU?$char_traits@_W@std@@V?$allocator@_W@2@@std@@AEAUPanelMode@@@Z 0000000180057c64     Pclass.obj
 0001:00056c84       $cppxdata$?generate_titles@@YAXAEBV?$basic_string@_WU?$char_traits@_W@std@@V?$allocator@_W@2@@std@@AEAUPanelMode@@@Z 0000000180057c84     Pclass.obj
 0001:00056c8d       $stateUnwindMap$?generate_titles@@YAXAEBV?$basic_string@_WU?$char_traits@_W@std@@V?$allocator@_W@2@@std@@AEAUPanelMode@@@Z 0000000180057c8d     Pclass.obj
 0001:00056c94       $ip2state$?generate_titles@@YAXAEBV?$basic_string@_WU?$char_traits@_W@std@@V?$allocator@_W@2@@std@@AEAUPanelMode@@@Z 0000000180057c94     Pclass.obj
 0001:00056c9c       $unwind$?EnumWndProc@@YAHPEAUHWND__@@_J@Z 0000000180057c9c     Pclass.obj
 0001:00056cac       $unwind$??1?$_Hash@V?$_Umap_traits@KPEAUHWND__@@V?$_Uhash_compare@KU?$hash@K@std@@U?$equal_to@K@2@@std@@V?$allocator@U?$pair@$$CBKPEAUHWND__@@@std@@@3@$0A@@std@@@std@@QEAA@XZ 0000000180057cac     Pclass.obj
 0001:00056cac       $unwind$??1?$list@U?$pair@$$CBKPEAUHWND__@@@std@@V?$allocator@U?$pair@$$CBKPEAUHWND__@@@std@@@2@@std@@QEAA@XZ 0000000180057cac     Pclass.obj
 0001:00056cb4       $chain$0$??1?$list@U?$pair@$$CBKPEAUHWND__@@@std@@V?$allocator@U?$pair@$$CBKPEAUHWND__@@@std@@@2@@std@@QEAA@XZ 0000000180057cb4     Pclass.obj
 0001:00056cc8       $chain$1$??1?$list@U?$pair@$$CBKPEAUHWND__@@@std@@V?$allocator@U?$pair@$$CBKPEAUHWND__@@@std@@@2@@std@@QEAA@XZ 0000000180057cc8     Pclass.obj
 0001:00056cd8       $unwind$?_Forced_rehash@?$_Hash@V?$_Umap_traits@KPEAUHWND__@@V?$_Uhash_compare@KU?$hash@K@std@@U?$equal_to@K@2@@std@@V?$allocator@U?$pair@$$CBKPEAUHWND__@@@std@@@3@$0A@@std@@@std@@IEAAX_K@Z 0000000180057cd8     Pclass.obj
 0001:00056ce4       $chain$1$?_Forced_rehash@?$_Hash@V?$_Umap_traits@KPEAUHWND__@@V?$_Uhash_compare@KU?$hash@K@std@@U?$equal_to@K@2@@std@@V?$allocator@U?$pair@$$CBKPEAUHWND__@@@std@@@3@$0A@@std@@@std@@IEAAX_K@Z 0000000180057ce4     Pclass.obj
 0001:00056cfc       $chain$2$?_Forced_rehash@?$_Hash@V?$_Umap_traits@KPEAUHWND__@@V?$_Uhash_compare@KU?$hash@K@std@@U?$equal_to@K@2@@std@@V?$allocator@U?$pair@$$CBKPEAUHWND__@@@std@@@3@$0A@@std@@@std@@IEAAX_K@Z 0000000180057cfc     Pclass.obj
 0001:00056d10       $chain$3$?_Forced_rehash@?$_Hash@V?$_Umap_traits@KPEAUHWND__@@V?$_Uhash_compare@KU?$hash@K@std@@U?$equal_to@K@2@@std@@V?$allocator@U?$pair@$$CBKPEAUHWND__@@@std@@@3@$0A@@std@@@std@@IEAAX_K@Z 0000000180057d10     Pclass.obj
 0001:00056d20       $chain$5$?_Forced_rehash@?$_Hash@V?$_Umap_traits@KPEAUHWND__@@V?$_Uhash_compare@KU?$hash@K@std@@U?$equal_to@K@2@@std@@V?$allocator@U?$pair@$$CBKPEAUHWND__@@@std@@@3@$0A@@std@@@std@@IEAAX_K@Z 0000000180057d20     Pclass.obj
 0001:00056d3c       $chain$6$?_Forced_rehash@?$_Hash@V?$_Umap_traits@KPEAUHWND__@@V?$_Uhash_compare@KU?$hash@K@std@@U?$equal_to@K@2@@std@@V?$allocator@U?$pair@$$CBKPEAUHWND__@@@std@@@3@$0A@@std@@@std@@IEAAX_K@Z 0000000180057d3c     Pclass.obj
 0001:00056d4c       $unwind$?_Assign_grow@?$_Hash_vec@V?$allocator@V?$_List_unchecked_iterator@V?$_List_val@U?$_List_simple_types@U?$pair@$$CBKPEAUHWND__@@@std@@@std@@@std@@@std@@@std@@@std@@QEAAX_KV?$_List_unchecked_iterator@V?$_List_val@U?$_List_simple_types@U?$pair@$$CBKPEAUHWND__@@@std@@@std@@@std@@@2@@Z 0000000180057d4c     Pclass.obj
 0001:00056d58       $chain$1$?_Assign_grow@?$_Hash_vec@V?$allocator@V?$_List_unchecked_iterator@V?$_List_val@U?$_List_simple_types@U?$pair@$$CBKPEAUHWND__@@@std@@@std@@@std@@@std@@@std@@@std@@QEAAX_KV?$_List_unchecked_iterator@V?$_List_val@U?$_List_simple_types@U?$pair@$$CBKPEAUHWND__@@@std@@@std@@@std@@@2@@Z 0000000180057d58     Pclass.obj
 0001:00056d70       $chain$2$?_Assign_grow@?$_Hash_vec@V?$allocator@V?$_List_unchecked_iterator@V?$_List_val@U?$_List_simple_types@U?$pair@$$CBKPEAUHWND__@@@std@@@std@@@std@@@std@@@std@@@std@@QEAAX_KV?$_List_unchecked_iterator@V?$_List_val@U?$_List_simple_types@U?$pair@$$CBKPEAUHWND__@@@std@@@std@@@std@@@2@@Z 0000000180057d70     Pclass.obj
 0001:00056d80       $chain$3$?_Assign_grow@?$_Hash_vec@V?$allocator@V?$_List_unchecked_iterator@V?$_List_val@U?$_List_simple_types@U?$pair@$$CBKPEAUHWND__@@@std@@@std@@@std@@@std@@@std@@@std@@QEAAX_KV?$_List_unchecked_iterator@V?$_List_val@U?$_List_simple_types@U?$pair@$$CBKPEAUHWND__@@@std@@@std@@@std@@@2@@Z 0000000180057d80     Pclass.obj
 0001:00056d98       $chain$0$??1?$_Hash@V?$_Umap_traits@KPEAUHWND__@@V?$_Uhash_compare@KU?$hash@K@std@@U?$equal_to@K@2@@std@@V?$allocator@U?$pair@$$CBKPEAUHWND__@@@std@@@3@$0A@@std@@@std@@QEAA@XZ 0000000180057d98     Pclass.obj
 0001:00056dac       $chain$1$??1?$_Hash@V?$_Umap_traits@KPEAUHWND__@@V?$_Uhash_compare@KU?$hash@K@std@@U?$equal_to@K@2@@std@@V?$allocator@U?$pair@$$CBKPEAUHWND__@@@std@@@3@$0A@@std@@@std@@QEAA@XZ 0000000180057dac     Pclass.obj
 0001:00056dbc       $unwind$?_Destroy@?$vector@V?$basic_string@_WU?$char_traits@_W@std@@V?$allocator@_W@2@@std@@V?$allocator@V?$basic_string@_WU?$char_traits@_W@std@@V?$allocator@_W@2@@std@@@2@@std@@AEAAXPEAV?$basic_string@_WU?$char_traits@_W@std@@V?$allocator@_W@2@@2@0@Z 0000000180057dbc     Pclass.obj
 0001:00056dbc       $unwind$??$free_environment@D@@YAXQEAPEAD@Z 0000000180057dbc     libucrt:environment_initialization.obj
 0001:00056dbc       $unwind$??$free_environment@_W@@YAXQEAPEA_W@Z 0000000180057dbc     libucrt:environment_initialization.obj
 0001:00056dc8       $chain$0$?_Tidy@?$vector@V?$basic_string@_WU?$char_traits@_W@std@@V?$allocator@_W@2@@std@@V?$allocator@V?$basic_string@_WU?$char_traits@_W@std@@V?$allocator@_W@2@@std@@@2@@std@@AEAAXXZ 0000000180057dc8     Pclass.obj
 0001:00056ddc       $chain$1$?_Tidy@?$vector@V?$basic_string@_WU?$char_traits@_W@std@@V?$allocator@_W@2@@std@@V?$allocator@V?$basic_string@_WU?$char_traits@_W@std@@V?$allocator@_W@2@@std@@@2@@std@@AEAAXXZ 0000000180057ddc     Pclass.obj
 0001:00056dec       $unwind$??$_Emplace_reallocate@V?$basic_string@_WU?$char_traits@_W@std@@V?$allocator@_W@2@@std@@@?$vector@V?$basic_string@_WU?$char_traits@_W@std@@V?$allocator@_W@2@@std@@V?$allocator@V?$basic_string@_WU?$char_traits@_W@std@@V?$allocator@_W@2@@std@@@2@@std@@QEAAPEAV?$basic_string@_WU?$char_traits@_W@std@@V?$allocator@_W@2@@1@QEAV21@$$QEAV21@@Z 0000000180057dec     Pclass.obj
 0001:00056e08       $cppxdata$??$_Emplace_reallocate@V?$basic_string@_WU?$char_traits@_W@std@@V?$allocator@_W@2@@std@@@?$vector@V?$basic_string@_WU?$char_traits@_W@std@@V?$allocator@_W@2@@std@@V?$allocator@V?$basic_string@_WU?$char_traits@_W@std@@V?$allocator@_W@2@@std@@@2@@std@@QEAAPEAV?$basic_string@_WU?$char_traits@_W@std@@V?$allocator@_W@2@@1@QEAV21@$$QEAV21@@Z 0000000180057e08     Pclass.obj
 0001:00056e15       $stateUnwindMap$??$_Emplace_reallocate@V?$basic_string@_WU?$char_traits@_W@std@@V?$allocator@_W@2@@std@@@?$vector@V?$basic_string@_WU?$char_traits@_W@std@@V?$allocator@_W@2@@std@@V?$allocator@V?$basic_string@_WU?$char_traits@_W@std@@V?$allocator@_W@2@@std@@@2@@std@@QEAAPEAV?$basic_string@_WU?$char_traits@_W@std@@V?$allocator@_W@2@@1@QEAV21@$$QEAV21@@Z 0000000180057e15     Pclass.obj
 0001:00056e15       $stateUnwindMap$??$_Resize_reallocate@U_Value_init_tag@std@@@?$vector@PEB_WV?$allocator@PEB_W@std@@@std@@AEAAX_KAEBU_Value_init_tag@1@@Z 0000000180057e15     Pclass.obj
 0001:00056e15       $stateUnwindMap$??$_Resize_reallocate@U_Value_init_tag@std@@@?$vector@PEAUHINSTANCE__@@V?$allocator@PEAUHINSTANCE__@@@std@@@std@@AEAAX_KAEBU_Value_init_tag@1@@Z 0000000180057e15     Plist.obj
 0001:00056e15       $stateUnwindMap$??$_Resize_reallocate@U_Value_init_tag@std@@@?$vector@EV?$allocator@E@std@@@std@@AEAAX_KAEBU_Value_init_tag@1@@Z 0000000180057e15     perfthread.obj
 0001:00056e18       $tryMap$??$_Emplace_reallocate@V?$basic_string@_WU?$char_traits@_W@std@@V?$allocator@_W@2@@std@@@?$vector@V?$basic_string@_WU?$char_traits@_W@std@@V?$allocator@_W@2@@std@@V?$allocator@V?$basic_string@_WU?$char_traits@_W@std@@V?$allocator@_W@2@@std@@@2@@std@@QEAAPEAV?$basic_string@_WU?$char_traits@_W@std@@V?$allocator@_W@2@@1@QEAV21@$$QEAV21@@Z 0000000180057e18     Pclass.obj
 0001:00056e20       $handlerMap$??$_Emplace_reallocate@V?$basic_string@_WU?$char_traits@_W@std@@V?$allocator@_W@2@@std@@@?$vector@V?$basic_string@_WU?$char_traits@_W@std@@V?$allocator@_W@2@@std@@V?$allocator@V?$basic_string@_WU?$char_traits@_W@std@@V?$allocator@_W@2@@std@@@2@@std@@QEAAPEAV?$basic_string@_WU?$char_traits@_W@std@@V?$allocator@_W@2@@1@QEAV21@$$QEAV21@@Z 0000000180057e20     Pclass.obj
 0001:00056e27       $ip2state$??$_Emplace_reallocate@V?$basic_string@_WU?$char_traits@_W@std@@V?$allocator@_W@2@@std@@@?$vector@V?$basic_string@_WU?$char_traits@_W@std@@V?$allocator@_W@2@@std@@V?$allocator@V?$basic_string@_WU?$char_traits@_W@std@@V?$allocator@_W@2@@std@@@2@@std@@QEAAPEAV?$basic_string@_WU?$char_traits@_W@std@@V?$allocator@_W@2@@1@QEAV21@$$QEAV21@@Z 0000000180057e27     Pclass.obj
 0001:00056e30       $unwind$?catch$8@?0???$_Emplace_reallocate@V?$basic_string@_WU?$char_traits@_W@std@@V?$allocator@_W@2@@std@@@?$vector@V?$basic_string@_WU?$char_traits@_W@std@@V?$allocator@_W@2@@std@@V?$allocator@V?$basic_string@_WU?$char_traits@_W@std@@V?$allocator@_W@2@@std@@@2@@std@@QEAAPEAV?$basic_string@_WU?$char_traits@_W@std@@V?$allocator@_W@2@@1@QEAV21@$$QEAV21@@Z@4HA 0000000180057e30     Pclass.obj
 0001:00056e3c       $unwind$?window_style@@YA@PEAUHWND__@@@Z 0000000180057e3c     Pclass.obj
 0001:00056e60       $cppxdata$?window_style@@YA@PEAUHWND__@@@Z 0000000180057e60     Pclass.obj
 0001:00056e69       $ip2state$?window_style@@YA@PEAUHWND__@@@Z 0000000180057e69     Pclass.obj
 0001:00056e74       $unwind$?window_ex_style@@YA@PEAUHWND__@@@Z 0000000180057e74     Pclass.obj
 0001:00056e98       $cppxdata$?window_ex_style@@YA@PEAUHWND__@@@Z 0000000180057e98     Pclass.obj
 0001:00056ea1       $ip2state$?window_ex_style@@YA@PEAUHWND__@@@Z 0000000180057ea1     Pclass.obj
 0001:00056eac       $unwind$?DumpNTCounters@@YAXPEAXAEAVPerfThread@@KK@Z 0000000180057eac     Pclass.obj
 0001:00056ed4       $cppxdata$?DumpNTCounters@@YAXPEAXAEAVPerfThread@@KK@Z 0000000180057ed4     Pclass.obj
 0001:00056edd       $stateUnwindMap$?DumpNTCounters@@YAXPEAXAEAVPerfThread@@KK@Z 0000000180057edd     Pclass.obj
 0001:00056f0a       $ip2state$?DumpNTCounters@@YAXPEAXAEAVPerfThread@@KK@Z 0000000180057f0a     Pclass.obj
 0001:00056f30       $unwind$??$_Try_emplace@AEBK$$V@?$_Hash@V?$_Umap_traits@KPEAUHWND__@@V?$_Uhash_compare@KU?$hash@K@std@@U?$equal_to@K@2@@std@@V?$allocator@U?$pair@$$CBKPEAUHWND__@@@std@@@3@$0A@@std@@@std@@IEAA?AU?$pair@PEAU?$_List_node@U?$pair@$$CBKPEAUHWND__@@@std@@PEAX@std@@_N@1@AEBK@Z 0000000180057f30     Pclass.obj
 0001:00056f54       $cppxdata$??$_Try_emplace@AEBK$$V@?$_Hash@V?$_Umap_traits@KPEAUHWND__@@V?$_Uhash_compare@KU?$hash@K@std@@U?$equal_to@K@2@@std@@V?$allocator@U?$pair@$$CBKPEAUHWND__@@@std@@@3@$0A@@std@@@std@@IEAA?AU?$pair@PEAU?$_List_node@U?$pair@$$CBKPEAUHWND__@@@std@@PEAX@std@@_N@1@AEBK@Z 0000000180057f54     Pclass.obj
 0001:00056f5d       $stateUnwindMap$??$_Try_emplace@AEBK$$V@?$_Hash@V?$_Umap_traits@KPEAUHWND__@@V?$_Uhash_compare@KU?$hash@K@std@@U?$equal_to@K@2@@std@@V?$allocator@U?$pair@$$CBKPEAUHWND__@@@std@@@3@$0A@@std@@@std@@IEAA?AU?$pair@PEAU?$_List_node@U?$pair@$$CBKPEAUHWND__@@@std@@PEAX@std@@_N@1@AEBK@Z 0000000180057f5d     Pclass.obj
 0001:00056f6a       $ip2state$??$_Try_emplace@AEBK$$V@?$_Hash@V?$_Umap_traits@KPEAUHWND__@@V?$_Uhash_compare@KU?$hash@K@std@@U?$equal_to@K@2@@std@@V?$allocator@U?$pair@$$CBKPEAUHWND__@@@std@@@3@$0A@@std@@@std@@IEAA?AU?$pair@PEAU?$_List_node@U?$pair@$$CBKPEAUHWND__@@@std@@PEAX@std@@_N@1@AEBK@Z 0000000180057f6a     Pclass.obj
 0001:00056f74       $unwind$??$_Assign_range@PEBUmode@@@?$vector@Umode@@V?$allocator@Umode@@@std@@@std@@AEAAXPEBUmode@@0Uforward_iterator_tag@1@@Z 0000000180057f74     Pclass.obj
 0001:00056f90       $cppxdata$??$_Assign_range@PEBUmode@@@?$vector@Umode@@V?$allocator@Umode@@@std@@@std@@AEAAXPEBUmode@@0Uforward_iterator_tag@1@@Z 0000000180057f90     Pclass.obj
 0001:00056f99       $stateUnwindMap$??$_Assign_range@PEBUmode@@@?$vector@Umode@@V?$allocator@Umode@@@std@@@std@@AEAAXPEBUmode@@0Uforward_iterator_tag@1@@Z 0000000180057f99     Pclass.obj
 0001:00056fbc       $ip2state$??$_Assign_range@PEBUmode@@@?$vector@Umode@@V?$allocator@Umode@@@std@@@std@@AEAAXPEBUmode@@0Uforward_iterator_tag@1@@Z 0000000180057fbc     Pclass.obj
 0001:00056fd0       $unwind$??$_Reallocate_grow_by@V<lambda_51c4cb9729979bd953fe6d1bff5c73b0>@@_K_K_W@?$basic_string@_WU?$char_traits@_W@std@@V?$allocator@_W@2@@std@@AEAAAEAV01@_KV<lambda_51c4cb9729979bd953fe6d1bff5c73b0>@@_K2_W@Z 0000000180057fd0     Pclass.obj
 0001:00056fe0       $chain$3$??$_Reallocate_grow_by@V<lambda_51c4cb9729979bd953fe6d1bff5c73b0>@@_K_K_W@?$basic_string@_WU?$char_traits@_W@std@@V?$allocator@_W@2@@std@@AEAAAEAV01@_KV<lambda_51c4cb9729979bd953fe6d1bff5c73b0>@@_K2_W@Z 0000000180057fe0     Pclass.obj
 0001:00057000       $chain$5$??$_Reallocate_grow_by@V<lambda_51c4cb9729979bd953fe6d1bff5c73b0>@@_K_K_W@?$basic_string@_WU?$char_traits@_W@std@@V?$allocator@_W@2@@std@@AEAAAEAV01@_KV<lambda_51c4cb9729979bd953fe6d1bff5c73b0>@@_K2_W@Z 0000000180058000     Pclass.obj
 0001:00057020       $chain$6$??$_Reallocate_grow_by@V<lambda_51c4cb9729979bd953fe6d1bff5c73b0>@@_K_K_W@?$basic_string@_WU?$char_traits@_W@std@@V?$allocator@_W@2@@std@@AEAAAEAV01@_KV<lambda_51c4cb9729979bd953fe6d1bff5c73b0>@@_K2_W@Z 0000000180058020     Pclass.obj
 0001:00057030       $unwind$??$_Reallocate_grow_by@V<lambda_967c2ed818824c5314a20ec3af46b793>@@_KPEB_W_K@?$basic_string@_WU?$char_traits@_W@std@@V?$allocator@_W@2@@std@@AEAAAEAV01@_KV<lambda_967c2ed818824c5314a20ec3af46b793>@@_KPEB_W2@Z 0000000180058030     Pclass.obj
 0001:00057040       $chain$3$??$_Reallocate_grow_by@V<lambda_967c2ed818824c5314a20ec3af46b793>@@_KPEB_W_K@?$basic_string@_WU?$char_traits@_W@std@@V?$allocator@_W@2@@std@@AEAAAEAV01@_KV<lambda_967c2ed818824c5314a20ec3af46b793>@@_KPEB_W2@Z 0000000180058040     Pclass.obj
 0001:00057060       $chain$5$??$_Reallocate_grow_by@V<lambda_967c2ed818824c5314a20ec3af46b793>@@_KPEB_W_K@?$basic_string@_WU?$char_traits@_W@std@@V?$allocator@_W@2@@std@@AEAAAEAV01@_KV<lambda_967c2ed818824c5314a20ec3af46b793>@@_KPEB_W2@Z 0000000180058060     Pclass.obj
 0001:00057080       $chain$6$??$_Reallocate_grow_by@V<lambda_967c2ed818824c5314a20ec3af46b793>@@_KPEB_W_K@?$basic_string@_WU?$char_traits@_W@std@@V?$allocator@_W@2@@std@@AEAAAEAV01@_KV<lambda_967c2ed818824c5314a20ec3af46b793>@@_KPEB_W2@Z 0000000180058080     Pclass.obj
 0001:00057090       $unwind$??$fill@PEAV?$_List_unchecked_iterator@V?$_List_val@U?$_List_simple_types@U?$pair@$$CBKPEAUHWND__@@@std@@@std@@@std@@@std@@V12@@std@@YAXQEAV?$_List_unchecked_iterator@V?$_List_val@U?$_List_simple_types@U?$pair@$$CBKPEAUHWND__@@@std@@@std@@@std@@@0@0AEBV10@@Z 0000000180058090     Pclass.obj
 0001:00057098       $chain$0$??$fill@PEAV?$_List_unchecked_iterator@V?$_List_val@U?$_List_simple_types@U?$pair@$$CBKPEAUHWND__@@@std@@@std@@@std@@@std@@V12@@std@@YAXQEAV?$_List_unchecked_iterator@V?$_List_val@U?$_List_simple_types@U?$pair@$$CBKPEAUHWND__@@@std@@@std@@@std@@@0@0AEBV10@@Z 0000000180058098     Pclass.obj
 0001:000570ac       $chain$1$??$fill@PEAV?$_List_unchecked_iterator@V?$_List_val@U?$_List_simple_types@U?$pair@$$CBKPEAUHWND__@@@std@@@std@@@std@@@std@@V12@@std@@YAXQEAV?$_List_unchecked_iterator@V?$_List_val@U?$_List_simple_types@U?$pair@$$CBKPEAUHWND__@@@std@@@std@@@std@@@0@0AEBV10@@Z 00000001800580ac     Pclass.obj
 0001:000570bc       $unwind$??$_Resize_reallocate@U_Value_init_tag@std@@@?$vector@PEB_WV?$allocator@PEB_W@std@@@std@@AEAAX_KAEBU_Value_init_tag@1@@Z 00000001800580bc     Pclass.obj
 0001:000570d4       $cppxdata$??$_Resize_reallocate@U_Value_init_tag@std@@@?$vector@PEB_WV?$allocator@PEB_W@std@@@std@@AEAAX_KAEBU_Value_init_tag@1@@Z 00000001800580d4     Pclass.obj
 0001:000570e1       $tryMap$??$_Resize_reallocate@U_Value_init_tag@std@@@?$vector@PEB_WV?$allocator@PEB_W@std@@@std@@AEAAX_KAEBU_Value_init_tag@1@@Z 00000001800580e1     Pclass.obj
 0001:000570e9       $handlerMap$??$_Resize_reallocate@U_Value_init_tag@std@@@?$vector@PEB_WV?$allocator@PEB_W@std@@@std@@AEAAX_KAEBU_Value_init_tag@1@@Z 00000001800580e9     Pclass.obj
 0001:000570f0       $ip2state$??$_Resize_reallocate@U_Value_init_tag@std@@@?$vector@PEB_WV?$allocator@PEB_W@std@@@std@@AEAAX_KAEBU_Value_init_tag@1@@Z 00000001800580f0     Pclass.obj
 0001:000570fc       $unwind$?catch$0@?0???$_Resize_reallocate@U_Value_init_tag@std@@@?$vector@PEB_WV?$allocator@PEB_W@std@@@std@@AEAAX_KAEBU_Value_init_tag@1@@Z@4HA 00000001800580fc     Pclass.obj
 0001:000570fc       $unwind$?catch$0@?0???$_Resize_reallocate@U_Value_init_tag@std@@@?$vector@PEAUHINSTANCE__@@V?$allocator@PEAUHINSTANCE__@@@std@@@std@@AEAAX_KAEBU_Value_init_tag@1@@Z@4HA 00000001800580fc     Plist.obj
 0001:000570fc       $unwind$?catch$0@?0???$_Resize_reallocate@U_Value_init_tag@std@@@?$vector@EV?$allocator@E@std@@@std@@AEAAX_KAEBU_Value_init_tag@1@@Z@4HA 00000001800580fc     perfthread.obj
 0001:00057104       $unwind$??0PerfThread@@QEAA@PEB_W00@Z 0000000180058104     perfthread.obj
 0001:00057128       $cppxdata$??0PerfThread@@QEAA@PEB_W00@Z 0000000180058128     perfthread.obj
 0001:00057131       $stateUnwindMap$??0PerfThread@@QEAA@PEB_W00@Z 0000000180058131     perfthread.obj
 0001:0005717c       $ip2state$??0PerfThread@@QEAA@PEB_W00@Z 000000018005817c     perfthread.obj
 0001:00057190       $unwind$?GetProcessData@PerfThread@@QEAAPEAUProcessPerfData@@KK@Z 0000000180058190     perfthread.obj
 0001:0005719c       $chain$0$?GetProcessData@PerfThread@@QEAAPEAUProcessPerfData@@KK@Z 000000018005819c     perfthread.obj
 0001:000571b0       $chain$1$?GetProcessData@PerfThread@@QEAAPEAUProcessPerfData@@KK@Z 00000001800581b0     perfthread.obj
 0001:000571c0       $unwind$?ThreadProc@PerfThread@@CAKPEAX@Z 00000001800581c0     perfthread.obj
 0001:000571c0       $unwind$parse_bcp47_language 00000001800581c0     libucrt:wsetlocale.obj
 0001:000571c0       $unwind$parse_bcp47_script 00000001800581c0     libucrt:wsetlocale.obj
 0001:000571cc       $unwind$?Refresh@PerfThread@@AEAAXXZ 00000001800581cc     perfthread.obj
 0001:000571ec       $cppxdata$?Refresh@PerfThread@@AEAAXXZ 00000001800581ec     perfthread.obj
 0001:000571f5       $stateUnwindMap$?Refresh@PerfThread@@AEAAXXZ 00000001800581f5     perfthread.obj
 0001:00057216       $ip2state$?Refresh@PerfThread@@AEAAXXZ 0000000180058216     perfthread.obj
 0001:00057230       $unwind$?RefreshWMIData@PerfThread@@AEAAXXZ 0000000180058230     perfthread.obj
 0001:00057254       $cppxdata$?RefreshWMIData@PerfThread@@AEAAXXZ 0000000180058254     perfthread.obj
 0001:0005725d       $stateUnwindMap$?RefreshWMIData@PerfThread@@AEAAXXZ 000000018005825d     perfthread.obj
 0001:00057264       $ip2state$?RefreshWMIData@PerfThread@@AEAAXXZ 0000000180058264     perfthread.obj
 0001:0005726c       $chain$0$?_Tidy@?$vector@UProcessPerfData@@V?$allocator@UProcessPerfData@@@std@@@std@@AEAAXXZ 000000018005826c     perfthread.obj
 0001:00057280       $chain$1$?_Tidy@?$vector@UProcessPerfData@@V?$allocator@UProcessPerfData@@@std@@@std@@AEAAXXZ 0000000180058280     perfthread.obj
 0001:00057290       $unwind$??$_Construct_n_copies_of_ty@U_Value_init_tag@std@@@?$vector@UProcessPerfData@@V?$allocator@UProcessPerfData@@@std@@@std@@AEAAX_KAEBU_Value_init_tag@1@@Z 0000000180058290     perfthread.obj
 0001:0005729c       $chain$2$??$_Construct_n_copies_of_ty@U_Value_init_tag@std@@@?$vector@UProcessPerfData@@V?$allocator@UProcessPerfData@@@std@@@std@@AEAAX_KAEBU_Value_init_tag@1@@Z 000000018005829c     perfthread.obj
 0001:000572b8       $chain$3$??$_Construct_n_copies_of_ty@U_Value_init_tag@std@@@?$vector@UProcessPerfData@@V?$allocator@UProcessPerfData@@@std@@@std@@AEAAX_KAEBU_Value_init_tag@1@@Z 00000001800582b8     perfthread.obj
 0001:000572cc       $chain$4$??$_Construct_n_copies_of_ty@U_Value_init_tag@std@@@?$vector@UProcessPerfData@@V?$allocator@UProcessPerfData@@@std@@@std@@AEAAX_KAEBU_Value_init_tag@1@@Z 00000001800582cc     perfthread.obj
 0001:000572cc       $chain$6$??$_Construct_n_copies_of_ty@U_Value_init_tag@std@@@?$vector@UProcessPerfData@@V?$allocator@UProcessPerfData@@@std@@@std@@AEAAX_KAEBU_Value_init_tag@1@@Z 00000001800582cc     perfthread.obj
 0001:000572e8       $chain$5$??$_Construct_n_copies_of_ty@U_Value_init_tag@std@@@?$vector@UProcessPerfData@@V?$allocator@UProcessPerfData@@@std@@@std@@AEAAX_KAEBU_Value_init_tag@1@@Z 00000001800582e8     perfthread.obj
 0001:000572f8       $unwind$??$_Resize_reallocate@U_Value_init_tag@std@@@?$vector@EV?$allocator@E@std@@@std@@AEAAX_KAEBU_Value_init_tag@1@@Z 00000001800582f8     perfthread.obj
 0001:00057310       $cppxdata$??$_Resize_reallocate@U_Value_init_tag@std@@@?$vector@EV?$allocator@E@std@@@std@@AEAAX_KAEBU_Value_init_tag@1@@Z 0000000180058310     perfthread.obj
 0001:0005731d       $tryMap$??$_Resize_reallocate@U_Value_init_tag@std@@@?$vector@EV?$allocator@E@std@@@std@@AEAAX_KAEBU_Value_init_tag@1@@Z 000000018005831d     perfthread.obj
 0001:00057325       $handlerMap$??$_Resize_reallocate@U_Value_init_tag@std@@@?$vector@EV?$allocator@E@std@@@std@@AEAAX_KAEBU_Value_init_tag@1@@Z 0000000180058325     perfthread.obj
 0001:0005732c       $ip2state$??$_Resize_reallocate@U_Value_init_tag@std@@@?$vector@EV?$allocator@E@std@@@std@@AEAAX_KAEBU_Value_init_tag@1@@Z 000000018005832c     perfthread.obj
 0001:00057334       $unwind$?GetList@@YA_NAEAPEAUPluginPanelItem@@AEA_KAEAVPerfThread@@@Z 0000000180058334     Plist.obj
 0001:00057354       $cppxdata$?GetList@@YA_NAEAPEAUPluginPanelItem@@AEA_KAEAVPerfThread@@@Z 0000000180058354     Plist.obj
 0001:0005735d       $stateUnwindMap$?GetList@@YA_NAEAPEAUPluginPanelItem@@AEA_KAEAVPerfThread@@@Z 000000018005835d     Plist.obj
 0001:00057364       $ip2state$?GetList@@YA_NAEAPEAUPluginPanelItem@@AEA_KAEAVPerfThread@@@Z 0000000180058364     Plist.obj
 0001:0005736c       $unwind$?KillProcess@@YA_NKPEAUHWND__@@@Z 000000018005836c     Plist.obj
 0001:00057388       $cppxdata$?KillProcess@@YA_NKPEAUHWND__@@@Z 0000000180058388     Plist.obj
 0001:00057391       $stateUnwindMap$?KillProcess@@YA_NKPEAUHWND__@@@Z 0000000180058391     Plist.obj
 0001:0005739f       $ip2state$?KillProcess@@YA_NKPEAUHWND__@@@Z 000000018005839f     Plist.obj
 0001:000573a8       $chain$1$?CreateToken@DebugToken@@SA_NXZ 00000001800583a8     Plist.obj
 0001:000573c0       $chain$2$?CreateToken@DebugToken@@SA_NXZ 00000001800583c0     Plist.obj
 0001:000573d4       $unwind$?PrintNTCurDirAndEnv@@YAXPEAX0H@Z 00000001800583d4     Plist.obj
 0001:000573fc       $cppxdata$?PrintNTCurDirAndEnv@@YAXPEAX0H@Z 00000001800583fc     Plist.obj
 0001:00057405       $stateUnwindMap$?PrintNTCurDirAndEnv@@YAXPEAX0H@Z 0000000180058405     Plist.obj
 0001:00057421       $ip2state$?PrintNTCurDirAndEnv@@YAXPEAX0H@Z 0000000180058421     Plist.obj
 0001:00057434       $unwind$?PrintModules@@YAXPEAXKAEAUoptions@@@Z 0000000180058434     Plist.obj
 0001:00057460       $cppxdata$?PrintModules@@YAXPEAXKAEAUoptions@@@Z 0000000180058460     Plist.obj
 0001:00057469       $stateUnwindMap$?PrintModules@@YAXPEAXKAEAUoptions@@@Z 0000000180058469     Plist.obj
 0001:00057483       $ip2state$?PrintModules@@YAXPEAXKAEAUoptions@@@Z 0000000180058483     Plist.obj
 0001:00057498       $unwind$?GetPData@@YA_NAEAUProcessData@@AEBUProcessPerfData@@@Z 0000000180058498     Plist.obj
 0001:000574ac       $chain$1$?GetPData@@YA_NAEAUProcessData@@AEBUProcessPerfData@@@Z 00000001800584ac     Plist.obj
 0001:000574c4       $chain$3$?GetPData@@YA_NAEAUProcessData@@AEBUProcessPerfData@@@Z 00000001800584c4     Plist.obj
 0001:000574dc       $chain$4$?GetPData@@YA_NAEAUProcessData@@AEBUProcessPerfData@@@Z 00000001800584dc     Plist.obj
 0001:000574ec       $unwind$??0?$vector@UProcessPerfData@@V?$allocator@UProcessPerfData@@@std@@@std@@QEAA@AEBV01@@Z 00000001800584ec     Plist.obj
 0001:00057508       $cppxdata$??0?$vector@UProcessPerfData@@V?$allocator@UProcessPerfData@@@std@@@std@@QEAA@AEBV01@@Z 0000000180058508     Plist.obj
 0001:00057511       $stateUnwindMap$??0?$vector@UProcessPerfData@@V?$allocator@UProcessPerfData@@@std@@@std@@QEAA@AEBV01@@Z 0000000180058511     Plist.obj
 0001:0005752d       $ip2state$??0?$vector@UProcessPerfData@@V?$allocator@UProcessPerfData@@@std@@@std@@QEAA@AEBV01@@Z 000000018005852d     Plist.obj
 0001:00057540       $unwind$?FreeUserData@@YAXQEAXQEBUFarPanelItemFreeInfo@@@Z 0000000180058540     Plist.obj
 0001:00057540       $unwind$_free_base         0000000180058540     libucrt:free_base.obj
 0001:00057540       $unwind$?destroy_fls@@YAXPEAX@Z 0000000180058540     libucrt:per_thread_data.obj
 0001:00057540       $unwind$__acrt_locale_free_numeric 0000000180058540     libucrt:initnum.obj
 0001:00057540       $unwind$__acrt_locale_free_lc_time_if_unreferenced 0000000180058540     libucrt:locale_refcounting.obj
 0001:00057548       $unwind$?read_string@?$ipc_functions@$0A@@@SA?AV?$basic_string@_WU?$char_traits@_W@std@@V?$allocator@_W@2@@std@@PEAXAEBUUNICODE_STRING_SAME@detail@@@Z 0000000180058548     Plist.obj
 0001:0005755c       $unwind$?GetOpenProcessData@?$ipc_functions@$0A@@@SAXPEAXPEAV?$basic_string@_WU?$char_traits@_W@std@@V?$allocator@_W@2@@std@@1111@Z 000000018005855c     Plist.obj
 0001:00057578       $chain$0$?GetOpenProcessData@?$ipc_functions@$0A@@@SAXPEAXPEAV?$basic_string@_WU?$char_traits@_W@std@@V?$allocator@_W@2@@std@@1111@Z 0000000180058578     Plist.obj
 0001:0005758c       $chain$1$?GetOpenProcessData@?$ipc_functions@$0A@@@SAXPEAXPEAV?$basic_string@_WU?$char_traits@_W@std@@V?$allocator@_W@2@@std@@1111@Z 000000018005858c     Plist.obj
 0001:0005759c       $chain$2$?GetOpenProcessData@?$ipc_functions@$0A@@@SAXPEAXPEAV?$basic_string@_WU?$char_traits@_W@std@@V?$allocator@_W@2@@std@@1111@Z 000000018005859c     Plist.obj
 0001:000575b0       $unwind$?print_module_impl@@YAXQEAXAEBV?$basic_string@_WU?$char_traits@_W@std@@V?$allocator@_W@2@@std@@KAEBUoptions@@AEBV?$function@$$A6A_NPEA_W_K@Z@2@@Z 00000001800585b0     Plist.obj
 0001:000575d0       $cppxdata$?print_module_impl@@YAXQEAXAEBV?$basic_string@_WU?$char_traits@_W@std@@V?$allocator@_W@2@@std@@KAEBUoptions@@AEBV?$function@$$A6A_NPEA_W_K@Z@2@@Z 00000001800585d0     Plist.obj
 0001:000575d9       $stateUnwindMap$?print_module_impl@@YAXQEAXAEBV?$basic_string@_WU?$char_traits@_W@std@@V?$allocator@_W@2@@std@@KAEBUoptions@@AEBV?$function@$$A6A_NPEA_W_K@Z@2@@Z 00000001800585d9     Plist.obj
 0001:000575ed       $ip2state$?print_module_impl@@YAXQEAXAEBV?$basic_string@_WU?$char_traits@_W@std@@V?$allocator@_W@2@@std@@KAEBUoptions@@AEBV?$function@$$A6A_NPEA_W_K@Z@2@@Z 00000001800585ed     Plist.obj
 0001:00057600       $unwind$??$print_module@PEAX@@YAXQEAXPEAXKAEAUoptions@@AEBV?$function@$$A6A_NPEA_W_K@Z@std@@@Z 0000000180058600     Plist.obj
 0001:00057620       $cppxdata$??$print_module@PEAX@@YAXQEAXPEAXKAEAUoptions@@AEBV?$function@$$A6A_NPEA_W_K@Z@std@@@Z 0000000180058620     Plist.obj
 0001:00057629       $stateUnwindMap$??$print_module@PEAX@@YAXQEAXPEAXKAEAUoptions@@AEBV?$function@$$A6A_NPEA_W_K@Z@std@@@Z 0000000180058629     Plist.obj
 0001:00057630       $ip2state$??$print_module@PEAX@@YAXQEAXPEAXKAEAUoptions@@AEBV?$function@$$A6A_NPEA_W_K@Z@std@@@Z 0000000180058630     Plist.obj
 0001:00057638       $unwind$??$_Resize_reallocate@U_Value_init_tag@std@@@?$vector@PEAUHINSTANCE__@@V?$allocator@PEAUHINSTANCE__@@@std@@@std@@AEAAX_KAEBU_Value_init_tag@1@@Z 0000000180058638     Plist.obj
 0001:00057650       $cppxdata$??$_Resize_reallocate@U_Value_init_tag@std@@@?$vector@PEAUHINSTANCE__@@V?$allocator@PEAUHINSTANCE__@@@std@@@std@@AEAAX_KAEBU_Value_init_tag@1@@Z 0000000180058650     Plist.obj
 0001:0005765d       $tryMap$??$_Resize_reallocate@U_Value_init_tag@std@@@?$vector@PEAUHINSTANCE__@@V?$allocator@PEAUHINSTANCE__@@@std@@@std@@AEAAX_KAEBU_Value_init_tag@1@@Z 000000018005865d     Plist.obj
 0001:00057665       $handlerMap$??$_Resize_reallocate@U_Value_init_tag@std@@@?$vector@PEAUHINSTANCE__@@V?$allocator@PEAUHINSTANCE__@@@std@@@std@@AEAAX_KAEBU_Value_init_tag@1@@Z 0000000180058665     Plist.obj
 0001:0005766c       $ip2state$??$_Resize_reallocate@U_Value_init_tag@std@@@?$vector@PEAUHINSTANCE__@@V?$allocator@PEAUHINSTANCE__@@@std@@@std@@AEAAX_KAEBU_Value_init_tag@1@@Z 000000018005866c     Plist.obj
 0001:00057670       $unwind$?ConvertDate@@YAXAEBU_FILETIME@@PEA_W1@Z 0000000180058670     Pmix.obj
 0001:0005767c       $unwind$?WinError@@YAHPEB_W@Z 000000018005867c     Pmix.obj
 0001:0005769c       $cppxdata$?WinError@@YAHPEB_W@Z 000000018005869c     Pmix.obj
 0001:000576a5       $stateUnwindMap$?WinError@@YAHPEB_W@Z 00000001800586a5     Pmix.obj
 0001:000576b3       $ip2state$?WinError@@YAHPEB_W@Z 00000001800586b3     Pmix.obj
 0001:000576bc       $unwind$??0WMIConnection@@QEAA@XZ 00000001800586bc     WMI.obj
 0001:000576cc       $cppxdata$??0WMIConnection@@QEAA@XZ 00000001800586cc     WMI.obj
 0001:000576d5       $stateUnwindMap$??0WMIConnection@@QEAA@XZ 00000001800586d5     WMI.obj
 0001:000576dc       $ip2state$??0WMIConnection@@QEAA@XZ 00000001800586dc     WMI.obj
 0001:000576e0       $unwind$??1WMIConnection@@QEAA@XZ 00000001800586e0     WMI.obj
 0001:000576f0       $cppxdata$??1WMIConnection@@QEAA@XZ 00000001800586f0     WMI.obj
 0001:000576f9       $ip2state$??1WMIConnection@@QEAA@XZ 00000001800586f9     WMI.obj
 0001:00057700       $unwind$?Connect@WMIConnection@@QEAA_NPEB_W00@Z 0000000180058700     WMI.obj
 0001:00057728       $cppxdata$?Connect@WMIConnection@@QEAA_NPEB_W00@Z 0000000180058728     WMI.obj
 0001:00057731       $stateUnwindMap$?Connect@WMIConnection@@QEAA_NPEB_W00@Z 0000000180058731     WMI.obj
 0001:0005775d       $ip2state$?Connect@WMIConnection@@QEAA_NPEB_W00@Z 000000018005875d     WMI.obj
 0001:0005776c       $unwind$?GetProcessPriority@WMIConnection@@QEAAKK@Z 000000018005876c     WMI.obj
 0001:0005776c       $unwind$?GetProcessSessionId@WMIConnection@@QEAAKK@Z 000000018005876c     WMI.obj
 0001:0005777c       $cppxdata$?GetProcessPriority@WMIConnection@@QEAAKK@Z 000000018005877c     WMI.obj
 0001:0005777c       $cppxdata$?GetProcessSessionId@WMIConnection@@QEAAKK@Z 000000018005877c     WMI.obj
 0001:00057785       $stateUnwindMap$?GetProcessPriority@WMIConnection@@QEAAKK@Z 0000000180058785     WMI.obj
 0001:00057785       $stateUnwindMap$?GetProcessSessionId@WMIConnection@@QEAAKK@Z 0000000180058785     WMI.obj
 0001:0005778c       $ip2state$?GetProcessPriority@WMIConnection@@QEAAKK@Z 000000018005878c     WMI.obj
 0001:0005778c       $ip2state$?GetProcessSessionId@WMIConnection@@QEAAKK@Z 000000018005878c     WMI.obj
 0001:00057790       $unwind$?GetProcessOwner@WMIConnection@@QEAA?AV?$basic_string@_WU?$char_traits@_W@std@@V?$allocator@_W@2@@std@@KPEAV23@@Z 0000000180058790     WMI.obj
 0001:000577b0       $cppxdata$?GetProcessOwner@WMIConnection@@QEAA?AV?$basic_string@_WU?$char_traits@_W@std@@V?$allocator@_W@2@@std@@KPEAV23@@Z 00000001800587b0     WMI.obj
 0001:000577b9       $stateUnwindMap$?GetProcessOwner@WMIConnection@@QEAA?AV?$basic_string@_WU?$char_traits@_W@std@@V?$allocator@_W@2@@std@@KPEAV23@@Z 00000001800587b9     WMI.obj
 0001:000577e6       $ip2state$?GetProcessOwner@WMIConnection@@QEAA?AV?$basic_string@_WU?$char_traits@_W@std@@V?$allocator@_W@2@@std@@KPEAV23@@Z 00000001800587e6     WMI.obj
 0001:000577f4       $unwind$?GetProcessUserSid@WMIConnection@@QEAA?AV?$basic_string@_WU?$char_traits@_W@std@@V?$allocator@_W@2@@std@@K@Z 00000001800587f4     WMI.obj
 0001:00057814       $cppxdata$?GetProcessUserSid@WMIConnection@@QEAA?AV?$basic_string@_WU?$char_traits@_W@std@@V?$allocator@_W@2@@std@@K@Z 0000000180058814     WMI.obj
 0001:0005781d       $stateUnwindMap$?GetProcessUserSid@WMIConnection@@QEAA?AV?$basic_string@_WU?$char_traits@_W@std@@V?$allocator@_W@2@@std@@K@Z 000000018005881d     WMI.obj
 0001:0005784a       $ip2state$?GetProcessUserSid@WMIConnection@@QEAA?AV?$basic_string@_WU?$char_traits@_W@std@@V?$allocator@_W@2@@std@@K@Z 000000018005884a     WMI.obj
 0001:00057858       $unwind$?GetProcessCommandLine@WMIConnection@@QEAA?AV?$basic_string@_WU?$char_traits@_W@std@@V?$allocator@_W@2@@std@@K@Z 0000000180058858     WMI.obj
 0001:00057858       $unwind$?GetProcessExecutablePath@WMIConnection@@QEAA?AV?$basic_string@_WU?$char_traits@_W@std@@V?$allocator@_W@2@@std@@K@Z 0000000180058858     WMI.obj
 0001:00057868       $cppxdata$?GetProcessCommandLine@WMIConnection@@QEAA?AV?$basic_string@_WU?$char_traits@_W@std@@V?$allocator@_W@2@@std@@K@Z 0000000180058868     WMI.obj
 0001:00057868       $cppxdata$?GetProcessExecutablePath@WMIConnection@@QEAA?AV?$basic_string@_WU?$char_traits@_W@std@@V?$allocator@_W@2@@std@@K@Z 0000000180058868     WMI.obj
 0001:00057871       $stateUnwindMap$?GetProcessCommandLine@WMIConnection@@QEAA?AV?$basic_string@_WU?$char_traits@_W@std@@V?$allocator@_W@2@@std@@K@Z 0000000180058871     WMI.obj
 0001:00057871       $stateUnwindMap$?GetProcessExecutablePath@WMIConnection@@QEAA?AV?$basic_string@_WU?$char_traits@_W@std@@V?$allocator@_W@2@@std@@K@Z 0000000180058871     WMI.obj
 0001:0005787d       $ip2state$?GetProcessCommandLine@WMIConnection@@QEAA?AV?$basic_string@_WU?$char_traits@_W@std@@V?$allocator@_W@2@@std@@K@Z 000000018005887d     WMI.obj
 0001:0005787d       $ip2state$?GetProcessExecutablePath@WMIConnection@@QEAA?AV?$basic_string@_WU?$char_traits@_W@std@@V?$allocator@_W@2@@std@@K@Z 000000018005887d     WMI.obj
 0001:00057880       $unwind$?ExecMethod@WMIConnection@@AEAAHKPEB_W0K@Z 0000000180058880     WMI.obj
 0001:000578a4       $cppxdata$?ExecMethod@WMIConnection@@AEAAHKPEB_W0K@Z 00000001800588a4     WMI.obj
 0001:000578ad       $stateUnwindMap$?ExecMethod@WMIConnection@@AEAAHKPEB_W0K@Z 00000001800588ad     WMI.obj
 0001:0005790c       $ip2state$?ExecMethod@WMIConnection@@AEAAHKPEB_W0K@Z 000000018005890c     WMI.obj
 0001:0005792c       $unwind$?GetProcessProperty@WMIConnection@@AEAA_NKPEB_WAEBV?$function@$$A6AXAEBUtagVARIANT@@@Z@std@@@Z 000000018005892c     WMI.obj
 0001:0005794c       $cppxdata$?GetProcessProperty@WMIConnection@@AEAA_NKPEB_WAEBV?$function@$$A6AXAEBUtagVARIANT@@@Z@std@@@Z 000000018005894c     WMI.obj
 0001:00057955       $stateUnwindMap$?GetProcessProperty@WMIConnection@@AEAA_NKPEB_WAEBV?$function@$$A6AXAEBUtagVARIANT@@@Z@std@@@Z 0000000180058955     WMI.obj
 0001:00057975       $ip2state$?GetProcessProperty@WMIConnection@@AEAA_NKPEB_WAEBV?$function@$$A6AXAEBUtagVARIANT@@@Z@std@@@Z 0000000180058975     WMI.obj
 0001:00057984       $unwind$?ProcessPath@@YA@K@Z 0000000180058984     WMI.obj
 0001:0005798c       $unwind$??1?$unique_ptr@UIWbemClassObject@@Ucom_closer@@@std@@QEAA@XZ 000000018005898c     WMI.obj
 0001:0005798c       $unwind$??1?$unique_ptr@UIWbemLocator@@Ucom_closer@@@std@@QEAA@XZ 000000018005898c     WMI.obj
 0001:0005799c       $cppxdata$??1?$unique_ptr@UIWbemClassObject@@Ucom_closer@@@std@@QEAA@XZ 000000018005899c     WMI.obj
 0001:0005799c       $cppxdata$??1?$unique_ptr@UIWbemLocator@@Ucom_closer@@@std@@QEAA@XZ 000000018005899c     WMI.obj
 0001:000579a1       $ip2state$??1?$unique_ptr@UIWbemClassObject@@Ucom_closer@@@std@@QEAA@XZ 00000001800589a1     WMI.obj
 0001:000579a1       $ip2state$??1?$unique_ptr@UIWbemLocator@@Ucom_closer@@@std@@QEAA@XZ 00000001800589a1     WMI.obj
 0001:000579a4       $unwind$??1?$ptr_setter@V?$unique_ptr@UIWbemClassObject@@Ucom_closer@@@std@@@@QEAA@XZ 00000001800589a4     WMI.obj
 0001:000579b4       $cppxdata$??1?$ptr_setter@V?$unique_ptr@UIWbemClassObject@@Ucom_closer@@@std@@@@QEAA@XZ 00000001800589b4     WMI.obj
 0001:000579bd       $ip2state$??1?$ptr_setter@V?$unique_ptr@UIWbemClassObject@@Ucom_closer@@@std@@@@QEAA@XZ 00000001800589bd     WMI.obj
 0001:000579c0       $chain$0$?dynamic_bind@@YAXXZ 00000001800589c0     Proclist.obj
 0001:000579d4       $chain$1$?dynamic_bind@@YAXXZ 00000001800589d4     Proclist.obj
 0001:000579e4       $unwind$?_Init@locale@std@@CAPEAV_Locimp@12@_N@Z 00000001800589e4     libcpmt:locale0.obj
 0001:000579f8       $stateUnwindMap$?_Init@locale@std@@CAPEAV_Locimp@12@_N@Z 00000001800589f8     libcpmt:locale0.obj
 0001:00057a00       $ip2state$?_Init@locale@std@@CAPEAV_Locimp@12@_N@Z 0000000180058a00     libcpmt:locale0.obj
 0001:00057a10       $unwind$_Mbrtowc           0000000180058a10     libcpmt:xmbtowc.obj
 0001:00057a10       $unwind$?getStateFromIterators@UWMap4@FH4@@SAHAEBViterator@12@H0H0@Z 0000000180058a10     libvcruntime:frame.obj
 0001:00057a10       $unwind$?commit_locale_name@_expandlocale_locale_name_cache@@QEAAXQEB_W_K@Z 0000000180058a10     libucrt:wsetlocale.obj
 0001:00057a10       $unwind$__acrt_copy_locale_name 0000000180058a10     libucrt:wsetlocale.obj
 0001:00057a10       $unwind$strpbrk            0000000180058a10     libucrt:strpbrk.obj
 0001:00057a20       $unwind$??__Finit_atexit@@YAXXZ 0000000180058a20     libcpmt:iosptrs.obj
 0001:00057a30       $stateUnwindMap$??__Finit_atexit@@YAXXZ 0000000180058a30     libcpmt:iosptrs.obj
 0001:00057a38       $ip2state$??__Finit_atexit@@YAXXZ 0000000180058a38     libcpmt:iosptrs.obj
 0001:00057a40       $unwind$__scrt_is_nonwritable_in_current_image 0000000180058a40     LIBCMT:utility.obj
 0001:00057a60       $unwind$??_M@YAXPEAX_K1P6AX0@Z@Z 0000000180058a60     LIBCMT:ehvecdtr.obj
 0001:00057a88       $unwind$?__ArrayUnwind@@YAXPEAX_K1P6AX0@Z@Z 0000000180058a88     LIBCMT:ehvecdtr.obj
 0001:00057ab4       $unwind$?filt$0@?0??__ArrayUnwind@@YAXPEAX_K1P6AX0@Z@Z@4HA 0000000180058ab4     LIBCMT:ehvecdtr.obj
 0001:00057ab4       $unwind$__DestructExceptionObject$filt$0 0000000180058ab4     libvcruntime:ehhelpers.obj
 0001:00057ab4       $unwind$?fin$1@?0??CxxCallCatchBlock@__FrameHandler3@@SAPEAXPEAU_EXCEPTION_RECORD@@@Z@4HA 0000000180058ab4     libvcruntime:frame.obj
 0001:00057ab4       $unwind$?fin$1@?0??CxxCallCatchBlock@__FrameHandler4@@SAPEAXPEAU_EXCEPTION_RECORD@@@Z@4HA 0000000180058ab4     libvcruntime:frame.obj
 0001:00057ac0       $unwind$?dllmain_crt_process_attach@@YAHQEAUHINSTANCE__@@QEAX@Z 0000000180058ac0     LIBCMT:dll_dllmain.obj
 0001:00057afc       $unwind$?dllmain_crt_process_detach@@YAH_N@Z 0000000180058afc     LIBCMT:dll_dllmain.obj
 0001:00057b50       $unwind$?dllmain_dispatch@@YAHQEAUHINSTANCE__@@KQEAX@Z 0000000180058b50     LIBCMT:dll_dllmain.obj
 0001:00057b78       $unwind$?filt$0@?0??dllmain_dispatch@@YAHQEAUHINSTANCE__@@KQEAX@Z@4HA 0000000180058b78     LIBCMT:dll_dllmain.obj
 0001:00057b78       $unwind$?filt$0@?0??FrameUnwindToState@__FrameHandler4@@SAXPEA_KPEAU_xDISPATCHER_CONTEXT@@PEAUFuncInfo4@FH4@@H@Z@4HA 0000000180058b78     libvcruntime:frame.obj
 0001:00057b78       $unwind$?fin$1@?0??FrameUnwindToState@__FrameHandler4@@SAXPEA_KPEAU_xDISPATCHER_CONTEXT@@PEAUFuncInfo4@FH4@@H@Z@4HA 0000000180058b78     libvcruntime:frame.obj
 0001:00057b80       $unwind$__GSHandlerCheck_EH 0000000180058b80     LIBCMT:gshandlereh.obj
 0001:00057b80       $unwind$__GSHandlerCheck_SEH 0000000180058b80     LIBCMT:gshandlerseh.obj
 0001:00057b80       $unwind$??$TypeMatchHelper@V__FrameHandler3@@@@YAHPEBU_s_HandlerType@@PEBU_s_CatchableType@@PEBU_s_ThrowInfo@@@Z 0000000180058b80     libvcruntime:frame.obj
 0001:00057b80       $unwind$??$TypeMatchHelper@V__FrameHandler4@@@@YAHPEAUHandlerType4@FH4@@PEBU_s_CatchableType@@PEBU_s_ThrowInfo@@@Z 0000000180058b80     libvcruntime:frame.obj
 0001:00057b80       $unwind$?initialize_stdio_handles_nolock@@YAXXZ 0000000180058b80     libucrt:ioinit.obj
 0001:00057b80       $unwind$__acrt_initialize_stdio 0000000180058b80     libucrt:_file.obj
 0001:00057b98       $xdatasym                  0000000180058b98     LIBCMT:amdsecgs.obj
 0001:00057b9c       $unwind$__isa_available_init 0000000180058b9c     LIBCMT:cpu_disp.obj
 0001:00057bac       $unwind$__scrt_fastfail    0000000180058bac     LIBCMT:utility_desktop.obj
 0001:00057bbc       $unwind$__security_init_cookie 0000000180058bbc     LIBCMT:gs_support.obj
 0001:00057bc8       $xdatasym                  0000000180058bc8     LIBCMT:guard_dispatch.obj
 0001:00057bcc       $unwind$__report_securityfailure 0000000180058bcc     LIBCMT:gs_report.obj
 0001:00057bd4       $unwind$capture_current_context 0000000180058bd4     LIBCMT:gs_report.obj
 0001:00057be0       $unwind$capture_previous_context 0000000180058be0     LIBCMT:gs_report.obj
 0001:00057bec       $unwind$__DestructExceptionObject 0000000180058bec     libvcruntime:ehhelpers.obj
 0001:00057c0c       $unwind$__std_exception_copy 0000000180058c0c     libvcruntime:std_exception.obj
 0001:00057c0c       $unwind$_wcstombs_s_l      0000000180058c0c     libucrt:wcstombs.obj
 0001:00057c0c       $unwind$string_is_alpha    0000000180058c0c     libucrt:wsetlocale.obj
 0001:00057c0c       $unwind$_free_osfhnd       0000000180058c0c     libucrt:osfinfo.obj
 0001:00057c20       $unwind$_CxxThrowException 0000000180058c20     libvcruntime:throw.obj
 0001:00057c30       $unwind$?DecompFuncInfo@FH4@@YA_JPEAEAEAUFuncInfo4@1@_KH_N@Z 0000000180058c30     libvcruntime:risctrnsctrl.obj
 0001:00057c48       $unwind$?UnwindNestedFrames@__FrameHandler3@@SAXPEA_KPEAUEHExceptionRecord@@PEAU_CONTEXT@@0PEAXPEBU_s_FuncInfo@@HHPEBU_s_HandlerType@@PEAU_xDISPATCHER_CONTEXT@@E@Z 0000000180058c48     libvcruntime:risctrnsctrl.obj
 0001:00057c5c       $unwind$?GetRangeOfTrysToCheck@__FrameHandler3@@SA?AU?$pair@Viterator@TryBlockMap@__FrameHandler3@@V123@@std@@AEAVTryBlockMap@1@HPEAU_xDISPATCHER_CONTEXT@@PEBU_s_FuncInfo@@H@Z 0000000180058c5c     libvcruntime:risctrnsctrl.obj
 0001:00057c74       $unwind$?UnwindNestedFrames@__FrameHandler4@@SAXPEA_KPEAUEHExceptionRecord@@PEAU_CONTEXT@@0PEAXPEAUFuncInfo4@FH4@@HHPEAUHandlerType4@5@PEAU_xDISPATCHER_CONTEXT@@E@Z 0000000180058c74     libvcruntime:risctrnsctrl.obj
 0001:00057c88       $unwind$?GetRangeOfTrysToCheck@__FrameHandler4@@SA?AU?$pair@Viterator@TryBlockMap4@FH4@@V123@@std@@AEAVTryBlockMap4@FH4@@HPEAU_xDISPATCHER_CONTEXT@@PEAUFuncInfo4@5@H@Z 0000000180058c88     libvcruntime:risctrnsctrl.obj
 0001:00057ca4       $unwind$__CxxFrameHandler3 0000000180058ca4     libvcruntime:risctrnsctrl.obj
 0001:00057cb8       $unwind$__CxxFrameHandler4 0000000180058cb8     libvcruntime:risctrnsctrl.obj
 0001:00057ccc       $unwind$??$_CallSETranslator@V__FrameHandler4@@@@YAHPEAUEHExceptionRecord@@PEA_KPEAU_CONTEXT@@PEAU_xDISPATCHER_CONTEXT@@PEAUFuncInfo4@FH4@@K1@Z 0000000180058ccc     libvcruntime:risctrnsctrl.obj
 0001:00057cec       $unwind$?filt$0@?0???$_CallSETranslator@V__FrameHandler3@@@@YAHPEAUEHExceptionRecord@@PEA_KPEAU_CONTEXT@@PEAU_xDISPATCHER_CONTEXT@@PEBU_s_FuncInfo@@K1@Z@4HA 0000000180058cec     libvcruntime:risctrnsctrl.obj
 0001:00057cec       $unwind$?filt$0@?0???$_CallSETranslator@V__FrameHandler4@@@@YAHPEAUEHExceptionRecord@@PEA_KPEAU_CONTEXT@@PEAU_xDISPATCHER_CONTEXT@@PEAUFuncInfo4@FH4@@K1@Z@4HA 0000000180058cec     libvcruntime:risctrnsctrl.obj
 0001:00057cf8       $unwind$??$_CallSETranslator@V__FrameHandler3@@@@YAHPEAUEHExceptionRecord@@PEA_KPEAU_CONTEXT@@PEAU_xDISPATCHER_CONTEXT@@PEBU_s_FuncInfo@@K1@Z 0000000180058cf8     libvcruntime:risctrnsctrl.obj
 0001:00057d18       $xdatasym                  0000000180058d18     libvcruntime:memchr.obj
 0001:00057d20       $xdatasym                  0000000180058d20     libvcruntime:memcmp.obj
 0001:00057d28       $xdatasym                  0000000180058d28     libvcruntime:memcpy.obj
 0001:00057d38       $xdatasym                  0000000180058d38     libvcruntime:memset.obj
 0001:00057d48       $unwind$__C_specific_handler 0000000180058d48     libvcruntime:riscchandler.obj
 0001:00057d48       $unwind$__acrt_locale_initialize_numeric 0000000180058d48     libucrt:initnum.obj
 0001:00057d64       $unwind$?StateFromIp@__FrameHandler4@@SAHPEAUFuncInfo4@FH4@@PEAU_xDISPATCHER_CONTEXT@@_K@Z 0000000180058d64     libvcruntime:ehstate.obj
 0001:00057d78       $unwind$?getStartStop@UWMap4@FH4@@QEAAXHHAEAViterator@12@0@Z 0000000180058d78     libvcruntime:frame.obj
 0001:00057d90       $unwind$?FrameUnwindToState@__FrameHandler3@@SAXPEA_KPEAU_xDISPATCHER_CONTEXT@@PEBU_s_FuncInfo@@H@Z 0000000180058d90     libvcruntime:frame.obj
 0001:00057ddc       $unwind$?CxxCallCatchBlock@__FrameHandler3@@SAPEAXPEAU_EXCEPTION_RECORD@@@Z 0000000180058ddc     libvcruntime:frame.obj
 0001:00057e18       $unwind$?FrameUnwindToState@__FrameHandler4@@SAXPEA_KPEAU_xDISPATCHER_CONTEXT@@PEAUFuncInfo4@FH4@@H@Z 0000000180058e18     libvcruntime:frame.obj
 0001:00057e60       $unwind$?CxxCallCatchBlock@__FrameHandler4@@SAPEAXPEAU_EXCEPTION_RECORD@@@Z 0000000180058e60     libvcruntime:frame.obj
 0001:00057ebc       $unwind$?IsInExceptionSpec@@YAEPEAUEHExceptionRecord@@PEBU_s_ESTypeList@@@Z 0000000180058ebc     libvcruntime:frame.obj
 0001:00057ed8       $unwind$??$__InternalCxxFrameHandler@V__FrameHandler3@@@@YA?AW4_EXCEPTION_DISPOSITION@@PEAUEHExceptionRecord@@PEA_KPEAU_CONTEXT@@PEAU_xDISPATCHER_CONTEXT@@PEBU_s_FuncInfo@@H1E@Z 0000000180058ed8     libvcruntime:frame.obj
 0001:00057ef0       $unwind$??$__InternalCxxFrameHandler@V__FrameHandler4@@@@YA?AW4_EXCEPTION_DISPOSITION@@PEAUEHExceptionRecord@@PEA_KPEAU_CONTEXT@@PEAU_xDISPATCHER_CONTEXT@@PEAUFuncInfo4@FH4@@H1E@Z 0000000180058ef0     libvcruntime:frame.obj
 0001:00057f08       $unwind$??$BuildCatchObjectHelperInternal@V__FrameHandler3@@@@YAHPEAUEHExceptionRecord@@PEAXPEBU_s_HandlerType@@PEBU_s_CatchableType@@@Z 0000000180058f08     libvcruntime:frame.obj
 0001:00057f48       $unwind$??$BuildCatchObjectHelperInternal@V__FrameHandler4@@@@YAHPEAUEHExceptionRecord@@PEAXPEAUHandlerType4@FH4@@PEBU_s_CatchableType@@@Z 0000000180058f48     libvcruntime:frame.obj
 0001:00057f88       $unwind$??$BuildCatchObjectInternal@V__FrameHandler3@@@@YAXPEAUEHExceptionRecord@@PEAXPEBU_s_HandlerType@@PEBU_s_CatchableType@@@Z 0000000180058f88     libvcruntime:frame.obj
 0001:00057fb4       $unwind$??$BuildCatchObjectInternal@V__FrameHandler4@@@@YAXPEAUEHExceptionRecord@@PEAXPEAUHandlerType4@FH4@@PEBU_s_CatchableType@@@Z 0000000180058fb4     libvcruntime:frame.obj
 0001:00057fe0       $unwind$??$FindHandler@V__FrameHandler3@@@@YAXPEAUEHExceptionRecord@@PEA_KPEAU_CONTEXT@@PEAU_xDISPATCHER_CONTEXT@@PEBU_s_FuncInfo@@EH1@Z 0000000180058fe0     libvcruntime:frame.obj
 0001:00058000       $unwind$??$FindHandler@V__FrameHandler4@@@@YAXPEAUEHExceptionRecord@@PEA_KPEAU_CONTEXT@@PEAU_xDISPATCHER_CONTEXT@@PEAUFuncInfo4@FH4@@EH1@Z 0000000180059000     libvcruntime:frame.obj
 0001:00058020       $unwind$??$CatchIt@V__FrameHandler3@@@@YAXPEAUEHExceptionRecord@@PEA_KPEAU_CONTEXT@@PEAU_xDISPATCHER_CONTEXT@@PEBU_s_FuncInfo@@PEBU_s_HandlerType@@PEBU_s_CatchableType@@PEBU_s_TryBlockMapEntry@@H1EE@Z 0000000180059020     libvcruntime:frame.obj
 0001:00058020       $unwind$??$CatchIt@V__FrameHandler4@@@@YAXPEAUEHExceptionRecord@@PEA_KPEAU_CONTEXT@@PEAU_xDISPATCHER_CONTEXT@@PEAUFuncInfo4@FH4@@PEAUHandlerType4@4@PEBU_s_CatchableType@@PEAUTryBlockMapEntry4@4@H1EE@Z 0000000180059020     libvcruntime:frame.obj
 0001:00058038       $unwind$??$FindHandlerForForeignException@V__FrameHandler3@@@@YAXPEAUEHExceptionRecord@@PEA_KPEAU_CONTEXT@@PEAU_xDISPATCHER_CONTEXT@@PEBU_s_FuncInfo@@HH1@Z 0000000180059038     libvcruntime:frame.obj
 0001:00058054       $unwind$??$FindHandlerForForeignException@V__FrameHandler4@@@@YAXPEAUEHExceptionRecord@@PEA_KPEAU_CONTEXT@@PEAU_xDISPATCHER_CONTEXT@@PEAUFuncInfo4@FH4@@HH1@Z 0000000180059054     libvcruntime:frame.obj
 0001:00058078       $xdatasym                  0000000180059078     libvcruntime:notify.obj
 0001:00058088       $xdatasym                  0000000180059088     libvcruntime:handlers.obj
 0001:000580a8       $unwind$__acrt_call_reportfault 00000001800590a8     libucrt:invalid_parameter.obj
 0001:000580c8       $unwind$_dclass            00000001800590c8     libucrt:nan.obj
 0001:000580c8       $unwind$_fdclass           00000001800590c8     libucrt:nanf.obj
 0001:000580c8       $unwind$_ldclass           00000001800590c8     libucrt:nanl.obj
 0001:000580c8       $unwind$round              00000001800590c8     libucrt:round.obj
 0001:000580d0       $unwind$__stdio_common_vsnprintf_s 00000001800590d0     libucrt:output.obj
 0001:000580e8       $unwind$?write_string@?$string_output_adapter@D@__crt_stdio_output@@QEBAXQEBDHQEAHAEAV__crt_deferred_errno_cache@@@Z 00000001800590e8     libucrt:output.obj
 0001:00058100       $unwind$??$common_vsprintf@Vformat_validation_base@__crt_stdio_output@@D@@YAH_KQEAD0QEBDQEAU__crt_locale_pointers@@1@Z 0000000180059100     libucrt:output.obj
 0001:00058120       $unwind$??$write_multiple_characters@V?$string_output_adapter@D@__crt_stdio_output@@D@__crt_stdio_output@@YAXAEBV?$string_output_adapter@D@0@DHQEAH@Z 0000000180059120     libucrt:output.obj
 0001:0005812c       $unwind$?process@?$output_processor@DV?$string_output_adapter@D@__crt_stdio_output@@V?$format_validation_base@DV?$string_output_adapter@D@__crt_stdio_output@@@2@@__crt_stdio_output@@QEAAHXZ 000000018005912c     libucrt:output.obj
 0001:00058140       $unwind$?parse_int_from_format_string@?$output_processor@DV?$string_output_adapter@D@__crt_stdio_output@@V?$format_validation_base@DV?$string_output_adapter@D@__crt_stdio_output@@@2@@__crt_stdio_output@@AEAA_NQEAH@Z 0000000180059140     libucrt:output.obj
 0001:00058154       $unwind$?type_case_a@?$output_processor@DV?$string_output_adapter@D@__crt_stdio_output@@V?$format_validation_base@DV?$string_output_adapter@D@__crt_stdio_output@@@2@@__crt_stdio_output@@AEAA_NXZ 0000000180059154     libucrt:output.obj
 0001:00058160       $unwind$?write_stored_string_tchar@?$output_processor@DV?$string_output_adapter@D@__crt_stdio_output@@V?$format_validation_base@DV?$string_output_adapter@D@__crt_stdio_output@@@2@@__crt_stdio_output@@AEAA_ND@Z 0000000180059160     libucrt:output.obj
 0001:00058178       $unwind$??$type_case_integer_parse_into_buffer@I@?$output_processor@DV?$string_output_adapter@D@__crt_stdio_output@@V?$format_validation_base@DV?$string_output_adapter@D@__crt_stdio_output@@@2@@__crt_stdio_output@@AEAAXII_N@Z 0000000180059178     libucrt:output.obj
 0001:00058178       $unwind$??$type_case_integer_parse_into_buffer@_K@?$output_processor@DV?$string_output_adapter@D@__crt_stdio_output@@V?$format_validation_base@DV?$string_output_adapter@D@__crt_stdio_output@@@2@@__crt_stdio_output@@AEAAX_KI_N@Z 0000000180059178     libucrt:output.obj
 0001:00058178       $unwind$__acrt_wcstok_s_novalidation 0000000180059178     libucrt:wcstok_s.obj
 0001:00058180       $unwind$terminate          0000000180059180     libucrt:terminate.obj
 0001:000581a0       $unwind$__acrt_lowio_destroy_handle_array 00000001800591a0     libucrt:osfinfo.obj
 0001:000581b0       $unwind$__acrt_lowio_ensure_fh_exists 00000001800591b0     libucrt:osfinfo.obj
 0001:000581dc       $unwind$log2               00000001800591dc     libucrt:log2.obj
 0001:000581e8       $unwind$__dcrt_lowio_ensure_console_output_initialized 00000001800591e8     libucrt:initcon.obj
 0001:000581e8       $unwind$_isleadbyte_l      00000001800591e8     libucrt:_wctype.obj
 0001:000581e8       $unwind$?getSystemCP@@YAHH@Z 00000001800591e8     libucrt:mbctype.obj
 0001:000581f0       $unwind$__acrt_initialize_winapi_thunks 00000001800591f0     libucrt:winapi_thunks.obj
 0001:000581f0       $unwind$wcsncpy            00000001800591f0     libucrt:wcsncpy.obj
 0001:000581f8       $xdatasym                  00000001800591f8     libucrt:log10.obj
 0001:00058208       $xdatasym                  0000000180059208     libucrt:pow.obj
 0001:00058218       $unwind$setlocale          0000000180059218     libucrt:setlocale.obj
 0001:00058220       $unwind$??R<lambda_b37934c380d97b75fd242ea49540127a>@@QEBAPEADXZ 0000000180059220     libucrt:setlocale.obj
 0001:00058238       $unwind$??$?RV<lambda_41e84717acc955b55e9d0d529e507b68>@@AEAV<lambda_b37934c380d97b75fd242ea49540127a>@@V<lambda_bb6db9f9ac473960206e0d4b942b5506>@@@?$__crt_seh_guarded_call@PEAD@@QEAAPEAD$$QEAV<lambda_41e84717acc955b55e9d0d529e507b68>@@AEAV<lambda_b37934c380d97b75fd242ea49540127a>@@$$QEAV<lambda_bb6db9f9ac473960206e0d4b942b5506>@@@Z 0000000180059238     libucrt:setlocale.obj
 0001:0005825c       $unwind$__acrt_locale_initialize_ctype 000000018005925c     libucrt:initctype.obj
 0001:00058284       $unwind$?divide@__crt_strtox@@YA_KAEAUbig_integer@1@AEBU21@@Z 0000000180059284     libucrt:strtod.obj
 0001:0005829c       $chain$0$?divide@__crt_strtox@@YA_KAEAUbig_integer@1@AEBU21@@Z 000000018005929c     libucrt:strtod.obj
 0001:000582b0       $chain$1$?divide@__crt_strtox@@YA_KAEAUbig_integer@1@AEBU21@@Z 00000001800592b0     libucrt:strtod.obj
 0001:000582c0       $xdatasym                  00000001800592c0     libucrt:powf.obj
 0001:000582d0       $unwind$parse_bcp47_region 00000001800592d0     libucrt:wsetlocale.obj
 0001:000582d0       $unwind$??$__acrt_mbs_to_wcs_cp@U__crt_win32_buffer_internal_dynamic_resizing@@@@YAHQEBDAEAV?$__crt_win32_buffer@_WU__crt_win32_buffer_internal_dynamic_resizing@@@@I@Z 00000001800592d0     libucrt:strftime.obj
 0001:000582e8       $unwind$__dcrt_write_console 00000001800592e8     libucrt:initcon.obj
 0001:000582e8       $unwind$??$__acrt_wcs_to_mbs_cp@U__crt_win32_buffer_no_resizing@@@@YAHQEB_WAEAV?$__crt_win32_buffer@DU__crt_win32_buffer_no_resizing@@@@I@Z 00000001800592e8     libucrt:strftime.obj
 0001:000582fc       $unwind$?common_exit@@YAXHW4_crt_exit_cleanup_mode@@W4_crt_exit_return_mode@@@Z 00000001800592fc     libucrt:exit.obj
 0001:00058308       $unwind$??R<lambda_6e4b09c48022b2350581041d5f6b0c4c>@@QEBA@XZ 0000000180059308     libucrt:exit.obj
 0001:00058328       $unwind$??$?RV<lambda_d80eeec6fff315bfe5c115232f3240e3>@@AEAV<lambda_6e4b09c48022b2350581041d5f6b0c4c>@@V<lambda_2358e3775559c9db80273638284d5e45>@@@?$__crt_seh_guarded_call@X@@QEAAX$$QEAV<lambda_d80eeec6fff315bfe5c115232f3240e3>@@AEAV<lambda_6e4b09c48022b2350581041d5f6b0c4c>@@$$QEAV<lambda_2358e3775559c9db80273638284d5e45>@@@Z 0000000180059328     libucrt:exit.obj
 0001:0005834c       $unwind$_configure_narrow_argv 000000018005934c     libucrt:argv_parsing.obj
 0001:00058360       $unwind$TranslateName      0000000180059360     libucrt:get_qualified_locale.obj
 0001:00058360       $unwind$??$parse_command_line@D@@YAXPEADPEAPEAD0PEA_K2@Z 0000000180059360     libucrt:argv_parsing.obj
 0001:0005837c       $unwind$??$create_environment@D@@YAQEAPEADQEAD@Z 000000018005937c     libucrt:environment_initialization.obj
 0001:0005837c       $unwind$__lc_wcstolc       000000018005937c     libucrt:wsetlocale.obj
 0001:00058394       $unwind$_register_onexit_function 0000000180059394     libucrt:onexit.obj
 0001:0005839c       $unwind$_execute_onexit_table 000000018005939c     libucrt:onexit.obj
 0001:000583a4       $unwind$??R<lambda_22ebabd17bc4fa466a2aca6d8deb888d>@@QEBAHXZ 00000001800593a4     libucrt:onexit.obj
 0001:000583bc       $unwind$??$?RV<lambda_638799b9deba96c50f710eeac98168cd>@@AEAV<lambda_22ebabd17bc4fa466a2aca6d8deb888d>@@V<lambda_a6f7d7db0129f75315ebf26d50c089f1>@@@?$__crt_seh_guarded_call@H@@QEAAH$$QEAV<lambda_638799b9deba96c50f710eeac98168cd>@@AEAV<lambda_22ebabd17bc4fa466a2aca6d8deb888d>@@$$QEAV<lambda_a6f7d7db0129f75315ebf26d50c089f1>@@@Z 00000001800593bc     libucrt:onexit.obj
 0001:000583e0       $unwind$??$?RV<lambda_7777bce6b2f8c936911f934f8298dc43>@@AEAV<lambda_f03950bc5685219e0bcd2087efbe011e>@@V<lambda_3883c3dff614d5e0c5f61bb1ac94921c>@@@?$__crt_seh_guarded_call@H@@QEAAH$$QEAV<lambda_7777bce6b2f8c936911f934f8298dc43>@@AEAV<lambda_f03950bc5685219e0bcd2087efbe011e>@@$$QEAV<lambda_3883c3dff614d5e0c5f61bb1ac94921c>@@@Z 00000001800593e0     libucrt:onexit.obj
 0001:00058404       $unwind$_query_new_handler 0000000180059404     libucrt:new_handler.obj
 0001:00058424       $unwind$??$parse_integer@KV?$c_string_character_source@D@__crt_strtox@@@__crt_strtox@@YAKQEAU__crt_locale_pointers@@V?$c_string_character_source@D@0@H_N@Z 0000000180059424     libucrt:atox.obj
 0001:00058440       $unwind$??$parse_integer@KV?$c_string_character_source@_W@__crt_strtox@@@__crt_strtox@@YAKQEAU__crt_locale_pointers@@V?$c_string_character_source@_W@0@H_N@Z 0000000180059440     libucrt:atox.obj
 0001:00058458       $xdatasym                  0000000180059458     libucrt:strncmp.obj
 0001:0005845c       $unwind$?construct_ptd_array@@YAXQEAU__acrt_ptd@@@Z 000000018005945c     libucrt:per_thread_data.obj
 0001:00058464       $unwind$?destroy_ptd_array@@YAXQEAU__acrt_ptd@@@Z 0000000180059464     libucrt:per_thread_data.obj
 0001:0005846c       $unwind$??$?RV<lambda_0ae27a3a962d80f24befdcbee591983d>@@AEAV<lambda_8d0ee55de4b1038c4002e0adecdf1839>@@V<lambda_dc504788e8f1664fe9b84e20bfb512f2>@@@?$__crt_seh_guarded_call@X@@QEAAX$$QEAV<lambda_0ae27a3a962d80f24befdcbee591983d>@@AEAV<lambda_8d0ee55de4b1038c4002e0adecdf1839>@@$$QEAV<lambda_dc504788e8f1664fe9b84e20bfb512f2>@@@Z 000000018005946c     libucrt:per_thread_data.obj
 0001:00058490       $unwind$??$?RV<lambda_aa87e3671a710a21b5dc78c0bdf72e11>@@AEAV<lambda_92619d2358a28f41a33ba319515a20b9>@@V<lambda_6992ecaafeb10aed2b74cb1fae11a551>@@@?$__crt_seh_guarded_call@X@@QEAAX$$QEAV<lambda_aa87e3671a710a21b5dc78c0bdf72e11>@@AEAV<lambda_92619d2358a28f41a33ba319515a20b9>@@$$QEAV<lambda_6992ecaafeb10aed2b74cb1fae11a551>@@@Z 0000000180059490     libucrt:per_thread_data.obj
 0001:000584b4       $unwind$??$?RV<lambda_f2e299630e499de9f9a165e60fcd3db5>@@AEAV<lambda_2ae9d31cdba2644fcbeaf08da7c24588>@@V<lambda_40d01ff24d0e7b3814fdbdcee8eab3c7>@@@?$__crt_seh_guarded_call@X@@QEAAX$$QEAV<lambda_f2e299630e499de9f9a165e60fcd3db5>@@AEAV<lambda_2ae9d31cdba2644fcbeaf08da7c24588>@@$$QEAV<lambda_40d01ff24d0e7b3814fdbdcee8eab3c7>@@@Z 00000001800594b4     libucrt:per_thread_data.obj
 0001:000584d8       $unwind$??$?RV<lambda_2d41944a1d46af3157314b8a01080d33>@@AEAV<lambda_8f455de75cd7d7f24b4096f044d8b9e6>@@V<lambda_aa500f224e6afead328df44964fe2772>@@@?$__crt_seh_guarded_call@X@@QEAAX$$QEAV<lambda_2d41944a1d46af3157314b8a01080d33>@@AEAV<lambda_8f455de75cd7d7f24b4096f044d8b9e6>@@$$QEAV<lambda_aa500f224e6afead328df44964fe2772>@@@Z 00000001800594d8     libucrt:per_thread_data.obj
 0001:000584fc       $unwind$__acrt_EnumSystemLocalesEx 00000001800594fc     libucrt:winapi_thunks.obj
 0001:0005850c       $unwind$?fp_format_e@@YAHQEBNQEAD_K12H_NIQEAU__crt_locale_pointers@@@Z 000000018005950c     libucrt:cvt.obj
 0001:0005850c       $unwind$_mbtowc_l          000000018005950c     libucrt:mbtowc.obj
 0001:0005850c       $unwind$__acrt_LCMapStringEx 000000018005950c     libucrt:winapi_thunks.obj
 0001:0005850c       $unwind$__acrt_LCMapStringW 000000018005950c     libucrt:lcmapstringw.obj
 0001:00058520       $unwind$??$?RV<lambda_48fc4a32460bb0512d3b13f8499328be>@@AEAV<lambda_6c3dac0a4f3f9cefca9bb494422f9b77>@@V<lambda_0a2f2c9f9a56eb2b08bfa6ff61d331c5>@@@?$__crt_seh_guarded_call@H@@QEAAH$$QEAV<lambda_48fc4a32460bb0512d3b13f8499328be>@@AEAV<lambda_6c3dac0a4f3f9cefca9bb494422f9b77>@@$$QEAV<lambda_0a2f2c9f9a56eb2b08bfa6ff61d331c5>@@@Z 0000000180059520     libucrt:winapi_thunks.obj
 0001:00058544       $unwind$_fcloseall         0000000180059544     libucrt:closeall.obj
 0001:00058568       $unwind$?common_flush_all@@YAH_N@Z 0000000180059568     libucrt:fflush.obj
 0001:00058570       $unwind$??$?RV<lambda_842d9ff0dc9ef11c61343bbaebe7f885>@@AEAV<lambda_c5860995281e5c4ce005b3de8f5874ee>@@V<lambda_d90129c13df834fdcbf8d2b88dafcf2d>@@@?$__crt_seh_guarded_call@X@@QEAAX$$QEAV<lambda_842d9ff0dc9ef11c61343bbaebe7f885>@@AEAV<lambda_c5860995281e5c4ce005b3de8f5874ee>@@$$QEAV<lambda_d90129c13df834fdcbf8d2b88dafcf2d>@@@Z 0000000180059570     libucrt:fflush.obj
 0001:00058594       $unwind$??$?RV<lambda_886d6c58226a84441f68b9f2b8217b83>@@AEAV<lambda_ab61a845afdef5b7c387490eaf3616ee>@@V<lambda_f7f22ab5edc0698d5f6905b0d3f44752>@@@?$__crt_seh_guarded_call@X@@QEAAX$$QEAV<lambda_886d6c58226a84441f68b9f2b8217b83>@@AEAV<lambda_ab61a845afdef5b7c387490eaf3616ee>@@$$QEAV<lambda_f7f22ab5edc0698d5f6905b0d3f44752>@@@Z 0000000180059594     libucrt:fflush.obj
 0001:000585bc       $unwind$__acrt_initialize_lowio 00000001800595bc     libucrt:ioinit.obj
 0001:000585dc       $unwind$?initialize_inherited_file_handles_nolock@@YAXXZ 00000001800595dc     libucrt:ioinit.obj
 0001:000585f8       $unwind$_write             00000001800595f8     libucrt:write.obj
 0001:00058628       $unwind$_write_nolock      0000000180059628     libucrt:write.obj
 0001:00058640       $unwind$?write_double_translated_ansi_nolock@@YA?AUwrite_result@?A0x17268360@@HQEBDI@Z 0000000180059640     libucrt:write.obj
 0001:00058664       $unwind$?write_text_ansi_nolock@@YA?AUwrite_result@?A0x17268360@@HQEBDI@Z 0000000180059664     libucrt:write.obj
 0001:00058664       $unwind$?write_text_utf16le_nolock@@YA?AUwrite_result@?A0x17268360@@HQEBDI@Z 0000000180059664     libucrt:write.obj
 0001:00058684       $unwind$?write_text_utf8_nolock@@YA?AUwrite_result@?A0x17268360@@HQEBDI@Z 0000000180059684     libucrt:write.obj
 0001:000586a8       $unwind$_wctomb_s_l        00000001800596a8     libucrt:wctomb.obj
 0001:000586b8       $unwind$__acrt_fp_format   00000001800596b8     libucrt:cvt.obj
 0001:000586cc       $unwind$?fp_format_e_internal@@YAHQEAD_KH_NIQEAU_strflt@@2QEAU__crt_locale_pointers@@@Z 00000001800596cc     libucrt:cvt.obj
 0001:000586e4       $unwind$?fp_format_a@@YAHQEBNPEAD_KQEAD2H_NIQEAU__crt_locale_pointers@@@Z 00000001800596e4     libucrt:cvt.obj
 0001:00058700       $unwind$__dcrt_get_narrow_environment_from_os 0000000180059700     libucrt:get_environment_from_os.obj
 0001:00058700       $unwind$?fp_format_f_internal@@YAHQEAD_KHQEAU_strflt@@_NQEAU__crt_locale_pointers@@@Z 0000000180059700     libucrt:cvt.obj
 0001:00058700       $unwind$??$__acrt_wcs_to_mbs_cp@U__crt_win32_buffer_internal_dynamic_resizing@@@@YAHQEB_WAEAV?$__crt_win32_buffer@DU__crt_win32_buffer_internal_dynamic_resizing@@@@I@Z 0000000180059700     libucrt:argv_wildcards.obj
 0001:00058718       $unwind$?fp_format_g@@YAHQEBNQEAD_K12H_NIQEAU__crt_locale_pointers@@@Z 0000000180059718     libucrt:cvt.obj
 0001:0005872c       $unwind$_wsetlocale        000000018005972c     libucrt:wsetlocale.obj
 0001:00058734       $unwind$_expandlocale      0000000180059734     libucrt:wsetlocale.obj
 0001:00058754       $unwind$_wcscats           0000000180059754     libucrt:wsetlocale.obj
 0001:00058764       $unwind$_wsetlocale_set_cat 0000000180059764     libucrt:wsetlocale.obj
 0001:00058764       $unwind$??$expand_argument_wildcards@D@@YAHQEAD0AEAV?$argument_list@D@?A0x5f5c8891@@@Z 0000000180059764     libucrt:argv_wildcards.obj
 0001:00058788       $unwind$_wsetlocale_get_all 0000000180059788     libucrt:wsetlocale.obj
 0001:00058788       $unwind$??$copy_and_add_argument_to_buffer@D@@YAHQEBD0_KAEAV?$argument_list@D@?A0x5f5c8891@@@Z 0000000180059788     libucrt:argv_wildcards.obj
 0001:000587a4       $unwind$_wsetlocale_nolock 00000001800597a4     libucrt:wsetlocale.obj
 0001:000587c8       $unwind$__acrt_uninitialize_locale 00000001800597c8     libucrt:wsetlocale.obj
 0001:000587c8       $unwind$__acrt_get_sigabrt_handler 00000001800597c8     libucrt:signal.obj
 0001:000587d0       $unwind$??R<lambda_2a444430fde8c29194d880d93eed5e8f>@@QEBA@XZ 00000001800597d0     libucrt:wsetlocale.obj
 0001:000587dc       $unwind$parse_bcp47        00000001800597dc     libucrt:wsetlocale.obj
 0001:00058800       $unwind$??$?RV<lambda_410d79af7f07d98d83a3f525b3859a53>@@AEAV<lambda_3e16ef9562a7dcce91392c22ab16ea36>@@V<lambda_38119f0e861e05405d8a144b9b982f0a>@@@?$__crt_seh_guarded_call@X@@QEAAX$$QEAV<lambda_410d79af7f07d98d83a3f525b3859a53>@@AEAV<lambda_3e16ef9562a7dcce91392c22ab16ea36>@@$$QEAV<lambda_38119f0e861e05405d8a144b9b982f0a>@@@Z 0000000180059800     libucrt:wsetlocale.obj
 0001:00058828       $unwind$??$?RV<lambda_1d892b297fdedeee07ed8124eeb2f2fa>@@AEAV<lambda_ffc046909424fd52df0ac47e64813305>@@V<lambda_01a7098693036236037e7cdb9bca3d73>@@@?$__crt_seh_guarded_call@X@@QEAAX$$QEAV<lambda_1d892b297fdedeee07ed8124eeb2f2fa>@@AEAV<lambda_ffc046909424fd52df0ac47e64813305>@@$$QEAV<lambda_01a7098693036236037e7cdb9bca3d73>@@@Z 0000000180059828     libucrt:wsetlocale.obj
 0001:0005884c       $unwind$??$?RV<lambda_7f2adfce497ff2baa965cd4f576ecfd1>@@AEAV<lambda_2a444430fde8c29194d880d93eed5e8f>@@AEAV<lambda_8dff2cf36a5417162780cd64fa2883ef>@@@?$__crt_seh_guarded_call@X@@QEAAX$$QEAV<lambda_7f2adfce497ff2baa965cd4f576ecfd1>@@AEAV<lambda_2a444430fde8c29194d880d93eed5e8f>@@AEAV<lambda_8dff2cf36a5417162780cd64fa2883ef>@@@Z 000000018005984c     libucrt:wsetlocale.obj
 0001:0005886c       $unwind$_mbstowcs_s_l      000000018005986c     libucrt:mbstowcs.obj
 0001:00058884       $unwind$?_mbstowcs_l_helper@@YA_KPEA_WPEBD_KPEAU__crt_locale_pointers@@@Z 0000000180059884     libucrt:mbstowcs.obj
 0001:0005889c       $unwind$_handle_error      000000018005989c     libucrt:libm_error.obj
 0001:0005889c       $unwind$_handle_errorf     000000018005989c     libucrt:libm_error.obj
 0001:000588bc       $unwind$__acrt_initialize_fma3 00000001800598bc     libucrt:fma3_available.obj
 0001:000588c4       $unwind$_log_special_common 00000001800598c4     libucrt:log_special.obj
 0001:000588d0       $unwind$_powf_special      00000001800598d0     libucrt:pow_special.obj
 0001:000588e0       $unwind$_pow_special       00000001800598e0     libucrt:pow_special.obj
 0001:000588ec       $unwind$?_wcstombs_l_helper@@YA_KPEADPEB_W_KPEAU__crt_locale_pointers@@@Z 00000001800598ec     libucrt:wcstombs.obj
 0001:00058910       $stateUnwindMap$?_wcstombs_l_helper@@YA_KPEADPEB_W_KPEAU__crt_locale_pointers@@@Z 0000000180059910     libucrt:wcstombs.obj
 0001:00058918       $ip2state$?_wcstombs_l_helper@@YA_KPEADPEB_W_KPEAU__crt_locale_pointers@@@Z 0000000180059918     libucrt:wcstombs.obj
 0001:00058928       $unwind$__acrt_GetLocaleInfoA 0000000180059928     libucrt:getlocaleinfoa.obj
 0001:00058948       $unwind$?InternalGetLocaleInfoA@@YAHQEAU__crt_locale_pointers@@QEB_WKQEADH@Z 0000000180059948     libucrt:getlocaleinfoa.obj
 0001:00058970       $unwind$__acrt_GetStringTypeA 0000000180059970     libucrt:getstringtypea.obj
 0001:00058998       $unwind$__acrt_LCMapStringA 0000000180059998     libucrt:lcmapstringa.obj
 0001:000589a8       $unwind$?__acrt_LCMapStringA_stat@@YAHPEAU__crt_locale_pointers@@PEB_WKPEBDHPEADHHH@Z 00000001800599a8     libucrt:lcmapstringa.obj
 0001:000589d0       $unwind$_raise_exc_ex      00000001800599d0     libucrt:fpexcept.obj
 0001:000589e4       $unwind$_ctrlfp            00000001800599e4     libucrt:fpctrl.obj
 0001:00058a0c       $unwind$_isctype_l         0000000180059a0c     libucrt:isctype.obj
 0001:00058a28       $unwind$raise              0000000180059a28     libucrt:signal.obj
 0001:00058a64       $unwind$??$?RV<lambda_450d765d439847d4c735a33c368b5fc0>@@AEAV<lambda_44731a7d0e6d81c3e6aa82d741081786>@@V<lambda_601a2a7da3b7a96e9554ac7215c4b07c>@@@?$__crt_seh_guarded_call@P6AXH@Z@@QEAAP6AXH@Z$$QEAV<lambda_450d765d439847d4c735a33c368b5fc0>@@AEAV<lambda_44731a7d0e6d81c3e6aa82d741081786>@@$$QEAV<lambda_601a2a7da3b7a96e9554ac7215c4b07c>@@@Z 0000000180059a64     libucrt:signal.obj
 0001:00058a88       $unwind$_wcsicmp_l         0000000180059a88     libucrt:wcsicmp.obj
 0001:00058aa0       $unwind$??$common_expand_argv_wildcards@D@@YAHQEAPEADQEAPEAPEAD@Z 0000000180059aa0     libucrt:argv_wildcards.obj
 0001:00058ab8       $unwind$__acrt_GetModuleFileNameA 0000000180059ab8     libucrt:getmodulefilenamea.obj
 0001:00058ad4       $unwind$_setmbcp_nolock    0000000180059ad4     libucrt:mbctype.obj
 0001:00058af4       $unwind$?update_thread_multibyte_data_internal@@YAPEAU__crt_multibyte_data@@QEAU__acrt_ptd@@QEAPEAU1@@Z 0000000180059af4     libucrt:mbctype.obj
 0001:00058b1c       $unwind$?setmbcp_internal@@YAHH_NQEAU__acrt_ptd@@QEAPEAU__crt_multibyte_data@@@Z 0000000180059b1c     libucrt:mbctype.obj
 0001:00058b2c       $unwind$?setSBUpLow@@YAXPEAU__crt_multibyte_data@@@Z 0000000180059b2c     libucrt:mbctype.obj
 0001:00058b48       $unwind$??$?RV<lambda_efdfa57d1f175319df784efa44bb7b81>@@AEAV<lambda_5f0a4c1567f8adc6734073e5d1e1b35c>@@V<lambda_2e8a7d3640ea6ccb4c2413664c2db6fd>@@@?$__crt_seh_guarded_call@X@@QEAAX$$QEAV<lambda_efdfa57d1f175319df784efa44bb7b81>@@AEAV<lambda_5f0a4c1567f8adc6734073e5d1e1b35c>@@$$QEAV<lambda_2e8a7d3640ea6ccb4c2413664c2db6fd>@@@Z 0000000180059b48     libucrt:mbctype.obj
 0001:00058b6c       $unwind$?x_ismbbtype_l@@YAHPEAU__crt_locale_pointers@@IHH@Z 0000000180059b6c     libucrt:ismbbyte.obj
 0001:00058b7c       $unwind$__acrt_update_thread_locale_data 0000000180059b7c     libucrt:locale_refcounting.obj
 0001:00058ba0       $unwind$__acrt_fenv_set_control 0000000180059ba0     libucrt:_fenvutils.obj
 0001:00058bb0       $unwind$fclose             0000000180059bb0     libucrt:fclose.obj
 0001:00058bd4       $unwind$_close             0000000180059bd4     libucrt:close.obj
 0001:00058bd4       $unwind$_commit            0000000180059bd4     libucrt:commit.obj
 0001:00058bdc       $unwind$??$?RV<lambda_a37b2b86f63e897a80ea819b0eb08c01>@@AEAV<lambda_38ce7e780aa69e748d6df282ebc68efe>@@V<lambda_99fb1378e971ab6e7edea83e3a7a83a2>@@@?$__crt_seh_guarded_call@H@@QEAAH$$QEAV<lambda_a37b2b86f63e897a80ea819b0eb08c01>@@AEAV<lambda_38ce7e780aa69e748d6df282ebc68efe>@@$$QEAV<lambda_99fb1378e971ab6e7edea83e3a7a83a2>@@@Z 0000000180059bdc     libucrt:commit.obj
 0001:00058c00       $unwind$?__mbsrtowcs_utf8@__crt_mbstring@@YA_KPEA_WPEAPEBD_KPEAU_Mbstatet@@@Z 0000000180059c00     libucrt:mbrtowc.obj
 0001:00058c18       $unwind$_putwch_nolock     0000000180059c18     libucrt:putwch.obj
 0001:00058c20       $unwind$__acrt_fltout      0000000180059c20     libucrt:cfout.obj
 0001:00058c40       $unwind$__acrt_locale_initialize_monetary 0000000180059c40     libucrt:initmon.obj
 0001:00058c40       $unwind$?initialize_lc_time@@YA_NQEAU__crt_lc_time_data@@QEAU__crt_locale_data@@@Z 0000000180059c40     libucrt:inittime.obj
 0001:00058c5c       $unwind$__acrt_locale_free_monetary 0000000180059c5c     libucrt:initmon.obj
 0001:00058c64       $unwind$__acrt_locale_free_time 0000000180059c64     libucrt:inittime.obj
 0001:00058c74       $unwind$__acrt_get_qualified_locale 0000000180059c74     libucrt:get_qualified_locale.obj
 0001:00058c90       $unwind$LangCountryEnumProcEx 0000000180059c90     libucrt:get_qualified_locale.obj
 0001:00058cb0       $unwind$LanguageEnumProcEx 0000000180059cb0     libucrt:get_qualified_locale.obj
 0001:00058ccc       $unwind$GetLocaleNameFromDefault 0000000180059ccc     libucrt:get_qualified_locale.obj
 0001:00058ce4       $unwind$TestDefaultCountry 0000000180059ce4     libucrt:get_qualified_locale.obj
 0001:00058cf4       $unwind$__acrt_get_qualified_locale_downlevel 0000000180059cf4     libucrt:getqloc_downlevel.obj
 0001:00058d10       $unwind$LangCountryEnumProc 0000000180059d10     libucrt:getqloc_downlevel.obj
 0001:00058d30       $unwind$LanguageEnumProc   0000000180059d30     libucrt:getqloc_downlevel.obj
 0001:00058d4c       $unwind$CountryEnumProc    0000000180059d4c     libucrt:getqloc_downlevel.obj
 0001:00058d6c       $unwind$?__wcsrtombs_utf8@__crt_mbstring@@YA_KPEADPEAPEB_W_KPEAU_Mbstatet@@@Z 0000000180059d6c     libucrt:wcrtomb.obj
 0001:00058d90       $xdatasym                  0000000180059d90     libucrt:fpsr.obj
 0001:00058d98       $unwind$_towlower_l        0000000180059d98     libucrt:towlower.obj
 0001:00058da0       $unwind$qsort              0000000180059da0     libucrt:qsort.obj
 0001:00058db8       $chain$4$qsort             0000000180059db8     libucrt:qsort.obj
 0001:00058ddc       $chain$5$qsort             0000000180059ddc     libucrt:qsort.obj
 0001:00058dec       $unwind$fallbackMethod     0000000180059dec     libucrt:strpbrk.obj
 0001:00058dfc       $unwind$_mbsdec_l          0000000180059dfc     libucrt:mbsdec.obj
 0001:00058e08       $unwind$_wcsnicmp_l        0000000180059e08     libucrt:wcsnicmp.obj
 0001:00058e24       $unwind$??$?RV<lambda_751a882b2c74d4b022dec766aa51a29a>@@AEAV<lambda_628dfdc04ba53c8bfc02c9951375f3f5>@@V<lambda_f6c7be5f7998530c34de24c7437d6b54>@@@?$__crt_seh_guarded_call@H@@QEAAH$$QEAV<lambda_751a882b2c74d4b022dec766aa51a29a>@@AEAV<lambda_628dfdc04ba53c8bfc02c9951375f3f5>@@$$QEAV<lambda_f6c7be5f7998530c34de24c7437d6b54>@@@Z 0000000180059e24     libucrt:close.obj
 0001:00058e48       $unwind$?__mbrtoc32_utf8@__crt_mbstring@@YA_KPEA_UPEBD_KPEAU_Mbstatet@@@Z 0000000180059e48     libucrt:mbrtoc32.obj
 0001:00058e64       $unwind$_IsNonwritableInCurrentImage 0000000180059e64     LIBCMT:pesect.obj
 0001:00059260       .edata                     000000018005a260     ProcList.exp
 0001:00059288       rgpv                       000000018005a288     ProcList.exp
 0001:000592c4       rgszName                   000000018005a2c4     ProcList.exp
 0001:00059300       rgwOrd                     000000018005a300     ProcList.exp
 0001:0005931e       szName                     000000018005a31e     ProcList.exp
 0001:0005932b       $N00001                    000000018005a32b     ProcList.exp
 0001:00059337       $N00002                    000000018005a337     ProcList.exp
 0001:00059340       $N00003                    000000018005a340     ProcList.exp
 0001:0005934b       $N00004                    000000018005a34b     ProcList.exp
 0001:00059358       $N00005                    000000018005a358     ProcList.exp
 0001:00059361       $N00006                    000000018005a361     ProcList.exp
 0001:0005936f       $N00007                    000000018005a36f     ProcList.exp
 0001:00059379       $N00008                    000000018005a379     ProcList.exp
 0001:00059386       $N00009                    000000018005a386     ProcList.exp
 0001:00059395       $N00010                    000000018005a395     ProcList.exp
 0001:000593a7       $N00011                    000000018005a3a7     ProcList.exp
 0001:000593b6       $N00012                    000000018005a3b6     ProcList.exp
 0001:000593bc       $N00013                    000000018005a3bc     ProcList.exp
 0001:000593cf       $N00014                    000000018005a3cf     ProcList.exp
 0001:000593e2       $N00015                    000000018005a3e2     ProcList.exp
 0002:00000010       ?FKeys@?1??GetOpenPanelInfo@Plist@@QEAAXPEAUOpenPanelInfo@@@Z@4PAGA 000000018005b010     Pclass.obj
 0002:00000058       ?nr@?7??Connect@Plist@@QEAA_NPEB_W00@Z@4U_NETRESOURCEW@@A 000000018005b058     Pclass.obj
 0002:00000100       ?init@std@@3JA             000000018005b100     libcpmt:xlock.obj
 0002:00000108       ?atcount_cdecl@@3_KA       000000018005b108     libcpmt:iosptrs.obj
 0002:00000150       ?__vcrt_flsindex@@3KA      000000018005b150     libvcruntime:per_thread_data.obj
 0002:00000160       ?errno_no_memory@@3HA      000000018005b160     libucrt:errno.obj
 0002:00000164       ?doserrno_no_memory@@3KA   000000018005b164     libucrt:errno.obj
 0002:00000350       ?__acrt_flsindex@@3KA      000000018005b350     libucrt:per_thread_data.obj
 0002:00000358       _ctype_loc_style           000000018005b358     libucrt:wsetlocale.obj
 0002:000004d4       ?dazSupported@?1??_ctrlfp@@9@9 000000018005b4d4     libucrt:fpctrl.obj
 0002:000004e0       ?tzstd_program@@3PADA      000000018005b4e0     libucrt:timeset.obj
 0002:00000520       ?tzdst_program@@3PADA      000000018005b520     libucrt:timeset.obj
 0002:00000560       ?tzname_states@@3PAY01PEADA 000000018005b560     libucrt:timeset.obj
 0002:000007a0       _mbctypes                  000000018005b7a0     libucrt:mbctype.obj
 0002:000008b0       _mbcasemaps                000000018005b8b0     libucrt:mbctype.obj
 0002:000009b0       ?__rgctypeflag@@3PADA      000000018005b9b0     libucrt:mbctype.obj
 0002:000009c0       ?__rgcode_page_info@@3PAUcode_page_info@@A 000000018005b9c0     libucrt:mbctype.obj
 0002:00000bb0       ?__dcrt_lowio_console_output_handle@@3PEAXEA 000000018005bbb0     libucrt:initcon.obj
 0002:00000d00       ??_R0?AV<lambda_87e110110aa5c29eaf754372c3484d5b>@@@8 000000018005bd00     Plist.obj
 0002:00000d40       ??_R0?AV<lambda_6ecd11d6a952986d4bf89c34edf08f5f>@@@8 000000018005bd40     WMI.obj
 0002:00000d80       ??_R0?AV<lambda_aac7a801b46524f039ecb4f6852a8dbe>@@@8 000000018005bd80     WMI.obj
 0002:00000fe0       ?UserAccountID@?1??GetUserAccountID@@YA@XZ@4V?$basic_string@_WU?$char_traits@_W@std@@V?$allocator@_W@2@@std@@B 000000018005bfe0     handles.obj
 0002:00001000       ?$S1@?1??GetUserAccountID@@YA@XZ@4IA 000000018005c000     handles.obj
 0002:00001010       ?TitlesLocal@?1??PanelModes@Plist@@QEAAPEAUPanelMode@@AEA_K@Z@4V?$array@V?$array@PEA_W$0BI@@std@@$09@std@@A 000000018005c010     Pclass.obj
 0002:00001790       ?TitlesRemote@?1??PanelModes@Plist@@QEAAPEAUPanelMode@@AEA_K@Z@4V?$array@V?$array@PEA_W$0BI@@std@@$09@std@@A 000000018005c790     Pclass.obj
 0002:00001f10       ?PanelModesLocal@?1??PanelModes@Plist@@QEAAPEAUPanelMode@@AEA_K@Z@4V?$array@UPanelMode@@$09@std@@A 000000018005cf10     Pclass.obj
 0002:000020f0       ?PanelModesRemote@?1??PanelModes@Plist@@QEAAPEAUPanelMode@@AEA_K@Z@4V?$array@UPanelMode@@$09@std@@A 000000018005d0f0     Pclass.obj
 0002:000022d0       ?ArraysInited@?2??PanelModes@Plist@@QEAAPEAUPanelMode@@AEA_K@Z@4_NA 000000018005d2d0     Pclass.obj
 0002:000022d8       ?Title@?1??GetOpenPanelInfo@Plist@@QEAAXPEAUOpenPanelInfo@@@Z@4V?$basic_string@_WU?$char_traits@_W@std@@V?$allocator@_W@2@@std@@A 000000018005d2d8     Pclass.obj
 0002:000022f8       ?$S1@?1??GetOpenPanelInfo@Plist@@QEAAXPEAUOpenPanelInfo@@@Z@4IA 000000018005d2f8     Pclass.obj
 0002:00002300       ?kbl@?1??GetOpenPanelInfo@Plist@@QEAAXPEAUOpenPanelInfo@@@Z@4PAUKeyBarLabel@@A 000000018005d300     Pclass.obj
 0002:00002408       ?kbt@?1??GetOpenPanelInfo@Plist@@QEAAXPEAUOpenPanelInfo@@@Z@4UKeyBarTitles@@A 000000018005d408     Pclass.obj
 0002:00002418       ?$S2@?1??GetOpenPanelInfo@Plist@@QEAAXPEAUOpenPanelInfo@@@Z@4IA 000000018005d418     Pclass.obj
 0002:00002420       ?Styles@?1??window_style@@YA@PEAUHWND__@@@Z@4QBU?$pair@HPEB_W@std@@B 000000018005d420     Pclass.obj
 0002:00002520       ?$S3@?1??window_style@@YA@PEAUHWND__@@@Z@4IA 000000018005d520     Pclass.obj
 0002:00002530       ?ExtStyles@?1??window_ex_style@@YA@PEAUHWND__@@@Z@4QBU?$pair@HPEB_W@std@@B 000000018005d530     Pclass.obj
 0002:00002670       ?$S5@?1??window_ex_style@@YA@PEAUHWND__@@@Z@4IA 000000018005d670     Pclass.obj
 0002:00002678       ?hDebugToken@@3V?$unique_ptr@XUhandle_closer@@@std@@A 000000018005d678     Plist.obj
 0002:00002948       ?Inited@?1??dynamic_bind@@YAXXZ@4_NA 000000018005d948     Proclist.obj
 0002:00002950       ?PluginMenuStrings@?4??GetPluginInfoW@@9@4PAPEB_WA 000000018005d950     Proclist.obj
 0002:00002958       ?DiskMenuStrings@?7??GetPluginInfoW@@9@4PAPEB_WA 000000018005d958     Proclist.obj
 0002:00002960       ?PluginCfgStrings@?1??GetPluginInfoW@@9@4PAPEB_WA 000000018005d960     Proclist.obj
 0002:00002970       ?initlocks@std@@3V_Init_locks@1@A 000000018005d970     libcpmt:xlock.obj
 0002:00002980       ?mtx@std@@3PAU_RTL_CRITICAL_SECTION@@A 000000018005d980     libcpmt:xlock.obj
 0002:00002af0       ?classic_locale@std@@3Vlocale@1@A 000000018005daf0     libcpmt:locale0.obj
 0002:00002b08       ?_Fac_tidy_reg@std@@3U_Fac_tidy_reg_t@1@B 000000018005db08     libcpmt:locale0.obj
 0002:00002b10       ?_Fac_head@std@@3PEAU_Fac_node@1@EA 000000018005db10     libcpmt:locale0.obj
 0002:00002b18       global_locale              000000018005db18     libcpmt:locale0.obj
 0002:00002b20       ?registered@?1??_Setgloballocale@locale@std@@CAXPEAX@Z@4_NA 000000018005db20     libcpmt:locale0.obj
 0002:00002b80       ?initlocks@std@@3V_Init_locks@1@A 000000018005db80     libcpmt:iosptrs.obj
 0002:00002b81       ?init_atexit@@3U_Init_atexit@@A 000000018005db81     libcpmt:iosptrs.obj
 0002:00002b90       ?atfuns_cdecl@@3PAP6AXXZA  000000018005db90     libcpmt:iosptrs.obj
 0002:00002e18       ?is_initialized_as_dll@@3_NA 000000018005de18     LIBCMT:utility.obj
 0002:00002e19       ?module_local_atexit_table_initialized@@3_NA 000000018005de19     LIBCMT:utility.obj
 0002:00002e20       ?module_local_atexit_table@@3U_onexit_table_t@@A 000000018005de20     LIBCMT:utility.obj
 0002:00002e38       ?module_local_at_quick_exit_table@@3U_onexit_table_t@@A 000000018005de38     LIBCMT:utility.obj
 0002:00002e50       ?__proc_attached@@3HA      000000018005de50     LIBCMT:dll_dllmain.obj
 0002:00002e80       GS_ExceptionRecord         000000018005de80     LIBCMT:gs_report.obj
 0002:00002f20       GS_ContextRecord           000000018005df20     LIBCMT:gs_report.obj
 0002:00003400       ?__vcrt_startup_thread_ptd@@3U__vcrt_ptd@@A 000000018005e400     libvcruntime:per_thread_data.obj
 0002:00003480       __vcrt_lock_table          000000018005e480     libvcruntime:locks.obj
 0002:000034a8       __vcrt_locks_initialized   000000018005e4a8     libvcruntime:locks.obj
 0002:000034f0       ?heap@@3V_HeapManager@@A   000000018005e4f0     libvcruntime:undname.obj
 0002:00003518       ?module_handles@@3PAPEAUHINSTANCE__@@A 000000018005e518     libvcruntime:winapi_downlevel.obj
 0002:00003530       ?function_pointers@@3PAPEAXA 000000018005e530     libvcruntime:winapi_downlevel.obj
 0002:00003558       ?__acrt_invalid_parameter_handler@@3V?$dual_state_global@P6AXPEB_W00I_K@Z@__crt_state_management@@A 000000018005e558     libucrt:invalid_parameter.obj
 0002:00003580       ?__acrt_lock_table@@3PAU_RTL_CRITICAL_SECTION@@A 000000018005e580     libucrt:locks.obj
 0002:000037b0       ?__acrt_locks_initialized@@3IA 000000018005e7b0     libucrt:locks.obj
 0002:000037b4       ?c_termination_complete@@3JA 000000018005e7b4     libucrt:exit.obj
 0002:000037b8       ?thread_local_exit_callback_func@@3P6AXPEAXK0@ZEA 000000018005e7b8     libucrt:exit.obj
 0002:000037d0       ?program_name@?1???$common_configure_argv@D@@YAHW4_crt_argv_mode@@@Z@4PADA 000000018005e7d0     libucrt:argv_parsing.obj
 0002:00003928       ?__acrt_new_handler@@3V?$dual_state_global@P6AH_K@Z@__crt_state_management@@A 000000018005e928     libucrt:new_handler.obj
 0002:00003930       ?module_handles@@3PAPEAUHINSTANCE__@@A 000000018005e930     libucrt:winapi_thunks.obj
 0002:000039d0       ?encoded_function_pointers@@3PAPEAXA 000000018005e9d0     libucrt:winapi_thunks.obj
 0002:00003ae0       ?static_enum_proc@?1??enum_system_locales_ex_nolock@@YAHQ6AHPEA_WK_J@Z@Z@4P6AH0K1@ZEA 000000018005eae0     libucrt:winapi_thunks.obj
 0002:00003f08       ?internal_state@?1??_mbtowc_l@@9@4U_Mbstatet@@A 000000018005ef08     libucrt:mbtowc.obj
 0002:00003f10       ?enable_percent_n@@3_KA    000000018005ef10     libucrt:printf_count_output.obj
 0002:00003f28       ?__acrt_app_type@@3W4_crt_app_type@@A 000000018005ef28     libucrt:report_runtime_error.obj
 0002:00003f38       ?ctrlc_action@@3V?$dual_state_global@P6AXH@Z@__crt_state_management@@A 000000018005ef38     libucrt:signal.obj
 0002:00003f40       ?ctrlbreak_action@@3V?$dual_state_global@P6AXH@Z@__crt_state_management@@A 000000018005ef40     libucrt:signal.obj
 0002:00003f48       ?abort_action@@3V?$dual_state_global@P6AXH@Z@__crt_state_management@@A 000000018005ef48     libucrt:signal.obj
 0002:00003f50       ?term_action@@3V?$dual_state_global@P6AXH@Z@__crt_state_management@@A 000000018005ef50     libucrt:signal.obj
 0002:00003f68       ?_tzname@@3V?$dual_state_global@PEAPEAD@__crt_state_management@@A 000000018005ef68     libucrt:timeset.obj
 0002:00003f70       ?tz_api_used@@3HA          000000018005ef70     libucrt:tzset.obj
 0002:00003f80       ?tz_info@@3U_TIME_ZONE_INFORMATION@@A 000000018005ef80     libucrt:tzset.obj
 0002:00004048       ?fSystemSet@@3HA           000000018005f048     libucrt:mbctype.obj
 0002:0000404c       ?initialized@?1??__acrt_initialize_multibyte@@9@4_NA 000000018005f04c     libucrt:mbctype.obj
 0002:00004088       ?user_matherr@@3V?$dual_state_global@P6AHPEAU_exception@@@Z@__crt_state_management@@A 000000018005f088     libucrt:matherr.obj
 0002:00004090       ?__acrt_global_new_mode@@3V?$dual_state_global@J@__crt_state_management@@A 000000018005f090     libucrt:new_mode.obj
 0002:00004098       ?internal_pst@?1??__mbrtoc32_utf8@__crt_mbstring@@YA_KPEA_UPEBD_KPEAU_Mbstatet@@@Z@4U3@A 000000018005f098     libucrt:mbrtoc32.obj
 0002:000040a0       ?internal_pst@?1??__c16rtomb_utf8@__crt_mbstring@@YA_KPEAD_SPEAU_Mbstatet@@@Z@4U3@A 000000018005f0a0     libucrt:c16rtomb.obj
 0003:0000000c       $pdata$?deallocate@?$allocator@_W@std@@QEAAXQEA_W_K@Z 000000018006000c     fileio.obj
 0003:00000018       $pdata$??1?$basic_string@_WU?$char_traits@_W@std@@V?$allocator@_W@2@@std@@QEAA@XZ 0000000180060018     fileio.obj
 0003:00000018       $pdata$?_Tidy_deallocate@?$basic_string@_WU?$char_traits@_W@std@@V?$allocator@_W@2@@std@@AEAAXXZ 0000000180060018     fileio.obj
 0003:00000024       $pdata$??1columns@@QEAA@XZ 0000000180060024     fileio.obj
 0003:00000030       $pdata$??1mode@@QEAA@XZ    0000000180060030     fileio.obj
 0003:0000003c       $pdata$??1?$vector@Umode@@V?$allocator@Umode@@@std@@@std@@QEAA@XZ 000000018006003c     fileio.obj
 0003:00000048       $pdata$0$??1?$vector@Umode@@V?$allocator@Umode@@@std@@@std@@QEAA@XZ 0000000180060048     fileio.obj
 0003:00000054       $pdata$1$??1?$vector@Umode@@V?$allocator@Umode@@@std@@@std@@QEAA@XZ 0000000180060054     fileio.obj
 0003:00000060       $pdata$2$??1?$vector@Umode@@V?$allocator@Umode@@@std@@@std@@QEAA@XZ 0000000180060060     fileio.obj
 0003:0000006c       $pdata$3$??1?$vector@Umode@@V?$allocator@Umode@@@std@@@std@@QEAA@XZ 000000018006006c     fileio.obj
 0003:00000078       $pdata$?WriteToFile@@YA_KPEAXAEBV?$basic_string_view@_WU?$char_traits@_W@std@@@std@@@Z 0000000180060078     fileio.obj
 0003:00000084       $pdata$?WriteToFile@@YA_KPEAX_W@Z 0000000180060084     fileio.obj
 0003:00000090       $pdata$??$_Destroy_range@V?$allocator@Umode@@@std@@@std@@YAXPEAUmode@@QEAU1@AEAV?$allocator@Umode@@@0@@Z 0000000180060090     fileio.obj
 0003:0000009c       $pdata$0$??$_Destroy_range@V?$allocator@Umode@@@std@@@std@@YAXPEAUmode@@QEAU1@AEAV?$allocator@Umode@@@0@@Z 000000018006009c     fileio.obj
 0003:000000a8       $pdata$1$??$_Destroy_range@V?$allocator@Umode@@@std@@@std@@YAXPEAUmode@@QEAU1@AEAV?$allocator@Umode@@@0@@Z 00000001800600a8     fileio.obj
 0003:000000b4       $pdata$??0exception@std@@QEAA@AEBV01@@Z 00000001800600b4     format.obj
 0003:000000c0       $pdata$??_Gbad_alloc@std@@UEAAPEAXI@Z 00000001800600c0     format.obj
 0003:000000c0       $pdata$??_Gbad_array_new_length@std@@UEAAPEAXI@Z 00000001800600c0     format.obj
 0003:000000c0       $pdata$??_Gbad_cast@std@@UEAAPEAXI@Z 00000001800600c0     format.obj
 0003:000000c0       $pdata$??_Gexception@std@@UEAAPEAXI@Z 00000001800600c0     format.obj
 0003:000000c0       $pdata$??_Gformat_error@v6@fmt@@UEAAPEAXI@Z 00000001800600c0     format.obj
 0003:000000c0       $pdata$??_Gruntime_error@std@@UEAAPEAXI@Z 00000001800600c0     format.obj
 0003:000000c0       $pdata$??_Gbad_function_call@std@@UEAAPEAXI@Z 00000001800600c0     libcpmt:xthrow.obj
 0003:000000c0       $pdata$??_Glength_error@std@@UEAAPEAXI@Z 00000001800600c0     libcpmt:xthrow.obj
 0003:000000c0       $pdata$??_Glogic_error@std@@UEAAPEAXI@Z 00000001800600c0     libcpmt:xthrow.obj
 0003:000000c0       $pdata$??_Gout_of_range@std@@UEAAPEAXI@Z 00000001800600c0     libcpmt:xthrow.obj
 0003:000000c0       $pdata$??_Gbad_exception@std@@UEAAPEAXI@Z 00000001800600c0     libvcruntime:frame.obj
 0003:000000cc       $pdata$??0bad_alloc@std@@QEAA@AEBV01@@Z 00000001800600cc     format.obj
 0003:000000d8       $pdata$??0bad_array_new_length@std@@QEAA@AEBV01@@Z 00000001800600d8     format.obj
 0003:000000e4       $pdata$?_Throw_bad_array_new_length@std@@YAXXZ 00000001800600e4     format.obj
 0003:000000e4       $pdata$?__scrt_throw_std_bad_array_new_length@@YAXXZ 00000001800600e4     LIBCMT:throw_bad_alloc.obj
 0003:000000f0       $pdata$??0bad_cast@std@@QEAA@AEBV01@@Z 00000001800600f0     format.obj
 0003:000000fc       $pdata$?_Throw_bad_cast@std@@YAXXZ 00000001800600fc     format.obj
 0003:00000108       $pdata$??1?$basic_string@DU?$char_traits@D@std@@V?$allocator@D@2@@std@@QEAA@XZ 0000000180060108     format.obj
 0003:00000114       $pdata$?assign@?$basic_string@DU?$char_traits@D@std@@V?$allocator@D@2@@std@@QEAAAEAV12@QEBD_K@Z 0000000180060114     format.obj
 0003:00000120       $pdata$0$?assign@?$basic_string@DU?$char_traits@D@std@@V?$allocator@D@2@@std@@QEAAAEAV12@QEBD_K@Z 0000000180060120     format.obj
 0003:0000012c       $pdata$1$?assign@?$basic_string@DU?$char_traits@D@std@@V?$allocator@D@2@@std@@QEAAAEAV12@QEBD_K@Z 000000018006012c     format.obj
 0003:00000138       $pdata$2$?assign@?$basic_string@DU?$char_traits@D@std@@V?$allocator@D@2@@std@@QEAAAEAV12@QEBD_K@Z 0000000180060138     format.obj
 0003:00000144       $pdata$3$?assign@?$basic_string@DU?$char_traits@D@std@@V?$allocator@D@2@@std@@QEAAAEAV12@QEBD_K@Z 0000000180060144     format.obj
 0003:00000150       $pdata$?_Xlen@?$basic_string@DU?$char_traits@D@std@@V?$allocator@D@2@@std@@CAXXZ 0000000180060150     format.obj
 0003:00000150       $pdata$?_Xlen@?$basic_string@_WU?$char_traits@_W@std@@V?$allocator@_W@2@@std@@CAXXZ 0000000180060150     format.obj
 0003:0000015c       $pdata$?allocate@?$allocator@_W@std@@QEAAPEA_W_K@Z 000000018006015c     format.obj
 0003:00000168       $pdata$?assign@?$basic_string@_WU?$char_traits@_W@std@@V?$allocator@_W@2@@std@@QEAAAEAV12@QEB_W_K@Z 0000000180060168     format.obj
 0003:00000174       $pdata$??0runtime_error@std@@QEAA@PEBD@Z 0000000180060174     format.obj
 0003:00000180       $pdata$??0runtime_error@std@@QEAA@AEBV01@@Z 0000000180060180     format.obj
 0003:0000018c       $pdata$??_G_Facet_base@std@@UEAAPEAXI@Z 000000018006018c     format.obj
 0003:00000198       $pdata$??1_Locinfo@std@@QEAA@XZ 0000000180060198     format.obj
 0003:000001a4       $pdata$??1?$_Yarn@D@std@@QEAA@XZ 00000001800601a4     format.obj
 0003:000001a4       $pdata$??1?$_Yarn@_W@std@@QEAA@XZ 00000001800601a4     format.obj
 0003:000001b0       $pdata$??1locale@std@@QEAA@XZ 00000001800601b0     format.obj
 0003:000001bc       $pdata$??$_Maklocstr@D@std@@YAPEADPEBDPEADAEBU_Cvtvec@@@Z 00000001800601bc     format.obj
 0003:000001c8       $pdata$?on_error@error_handler@detail@v6@fmt@@QEAAXPEBD@Z 00000001800601c8     format.obj
 0003:000001d4       $pdata$??0format_error@v6@fmt@@QEAA@AEBV012@@Z 00000001800601d4     format.obj
 0003:000001e0       $pdata$??$grouping_impl@_W@detail@v6@fmt@@YA?AV?$basic_string@DU?$char_traits@D@std@@V?$allocator@D@2@@std@@Vlocale_ref@012@@Z 00000001800601e0     format.obj
 0003:000001ec       $pdata$??$thousands_sep_impl@_W@detail@v6@fmt@@YA_WVlocale_ref@012@@Z 00000001800601ec     format.obj
 0003:000001f8       $pdata$??$decimal_point_impl@_W@detail@v6@fmt@@YA_WVlocale_ref@012@@Z 00000001800601f8     format.obj
 0003:00000204       $pdata$?grow@?$basic_memory_buffer@_W$0BPE@V?$allocator@_W@std@@@v6@fmt@@MEAAX_K@Z 0000000180060204     format.obj
 0003:00000210       $pdata$??1?$basic_memory_buffer@_W$0BPE@V?$allocator@_W@std@@@v6@fmt@@UEAA@XZ 0000000180060210     format.obj
 0003:0000021c       $pdata$??_G?$basic_memory_buffer@_W$0BPE@V?$allocator@_W@std@@@v6@fmt@@UEAAPEAXI@Z 000000018006021c     format.obj
 0003:00000228       $pdata$?resize@?$buffer@D@detail@v6@fmt@@QEAAX_K@Z 0000000180060228     format.obj
 0003:00000234       $pdata$?grow@?$basic_memory_buffer@D$0BPE@V?$allocator@D@std@@@v6@fmt@@MEAAX_K@Z 0000000180060234     format.obj
 0003:00000240       $pdata$??1?$basic_memory_buffer@D$0BPE@V?$allocator@D@std@@@v6@fmt@@UEAA@XZ 0000000180060240     format.obj
 0003:0000024c       $pdata$??_G?$basic_memory_buffer@D$0BPE@V?$allocator@D@std@@@v6@fmt@@UEAAPEAXI@Z 000000018006024c     format.obj
 0003:00000258       $pdata$??$format_float@N@detail@v6@fmt@@YAHNHUfloat_specs@012@AEAV?$buffer@D@012@@Z 0000000180060258     format.obj
 0003:00000264       $pdata$1$??$format_float@N@detail@v6@fmt@@YAHNHUfloat_specs@012@AEAV?$buffer@D@012@@Z 0000000180060264     format.obj
 0003:00000270       $pdata$2$??$format_float@N@detail@v6@fmt@@YAHNHUfloat_specs@012@AEAV?$buffer@D@012@@Z 0000000180060270     format.obj
 0003:0000027c       $pdata$??$format_float@O@detail@v6@fmt@@YAHOHUfloat_specs@012@AEAV?$buffer@D@012@@Z 000000018006027c     format.obj
 0003:00000288       $pdata$1$??$format_float@O@detail@v6@fmt@@YAHOHUfloat_specs@012@AEAV?$buffer@D@012@@Z 0000000180060288     format.obj
 0003:00000294       $pdata$2$??$format_float@O@detail@v6@fmt@@YAHOHUfloat_specs@012@AEAV?$buffer@D@012@@Z 0000000180060294     format.obj
 0003:000002a0       $pdata$??$snprintf_float@N@detail@v6@fmt@@YAHNHUfloat_specs@012@AEAV?$buffer@D@012@@Z 00000001800602a0     format.obj
 0003:000002ac       $pdata$??$snprintf_float@O@detail@v6@fmt@@YAHOHUfloat_specs@012@AEAV?$buffer@D@012@@Z 00000001800602ac     format.obj
 0003:000002b8       $pdata$?fmt_snprintf@detail@v6@fmt@@YAHPEAD_KPEBDZZ 00000001800602b8     format.obj
 0003:000002c4       $pdata$?grow@?$basic_memory_buffer@I$0CA@V?$allocator@I@std@@@v6@fmt@@MEAAX_K@Z 00000001800602c4     format.obj
 0003:000002d0       $pdata$??1?$basic_memory_buffer@I$0CA@V?$allocator@I@std@@@v6@fmt@@UEAA@XZ 00000001800602d0     format.obj
 0003:000002d0       $pdata$??1bigint@detail@v6@fmt@@QEAA@XZ 00000001800602d0     format.obj
 0003:000002dc       $pdata$??_G?$basic_memory_buffer@I$0CA@V?$allocator@I@std@@@v6@fmt@@UEAAPEAXI@Z 00000001800602dc     format.obj
 0003:000002e8       $pdata$??_3bigint@detail@v6@fmt@@QEAAAEAV0123@H@Z 00000001800602e8     format.obj
 0003:000002f4       $pdata$1$??_3bigint@detail@v6@fmt@@QEAAAEAV0123@H@Z 00000001800602f4     format.obj
 0003:00000300       $pdata$2$??_3bigint@detail@v6@fmt@@QEAAAEAV0123@H@Z 0000000180060300     format.obj
 0003:0000030c       $pdata$?assign_pow10@bigint@detail@v6@fmt@@QEAAXH@Z 000000018006030c     format.obj
 0003:00000318       $pdata$1$?assign_pow10@bigint@detail@v6@fmt@@QEAAXH@Z 0000000180060318     format.obj
 0003:00000324       $pdata$2$?assign_pow10@bigint@detail@v6@fmt@@QEAAXH@Z 0000000180060324     format.obj
 0003:00000330       $pdata$?square@bigint@detail@v6@fmt@@QEAAXXZ 0000000180060330     format.obj
 0003:0000033c       $pdata$??$do_throw@Vformat_error@v6@fmt@@@detail@v6@fmt@@YAXAEBVformat_error@12@@Z 000000018006033c     format.obj
 0003:00000348       $pdata$??$get@Vlocale@std@@@locale_ref@detail@v6@fmt@@QEBA?AVlocale@std@@XZ 0000000180060348     format.obj
 0003:00000354       $pdata$??$_Allocate@$0BA@U_Default_allocate_traits@std@@$0A@@std@@YAPEAX_K@Z 0000000180060354     format.obj
 0003:00000360       $pdata$??$use_facet@V?$numpunct@_W@std@@@std@@YAAEBV?$numpunct@_W@0@AEBVlocale@0@@Z 0000000180060360     format.obj
 0003:0000036c       $pdata$?_Getcat@?$numpunct@_W@std@@SA_KPEAPEBVfacet@locale@2@PEBV42@@Z 000000018006036c     format.obj
 0003:00000378       $pdata$?dtor$0@?0??_Getcat@?$numpunct@_W@std@@SA_KPEAPEBVfacet@locale@2@PEBV42@@Z@4HA 0000000180060378     format.obj
 0003:00000384       $pdata$?dtor$1@?0??_Getcat@?$numpunct@_W@std@@SA_KPEAPEBVfacet@locale@2@PEBV42@@Z@4HA 0000000180060384     format.obj
 0003:00000390       $pdata$?_Init@?$numpunct@_W@std@@IEAAXAEBV_Locinfo@2@_N@Z 0000000180060390     format.obj
 0003:0000039c       $pdata$?do_grouping@?$numpunct@_W@std@@MEBA?AV?$basic_string@DU?$char_traits@D@std@@V?$allocator@D@2@@2@XZ 000000018006039c     format.obj
 0003:000003a8       $pdata$?do_falsename@?$numpunct@_W@std@@MEBA?AV?$basic_string@_WU?$char_traits@_W@std@@V?$allocator@_W@2@@2@XZ 00000001800603a8     format.obj
 0003:000003b4       $pdata$?do_truename@?$numpunct@_W@std@@MEBA?AV?$basic_string@_WU?$char_traits@_W@std@@V?$allocator@_W@2@@2@XZ 00000001800603b4     format.obj
 0003:000003c0       $pdata$??_G?$numpunct@_W@std@@MEAAPEAXI@Z 00000001800603c0     format.obj
 0003:000003cc       $pdata$??$grisu_gen_digits@Ugrisu_shortest_handler@detail@v6@fmt@@@detail@v6@fmt@@YA?AW4result@digits@012@Vfp@012@_KAEAHAEAUgrisu_shortest_handler@012@@Z 00000001800603cc     format.obj
 0003:000003d8       $pdata$??$fallback_format@N@detail@v6@fmt@@YAXNAEAV?$buffer@D@012@AEAH@Z 00000001800603d8     format.obj
 0003:000003d8       $pdata$??$fallback_format@O@detail@v6@fmt@@YAXOAEAV?$buffer@D@012@AEAH@Z 00000001800603d8     format.obj
 0003:000003e4       $pdata$??$grisu_gen_digits@Ufixed_handler@detail@v6@fmt@@@detail@v6@fmt@@YA?AW4result@digits@012@Vfp@012@_KAEAHAEAUfixed_handler@012@@Z 00000001800603e4     format.obj
 0003:000003f0       $pdata$??1?$_Tidy_guard@V?$numpunct@_W@std@@@std@@QEAA@XZ 00000001800603f0     format.obj
 0003:000003fc       $pdata$??0?$basic_string@_WU?$char_traits@_W@std@@V?$allocator@_W@2@@std@@QEAA@AEBV01@@Z 00000001800603fc     handles.obj
 0003:00000408       $pdata$?append@?$basic_string@_WU?$char_traits@_W@std@@V?$allocator@_W@2@@std@@QEAAAEAV12@QEB_W_K@Z 0000000180060408     handles.obj
 0003:00000414       $pdata$0$?append@?$basic_string@_WU?$char_traits@_W@std@@V?$allocator@_W@2@@std@@QEAAAEAV12@QEB_W_K@Z 0000000180060414     handles.obj
 0003:00000420       $pdata$1$?append@?$basic_string@_WU?$char_traits@_W@std@@V?$allocator@_W@2@@std@@QEAAAEAV12@QEB_W_K@Z 0000000180060420     handles.obj
 0003:0000042c       $pdata$2$?append@?$basic_string@_WU?$char_traits@_W@std@@V?$allocator@_W@2@@std@@QEAAAEAV12@QEB_W_K@Z 000000018006042c     handles.obj
 0003:00000438       $pdata$3$?append@?$basic_string@_WU?$char_traits@_W@std@@V?$allocator@_W@2@@std@@QEAAAEAV12@QEB_W_K@Z 0000000180060438     handles.obj
 0003:00000444       $pdata$??1DebugToken@@QEAA@XZ 0000000180060444     handles.obj
 0003:00000450       $pdata$?PrintHandleInfo@@YA_NKPEAX_NPEAVPerfThread@@@Z 0000000180060450     handles.obj
 0003:0000045c       $pdata$?query_object@@YA?AV?$unique_ptr@$$BY0A@DU?$default_delete@$$BY0A@D@std@@@std@@PEAXW4OBJECT_INFORMATION_CLASS@@@Z 000000018006045c     handles.obj
 0003:00000468       $pdata$?GetFileNameThread@test@?4??GetFileName@@YA?AV?$basic_string@_WU?$char_traits@_W@std@@V?$allocator@_W@2@@std@@PEAX@Z@SAK0@Z 0000000180060468     handles.obj
 0003:00000474       $pdata$??R<lambda_c3630acb37279cf92411e07a2b271fdf>@@QEBA?AV?$basic_string@_WU?$char_traits@_W@std@@V?$allocator@_W@2@@std@@XZ 0000000180060474     handles.obj
 0003:00000480       $pdata$??$make_unique@$$BY0A@_W$0A@@std@@YA?AV?$unique_ptr@$$BY0A@_WU?$default_delete@$$BY0A@_W@std@@@0@_K@Z 0000000180060480     handles.obj
 0003:0000048c       $pdata$??__FUserAccountID@?1??GetUserAccountID@@YA@XZ@YAXXZ 000000018006048c     handles.obj
 0003:00000498       $pdata$?GetNameByType@@YA?AV?$basic_string@_WU?$char_traits@_W@std@@V?$allocator@_W@2@@std@@PEAXGPEAVPerfThread@@@Z 0000000180060498     handles.obj
 0003:000004a4       $pdata$?dtor$20@?0??GetNameByType@@YA?AV?$basic_string@_WU?$char_traits@_W@std@@V?$allocator@_W@2@@std@@PEAXGPEAVPerfThread@@@Z@4HA 00000001800604a4     handles.obj
 0003:000004b0       $pdata$??1?$scoped_lock@VPerfThread@@@std@@QEAA@XZ 00000001800604b0     handles.obj
 0003:000004bc       $pdata$?duplicate_handle@@YA?AV?$unique_ptr@XUhandle_closer@@@std@@PEAXK@Z 00000001800604bc     handles.obj
 0003:000004c8       $pdata$??$vformat@_W$0A@@detail@v6@fmt@@YA?AV?$basic_string@_WU?$char_traits@_W@std@@V?$allocator@_W@2@@std@@V?$basic_string_view@_W@12@V?$basic_format_args@V?$basic_format_context@V?$back_insert_iterator@V?$buffer@_W@detail@v6@fmt@@@std@@_W@v6@fmt@@@12@@Z 00000001800604c8     handles.obj
 0003:000004d4       $pdata$?on_fill@?$specs_setter@_W@detail@v6@fmt@@QEAAXV?$basic_string_view@_W@34@@Z 00000001800604d4     handles.obj
 0003:000004e0       $pdata$??$reserve@V?$buffer@_W@detail@v6@fmt@@$0A@@detail@v6@fmt@@YAPEA_WV?$back_insert_iterator@V?$buffer@_W@detail@v6@fmt@@@std@@_K@Z 00000001800604e0     handles.obj
 0003:000004ec       $pdata$?write@?$arg_formatter_base@V?$back_insert_iterator@V?$buffer@_W@detail@v6@fmt@@@std@@_WUerror_handler@detail@v6@fmt@@@detail@v6@fmt@@IEAAX_N@Z 00000001800604ec     handles.obj
 0003:000004f8       $pdata$1$?write@?$arg_formatter_base@V?$back_insert_iterator@V?$buffer@_W@detail@v6@fmt@@@std@@_WUerror_handler@detail@v6@fmt@@@detail@v6@fmt@@IEAAX_N@Z 00000001800604f8     handles.obj
 0003:00000504       $pdata$2$?write@?$arg_formatter_base@V?$back_insert_iterator@V?$buffer@_W@detail@v6@fmt@@@std@@_WUerror_handler@detail@v6@fmt@@@detail@v6@fmt@@IEAAX_N@Z 0000000180060504     handles.obj
 0003:00000510       $pdata$?write@?$arg_formatter_base@V?$back_insert_iterator@V?$buffer@_W@detail@v6@fmt@@@std@@_WUerror_handler@detail@v6@fmt@@@detail@v6@fmt@@IEAAXPEB_W@Z 0000000180060510     handles.obj
 0003:0000051c       $pdata$??$visit_format_arg@U?$default_arg_formatter@V?$back_insert_iterator@V?$buffer@_W@detail@v6@fmt@@@std@@_W@detail@v6@fmt@@V?$basic_format_context@V?$back_insert_iterator@V?$buffer@_W@detail@v6@fmt@@@std@@_W@34@@v6@fmt@@YA?AV?$back_insert_iterator@V?$buffer@_W@detail@v6@fmt@@@std@@$$QEAU?$default_arg_formatter@V?$back_insert_iterator@V?$buffer@_W@detail@v6@fmt@@@std@@_W@detail@01@AEBV?$basic_format_arg@V?$basic_format_context@V?$back_insert_iterator@V?$buffer@_W@detail@v6@fmt@@@std@@_W@v6@fmt@@@01@@Z 000000018006051c     handles.obj
 0003:00000528       $pdata$?on_text@?$format_handler@V?$arg_formatter@V?$back_insert_iterator@V?$buffer@_W@detail@v6@fmt@@@std@@_W@detail@v6@fmt@@_WV?$basic_format_context@V?$back_insert_iterator@V?$buffer@_W@detail@v6@fmt@@@std@@_W@34@@detail@v6@fmt@@QEAAXPEB_W0@Z 0000000180060528     handles.obj
 0003:00000534       $pdata$?on_replacement_field@?$format_handler@V?$arg_formatter@V?$back_insert_iterator@V?$buffer@_W@detail@v6@fmt@@@std@@_W@detail@v6@fmt@@_WV?$basic_format_context@V?$back_insert_iterator@V?$buffer@_W@detail@v6@fmt@@@std@@_W@34@@detail@v6@fmt@@QEAAXHPEB_W@Z 0000000180060534     handles.obj
 0003:00000540       $pdata$?on_format_specs@?$format_handler@V?$arg_formatter@V?$back_insert_iterator@V?$buffer@_W@detail@v6@fmt@@@std@@_W@detail@v6@fmt@@_WV?$basic_format_context@V?$back_insert_iterator@V?$buffer@_W@detail@v6@fmt@@@std@@_W@34@@detail@v6@fmt@@QEAAPEB_WHPEB_W0@Z 0000000180060540     handles.obj
 0003:0000054c       $pdata$??$parse_format_string@$0A@_WAEAU?$format_handler@V?$arg_formatter@V?$back_insert_iterator@V?$buffer@_W@detail@v6@fmt@@@std@@_W@detail@v6@fmt@@_WV?$basic_format_context@V?$back_insert_iterator@V?$buffer@_W@detail@v6@fmt@@@std@@_W@34@@detail@v6@fmt@@@detail@v6@fmt@@YAXV?$basic_string_view@_W@12@AEAU?$format_handler@V?$arg_formatter@V?$back_insert_iterator@V?$buffer@_W@detail@v6@fmt@@@std@@_W@detail@v6@fmt@@_WV?$basic_format_context@V?$back_insert_iterator@V?$buffer@_W@detail@v6@fmt@@@std@@_W@34@@012@@Z 000000018006054c     handles.obj
 0003:00000558       $pdata$??Rwriter@?1???$parse_format_string@$0A@_WAEAU?$format_handler@V?$arg_formatter@V?$back_insert_iterator@V?$buffer@_W@detail@v6@fmt@@@std@@_W@detail@v6@fmt@@_WV?$basic_format_context@V?$back_insert_iterator@V?$buffer@_W@detail@v6@fmt@@@std@@_W@34@@detail@v6@fmt@@@detail@v6@fmt@@YAXV?$basic_string_view@_W@23@AEAU?$format_handler@V?$arg_formatter@V?$back_insert_iterator@V?$buffer@_W@detail@v6@fmt@@@std@@_W@detail@v6@fmt@@_WV?$basic_format_context@V?$back_insert_iterator@V?$buffer@_W@detail@v6@fmt@@@std@@_W@34@@123@@Z@QEAAXPEB_W2@Z 0000000180060558     handles.obj
 0003:00000564       $pdata$0$??Rwriter@?1???$parse_format_string@$0A@_WAEAU?$format_handler@V?$arg_formatter@V?$back_insert_iterator@V?$buffer@_W@detail@v6@fmt@@@std@@_W@detail@v6@fmt@@_WV?$basic_format_context@V?$back_insert_iterator@V?$buffer@_W@detail@v6@fmt@@@std@@_W@34@@detail@v6@fmt@@@detail@v6@fmt@@YAXV?$basic_string_view@_W@23@AEAU?$format_handler@V?$arg_formatter@V?$back_insert_iterator@V?$buffer@_W@detail@v6@fmt@@@std@@_W@detail@v6@fmt@@_WV?$basic_format_context@V?$back_insert_iterator@V?$buffer@_W@detail@v6@fmt@@@std@@_W@34@@123@@Z@QEAAXPEB_W2@Z 0000000180060564     handles.obj
 0003:00000570       $pdata$1$??Rwriter@?1???$parse_format_string@$0A@_WAEAU?$format_handler@V?$arg_formatter@V?$back_insert_iterator@V?$buffer@_W@detail@v6@fmt@@@std@@_W@detail@v6@fmt@@_WV?$basic_format_context@V?$back_insert_iterator@V?$buffer@_W@detail@v6@fmt@@@std@@_W@34@@detail@v6@fmt@@@detail@v6@fmt@@YAXV?$basic_string_view@_W@23@AEAU?$format_handler@V?$arg_formatter@V?$back_insert_iterator@V?$buffer@_W@detail@v6@fmt@@@std@@_W@detail@v6@fmt@@_WV?$basic_format_context@V?$back_insert_iterator@V?$buffer@_W@detail@v6@fmt@@@std@@_W@34@@123@@Z@QEAAXPEB_W2@Z 0000000180060570     handles.obj
 0003:0000057c       $pdata$2$??Rwriter@?1???$parse_format_string@$0A@_WAEAU?$format_handler@V?$arg_formatter@V?$back_insert_iterator@V?$buffer@_W@detail@v6@fmt@@@std@@_W@detail@v6@fmt@@_WV?$basic_format_context@V?$back_insert_iterator@V?$buffer@_W@detail@v6@fmt@@@std@@_W@34@@detail@v6@fmt@@@detail@v6@fmt@@YAXV?$basic_string_view@_W@23@AEAU?$format_handler@V?$arg_formatter@V?$back_insert_iterator@V?$buffer@_W@detail@v6@fmt@@@std@@_W@detail@v6@fmt@@_WV?$basic_format_context@V?$back_insert_iterator@V?$buffer@_W@detail@v6@fmt@@@std@@_W@34@@123@@Z@QEAAXPEB_W2@Z 000000018006057c     handles.obj
 0003:00000588       $pdata$??$write@_WV?$back_insert_iterator@V?$buffer@_W@detail@v6@fmt@@@std@@@detail@v6@fmt@@YA?AV?$back_insert_iterator@V?$buffer@_W@detail@v6@fmt@@@std@@V34@_W@Z 0000000180060588     handles.obj
 0003:00000594       $pdata$??$write@_WV?$back_insert_iterator@V?$buffer@_W@detail@v6@fmt@@@std@@@detail@v6@fmt@@YA?AV?$back_insert_iterator@V?$buffer@_W@detail@v6@fmt@@@std@@V34@_N@Z 0000000180060594     handles.obj
 0003:000005a0       $pdata$??$write@_WV?$back_insert_iterator@V?$buffer@_W@detail@v6@fmt@@@std@@H$0A@@detail@v6@fmt@@YA?AV?$back_insert_iterator@V?$buffer@_W@detail@v6@fmt@@@std@@V34@H@Z 00000001800605a0     handles.obj
 0003:000005ac       $pdata$??$write@_WV?$back_insert_iterator@V?$buffer@_W@detail@v6@fmt@@@std@@I$0A@@detail@v6@fmt@@YA?AV?$back_insert_iterator@V?$buffer@_W@detail@v6@fmt@@@std@@V34@I@Z 00000001800605ac     handles.obj
 0003:000005b8       $pdata$??$write@_WV?$back_insert_iterator@V?$buffer@_W@detail@v6@fmt@@@std@@_J$0A@@detail@v6@fmt@@YA?AV?$back_insert_iterator@V?$buffer@_W@detail@v6@fmt@@@std@@V34@_J@Z 00000001800605b8     handles.obj
 0003:000005c4       $pdata$??$write@_WV?$back_insert_iterator@V?$buffer@_W@detail@v6@fmt@@@std@@_K$0A@@detail@v6@fmt@@YA?AV?$back_insert_iterator@V?$buffer@_W@detail@v6@fmt@@@std@@V34@_K@Z 00000001800605c4     handles.obj
 0003:000005d0       $pdata$??$write@_WV?$back_insert_iterator@V?$buffer@_W@detail@v6@fmt@@@std@@M$0A@@detail@v6@fmt@@YA?AV?$back_insert_iterator@V?$buffer@_W@detail@v6@fmt@@@std@@V34@M@Z 00000001800605d0     handles.obj
 0003:000005dc       $pdata$??$write@_WV?$back_insert_iterator@V?$buffer@_W@detail@v6@fmt@@@std@@N$0A@@detail@v6@fmt@@YA?AV?$back_insert_iterator@V?$buffer@_W@detail@v6@fmt@@@std@@V34@N@Z 00000001800605dc     handles.obj
 0003:000005e8       $pdata$??$write@_WV?$back_insert_iterator@V?$buffer@_W@detail@v6@fmt@@@std@@O$0A@@detail@v6@fmt@@YA?AV?$back_insert_iterator@V?$buffer@_W@detail@v6@fmt@@@std@@V34@O@Z 00000001800605e8     handles.obj
 0003:000005f4       $pdata$??$parse_arg_id@_WAEAU?$id_adapter@AEAU?$format_handler@V?$arg_formatter@V?$back_insert_iterator@V?$buffer@_W@detail@v6@fmt@@@std@@_W@detail@v6@fmt@@_WV?$basic_format_context@V?$back_insert_iterator@V?$buffer@_W@detail@v6@fmt@@@std@@_W@34@@detail@v6@fmt@@_W@detail@v6@fmt@@@detail@v6@fmt@@YAPEB_WPEB_W0AEAU?$id_adapter@AEAU?$format_handler@V?$arg_formatter@V?$back_insert_iterator@V?$buffer@_W@detail@v6@fmt@@@std@@_W@detail@v6@fmt@@_WV?$basic_format_context@V?$back_insert_iterator@V?$buffer@_W@detail@v6@fmt@@@std@@_W@34@@detail@v6@fmt@@_W@012@@Z 00000001800605f4     handles.obj
 0003:00000600       $pdata$?check_sign@?$numeric_specs_checker@V?$specs_handler@V?$basic_format_parse_context@_WUerror_handler@detail@v6@fmt@@@v6@fmt@@V?$basic_format_context@V?$back_insert_iterator@V?$buffer@_W@detail@v6@fmt@@@std@@_W@23@@detail@v6@fmt@@@detail@v6@fmt@@QEAAXXZ 0000000180060600     handles.obj
 0003:0000060c       $pdata$??$parse_format_specs@_WAEAV?$specs_checker@V?$specs_handler@V?$basic_format_parse_context@_WUerror_handler@detail@v6@fmt@@@v6@fmt@@V?$basic_format_context@V?$back_insert_iterator@V?$buffer@_W@detail@v6@fmt@@@std@@_W@23@@detail@v6@fmt@@@detail@v6@fmt@@@detail@v6@fmt@@YAPEB_WPEB_W0AEAV?$specs_checker@V?$specs_handler@V?$basic_format_parse_context@_WUerror_handler@detail@v6@fmt@@@v6@fmt@@V?$basic_format_context@V?$back_insert_iterator@V?$buffer@_W@detail@v6@fmt@@@std@@_W@23@@detail@v6@fmt@@@012@@Z 000000018006060c     handles.obj
 0003:00000618       $pdata$1$??$parse_format_specs@_WAEAV?$specs_checker@V?$specs_handler@V?$basic_format_parse_context@_WUerror_handler@detail@v6@fmt@@@v6@fmt@@V?$basic_format_context@V?$back_insert_iterator@V?$buffer@_W@detail@v6@fmt@@@std@@_W@23@@detail@v6@fmt@@@detail@v6@fmt@@@detail@v6@fmt@@YAPEB_WPEB_W0AEAV?$specs_checker@V?$specs_handler@V?$basic_format_parse_context@_WUerror_handler@detail@v6@fmt@@@v6@fmt@@V?$basic_format_context@V?$back_insert_iterator@V?$buffer@_W@detail@v6@fmt@@@std@@_W@23@@detail@v6@fmt@@@012@@Z 0000000180060618     handles.obj
 0003:00000624       $pdata$3$??$parse_format_specs@_WAEAV?$specs_checker@V?$specs_handler@V?$basic_format_parse_context@_WUerror_handler@detail@v6@fmt@@@v6@fmt@@V?$basic_format_context@V?$back_insert_iterator@V?$buffer@_W@detail@v6@fmt@@@std@@_W@23@@detail@v6@fmt@@@detail@v6@fmt@@@detail@v6@fmt@@YAPEB_WPEB_W0AEAV?$specs_checker@V?$specs_handler@V?$basic_format_parse_context@_WUerror_handler@detail@v6@fmt@@@v6@fmt@@V?$basic_format_context@V?$back_insert_iterator@V?$buffer@_W@detail@v6@fmt@@@std@@_W@23@@detail@v6@fmt@@@012@@Z 0000000180060624     handles.obj
 0003:00000630       $pdata$4$??$parse_format_specs@_WAEAV?$specs_checker@V?$specs_handler@V?$basic_format_parse_context@_WUerror_handler@detail@v6@fmt@@@v6@fmt@@V?$basic_format_context@V?$back_insert_iterator@V?$buffer@_W@detail@v6@fmt@@@std@@_W@23@@detail@v6@fmt@@@detail@v6@fmt@@@detail@v6@fmt@@YAPEB_WPEB_W0AEAV?$specs_checker@V?$specs_handler@V?$basic_format_parse_context@_WUerror_handler@detail@v6@fmt@@@v6@fmt@@V?$basic_format_context@V?$back_insert_iterator@V?$buffer@_W@detail@v6@fmt@@@std@@_W@23@@detail@v6@fmt@@@012@@Z 0000000180060630     handles.obj
 0003:0000063c       $pdata$??$?RH$0A@@?$arg_formatter_base@V?$back_insert_iterator@V?$buffer@_W@detail@v6@fmt@@@std@@_WUerror_handler@detail@v6@fmt@@@detail@v6@fmt@@QEAA?AV?$back_insert_iterator@V?$buffer@_W@detail@v6@fmt@@@std@@H@Z 000000018006063c     handles.obj
 0003:00000648       $pdata$??$visit_format_arg@V?$arg_formatter@V?$back_insert_iterator@V?$buffer@_W@detail@v6@fmt@@@std@@_W@detail@v6@fmt@@V?$basic_format_context@V?$back_insert_iterator@V?$buffer@_W@detail@v6@fmt@@@std@@_W@34@@v6@fmt@@YA?AV?$back_insert_iterator@V?$buffer@_W@detail@v6@fmt@@@std@@$$QEAV?$arg_formatter@V?$back_insert_iterator@V?$buffer@_W@detail@v6@fmt@@@std@@_W@detail@01@AEBV?$basic_format_arg@V?$basic_format_context@V?$back_insert_iterator@V?$buffer@_W@detail@v6@fmt@@@std@@_W@v6@fmt@@@01@@Z 0000000180060648     handles.obj
 0003:00000654       $pdata$??$write_ptr@_WV?$back_insert_iterator@V?$buffer@_W@detail@v6@fmt@@@std@@_K@detail@v6@fmt@@YA?AV?$back_insert_iterator@V?$buffer@_W@detail@v6@fmt@@@std@@V34@_KPEBU?$basic_format_specs@_W@12@@Z 0000000180060654     handles.obj
 0003:00000660       $pdata$2$??$write_ptr@_WV?$back_insert_iterator@V?$buffer@_W@detail@v6@fmt@@@std@@_K@detail@v6@fmt@@YA?AV?$back_insert_iterator@V?$buffer@_W@detail@v6@fmt@@@std@@V34@_KPEBU?$basic_format_specs@_W@12@@Z 0000000180060660     handles.obj
 0003:0000066c       $pdata$3$??$write_ptr@_WV?$back_insert_iterator@V?$buffer@_W@detail@v6@fmt@@@std@@_K@detail@v6@fmt@@YA?AV?$back_insert_iterator@V?$buffer@_W@detail@v6@fmt@@@std@@V34@_KPEBU?$basic_format_specs@_W@12@@Z 000000018006066c     handles.obj
 0003:00000678       $pdata$??$format_decimal@_W_K@detail@v6@fmt@@YA?AU?$format_decimal_result@PEA_W@012@PEA_W_KH@Z 0000000180060678     handles.obj
 0003:00000684       $pdata$0$??$format_decimal@_W_K@detail@v6@fmt@@YA?AU?$format_decimal_result@PEA_W@012@PEA_W_KH@Z 0000000180060684     handles.obj
 0003:00000690       $pdata$1$??$format_decimal@_W_K@detail@v6@fmt@@YA?AU?$format_decimal_result@PEA_W@012@PEA_W_KH@Z 0000000180060690     handles.obj
 0003:0000069c       $pdata$??$write_nonfinite@_WV?$back_insert_iterator@V?$buffer@_W@detail@v6@fmt@@@std@@@detail@v6@fmt@@YA?AV?$back_insert_iterator@V?$buffer@_W@detail@v6@fmt@@@std@@V34@_NAEBU?$basic_format_specs@_W@12@AEBUfloat_specs@012@@Z 000000018006069c     handles.obj
 0003:000006a8       $pdata$??0?$float_writer@_W@detail@v6@fmt@@QEAA@PEBDHHUfloat_specs@123@_W@Z 00000001800606a8     handles.obj
 0003:000006b4       $pdata$?on_char@char_spec_handler@?$arg_formatter_base@V?$back_insert_iterator@V?$buffer@_W@detail@v6@fmt@@@std@@_WUerror_handler@detail@v6@fmt@@@detail@v6@fmt@@QEAAXXZ 00000001800606b4     handles.obj
 0003:000006c0       $pdata$0$?on_char@char_spec_handler@?$arg_formatter_base@V?$back_insert_iterator@V?$buffer@_W@detail@v6@fmt@@@std@@_WUerror_handler@detail@v6@fmt@@@detail@v6@fmt@@QEAAXXZ 00000001800606c0     handles.obj
 0003:000006cc       $pdata$1$?on_char@char_spec_handler@?$arg_formatter_base@V?$back_insert_iterator@V?$buffer@_W@detail@v6@fmt@@@std@@_WUerror_handler@detail@v6@fmt@@@detail@v6@fmt@@QEAAXXZ 00000001800606cc     handles.obj
 0003:000006d8       $pdata$??$get_id@_W@?$basic_format_args@V?$basic_format_context@V?$back_insert_iterator@V?$buffer@_W@detail@v6@fmt@@@std@@_W@v6@fmt@@@v6@fmt@@QEBAHV?$basic_string_view@_W@12@@Z 00000001800606d8     handles.obj
 0003:000006e4       $pdata$5$??$get_id@_W@?$basic_format_args@V?$basic_format_context@V?$back_insert_iterator@V?$buffer@_W@detail@v6@fmt@@@std@@_W@v6@fmt@@@v6@fmt@@QEBAHV?$basic_string_view@_W@12@@Z 00000001800606e4     handles.obj
 0003:000006f0       $pdata$7$??$get_id@_W@?$basic_format_args@V?$basic_format_context@V?$back_insert_iterator@V?$buffer@_W@detail@v6@fmt@@@std@@_W@v6@fmt@@@v6@fmt@@QEBAHV?$basic_string_view@_W@12@@Z 00000001800606f0     handles.obj
 0003:000006fc       $pdata$??$write_int@H@?$arg_formatter_base@V?$back_insert_iterator@V?$buffer@_W@detail@v6@fmt@@@std@@_WUerror_handler@detail@v6@fmt@@@detail@v6@fmt@@AEAAXHAEBU?$basic_format_specs@_W@23@@Z 00000001800606fc     handles.obj
 0003:00000708       $pdata$??$prettify@PEA_W@?$float_writer@_W@detail@v6@fmt@@AEBAPEA_WPEA_W@Z 0000000180060708     handles.obj
 0003:00000714       $pdata$0$??$prettify@PEA_W@?$float_writer@_W@detail@v6@fmt@@AEBAPEA_WPEA_W@Z 0000000180060714     handles.obj
 0003:00000720       $pdata$??$parse_arg_id@_WU?$width_adapter@AEAV?$specs_checker@V?$specs_handler@V?$basic_format_parse_context@_WUerror_handler@detail@v6@fmt@@@v6@fmt@@V?$basic_format_context@V?$back_insert_iterator@V?$buffer@_W@detail@v6@fmt@@@std@@_W@23@@detail@v6@fmt@@@detail@v6@fmt@@_W@detail@v6@fmt@@@detail@v6@fmt@@YAPEB_WPEB_W0$$QEAU?$width_adapter@AEAV?$specs_checker@V?$specs_handler@V?$basic_format_parse_context@_WUerror_handler@detail@v6@fmt@@@v6@fmt@@V?$basic_format_context@V?$back_insert_iterator@V?$buffer@_W@detail@v6@fmt@@@std@@_W@23@@detail@v6@fmt@@@detail@v6@fmt@@_W@012@@Z 0000000180060720     handles.obj
 0003:0000072c       $pdata$??$parse_arg_id@_WU?$precision_adapter@AEAV?$specs_checker@V?$specs_handler@V?$basic_format_parse_context@_WUerror_handler@detail@v6@fmt@@@v6@fmt@@V?$basic_format_context@V?$back_insert_iterator@V?$buffer@_W@detail@v6@fmt@@@std@@_W@23@@detail@v6@fmt@@@detail@v6@fmt@@_W@detail@v6@fmt@@@detail@v6@fmt@@YAPEB_WPEB_W0$$QEAU?$precision_adapter@AEAV?$specs_checker@V?$specs_handler@V?$basic_format_parse_context@_WUerror_handler@detail@v6@fmt@@@v6@fmt@@V?$basic_format_context@V?$back_insert_iterator@V?$buffer@_W@detail@v6@fmt@@@std@@_W@23@@detail@v6@fmt@@@detail@v6@fmt@@_W@012@@Z 000000018006072c     handles.obj
 0003:00000738       $pdata$??$write@_WV?$back_insert_iterator@V?$buffer@_W@detail@v6@fmt@@@std@@M$0A@@detail@v6@fmt@@YA?AV?$back_insert_iterator@V?$buffer@_W@detail@v6@fmt@@@std@@V34@MU?$basic_format_specs@_W@12@Vlocale_ref@012@@Z 0000000180060738     handles.obj
 0003:00000744       $pdata$??$write@_WV?$back_insert_iterator@V?$buffer@_W@detail@v6@fmt@@@std@@N$0A@@detail@v6@fmt@@YA?AV?$back_insert_iterator@V?$buffer@_W@detail@v6@fmt@@@std@@V34@NU?$basic_format_specs@_W@12@Vlocale_ref@012@@Z 0000000180060744     handles.obj
 0003:00000750       $pdata$??$write@_WV?$back_insert_iterator@V?$buffer@_W@detail@v6@fmt@@@std@@O$0A@@detail@v6@fmt@@YA?AV?$back_insert_iterator@V?$buffer@_W@detail@v6@fmt@@@std@@V34@OU?$basic_format_specs@_W@12@Vlocale_ref@012@@Z 0000000180060750     handles.obj
 0003:0000075c       $pdata$??$write@_W_WV?$back_insert_iterator@V?$buffer@_W@detail@v6@fmt@@@std@@@detail@v6@fmt@@YA?AV?$back_insert_iterator@V?$buffer@_W@detail@v6@fmt@@@std@@V34@V?$basic_string_view@_W@12@AEBU?$basic_format_specs@_W@12@@Z 000000018006075c     handles.obj
 0003:00000768       $pdata$?on_dec@?$int_writer@V?$back_insert_iterator@V?$buffer@_W@detail@v6@fmt@@@std@@_WI@detail@v6@fmt@@QEAAXXZ 0000000180060768     handles.obj
 0003:00000774       $pdata$?on_num@?$int_writer@V?$back_insert_iterator@V?$buffer@_W@detail@v6@fmt@@@std@@_WI@detail@v6@fmt@@QEAAXXZ 0000000180060774     handles.obj
 0003:00000780       $pdata$??$handle_int_type_spec@AEAU?$int_writer@V?$back_insert_iterator@V?$buffer@_W@detail@v6@fmt@@@std@@_WI@detail@v6@fmt@@@detail@v6@fmt@@YAXDAEAU?$int_writer@V?$back_insert_iterator@V?$buffer@_W@detail@v6@fmt@@@std@@_WI@012@@Z 0000000180060780     handles.obj
 0003:0000078c       $pdata$?on_dec@?$int_writer@V?$back_insert_iterator@V?$buffer@_W@detail@v6@fmt@@@std@@_W_K@detail@v6@fmt@@QEAAXXZ 000000018006078c     handles.obj
 0003:00000798       $pdata$?on_num@?$int_writer@V?$back_insert_iterator@V?$buffer@_W@detail@v6@fmt@@@std@@_W_K@detail@v6@fmt@@QEAAXXZ 0000000180060798     handles.obj
 0003:000007a4       $pdata$??$handle_int_type_spec@AEAU?$int_writer@V?$back_insert_iterator@V?$buffer@_W@detail@v6@fmt@@@std@@_W_K@detail@v6@fmt@@@detail@v6@fmt@@YAXDAEAU?$int_writer@V?$back_insert_iterator@V?$buffer@_W@detail@v6@fmt@@@std@@_W_K@012@@Z 00000001800607a4     handles.obj
 0003:000007b0       $pdata$??$parse_float_type_spec@Uerror_handler@detail@v6@fmt@@_W@detail@v6@fmt@@YA?AUfloat_specs@012@AEBU?$basic_format_specs@_W@12@$$QEAUerror_handler@012@@Z 00000001800607b0     handles.obj
 0003:000007bc       $pdata$??$write_bytes@_WV?$back_insert_iterator@V?$buffer@_W@detail@v6@fmt@@@std@@@detail@v6@fmt@@YA?AV?$back_insert_iterator@V?$buffer@_W@detail@v6@fmt@@@std@@V34@V?$basic_string_view@D@12@AEBU?$basic_format_specs@_W@12@@Z 00000001800607bc     handles.obj
 0003:000007c8       $pdata$??$write_padded@$01V?$back_insert_iterator@V?$buffer@_W@detail@v6@fmt@@@std@@_WV?$float_writer@_W@detail@v6@fmt@@@detail@v6@fmt@@YA?AV?$back_insert_iterator@V?$buffer@_W@detail@v6@fmt@@@std@@V34@AEBU?$basic_format_specs@_W@12@_KAEBV?$float_writer@_W@012@@Z 00000001800607c8     handles.obj
 0003:000007d4       $pdata$??$fill@PEA_W_W@detail@v6@fmt@@YAPEA_WPEA_W_KAEBU?$fill_t@_W@012@@Z 00000001800607d4     handles.obj
 0003:000007e0       $pdata$0$??$fill@PEA_W_W@detail@v6@fmt@@YAPEA_WPEA_W_KAEBU?$fill_t@_W@012@@Z 00000001800607e0     handles.obj
 0003:000007ec       $pdata$1$??$fill@PEA_W_W@detail@v6@fmt@@YAPEA_WPEA_W_KAEBU?$fill_t@_W@012@@Z 00000001800607ec     handles.obj
 0003:000007f8       $pdata$??$get_dynamic_spec@Vprecision_checker@detail@v6@fmt@@V?$basic_format_arg@V?$basic_format_context@V?$back_insert_iterator@V?$buffer@_W@detail@v6@fmt@@@std@@_W@v6@fmt@@@34@Uerror_handler@234@@detail@v6@fmt@@YAHV?$basic_format_arg@V?$basic_format_context@V?$back_insert_iterator@V?$buffer@_W@detail@v6@fmt@@@std@@_W@v6@fmt@@@12@Uerror_handler@012@@Z 00000001800607f8     handles.obj
 0003:00000804       $pdata$??$get_dynamic_spec@Vwidth_checker@detail@v6@fmt@@V?$basic_format_arg@V?$basic_format_context@V?$back_insert_iterator@V?$buffer@_W@detail@v6@fmt@@@std@@_W@v6@fmt@@@34@Uerror_handler@234@@detail@v6@fmt@@YAHV?$basic_format_arg@V?$basic_format_context@V?$back_insert_iterator@V?$buffer@_W@detail@v6@fmt@@@std@@_W@v6@fmt@@@12@Uerror_handler@012@@Z 0000000180060804     handles.obj
 0003:00000810       $pdata$??$write_int@V?$back_insert_iterator@V?$buffer@_W@detail@v6@fmt@@@std@@_WV<lambda_dbc99c5d30ad811266da5b27d7d4d7eb>@@@detail@v6@fmt@@YA?AV?$back_insert_iterator@V?$buffer@_W@detail@v6@fmt@@@std@@V34@HV?$basic_string_view@D@12@AEBU?$basic_format_specs@_W@12@V<lambda_dbc99c5d30ad811266da5b27d7d4d7eb>@@@Z 0000000180060810     handles.obj
 0003:0000081c       $pdata$??$write_int@V?$back_insert_iterator@V?$buffer@_W@detail@v6@fmt@@@std@@_WV<lambda_0273f2d8c97c19346923ccbca9d35cd0>@@@detail@v6@fmt@@YA?AV?$back_insert_iterator@V?$buffer@_W@detail@v6@fmt@@@std@@V34@HV?$basic_string_view@D@12@AEBU?$basic_format_specs@_W@12@V<lambda_0273f2d8c97c19346923ccbca9d35cd0>@@@Z 000000018006081c     handles.obj
 0003:00000828       $pdata$??$write_int@V?$back_insert_iterator@V?$buffer@_W@detail@v6@fmt@@@std@@_WV<lambda_1584a04d9a5f951756080462468a1c79>@@@detail@v6@fmt@@YA?AV?$back_insert_iterator@V?$buffer@_W@detail@v6@fmt@@@std@@V34@HV?$basic_string_view@D@12@AEBU?$basic_format_specs@_W@12@V<lambda_1584a04d9a5f951756080462468a1c79>@@@Z 0000000180060828     handles.obj
 0003:00000834       $pdata$??$write_int@V?$back_insert_iterator@V?$buffer@_W@detail@v6@fmt@@@std@@_WV<lambda_766228445ed89183d7065b0051936627>@@@detail@v6@fmt@@YA?AV?$back_insert_iterator@V?$buffer@_W@detail@v6@fmt@@@std@@V34@HV?$basic_string_view@D@12@AEBU?$basic_format_specs@_W@12@V<lambda_766228445ed89183d7065b0051936627>@@@Z 0000000180060834     handles.obj
 0003:00000840       $pdata$??$write_int@V?$back_insert_iterator@V?$buffer@_W@detail@v6@fmt@@@std@@_WV<lambda_ee8e8661040b0e68e19c307d8706693d>@@@detail@v6@fmt@@YA?AV?$back_insert_iterator@V?$buffer@_W@detail@v6@fmt@@@std@@V34@HV?$basic_string_view@D@12@AEBU?$basic_format_specs@_W@12@V<lambda_ee8e8661040b0e68e19c307d8706693d>@@@Z 0000000180060840     handles.obj
 0003:0000084c       $pdata$??$write_int@V?$back_insert_iterator@V?$buffer@_W@detail@v6@fmt@@@std@@_WV<lambda_c4159916ea5054600e9c49615e89ce82>@@@detail@v6@fmt@@YA?AV?$back_insert_iterator@V?$buffer@_W@detail@v6@fmt@@@std@@V34@HV?$basic_string_view@D@12@AEBU?$basic_format_specs@_W@12@V<lambda_c4159916ea5054600e9c49615e89ce82>@@@Z 000000018006084c     handles.obj
 0003:00000858       $pdata$??$write_int@V?$back_insert_iterator@V?$buffer@_W@detail@v6@fmt@@@std@@_WV<lambda_46028ac11bf91aacf0795357afd8c72d>@@@detail@v6@fmt@@YA?AV?$back_insert_iterator@V?$buffer@_W@detail@v6@fmt@@@std@@V34@HV?$basic_string_view@D@12@AEBU?$basic_format_specs@_W@12@V<lambda_46028ac11bf91aacf0795357afd8c72d>@@@Z 0000000180060858     handles.obj
 0003:00000864       $pdata$??$write_padded@$01V?$back_insert_iterator@V?$buffer@_W@detail@v6@fmt@@@std@@_WV<lambda_2c6139bafe179ad98da6b2e77db1d169>@@@detail@v6@fmt@@YA?AV?$back_insert_iterator@V?$buffer@_W@detail@v6@fmt@@@std@@V34@AEBU?$basic_format_specs@_W@12@_K2AEBV<lambda_2c6139bafe179ad98da6b2e77db1d169>@@@Z 0000000180060864     handles.obj
 0003:00000870       $pdata$??1PluginSettings@@QEAA@XZ 0000000180060870     Pcfg.obj
 0003:0000087c       $pdata$?SaveValue@PluginCheckBoxBinding@@UEAAXPEBUFarDialogItem@@H@Z 000000018006087c     Pcfg.obj
 0003:00000888       $pdata$??_GPluginCheckBoxBinding@@UEAAPEAXI@Z 0000000180060888     Pcfg.obj
 0003:00000888       $pdata$??_GPluginEditFieldBinding@@UEAAPEAXI@Z 0000000180060888     Pclass.obj
 0003:00000894       $pdata$??1PluginDialogBuilder@@QEAA@XZ 0000000180060894     Pcfg.obj
 0003:000008a0       $pdata$?AddButtons@PluginDialogBuilder@@QEAAXHPEBHHH@Z 00000001800608a0     Pcfg.obj
 0003:000008ac       $pdata$4$?AddButtons@PluginDialogBuilder@@QEAAXHPEBHHH@Z 00000001800608ac     Pcfg.obj
 0003:000008b8       $pdata$5$?AddButtons@PluginDialogBuilder@@QEAAXHPEBHHH@Z 00000001800608b8     Pcfg.obj
 0003:000008c4       $pdata$?ShowDialogEx@PluginDialogBuilder@@QEAA_JXZ 00000001800608c4     Pcfg.obj
 0003:000008d0       $pdata$4$?ShowDialogEx@PluginDialogBuilder@@QEAA_JXZ 00000001800608d0     Pcfg.obj
 0003:000008dc       $pdata$6$?ShowDialogEx@PluginDialogBuilder@@QEAA_JXZ 00000001800608dc     Pcfg.obj
 0003:000008e8       $pdata$7$?ShowDialogEx@PluginDialogBuilder@@QEAA_JXZ 00000001800608e8     Pcfg.obj
 0003:000008f4       $pdata$8$?ShowDialogEx@PluginDialogBuilder@@QEAA_JXZ 00000001800608f4     Pcfg.obj
 0003:00000900       $pdata$?AddDialogItem@PluginDialogBuilder@@AEAAPEAUFarDialogItem@@W4FARDIALOGITEMTYPES@@PEB_W@Z 0000000180060900     Pcfg.obj
 0003:0000090c       $pdata$0$?AddDialogItem@PluginDialogBuilder@@AEAAPEAUFarDialogItem@@W4FARDIALOGITEMTYPES@@PEB_W@Z 000000018006090c     Pcfg.obj
 0003:00000918       $pdata$1$?AddDialogItem@PluginDialogBuilder@@AEAAPEAUFarDialogItem@@W4FARDIALOGITEMTYPES@@PEB_W@Z 0000000180060918     Pcfg.obj
 0003:00000924       $pdata$2$?AddDialogItem@PluginDialogBuilder@@AEAAPEAUFarDialogItem@@W4FARDIALOGITEMTYPES@@PEB_W@Z 0000000180060924     Pcfg.obj
 0003:00000930       $pdata$3$?AddDialogItem@PluginDialogBuilder@@AEAAPEAUFarDialogItem@@W4FARDIALOGITEMTYPES@@PEB_W@Z 0000000180060930     Pcfg.obj
 0003:0000093c       $pdata$?ItemWidth@PluginDialogBuilder@@CA_JAEBUFarDialogItem@@@Z 000000018006093c     Pcfg.obj
 0003:00000948       $pdata$?Read@options@@QEAAXXZ 0000000180060948     Pcfg.obj
 0003:00000954       $pdata$?Write@options@@QEBAXXZ 0000000180060954     Pcfg.obj
 0003:00000960       $pdata$?Config@@YAHXZ      0000000180060960     Pcfg.obj
 0003:0000096c       $pdata$?_Xran@?$_String_val@U?$_Simple_types@_W@std@@@std@@SAXXZ 000000018006096c     Pclass.obj
 0003:00000978       $pdata$?append@?$basic_string@_WU?$char_traits@_W@std@@V?$allocator@_W@2@@std@@QEAAAEAV12@_K_W@Z 0000000180060978     Pclass.obj
 0003:00000984       $pdata$1$?append@?$basic_string@_WU?$char_traits@_W@std@@V?$allocator@_W@2@@std@@QEAAAEAV12@_K_W@Z 0000000180060984     Pclass.obj
 0003:00000990       $pdata$2$?append@?$basic_string@_WU?$char_traits@_W@std@@V?$allocator@_W@2@@std@@QEAAAEAV12@_K_W@Z 0000000180060990     Pclass.obj
 0003:0000099c       $pdata$3$?append@?$basic_string@_WU?$char_traits@_W@std@@V?$allocator@_W@2@@std@@QEAAAEAV12@_K_W@Z 000000018006099c     Pclass.obj
 0003:000009a8       $pdata$4$?append@?$basic_string@_WU?$char_traits@_W@std@@V?$allocator@_W@2@@std@@QEAAAEAV12@_K_W@Z 00000001800609a8     Pclass.obj
 0003:000009b4       $pdata$?insert@?$basic_string@_WU?$char_traits@_W@std@@V?$allocator@_W@2@@std@@QEAAAEAV12@_KQEB_W0@Z 00000001800609b4     Pclass.obj
 0003:000009c0       $pdata$2$?insert@?$basic_string@_WU?$char_traits@_W@std@@V?$allocator@_W@2@@std@@QEAAAEAV12@_KQEB_W0@Z 00000001800609c0     Pclass.obj
 0003:000009cc       $pdata$3$?insert@?$basic_string@_WU?$char_traits@_W@std@@V?$allocator@_W@2@@std@@QEAAAEAV12@_KQEB_W0@Z 00000001800609cc     Pclass.obj
 0003:000009d8       $pdata$??4columns@@QEAAAEAU0@AEBU0@@Z 00000001800609d8     Pclass.obj
 0003:000009e4       $pdata$??0Plist@@QEAA@XZ   00000001800609e4     Pclass.obj
 0003:000009f0       $pdata$?dtor$7@?0???0Plist@@QEAA@XZ@4HA 00000001800609f0     Pclass.obj
 0003:000009fc       $pdata$??1Plist@@QEAA@XZ   00000001800609fc     Pclass.obj
 0003:00000a08       $pdata$?Connect@Plist@@QEAA_NPEB_W00@Z 0000000180060a08     Pclass.obj
 0003:00000a14       $pdata$?dtor$3@?0??Connect@Plist@@QEAA_NPEB_W00@Z@4HA 0000000180060a14     Pclass.obj
 0003:00000a20       $pdata$?GetFindData@Plist@@QEAAHAEAPEAUPluginPanelItem@@AEA_K_K@Z 0000000180060a20     Pclass.obj
 0003:00000a2c       $pdata$?FreeFindData@Plist@@SAXPEAUPluginPanelItem@@_K@Z 0000000180060a2c     Pclass.obj
 0003:00000a38       $pdata$?GetOpenPanelInfo@Plist@@QEAAXPEAUOpenPanelInfo@@@Z 0000000180060a38     Pclass.obj
 0003:00000a44       $pdata$?GetFiles@Plist@@QEAAHPEAUPluginPanelItem@@_KHPEAPEB_W1AEAUoptions@@@Z 0000000180060a44     Pclass.obj
 0003:00000a50       $pdata$?DeleteFiles@Plist@@QEAAHPEAUPluginPanelItem@@_K1@Z 0000000180060a50     Pclass.obj
 0003:00000a5c       $pdata$?ProcessEvent@Plist@@QEAAH_JPEAX@Z 0000000180060a5c     Pclass.obj
 0003:00000a68       $pdata$?Compare@Plist@@QEBAHPEBUPluginPanelItem@@0I@Z 0000000180060a68     Pclass.obj
 0003:00000a74       $pdata$?ProcessKey@Plist@@QEAAHPEBU_INPUT_RECORD@@@Z 0000000180060a74     Pclass.obj
 0003:00000a80       $pdata$?dtor$25@?0??ProcessKey@Plist@@QEAAHPEBU_INPUT_RECORD@@@Z@4HA 0000000180060a80     Pclass.obj
 0003:00000a80       $pdata$?dtor$28@?0??ProcessKey@Plist@@QEAAHPEBU_INPUT_RECORD@@@Z@4HA 0000000180060a80     Pclass.obj
 0003:00000a8c       $pdata$?PanelModes@Plist@@QEAAPEAUPanelMode@@AEA_K@Z 0000000180060a8c     Pclass.obj
 0003:00000a98       $pdata$2$?PanelModes@Plist@@QEAAPEAUPanelMode@@AEA_K@Z 0000000180060a98     Pclass.obj
 0003:00000aa4       $pdata$3$?PanelModes@Plist@@QEAAPEAUPanelMode@@AEA_K@Z 0000000180060aa4     Pclass.obj
 0003:00000ab0       $pdata$?GetVersionInfo@Plist@@SA_NPEB_WAEAV?$unique_ptr@$$BY0A@DU?$default_delete@$$BY0A@D@std@@@std@@AEAPEB_W2@Z 0000000180060ab0     Pclass.obj
 0003:00000abc       $pdata$?SavePanelModes@Plist@@SAXXZ 0000000180060abc     Pclass.obj
 0003:00000ac8       $pdata$?InitializePanelModes@Plist@@SAXXZ 0000000180060ac8     Pclass.obj
 0003:00000ad4       $pdata$?dtor$90@?0??InitializePanelModes@Plist@@SAXXZ@4HA 0000000180060ad4     Pclass.obj
 0003:00000ae0       $pdata$?dtor$181@?0??InitializePanelModes@Plist@@SAXXZ@4HA 0000000180060ae0     Pclass.obj
 0003:00000aec       $pdata$?PrintVersionInfo@Plist@@CAXPEAXPEB_W@Z 0000000180060aec     Pclass.obj
 0003:00000af8       $pdata$?Reread@Plist@@AEAAXXZ 0000000180060af8     Pclass.obj
 0003:00000b04       $pdata$?PrintOwnerInfo@Plist@@AEAAXPEAXK@Z 0000000180060b04     Pclass.obj
 0003:00000b10       $pdata$?ConnectWMI@Plist@@AEAA_NXZ 0000000180060b10     Pclass.obj
 0003:00000b1c       $pdata$?dtor$1@?0??ConnectWMI@Plist@@AEAA_NXZ@4HA 0000000180060b1c     Pclass.obj
 0003:00000b28       $pdata$?WmiError@Plist@@AEBAXXZ 0000000180060b28     Pclass.obj
 0003:00000b34       $pdata$0$?WmiError@Plist@@AEBAXXZ 0000000180060b34     Pclass.obj
 0003:00000b40       $pdata$1$?WmiError@Plist@@AEBAXXZ 0000000180060b40     Pclass.obj
 0003:00000b4c       $pdata$??4?$unique_ptr@VPerfThread@@U?$default_delete@VPerfThread@@@std@@@std@@QEAAAEAV01@$$QEAV01@@Z 0000000180060b4c     Pclass.obj
 0003:00000b58       $pdata$0$??4?$unique_ptr@VPerfThread@@U?$default_delete@VPerfThread@@@std@@@std@@QEAAAEAV01@$$QEAV01@@Z 0000000180060b58     Pclass.obj
 0003:00000b64       $pdata$1$??4?$unique_ptr@VPerfThread@@U?$default_delete@VPerfThread@@@std@@@std@@QEAAAEAV01@$$QEAV01@@Z 0000000180060b64     Pclass.obj
 0003:00000b70       $pdata$??1?$unique_ptr@VPerfThread@@U?$default_delete@VPerfThread@@@std@@@std@@QEAA@XZ 0000000180060b70     Pclass.obj
 0003:00000b7c       $pdata$??1?$unique_ptr@VWMIConnection@@U?$default_delete@VWMIConnection@@@std@@@std@@QEAA@XZ 0000000180060b7c     Pclass.obj
 0003:00000b88       $pdata$?_Clear_and_reserve_geometric@?$vector@Umode@@V?$allocator@Umode@@@std@@@std@@AEAAX_K@Z 0000000180060b88     Pclass.obj
 0003:00000b94       $pdata$0$?_Clear_and_reserve_geometric@?$vector@Umode@@V?$allocator@Umode@@@std@@@std@@AEAAX_K@Z 0000000180060b94     Pclass.obj
 0003:00000ba0       $pdata$1$?_Clear_and_reserve_geometric@?$vector@Umode@@V?$allocator@Umode@@@std@@@std@@AEAAX_K@Z 0000000180060ba0     Pclass.obj
 0003:00000bac       $pdata$3$?_Clear_and_reserve_geometric@?$vector@Umode@@V?$allocator@Umode@@@std@@@std@@AEAAX_K@Z 0000000180060bac     Pclass.obj
 0003:00000bb8       $pdata$4$?_Clear_and_reserve_geometric@?$vector@Umode@@V?$allocator@Umode@@@std@@@std@@AEAAX_K@Z 0000000180060bb8     Pclass.obj
 0003:00000bc4       $pdata$?_Xlength@?$vector@PEB_WV?$allocator@PEB_W@std@@@std@@CAXXZ 0000000180060bc4     Pclass.obj
 0003:00000bc4       $pdata$?_Xlength@?$vector@Umode@@V?$allocator@Umode@@@std@@@std@@CAXXZ 0000000180060bc4     Pclass.obj
 0003:00000bc4       $pdata$?_Xlength@?$vector@V?$basic_string@_WU?$char_traits@_W@std@@V?$allocator@_W@2@@std@@V?$allocator@V?$basic_string@_WU?$char_traits@_W@std@@V?$allocator@_W@2@@std@@@2@@std@@CAXXZ 0000000180060bc4     Pclass.obj
 0003:00000bc4       $pdata$?_Xlength@?$vector@PEAUHINSTANCE__@@V?$allocator@PEAUHINSTANCE__@@@std@@@std@@CAXXZ 0000000180060bc4     Plist.obj
 0003:00000bc4       $pdata$?_Xlength@?$vector@EV?$allocator@E@std@@@std@@CAXXZ 0000000180060bc4     perfthread.obj
 0003:00000bc4       $pdata$?_Xlength@?$vector@UProcessPerfData@@V?$allocator@UProcessPerfData@@@std@@@std@@CAXXZ 0000000180060bc4     perfthread.obj
 0003:00000bd0       $pdata$??1ProcessData@@QEAA@XZ 0000000180060bd0     Pclass.obj
 0003:00000bdc       $pdata$?DurationToText@@YA?AV?$basic_string@_WU?$char_traits@_W@std@@V?$allocator@_W@2@@std@@_K@Z 0000000180060bdc     Pclass.obj
 0003:00000be8       $pdata$?SaveValue@PluginEditFieldBinding@@UEAAXPEBUFarDialogItem@@H@Z 0000000180060be8     Pclass.obj
 0003:00000bf4       $pdata$?AddEditField@PluginDialogBuilder@@QEAAPEAUFarDialogItem@@PEA_WHHPEB_W_N@Z 0000000180060bf4     Pclass.obj
 0003:00000c00       $pdata$?ui64toa_width@@YA?AV?$basic_string@_WU?$char_traits@_W@std@@V?$allocator@_W@2@@std@@_KI_N@Z 0000000180060c00     Pclass.obj
 0003:00000c0c       $pdata$?PrintTitle@@YA?AV?$basic_string@_WU?$char_traits@_W@std@@V?$allocator@_W@2@@std@@H@Z 0000000180060c0c     Pclass.obj
 0003:00000c18       $pdata$?TranslateMode@@YA_NAEBV?$basic_string@_WU?$char_traits@_W@std@@V?$allocator@_W@2@@std@@AEAV12@@Z 0000000180060c18     Pclass.obj
 0003:00000c24       $pdata$?generate_titles@@YAXAEBV?$basic_string@_WU?$char_traits@_W@std@@V?$allocator@_W@2@@std@@AEAUPanelMode@@@Z 0000000180060c24     Pclass.obj
 0003:00000c30       $pdata$??__FTitle@?1??GetOpenPanelInfo@Plist@@QEAAXPEAUOpenPanelInfo@@@Z@YAXXZ 0000000180060c30     Pclass.obj
 0003:00000c3c       $pdata$?EnumWndProc@@YAHPEAUHWND__@@_J@Z 0000000180060c3c     Pclass.obj
 0003:00000c48       $pdata$??1?$list@U?$pair@$$CBKPEAUHWND__@@@std@@V?$allocator@U?$pair@$$CBKPEAUHWND__@@@std@@@2@@std@@QEAA@XZ 0000000180060c48     Pclass.obj
 0003:00000c54       $pdata$0$??1?$list@U?$pair@$$CBKPEAUHWND__@@@std@@V?$allocator@U?$pair@$$CBKPEAUHWND__@@@std@@@2@@std@@QEAA@XZ 0000000180060c54     Pclass.obj
 0003:00000c60       $pdata$1$??1?$list@U?$pair@$$CBKPEAUHWND__@@@std@@V?$allocator@U?$pair@$$CBKPEAUHWND__@@@std@@@2@@std@@QEAA@XZ 0000000180060c60     Pclass.obj
 0003:00000c6c       $pdata$?_Forced_rehash@?$_Hash@V?$_Umap_traits@KPEAUHWND__@@V?$_Uhash_compare@KU?$hash@K@std@@U?$equal_to@K@2@@std@@V?$allocator@U?$pair@$$CBKPEAUHWND__@@@std@@@3@$0A@@std@@@std@@IEAAX_K@Z 0000000180060c6c     Pclass.obj
 0003:00000c78       $pdata$1$?_Forced_rehash@?$_Hash@V?$_Umap_traits@KPEAUHWND__@@V?$_Uhash_compare@KU?$hash@K@std@@U?$equal_to@K@2@@std@@V?$allocator@U?$pair@$$CBKPEAUHWND__@@@std@@@3@$0A@@std@@@std@@IEAAX_K@Z 0000000180060c78     Pclass.obj
 0003:00000c84       $pdata$2$?_Forced_rehash@?$_Hash@V?$_Umap_traits@KPEAUHWND__@@V?$_Uhash_compare@KU?$hash@K@std@@U?$equal_to@K@2@@std@@V?$allocator@U?$pair@$$CBKPEAUHWND__@@@std@@@3@$0A@@std@@@std@@IEAAX_K@Z 0000000180060c84     Pclass.obj
 0003:00000c90       $pdata$3$?_Forced_rehash@?$_Hash@V?$_Umap_traits@KPEAUHWND__@@V?$_Uhash_compare@KU?$hash@K@std@@U?$equal_to@K@2@@std@@V?$allocator@U?$pair@$$CBKPEAUHWND__@@@std@@@3@$0A@@std@@@std@@IEAAX_K@Z 0000000180060c90     Pclass.obj
 0003:00000c9c       $pdata$5$?_Forced_rehash@?$_Hash@V?$_Umap_traits@KPEAUHWND__@@V?$_Uhash_compare@KU?$hash@K@std@@U?$equal_to@K@2@@std@@V?$allocator@U?$pair@$$CBKPEAUHWND__@@@std@@@3@$0A@@std@@@std@@IEAAX_K@Z 0000000180060c9c     Pclass.obj
 0003:00000ca8       $pdata$6$?_Forced_rehash@?$_Hash@V?$_Umap_traits@KPEAUHWND__@@V?$_Uhash_compare@KU?$hash@K@std@@U?$equal_to@K@2@@std@@V?$allocator@U?$pair@$$CBKPEAUHWND__@@@std@@@3@$0A@@std@@@std@@IEAAX_K@Z 0000000180060ca8     Pclass.obj
 0003:00000cb4       $pdata$?_Assign_grow@?$_Hash_vec@V?$allocator@V?$_List_unchecked_iterator@V?$_List_val@U?$_List_simple_types@U?$pair@$$CBKPEAUHWND__@@@std@@@std@@@std@@@std@@@std@@@std@@QEAAX_KV?$_List_unchecked_iterator@V?$_List_val@U?$_List_simple_types@U?$pair@$$CBKPEAUHWND__@@@std@@@std@@@std@@@2@@Z 0000000180060cb4     Pclass.obj
 0003:00000cc0       $pdata$1$?_Assign_grow@?$_Hash_vec@V?$allocator@V?$_List_unchecked_iterator@V?$_List_val@U?$_List_simple_types@U?$pair@$$CBKPEAUHWND__@@@std@@@std@@@std@@@std@@@std@@@std@@QEAAX_KV?$_List_unchecked_iterator@V?$_List_val@U?$_List_simple_types@U?$pair@$$CBKPEAUHWND__@@@std@@@std@@@std@@@2@@Z 0000000180060cc0     Pclass.obj
 0003:00000ccc       $pdata$2$?_Assign_grow@?$_Hash_vec@V?$allocator@V?$_List_unchecked_iterator@V?$_List_val@U?$_List_simple_types@U?$pair@$$CBKPEAUHWND__@@@std@@@std@@@std@@@std@@@std@@@std@@QEAAX_KV?$_List_unchecked_iterator@V?$_List_val@U?$_List_simple_types@U?$pair@$$CBKPEAUHWND__@@@std@@@std@@@std@@@2@@Z 0000000180060ccc     Pclass.obj
 0003:00000cd8       $pdata$3$?_Assign_grow@?$_Hash_vec@V?$allocator@V?$_List_unchecked_iterator@V?$_List_val@U?$_List_simple_types@U?$pair@$$CBKPEAUHWND__@@@std@@@std@@@std@@@std@@@std@@@std@@QEAAX_KV?$_List_unchecked_iterator@V?$_List_val@U?$_List_simple_types@U?$pair@$$CBKPEAUHWND__@@@std@@@std@@@std@@@2@@Z 0000000180060cd8     Pclass.obj
 0003:00000ce4       $pdata$??1?$_Hash_vec@V?$allocator@V?$_List_unchecked_iterator@V?$_List_val@U?$_List_simple_types@U?$pair@$$CBKPEAUHWND__@@@std@@@std@@@std@@@std@@@std@@@std@@QEAA@XZ 0000000180060ce4     Pclass.obj
 0003:00000cf0       $pdata$??1?$_Hash@V?$_Umap_traits@KPEAUHWND__@@V?$_Uhash_compare@KU?$hash@K@std@@U?$equal_to@K@2@@std@@V?$allocator@U?$pair@$$CBKPEAUHWND__@@@std@@@3@$0A@@std@@@std@@QEAA@XZ 0000000180060cf0     Pclass.obj
 0003:00000cfc       $pdata$0$??1?$_Hash@V?$_Umap_traits@KPEAUHWND__@@V?$_Uhash_compare@KU?$hash@K@std@@U?$equal_to@K@2@@std@@V?$allocator@U?$pair@$$CBKPEAUHWND__@@@std@@@3@$0A@@std@@@std@@QEAA@XZ 0000000180060cfc     Pclass.obj
 0003:00000d08       $pdata$1$??1?$_Hash@V?$_Umap_traits@KPEAUHWND__@@V?$_Uhash_compare@KU?$hash@K@std@@U?$equal_to@K@2@@std@@V?$allocator@U?$pair@$$CBKPEAUHWND__@@@std@@@3@$0A@@std@@@std@@QEAA@XZ 0000000180060d08     Pclass.obj
 0003:00000d14       $pdata$?deallocate@?$allocator@V?$basic_string@_WU?$char_traits@_W@std@@V?$allocator@_W@2@@std@@@std@@QEAAXQEAV?$basic_string@_WU?$char_traits@_W@std@@V?$allocator@_W@2@@2@_K@Z 0000000180060d14     Pclass.obj
 0003:00000d20       $pdata$?_Destroy@?$vector@V?$basic_string@_WU?$char_traits@_W@std@@V?$allocator@_W@2@@std@@V?$allocator@V?$basic_string@_WU?$char_traits@_W@std@@V?$allocator@_W@2@@std@@@2@@std@@AEAAXPEAV?$basic_string@_WU?$char_traits@_W@std@@V?$allocator@_W@2@@2@0@Z 0000000180060d20     Pclass.obj
 0003:00000d2c       $pdata$?_Tidy@?$vector@V?$basic_string@_WU?$char_traits@_W@std@@V?$allocator@_W@2@@std@@V?$allocator@V?$basic_string@_WU?$char_traits@_W@std@@V?$allocator@_W@2@@std@@@2@@std@@AEAAXXZ 0000000180060d2c     Pclass.obj
 0003:00000d38       $pdata$0$?_Tidy@?$vector@V?$basic_string@_WU?$char_traits@_W@std@@V?$allocator@_W@2@@std@@V?$allocator@V?$basic_string@_WU?$char_traits@_W@std@@V?$allocator@_W@2@@std@@@2@@std@@AEAAXXZ 0000000180060d38     Pclass.obj
 0003:00000d44       $pdata$1$?_Tidy@?$vector@V?$basic_string@_WU?$char_traits@_W@std@@V?$allocator@_W@2@@std@@V?$allocator@V?$basic_string@_WU?$char_traits@_W@std@@V?$allocator@_W@2@@std@@@2@@std@@AEAAXXZ 0000000180060d44     Pclass.obj
 0003:00000d50       $pdata$?deallocate@?$allocator@PEB_W@std@@QEAAXQEAPEB_W_K@Z 0000000180060d50     Pclass.obj
 0003:00000d50       $pdata$?deallocate@?$allocator@PEAUHINSTANCE__@@@std@@QEAAXQEAPEAUHINSTANCE__@@_K@Z 0000000180060d50     Plist.obj
 0003:00000d5c       $pdata$??$_Emplace_reallocate@V?$basic_string@_WU?$char_traits@_W@std@@V?$allocator@_W@2@@std@@@?$vector@V?$basic_string@_WU?$char_traits@_W@std@@V?$allocator@_W@2@@std@@V?$allocator@V?$basic_string@_WU?$char_traits@_W@std@@V?$allocator@_W@2@@std@@@2@@std@@QEAAPEAV?$basic_string@_WU?$char_traits@_W@std@@V?$allocator@_W@2@@1@QEAV21@$$QEAV21@@Z 0000000180060d5c     Pclass.obj
 0003:00000d68       $pdata$?catch$8@?0???$_Emplace_reallocate@V?$basic_string@_WU?$char_traits@_W@std@@V?$allocator@_W@2@@std@@@?$vector@V?$basic_string@_WU?$char_traits@_W@std@@V?$allocator@_W@2@@std@@V?$allocator@V?$basic_string@_WU?$char_traits@_W@std@@V?$allocator@_W@2@@std@@@2@@std@@QEAAPEAV?$basic_string@_WU?$char_traits@_W@std@@V?$allocator@_W@2@@1@QEAV21@$$QEAV21@@Z@4HA 0000000180060d68     Pclass.obj
 0003:00000d74       $pdata$?window_style@@YA@PEAUHWND__@@@Z 0000000180060d74     Pclass.obj
 0003:00000d80       $pdata$?window_ex_style@@YA@PEAUHWND__@@@Z 0000000180060d80     Pclass.obj
 0003:00000d8c       $pdata$?DumpNTCounters@@YAXPEAXAEAVPerfThread@@KK@Z 0000000180060d8c     Pclass.obj
 0003:00000d98       $pdata$?_Tidy@?$vector@UFarMenuItem@@V?$allocator@UFarMenuItem@@@std@@@std@@AEAAXXZ 0000000180060d98     Pclass.obj
 0003:00000da4       $pdata$??$_Try_emplace@AEBK$$V@?$_Hash@V?$_Umap_traits@KPEAUHWND__@@V?$_Uhash_compare@KU?$hash@K@std@@U?$equal_to@K@2@@std@@V?$allocator@U?$pair@$$CBKPEAUHWND__@@@std@@@3@$0A@@std@@@std@@IEAA?AU?$pair@PEAU?$_List_node@U?$pair@$$CBKPEAUHWND__@@@std@@PEAX@std@@_N@1@AEBK@Z 0000000180060da4     Pclass.obj
 0003:00000db0       $pdata$??$_Assign_range@PEBUmode@@@?$vector@Umode@@V?$allocator@Umode@@@std@@@std@@AEAAXPEBUmode@@0Uforward_iterator_tag@1@@Z 0000000180060db0     Pclass.obj
 0003:00000dbc       $pdata$??$_Reallocate_grow_by@V<lambda_51c4cb9729979bd953fe6d1bff5c73b0>@@_K_K_W@?$basic_string@_WU?$char_traits@_W@std@@V?$allocator@_W@2@@std@@AEAAAEAV01@_KV<lambda_51c4cb9729979bd953fe6d1bff5c73b0>@@_K2_W@Z 0000000180060dbc     Pclass.obj
 0003:00000dc8       $pdata$3$??$_Reallocate_grow_by@V<lambda_51c4cb9729979bd953fe6d1bff5c73b0>@@_K_K_W@?$basic_string@_WU?$char_traits@_W@std@@V?$allocator@_W@2@@std@@AEAAAEAV01@_KV<lambda_51c4cb9729979bd953fe6d1bff5c73b0>@@_K2_W@Z 0000000180060dc8     Pclass.obj
 0003:00000dd4       $pdata$5$??$_Reallocate_grow_by@V<lambda_51c4cb9729979bd953fe6d1bff5c73b0>@@_K_K_W@?$basic_string@_WU?$char_traits@_W@std@@V?$allocator@_W@2@@std@@AEAAAEAV01@_KV<lambda_51c4cb9729979bd953fe6d1bff5c73b0>@@_K2_W@Z 0000000180060dd4     Pclass.obj
 0003:00000de0       $pdata$6$??$_Reallocate_grow_by@V<lambda_51c4cb9729979bd953fe6d1bff5c73b0>@@_K_K_W@?$basic_string@_WU?$char_traits@_W@std@@V?$allocator@_W@2@@std@@AEAAAEAV01@_KV<lambda_51c4cb9729979bd953fe6d1bff5c73b0>@@_K2_W@Z 0000000180060de0     Pclass.obj
 0003:00000dec       $pdata$??$_Reallocate_grow_by@V<lambda_967c2ed818824c5314a20ec3af46b793>@@_KPEB_W_K@?$basic_string@_WU?$char_traits@_W@std@@V?$allocator@_W@2@@std@@AEAAAEAV01@_KV<lambda_967c2ed818824c5314a20ec3af46b793>@@_KPEB_W2@Z 0000000180060dec     Pclass.obj
 0003:00000df8       $pdata$3$??$_Reallocate_grow_by@V<lambda_967c2ed818824c5314a20ec3af46b793>@@_KPEB_W_K@?$basic_string@_WU?$char_traits@_W@std@@V?$allocator@_W@2@@std@@AEAAAEAV01@_KV<lambda_967c2ed818824c5314a20ec3af46b793>@@_KPEB_W2@Z 0000000180060df8     Pclass.obj
 0003:00000e04       $pdata$5$??$_Reallocate_grow_by@V<lambda_967c2ed818824c5314a20ec3af46b793>@@_KPEB_W_K@?$basic_string@_WU?$char_traits@_W@std@@V?$allocator@_W@2@@std@@AEAAAEAV01@_KV<lambda_967c2ed818824c5314a20ec3af46b793>@@_KPEB_W2@Z 0000000180060e04     Pclass.obj
 0003:00000e10       $pdata$6$??$_Reallocate_grow_by@V<lambda_967c2ed818824c5314a20ec3af46b793>@@_KPEB_W_K@?$basic_string@_WU?$char_traits@_W@std@@V?$allocator@_W@2@@std@@AEAAAEAV01@_KV<lambda_967c2ed818824c5314a20ec3af46b793>@@_KPEB_W2@Z 0000000180060e10     Pclass.obj
 0003:00000e1c       $pdata$??$fill@PEAV?$_List_unchecked_iterator@V?$_List_val@U?$_List_simple_types@U?$pair@$$CBKPEAUHWND__@@@std@@@std@@@std@@@std@@V12@@std@@YAXQEAV?$_List_unchecked_iterator@V?$_List_val@U?$_List_simple_types@U?$pair@$$CBKPEAUHWND__@@@std@@@std@@@std@@@0@0AEBV10@@Z 0000000180060e1c     Pclass.obj
 0003:00000e28       $pdata$0$??$fill@PEAV?$_List_unchecked_iterator@V?$_List_val@U?$_List_simple_types@U?$pair@$$CBKPEAUHWND__@@@std@@@std@@@std@@@std@@V12@@std@@YAXQEAV?$_List_unchecked_iterator@V?$_List_val@U?$_List_simple_types@U?$pair@$$CBKPEAUHWND__@@@std@@@std@@@std@@@0@0AEBV10@@Z 0000000180060e28     Pclass.obj
 0003:00000e34       $pdata$1$??$fill@PEAV?$_List_unchecked_iterator@V?$_List_val@U?$_List_simple_types@U?$pair@$$CBKPEAUHWND__@@@std@@@std@@@std@@@std@@V12@@std@@YAXQEAV?$_List_unchecked_iterator@V?$_List_val@U?$_List_simple_types@U?$pair@$$CBKPEAUHWND__@@@std@@@std@@@std@@@0@0AEBV10@@Z 0000000180060e34     Pclass.obj
 0003:00000e40       $pdata$??$_Resize_reallocate@U_Value_init_tag@std@@@?$vector@PEB_WV?$allocator@PEB_W@std@@@std@@AEAAX_KAEBU_Value_init_tag@1@@Z 0000000180060e40     Pclass.obj
 0003:00000e4c       $pdata$?catch$0@?0???$_Resize_reallocate@U_Value_init_tag@std@@@?$vector@PEB_WV?$allocator@PEB_W@std@@@std@@AEAAX_KAEBU_Value_init_tag@1@@Z@4HA 0000000180060e4c     Pclass.obj
 0003:00000e58       $pdata$??$_Copy_unchecked@PEBUmode@@PEAU1@@std@@YAPEAUmode@@PEBU1@0PEAU1@@Z 0000000180060e58     Pclass.obj
 0003:00000e64       $pdata$??4ProcessPerfData@@QEAAAEAU0@AEBU0@@Z 0000000180060e64     perfthread.obj
 0003:00000e70       $pdata$??0PerfThread@@QEAA@PEB_W00@Z 0000000180060e70     perfthread.obj
 0003:00000e7c       $pdata$??1PerfThread@@QEAA@XZ 0000000180060e7c     perfthread.obj
 0003:00000e88       $pdata$?GetProcessData@PerfThread@@QEAAPEAUProcessPerfData@@KK@Z 0000000180060e88     perfthread.obj
 0003:00000e94       $pdata$0$?GetProcessData@PerfThread@@QEAAPEAUProcessPerfData@@KK@Z 0000000180060e94     perfthread.obj
 0003:00000ea0       $pdata$1$?GetProcessData@PerfThread@@QEAAPEAUProcessPerfData@@KK@Z 0000000180060ea0     perfthread.obj
 0003:00000eac       $pdata$?SyncReread@PerfThread@@QEAAXXZ 0000000180060eac     perfthread.obj
 0003:00000eb8       $pdata$?ThreadProc@PerfThread@@CAKPEAX@Z 0000000180060eb8     perfthread.obj
 0003:00000ec4       $pdata$?Refresh@PerfThread@@AEAAXXZ 0000000180060ec4     perfthread.obj
 0003:00000ed0       $pdata$?RefreshWMIData@PerfThread@@AEAAXXZ 0000000180060ed0     perfthread.obj
 0003:00000edc       $pdata$?_Tidy@?$vector@UProcessPerfData@@V?$allocator@UProcessPerfData@@@std@@@std@@AEAAXXZ 0000000180060edc     perfthread.obj
 0003:00000ee8       $pdata$0$?_Tidy@?$vector@UProcessPerfData@@V?$allocator@UProcessPerfData@@@std@@@std@@AEAAXXZ 0000000180060ee8     perfthread.obj
 0003:00000ef4       $pdata$1$?_Tidy@?$vector@UProcessPerfData@@V?$allocator@UProcessPerfData@@@std@@@std@@AEAAXXZ 0000000180060ef4     perfthread.obj
 0003:00000f00       $pdata$??1?$vector@_WV?$allocator@_W@std@@@std@@QEAA@XZ 0000000180060f00     perfthread.obj
 0003:00000f0c       $pdata$?deallocate@?$allocator@E@std@@QEAAXQEAE_K@Z 0000000180060f0c     perfthread.obj
 0003:00000f18       $pdata$??1?$vector@EV?$allocator@E@std@@@std@@QEAA@XZ 0000000180060f18     perfthread.obj
 0003:00000f24       $pdata$??$_Construct_n_copies_of_ty@U_Value_init_tag@std@@@?$vector@UProcessPerfData@@V?$allocator@UProcessPerfData@@@std@@@std@@AEAAX_KAEBU_Value_init_tag@1@@Z 0000000180060f24     perfthread.obj
 0003:00000f30       $pdata$2$??$_Construct_n_copies_of_ty@U_Value_init_tag@std@@@?$vector@UProcessPerfData@@V?$allocator@UProcessPerfData@@@std@@@std@@AEAAX_KAEBU_Value_init_tag@1@@Z 0000000180060f30     perfthread.obj
 0003:00000f3c       $pdata$3$??$_Construct_n_copies_of_ty@U_Value_init_tag@std@@@?$vector@UProcessPerfData@@V?$allocator@UProcessPerfData@@@std@@@std@@AEAAX_KAEBU_Value_init_tag@1@@Z 0000000180060f3c     perfthread.obj
 0003:00000f48       $pdata$4$??$_Construct_n_copies_of_ty@U_Value_init_tag@std@@@?$vector@UProcessPerfData@@V?$allocator@UProcessPerfData@@@std@@@std@@AEAAX_KAEBU_Value_init_tag@1@@Z 0000000180060f48     perfthread.obj
 0003:00000f54       $pdata$5$??$_Construct_n_copies_of_ty@U_Value_init_tag@std@@@?$vector@UProcessPerfData@@V?$allocator@UProcessPerfData@@@std@@@std@@AEAAX_KAEBU_Value_init_tag@1@@Z 0000000180060f54     perfthread.obj
 0003:00000f60       $pdata$6$??$_Construct_n_copies_of_ty@U_Value_init_tag@std@@@?$vector@UProcessPerfData@@V?$allocator@UProcessPerfData@@@std@@@std@@AEAAX_KAEBU_Value_init_tag@1@@Z 0000000180060f60     perfthread.obj
 0003:00000f6c       $pdata$??$_Resize_reallocate@U_Value_init_tag@std@@@?$vector@EV?$allocator@E@std@@@std@@AEAAX_KAEBU_Value_init_tag@1@@Z 0000000180060f6c     perfthread.obj
 0003:00000f78       $pdata$?catch$0@?0???$_Resize_reallocate@U_Value_init_tag@std@@@?$vector@EV?$allocator@E@std@@@std@@AEAAX_KAEBU_Value_init_tag@1@@Z@4HA 0000000180060f78     perfthread.obj
 0003:00000f84       $pdata$??1?$_Uninitialized_backout_al@V?$allocator@UProcessPerfData@@@std@@@std@@QEAA@XZ 0000000180060f84     perfthread.obj
 0003:00000f90       $pdata$??0?$basic_string@_WU?$char_traits@_W@std@@V?$allocator@_W@2@@std@@QEAA@_K_W@Z 0000000180060f90     Plist.obj
 0003:00000f9c       $pdata$?GetList@@YA_NAEAPEAUPluginPanelItem@@AEA_KAEAVPerfThread@@@Z 0000000180060f9c     Plist.obj
 0003:00000fa8       $pdata$?KillProcess@@YA_NKPEAUHWND__@@@Z 0000000180060fa8     Plist.obj
 0003:00000fb4       $pdata$?Enable@DebugToken@@QEAA_NXZ 0000000180060fb4     Plist.obj
 0003:00000fc0       $pdata$?Revert@DebugToken@@QEAA_NXZ 0000000180060fc0     Plist.obj
 0003:00000fcc       $pdata$?CreateToken@DebugToken@@SA_NXZ 0000000180060fcc     Plist.obj
 0003:00000fd8       $pdata$1$?CreateToken@DebugToken@@SA_NXZ 0000000180060fd8     Plist.obj
 0003:00000fe4       $pdata$2$?CreateToken@DebugToken@@SA_NXZ 0000000180060fe4     Plist.obj
 0003:00000ff0       $pdata$?OpenProcessForced@@YAPEAXPEAVDebugToken@@KKH@Z 0000000180060ff0     Plist.obj
 0003:00000ffc       $pdata$?PrintNTCurDirAndEnv@@YAXPEAX0H@Z 0000000180060ffc     Plist.obj
 0003:00001008       $pdata$?PrintModules@@YAXPEAXKAEAUoptions@@@Z 0000000180061008     Plist.obj
 0003:00001014       $pdata$?GetPData@@YA_NAEAUProcessData@@AEBUProcessPerfData@@@Z 0000000180061014     Plist.obj
 0003:00001020       $pdata$1$?GetPData@@YA_NAEAUProcessData@@AEBUProcessPerfData@@@Z 0000000180061020     Plist.obj
 0003:0000102c       $pdata$3$?GetPData@@YA_NAEAUProcessData@@AEBUProcessPerfData@@@Z 000000018006102c     Plist.obj
 0003:00001038       $pdata$4$?GetPData@@YA_NAEAUProcessData@@AEBUProcessPerfData@@@Z 0000000180061038     Plist.obj
 0003:00001044       $pdata$??0?$vector@UProcessPerfData@@V?$allocator@UProcessPerfData@@@std@@@std@@QEAA@AEBV01@@Z 0000000180061044     Plist.obj
 0003:00001050       $pdata$?FreeUserData@@YAXQEAXQEBUFarPanelItemFreeInfo@@@Z 0000000180061050     Plist.obj
 0003:0000105c       $pdata$?read_string@?$ipc_functions@$0A@@@SA?AV?$basic_string@_WU?$char_traits@_W@std@@V?$allocator@_W@2@@std@@PEAXAEBUUNICODE_STRING_SAME@detail@@@Z 000000018006105c     Plist.obj
 0003:00001068       $pdata$?GetOpenProcessData@?$ipc_functions@$0A@@@SAXPEAXPEAV?$basic_string@_WU?$char_traits@_W@std@@V?$allocator@_W@2@@std@@1111@Z 0000000180061068     Plist.obj
 0003:00001074       $pdata$0$?GetOpenProcessData@?$ipc_functions@$0A@@@SAXPEAXPEAV?$basic_string@_WU?$char_traits@_W@std@@V?$allocator@_W@2@@std@@1111@Z 0000000180061074     Plist.obj
 0003:00001080       $pdata$1$?GetOpenProcessData@?$ipc_functions@$0A@@@SAXPEAXPEAV?$basic_string@_WU?$char_traits@_W@std@@V?$allocator@_W@2@@std@@1111@Z 0000000180061080     Plist.obj
 0003:0000108c       $pdata$2$?GetOpenProcessData@?$ipc_functions@$0A@@@SAXPEAXPEAV?$basic_string@_WU?$char_traits@_W@std@@V?$allocator@_W@2@@std@@1111@Z 000000018006108c     Plist.obj
 0003:00001098       $pdata$?print_module_impl@@YAXQEAXAEBV?$basic_string@_WU?$char_traits@_W@std@@V?$allocator@_W@2@@std@@KAEBUoptions@@AEBV?$function@$$A6A_NPEA_W_K@Z@2@@Z 0000000180061098     Plist.obj
 0003:000010a4       $pdata$??1?$function@$$A6A_NPEA_W_K@Z@std@@QEAA@XZ 00000001800610a4     Plist.obj
 0003:000010a4       $pdata$??1?$function@$$A6AXAEBUtagVARIANT@@@Z@std@@QEAA@XZ 00000001800610a4     WMI.obj
 0003:000010b0       $pdata$?allocate@?$allocator@PEAUHINSTANCE__@@@std@@QEAAPEAPEAUHINSTANCE__@@_K@Z 00000001800610b0     Plist.obj
 0003:000010bc       $pdata$??1?$vector@PEAUHINSTANCE__@@V?$allocator@PEAUHINSTANCE__@@@std@@@std@@QEAA@XZ 00000001800610bc     Plist.obj
 0003:000010c8       $pdata$??R<lambda_fbad59960194a21b5f35257a64aadaa4>@@QEBAXXZ 00000001800610c8     Plist.obj
 0003:000010d4       $pdata$??$print_module@PEAX@@YAXQEAXPEAXKAEAUoptions@@AEBV?$function@$$A6A_NPEA_W_K@Z@std@@@Z 00000001800610d4     Plist.obj
 0003:000010e0       $pdata$??$_Resize_reallocate@U_Value_init_tag@std@@@?$vector@PEAUHINSTANCE__@@V?$allocator@PEAUHINSTANCE__@@@std@@@std@@AEAAX_KAEBU_Value_init_tag@1@@Z 00000001800610e0     Plist.obj
 0003:000010ec       $pdata$?catch$0@?0???$_Resize_reallocate@U_Value_init_tag@std@@@?$vector@PEAUHINSTANCE__@@V?$allocator@PEAUHINSTANCE__@@@std@@@std@@AEAAX_KAEBU_Value_init_tag@1@@Z@4HA 00000001800610ec     Plist.obj
 0003:000010f8       $pdata$?_Do_call@?$_Func_impl_no_alloc@V<lambda_87e110110aa5c29eaf754372c3484d5b>@@_NPEA_W_K@std@@EEAA_N$$QEAPEA_W$$QEA_K@Z 00000001800610f8     Plist.obj
 0003:00001104       $pdata$?_Do_call@?$_Func_impl_no_alloc@V<lambda_c6a5923e4ab0669d9f7c2a6c892502eb>@@_NPEA_W_K@std@@EEAA_N$$QEAPEA_W$$QEA_K@Z 0000000180061104     Plist.obj
 0003:00001110       $pdata$?ConvertDate@@YAXAEBU_FILETIME@@PEA_W1@Z 0000000180061110     Pmix.obj
 0003:0000111c       $pdata$?WinError@@YAHPEB_W@Z 000000018006111c     Pmix.obj
 0003:00001128       $pdata$??0WMIConnection@@QEAA@XZ 0000000180061128     WMI.obj
 0003:00001134       $pdata$??1WMIConnection@@QEAA@XZ 0000000180061134     WMI.obj
 0003:00001140       $pdata$?Connect@WMIConnection@@QEAA_NPEB_W00@Z 0000000180061140     WMI.obj
 0003:0000114c       $pdata$?Disconnect@WMIConnection@@QEAAXXZ 000000018006114c     WMI.obj
 0003:00001158       $pdata$?GetProcessPriority@WMIConnection@@QEAAKK@Z 0000000180061158     WMI.obj
 0003:00001164       $pdata$?SetProcessPriority@WMIConnection@@QEAAHKK@Z 0000000180061164     WMI.obj
 0003:00001170       $pdata$?TerminateProcess@WMIConnection@@QEAAHK@Z 0000000180061170     WMI.obj
 0003:0000117c       $pdata$?GetProcessOwner@WMIConnection@@QEAA?AV?$basic_string@_WU?$char_traits@_W@std@@V?$allocator@_W@2@@std@@KPEAV23@@Z 000000018006117c     WMI.obj
 0003:00001188       $pdata$?GetProcessUserSid@WMIConnection@@QEAA?AV?$basic_string@_WU?$char_traits@_W@std@@V?$allocator@_W@2@@std@@K@Z 0000000180061188     WMI.obj
 0003:00001194       $pdata$?GetProcessSessionId@WMIConnection@@QEAAKK@Z 0000000180061194     WMI.obj
 0003:000011a0       $pdata$?GetProcessExecutablePath@WMIConnection@@QEAA?AV?$basic_string@_WU?$char_traits@_W@std@@V?$allocator@_W@2@@std@@K@Z 00000001800611a0     WMI.obj
 0003:000011ac       $pdata$?dtor$1@?0??GetProcessCommandLine@WMIConnection@@QEAA?AV?$basic_string@_WU?$char_traits@_W@std@@V?$allocator@_W@2@@std@@K@Z@4HA 00000001800611ac     WMI.obj
 0003:000011ac       $pdata$?dtor$1@?0??GetProcessExecutablePath@WMIConnection@@QEAA?AV?$basic_string@_WU?$char_traits@_W@std@@V?$allocator@_W@2@@std@@K@Z@4HA 00000001800611ac     WMI.obj
 0003:000011b8       $pdata$?GetProcessCommandLine@WMIConnection@@QEAA?AV?$basic_string@_WU?$char_traits@_W@std@@V?$allocator@_W@2@@std@@K@Z 00000001800611b8     WMI.obj
 0003:000011c4       $pdata$?ExecMethod@WMIConnection@@AEAAHKPEB_W0K@Z 00000001800611c4     WMI.obj
 0003:000011d0       $pdata$?GetProcessProperty@WMIConnection@@AEAA_NKPEB_WAEBV?$function@$$A6AXAEBUtagVARIANT@@@Z@std@@@Z 00000001800611d0     WMI.obj
 0003:000011dc       $pdata$?ProcessPath@@YA@K@Z 00000001800611dc     WMI.obj
 0003:000011e8       $pdata$??1?$unique_ptr@UIWbemClassObject@@Ucom_closer@@@std@@QEAA@XZ 00000001800611e8     WMI.obj
 0003:000011e8       $pdata$??1?$unique_ptr@UIWbemLocator@@Ucom_closer@@@std@@QEAA@XZ 00000001800611e8     WMI.obj
 0003:000011f4       $pdata$??1?$ptr_setter@V?$unique_ptr@UIWbemClassObject@@Ucom_closer@@@std@@@@QEAA@XZ 00000001800611f4     WMI.obj
 0003:00001200       $pdata$ClosePanelW         0000000180061200     Proclist.obj
 0003:0000120c       $pdata$CompareW            000000018006120c     Proclist.obj
 0003:00001218       $pdata$ConfigureW          0000000180061218     Proclist.obj
 0003:00001224       $pdata$DeleteFilesW        0000000180061224     Proclist.obj
 0003:00001230       $pdata$GetFilesW           0000000180061230     Proclist.obj
 0003:0000123c       $pdata$GetFindDataW        000000018006123c     Proclist.obj
 0003:00001248       $pdata$GetGlobalInfoW      0000000180061248     Proclist.obj
 0003:00001254       $pdata$GetPluginInfoW      0000000180061254     Proclist.obj
 0003:00001260       $pdata$OpenW               0000000180061260     Proclist.obj
 0003:0000126c       $pdata$ProcessPanelEventW  000000018006126c     Proclist.obj
 0003:00001278       $pdata$ProcessPanelInputW  0000000180061278     Proclist.obj
 0003:00001284       $pdata$SetStartupInfoW     0000000180061284     Proclist.obj
 0003:00001290       $pdata$?Message@@YAHIPEB_WPEAPEB_W_K2@Z 0000000180061290     Proclist.obj
 0003:0000129c       $pdata$?is_wow64_process@@YA_NPEAX@Z 000000018006129c     Proclist.obj
 0003:000012a8       $pdata$?dynamic_bind@@YAXXZ 00000001800612a8     Proclist.obj
 0003:000012b4       $pdata$0$?dynamic_bind@@YAXXZ 00000001800612b4     Proclist.obj
 0003:000012c0       $pdata$1$?dynamic_bind@@YAXXZ 00000001800612c0     Proclist.obj
 0003:000012cc       $pdata$??0_Lockit@std@@QEAA@H@Z 00000001800612cc     libcpmt:xlock.obj
 0003:000012d8       $pdata$??1_Lockit@std@@QEAA@XZ 00000001800612d8     libcpmt:xlock.obj
 0003:000012e4       $pdata$??0_Init_locks@std@@QEAA@XZ 00000001800612e4     libcpmt:xlock.obj
 0003:000012f0       $pdata$??1_Init_locks@std@@QEAA@XZ 00000001800612f0     libcpmt:xlock.obj
 0003:000012fc       $pdata$??__Einitlocks@std@@YAXXZ 00000001800612fc     libcpmt:xlock.obj
 0003:00001308       $pdata$?__scrt_throw_std_bad_alloc@@YAXXZ 0000000180061308     LIBCMT:throw_bad_alloc.obj
 0003:00001308       $pdata$?_Xbad_alloc@std@@YAXXZ 0000000180061308     libcpmt:xthrow.obj
 0003:00001314       $pdata$?_Xlength_error@std@@YAXPEBD@Z 0000000180061314     libcpmt:xthrow.obj
 0003:00001320       $pdata$?_Xout_of_range@std@@YAXPEBD@Z 0000000180061320     libcpmt:xthrow.obj
 0003:0000132c       $pdata$?_Xruntime_error@std@@YAXPEBD@Z 000000018006132c     libcpmt:xthrow.obj
 0003:00001338       $pdata$??0logic_error@std@@QEAA@AEBV01@@Z 0000000180061338     libcpmt:xthrow.obj
 0003:00001344       $pdata$??0length_error@std@@QEAA@PEBD@Z 0000000180061344     libcpmt:xthrow.obj
 0003:00001350       $pdata$??0length_error@std@@QEAA@AEBV01@@Z 0000000180061350     libcpmt:xthrow.obj
 0003:0000135c       $pdata$??0out_of_range@std@@QEAA@PEBD@Z 000000018006135c     libcpmt:xthrow.obj
 0003:00001368       $pdata$??0out_of_range@std@@QEAA@AEBV01@@Z 0000000180061368     libcpmt:xthrow.obj
 0003:00001374       $pdata$??0bad_function_call@std@@QEAA@AEBV01@@Z 0000000180061374     libcpmt:xthrow.obj
 0003:00001380       $pdata$?_Xbad_function_call@std@@YAXXZ 0000000180061380     libcpmt:xthrow.obj
 0003:0000138c       $pdata$?_Facet_Register@std@@YAXPEAV_Facet_base@1@@Z 000000018006138c     libcpmt:locale0.obj
 0003:00001398       $pdata$??__F_Fac_tidy_reg@std@@YAXXZ 0000000180061398     libcpmt:locale0.obj
 0003:000013a4       $pdata$?_Locinfo_ctor@_Locinfo@std@@SAXPEAV12@PEBD@Z 00000001800613a4     libcpmt:locale0.obj
 0003:000013b0       $pdata$?_Locinfo_dtor@_Locinfo@std@@SAXPEAV12@@Z 00000001800613b0     libcpmt:locale0.obj
 0003:000013bc       $pdata$??4?$_Yarn@D@std@@QEAAAEAV01@PEBD@Z 00000001800613bc     libcpmt:locale0.obj
 0003:000013c8       $pdata$?_New_Locimp@_Locimp@locale@std@@CAPEAV123@_N@Z 00000001800613c8     libcpmt:locale0.obj
 0003:000013d4       $pdata$?_Locimp_dtor@_Locimp@locale@std@@CAXPEAV123@@Z 00000001800613d4     libcpmt:locale0.obj
 0003:000013e0       $pdata$??_G_Locimp@locale@std@@MEAAPEAXI@Z 00000001800613e0     libcpmt:locale0.obj
 0003:000013ec       $pdata$?_Init@locale@std@@CAPEAV_Locimp@12@_N@Z 00000001800613ec     libcpmt:locale0.obj
 0003:000013f8       $pdata$?_Setgloballocale@locale@std@@CAXPEAX@Z 00000001800613f8     libcpmt:locale0.obj
 0003:00001404       $pdata$_Deletegloballocale 0000000180061404     libcpmt:locale0.obj
 0003:00001410       $pdata$tidy_global         0000000180061410     libcpmt:locale0.obj
 0003:0000141c       $pdata$??__Fclassic_locale@std@@YAXXZ 000000018006141c     libcpmt:locale0.obj
 0003:00001428       $pdata$_Getcvt             0000000180061428     libcpmt:xwctomb.obj
 0003:00001434       $pdata$_Mbrtowc            0000000180061434     libcpmt:xmbtowc.obj
 0003:00001440       $pdata$??__Einitlocks@std@@YAXXZ 0000000180061440     libcpmt:iosptrs.obj
 0003:0000144c       $pdata$?_Atexit@@YAXP6AXXZ@Z 000000018006144c     libcpmt:iosptrs.obj
 0003:00001458       $pdata$??__Finit_atexit@@YAXXZ 0000000180061458     libcpmt:iosptrs.obj
 0003:00001464       $pdata$__crtInitializeCriticalSectionEx 0000000180061464     libcpmt:winapisupp.obj
 0003:00001470       $pdata$?initialize_pointers@@YAHXZ 0000000180061470     libcpmt:winapisupp.obj
 0003:0000147c       $pdata$atexit              000000018006147c     LIBCMT:utility.obj
 0003:00001488       $pdata$_onexit             0000000180061488     LIBCMT:utility.obj
 0003:00001494       $pdata$__scrt_is_nonwritable_in_current_image 0000000180061494     LIBCMT:utility.obj
 0003:000014a0       $pdata$__scrt_is_nonwritable_in_current_image$filt$0 00000001800614a0     LIBCMT:utility.obj
 0003:000014ac       $pdata$__scrt_acquire_startup_lock 00000001800614ac     LIBCMT:utility.obj
 0003:000014b8       $pdata$__scrt_release_startup_lock 00000001800614b8     LIBCMT:utility.obj
 0003:000014c4       $pdata$__scrt_initialize_crt 00000001800614c4     LIBCMT:utility.obj
 0003:000014d0       $pdata$__scrt_uninitialize_crt 00000001800614d0     LIBCMT:utility.obj
 0003:000014dc       $pdata$__scrt_initialize_onexit_tables 00000001800614dc     LIBCMT:utility.obj
 0003:000014e8       $pdata$__scrt_dllmain_exception_filter 00000001800614e8     LIBCMT:utility.obj
 0003:000014f4       $pdata$__scrt_dllmain_before_initialize_c 00000001800614f4     LIBCMT:utility.obj
 0003:00001500       $pdata$__scrt_dllmain_after_initialize_c 0000000180061500     LIBCMT:utility.obj
 0003:0000150c       $pdata$__scrt_dllmain_uninitialize_c 000000018006150c     LIBCMT:utility.obj
 0003:00001518       $pdata$__scrt_dllmain_uninitialize_critical 0000000180061518     LIBCMT:utility.obj
 0003:00001524       $pdata$__scrt_dllmain_crt_thread_attach 0000000180061524     LIBCMT:utility.obj
 0003:00001530       $pdata$__scrt_dllmain_crt_thread_detach 0000000180061530     LIBCMT:utility.obj
 0003:0000153c       $pdata$??2@YAPEAX_K@Z      000000018006153c     LIBCMT:new_scalar.obj
 0003:00001548       $pdata$??_Gtype_info@@UEAAPEAXI@Z 0000000180061548     LIBCMT:std_type_info_static.obj
 0003:00001554       $pdata$??_M@YAXPEAX_K1P6AX0@Z@Z 0000000180061554     LIBCMT:ehvecdtr.obj
 0003:00001560       $pdata$?fin$0@?0???_M@YAXPEAX_K1P6AX0@Z@Z@4HA 0000000180061560     LIBCMT:ehvecdtr.obj
 0003:0000156c       $pdata$?__ArrayUnwind@@YAXPEAX_K1P6AX0@Z@Z 000000018006156c     LIBCMT:ehvecdtr.obj
 0003:00001578       $pdata$?filt$0@?0??__ArrayUnwind@@YAXPEAX_K1P6AX0@Z@Z@4HA 0000000180061578     LIBCMT:ehvecdtr.obj
 0003:00001584       $pdata$?dllmain_crt_process_attach@@YAHQEAUHINSTANCE__@@QEAX@Z 0000000180061584     LIBCMT:dll_dllmain.obj
 0003:00001590       $pdata$?fin$0@?0??dllmain_crt_process_attach@@YAHQEAUHINSTANCE__@@QEAX@Z@4HA 0000000180061590     LIBCMT:dll_dllmain.obj
 0003:0000159c       $pdata$?dllmain_crt_process_detach@@YAH_N@Z 000000018006159c     LIBCMT:dll_dllmain.obj
 0003:000015a8       $pdata$?fin$0@?0??dllmain_crt_process_detach@@YAH_N@Z@4HA 00000001800615a8     LIBCMT:dll_dllmain.obj
 0003:000015b4       $pdata$?fin$1@?0??dllmain_crt_process_detach@@YAH_N@Z@4HA 00000001800615b4     LIBCMT:dll_dllmain.obj
 0003:000015c0       $pdata$?dllmain_crt_dispatch@@YAHQEAUHINSTANCE__@@KQEAX@Z 00000001800615c0     LIBCMT:dll_dllmain.obj
 0003:000015cc       $pdata$?dllmain_dispatch@@YAHQEAUHINSTANCE__@@KQEAX@Z 00000001800615cc     LIBCMT:dll_dllmain.obj
 0003:000015d8       $pdata$?filt$0@?0??dllmain_dispatch@@YAHQEAUHINSTANCE__@@KQEAX@Z@4HA 00000001800615d8     LIBCMT:dll_dllmain.obj
 0003:000015e4       $pdata$_DllMainCRTStartup  00000001800615e4     LIBCMT:dll_dllmain.obj
 0003:000015f0       $pdata$__GSHandlerCheckCommon 00000001800615f0     LIBCMT:gshandler.obj
 0003:000015fc       $pdata$__GSHandlerCheck    00000001800615fc     LIBCMT:gshandler.obj
 0003:00001608       $pdata$__GSHandlerCheck_EH 0000000180061608     LIBCMT:gshandlereh.obj
 0003:00001620       $pdata$__isa_available_init 0000000180061620     LIBCMT:cpu_disp.obj
 0003:0000162c       $pdata$__scrt_fastfail     000000018006162c     LIBCMT:utility_desktop.obj
 0003:00001638       $pdata$__security_init_cookie 0000000180061638     LIBCMT:gs_support.obj
 0003:00001644       $pdata$__scrt_initialize_default_local_stdio_options 0000000180061644     LIBCMT:default_local_stdio_options.obj
 0003:00001650       $pdata$_RTC_Initialize     0000000180061650     LIBCMT:initsect.obj
 0003:0000165c       $pdata$_RTC_Terminate      000000018006165c     LIBCMT:initsect.obj
 0003:00001674       $pdata$__report_securityfailure 0000000180061674     LIBCMT:gs_report.obj
 0003:00001680       $pdata$__report_rangecheckfailure 0000000180061680     LIBCMT:gs_report.obj
 0003:0000168c       $pdata$__report_gsfailure  000000018006168c     LIBCMT:gs_report.obj
 0003:00001698       $pdata$capture_current_context 0000000180061698     LIBCMT:gs_report.obj
 0003:000016a4       $pdata$capture_previous_context 00000001800616a4     LIBCMT:gs_report.obj
 0003:000016b0       $pdata$__raise_securityfailure 00000001800616b0     LIBCMT:gs_report.obj
 0003:000016bc       $pdata$_purecall           00000001800616bc     libvcruntime:purevirt.obj
 0003:000016c8       $pdata$__std_terminate     00000001800616c8     libvcruntime:ehhelpers.obj
 0003:000016d4       $pdata$_IsExceptionObjectToBeDestroyed 00000001800616d4     libvcruntime:ehhelpers.obj
 0003:000016e0       $pdata$__current_exception 00000001800616e0     libvcruntime:ehhelpers.obj
 0003:000016ec       $pdata$__current_exception_context 00000001800616ec     libvcruntime:ehhelpers.obj
 0003:000016f8       $pdata$__FrameUnwindFilter 00000001800616f8     libvcruntime:ehhelpers.obj
 0003:00001704       $pdata$__DestructExceptionObject 0000000180061704     libvcruntime:ehhelpers.obj
 0003:00001710       $pdata$__DestructExceptionObject$filt$0 0000000180061710     libvcruntime:ehhelpers.obj
 0003:0000171c       $pdata$__std_exception_copy 000000018006171c     libvcruntime:std_exception.obj
 0003:00001728       $pdata$__std_exception_destroy 0000000180061728     libvcruntime:std_exception.obj
 0003:00001734       $pdata$_CxxThrowException  0000000180061734     libvcruntime:throw.obj
 0003:00001740       $pdata$?DecompFuncInfo@FH4@@YA_JPEAEAEAUFuncInfo4@1@_KH_N@Z 0000000180061740     libvcruntime:risctrnsctrl.obj
 0003:0000174c       $pdata$?CatchTryBlock@__FrameHandler3@@SAPEBU_s_TryBlockMapEntry@@PEBU_s_FuncInfo@@H@Z 000000018006174c     libvcruntime:risctrnsctrl.obj
 0003:00001758       $pdata$?ExecutionInCatch@__FrameHandler3@@SA_NPEAU_xDISPATCHER_CONTEXT@@PEBU_s_FuncInfo@@@Z 0000000180061758     libvcruntime:risctrnsctrl.obj
 0003:00001764       $pdata$?FrameUnwindToEmptyState@__FrameHandler3@@SAXPEA_KPEAU_xDISPATCHER_CONTEXT@@PEBU_s_FuncInfo@@@Z 0000000180061764     libvcruntime:risctrnsctrl.obj
 0003:00001770       $pdata$?GetEstablisherFrame@__FrameHandler3@@SAPEA_KPEA_KPEAU_xDISPATCHER_CONTEXT@@PEBU_s_FuncInfo@@0@Z 0000000180061770     libvcruntime:risctrnsctrl.obj
 0003:0000177c       $pdata$?UnwindNestedFrames@__FrameHandler3@@SAXPEA_KPEAUEHExceptionRecord@@PEAU_CONTEXT@@0PEAXPEBU_s_FuncInfo@@HHPEBU_s_HandlerType@@PEAU_xDISPATCHER_CONTEXT@@E@Z 000000018006177c     libvcruntime:risctrnsctrl.obj
 0003:00001788       $pdata$?GetRangeOfTrysToCheck@__FrameHandler3@@SA?AU?$pair@Viterator@TryBlockMap@__FrameHandler3@@V123@@std@@AEAVTryBlockMap@1@HPEAU_xDISPATCHER_CONTEXT@@PEBU_s_FuncInfo@@H@Z 0000000180061788     libvcruntime:risctrnsctrl.obj
 0003:00001794       $pdata$?FrameUnwindToEmptyState@__FrameHandler4@@SAXPEA_KPEAU_xDISPATCHER_CONTEXT@@PEAUFuncInfo4@FH4@@@Z 0000000180061794     libvcruntime:risctrnsctrl.obj
 0003:000017a0       $pdata$?UnwindNestedFrames@__FrameHandler4@@SAXPEA_KPEAUEHExceptionRecord@@PEAU_CONTEXT@@0PEAXPEAUFuncInfo4@FH4@@HHPEAUHandlerType4@5@PEAU_xDISPATCHER_CONTEXT@@E@Z 00000001800617a0     libvcruntime:risctrnsctrl.obj
 0003:000017ac       $pdata$?GetRangeOfTrysToCheck@__FrameHandler4@@SA?AU?$pair@Viterator@TryBlockMap4@FH4@@V123@@std@@AEAVTryBlockMap4@FH4@@HPEAU_xDISPATCHER_CONTEXT@@PEAUFuncInfo4@5@H@Z 00000001800617ac     libvcruntime:risctrnsctrl.obj
 0003:000017b8       $pdata$_GetImageBase       00000001800617b8     libvcruntime:risctrnsctrl.obj
 0003:000017c4       $pdata$_SetImageBase       00000001800617c4     libvcruntime:risctrnsctrl.obj
 0003:000017d0       $pdata$_GetThrowImageBase  00000001800617d0     libvcruntime:risctrnsctrl.obj
 0003:000017dc       $pdata$_SetThrowImageBase  00000001800617dc     libvcruntime:risctrnsctrl.obj
 0003:000017e8       $pdata$_CreateFrameInfo    00000001800617e8     libvcruntime:risctrnsctrl.obj
 0003:000017f4       $pdata$_FindAndUnlinkFrame 00000001800617f4     libvcruntime:risctrnsctrl.obj
 0003:00001800       $pdata$__CxxFrameHandler3  0000000180061800     libvcruntime:risctrnsctrl.obj
 0003:0000180c       $pdata$__CxxFrameHandler4  000000018006180c     libvcruntime:risctrnsctrl.obj
 0003:00001818       $pdata$??$_CallSETranslator@V__FrameHandler4@@@@YAHPEAUEHExceptionRecord@@PEA_KPEAU_CONTEXT@@PEAU_xDISPATCHER_CONTEXT@@PEAUFuncInfo4@FH4@@K1@Z 0000000180061818     libvcruntime:risctrnsctrl.obj
 0003:00001824       $pdata$?filt$0@?0???$_CallSETranslator@V__FrameHandler4@@@@YAHPEAUEHExceptionRecord@@PEA_KPEAU_CONTEXT@@PEAU_xDISPATCHER_CONTEXT@@PEAUFuncInfo4@FH4@@K1@Z@4HA 0000000180061824     libvcruntime:risctrnsctrl.obj
 0003:00001830       $pdata$??$_CallSETranslator@V__FrameHandler3@@@@YAHPEAUEHExceptionRecord@@PEA_KPEAU_CONTEXT@@PEAU_xDISPATCHER_CONTEXT@@PEBU_s_FuncInfo@@K1@Z 0000000180061830     libvcruntime:risctrnsctrl.obj
 0003:0000183c       $pdata$?filt$0@?0???$_CallSETranslator@V__FrameHandler3@@@@YAHPEAUEHExceptionRecord@@PEA_KPEAU_CONTEXT@@PEAU_xDISPATCHER_CONTEXT@@PEBU_s_FuncInfo@@K1@Z@4HA 000000018006183c     libvcruntime:risctrnsctrl.obj
 0003:00001890       $pdata$__vcrt_initialize   0000000180061890     libvcruntime:initialization.obj
 0003:0000189c       $pdata$__vcrt_uninitialize 000000018006189c     libvcruntime:initialization.obj
 0003:000018a8       $pdata$__vcrt_uninitialize_critical 00000001800618a8     libvcruntime:initialization.obj
 0003:000018b4       $pdata$__vcrt_thread_attach 00000001800618b4     libvcruntime:initialization.obj
 0003:000018c0       $pdata$__vcrt_thread_detach 00000001800618c0     libvcruntime:initialization.obj
 0003:000018cc       $pdata$__C_specific_handler 00000001800618cc     libvcruntime:riscchandler.obj
 0003:000018d8       $pdata$__std_type_info_destroy_list 00000001800618d8     libvcruntime:std_type_info.obj
 0003:000018e4       $pdata$__vcrt_initialize_ptd 00000001800618e4     libvcruntime:per_thread_data.obj
 0003:000018f0       $pdata$__vcrt_uninitialize_ptd 00000001800618f0     libvcruntime:per_thread_data.obj
 0003:000018fc       $pdata$__vcrt_getptd       00000001800618fc     libvcruntime:per_thread_data.obj
 0003:00001908       $pdata$__vcrt_getptd_noexit 0000000180061908     libvcruntime:per_thread_data.obj
 0003:00001914       $pdata$__vcrt_freeptd      0000000180061914     libvcruntime:per_thread_data.obj
 0003:00001920       $pdata$__vcrt_freefls      0000000180061920     libvcruntime:per_thread_data.obj
 0003:0000192c       $pdata$?StateFromIp@__FrameHandler3@@SAHPEBU_s_FuncInfo@@PEAU_xDISPATCHER_CONTEXT@@_K@Z 000000018006192c     libvcruntime:ehstate.obj
 0003:00001938       $pdata$?GetCurrentState@__FrameHandler3@@SAHPEA_KPEAU_xDISPATCHER_CONTEXT@@PEBU_s_FuncInfo@@@Z 0000000180061938     libvcruntime:ehstate.obj
 0003:00001944       $pdata$?SetUnwindTryBlock@__FrameHandler3@@SAXPEA_KPEAU_xDISPATCHER_CONTEXT@@PEBU_s_FuncInfo@@H@Z 0000000180061944     libvcruntime:ehstate.obj
 0003:00001950       $pdata$?GetUnwindTryBlock@__FrameHandler3@@SAHPEA_KPEAU_xDISPATCHER_CONTEXT@@PEBU_s_FuncInfo@@@Z 0000000180061950     libvcruntime:ehstate.obj
 0003:0000195c       $pdata$?StateFromIp@__FrameHandler4@@SAHPEAUFuncInfo4@FH4@@PEAU_xDISPATCHER_CONTEXT@@_K@Z 000000018006195c     libvcruntime:ehstate.obj
 0003:00001968       $pdata$?getStartStop@UWMap4@FH4@@QEAAXHHAEAViterator@12@0@Z 0000000180061968     libvcruntime:frame.obj
 0003:00001974       $pdata$?getStateFromIterators@UWMap4@FH4@@SAHAEBViterator@12@H0H0@Z 0000000180061974     libvcruntime:frame.obj
 0003:00001980       $pdata$??0HandlerMap4@FH4@@QEAA@PEBUTryBlockMapEntry4@1@_KH@Z 0000000180061980     libvcruntime:frame.obj
 0003:0000198c       $pdata$?FrameUnwindToState@__FrameHandler3@@SAXPEA_KPEAU_xDISPATCHER_CONTEXT@@PEBU_s_FuncInfo@@H@Z 000000018006198c     libvcruntime:frame.obj
 0003:00001998       $pdata$?filt$0@?0??FrameUnwindToState@__FrameHandler3@@SAXPEA_KPEAU_xDISPATCHER_CONTEXT@@PEBU_s_FuncInfo@@H@Z@4HA 0000000180061998     libvcruntime:frame.obj
 0003:000019a4       $pdata$?fin$1@?0??FrameUnwindToState@__FrameHandler3@@SAXPEA_KPEAU_xDISPATCHER_CONTEXT@@PEBU_s_FuncInfo@@H@Z@4HA 00000001800619a4     libvcruntime:frame.obj
 0003:000019b0       $pdata$?GetHandlerSearchState@__FrameHandler3@@SAHPEA_KPEAU_xDISPATCHER_CONTEXT@@PEBU_s_FuncInfo@@@Z 00000001800619b0     libvcruntime:frame.obj
 0003:000019bc       $pdata$?CxxCallCatchBlock@__FrameHandler3@@SAPEAXPEAU_EXCEPTION_RECORD@@@Z 00000001800619bc     libvcruntime:frame.obj
 0003:000019c8       $pdata$?filt$0@?0??CxxCallCatchBlock@__FrameHandler3@@SAPEAXPEAU_EXCEPTION_RECORD@@@Z@4HA 00000001800619c8     libvcruntime:frame.obj
 0003:000019d4       $pdata$?fin$1@?0??CxxCallCatchBlock@__FrameHandler3@@SAPEAXPEAU_EXCEPTION_RECORD@@@Z@4HA 00000001800619d4     libvcruntime:frame.obj
 0003:000019e0       $pdata$?FrameUnwindToState@__FrameHandler4@@SAXPEA_KPEAU_xDISPATCHER_CONTEXT@@PEAUFuncInfo4@FH4@@H@Z 00000001800619e0     libvcruntime:frame.obj
 0003:000019ec       $pdata$?filt$0@?0??FrameUnwindToState@__FrameHandler4@@SAXPEA_KPEAU_xDISPATCHER_CONTEXT@@PEAUFuncInfo4@FH4@@H@Z@4HA 00000001800619ec     libvcruntime:frame.obj
 0003:000019f8       $pdata$?fin$1@?0??FrameUnwindToState@__FrameHandler4@@SAXPEA_KPEAU_xDISPATCHER_CONTEXT@@PEAUFuncInfo4@FH4@@H@Z@4HA 00000001800619f8     libvcruntime:frame.obj
 0003:00001a04       $pdata$?CxxCallCatchBlock@__FrameHandler4@@SAPEAXPEAU_EXCEPTION_RECORD@@@Z 0000000180061a04     libvcruntime:frame.obj
 0003:00001a10       $pdata$?filt$0@?0??CxxCallCatchBlock@__FrameHandler4@@SAPEAXPEAU_EXCEPTION_RECORD@@@Z@4HA 0000000180061a10     libvcruntime:frame.obj
 0003:00001a1c       $pdata$?fin$1@?0??CxxCallCatchBlock@__FrameHandler4@@SAPEAXPEAU_EXCEPTION_RECORD@@@Z@4HA 0000000180061a1c     libvcruntime:frame.obj
 0003:00001a28       $pdata$??0bad_exception@std@@QEAA@AEBV01@@Z 0000000180061a28     libvcruntime:frame.obj
 0003:00001a34       $pdata$?ExFilterRethrow@@YAHPEAU_EXCEPTION_POINTERS@@PEAUEHExceptionRecord@@PEAH@Z 0000000180061a34     libvcruntime:frame.obj
 0003:00001a40       $pdata$?ExFilterRethrowFH4@@YAHPEAU_EXCEPTION_POINTERS@@PEAUEHExceptionRecord@@HPEAH@Z 0000000180061a40     libvcruntime:frame.obj
 0003:00001a4c       $pdata$?IsInExceptionSpec@@YAEPEAUEHExceptionRecord@@PEBU_s_ESTypeList@@@Z 0000000180061a4c     libvcruntime:frame.obj
 0003:00001a58       $pdata$?Is_bad_exception_allowed@@YAEPEBU_s_ESTypeList@@@Z 0000000180061a58     libvcruntime:frame.obj
 0003:00001a64       $pdata$??$__InternalCxxFrameHandler@V__FrameHandler3@@@@YA?AW4_EXCEPTION_DISPOSITION@@PEAUEHExceptionRecord@@PEA_KPEAU_CONTEXT@@PEAU_xDISPATCHER_CONTEXT@@PEBU_s_FuncInfo@@H1E@Z 0000000180061a64     libvcruntime:frame.obj
 0003:00001a70       $pdata$??$__InternalCxxFrameHandler@V__FrameHandler4@@@@YA?AW4_EXCEPTION_DISPOSITION@@PEAUEHExceptionRecord@@PEA_KPEAU_CONTEXT@@PEAU_xDISPATCHER_CONTEXT@@PEAUFuncInfo4@FH4@@H1E@Z 0000000180061a70     libvcruntime:frame.obj
 0003:00001a7c       $pdata$??$TypeMatchHelper@V__FrameHandler3@@@@YAHPEBU_s_HandlerType@@PEBU_s_CatchableType@@PEBU_s_ThrowInfo@@@Z 0000000180061a7c     libvcruntime:frame.obj
 0003:00001a88       $pdata$??$TypeMatchHelper@V__FrameHandler4@@@@YAHPEAUHandlerType4@FH4@@PEBU_s_CatchableType@@PEBU_s_ThrowInfo@@@Z 0000000180061a88     libvcruntime:frame.obj
 0003:00001a94       $pdata$??$BuildCatchObjectHelperInternal@V__FrameHandler3@@@@YAHPEAUEHExceptionRecord@@PEAXPEBU_s_HandlerType@@PEBU_s_CatchableType@@@Z 0000000180061a94     libvcruntime:frame.obj
 0003:00001aa0       $pdata$??$BuildCatchObjectHelperInternal@V__FrameHandler4@@@@YAHPEAUEHExceptionRecord@@PEAXPEAUHandlerType4@FH4@@PEBU_s_CatchableType@@@Z 0000000180061aa0     libvcruntime:frame.obj
 0003:00001aac       $pdata$??$BuildCatchObjectInternal@V__FrameHandler3@@@@YAXPEAUEHExceptionRecord@@PEAXPEBU_s_HandlerType@@PEBU_s_CatchableType@@@Z 0000000180061aac     libvcruntime:frame.obj
 0003:00001ab8       $pdata$??$BuildCatchObjectInternal@V__FrameHandler4@@@@YAXPEAUEHExceptionRecord@@PEAXPEAUHandlerType4@FH4@@PEBU_s_CatchableType@@@Z 0000000180061ab8     libvcruntime:frame.obj
 0003:00001ac4       $pdata$??$FindHandler@V__FrameHandler3@@@@YAXPEAUEHExceptionRecord@@PEA_KPEAU_CONTEXT@@PEAU_xDISPATCHER_CONTEXT@@PEBU_s_FuncInfo@@EH1@Z 0000000180061ac4     libvcruntime:frame.obj
 0003:00001ad0       $pdata$??$FindHandler@V__FrameHandler4@@@@YAXPEAUEHExceptionRecord@@PEA_KPEAU_CONTEXT@@PEAU_xDISPATCHER_CONTEXT@@PEAUFuncInfo4@FH4@@EH1@Z 0000000180061ad0     libvcruntime:frame.obj
 0003:00001adc       $pdata$??$CatchIt@V__FrameHandler3@@@@YAXPEAUEHExceptionRecord@@PEA_KPEAU_CONTEXT@@PEAU_xDISPATCHER_CONTEXT@@PEBU_s_FuncInfo@@PEBU_s_HandlerType@@PEBU_s_CatchableType@@PEBU_s_TryBlockMapEntry@@H1EE@Z 0000000180061adc     libvcruntime:frame.obj
 0003:00001ae8       $pdata$??$FindHandlerForForeignException@V__FrameHandler3@@@@YAXPEAUEHExceptionRecord@@PEA_KPEAU_CONTEXT@@PEAU_xDISPATCHER_CONTEXT@@PEBU_s_FuncInfo@@HH1@Z 0000000180061ae8     libvcruntime:frame.obj
 0003:00001af4       $pdata$??$CatchIt@V__FrameHandler4@@@@YAXPEAUEHExceptionRecord@@PEA_KPEAU_CONTEXT@@PEAU_xDISPATCHER_CONTEXT@@PEAUFuncInfo4@FH4@@PEAUHandlerType4@4@PEBU_s_CatchableType@@PEAUTryBlockMapEntry4@4@H1EE@Z 0000000180061af4     libvcruntime:frame.obj
 0003:00001b00       $pdata$??$FindHandlerForForeignException@V__FrameHandler4@@@@YAXPEAUEHExceptionRecord@@PEA_KPEAU_CONTEXT@@PEAU_xDISPATCHER_CONTEXT@@PEAUFuncInfo4@FH4@@HH1@Z 0000000180061b00     libvcruntime:frame.obj
 0003:00001b0c       $pdata$__vcrt_initialize_locks 0000000180061b0c     libvcruntime:locks.obj
 0003:00001b18       $pdata$__vcrt_uninitialize_locks 0000000180061b18     libvcruntime:locks.obj
 0003:00001b48       $pdata$__vcrt_FlsAlloc     0000000180061b48     libvcruntime:winapi_downlevel.obj
 0003:00001b54       $pdata$__vcrt_FlsFree      0000000180061b54     libvcruntime:winapi_downlevel.obj
 0003:00001b60       $pdata$__vcrt_FlsGetValue  0000000180061b60     libvcruntime:winapi_downlevel.obj
 0003:00001b6c       $pdata$__vcrt_FlsSetValue  0000000180061b6c     libvcruntime:winapi_downlevel.obj
 0003:00001b78       $pdata$__vcrt_InitializeCriticalSectionEx 0000000180061b78     libvcruntime:winapi_downlevel.obj
 0003:00001b84       $pdata$?try_get_function@@YAPEAXW4function_id@?A0x81a78551@@QEBDQEBW4module_id@2@2@Z 0000000180061b84     libvcruntime:winapi_downlevel.obj
 0003:00001bc0       $pdata$_invalid_parameter_noinfo 0000000180061bc0     libucrt:invalid_parameter.obj
 0003:00001bcc       $pdata$_invalid_parameter_noinfo_noreturn 0000000180061bcc     libucrt:invalid_parameter.obj
 0003:00001bd8       $pdata$_invoke_watson      0000000180061bd8     libucrt:invalid_parameter.obj
 0003:00001be4       $pdata$__acrt_call_reportfault 0000000180061be4     libucrt:invalid_parameter.obj
 0003:00001bf0       $pdata$_invalid_parameter  0000000180061bf0     libucrt:invalid_parameter.obj
 0003:00001bfc       $pdata$_dclass             0000000180061bfc     libucrt:nan.obj
 0003:00001c08       $pdata$_ldclass            0000000180061c08     libucrt:nanl.obj
 0003:00001c14       $pdata$_fdclass            0000000180061c14     libucrt:nanf.obj
 0003:00001c20       $pdata$_errno              0000000180061c20     libucrt:errno.obj
 0003:00001c2c       $pdata$__doserrno          0000000180061c2c     libucrt:errno.obj
 0003:00001c38       $pdata$__acrt_errno_map_os_error 0000000180061c38     libucrt:errno.obj
 0003:00001c44       $pdata$__acrt_initialize_stdio 0000000180061c44     libucrt:_file.obj
 0003:00001c50       $pdata$__acrt_uninitialize_stdio 0000000180061c50     libucrt:_file.obj
 0003:00001c5c       $pdata$_fileno             0000000180061c5c     libucrt:fileno.obj
 0003:00001c68       $pdata$??0_LocaleUpdate@@QEAA@QEAU__crt_locale_pointers@@@Z 0000000180061c68     libucrt:output.obj
 0003:00001c74       $pdata$__stdio_common_vsnprintf_s 0000000180061c74     libucrt:output.obj
 0003:00001c80       $pdata$?write_string@?$string_output_adapter@D@__crt_stdio_output@@QEBAXQEBDHQEAHAEAV__crt_deferred_errno_cache@@@Z 0000000180061c80     libucrt:output.obj
 0003:00001c8c       $pdata$??$common_vsprintf@Vformat_validation_base@__crt_stdio_output@@D@@YAH_KQEAD0QEBDQEAU__crt_locale_pointers@@1@Z 0000000180061c8c     libucrt:output.obj
 0003:00001c98       $pdata$??$write_multiple_characters@V?$string_output_adapter@D@__crt_stdio_output@@D@__crt_stdio_output@@YAXAEBV?$string_output_adapter@D@0@DHQEAH@Z 0000000180061c98     libucrt:output.obj
 0003:00001ca4       $pdata$??$ensure_buffer_is_big_enough@D@formatting_buffer@__crt_stdio_output@@QEAA_N_K@Z 0000000180061ca4     libucrt:output.obj
 0003:00001cb0       $pdata$?process@?$output_processor@DV?$string_output_adapter@D@__crt_stdio_output@@V?$format_validation_base@DV?$string_output_adapter@D@__crt_stdio_output@@@2@@__crt_stdio_output@@QEAAHXZ 0000000180061cb0     libucrt:output.obj
 0003:00001cbc       $pdata$?state_case_normal@?$output_processor@DV?$string_output_adapter@D@__crt_stdio_output@@V?$format_validation_base@DV?$string_output_adapter@D@__crt_stdio_output@@@2@@__crt_stdio_output@@AEAA_NXZ 0000000180061cbc     libucrt:output.obj
 0003:00001cc8       $pdata$?state_case_normal_tchar@?$output_processor@DV?$string_output_adapter@D@__crt_stdio_output@@V?$format_validation_base@DV?$string_output_adapter@D@__crt_stdio_output@@@2@@__crt_stdio_output@@AEAA_ND@Z 0000000180061cc8     libucrt:output.obj
 0003:00001cd4       $pdata$?parse_int_from_format_string@?$output_processor@DV?$string_output_adapter@D@__crt_stdio_output@@V?$format_validation_base@DV?$string_output_adapter@D@__crt_stdio_output@@@2@@__crt_stdio_output@@AEAA_NQEAH@Z 0000000180061cd4     libucrt:output.obj
 0003:00001ce0       $pdata$?state_case_size@?$output_processor@DV?$string_output_adapter@D@__crt_stdio_output@@V?$format_validation_base@DV?$string_output_adapter@D@__crt_stdio_output@@@2@@__crt_stdio_output@@AEAA_NXZ 0000000180061ce0     libucrt:output.obj
 0003:00001cec       $pdata$?state_case_type@?$output_processor@DV?$string_output_adapter@D@__crt_stdio_output@@V?$format_validation_base@DV?$string_output_adapter@D@__crt_stdio_output@@@2@@__crt_stdio_output@@AEAA_NXZ 0000000180061cec     libucrt:output.obj
 0003:00001cf8       $pdata$?type_case_c_tchar@?$output_processor@DV?$string_output_adapter@D@__crt_stdio_output@@V?$format_validation_base@DV?$string_output_adapter@D@__crt_stdio_output@@@2@@__crt_stdio_output@@AEAA_ND@Z 0000000180061cf8     libucrt:output.obj
 0003:00001d04       $pdata$?type_case_s@?$output_processor@DV?$string_output_adapter@D@__crt_stdio_output@@V?$format_validation_base@DV?$string_output_adapter@D@__crt_stdio_output@@@2@@__crt_stdio_output@@AEAA_NXZ 0000000180061d04     libucrt:output.obj
 0003:00001d10       $pdata$?type_case_a@?$output_processor@DV?$string_output_adapter@D@__crt_stdio_output@@V?$format_validation_base@DV?$string_output_adapter@D@__crt_stdio_output@@@2@@__crt_stdio_output@@AEAA_NXZ 0000000180061d10     libucrt:output.obj
 0003:00001d1c       $pdata$?type_case_integer@?$output_processor@DV?$string_output_adapter@D@__crt_stdio_output@@V?$format_validation_base@DV?$string_output_adapter@D@__crt_stdio_output@@@2@@__crt_stdio_output@@AEAA_NI_N@Z 0000000180061d1c     libucrt:output.obj
 0003:00001d28       $pdata$?type_case_n@?$output_processor@DV?$string_output_adapter@D@__crt_stdio_output@@V?$format_validation_base@DV?$string_output_adapter@D@__crt_stdio_output@@@2@@__crt_stdio_output@@AEAA_NXZ 0000000180061d28     libucrt:output.obj
 0003:00001d34       $pdata$?write_stored_string_tchar@?$output_processor@DV?$string_output_adapter@D@__crt_stdio_output@@V?$format_validation_base@DV?$string_output_adapter@D@__crt_stdio_output@@@2@@__crt_stdio_output@@AEAA_ND@Z 0000000180061d34     libucrt:output.obj
 0003:00001d40       $pdata$??$type_case_integer_parse_into_buffer@_K@?$output_processor@DV?$string_output_adapter@D@__crt_stdio_output@@V?$format_validation_base@DV?$string_output_adapter@D@__crt_stdio_output@@@2@@__crt_stdio_output@@AEAAX_KI_N@Z 0000000180061d40     libucrt:output.obj
 0003:00001d4c       $pdata$??$type_case_integer_parse_into_buffer@I@?$output_processor@DV?$string_output_adapter@D@__crt_stdio_output@@V?$format_validation_base@DV?$string_output_adapter@D@__crt_stdio_output@@@2@@__crt_stdio_output@@AEAAXII_N@Z 0000000180061d4c     libucrt:output.obj
 0003:00001d58       $pdata$terminate           0000000180061d58     libucrt:terminate.obj
 0003:00001d64       $pdata$localeconv          0000000180061d64     libucrt:localeconv.obj
 0003:00001d70       $pdata$_get_osfhandle      0000000180061d70     libucrt:osfinfo.obj
 0003:00001d7c       $pdata$_free_osfhnd        0000000180061d7c     libucrt:osfinfo.obj
 0003:00001d88       $pdata$__acrt_lowio_create_handle_array 0000000180061d88     libucrt:osfinfo.obj
 0003:00001d94       $pdata$__acrt_lowio_destroy_handle_array 0000000180061d94     libucrt:osfinfo.obj
 0003:00001da0       $pdata$__acrt_lowio_ensure_fh_exists 0000000180061da0     libucrt:osfinfo.obj
 0003:00001dac       $pdata$__acrt_initialize_lowio$fin$0 0000000180061dac     libucrt:ioinit.obj
 0003:00001dac       $pdata$__acrt_lowio_ensure_fh_exists$fin$0 0000000180061dac     libucrt:osfinfo.obj
 0003:00001db8       $pdata$_isatty             0000000180061db8     libucrt:isatty.obj
 0003:00001dc4       $pdata$log2                0000000180061dc4     libucrt:log2.obj
 0003:00001dd0       $pdata$round               0000000180061dd0     libucrt:round.obj
 0003:00001ddc       $pdata$_isleadbyte_l       0000000180061ddc     libucrt:_wctype.obj
 0003:00001de8       $pdata$wcsncpy             0000000180061de8     libucrt:wcsncpy.obj
 0003:00001df4       $pdata$wcstok              0000000180061df4     libucrt:wcstok.obj
 0003:00001e18       $pdata$__acrt_initialize_locks 0000000180061e18     libucrt:locks.obj
 0003:00001e24       $pdata$__acrt_uninitialize_locks 0000000180061e24     libucrt:locks.obj
 0003:00001e30       $pdata$_lock_locales       0000000180061e30     libucrt:locks.obj
 0003:00001e3c       $pdata$setlocale           0000000180061e3c     libucrt:setlocale.obj
 0003:00001e48       $pdata$??R<lambda_b37934c380d97b75fd242ea49540127a>@@QEBAPEADXZ 0000000180061e48     libucrt:setlocale.obj
 0003:00001e54       $pdata$??$?RV<lambda_41e84717acc955b55e9d0d529e507b68>@@AEAV<lambda_b37934c380d97b75fd242ea49540127a>@@V<lambda_bb6db9f9ac473960206e0d4b942b5506>@@@?$__crt_seh_guarded_call@PEAD@@QEAAPEAD$$QEAV<lambda_41e84717acc955b55e9d0d529e507b68>@@AEAV<lambda_b37934c380d97b75fd242ea49540127a>@@$$QEAV<lambda_bb6db9f9ac473960206e0d4b942b5506>@@@Z 0000000180061e54     libucrt:setlocale.obj
 0003:00001e60       $pdata$?fin$0@?0???$?RV<lambda_0ae27a3a962d80f24befdcbee591983d>@@AEAV<lambda_8d0ee55de4b1038c4002e0adecdf1839>@@V<lambda_dc504788e8f1664fe9b84e20bfb512f2>@@@?$__crt_seh_guarded_call@X@@QEAAX$$QEAV<lambda_0ae27a3a962d80f24befdcbee591983d>@@AEAV<lambda_8d0ee55de4b1038c4002e0adecdf1839>@@$$QEAV<lambda_dc504788e8f1664fe9b84e20bfb512f2>@@@Z@4HA 0000000180061e60     libucrt:per_thread_data.obj
 0003:00001e60       $pdata$?fin$0@?0???$?RV<lambda_2d41944a1d46af3157314b8a01080d33>@@AEAV<lambda_8f455de75cd7d7f24b4096f044d8b9e6>@@V<lambda_aa500f224e6afead328df44964fe2772>@@@?$__crt_seh_guarded_call@X@@QEAAX$$QEAV<lambda_2d41944a1d46af3157314b8a01080d33>@@AEAV<lambda_8f455de75cd7d7f24b4096f044d8b9e6>@@$$QEAV<lambda_aa500f224e6afead328df44964fe2772>@@@Z@4HA 0000000180061e60     libucrt:per_thread_data.obj
 0003:00001e60       $pdata$?fin$0@?0???$?RV<lambda_aa87e3671a710a21b5dc78c0bdf72e11>@@AEAV<lambda_92619d2358a28f41a33ba319515a20b9>@@V<lambda_6992ecaafeb10aed2b74cb1fae11a551>@@@?$__crt_seh_guarded_call@X@@QEAAX$$QEAV<lambda_aa87e3671a710a21b5dc78c0bdf72e11>@@AEAV<lambda_92619d2358a28f41a33ba319515a20b9>@@$$QEAV<lambda_6992ecaafeb10aed2b74cb1fae11a551>@@@Z@4HA 0000000180061e60     libucrt:per_thread_data.obj
 0003:00001e60       $pdata$?fin$0@?0???$?RV<lambda_f2e299630e499de9f9a165e60fcd3db5>@@AEAV<lambda_2ae9d31cdba2644fcbeaf08da7c24588>@@V<lambda_40d01ff24d0e7b3814fdbdcee8eab3c7>@@@?$__crt_seh_guarded_call@X@@QEAAX$$QEAV<lambda_f2e299630e499de9f9a165e60fcd3db5>@@AEAV<lambda_2ae9d31cdba2644fcbeaf08da7c24588>@@$$QEAV<lambda_40d01ff24d0e7b3814fdbdcee8eab3c7>@@@Z@4HA 0000000180061e60     libucrt:per_thread_data.obj
 0003:00001e60       $pdata$?fin$0@?0???$?RV<lambda_48fc4a32460bb0512d3b13f8499328be>@@AEAV<lambda_6c3dac0a4f3f9cefca9bb494422f9b77>@@V<lambda_0a2f2c9f9a56eb2b08bfa6ff61d331c5>@@@?$__crt_seh_guarded_call@H@@QEAAH$$QEAV<lambda_48fc4a32460bb0512d3b13f8499328be>@@AEAV<lambda_6c3dac0a4f3f9cefca9bb494422f9b77>@@$$QEAV<lambda_0a2f2c9f9a56eb2b08bfa6ff61d331c5>@@@Z@4HA 0000000180061e60     libucrt:winapi_thunks.obj
 0003:00001e60       $pdata$?fin$0@?0???$?RV<lambda_41e84717acc955b55e9d0d529e507b68>@@AEAV<lambda_b37934c380d97b75fd242ea49540127a>@@V<lambda_bb6db9f9ac473960206e0d4b942b5506>@@@?$__crt_seh_guarded_call@PEAD@@QEAAPEAD$$QEAV<lambda_41e84717acc955b55e9d0d529e507b68>@@AEAV<lambda_b37934c380d97b75fd242ea49540127a>@@$$QEAV<lambda_bb6db9f9ac473960206e0d4b942b5506>@@@Z@4HA 0000000180061e60     libucrt:setlocale.obj
 0003:00001e60       $pdata$?fin$0@?0???$?RV<lambda_1d892b297fdedeee07ed8124eeb2f2fa>@@AEAV<lambda_ffc046909424fd52df0ac47e64813305>@@V<lambda_01a7098693036236037e7cdb9bca3d73>@@@?$__crt_seh_guarded_call@X@@QEAAX$$QEAV<lambda_1d892b297fdedeee07ed8124eeb2f2fa>@@AEAV<lambda_ffc046909424fd52df0ac47e64813305>@@$$QEAV<lambda_01a7098693036236037e7cdb9bca3d73>@@@Z@4HA 0000000180061e60     libucrt:wsetlocale.obj
 0003:00001e60       $pdata$?fin$0@?0???$?RV<lambda_efdfa57d1f175319df784efa44bb7b81>@@AEAV<lambda_5f0a4c1567f8adc6734073e5d1e1b35c>@@V<lambda_2e8a7d3640ea6ccb4c2413664c2db6fd>@@@?$__crt_seh_guarded_call@X@@QEAAX$$QEAV<lambda_efdfa57d1f175319df784efa44bb7b81>@@AEAV<lambda_5f0a4c1567f8adc6734073e5d1e1b35c>@@$$QEAV<lambda_2e8a7d3640ea6ccb4c2413664c2db6fd>@@@Z@4HA 0000000180061e60     libucrt:mbctype.obj
 0003:00001e60       $pdata$?fin$0@?0???$?RV<lambda_450d765d439847d4c735a33c368b5fc0>@@AEAV<lambda_44731a7d0e6d81c3e6aa82d741081786>@@V<lambda_601a2a7da3b7a96e9554ac7215c4b07c>@@@?$__crt_seh_guarded_call@P6AXH@Z@@QEAAP6AXH@Z$$QEAV<lambda_450d765d439847d4c735a33c368b5fc0>@@AEAV<lambda_44731a7d0e6d81c3e6aa82d741081786>@@$$QEAV<lambda_601a2a7da3b7a96e9554ac7215c4b07c>@@@Z@4HA 0000000180061e60     libucrt:signal.obj
 0003:00001e60       $pdata$?fin$0@?0???$?RV<lambda_d80eeec6fff315bfe5c115232f3240e3>@@AEAV<lambda_6e4b09c48022b2350581041d5f6b0c4c>@@V<lambda_2358e3775559c9db80273638284d5e45>@@@?$__crt_seh_guarded_call@X@@QEAAX$$QEAV<lambda_d80eeec6fff315bfe5c115232f3240e3>@@AEAV<lambda_6e4b09c48022b2350581041d5f6b0c4c>@@$$QEAV<lambda_2358e3775559c9db80273638284d5e45>@@@Z@4HA 0000000180061e60     libucrt:exit.obj
 0003:00001e60       $pdata$?fin$0@?0???$?RV<lambda_638799b9deba96c50f710eeac98168cd>@@AEAV<lambda_22ebabd17bc4fa466a2aca6d8deb888d>@@V<lambda_a6f7d7db0129f75315ebf26d50c089f1>@@@?$__crt_seh_guarded_call@H@@QEAAH$$QEAV<lambda_638799b9deba96c50f710eeac98168cd>@@AEAV<lambda_22ebabd17bc4fa466a2aca6d8deb888d>@@$$QEAV<lambda_a6f7d7db0129f75315ebf26d50c089f1>@@@Z@4HA 0000000180061e60     libucrt:onexit.obj
 0003:00001e60       $pdata$?fin$0@?0???$?RV<lambda_7777bce6b2f8c936911f934f8298dc43>@@AEAV<lambda_f03950bc5685219e0bcd2087efbe011e>@@V<lambda_3883c3dff614d5e0c5f61bb1ac94921c>@@@?$__crt_seh_guarded_call@H@@QEAAH$$QEAV<lambda_7777bce6b2f8c936911f934f8298dc43>@@AEAV<lambda_f03950bc5685219e0bcd2087efbe011e>@@$$QEAV<lambda_3883c3dff614d5e0c5f61bb1ac94921c>@@@Z@4HA 0000000180061e60     libucrt:onexit.obj
 0003:00001e6c       $pdata$___mb_cur_max_func  0000000180061e6c     libucrt:initctype.obj
 0003:00001e78       $pdata$__acrt_locale_initialize_ctype 0000000180061e78     libucrt:initctype.obj
 0003:00001e84       $pdata$___lc_locale_name_func 0000000180061e84     libucrt:initctype.obj
 0003:00001e90       $pdata$___lc_codepage_func 0000000180061e90     libucrt:initctype.obj
 0003:00001e9c       $pdata$__pctype_func       0000000180061e9c     libucrt:ctype.obj
 0003:00001ea8       $pdata$_ischartype_l       0000000180061ea8     libucrt:strtod.obj
 0003:00001eb4       $pdata$memcpy_s            0000000180061eb4     libucrt:cfout.obj
 0003:00001eb4       $pdata$memcpy_s            0000000180061eb4     libucrt:strtod.obj
 0003:00001ec0       $pdata$?divide@__crt_strtox@@YA_KAEAUbig_integer@1@AEBU21@@Z 0000000180061ec0     libucrt:strtod.obj
 0003:00001ecc       $pdata$0$?divide@__crt_strtox@@YA_KAEAUbig_integer@1@AEBU21@@Z 0000000180061ecc     libucrt:strtod.obj
 0003:00001ed8       $pdata$1$?divide@__crt_strtox@@YA_KAEAUbig_integer@1@AEBU21@@Z 0000000180061ed8     libucrt:strtod.obj
 0003:00001ef0       $pdata$abort               0000000180061ef0     libucrt:abort.obj
 0003:00001efc       $pdata$_wcsdup             0000000180061efc     libucrt:wcsdup.obj
 0003:00001f08       $pdata$??$__acrt_mbs_to_wcs_cp@U__crt_win32_buffer_internal_dynamic_resizing@@@@YAHQEBDAEAV?$__crt_win32_buffer@_WU__crt_win32_buffer_internal_dynamic_resizing@@@@I@Z 0000000180061f08     libucrt:strftime.obj
 0003:00001f14       $pdata$??$__acrt_wcs_to_mbs_cp@U__crt_win32_buffer_no_resizing@@@@YAHQEB_WAEAV?$__crt_win32_buffer@DU__crt_win32_buffer_no_resizing@@@@I@Z 0000000180061f14     libucrt:strftime.obj
 0003:00001f20       $pdata$wcscpy_s            0000000180061f20     libucrt:wcscpy_s.obj
 0003:00001f2c       $pdata$_seh_filter_exe     0000000180061f2c     libucrt:exception_filter.obj
 0003:00001f38       $pdata$?try_cor_exit_process@@YAXI@Z 0000000180061f38     libucrt:exit.obj
 0003:00001f44       $pdata$?exit_or_terminate_process@@YAXI@Z 0000000180061f44     libucrt:exit.obj
 0003:00001f50       $pdata$?common_exit@@YAXHW4_crt_exit_cleanup_mode@@W4_crt_exit_return_mode@@@Z 0000000180061f50     libucrt:exit.obj
 0003:00001f5c       $pdata$??R<lambda_6e4b09c48022b2350581041d5f6b0c4c>@@QEBA@XZ 0000000180061f5c     libucrt:exit.obj
 0003:00001f68       $pdata$?filt$0@?0???R<lambda_6e4b09c48022b2350581041d5f6b0c4c>@@QEBA@XZ@4HA 0000000180061f68     libucrt:exit.obj
 0003:00001f74       $pdata$??$?RV<lambda_d80eeec6fff315bfe5c115232f3240e3>@@AEAV<lambda_6e4b09c48022b2350581041d5f6b0c4c>@@V<lambda_2358e3775559c9db80273638284d5e45>@@@?$__crt_seh_guarded_call@X@@QEAAX$$QEAV<lambda_d80eeec6fff315bfe5c115232f3240e3>@@AEAV<lambda_6e4b09c48022b2350581041d5f6b0c4c>@@$$QEAV<lambda_2358e3775559c9db80273638284d5e45>@@@Z 0000000180061f74     libucrt:exit.obj
 0003:00001f80       $pdata$_configure_narrow_argv 0000000180061f80     libucrt:argv_parsing.obj
 0003:00001f8c       $pdata$__acrt_allocate_buffer_for_argv 0000000180061f8c     libucrt:argv_parsing.obj
 0003:00001f98       $pdata$??$parse_command_line@D@@YAXPEADPEAPEAD0PEA_K2@Z 0000000180061f98     libucrt:argv_parsing.obj
 0003:00001fa4       $pdata$__dcrt_uninitialize_environments_nolock 0000000180061fa4     libucrt:environment_initialization.obj
 0003:00001fb0       $pdata$??$common_initialize_environment_nolock@D@@YAHXZ 0000000180061fb0     libucrt:environment_initialization.obj
 0003:00001fbc       $pdata$??$uninitialize_environment_internal@D@@YAXAEAPEAPEAD@Z 0000000180061fbc     libucrt:environment_initialization.obj
 0003:00001fc8       $pdata$??$uninitialize_environment_internal@_W@@YAXAEAPEAPEA_W@Z 0000000180061fc8     libucrt:environment_initialization.obj
 0003:00001fd4       $pdata$??$free_environment@D@@YAXQEAPEAD@Z 0000000180061fd4     libucrt:environment_initialization.obj
 0003:00001fd4       $pdata$??$free_environment@_W@@YAXQEAPEA_W@Z 0000000180061fd4     libucrt:environment_initialization.obj
 0003:00001fe0       $pdata$??$create_environment@D@@YAQEAPEADQEAD@Z 0000000180061fe0     libucrt:environment_initialization.obj
 0003:00001fec       $pdata$_register_onexit_function 0000000180061fec     libucrt:onexit.obj
 0003:00001ff8       $pdata$_execute_onexit_table 0000000180061ff8     libucrt:onexit.obj
 0003:00002004       $pdata$??R<lambda_22ebabd17bc4fa466a2aca6d8deb888d>@@QEBAHXZ 0000000180062004     libucrt:onexit.obj
 0003:00002010       $pdata$??R<lambda_f03950bc5685219e0bcd2087efbe011e>@@QEBAHXZ 0000000180062010     libucrt:onexit.obj
 0003:0000201c       $pdata$??$?RV<lambda_638799b9deba96c50f710eeac98168cd>@@AEAV<lambda_22ebabd17bc4fa466a2aca6d8deb888d>@@V<lambda_a6f7d7db0129f75315ebf26d50c089f1>@@@?$__crt_seh_guarded_call@H@@QEAAH$$QEAV<lambda_638799b9deba96c50f710eeac98168cd>@@AEAV<lambda_22ebabd17bc4fa466a2aca6d8deb888d>@@$$QEAV<lambda_a6f7d7db0129f75315ebf26d50c089f1>@@@Z 000000018006201c     libucrt:onexit.obj
 0003:00002028       $pdata$??$?RV<lambda_7777bce6b2f8c936911f934f8298dc43>@@AEAV<lambda_f03950bc5685219e0bcd2087efbe011e>@@V<lambda_3883c3dff614d5e0c5f61bb1ac94921c>@@@?$__crt_seh_guarded_call@H@@QEAAH$$QEAV<lambda_7777bce6b2f8c936911f934f8298dc43>@@AEAV<lambda_f03950bc5685219e0bcd2087efbe011e>@@$$QEAV<lambda_3883c3dff614d5e0c5f61bb1ac94921c>@@@Z 0000000180062028     libucrt:onexit.obj
 0003:00002034       $pdata$__acrt_uninitialize 0000000180062034     libucrt:initialization.obj
 0003:00002040       $pdata$__acrt_uninitialize_critical 0000000180062040     libucrt:initialization.obj
 0003:0000204c       $pdata$__acrt_thread_attach 000000018006204c     libucrt:initialization.obj
 0003:00002058       $pdata$__acrt_thread_detach 0000000180062058     libucrt:initialization.obj
 0003:00002064       $pdata$initialize_c        0000000180062064     libucrt:initialization.obj
 0003:00002070       $pdata$uninitialize_environment 0000000180062070     libucrt:initialization.obj
 0003:0000207c       $pdata$initialize_pointers 000000018006207c     libucrt:initialization.obj
 0003:00002088       $pdata$uninitialize_allocated_memory 0000000180062088     libucrt:initialization.obj
 0003:00002094       $pdata$uninitialize_allocated_io_buffers 0000000180062094     libucrt:initialization.obj
 0003:000020a0       $pdata$_callnewh           00000001800620a0     libucrt:new_handler.obj
 0003:000020ac       $pdata$_query_new_handler  00000001800620ac     libucrt:new_handler.obj
 0003:000020b8       $pdata$_query_new_handler$fin$0 00000001800620b8     libucrt:new_handler.obj
 0003:000020c4       $pdata$_initterm           00000001800620c4     libucrt:initterm.obj
 0003:000020d0       $pdata$_initterm_e         00000001800620d0     libucrt:initterm.obj
 0003:000020dc       $pdata$strcpy_s            00000001800620dc     libucrt:strcpy_s.obj
 0003:000020e8       $pdata$_wtol               00000001800620e8     libucrt:atox.obj
 0003:000020f4       $pdata$??$parse_integer@KV?$c_string_character_source@D@__crt_strtox@@@__crt_strtox@@YAKQEAU__crt_locale_pointers@@V?$c_string_character_source@D@0@H_N@Z 00000001800620f4     libucrt:atox.obj
 0003:00002100       $pdata$??$parse_integer@KV?$c_string_character_source@_W@__crt_strtox@@@__crt_strtox@@YAKQEAU__crt_locale_pointers@@V?$c_string_character_source@_W@0@H_N@Z 0000000180062100     libucrt:atox.obj
 0003:00002118       $pdata$__acrt_initialize_ptd 0000000180062118     libucrt:per_thread_data.obj
 0003:00002124       $pdata$__acrt_uninitialize_ptd 0000000180062124     libucrt:per_thread_data.obj
 0003:00002130       $pdata$__acrt_getptd       0000000180062130     libucrt:per_thread_data.obj
 0003:0000213c       $pdata$__acrt_getptd_head  000000018006213c     libucrt:per_thread_data.obj
 0003:00002148       $pdata$__acrt_getptd_noexit 0000000180062148     libucrt:per_thread_data.obj
 0003:00002154       $pdata$__acrt_freeptd      0000000180062154     libucrt:per_thread_data.obj
 0003:00002160       $pdata$?destroy_fls@@YAXPEAX@Z 0000000180062160     libucrt:per_thread_data.obj
 0003:0000216c       $pdata$?replace_current_thread_locale_nolock@@YAXQEAU__acrt_ptd@@QEAU__crt_locale_data@@@Z 000000018006216c     libucrt:per_thread_data.obj
 0003:00002178       $pdata$?construct_ptd_array@@YAXQEAU__acrt_ptd@@@Z 0000000180062178     libucrt:per_thread_data.obj
 0003:00002184       $pdata$?destroy_ptd_array@@YAXQEAU__acrt_ptd@@@Z 0000000180062184     libucrt:per_thread_data.obj
 0003:00002190       $pdata$??$?RV<lambda_0ae27a3a962d80f24befdcbee591983d>@@AEAV<lambda_8d0ee55de4b1038c4002e0adecdf1839>@@V<lambda_dc504788e8f1664fe9b84e20bfb512f2>@@@?$__crt_seh_guarded_call@X@@QEAAX$$QEAV<lambda_0ae27a3a962d80f24befdcbee591983d>@@AEAV<lambda_8d0ee55de4b1038c4002e0adecdf1839>@@$$QEAV<lambda_dc504788e8f1664fe9b84e20bfb512f2>@@@Z 0000000180062190     libucrt:per_thread_data.obj
 0003:0000219c       $pdata$??$?RV<lambda_aa87e3671a710a21b5dc78c0bdf72e11>@@AEAV<lambda_92619d2358a28f41a33ba319515a20b9>@@V<lambda_6992ecaafeb10aed2b74cb1fae11a551>@@@?$__crt_seh_guarded_call@X@@QEAAX$$QEAV<lambda_aa87e3671a710a21b5dc78c0bdf72e11>@@AEAV<lambda_92619d2358a28f41a33ba319515a20b9>@@$$QEAV<lambda_6992ecaafeb10aed2b74cb1fae11a551>@@@Z 000000018006219c     libucrt:per_thread_data.obj
 0003:000021a8       $pdata$??$?RV<lambda_f2e299630e499de9f9a165e60fcd3db5>@@AEAV<lambda_2ae9d31cdba2644fcbeaf08da7c24588>@@V<lambda_40d01ff24d0e7b3814fdbdcee8eab3c7>@@@?$__crt_seh_guarded_call@X@@QEAAX$$QEAV<lambda_f2e299630e499de9f9a165e60fcd3db5>@@AEAV<lambda_2ae9d31cdba2644fcbeaf08da7c24588>@@$$QEAV<lambda_40d01ff24d0e7b3814fdbdcee8eab3c7>@@@Z 00000001800621a8     libucrt:per_thread_data.obj
 0003:000021b4       $pdata$??$?RV<lambda_2d41944a1d46af3157314b8a01080d33>@@AEAV<lambda_8f455de75cd7d7f24b4096f044d8b9e6>@@V<lambda_aa500f224e6afead328df44964fe2772>@@@?$__crt_seh_guarded_call@X@@QEAAX$$QEAV<lambda_2d41944a1d46af3157314b8a01080d33>@@AEAV<lambda_8f455de75cd7d7f24b4096f044d8b9e6>@@$$QEAV<lambda_aa500f224e6afead328df44964fe2772>@@@Z 00000001800621b4     libucrt:per_thread_data.obj
 0003:000021c0       $pdata$_calloc_base        00000001800621c0     libucrt:calloc_base.obj
 0003:000021cc       $pdata$_free_base          00000001800621cc     libucrt:free_base.obj
 0003:000021d8       $pdata$__acrt_initialize_winapi_thunks 00000001800621d8     libucrt:winapi_thunks.obj
 0003:000021e4       $pdata$__acrt_uninitialize_winapi_thunks 00000001800621e4     libucrt:winapi_thunks.obj
 0003:000021f0       $pdata$__acrt_AreFileApisANSI 00000001800621f0     libucrt:winapi_thunks.obj
 0003:000021fc       $pdata$__acrt_EnumSystemLocalesEx 00000001800621fc     libucrt:winapi_thunks.obj
 0003:00002208       $pdata$__acrt_FlsAlloc     0000000180062208     libucrt:winapi_thunks.obj
 0003:00002214       $pdata$__acrt_FlsFree      0000000180062214     libucrt:winapi_thunks.obj
 0003:00002220       $pdata$__acrt_FlsGetValue  0000000180062220     libucrt:winapi_thunks.obj
 0003:0000222c       $pdata$__acrt_FlsSetValue  000000018006222c     libucrt:winapi_thunks.obj
 0003:00002238       $pdata$__acrt_GetLocaleInfoEx 0000000180062238     libucrt:winapi_thunks.obj
 0003:00002244       $pdata$__acrt_GetUserDefaultLocaleName 0000000180062244     libucrt:winapi_thunks.obj
 0003:00002250       $pdata$__acrt_InitializeCriticalSectionEx 0000000180062250     libucrt:winapi_thunks.obj
 0003:0000225c       $pdata$__acrt_IsValidLocaleName 000000018006225c     libucrt:winapi_thunks.obj
 0003:00002268       $pdata$__acrt_LCMapStringEx 0000000180062268     libucrt:winapi_thunks.obj
 0003:00002274       $pdata$__acrt_LCIDToLocaleName 0000000180062274     libucrt:winapi_thunks.obj
 0003:00002280       $pdata$__acrt_LocaleNameToLCID 0000000180062280     libucrt:winapi_thunks.obj
 0003:0000228c       $pdata$__acrt_AppPolicyGetProcessTerminationMethodInternal 000000018006228c     libucrt:winapi_thunks.obj
 0003:00002298       $pdata$__acrt_can_use_vista_locale_apis 0000000180062298     libucrt:winapi_thunks.obj
 0003:000022a4       $pdata$__acrt_eagerly_load_locale_apis 00000001800622a4     libucrt:winapi_thunks.obj
 0003:000022b0       $pdata$?try_get_function@@YAPEAXW4function_id@?A0x391cf84c@@QEBDQEBW4module_id@2@2@Z 00000001800622b0     libucrt:winapi_thunks.obj
 0003:000022bc       $pdata$??$?RV<lambda_48fc4a32460bb0512d3b13f8499328be>@@AEAV<lambda_6c3dac0a4f3f9cefca9bb494422f9b77>@@V<lambda_0a2f2c9f9a56eb2b08bfa6ff61d331c5>@@@?$__crt_seh_guarded_call@H@@QEAAH$$QEAV<lambda_48fc4a32460bb0512d3b13f8499328be>@@AEAV<lambda_6c3dac0a4f3f9cefca9bb494422f9b77>@@$$QEAV<lambda_0a2f2c9f9a56eb2b08bfa6ff61d331c5>@@@Z 00000001800622bc     libucrt:winapi_thunks.obj
 0003:000022c8       $pdata$_fcloseall          00000001800622c8     libucrt:closeall.obj
 0003:000022d4       $pdata$_fcloseall$fin$0    00000001800622d4     libucrt:closeall.obj
 0003:000022e0       $pdata$_fflush_nolock      00000001800622e0     libucrt:fflush.obj
 0003:000022ec       $pdata$__acrt_stdio_flush_nolock 00000001800622ec     libucrt:fflush.obj
 0003:000022f8       $pdata$?common_flush_all@@YAH_N@Z 00000001800622f8     libucrt:fflush.obj
 0003:00002304       $pdata$??$?RV<lambda_842d9ff0dc9ef11c61343bbaebe7f885>@@AEAV<lambda_c5860995281e5c4ce005b3de8f5874ee>@@V<lambda_d90129c13df834fdcbf8d2b88dafcf2d>@@@?$__crt_seh_guarded_call@X@@QEAAX$$QEAV<lambda_842d9ff0dc9ef11c61343bbaebe7f885>@@AEAV<lambda_c5860995281e5c4ce005b3de8f5874ee>@@$$QEAV<lambda_d90129c13df834fdcbf8d2b88dafcf2d>@@@Z 0000000180062304     libucrt:fflush.obj
 0003:00002310       $pdata$?fin$0@?0???$?RV<lambda_842d9ff0dc9ef11c61343bbaebe7f885>@@AEAV<lambda_c5860995281e5c4ce005b3de8f5874ee>@@V<lambda_d90129c13df834fdcbf8d2b88dafcf2d>@@@?$__crt_seh_guarded_call@X@@QEAAX$$QEAV<lambda_842d9ff0dc9ef11c61343bbaebe7f885>@@AEAV<lambda_c5860995281e5c4ce005b3de8f5874ee>@@$$QEAV<lambda_d90129c13df834fdcbf8d2b88dafcf2d>@@@Z@4HA 0000000180062310     libucrt:fflush.obj
 0003:0000231c       $pdata$??$?RV<lambda_886d6c58226a84441f68b9f2b8217b83>@@AEAV<lambda_ab61a845afdef5b7c387490eaf3616ee>@@V<lambda_f7f22ab5edc0698d5f6905b0d3f44752>@@@?$__crt_seh_guarded_call@X@@QEAAX$$QEAV<lambda_886d6c58226a84441f68b9f2b8217b83>@@AEAV<lambda_ab61a845afdef5b7c387490eaf3616ee>@@$$QEAV<lambda_f7f22ab5edc0698d5f6905b0d3f44752>@@@Z 000000018006231c     libucrt:fflush.obj
 0003:00002328       $pdata$?fin$0@?0???$?RV<lambda_886d6c58226a84441f68b9f2b8217b83>@@AEAV<lambda_ab61a845afdef5b7c387490eaf3616ee>@@V<lambda_f7f22ab5edc0698d5f6905b0d3f44752>@@@?$__crt_seh_guarded_call@X@@QEAAX$$QEAV<lambda_886d6c58226a84441f68b9f2b8217b83>@@AEAV<lambda_ab61a845afdef5b7c387490eaf3616ee>@@$$QEAV<lambda_f7f22ab5edc0698d5f6905b0d3f44752>@@@Z@4HA 0000000180062328     libucrt:fflush.obj
 0003:00002334       $pdata$__acrt_stdio_free_buffer_nolock 0000000180062334     libucrt:_freebuf.obj
 0003:00002340       $pdata$__acrt_initialize_lowio 0000000180062340     libucrt:ioinit.obj
 0003:0000234c       $pdata$__acrt_uninitialize_lowio 000000018006234c     libucrt:ioinit.obj
 0003:00002358       $pdata$?initialize_inherited_file_handles_nolock@@YAXXZ 0000000180062358     libucrt:ioinit.obj
 0003:00002364       $pdata$?initialize_stdio_handles_nolock@@YAXXZ 0000000180062364     libucrt:ioinit.obj
 0003:00002370       $pdata$_write              0000000180062370     libucrt:write.obj
 0003:0000237c       $pdata$_write$fin$0        000000018006237c     libucrt:write.obj
 0003:00002388       $pdata$_write_nolock       0000000180062388     libucrt:write.obj
 0003:00002394       $pdata$?write_double_translated_ansi_nolock@@YA?AUwrite_result@?A0x17268360@@HQEBDI@Z 0000000180062394     libucrt:write.obj
 0003:000023a0       $pdata$?write_text_ansi_nolock@@YA?AUwrite_result@?A0x17268360@@HQEBDI@Z 00000001800623a0     libucrt:write.obj
 0003:000023ac       $pdata$?write_text_utf16le_nolock@@YA?AUwrite_result@?A0x17268360@@HQEBDI@Z 00000001800623ac     libucrt:write.obj
 0003:000023b8       $pdata$?write_text_utf8_nolock@@YA?AUwrite_result@?A0x17268360@@HQEBDI@Z 00000001800623b8     libucrt:write.obj
 0003:000023c4       $pdata$_malloc_base        00000001800623c4     libucrt:malloc_base.obj
 0003:000023d0       $pdata$strtol              00000001800623d0     libucrt:strtox.obj
 0003:000023dc       $pdata$_mbtowc_l           00000001800623dc     libucrt:mbtowc.obj
 0003:000023e8       $pdata$wctomb_s            00000001800623e8     libucrt:wctomb.obj
 0003:000023f4       $pdata$_wctomb_s_l         00000001800623f4     libucrt:wctomb.obj
 0003:00002400       $pdata$__acrt_update_locale_info 0000000180062400     libucrt:locale_update.obj
 0003:0000240c       $pdata$__acrt_update_multibyte_info 000000018006240c     libucrt:locale_update.obj
 0003:00002418       $pdata$__acrt_fp_format    0000000180062418     libucrt:cvt.obj
 0003:00002424       $pdata$?fp_format_e_internal@@YAHQEAD_KH_NIQEAU_strflt@@2QEAU__crt_locale_pointers@@@Z 0000000180062424     libucrt:cvt.obj
 0003:00002430       $pdata$?fp_format_e@@YAHQEBNQEAD_K12H_NIQEAU__crt_locale_pointers@@@Z 0000000180062430     libucrt:cvt.obj
 0003:0000243c       $pdata$?fp_format_a@@YAHQEBNPEAD_KQEAD2H_NIQEAU__crt_locale_pointers@@@Z 000000018006243c     libucrt:cvt.obj
 0003:00002448       $pdata$?fp_format_f_internal@@YAHQEAD_KHQEAU_strflt@@_NQEAU__crt_locale_pointers@@@Z 0000000180062448     libucrt:cvt.obj
 0003:00002454       $pdata$?fp_format_g@@YAHQEBNQEAD_K12H_NIQEAU__crt_locale_pointers@@@Z 0000000180062454     libucrt:cvt.obj
 0003:00002460       $pdata$__acrt_copy_locale_name 0000000180062460     libucrt:wsetlocale.obj
 0003:0000246c       $pdata$_wsetlocale         000000018006246c     libucrt:wsetlocale.obj
 0003:00002478       $pdata$_expandlocale       0000000180062478     libucrt:wsetlocale.obj
 0003:00002484       $pdata$_wcscats            0000000180062484     libucrt:wsetlocale.obj
 0003:00002490       $pdata$__lc_lctowcs        0000000180062490     libucrt:wsetlocale.obj
 0003:0000249c       $pdata$__lc_wcstolc        000000018006249c     libucrt:wsetlocale.obj
 0003:000024a8       $pdata$_wsetlocale_set_cat 00000001800624a8     libucrt:wsetlocale.obj
 0003:000024b4       $pdata$_wsetlocale_get_all 00000001800624b4     libucrt:wsetlocale.obj
 0003:000024c0       $pdata$_wsetlocale_nolock  00000001800624c0     libucrt:wsetlocale.obj
 0003:000024cc       $pdata$__acrt_uninitialize_locale 00000001800624cc     libucrt:wsetlocale.obj
 0003:000024d8       $pdata$_copytlocinfo_nolock 00000001800624d8     libucrt:wsetlocale.obj
 0003:000024e4       $pdata$??R<lambda_2a444430fde8c29194d880d93eed5e8f>@@QEBA@XZ 00000001800624e4     libucrt:wsetlocale.obj
 0003:000024f0       $pdata$string_is_alpha     00000001800624f0     libucrt:wsetlocale.obj
 0003:000024fc       $pdata$parse_bcp47_language 00000001800624fc     libucrt:wsetlocale.obj
 0003:00002508       $pdata$parse_bcp47_script  0000000180062508     libucrt:wsetlocale.obj
 0003:00002514       $pdata$parse_bcp47_region  0000000180062514     libucrt:wsetlocale.obj
 0003:00002520       $pdata$parse_bcp47_code_page 0000000180062520     libucrt:wsetlocale.obj
 0003:0000252c       $pdata$parse_bcp47         000000018006252c     libucrt:wsetlocale.obj
 0003:00002538       $pdata$?commit_locale_name@_expandlocale_locale_name_cache@@QEAAXQEB_W_K@Z 0000000180062538     libucrt:wsetlocale.obj
 0003:00002544       $pdata$??$?RV<lambda_410d79af7f07d98d83a3f525b3859a53>@@AEAV<lambda_3e16ef9562a7dcce91392c22ab16ea36>@@V<lambda_38119f0e861e05405d8a144b9b982f0a>@@@?$__crt_seh_guarded_call@X@@QEAAX$$QEAV<lambda_410d79af7f07d98d83a3f525b3859a53>@@AEAV<lambda_3e16ef9562a7dcce91392c22ab16ea36>@@$$QEAV<lambda_38119f0e861e05405d8a144b9b982f0a>@@@Z 0000000180062544     libucrt:wsetlocale.obj
 0003:00002550       $pdata$?fin$0@?0???$?RV<lambda_410d79af7f07d98d83a3f525b3859a53>@@AEAV<lambda_3e16ef9562a7dcce91392c22ab16ea36>@@V<lambda_38119f0e861e05405d8a144b9b982f0a>@@@?$__crt_seh_guarded_call@X@@QEAAX$$QEAV<lambda_410d79af7f07d98d83a3f525b3859a53>@@AEAV<lambda_3e16ef9562a7dcce91392c22ab16ea36>@@$$QEAV<lambda_38119f0e861e05405d8a144b9b982f0a>@@@Z@4HA 0000000180062550     libucrt:wsetlocale.obj
 0003:0000255c       $pdata$??$?RV<lambda_1d892b297fdedeee07ed8124eeb2f2fa>@@AEAV<lambda_ffc046909424fd52df0ac47e64813305>@@V<lambda_01a7098693036236037e7cdb9bca3d73>@@@?$__crt_seh_guarded_call@X@@QEAAX$$QEAV<lambda_1d892b297fdedeee07ed8124eeb2f2fa>@@AEAV<lambda_ffc046909424fd52df0ac47e64813305>@@$$QEAV<lambda_01a7098693036236037e7cdb9bca3d73>@@@Z 000000018006255c     libucrt:wsetlocale.obj
 0003:00002568       $pdata$??$?RV<lambda_7f2adfce497ff2baa965cd4f576ecfd1>@@AEAV<lambda_2a444430fde8c29194d880d93eed5e8f>@@AEAV<lambda_8dff2cf36a5417162780cd64fa2883ef>@@@?$__crt_seh_guarded_call@X@@QEAAX$$QEAV<lambda_7f2adfce497ff2baa965cd4f576ecfd1>@@AEAV<lambda_2a444430fde8c29194d880d93eed5e8f>@@AEAV<lambda_8dff2cf36a5417162780cd64fa2883ef>@@@Z 0000000180062568     libucrt:wsetlocale.obj
 0003:00002574       $pdata$?fin$0@?0???$?RV<lambda_7f2adfce497ff2baa965cd4f576ecfd1>@@AEAV<lambda_2a444430fde8c29194d880d93eed5e8f>@@AEAV<lambda_8dff2cf36a5417162780cd64fa2883ef>@@@?$__crt_seh_guarded_call@X@@QEAAX$$QEAV<lambda_7f2adfce497ff2baa965cd4f576ecfd1>@@AEAV<lambda_2a444430fde8c29194d880d93eed5e8f>@@AEAV<lambda_8dff2cf36a5417162780cd64fa2883ef>@@@Z@4HA 0000000180062574     libucrt:wsetlocale.obj
 0003:00002580       $pdata$mbstowcs_s          0000000180062580     libucrt:mbstowcs.obj
 0003:0000258c       $pdata$_mbstowcs_s_l       000000018006258c     libucrt:mbstowcs.obj
 0003:00002598       $pdata$?_mbstowcs_l_helper@@YA_KPEA_WPEBD_KPEAU__crt_locale_pointers@@@Z 0000000180062598     libucrt:mbstowcs.obj
 0003:000025a4       $pdata$strncpy_s           00000001800625a4     libucrt:strncpy_s.obj
 0003:000025b0       $pdata$_call_matherr       00000001800625b0     libucrt:libm_error.obj
 0003:000025bc       $pdata$_exception_enabled  00000001800625bc     libucrt:libm_error.obj
 0003:000025c8       $pdata$_handle_errorf      00000001800625c8     libucrt:libm_error.obj
 0003:000025d4       $pdata$_handle_error       00000001800625d4     libucrt:libm_error.obj
 0003:000025e0       $pdata$iswctype            00000001800625e0     libucrt:iswctype.obj
 0003:000025ec       $pdata$__acrt_wcstok_s_novalidation 00000001800625ec     libucrt:wcstok_s.obj
 0003:000025f8       $pdata$__acrt_initialize_fma3 00000001800625f8     libucrt:fma3_available.obj
 0003:00002604       $pdata$_log_special_common 0000000180062604     libucrt:log_special.obj
 0003:00002610       $pdata$_log10_special      0000000180062610     libucrt:log_special.obj
 0003:0000261c       $pdata$_powf_special       000000018006261c     libucrt:pow_special.obj
 0003:00002628       $pdata$_pow_special        0000000180062628     libucrt:pow_special.obj
 0003:00002634       $pdata$_wcstombs_s_l       0000000180062634     libucrt:wcstombs.obj
 0003:00002640       $pdata$?_wcstombs_l_helper@@YA_KPEADPEB_W_KPEAU__crt_locale_pointers@@@Z 0000000180062640     libucrt:wcstombs.obj
 0003:0000264c       $pdata$__acrt_GetLocaleInfoA 000000018006264c     libucrt:getlocaleinfoa.obj
 0003:00002658       $pdata$?InternalGetLocaleInfoA@@YAHQEAU__crt_locale_pointers@@QEB_WKQEADH@Z 0000000180062658     libucrt:getlocaleinfoa.obj
 0003:00002664       $pdata$__acrt_GetStringTypeA 0000000180062664     libucrt:getstringtypea.obj
 0003:00002670       $pdata$__acrt_LCMapStringA 0000000180062670     libucrt:lcmapstringa.obj
 0003:0000267c       $pdata$?__acrt_LCMapStringA_stat@@YAHPEAU__crt_locale_pointers@@PEB_WKPEBDHPEADHHH@Z 000000018006267c     libucrt:lcmapstringa.obj
 0003:00002688       $pdata$_set_errno_from_matherr 0000000180062688     libucrt:fpexcept.obj
 0003:00002694       $pdata$_raise_excf         0000000180062694     libucrt:fpexcept.obj
 0003:000026a0       $pdata$_raise_exc          00000001800626a0     libucrt:fpexcept.obj
 0003:000026ac       $pdata$_raise_exc_ex       00000001800626ac     libucrt:fpexcept.obj
 0003:000026b8       $pdata$_clrfp              00000001800626b8     libucrt:fpctrl.obj
 0003:000026c4       $pdata$_ctrlfp             00000001800626c4     libucrt:fpctrl.obj
 0003:000026d0       $pdata$_ctrlfp$filt$0      00000001800626d0     libucrt:fpctrl.obj
 0003:000026dc       $pdata$_statfp             00000001800626dc     libucrt:fpctrl.obj
 0003:000026e8       $pdata$_set_statfp         00000001800626e8     libucrt:fpctrl.obj
 0003:000026f4       $pdata$_realloc_base       00000001800626f4     libucrt:realloc_base.obj
 0003:00002700       $pdata$_isctype_l          0000000180062700     libucrt:isctype.obj
 0003:0000270c       $pdata$__acrt_get_sigabrt_handler 000000018006270c     libucrt:signal.obj
 0003:00002718       $pdata$raise               0000000180062718     libucrt:signal.obj
 0003:00002724       $pdata$raise$fin$0         0000000180062724     libucrt:signal.obj
 0003:00002730       $pdata$??$?RV<lambda_450d765d439847d4c735a33c368b5fc0>@@AEAV<lambda_44731a7d0e6d81c3e6aa82d741081786>@@V<lambda_601a2a7da3b7a96e9554ac7215c4b07c>@@@?$__crt_seh_guarded_call@P6AXH@Z@@QEAAP6AXH@Z$$QEAV<lambda_450d765d439847d4c735a33c368b5fc0>@@AEAV<lambda_44731a7d0e6d81c3e6aa82d741081786>@@$$QEAV<lambda_601a2a7da3b7a96e9554ac7215c4b07c>@@@Z 0000000180062730     libucrt:signal.obj
 0003:0000273c       $pdata$__acrt_WideCharToMultiByte 000000018006273c     libucrt:widechartomultibyte.obj
 0003:00002748       $pdata$_wcsicmp            0000000180062748     libucrt:wcsicmp.obj
 0003:00002754       $pdata$_wcsicmp_l          0000000180062754     libucrt:wcsicmp.obj
 0003:00002760       $pdata$__acrt_get_process_end_policy 0000000180062760     libucrt:win_policies.obj
 0003:0000276c       $pdata$??$__acrt_wcs_to_mbs_cp@U__crt_win32_buffer_internal_dynamic_resizing@@@@YAHQEB_WAEAV?$__crt_win32_buffer@DU__crt_win32_buffer_internal_dynamic_resizing@@@@I@Z 000000018006276c     libucrt:argv_wildcards.obj
 0003:00002778       $pdata$??$common_expand_argv_wildcards@D@@YAHQEAPEADQEAPEAPEAD@Z 0000000180062778     libucrt:argv_wildcards.obj
 0003:00002784       $pdata$??$copy_and_add_argument_to_buffer@D@@YAHQEBD0_KAEAV?$argument_list@D@?A0x5f5c8891@@@Z 0000000180062784     libucrt:argv_wildcards.obj
 0003:00002790       $pdata$??$expand_argument_wildcards@D@@YAHQEAD0AEAV?$argument_list@D@?A0x5f5c8891@@@Z 0000000180062790     libucrt:argv_wildcards.obj
 0003:0000279c       $pdata$__acrt_GetModuleFileNameA 000000018006279c     libucrt:getmodulefilenamea.obj
 0003:000027a8       $pdata$__acrt_update_thread_multibyte_data 00000001800627a8     libucrt:mbctype.obj
 0003:000027b4       $pdata$__acrt_initialize_multibyte 00000001800627b4     libucrt:mbctype.obj
 0003:000027c0       $pdata$_setmbcp_nolock     00000001800627c0     libucrt:mbctype.obj
 0003:000027cc       $pdata$?getSystemCP@@YAHH@Z 00000001800627cc     libucrt:mbctype.obj
 0003:000027d8       $pdata$?setSBCS@@YAXPEAU__crt_multibyte_data@@@Z 00000001800627d8     libucrt:mbctype.obj
 0003:000027e4       $pdata$?update_thread_multibyte_data_internal@@YAPEAU__crt_multibyte_data@@QEAU__acrt_ptd@@QEAPEAU1@@Z 00000001800627e4     libucrt:mbctype.obj
 0003:000027f0       $pdata$?fin$0@?0??update_thread_multibyte_data_internal@@YAPEAU__crt_multibyte_data@@QEAU__acrt_ptd@@QEAPEAU1@@Z@4HA 00000001800627f0     libucrt:mbctype.obj
 0003:000027fc       $pdata$?setmbcp_internal@@YAHH_NQEAU__acrt_ptd@@QEAPEAU__crt_multibyte_data@@@Z 00000001800627fc     libucrt:mbctype.obj
 0003:00002808       $pdata$?setSBUpLow@@YAXPEAU__crt_multibyte_data@@@Z 0000000180062808     libucrt:mbctype.obj
 0003:00002814       $pdata$??$?RV<lambda_efdfa57d1f175319df784efa44bb7b81>@@AEAV<lambda_5f0a4c1567f8adc6734073e5d1e1b35c>@@V<lambda_2e8a7d3640ea6ccb4c2413664c2db6fd>@@@?$__crt_seh_guarded_call@X@@QEAAX$$QEAV<lambda_efdfa57d1f175319df784efa44bb7b81>@@AEAV<lambda_5f0a4c1567f8adc6734073e5d1e1b35c>@@$$QEAV<lambda_2e8a7d3640ea6ccb4c2413664c2db6fd>@@@Z 0000000180062814     libucrt:mbctype.obj
 0003:00002820       $pdata$?x_ismbbtype_l@@YAHPEAU__crt_locale_pointers@@IHH@Z 0000000180062820     libucrt:ismbbyte.obj
 0003:0000282c       $pdata$__acrt_initialize_command_line 000000018006282c     libucrt:argv_data.obj
 0003:00002838       $pdata$__dcrt_get_narrow_environment_from_os 0000000180062838     libucrt:get_environment_from_os.obj
 0003:00002844       $pdata$_recalloc_base      0000000180062844     libucrt:recalloc.obj
 0003:00002850       $pdata$__acrt_initialize_heap 0000000180062850     libucrt:heap_handle.obj
 0003:0000285c       $pdata$__acrt_execute_initializers 000000018006285c     libucrt:shared_initialization.obj
 0003:00002868       $pdata$__acrt_execute_uninitializers 0000000180062868     libucrt:shared_initialization.obj
 0003:00002874       $pdata$__acrt_release_locale_ref 0000000180062874     libucrt:locale_refcounting.obj
 0003:00002880       $pdata$__acrt_free_locale  0000000180062880     libucrt:locale_refcounting.obj
 0003:0000288c       $pdata$__acrt_locale_free_lc_time_if_unreferenced 000000018006288c     libucrt:locale_refcounting.obj
 0003:00002898       $pdata$__acrt_update_thread_locale_data 0000000180062898     libucrt:locale_refcounting.obj
 0003:000028a4       $pdata$__acrt_update_thread_locale_data$fin$0 00000001800628a4     libucrt:locale_refcounting.obj
 0003:000028b0       $pdata$_updatetlocinfoEx_nolock 00000001800628b0     libucrt:locale_refcounting.obj
 0003:000028bc       $pdata$__acrt_fenv_set_control 00000001800628bc     libucrt:_fenvutils.obj
 0003:000028c8       $pdata$__acrt_DownlevelLocaleNameToLCID 00000001800628c8     libucrt:lcidtoname_downlevel.obj
 0003:000028d4       $pdata$__acrt_DownlevelLCIDToLocaleName 00000001800628d4     libucrt:lcidtoname_downlevel.obj
 0003:000028e0       $pdata$fclose              00000001800628e0     libucrt:fclose.obj
 0003:000028ec       $pdata$fclose$fin$0        00000001800628ec     libucrt:fclose.obj
 0003:000028f8       $pdata$_fclose_nolock      00000001800628f8     libucrt:fclose.obj
 0003:00002904       $pdata$_commit             0000000180062904     libucrt:commit.obj
 0003:00002910       $pdata$??$?RV<lambda_a37b2b86f63e897a80ea819b0eb08c01>@@AEAV<lambda_38ce7e780aa69e748d6df282ebc68efe>@@V<lambda_99fb1378e971ab6e7edea83e3a7a83a2>@@@?$__crt_seh_guarded_call@H@@QEAAH$$QEAV<lambda_a37b2b86f63e897a80ea819b0eb08c01>@@AEAV<lambda_38ce7e780aa69e748d6df282ebc68efe>@@$$QEAV<lambda_99fb1378e971ab6e7edea83e3a7a83a2>@@@Z 0000000180062910     libucrt:commit.obj
 0003:0000291c       $pdata$?fin$0@?0???$?RV<lambda_751a882b2c74d4b022dec766aa51a29a>@@AEAV<lambda_628dfdc04ba53c8bfc02c9951375f3f5>@@V<lambda_f6c7be5f7998530c34de24c7437d6b54>@@@?$__crt_seh_guarded_call@H@@QEAAH$$QEAV<lambda_751a882b2c74d4b022dec766aa51a29a>@@AEAV<lambda_628dfdc04ba53c8bfc02c9951375f3f5>@@$$QEAV<lambda_f6c7be5f7998530c34de24c7437d6b54>@@@Z@4HA 000000018006291c     libucrt:close.obj
 0003:0000291c       $pdata$?fin$0@?0???$?RV<lambda_a37b2b86f63e897a80ea819b0eb08c01>@@AEAV<lambda_38ce7e780aa69e748d6df282ebc68efe>@@V<lambda_99fb1378e971ab6e7edea83e3a7a83a2>@@@?$__crt_seh_guarded_call@H@@QEAAH$$QEAV<lambda_a37b2b86f63e897a80ea819b0eb08c01>@@AEAV<lambda_38ce7e780aa69e748d6df282ebc68efe>@@$$QEAV<lambda_99fb1378e971ab6e7edea83e3a7a83a2>@@@Z@4HA 000000018006291c     libucrt:commit.obj
 0003:00002928       $pdata$??$common_lseek_nolock@_J@@YA_JH_JH@Z 0000000180062928     libucrt:lseek.obj
 0003:00002934       $pdata$?__mbrtowc_utf8@__crt_mbstring@@YA_KPEA_WPEBD_KPEAU_Mbstatet@@@Z 0000000180062934     libucrt:mbrtowc.obj
 0003:00002940       $pdata$?__mbsrtowcs_utf8@__crt_mbstring@@YA_KPEA_WPEAPEBD_KPEAU_Mbstatet@@@Z 0000000180062940     libucrt:mbrtowc.obj
 0003:0000294c       $pdata$_putwch_nolock      000000018006294c     libucrt:putwch.obj
 0003:00002958       $pdata$?__c32rtomb_utf8@__crt_mbstring@@YA_KPEAD_UPEAU_Mbstatet@@@Z 0000000180062958     libucrt:c32rtomb.obj
 0003:00002964       $pdata$__acrt_fp_strflt_to_string 0000000180062964     libucrt:_fptostr.obj
 0003:00002970       $pdata$__acrt_fltout       0000000180062970     libucrt:cfout.obj
 0003:0000297c       $pdata$__acrt_locale_initialize_monetary 000000018006297c     libucrt:initmon.obj
 0003:00002988       $pdata$__acrt_locale_free_monetary 0000000180062988     libucrt:initmon.obj
 0003:00002994       $pdata$__acrt_locale_initialize_numeric 0000000180062994     libucrt:initnum.obj
 0003:000029a0       $pdata$__acrt_locale_free_numeric 00000001800629a0     libucrt:initnum.obj
 0003:000029ac       $pdata$__acrt_locale_initialize_time 00000001800629ac     libucrt:inittime.obj
 0003:000029b8       $pdata$__acrt_locale_free_time 00000001800629b8     libucrt:inittime.obj
 0003:000029c4       $pdata$?initialize_lc_time@@YA_NQEAU__crt_lc_time_data@@QEAU__crt_locale_data@@@Z 00000001800629c4     libucrt:inittime.obj
 0003:000029d0       $pdata$?free_crt_array_internal@@YAXQEAPEBX_K@Z 00000001800629d0     libucrt:inittime.obj
 0003:000029dc       $pdata$wcscat_s            00000001800629dc     libucrt:wcscat_s.obj
 0003:000029e8       $pdata$wcsncat_s           00000001800629e8     libucrt:wcsncat_s.obj
 0003:000029f4       $pdata$wcsncpy_s           00000001800629f4     libucrt:wcsncpy_s.obj
 0003:00002a00       $pdata$__acrt_get_qualified_locale 0000000180062a00     libucrt:get_qualified_locale.obj
 0003:00002a0c       $pdata$TranslateName       0000000180062a0c     libucrt:get_qualified_locale.obj
 0003:00002a18       $pdata$GetLocaleNameFromLangCountry 0000000180062a18     libucrt:get_qualified_locale.obj
 0003:00002a24       $pdata$LangCountryEnumProcEx 0000000180062a24     libucrt:get_qualified_locale.obj
 0003:00002a30       $pdata$GetLocaleNameFromLanguage 0000000180062a30     libucrt:get_qualified_locale.obj
 0003:00002a3c       $pdata$LanguageEnumProcEx  0000000180062a3c     libucrt:get_qualified_locale.obj
 0003:00002a48       $pdata$GetLocaleNameFromDefault 0000000180062a48     libucrt:get_qualified_locale.obj
 0003:00002a54       $pdata$ProcessCodePage     0000000180062a54     libucrt:get_qualified_locale.obj
 0003:00002a60       $pdata$TestDefaultCountry  0000000180062a60     libucrt:get_qualified_locale.obj
 0003:00002a6c       $pdata$__acrt_get_qualified_locale_downlevel 0000000180062a6c     libucrt:getqloc_downlevel.obj
 0003:00002a78       $pdata$TranslateName       0000000180062a78     libucrt:getqloc_downlevel.obj
 0003:00002a84       $pdata$GetLcidFromLangCountry 0000000180062a84     libucrt:getqloc_downlevel.obj
 0003:00002a90       $pdata$LangCountryEnumProc 0000000180062a90     libucrt:getqloc_downlevel.obj
 0003:00002a9c       $pdata$GetLcidFromLanguage 0000000180062a9c     libucrt:getqloc_downlevel.obj
 0003:00002aa8       $pdata$LanguageEnumProc    0000000180062aa8     libucrt:getqloc_downlevel.obj
 0003:00002ab4       $pdata$CountryEnumProc     0000000180062ab4     libucrt:getqloc_downlevel.obj
 0003:00002ac0       $pdata$ProcessCodePage     0000000180062ac0     libucrt:getqloc_downlevel.obj
 0003:00002acc       $pdata$TestDefaultLanguage 0000000180062acc     libucrt:getqloc_downlevel.obj
 0003:00002ad8       $pdata$?__wcsrtombs_utf8@__crt_mbstring@@YA_KPEADPEAPEB_W_KPEAU_Mbstatet@@@Z 0000000180062ad8     libucrt:wcrtomb.obj
 0003:00002af0       $pdata$_towlower_l         0000000180062af0     libucrt:towlower.obj
 0003:00002afc       $pdata$qsort               0000000180062afc     libucrt:qsort.obj
 0003:00002b08       $pdata$4$qsort             0000000180062b08     libucrt:qsort.obj
 0003:00002b14       $pdata$5$qsort             0000000180062b14     libucrt:qsort.obj
 0003:00002b20       $pdata$strpbrk             0000000180062b20     libucrt:strpbrk.obj
 0003:00002b2c       $pdata$fallbackMethod      0000000180062b2c     libucrt:strpbrk.obj
 0003:00002b38       $pdata$_mbsdec_l           0000000180062b38     libucrt:mbsdec.obj
 0003:00002b44       $pdata$?initialize_multibyte@@YAHXZ 0000000180062b44     libucrt:multibyte_initializer.obj
 0003:00002b50       $pdata$_msize_base         0000000180062b50     libucrt:msize.obj
 0003:00002b5c       $pdata$_wcsnicmp           0000000180062b5c     libucrt:wcsnicmp.obj
 0003:00002b68       $pdata$_wcsnicmp_l         0000000180062b68     libucrt:wcsnicmp.obj
 0003:00002b74       $pdata$_close              0000000180062b74     libucrt:close.obj
 0003:00002b80       $pdata$_close_nolock       0000000180062b80     libucrt:close.obj
 0003:00002b8c       $pdata$??$?RV<lambda_751a882b2c74d4b022dec766aa51a29a>@@AEAV<lambda_628dfdc04ba53c8bfc02c9951375f3f5>@@V<lambda_f6c7be5f7998530c34de24c7437d6b54>@@@?$__crt_seh_guarded_call@H@@QEAAH$$QEAV<lambda_751a882b2c74d4b022dec766aa51a29a>@@AEAV<lambda_628dfdc04ba53c8bfc02c9951375f3f5>@@$$QEAV<lambda_f6c7be5f7998530c34de24c7437d6b54>@@@Z 0000000180062b8c     libucrt:close.obj
 0003:00002b98       $pdata$?__mbrtoc32_utf8@__crt_mbstring@@YA_KPEA_UPEBD_KPEAU_Mbstatet@@@Z 0000000180062b98     libucrt:mbrtoc32.obj
 0003:00002ba4       $pdata$__dcrt_lowio_ensure_console_output_initialized 0000000180062ba4     libucrt:initcon.obj
 0003:00002bb0       $pdata$__dcrt_write_console 0000000180062bb0     libucrt:initcon.obj
 0003:00002bbc       $pdata$__dcrt_terminate_console_output 0000000180062bbc     libucrt:initcon.obj
 0003:00002bc8       $pdata$fegetenv            0000000180062bc8     libucrt:fegetenv.obj
 0003:00002bd4       $pdata$fesetenv            0000000180062bd4     libucrt:fesetenv.obj
 0003:00002be0       $pdata$feholdexcept        0000000180062be0     libucrt:feholdexcept.obj
 0003:00002bec       $pdata$_itow_s             0000000180062bec     libucrt:xtoa.obj
 0003:00002bf8       $pdata$??$common_xtox_s@K_W@@YAHKQEA_W_KI_N@Z 0000000180062bf8     libucrt:xtoa.obj
 0003:00002c04       $pdata$??$common_xtox@K_W@@YAHKQEA_W_KI_N@Z 0000000180062c04     libucrt:xtoa.obj
 0003:00002c10       $pdata$?__c16rtomb_utf8@__crt_mbstring@@YA_KPEAD_SPEAU_Mbstatet@@@Z 0000000180062c10     libucrt:c16rtomb.obj
 0003:00002c1c       $pdata$__acrt_LCMapStringW 0000000180062c1c     libucrt:lcmapstringw.obj
 0003:00002c28       $pdata$_clearfp            0000000180062c28     libucrt:ieee.obj
 0003:00002c34       $pdata$_IsNonwritableInCurrentImage 0000000180062c34     LIBCMT:pesect.obj
 0003:00002c40       $pdata$_IsNonwritableInCurrentImage$filt$0 0000000180062c40     LIBCMT:pesect.obj
 0003:00002c4c       $pdata$__GSHandlerCheck_SEH 0000000180062c4c     LIBCMT:gshandlerseh.obj
 0004:00000d28       .idata$6                   0000000180063d28     kernel32:KERNEL32.dll
 0004:00000e0e       .idata$6                   0000000180063e0e     user32:USER32.dll
 0004:00000f1e       .idata$6                   0000000180063f1e     advapi32:ADVAPI32.dll
 0004:00000f62       .idata$6                   0000000180063f62     ole32:ole32.dll
 0004:00000f9c       .idata$6                   0000000180063f9c     mpr:MPR.dll
 0004:00000fe6       .idata$6                   0000000180063fe6     version:VERSION.dll
 0004:00000ff2       .idata$6                   0000000180063ff2     oleaut32:OLEAUT32.dll
 0004:00001030       .idata$6                   0000000180064030     psapi:PSAPI.DLL
 0005:00000000       MoveSmall                  0000000180065000     libvcruntime:memcpy.obj
 0005:00000050       MsetTab                    0000000180065050     libvcruntime:memset.obj
 0006:00000060       $R000000                   0000000180066060     ProcList.res
